 MFC42UD

 Timestamp is 358872ad (Wed Jun 17 18:51:41 1998)

 Preferred load address is 5f800000

 Start         Length     Name                   Class
 0001:00000000 00003851H .text                   CODE
 0001:00003860 0000704fH .text$AFX_AUX           CODE
 0001:0000a8b0 0000efb0H .text$AFX_CMNCTL        CODE
 0001:00019860 00007dfeH .text$AFX_COL1          CODE
 0001:00021660 00004388H .text$AFX_COL2          CODE
 0001:000259f0 00014960H .text$AFX_CORE1         CODE
 0001:0003a350 0000e3ffH .text$AFX_CORE2         CODE
 0001:00048750 0001870fH .text$AFX_CORE3         CODE
 0001:00060e60 00014829H .text$AFX_CORE4         CODE
 0001:00075690 00004bfeH .text$AFX_DBG1          CODE
 0001:0007a290 0000c8d3H .text$AFX_DBG2          CODE
 0001:00086b70 00007884H .text$AFX_INET          CODE
 0001:0008e400 0000ae7bH .text$AFX_INIT          CODE
 0001:00099280 000007dbH .text$AFX_MAPI          CODE
 0001:00099a60 0000748bH .text$AFX_PRNT          CODE
 0001:000a0ef0 000005e4H .text$AFX_TERM          CODE
 0001:000a14e0 00004849H .text$AFX_VDEL          CODE
 0001:000a5d30 00003c6dH .text$x                 CODE
 0002:00000000 00000a24H .idata$5                DATA
 0002:00000a30 00010cecH .rdata                  DATA
 0002:00011720 00003694H .rdata$r                DATA
 0002:00014db8 00005f50H .xdata$x                DATA
 0002:0001ad08 000000c0H .didat$2                DATA
 0002:0001adc8 00000020H .didat$3                DATA
 0002:0001ade8 000001ccH .didat$4                DATA
 0002:0001afb4 00000872H .didat$6                DATA
 0002:0001b828 000001ccH .didat$7                DATA
 0002:0001b9f4 00000050H .idata$2                DATA
 0002:0001ba44 00000014H .idata$3                DATA
 0002:0001ba58 00000a24H .idata$4                DATA
 0002:0001c47c 00002964H .idata$6                DATA
 0002:0001ede0 00004c14H .edata                  DATA
 0003:00000000 00000004H .CRT$XCA                DATA
 0003:00000004 0000000cH .CRT$XCC                DATA
 0003:00000010 00000024H .CRT$XCL                DATA
 0003:00000034 0000007cH .CRT$XCU                DATA
 0003:000000b0 00000004H .CRT$XCZ                DATA
 0003:000000b4 00000004H .CRT$XIA                DATA
 0003:000000b8 00000004H .CRT$XIZ                DATA
 0003:000000c0 00001d10H .data                   DATA
 0003:00001dd0 000001ccH .didat$5                DATA
 0003:00001fa0 00002260H .bss                    DATA
 0004:00000000 00000e98H .rsrc$01                DATA
 0004:00000ea0 000065a8H .rsrc$02                DATA

  Address         Publics by Value              Rva+Base     Lib:Object

 0001:00000000       ?GetHead@CSimpleList@@QBEPAXXZ 5f801000 f i objcore.obj
 0001:00000010       ?AtlW2AHelper@@YGPADPADPBGH@Z 5f801010 f i dumpcont.obj
 0001:00000030       ?AtlW2AHelper@@YGPADPADPBGHI@Z 5f801030 f i dumpcont.obj
 0001:000000c0       ??8@YAHABU_GUID@@0@Z       5f8010c0 f i arcstrm.obj
 0001:000000c0       ?IsEqualGUID@@YAHABU_GUID@@0@Z 5f8010c0 f i arcstrm.obj
 0001:000000e0       ??1CNoTrackObject@@UAE@XZ  5f8010e0 f i dumpinit.obj
 0001:00000100       ??_ECNoTrackObject@@UAEPAXI@Z 5f801100 f i dumpinit.obj
 0001:00000100       ??_GCNoTrackObject@@UAEPAXI@Z 5f801100 f i dumpinit.obj
 0001:00000130       ?DrawState@@YGHPAUHDC__@@PAUHBRUSH__@@P6GH0JIHH@ZJIHHHHI@Z 5f801130 f i afxinl2.obj
 0001:00000170       ?GetNextWindow@@YAPAUHWND__@@PAU1@I@Z 5f801170 f i afxinl3.obj
 0001:00000190       __wcsinc                   5f801190 f i filecore.obj
 0001:000001a0       ?GetFileTitle@@YGFPBGPAGG@Z 5f8011a0 f i filecore.obj
 0001:000001c0       ??0AFX_CLASSINIT@@QAE@PAUCRuntimeClass@@@Z 5f8011c0 f i array_b.obj
 0001:000001e0       ?data@CStringData@@QAEPAGXZ 5f8011e0 f i strcore.obj
 0001:00000200       ?wcschr@@YAPAGPAGG@Z       5f801200 f i strcore.obj
 0001:00000220       ?wcspbrk@@YAPAGPAGPBG@Z    5f801220 f i strcore.obj
 0001:00000240       ?wcsstr@@YAPAGPAGPBG@Z     5f801240 f i strex.obj
 0001:00000260       ?wcsrchr@@YAPAGPAGG@Z      5f801260 f i strex.obj
 0001:00000280       __tclen                    5f801280 f i strex.obj
 0001:00000290       ?Construct@CSimpleList@@QAEXH@Z 5f801290 f i afxstate.obj
 0001:000002d0       ??0CTypeLibCache@@QAE@XZ   5f8012d0 f i afxstate.obj
 0001:00000310       ??0CSimpleList@@QAE@H@Z    5f801310 f i afxstate.obj
 0001:00000340       ??1CHandleMap@@QAE@XZ      5f801340 f i afxstate.obj
 0001:000003a0       ??2@YAPAXIPAX@Z            5f8013a0 f i afxstate.obj
 0001:000003b0       ??3@YAXPAX0@Z              5f8013b0 f i afxstate.obj
 0001:000003c0       ?GetNextPtr@CSimpleList@@QBEPAPAXPAX@Z 5f8013c0 f i afxtls.obj
 0001:00000400       ??2CThreadSlotData@@SGPAXIPAX@Z 5f801400 f i afxtls.obj
 0001:00000410       ??0CFixedAlloc@@QAE@II@Z   5f801410 f   fixalloc.obj
 0001:00000492       ??1CFixedAlloc@@QAE@XZ     5f801492 f   fixalloc.obj
 0001:000004b2       ?FreeAll@CFixedAlloc@@QAEXXZ 5f8014b2 f   fixalloc.obj
 0001:000004f6       ?Alloc@CFixedAlloc@@QAEPAXXZ 5f8014f6 f   fixalloc.obj
 0001:00000666       ?Free@CFixedAlloc@@QAEXPAX@Z 5f801666 f   fixalloc.obj
 0001:000006b0       ??0CSyncObject@@QAE@PBG@Z  5f8016b0 f   mtcore.obj
 0001:00000726       ??1CSyncObject@@UAE@XZ     5f801726 f   mtcore.obj
 0001:0000079a       ?Lock@CSyncObject@@UAEHK@Z 5f80179a f   mtcore.obj
 0001:000007c5       ?Dump@CSyncObject@@UBEXAAVCDumpContext@@@Z 5f8017c5 f   mtcore.obj
 0001:00000820       ?AssertValid@CSyncObject@@UBEXXZ 5f801820 f   mtcore.obj
 0001:00000833       ??BCSyncObject@@QBEPAXXZ   5f801833 f   mtcore.obj
 0001:00000844       ?Unlock@CSemaphore@@UAEHXZ 5f801844 f   mtcore.obj
 0001:0000085e       ?SetEvent@CEvent@@QAEHXZ   5f80185e f   mtcore.obj
 0001:0000089c       ?PulseEvent@CEvent@@QAEHXZ 5f80189c f   mtcore.obj
 0001:000008da       ?ResetEvent@CEvent@@QAEHXZ 5f8018da f   mtcore.obj
 0001:00000918       ??1CSingleLock@@QAE@XZ     5f801918 f   mtcore.obj
 0001:0000092b       ?IsLocked@CSingleLock@@QAEHXZ 5f80192b f   mtcore.obj
 0001:0000093c       ?IsLocked@CMultiLock@@QAEHK@Z 5f80193c f   mtcore.obj
 0001:00000983       ??0CCriticalSection@@QAE@XZ 5f801983 f   mtcore.obj
 0001:000009b1       ??BCCriticalSection@@QAEPAU_RTL_CRITICAL_SECTION@@XZ 5f8019b1 f   mtcore.obj
 0001:000009c2       ??1CCriticalSection@@UAE@XZ 5f8019c2 f   mtcore.obj
 0001:000009eb       ?Lock@CCriticalSection@@QAEHXZ 5f8019eb f   mtcore.obj
 0001:00000a08       ?Lock@CCriticalSection@@UAEHK@Z 5f801a08 f   mtcore.obj
 0001:00000a1d       ?Unlock@CCriticalSection@@UAEHXZ 5f801a1d f   mtcore.obj
 0001:00000a40       ??_ECSyncObject@@UAEPAXI@Z 5f801a40 f i mtcore.obj
 0001:00000a40       ??_GCSyncObject@@UAEPAXI@Z 5f801a40 f i mtcore.obj
 0001:00000a70       ?Unlock@CSyncObject@@UAEHJPAJ@Z 5f801a70 f i mtcore.obj
 0001:00000a90       ??0CSemaphore@@QAE@JJPBGPAU_SECURITY_ATTRIBUTES@@@Z 5f801a90 f   mtex.obj
 0001:00000b4e       ??1CSemaphore@@UAE@XZ      5f801b4e f   mtex.obj
 0001:00000b6a       ?Unlock@CSemaphore@@UAEHJPAJ@Z 5f801b6a f   mtex.obj
 0001:00000b8c       ??0CMutex@@QAE@HPBGPAU_SECURITY_ATTRIBUTES@@@Z 5f801b8c f   mtex.obj
 0001:00000c04       ??1CMutex@@UAE@XZ          5f801c04 f   mtex.obj
 0001:00000c20       ?Unlock@CMutex@@UAEHXZ     5f801c20 f   mtex.obj
 0001:00000c38       ??0CEvent@@QAE@HHPBGPAU_SECURITY_ATTRIBUTES@@@Z 5f801c38 f   mtex.obj
 0001:00000cb4       ??1CEvent@@UAE@XZ          5f801cb4 f   mtex.obj
 0001:00000cd0       ?Unlock@CEvent@@UAEHXZ     5f801cd0 f   mtex.obj
 0001:00000ce0       ??0CSingleLock@@QAE@PAVCSyncObject@@H@Z 5f801ce0 f   mtex.obj
 0001:00000d69       ?Lock@CSingleLock@@QAEHK@Z 5f801d69 f   mtex.obj
 0001:00000de3       ?Unlock@CSingleLock@@QAEHXZ 5f801de3 f   mtex.obj
 0001:00000e42       ?Unlock@CSingleLock@@QAEHJPAJ@Z 5f801e42 f   mtex.obj
 0001:00000eab       ??0CMultiLock@@QAE@QAPAVCSyncObject@@KH@Z 5f801eab f   mtex.obj
 0001:00001068       ??1CMultiLock@@QAE@XZ      5f802068 f   mtex.obj
 0001:000010b2       ?Lock@CMultiLock@@QAEKKHK@Z 5f8020b2 f   mtex.obj
 0001:0000118c       ?Unlock@CMultiLock@@QAEHXZ 5f80218c f   mtex.obj
 0001:000011fa       ?Unlock@CMultiLock@@QAEHJPAJ@Z 5f8021fa f   mtex.obj
 0001:000012b0       _InitMultipleMonitorStubs  5f8022b0 f   wincore.obj
 0001:000013f9       _xGetSystemMetrics@4       5f8023f9 f   wincore.obj
 0001:00001474       _xMonitorFromPoint@12      5f802474 f   wincore.obj
 0001:000014d1       _xMonitorFromRect@8        5f8024d1 f   wincore.obj
 0001:00001535       _xMonitorFromWindow@8      5f802535 f   wincore.obj
 0001:000015b4       _xGetMonitorInfo@8         5f8025b4 f   wincore.obj
 0001:0000168d       _xEnumDisplayMonitors@16   5f80268d f   wincore.obj
 0001:000017c0       ?LookupPermanent@CHandleMap@@QAEPAVCObject@@PAX@Z 5f8027c0 f i wincore.obj
 0001:000017e0       ?LookupTemporary@CHandleMap@@QAEPAVCObject@@PAX@Z 5f8027e0 f i wincore.obj
 0001:00001800       ?UnlockResource@@YGHPAX@Z  5f802800 f i wincore.obj
 0001:00001810       ?AtlA2WHelper@@YGPAGPAGPBDH@Z 5f802810 f i wincore.obj
 0001:00001830       ?AtlA2WHelper@@YGPAGPAGPBDHI@Z 5f802830 f i wincore.obj
 0001:000018c0       ??0CPushRoutingFrame@@QAE@PAVCFrameWnd@@@Z 5f8028c0 f i winfrm.obj
 0001:00001900       ??1CPushRoutingFrame@@QAE@XZ 5f802900 f i winfrm.obj
 0001:00001920       ?GetWindowTask@@YAPAUHTASK__@@PAUHWND__@@@Z 5f802920 f i winfrmx.obj
 0001:00001940       ??_9@$BMM@AE               5f802940 f i dlgcore.obj
 0001:00001950       ??_9@$BNA@AE               5f802950 f i dlgcore.obj
 0001:00001960       ?T2COLE@@YAPBGPBG@Z        5f802960 f i doccore.obj
 0001:00001960       ?T2W@@YAPAGPAG@Z           5f802960 f i doccore.obj
 0001:00001970       __wcsdec                   5f802970 f i docmgr.obj
 0001:000019a0       ??_9@$BOI@AE               5f8029a0 f i viewcore.obj
 0001:000019b0       ??0CPushRoutingView@@QAE@PAVCView@@@Z 5f8029b0 f i viewcore.obj
 0001:000019f0       ??1CPushRoutingView@@QAE@XZ 5f8029f0 f i viewcore.obj
 0001:00001a10       ?GetSize@CRecentFileList@@QBEHXZ 5f802a10 f i appcore.obj
 0001:00001a30       ??ACRecentFileList@@QAEAAVCString@@H@Z 5f802a30 f i appcore.obj
 0001:00001a80       ??0CFileFind@@QAE@XZ       5f802a80 f   filefind.obj
 0001:00001afe       ??1CFileFind@@UAE@XZ       5f802afe f   filefind.obj
 0001:00001b5e       ?Close@CFileFind@@QAEXXZ   5f802b5e f   filefind.obj
 0001:00001be2       ?CloseContext@CFileFind@@MAEXXZ 5f802be2 f   filefind.obj
 0001:00001bfa       ?FindFile@CFileFind@@UAEHPBGK@Z 5f802bfa f   filefind.obj
 0001:00001d7f       ?MatchesMask@CFileFind@@UBEHK@Z 5f802d7f f   filefind.obj
 0001:00001de0       ?GetLastAccessTime@CFileFind@@UBEHPAU_FILETIME@@@Z 5f802de0 f   filefind.obj
 0001:00001e75       ?GetLastWriteTime@CFileFind@@UBEHPAU_FILETIME@@@Z 5f802e75 f   filefind.obj
 0001:00001f0a       ?GetCreationTime@CFileFind@@UBEHPAU_FILETIME@@@Z 5f802f0a f   filefind.obj
 0001:00001f7f       ?GetLastAccessTime@CFileFind@@UBEHAAVCTime@@@Z 5f802f7f f   filefind.obj
 0001:00001ff9       ?GetLastWriteTime@CFileFind@@UBEHAAVCTime@@@Z 5f802ff9 f   filefind.obj
 0001:00002073       ?GetCreationTime@CFileFind@@UBEHAAVCTime@@@Z 5f803073 f   filefind.obj
 0001:000020ed       ?IsDots@CFileFind@@UBEHXZ  5f8030ed f   filefind.obj
 0001:0000219b       ?FindNextFileW@CFileFind@@UAEHXZ 5f80319b f   filefind.obj
 0001:00002245       ?GetFileURL@CFileFind@@UBE?AVCString@@XZ 5f803245 f   filefind.obj
 0001:00002321       ?GetRoot@CFileFind@@UBE?AVCString@@XZ 5f803321 f   filefind.obj
 0001:0000238e       ?GetFilePath@CFileFind@@UBE?AVCString@@XZ 5f80338e f   filefind.obj
 0001:000024b8       ?GetFileTitle@CFileFind@@UBE?AVCString@@XZ 5f8034b8 f   filefind.obj
 0001:000025ab       ?GetFileName@CFileFind@@UBE?AVCString@@XZ 5f8035ab f   filefind.obj
 0001:0000266a       ?GetLength@CFileFind@@QBEKXZ 5f80366a f   filefind.obj
 0001:000026c7       ?GetLength64@CFileFind@@QBE_JXZ 5f8036c7 f   filefind.obj
 0001:00002736       ?Dump@CFileFind@@MBEXAAVCDumpContext@@@Z 5f803736 f   filefind.obj
 0001:0000276a       ?AssertValid@CFileFind@@MBEXXZ 5f80376a f   filefind.obj
 0001:000027e0       ?IsEmpty@CSimpleList@@QBEHXZ 5f8037e0 f i dllinit.obj
 0001:00002800       ??_Gtype_info@@UAEPAXI@Z   5f803800 f i msvcrtd:ti_inst.obj
 0001:00002800       ??_Etype_info@@UAEPAXI@Z   5f803800 f i msvcrtd:ti_inst.obj
 0001:0000282e       ___CxxFrameHandler         5f80382e f   msvcrtd:MSVCRTD.dll
 0001:00002840       __onexit                   5f803840 f   msvcrtd:atonexit.obj
 0001:00002880       _atexit                    5f803880 f   msvcrtd:atonexit.obj
 0001:00002898       __CxxThrowException@8      5f803898 f   msvcrtd:MSVCRTD.dll
 0001:000028a0       __chkstk                   5f8038a0 f   msvcrtd:chkstk.obj
 0001:000028a0       __alloca_probe             5f8038a0 f   msvcrtd:chkstk.obj
 0001:000028d0       _memcpy                    5f8038d0 f   msvcrtd:MSVCRTD.dll
 0001:000028d6       _memcmp                    5f8038d6 f   msvcrtd:MSVCRTD.dll
 0001:000028dc       __except_handler3          5f8038dc f   msvcrtd:MSVCRTD.dll
 0001:000028e2       _memset                    5f8038e2 f   msvcrtd:MSVCRTD.dll
 0001:000028e8       __purecall                 5f8038e8 f   msvcrtd:MSVCRTD.dll
 0001:000028f0       __alldiv                   5f8038f0 f   msvcrtd:lldiv.obj
 0001:000029a0       __allshr                   5f8039a0 f   msvcrtd:llshr.obj
 0001:000029d0       __allmul                   5f8039d0 f   msvcrtd:llmul.obj
 0001:00002a04       _abs                       5f803a04 f   msvcrtd:MSVCRTD.dll
 0001:00002a10       ??_L@YGXPAXIHP6EX0@Z1@Z    5f803a10 f   msvcrtd:ehvecctr.obj
 0001:00002ab0       ??_M@YGXPAXIHP6EX0@Z@Z     5f803ab0 f   msvcrtd:ehvecdtr.obj
 0001:00002b60       ?__ArrayUnwind@@YGXPAXIHP6EX0@Z@Z 5f803b60 f   msvcrtd:ehvecdtr.obj
 0001:00002c10       __CRT_INIT@12              5f803c10 f   msvcrtd:crtdll.obj
 0001:00002d20       __DllMainCRTStartup@12     5f803d20 f   msvcrtd:crtdll.obj
 0001:00002e14       ??1type_info@@UAE@XZ       5f803e14 f   msvcrtd:MSVCRTD.dll
 0001:00002e1a       ___dllonexit               5f803e1a f   msvcrtd:MSVCRTD.dll
 0001:00002e20       ?terminate@@YAXXZ          5f803e20 f   msvcrtd:MSVCRTD.dll
 0001:00002e26       __initterm                 5f803e26 f   msvcrtd:MSVCRTD.dll
 0001:00002e2c       _ReuseDDElParam@20         5f803e2c f   user32:USER32.dll
 0001:00002e32       _UnpackDDElParam@16        5f803e32 f   user32:USER32.dll
 0001:00002e38       __imp_load__RegCloseKey@4  5f803e38     advapi32:ADVAPI32.dll
 0001:00002e44       __tailMerge_ADVAPI32       5f803e44     advapi32:ADVAPI32.dll
 0001:00002e52       _RegCloseKey@4             5f803e52     advapi32:ADVAPI32.dll
 0001:00002e58       __imp_load__RegQueryValueExW@24 5f803e58     advapi32:ADVAPI32.dll
 0001:00002e64       _RegQueryValueExW@24       5f803e64     advapi32:ADVAPI32.dll
 0001:00002e6a       __imp_load__RegOpenKeyW@12 5f803e6a     advapi32:ADVAPI32.dll
 0001:00002e76       _RegOpenKeyW@12            5f803e76     advapi32:ADVAPI32.dll
 0001:00002e7c       __imp_load__SetFileSecurityW@12 5f803e7c     advapi32:ADVAPI32.dll
 0001:00002e88       _SetFileSecurityW@12       5f803e88     advapi32:ADVAPI32.dll
 0001:00002e8e       __imp_load__GetFileSecurityW@20 5f803e8e     advapi32:ADVAPI32.dll
 0001:00002e9a       _GetFileSecurityW@20       5f803e9a     advapi32:ADVAPI32.dll
 0001:00002ea0       __imp_load__RegDeleteKeyW@8 5f803ea0     advapi32:ADVAPI32.dll
 0001:00002eac       _RegDeleteKeyW@8           5f803eac     advapi32:ADVAPI32.dll
 0001:00002eb2       __imp_load__RegEnumKeyW@16 5f803eb2     advapi32:ADVAPI32.dll
 0001:00002ebe       _RegEnumKeyW@16            5f803ebe     advapi32:ADVAPI32.dll
 0001:00002ec4       __imp_load__RegSetValueExW@24 5f803ec4     advapi32:ADVAPI32.dll
 0001:00002ed0       _RegSetValueExW@24         5f803ed0     advapi32:ADVAPI32.dll
 0001:00002ed6       __imp_load__RegCreateKeyW@12 5f803ed6     advapi32:ADVAPI32.dll
 0001:00002ee2       _RegCreateKeyW@12          5f803ee2     advapi32:ADVAPI32.dll
 0001:00002ee8       __imp_load__RegSetValueW@20 5f803ee8     advapi32:ADVAPI32.dll
 0001:00002ef4       _RegSetValueW@20           5f803ef4     advapi32:ADVAPI32.dll
 0001:00002efa       __imp_load__RegQueryValueW@16 5f803efa     advapi32:ADVAPI32.dll
 0001:00002f06       _RegQueryValueW@16         5f803f06     advapi32:ADVAPI32.dll
 0001:00002f0c       __imp_load__RegOpenKeyExW@20 5f803f0c     advapi32:ADVAPI32.dll
 0001:00002f18       _RegOpenKeyExW@20          5f803f18     advapi32:ADVAPI32.dll
 0001:00002f1e       __imp_load__RegCreateKeyExW@36 5f803f1e     advapi32:ADVAPI32.dll
 0001:00002f2a       _RegCreateKeyExW@36        5f803f2a     advapi32:ADVAPI32.dll
 0001:00002f30       __imp_load__RegDeleteValueW@8 5f803f30     advapi32:ADVAPI32.dll
 0001:00002f3c       _RegDeleteValueW@8         5f803f3c     advapi32:ADVAPI32.dll
 0001:00002f42       __imp_load__CreateMappedBitmap@20 5f803f42     comctl32:COMCTL32.dll
 0001:00002f4e       __tailMerge_COMCTL32       5f803f4e     comctl32:COMCTL32.dll
 0001:00002f5c       _CreateMappedBitmap@20     5f803f5c     comctl32:COMCTL32.dll
 0001:00002f62       __imp_load__InitCommonControlsEx@4 5f803f62     comctl32:COMCTL32.dll
 0001:00002f6e       _InitCommonControlsEx@4    5f803f6e     comctl32:COMCTL32.dll
 0001:00002f74       __imp_load__InitCommonControls@0 5f803f74     comctl32:COMCTL32.dll
 0001:00002f80       _InitCommonControls@0      5f803f80     comctl32:COMCTL32.dll
 0001:00002f86       __imp_load__MakeDragList@4 5f803f86     comctl32:COMCTL32.dll
 0001:00002f92       _MakeDragList@4            5f803f92     comctl32:COMCTL32.dll
 0001:00002f98       __imp_load__ImageList_Destroy@4 5f803f98     comctl32:COMCTL32.dll
 0001:00002fa4       _ImageList_Destroy@4       5f803fa4     comctl32:COMCTL32.dll
 0001:00002faa       __imp_load__ImageList_Create@20 5f803faa     comctl32:COMCTL32.dll
 0001:00002fb6       _ImageList_Create@20       5f803fb6     comctl32:COMCTL32.dll
 0001:00002fbc       __imp_load__ImageList_LoadImageW@28 5f803fbc     comctl32:COMCTL32.dll
 0001:00002fc8       _ImageList_LoadImageW@28   5f803fc8     comctl32:COMCTL32.dll
 0001:00002fce       __imp_load__ImageList_Merge@24 5f803fce     comctl32:COMCTL32.dll
 0001:00002fda       _ImageList_Merge@24        5f803fda     comctl32:COMCTL32.dll
 0001:00002fe0       __imp_load__ImageList_Read@4 5f803fe0     comctl32:COMCTL32.dll
 0001:00002fec       _ImageList_Read@4          5f803fec     comctl32:COMCTL32.dll
 0001:00002ff2       __imp_load__ImageList_Write@8 5f803ff2     comctl32:COMCTL32.dll
 0001:00002ffe       _ImageList_Write@8         5f803ffe     comctl32:COMCTL32.dll
 0001:00003004       __imp_load__LBItemFromPt@16 5f804004     comctl32:COMCTL32.dll
 0001:00003010       _LBItemFromPt@16           5f804010     comctl32:COMCTL32.dll
 0001:00003016       __imp_load__ImageList_GetImageCount@4 5f804016     comctl32:COMCTL32.dll
 0001:00003022       _ImageList_GetImageCount@4 5f804022     comctl32:COMCTL32.dll
 0001:00003028       __imp_load__ImageList_Add@12 5f804028     comctl32:COMCTL32.dll
 0001:00003034       _ImageList_Add@12          5f804034     comctl32:COMCTL32.dll
 0001:0000303a       __imp_load__ImageList_AddMasked@12 5f80403a     comctl32:COMCTL32.dll
 0001:00003046       _ImageList_AddMasked@12    5f804046     comctl32:COMCTL32.dll
 0001:0000304c       __imp_load__ImageList_Remove@8 5f80404c     comctl32:COMCTL32.dll
 0001:00003058       _ImageList_Remove@8        5f804058     comctl32:COMCTL32.dll
 0001:0000305e       __imp_load__ImageList_Replace@16 5f80405e     comctl32:COMCTL32.dll
 0001:0000306a       _ImageList_Replace@16      5f80406a     comctl32:COMCTL32.dll
 0001:00003070       __imp_load__ImageList_ReplaceIcon@12 5f804070     comctl32:COMCTL32.dll
 0001:0000307c       _ImageList_ReplaceIcon@12  5f80407c     comctl32:COMCTL32.dll
 0001:00003082       __imp_load__ImageList_GetIcon@12 5f804082     comctl32:COMCTL32.dll
 0001:0000308e       _ImageList_GetIcon@12      5f80408e     comctl32:COMCTL32.dll
 0001:00003094       __imp_load__ImageList_Draw@24 5f804094     comctl32:COMCTL32.dll
 0001:000030a0       _ImageList_Draw@24         5f8040a0     comctl32:COMCTL32.dll
 0001:000030a6       __imp_load__ImageList_SetBkColor@8 5f8040a6     comctl32:COMCTL32.dll
 0001:000030b2       _ImageList_SetBkColor@8    5f8040b2     comctl32:COMCTL32.dll
 0001:000030b8       __imp_load__ImageList_GetBkColor@4 5f8040b8     comctl32:COMCTL32.dll
 0001:000030c4       _ImageList_GetBkColor@4    5f8040c4     comctl32:COMCTL32.dll
 0001:000030ca       __imp_load__ImageList_SetOverlayImage@12 5f8040ca     comctl32:COMCTL32.dll
 0001:000030d6       _ImageList_SetOverlayImage@12 5f8040d6     comctl32:COMCTL32.dll
 0001:000030dc       __imp_load__ImageList_GetImageInfo@12 5f8040dc     comctl32:COMCTL32.dll
 0001:000030e8       _ImageList_GetImageInfo@12 5f8040e8     comctl32:COMCTL32.dll
 0001:000030ee       __imp_load__ImageList_BeginDrag@16 5f8040ee     comctl32:COMCTL32.dll
 0001:000030fa       _ImageList_BeginDrag@16    5f8040fa     comctl32:COMCTL32.dll
 0001:00003100       __imp_load__ImageList_EndDrag@0 5f804100     comctl32:COMCTL32.dll
 0001:0000310c       _ImageList_EndDrag@0       5f80410c     comctl32:COMCTL32.dll
 0001:00003112       __imp_load__ImageList_DragMove@8 5f804112     comctl32:COMCTL32.dll
 0001:0000311e       _ImageList_DragMove@8      5f80411e     comctl32:COMCTL32.dll
 0001:00003124       __imp_load__ImageList_SetDragCursorImage@16 5f804124     comctl32:COMCTL32.dll
 0001:00003130       _ImageList_SetDragCursorImage@16 5f804130     comctl32:COMCTL32.dll
 0001:00003136       __imp_load__ImageList_DragShowNolock@4 5f804136     comctl32:COMCTL32.dll
 0001:00003142       _ImageList_DragShowNolock@4 5f804142     comctl32:COMCTL32.dll
 0001:00003148       __imp_load__ImageList_GetDragImage@8 5f804148     comctl32:COMCTL32.dll
 0001:00003154       _ImageList_GetDragImage@8  5f804154     comctl32:COMCTL32.dll
 0001:0000315a       __imp_load__ImageList_DragEnter@12 5f80415a     comctl32:COMCTL32.dll
 0001:00003166       _ImageList_DragEnter@12    5f804166     comctl32:COMCTL32.dll
 0001:0000316c       __imp_load__ImageList_DragLeave@4 5f80416c     comctl32:COMCTL32.dll
 0001:00003178       _ImageList_DragLeave@4     5f804178     comctl32:COMCTL32.dll
 0001:0000317e       __imp_load__PropertySheetW@4 5f80417e     comctl32:COMCTL32.dll
 0001:0000318a       _PropertySheetW@4          5f80418a     comctl32:COMCTL32.dll
 0001:00003190       __imp_load__DestroyPropertySheetPage@4 5f804190     comctl32:COMCTL32.dll
 0001:0000319c       _DestroyPropertySheetPage@4 5f80419c     comctl32:COMCTL32.dll
 0001:000031a2       __imp_load__CreatePropertySheetPageW@4 5f8041a2     comctl32:COMCTL32.dll
 0001:000031ae       _CreatePropertySheetPageW@4 5f8041ae     comctl32:COMCTL32.dll
 0001:000031b4       __imp_load__ImageList_SetImageCount@8 5f8041b4     comctl32:COMCTL32.dll
 0001:000031c0       _ImageList_SetImageCount@8 5f8041c0     comctl32:COMCTL32.dll
 0001:000031c6       __imp_load__ImageList_Copy@20 5f8041c6     comctl32:COMCTL32.dll
 0001:000031d2       _ImageList_Copy@20         5f8041d2     comctl32:COMCTL32.dll
 0001:000031d8       __imp_load__ImageList_DrawIndirect@4 5f8041d8     comctl32:COMCTL32.dll
 0001:000031e4       _ImageList_DrawIndirect@4  5f8041e4     comctl32:COMCTL32.dll
 0001:000031ea       __imp_load__ImageList_Duplicate@4 5f8041ea     comctl32:COMCTL32.dll
 0001:000031f6       _ImageList_Duplicate@4     5f8041f6     comctl32:COMCTL32.dll
 0001:000031fc       __imp_load__SHGetFileInfoW@20 5f8041fc     shell32:SHELL32.dll
 0001:00003208       __tailMerge_SHELL32        5f804208     shell32:SHELL32.dll
 0001:00003216       _SHGetFileInfoW@20         5f804216     shell32:SHELL32.dll
 0001:0000321c       __imp_load__DragAcceptFiles@8 5f80421c     shell32:SHELL32.dll
 0001:00003228       _DragAcceptFiles@8         5f804228     shell32:SHELL32.dll
 0001:0000322e       __imp_load__DragFinish@4   5f80422e     shell32:SHELL32.dll
 0001:0000323a       _DragFinish@4              5f80423a     shell32:SHELL32.dll
 0001:00003240       __imp_load__DragQueryFileW@16 5f804240     shell32:SHELL32.dll
 0001:0000324c       _DragQueryFileW@16         5f80424c     shell32:SHELL32.dll
 0001:00003252       __imp_load__ExtractIconW@12 5f804252     shell32:SHELL32.dll
 0001:0000325e       _ExtractIconW@12           5f80425e     shell32:SHELL32.dll
 0001:00003264       __imp_load__GetFileTitleW@12 5f804264     comdlg32:comdlg32.dll
 0001:00003270       __tailMerge_comdlg32       5f804270     comdlg32:comdlg32.dll
 0001:0000327e       _GetFileTitleW@12          5f80427e     comdlg32:comdlg32.dll
 0001:00003284       __imp_load__GetSaveFileNameW@4 5f804284     comdlg32:comdlg32.dll
 0001:00003290       _GetSaveFileNameW@4        5f804290     comdlg32:comdlg32.dll
 0001:00003296       __imp_load__GetOpenFileNameW@4 5f804296     comdlg32:comdlg32.dll
 0001:000032a2       _GetOpenFileNameW@4        5f8042a2     comdlg32:comdlg32.dll
 0001:000032a8       __imp_load__PageSetupDlgW@4 5f8042a8     comdlg32:comdlg32.dll
 0001:000032b4       _PageSetupDlgW@4           5f8042b4     comdlg32:comdlg32.dll
 0001:000032ba       __imp_load__PrintDlgW@4    5f8042ba     comdlg32:comdlg32.dll
 0001:000032c6       _PrintDlgW@4               5f8042c6     comdlg32:comdlg32.dll
 0001:000032cc       __imp_load__ChooseColorW@4 5f8042cc     comdlg32:comdlg32.dll
 0001:000032d8       _ChooseColorW@4            5f8042d8     comdlg32:comdlg32.dll
 0001:000032de       __imp_load__ChooseFontW@4  5f8042de     comdlg32:comdlg32.dll
 0001:000032ea       _ChooseFontW@4             5f8042ea     comdlg32:comdlg32.dll
 0001:000032f0       __imp_load__ReplaceTextW@4 5f8042f0     comdlg32:comdlg32.dll
 0001:000032fc       _ReplaceTextW@4            5f8042fc     comdlg32:comdlg32.dll
 0001:00003302       __imp_load__FindTextW@4    5f804302     comdlg32:comdlg32.dll
 0001:0000330e       _FindTextW@4               5f80430e     comdlg32:comdlg32.dll
 0001:00003314       __imp_load__CommDlgExtendedError@0 5f804314     comdlg32:comdlg32.dll
 0001:00003320       _CommDlgExtendedError@0    5f804320     comdlg32:comdlg32.dll
 0001:00003326       __imp_load__ClosePrinter@4 5f804326     winspool:WINSPOOL.DRV
 0001:00003332       __tailMerge_WINSPOOL       5f804332     winspool:WINSPOOL.DRV
 0001:00003340       _ClosePrinter@4            5f804340     winspool:WINSPOOL.DRV
 0001:00003346       __imp_load__DocumentPropertiesW@24 5f804346     winspool:WINSPOOL.DRV
 0001:00003352       _DocumentPropertiesW@24    5f804352     winspool:WINSPOOL.DRV
 0001:00003358       __imp_load__OpenPrinterW@12 5f804358     winspool:WINSPOOL.DRV
 0001:00003364       _OpenPrinterW@12           5f804364     winspool:WINSPOOL.DRV
 0001:0000336a       __imp_load__InternetCrackUrlW@16 5f80436a     wininet:WININET.dll
 0001:00003376       __tailMerge_WININET        5f804376     wininet:WININET.dll
 0001:00003384       _InternetCrackUrlW@16      5f804384     wininet:WININET.dll
 0001:0000338a       __imp_load__InternetCanonicalizeUrlW@16 5f80438a     wininet:WININET.dll
 0001:00003396       _InternetCanonicalizeUrlW@16 5f804396     wininet:WININET.dll
 0001:0000339c       __imp_load__InternetQueryOptionW@16 5f80439c     wininet:WININET.dll
 0001:000033a8       _InternetQueryOptionW@16   5f8043a8     wininet:WININET.dll
 0001:000033ae       __imp_load__InternetOpenW@20 5f8043ae     wininet:WININET.dll
 0001:000033ba       _InternetOpenW@20          5f8043ba     wininet:WININET.dll
 0001:000033c0       __imp_load__InternetCloseHandle@4 5f8043c0     wininet:WININET.dll
 0001:000033cc       _InternetCloseHandle@4     5f8043cc     wininet:WININET.dll
 0001:000033d2       __imp_load__InternetOpenUrlW@24 5f8043d2     wininet:WININET.dll
 0001:000033de       _InternetOpenUrlW@24       5f8043de     wininet:WININET.dll
 0001:000033e4       __imp_load__InternetSetOptionExW@20 5f8043e4     wininet:WININET.dll
 0001:000033f0       _InternetSetOptionExW@20   5f8043f0     wininet:WININET.dll
 0001:000033f6       __imp_load__InternetSetStatusCallback@8 5f8043f6     wininet:WININET.dll
 0001:00003402       _InternetSetStatusCallback@8 5f804402     wininet:WININET.dll
 0001:00003408       __imp_load__InternetSetCookieW@12 5f804408     wininet:WININET.dll
 0001:00003414       _InternetSetCookieW@12     5f804414     wininet:WININET.dll
 0001:0000341a       __imp_load__InternetGetCookieW@16 5f80441a     wininet:WININET.dll
 0001:00003426       _InternetGetCookieW@16     5f804426     wininet:WININET.dll
 0001:0000342c       __imp_load__InternetSetFilePointer@20 5f80442c     wininet:WININET.dll
 0001:00003438       _InternetSetFilePointer@20 5f804438     wininet:WININET.dll
 0001:0000343e       __imp_load__InternetWriteFile@16 5f80443e     wininet:WININET.dll
 0001:0000344a       _InternetWriteFile@16      5f80444a     wininet:WININET.dll
 0001:00003450       __imp_load__InternetReadFile@16 5f804450     wininet:WININET.dll
 0001:0000345c       _InternetReadFile@16       5f80445c     wininet:WININET.dll
 0001:00003462       __imp_load__InternetQueryDataAvailable@16 5f804462     wininet:WININET.dll
 0001:0000346e       _InternetQueryDataAvailable@16 5f80446e     wininet:WININET.dll
 0001:00003474       __imp_load__InternetConnectW@32 5f804474     wininet:WININET.dll
 0001:00003480       _InternetConnectW@32       5f804480     wininet:WININET.dll
 0001:00003486       __imp_load__FtpDeleteFileW@8 5f804486     wininet:WININET.dll
 0001:00003492       _FtpDeleteFileW@8          5f804492     wininet:WININET.dll
 0001:00003498       __imp_load__FtpRenameFileW@12 5f804498     wininet:WININET.dll
 0001:000034a4       _FtpRenameFileW@12         5f8044a4     wininet:WININET.dll
 0001:000034aa       __imp_load__FtpCreateDirectoryW@8 5f8044aa     wininet:WININET.dll
 0001:000034b6       _FtpCreateDirectoryW@8     5f8044b6     wininet:WININET.dll
 0001:000034bc       __imp_load__FtpRemoveDirectoryW@8 5f8044bc     wininet:WININET.dll
 0001:000034c8       _FtpRemoveDirectoryW@8     5f8044c8     wininet:WININET.dll
 0001:000034ce       __imp_load__FtpSetCurrentDirectoryW@8 5f8044ce     wininet:WININET.dll
 0001:000034da       _FtpSetCurrentDirectoryW@8 5f8044da     wininet:WININET.dll
 0001:000034e0       __imp_load__FtpGetCurrentDirectoryW@12 5f8044e0     wininet:WININET.dll
 0001:000034ec       _FtpGetCurrentDirectoryW@12 5f8044ec     wininet:WININET.dll
 0001:000034f2       __imp_load__FtpOpenFileW@20 5f8044f2     wininet:WININET.dll
 0001:000034fe       _FtpOpenFileW@20           5f8044fe     wininet:WININET.dll
 0001:00003504       __imp_load__FtpPutFileW@20 5f804504     wininet:WININET.dll
 0001:00003510       _FtpPutFileW@20            5f804510     wininet:WININET.dll
 0001:00003516       __imp_load__FtpGetFileW@28 5f804516     wininet:WININET.dll
 0001:00003522       _FtpGetFileW@28            5f804522     wininet:WININET.dll
 0001:00003528       __imp_load__GopherCreateLocatorW@28 5f804528     wininet:WININET.dll
 0001:00003534       _GopherCreateLocatorW@28   5f804534     wininet:WININET.dll
 0001:0000353a       __imp_load__GopherGetAttributeW@32 5f80453a     wininet:WININET.dll
 0001:00003546       _GopherGetAttributeW@32    5f804546     wininet:WININET.dll
 0001:0000354c       __imp_load__GopherOpenFileW@20 5f80454c     wininet:WININET.dll
 0001:00003558       _GopherOpenFileW@20        5f804558     wininet:WININET.dll
 0001:0000355e       __imp_load__HttpOpenRequestW@32 5f80455e     wininet:WININET.dll
 0001:0000356a       _HttpOpenRequestW@32       5f80456a     wininet:WININET.dll
 0001:00003570       __imp_load__InternetErrorDlg@20 5f804570     wininet:WININET.dll
 0001:0000357c       _InternetErrorDlg@20       5f80457c     wininet:WININET.dll
 0001:00003582       __imp_load__HttpAddRequestHeadersW@16 5f804582     wininet:WININET.dll
 0001:0000358e       _HttpAddRequestHeadersW@16 5f80458e     wininet:WININET.dll
 0001:00003594       __imp_load__HttpSendRequestW@20 5f804594     wininet:WININET.dll
 0001:000035a0       _HttpSendRequestW@20       5f8045a0     wininet:WININET.dll
 0001:000035a6       __imp_load__HttpEndRequestW@16 5f8045a6     wininet:WININET.dll
 0001:000035b2       _HttpEndRequestW@16        5f8045b2     wininet:WININET.dll
 0001:000035b8       __imp_load__HttpSendRequestExW@20 5f8045b8     wininet:WININET.dll
 0001:000035c4       _HttpSendRequestExW@20     5f8045c4     wininet:WININET.dll
 0001:000035ca       __imp_load__HttpQueryInfoW@20 5f8045ca     wininet:WININET.dll
 0001:000035d6       _HttpQueryInfoW@20         5f8045d6     wininet:WININET.dll
 0001:000035dc       __imp_load__FtpFindFirstFileW@20 5f8045dc     wininet:WININET.dll
 0001:000035e8       _FtpFindFirstFileW@20      5f8045e8     wininet:WININET.dll
 0001:000035ee       __imp_load__InternetFindNextFileW@8 5f8045ee     wininet:WININET.dll
 0001:000035fa       _InternetFindNextFileW@8   5f8045fa     wininet:WININET.dll
 0001:00003600       __imp_load__GopherFindFirstFileW@24 5f804600     wininet:WININET.dll
 0001:0000360c       _GopherFindFirstFileW@24   5f80460c     wininet:WININET.dll
 0001:00003612       __imp_load__InternetGetLastResponseInfoW@12 5f804612     wininet:WININET.dll
 0001:0000361e       _InternetGetLastResponseInfoW@12 5f80461e     wininet:WININET.dll
 0001:00003624       __imp_load__GopherGetLocatorTypeW@8 5f804624     wininet:WININET.dll
 0001:00003630       _GopherGetLocatorTypeW@8   5f804630     wininet:WININET.dll
 0001:00003636       ___delayLoadHelper@8       5f804636 f   delayimp:delayhlp.obj
 0001:00003860       ?InitString@CSimpleException@@QAEXXZ 5f804860 f   except.obj
 0001:0000389c       ?GetErrorMessage@CSimpleException@@UAEHPAGIPAI@Z 5f80489c f   except.obj
 0001:0000392e       ?AfxThrowMemoryException@@YGXXZ 5f80492e f   except.obj
 0001:0000394b       ?AfxThrowNotSupportedException@@YGXXZ 5f80494b f   except.obj
 0001:00003970       ?AfxIsValidString@@YGHPBGH@Z 5f804970 f   validadd.obj
 0001:000039b2       ?AfxIsValidString@@YGHPBDH@Z 5f8049b2 f   validadd.obj
 0001:000039d6       ?AfxIsValidAddress@@YGHPBXIH@Z 5f8049d6 f   validadd.obj
 0001:00003a64       ?_AfxCrtDumpClient@@YAXPAXI@Z 5f804a64 f   dumpinit.obj
 0001:00003bd6       ?_AfxCrtReportHook@@YAHHPADPAH@Z 5f804bd6 f   dumpinit.obj
 0001:00003c33       ??0_AFX_DEBUG_STATE@@QAE@XZ 5f804c33 f   dumpinit.obj
 0001:00003d30       ??1_AFX_DEBUG_STATE@@UAE@XZ 5f804d30 f   dumpinit.obj
 0001:00003dc6       ?AfxDiagnosticInit@@YGHXZ  5f804dc6 f   dumpinit.obj
 0001:00003e10       ??_G_AFX_DEBUG_STATE@@UAEPAXI@Z 5f804e10 f i dumpinit.obj
 0001:00003e10       ??_E_AFX_DEBUG_STATE@@UAEPAXI@Z 5f804e10 f i dumpinit.obj
 0001:00003e40       ??0CNoTrackObject@@QAE@XZ  5f804e40 f i dumpinit.obj
 0001:00003e60       ??1?$CProcessLocal@V_AFX_DEBUG_STATE@@@@QAE@XZ 5f804e60 f i dumpinit.obj
 0001:00003e80       ?GetData@?$CProcessLocal@V_AFX_DEBUG_STATE@@@@QAEPAV_AFX_DEBUG_STATE@@XZ 5f804e80 f i dumpinit.obj
 0001:00003ed0       ?CreateObject@?$CProcessLocal@V_AFX_DEBUG_STATE@@@@SGPAVCNoTrackObject@@XZ 5f804ed0 f i dumpinit.obj
 0001:00003f40       ?AfxDump@@YGXPBVCObject@@@Z 5f804f40 f   dumpout.obj
 0001:00003f55       ?AfxTrace@@YAXPBGZZ        5f804f55 f   dumpout.obj
 0001:00004020       ?AfxAbort@@YGXXZ           5f805020 f   afxabort.obj
 0001:00004050       ??0CString@@QAE@GH@Z       5f805050 f   strex.obj
 0001:000040a8       ??0CString@@QAE@PBGH@Z     5f8050a8 f   strex.obj
 0001:0000411a       ??0CString@@QAE@PBDH@Z     5f80511a f   strex.obj
 0001:00004189       ??4CString@@QAEABV0@G@Z    5f805189 f   strex.obj
 0001:000041a7       ??H@YG?AVCString@@ABV0@G@Z 5f8051a7 f   strex.obj
 0001:0000422c       ??H@YG?AVCString@@GABV0@@Z 5f80522c f   strex.obj
 0001:000042b1       ?Delete@CString@@QAEHHH@Z  5f8052b1 f   strex.obj
 0001:00004344       ?Insert@CString@@QAEHHG@Z  5f805344 f   strex.obj
 0001:0000442d       ?Insert@CString@@QAEHHPBG@Z 5f80542d f   strex.obj
 0001:00004544       ?Replace@CString@@QAEHGG@Z 5f805544 f   strex.obj
 0001:000045d7       ?Replace@CString@@QAEHPBG0@Z 5f8055d7 f   strex.obj
 0001:00004828       ?Remove@CString@@QAEHG@Z   5f805828 f   strex.obj
 0001:000048df       ?Mid@CString@@QBE?AV1@H@Z  5f8058df f   strex.obj
 0001:0000491f       ?Mid@CString@@QBE?AV1@HH@Z 5f80591f f   strex.obj
 0001:00004a78       ?Right@CString@@QBE?AV1@H@Z 5f805a78 f   strex.obj
 0001:00004b37       ?Left@CString@@QBE?AV1@H@Z 5f805b37 f   strex.obj
 0001:00004be9       ?SpanIncluding@CString@@QBE?AV1@PBG@Z 5f805be9 f   strex.obj
 0001:00004c59       ?SpanExcluding@CString@@QBE?AV1@PBG@Z 5f805c59 f   strex.obj
 0001:00004cc9       ?ReverseFind@CString@@QBEHG@Z 5f805cc9 f   strex.obj
 0001:00004d0d       ?Find@CString@@QBEHPBG@Z   5f805d0d f   strex.obj
 0001:00004d28       ?Find@CString@@QBEHPBGH@Z  5f805d28 f   strex.obj
 0001:00004dbb       ?FormatV@CString@@QAEXPBGPAD@Z 5f805dbb f   strex.obj
 0001:00005578       ?Format@CString@@QAAXPBGZZ 5f806578 f   strex.obj
 0001:000055cc       ?Format@CString@@QAAXIZZ   5f8065cc f   strex.obj
 0001:00005665       ?FormatMessageW@CString@@QAAXPBGZZ 5f806665 f   strex.obj
 0001:000056be       ?FormatMessageW@CString@@QAAXIZZ 5f8066be f   strex.obj
 0001:00005789       ?TrimRight@CString@@QAEXPBG@Z 5f806789 f   strex.obj
 0001:0000581e       ?TrimRight@CString@@QAEXG@Z 5f80681e f   strex.obj
 0001:000058af       ?TrimRight@CString@@QAEXXZ 5f8068af f   strex.obj
 0001:0000593e       ?TrimLeft@CString@@QAEXPBG@Z 5f80693e f   strex.obj
 0001:000059f3       ?TrimLeft@CString@@QAEXG@Z 5f8069f3 f   strex.obj
 0001:00005a85       ?TrimLeft@CString@@QAEXXZ  5f806a85 f   strex.obj
 0001:00005b14       ?ConstructElements@@YGXPAVCString@@H@Z 5f806b14 f   strex.obj
 0001:00005b88       ?DestructElements@@YGXPAVCString@@H@Z 5f806b88 f   strex.obj
 0001:00005bf2       ?CopyElements@@YGXPAVCString@@PBV1@H@Z 5f806bf2 f   strex.obj
 0001:00005c9d       ?HashKey@@YGIPBG@Z         5f806c9d f   strex.obj
 0001:00005cde       ?HashKey@@YGIPBD@Z         5f806cde f   strex.obj
 0001:00005d20       ??0CTime@@QAE@HHHHHHH@Z    5f806d20 f   timecore.obj
 0001:00005e02       ??0CTime@@QAE@GGH@Z        5f806e02 f   timecore.obj
 0001:00005ebb       ??0CTime@@QAE@ABU_SYSTEMTIME@@H@Z 5f806ebb f   timecore.obj
 0001:00005f51       ??0CTime@@QAE@ABU_FILETIME@@H@Z 5f806f51 f   timecore.obj
 0001:00005fb9       ?GetTickCount@CTime@@SG?AV1@XZ 5f806fb9 f   timecore.obj
 0001:00005fe3       ?GetGmtTm@CTime@@QBEPAUtm@@PAU2@@Z 5f806fe3 f   timecore.obj
 0001:00006025       ?GetLocalTm@CTime@@QBEPAUtm@@PAU2@@Z 5f807025 f   timecore.obj
 0001:00006077       ?GetAsSystemTime@CTime@@QBEHAAU_SYSTEMTIME@@@Z 5f807077 f   timecore.obj
 0001:00006112       ??6@YGAAVCDumpContext@@AAV0@VCTime@@@Z 5f807112 f   timecore.obj
 0001:00006189       ??6@YGAAVCArchive@@AAV0@VCTime@@@Z 5f807189 f   timecore.obj
 0001:0000619c       ??5@YGAAVCArchive@@AAV0@AAVCTime@@@Z 5f80719c f   timecore.obj
 0001:000061af       ??6@YGAAVCDumpContext@@AAV0@VCTimeSpan@@@Z 5f8071af f   timecore.obj
 0001:00006233       ??6@YGAAVCArchive@@AAV0@VCTimeSpan@@@Z 5f807233 f   timecore.obj
 0001:00006246       ??5@YGAAVCArchive@@AAV0@AAVCTimeSpan@@@Z 5f807246 f   timecore.obj
 0001:00006259       ?Format@CTimeSpan@@QBE?AVCString@@PBG@Z 5f807259 f   timecore.obj
 0001:00006549       ?Format@CTimeSpan@@QBE?AVCString@@I@Z 5f807549 f   timecore.obj
 0001:000065e9       ?Format@CTime@@QBE?AVCString@@PBG@Z 5f8075e9 f   timecore.obj
 0001:00006675       ?FormatGmt@CTime@@QBE?AVCString@@PBG@Z 5f807675 f   timecore.obj
 0001:00006701       ?Format@CTime@@QBE?AVCString@@I@Z 5f807701 f   timecore.obj
 0001:000067a1       ?FormatGmt@CTime@@QBE?AVCString@@I@Z 5f8077a1 f   timecore.obj
 0001:00006841       ?Format@CTime@@QBE?AVCString@@PBD@Z 5f807841 f   timecore.obj
 0001:000068b6       ?FormatGmt@CTime@@QBE?AVCString@@PBD@Z 5f8078b6 f   timecore.obj
 0001:0000692b       ?Format@CTimeSpan@@QBE?AVCString@@PBD@Z 5f80792b f   timecore.obj
 0001:000069a0       ?LoadBitmaps@CBitmapButton@@QAEHPBG000@Z 5f8079a0 f   winbtn.obj
 0001:00006a80       ?SizeToContent@CBitmapButton@@QAEXXZ 5f807a80 f   winbtn.obj
 0001:00006b1b       ?AutoLoad@CBitmapButton@@QAEHIPAVCWnd@@@Z 5f807b1b f   winbtn.obj
 0001:00006cc5       ?DrawItem@CBitmapButton@@MAEXPAUtagDRAWITEMSTRUCT@@@Z 5f807cc5 f   winbtn.obj
 0001:00006e51       ?AssertValid@CBitmapButton@@UBEXXZ 5f807e51 f   winbtn.obj
 0001:00006ea0       ?Dump@CBitmapButton@@UBEXAAVCDumpContext@@@Z 5f807ea0 f   winbtn.obj
 0001:00006f40       ?_GetBaseMessageMap@CCommonDialog@@KGPBUAFX_MSGMAP@@XZ 5f807f40 f   dlgcomm.obj
 0001:00006f4a       ?GetMessageMap@CCommonDialog@@MBEPBUAFX_MSGMAP@@XZ 5f807f4a f   dlgcomm.obj
 0001:00006f5a       ?_AfxCommDlgProc@@YGIPAUHWND__@@IIJ@Z 5f807f5a f   dlgcomm.obj
 0001:000072b9       ?OnOK@CCommonDialog@@MAEXXZ 5f8082b9 f   dlgcomm.obj
 0001:00007301       ?OnCancel@CCommonDialog@@MAEXXZ 5f808301 f   dlgcomm.obj
 0001:00007327       ?OnHelpInfo@CCommonDialog@@IAEHPAUtagHELPINFO@@@Z 5f808327 f   dlgcomm.obj
 0001:00007340       ??0CFileDialog@@QAE@HPBG0K0PAVCWnd@@@Z 5f808340 f   dlgfile.obj
 0001:00007554       ?DoModal@CFileDialog@@UAEHXZ 5f808554 f   dlgfile.obj
 0001:0000779d       ?GetPathName@CFileDialog@@QBE?AVCString@@XZ 5f80879d f   dlgfile.obj
 0001:00007913       ?GetFileName@CFileDialog@@QBE?AVCString@@XZ 5f808913 f   dlgfile.obj
 0001:00007a41       ?GetFileExt@CFileDialog@@QBE?AVCString@@XZ 5f808a41 f   dlgfile.obj
 0001:00007c61       ?GetFileTitle@CFileDialog@@QBE?AVCString@@XZ 5f808c61 f   dlgfile.obj
 0001:00007d09       ?GetNextPathName@CFileDialog@@QBE?AVCString@@AAPAU__POSITION@@@Z 5f808d09 f   dlgfile.obj
 0001:000080c0       ?SetTemplate@CFileDialog@@QAEXPBG0@Z 5f8090c0 f   dlgfile.obj
 0001:0000810f       ?GetFolderPath@CFileDialog@@QBE?AVCString@@XZ 5f80910f f   dlgfile.obj
 0001:00008214       ?SetControlText@CFileDialog@@QAEXHPBD@Z 5f809214 f   dlgfile.obj
 0001:0000829b       ?HideControl@CFileDialog@@QAEXH@Z 5f80929b f   dlgfile.obj
 0001:00008320       ?SetDefExt@CFileDialog@@QAEXPBD@Z 5f809320 f   dlgfile.obj
 0001:000083a5       ?OnShareViolation@CFileDialog@@MAEIPBG@Z 5f8093a5 f   dlgfile.obj
 0001:000083c7       ?OnFileNameOK@CFileDialog@@MAEHXZ 5f8093c7 f   dlgfile.obj
 0001:000083e7       ?OnLBSelChangedNotify@CFileDialog@@MAEXIII@Z 5f8093e7 f   dlgfile.obj
 0001:00008407       ?OnInitDone@CFileDialog@@MAEXXZ 5f809407 f   dlgfile.obj
 0001:00008436       ?OnFileNameChange@CFileDialog@@MAEXXZ 5f809436 f   dlgfile.obj
 0001:00008454       ?OnFolderChange@CFileDialog@@MAEXXZ 5f809454 f   dlgfile.obj
 0001:00008472       ?OnTypeChange@CFileDialog@@MAEXXZ 5f809472 f   dlgfile.obj
 0001:00008490       ?OnNotify@CFileDialog@@MAEHIJPAJ@Z 5f809490 f   dlgfile.obj
 0001:000085fc       ?Dump@CFileDialog@@UBEXAAVCDumpContext@@@Z 5f8095fc f   dlgfile.obj
 0001:00008890       ??_ECFileDialog@@UAEPAXI@Z 5f809890 f i dlgfile.obj
 0001:00008890       ??_GCFileDialog@@UAEPAXI@Z 5f809890 f i dlgfile.obj
 0001:000088c0       ??1CFileDialog@@UAE@XZ     5f8098c0 f i dlgfile.obj
 0001:00008910       ??0CPageSetupDialog@@QAE@KPAVCWnd@@@Z 5f809910 f   dlgprnt.obj
 0001:000089cc       ?DoModal@CPageSetupDialog@@UAEHXZ 5f8099cc f   dlgprnt.obj
 0001:00008ac0       ?GetDevMode@CPageSetupDialog@@QBEPAU_devicemodeW@@XZ 5f809ac0 f   dlgprnt.obj
 0001:00008ae5       ?GetDriverName@CPageSetupDialog@@QBE?AVCString@@XZ 5f809ae5 f   dlgprnt.obj
 0001:00008b53       ?GetDeviceName@CPageSetupDialog@@QBE?AVCString@@XZ 5f809b53 f   dlgprnt.obj
 0001:00008bc2       ?GetPortName@CPageSetupDialog@@QBE?AVCString@@XZ 5f809bc2 f   dlgprnt.obj
 0001:00008c31       ?CreatePrinterDC@CPageSetupDialog@@QAEPAUHDC__@@XZ 5f809c31 f   dlgprnt.obj
 0001:00008c5f       ?GetMargins@CPageSetupDialog@@QBEXPAUtagRECT@@0@Z 5f809c5f f   dlgprnt.obj
 0001:00008ca4       ?Dump@CPageSetupDialog@@UBEXAAVCDumpContext@@@Z 5f809ca4 f   dlgprnt.obj
 0001:00008da8       ?PreDrawPage@CPageSetupDialog@@UAEIGGPAUtagPSDW@@@Z 5f809da8 f   dlgprnt.obj
 0001:00008db7       ?OnDrawPage@CPageSetupDialog@@UAEIPAVCDC@@IPAUtagRECT@@@Z 5f809db7 f   dlgprnt.obj
 0001:00008dc6       ?PaintHookProc@CPageSetupDialog@@KGIPAUHWND__@@IIJ@Z 5f809dc6 f   dlgprnt.obj
 0001:00008e76       ?_GetBaseMessageMap@CPrintDialog@@KGPBUAFX_MSGMAP@@XZ 5f809e76 f   dlgprnt.obj
 0001:00008e80       ?GetMessageMap@CPrintDialog@@MBEPBUAFX_MSGMAP@@XZ 5f809e80 f   dlgprnt.obj
 0001:00008e90       ??0CPrintDialog@@QAE@HKPAVCWnd@@@Z 5f809e90 f   dlgprnt.obj
 0001:00008fb5       ??0CPrintDialog@@IAE@AAUtagPDW@@@Z 5f809fb5 f   dlgprnt.obj
 0001:00008fe1       ?AttachOnSetup@CPrintDialog@@MAEPAV1@XZ 5f809fe1 f   dlgprnt.obj
 0001:00009095       ?OnPrintSetup@CPrintDialog@@IAEXXZ 5f80a095 f   dlgprnt.obj
 0001:0000912d       ?DoModal@CPrintDialog@@UAEHXZ 5f80a12d f   dlgprnt.obj
 0001:0000918d       ?CreatePrinterDC@CPrintDialog@@QAEPAUHDC__@@XZ 5f80a18d f   dlgprnt.obj
 0001:000091d6       ?GetCopies@CPrintDialog@@QBEHXZ 5f80a1d6 f   dlgprnt.obj
 0001:00009220       ?GetDevMode@CPrintDialog@@QBEPAU_devicemodeW@@XZ 5f80a220 f   dlgprnt.obj
 0001:0000924b       ?GetDriverName@CPrintDialog@@QBE?AVCString@@XZ 5f80a24b f   dlgprnt.obj
 0001:000092bf       ?GetDeviceName@CPrintDialog@@QBE?AVCString@@XZ 5f80a2bf f   dlgprnt.obj
 0001:00009334       ?GetPortName@CPrintDialog@@QBE?AVCString@@XZ 5f80a334 f   dlgprnt.obj
 0001:000093a9       ?GetDefaults@CPrintDialog@@QAEHXZ 5f80a3a9 f   dlgprnt.obj
 0001:000093d5       ?Dump@CPrintDialog@@UBEXAAVCDumpContext@@@Z 5f80a3d5 f   dlgprnt.obj
 0001:00009558       ?AfxCreateDC@@YGPAUHDC__@@PAX0@Z 5f80a558 f   dlgprnt.obj
 0001:00009610       ??_ECColorDialog@@UAEPAXI@Z 5f80a610 f i dlgprnt.obj
 0001:00009610       ??_ECFontDialog@@UAEPAXI@Z 5f80a610 f i dlgprnt.obj
 0001:00009610       ??_ECFindReplaceDialog@@UAEPAXI@Z 5f80a610 f i dlgprnt.obj
 0001:00009610       ??_ECPrintDialog@@UAEPAXI@Z 5f80a610 f i dlgprnt.obj
 0001:00009610       ??_GCPrintDialog@@UAEPAXI@Z 5f80a610 f i dlgprnt.obj
 0001:00009610       ??_GCColorDialog@@UAEPAXI@Z 5f80a610 f i dlgprnt.obj
 0001:00009610       ??_GCFontDialog@@UAEPAXI@Z 5f80a610 f i dlgprnt.obj
 0001:00009610       ??_GCFindReplaceDialog@@UAEPAXI@Z 5f80a610 f i dlgprnt.obj
 0001:00009640       ??1CFontDialog@@UAE@XZ     5f80a640 f i dlgprnt.obj
 0001:00009640       ??1CPrintDialog@@UAE@XZ    5f80a640 f i dlgprnt.obj
 0001:00009640       ??1CPageSetupDialog@@UAE@XZ 5f80a640 f i dlgprnt.obj
 0001:00009640       ??1CColorDialog@@UAE@XZ    5f80a640 f i dlgprnt.obj
 0001:00009640       ??1CFindReplaceDialog@@UAE@XZ 5f80a640 f i dlgprnt.obj
 0001:00009660       ??0_AFX_COLOR_STATE@@QAE@XZ 5f80a660 f   dlgclr.obj
 0001:000096a9       ?_GetBaseMessageMap@CColorDialog@@KGPBUAFX_MSGMAP@@XZ 5f80a6a9 f   dlgclr.obj
 0001:000096b3       ?GetMessageMap@CColorDialog@@MBEPBUAFX_MSGMAP@@XZ 5f80a6b3 f   dlgclr.obj
 0001:000096c3       ??0CColorDialog@@QAE@KKPAVCWnd@@@Z 5f80a6c3 f   dlgclr.obj
 0001:00009799       ?DoModal@CColorDialog@@UAEHXZ 5f80a799 f   dlgclr.obj
 0001:0000983d       ?OnColorOK@CColorDialog@@MAEHXZ 5f80a83d f   dlgclr.obj
 0001:0000985a       ?SetCurrentColor@CColorDialog@@QAEXK@Z 5f80a85a f   dlgclr.obj
 0001:000098b2       ?GetSavedCustomColors@CColorDialog@@SGPAKXZ 5f80a8b2 f   dlgclr.obj
 0001:000098c4       ?OnCtlColor@CColorDialog@@IAEPAUHBRUSH__@@PAVCDC@@PAVCWnd@@I@Z 5f80a8c4 f   dlgclr.obj
 0001:000098d9       ?Dump@CColorDialog@@UBEXAAVCDumpContext@@@Z 5f80a8d9 f   dlgclr.obj
 0001:000099d0       ??_E_AFX_COLOR_STATE@@UAEPAXI@Z 5f80a9d0 f i dlgclr.obj
 0001:000099d0       ??_G_AFX_COLOR_STATE@@UAEPAXI@Z 5f80a9d0 f i dlgclr.obj
 0001:00009a00       ??1_AFX_COLOR_STATE@@UAE@XZ 5f80aa00 f i dlgclr.obj
 0001:00009a20       ??0CFontDialog@@QAE@PAUtagLOGFONTW@@KPAVCDC@@PAVCWnd@@@Z 5f80aa20 f   dlgfnt.obj
 0001:00009ba1       ??0CFontDialog@@QAE@ABU_charformat@@KPAVCDC@@PAVCWnd@@@Z 5f80aba1 f   dlgfnt.obj
 0001:00009d21       ?DoModal@CFontDialog@@UAEHXZ 5f80ad21 f   dlgfnt.obj
 0001:00009df0       ?GetCurrentFont@CFontDialog@@QAEXPAUtagLOGFONTW@@@Z 5f80adf0 f   dlgfnt.obj
 0001:00009e51       ?FillInLogFont@CFontDialog@@QAEKABU_charformat@@@Z 5f80ae51 f   dlgfnt.obj
 0001:0000a0fa       ?GetCharFormat@CFontDialog@@QBEXAAU_charformat@@@Z 5f80b0fa f   dlgfnt.obj
 0001:0000a345       ?Dump@CFontDialog@@UBEXAAVCDumpContext@@@Z 5f80b345 f   dlgfnt.obj
 0001:0000a4a0       ??0CFindReplaceDialog@@QAE@XZ 5f80b4a0 f   dlgfr.obj
 0001:0000a569       ?PostNcDestroy@CFindReplaceDialog@@MAEXXZ 5f80b569 f   dlgfr.obj
 0001:0000a5c7       ?Create@CFindReplaceDialog@@QAEHHPBG0KPAVCWnd@@@Z 5f80b5c7 f   dlgfr.obj
 0001:0000a781       ?GetNotifier@CFindReplaceDialog@@SGPAV1@J@Z 5f80b781 f   dlgfr.obj
 0001:0000a7f2       ?Dump@CFindReplaceDialog@@UBEXAAVCDumpContext@@@Z 5f80b7f2 f   dlgfr.obj
 0001:0000a8b0       ??0CArchiveStream@@QAE@PAVCArchive@@@Z 5f80b8b0 f   arcstrm.obj
 0001:0000a8da       ?AddRef@CArchiveStream@@UAGKXZ 5f80b8da f   arcstrm.obj
 0001:0000a8e6       ?Release@CArchiveStream@@UAGKXZ 5f80b8e6 f   arcstrm.obj
 0001:0000a8ef       ?QueryInterface@CArchiveStream@@UAGJABU_GUID@@PAPAX@Z 5f80b8ef f   arcstrm.obj
 0001:0000a931       ?Read@CArchiveStream@@UAGJPAXKPAK@Z 5f80b931 f   arcstrm.obj
 0001:0000aa37       ?Write@CArchiveStream@@UAGJPBXKPAK@Z 5f80ba37 f   arcstrm.obj
 0001:0000ab3a       ?Seek@CArchiveStream@@UAGJT_LARGE_INTEGER@@KPAT_ULARGE_INTEGER@@@Z 5f80bb3a f   arcstrm.obj
 0001:0000ac69       ?SetSize@CArchiveStream@@UAGJT_ULARGE_INTEGER@@@Z 5f80bc69 f   arcstrm.obj
 0001:0000ac75       ?CopyTo@CArchiveStream@@UAGJPAUIStream@@T_ULARGE_INTEGER@@PAT3@2@Z 5f80bc75 f   arcstrm.obj
 0001:0000ac81       ?Commit@CArchiveStream@@UAGJK@Z 5f80bc81 f   arcstrm.obj
 0001:0000ac8d       ?Revert@CArchiveStream@@UAGJXZ 5f80bc8d f   arcstrm.obj
 0001:0000ac99       ?LockRegion@CArchiveStream@@UAGJT_ULARGE_INTEGER@@0K@Z 5f80bc99 f   arcstrm.obj
 0001:0000aca5       ?UnlockRegion@CArchiveStream@@UAGJT_ULARGE_INTEGER@@0K@Z 5f80bca5 f   arcstrm.obj
 0001:0000acb1       ?Stat@CArchiveStream@@UAGJPAUtagSTATSTG@@K@Z 5f80bcb1 f   arcstrm.obj
 0001:0000acbd       ?Clone@CArchiveStream@@UAGJPAPAUIStream@@@Z 5f80bcbd f   arcstrm.obj
 0001:0000acd0       ??0IStream@@QAE@XZ         5f80bcd0 f i arcstrm.obj
 0001:0000acf0       ??0ISequentialStream@@QAE@XZ 5f80bcf0 f i arcstrm.obj
 0001:0000ad10       ??0IUnknown@@QAE@XZ        5f80bd10 f i arcstrm.obj
 0001:0000ad20       ?_GetBaseMessageMap@CToolTipCtrl@@KGPBUAFX_MSGMAP@@XZ 5f80bd20 f   tooltip.obj
 0001:0000ad2a       ?GetMessageMap@CToolTipCtrl@@MBEPBUAFX_MSGMAP@@XZ 5f80bd2a f   tooltip.obj
 0001:0000ad3a       ??0CToolTipCtrl@@QAE@XZ    5f80bd3a f   tooltip.obj
 0001:0000ad93       ?Create@CToolTipCtrl@@QAEHPAVCWnd@@K@Z 5f80bd93 f   tooltip.obj
 0001:0000ae21       ??1CToolTipCtrl@@UAE@XZ    5f80be21 f   tooltip.obj
 0001:0000ae81       ?DestroyToolTipCtrl@CToolTipCtrl@@QAEHXZ 5f80be81 f   tooltip.obj
 0001:0000aee0       ?OnAddTool@CToolTipCtrl@@IAEJIJ@Z 5f80bee0 f   tooltip.obj
 0001:0000af85       ?OnDisableModal@CToolTipCtrl@@IAEJIJ@Z 5f80bf85 f   tooltip.obj
 0001:0000afa5       ?OnEnable@CToolTipCtrl@@IAEXH@Z 5f80bfa5 f   tooltip.obj
 0001:0000afc5       ?OnWindowFromPoint@CToolTipCtrl@@IAEJIJ@Z 5f80bfc5 f   tooltip.obj
 0001:0000b0a1       ?AddTool@CToolTipCtrl@@QAEHPAVCWnd@@PBGPBUtagRECT@@I@Z 5f80c0a1 f   tooltip.obj
 0001:0000b19d       ?AddTool@CToolTipCtrl@@QAEHPAVCWnd@@IPBUtagRECT@@I@Z 5f80c19d f   tooltip.obj
 0001:0000b2d9       ?DelTool@CToolTipCtrl@@QAEXPAVCWnd@@I@Z 5f80c2d9 f   tooltip.obj
 0001:0000b365       ?GetText@CToolTipCtrl@@QBEXAAVCString@@PAVCWnd@@I@Z 5f80c365 f   tooltip.obj
 0001:0000b40b       ?GetToolInfo@CToolTipCtrl@@QBEHAAVCToolInfo@@PAVCWnd@@I@Z 5f80c40b f   tooltip.obj
 0001:0000b4a1       ?HitTest@CToolTipCtrl@@QBEHPAVCWnd@@VCPoint@@PAUtagTOOLINFOW@@@Z 5f80c4a1 f   tooltip.obj
 0001:0000b586       ?SetToolRect@CToolTipCtrl@@QAEXPAVCWnd@@IPBUtagRECT@@@Z 5f80c586 f   tooltip.obj
 0001:0000b644       ?UpdateTipText@CToolTipCtrl@@QAEXPBGPAVCWnd@@I@Z 5f80c644 f   tooltip.obj
 0001:0000b6d6       ?UpdateTipText@CToolTipCtrl@@QAEXIPAVCWnd@@I@Z 5f80c6d6 f   tooltip.obj
 0001:0000b78b       ?FillInToolInfo@CToolTipCtrl@@QBEXAAUtagTOOLINFOW@@PAVCWnd@@I@Z 5f80c78b f   tooltip.obj
 0001:0000b805       ?_EnableToolTips@CWnd@@QAEHHI@Z 5f80c805 f   tooltip.obj
 0001:0000b92d       ?EnableToolTips@CWnd@@QAEHH@Z 5f80c92d f   tooltip.obj
 0001:0000b948       ?EnableTrackingToolTips@CWnd@@QAEHH@Z 5f80c948 f   tooltip.obj
 0001:0000b966       ?_AfxRelayToolTipMessage@@YGXPAVCToolTipCtrl@@PAUtagMSG@@@Z 5f80c966 f   tooltip.obj
 0001:0000b9f8       ?_FilterToolTipMessage@CWnd@@SGXPAUtagMSG@@PAV1@@Z 5f80c9f8 f   tooltip.obj
 0001:0000ba0b       ?FilterToolTipMessage@CWnd@@QAEXPAUtagMSG@@@Z 5f80ca0b f   tooltip.obj
 0001:0000c1b0       ??1CDragListBox@@UAE@XZ    5f80d1b0 f   winctrl2.obj
 0001:0000c201       ?PreSubclassWindow@CDragListBox@@UAEXXZ 5f80d201 f   winctrl2.obj
 0001:0000c26d       ?BeginDrag@CDragListBox@@UAEHVCPoint@@@Z 5f80d26d f   winctrl2.obj
 0001:0000c2aa       ?CancelDrag@CDragListBox@@UAEXVCPoint@@@Z 5f80d2aa f   winctrl2.obj
 0001:0000c2c7       ?Dragging@CDragListBox@@UAEIVCPoint@@@Z 5f80d2c7 f   winctrl2.obj
 0001:0000c31f       ?Dropped@CDragListBox@@UAEXHVCPoint@@@Z 5f80d31f f   winctrl2.obj
 0001:0000c464       ?DrawInsert@CDragListBox@@UAEXH@Z 5f80d464 f   winctrl2.obj
 0001:0000c4a0       ?DrawSingle@CDragListBox@@QAEXH@Z 5f80d4a0 f   winctrl2.obj
 0001:0000c5a6       ?OnChildNotify@CDragListBox@@MAEHIIJPAJ@Z 5f80d5a6 f   winctrl2.obj
 0001:0000c70b       ?_GetBaseMessageMap@CToolBarCtrl@@KGPBUAFX_MSGMAP@@XZ 5f80d70b f   winctrl2.obj
 0001:0000c715       ?GetMessageMap@CToolBarCtrl@@MBEPBUAFX_MSGMAP@@XZ 5f80d715 f   winctrl2.obj
 0001:0000c725       ?Create@CToolBarCtrl@@QAEHKABUtagRECT@@PAVCWnd@@I@Z 5f80d725 f   winctrl2.obj
 0001:0000c78c       ??1CToolBarCtrl@@UAE@XZ    5f80d78c f   winctrl2.obj
 0001:0000c7dd       ?AddBitmap@CToolBarCtrl@@QAEHHPAVCBitmap@@@Z 5f80d7dd f   winctrl2.obj
 0001:0000c849       ?AddBitmap@CToolBarCtrl@@QAEHHI@Z 5f80d849 f   winctrl2.obj
 0001:0000c8d7       ?SaveState@CToolBarCtrl@@QAEXPAUHKEY__@@PBG1@Z 5f80d8d7 f   winctrl2.obj
 0001:0000c941       ?RestoreState@CToolBarCtrl@@QAEXPAUHKEY__@@PBG1@Z 5f80d941 f   winctrl2.obj
 0001:0000c9ab       ?AddString@CToolBarCtrl@@QAEHI@Z 5f80d9ab f   winctrl2.obj
 0001:0000ca3e       ?OnCreate@CToolBarCtrl@@IAEHPAUtagCREATESTRUCTW@@@Z 5f80da3e f   winctrl2.obj
 0001:0000ca6d       ?GetDropTarget@CToolBarCtrl@@QBEJPAPAUIDropTarget@@@Z 5f80da6d f   winctrl2.obj
 0001:0000cae6       ?Create@CStatusBarCtrl@@QAEHKABUtagRECT@@PAVCWnd@@I@Z 5f80dae6 f   winctrl2.obj
 0001:0000cb4d       ??1CStatusBarCtrl@@UAE@XZ  5f80db4d f   winctrl2.obj
 0001:0000cb9e       ?GetText@CStatusBarCtrl@@QBEHPBGHPAH@Z 5f80db9e f   winctrl2.obj
 0001:0000cc43       ?GetText@CStatusBarCtrl@@QBE?AVCString@@HPAH@Z 5f80dc43 f   winctrl2.obj
 0001:0000cd6f       ?GetTextLength@CStatusBarCtrl@@QBEHHPAH@Z 5f80dd6f f   winctrl2.obj
 0001:0000ce12       ?GetTipText@CStatusBarCtrl@@QBE?AVCString@@H@Z 5f80de12 f   winctrl2.obj
 0001:0000ced4       ?GetBorders@CStatusBarCtrl@@QBEHAAH00@Z 5f80ded4 f   winctrl2.obj
 0001:0000cf50       ?DrawItem@CStatusBarCtrl@@UAEXPAUtagDRAWITEMSTRUCT@@@Z 5f80df50 f   winctrl2.obj
 0001:0000cf86       ?OnChildNotify@CStatusBarCtrl@@MAEHIIJPAJ@Z 5f80df86 f   winctrl2.obj
 0001:0000cff0       ?_GetBaseMessageMap@CListCtrl@@KGPBUAFX_MSGMAP@@XZ 5f80dff0 f   winctrl2.obj
 0001:0000cffa       ?GetMessageMap@CListCtrl@@MBEPBUAFX_MSGMAP@@XZ 5f80dffa f   winctrl2.obj
 0001:0000d00a       ?Create@CListCtrl@@QAEHKABUtagRECT@@PAVCWnd@@I@Z 5f80e00a f   winctrl2.obj
 0001:0000d071       ??1CListCtrl@@UAE@XZ       5f80e071 f   winctrl2.obj
 0001:0000d0c2       ?GetItemRect@CListCtrl@@QBEHHPAUtagRECT@@I@Z 5f80e0c2 f   winctrl2.obj
 0001:0000d122       ?SetItemCountEx@CListCtrl@@QAEHHK@Z 5f80e122 f   winctrl2.obj
 0001:0000d1ab       ?SetIconSpacing@CListCtrl@@QAE?AVCSize@@HH@Z 5f80e1ab f   winctrl2.obj
 0001:0000d235       ?SetIconSpacing@CListCtrl@@QAE?AVCSize@@V2@@Z 5f80e235 f   winctrl2.obj
 0001:0000d2bf       ?GetSubItemRect@CListCtrl@@QAEHHHHAAVCRect@@@Z 5f80e2bf f   winctrl2.obj
 0001:0000d369       ?InsertColumn@CListCtrl@@QAEHHPBGHHH@Z 5f80e369 f   winctrl2.obj
 0001:0000d3c5       ?InsertItem@CListCtrl@@QAEHIHPBGIIHJ@Z 5f80e3c5 f   winctrl2.obj
 0001:0000d442       ?HitTest@CListCtrl@@QBEHVCPoint@@PAI@Z 5f80e442 f   winctrl2.obj
 0001:0000d4ba       ?SetItem@CListCtrl@@QAEHHHIPBGHIIJ@Z 5f80e4ba f   winctrl2.obj
 0001:0000d56d       ?SetItemState@CListCtrl@@QAEHHII@Z 5f80e56d f   winctrl2.obj
 0001:0000d5d3       ?SetItemText@CListCtrl@@QAEHHHPBG@Z 5f80e5d3 f   winctrl2.obj
 0001:0000d664       ?GetItemText@CListCtrl@@QBE?AVCString@@HH@Z 5f80e664 f   winctrl2.obj
 0001:0000d769       ?GetItemText@CListCtrl@@QBEHHHPAGH@Z 5f80e769 f   winctrl2.obj
 0001:0000d7e5       ?GetItemData@CListCtrl@@QBEKH@Z 5f80e7e5 f   winctrl2.obj
 0001:0000d87b       ?DrawItem@CListCtrl@@UAEXPAUtagDRAWITEMSTRUCT@@@Z 5f80e87b f   winctrl2.obj
 0001:0000d8b1       ?OnChildNotify@CListCtrl@@MAEHIIJPAJ@Z 5f80e8b1 f   winctrl2.obj
 0001:0000d91b       ?RemoveImageList@CListCtrl@@IAEXH@Z 5f80e91b f   winctrl2.obj
 0001:0000d960       ?OnNcDestroy@CListCtrl@@IAEXXZ 5f80e960 f   winctrl2.obj
 0001:0000d991       ?CreateDragImage@CListCtrl@@QAEPAVCImageList@@HPAUtagPOINT@@@Z 5f80e991 f   winctrl2.obj
 0001:0000da8c       ?_GetBaseMessageMap@CTreeCtrl@@KGPBUAFX_MSGMAP@@XZ 5f80ea8c f   winctrl2.obj
 0001:0000da96       ?GetMessageMap@CTreeCtrl@@MBEPBUAFX_MSGMAP@@XZ 5f80ea96 f   winctrl2.obj
 0001:0000daa6       ?Create@CTreeCtrl@@QAEHKABUtagRECT@@PAVCWnd@@I@Z 5f80eaa6 f   winctrl2.obj
 0001:0000db0d       ??1CTreeCtrl@@UAE@XZ       5f80eb0d f   winctrl2.obj
 0001:0000db5e       ?GetItemRect@CTreeCtrl@@QBEHPAU_TREEITEM@@PAUtagRECT@@H@Z 5f80eb5e f   winctrl2.obj
 0001:0000dbbe       ?GetItemText@CTreeCtrl@@QBE?AVCString@@PAU_TREEITEM@@@Z 5f80ebbe f   winctrl2.obj
 0001:0000dcc2       ?GetItemImage@CTreeCtrl@@QBEHPAU_TREEITEM@@AAH1@Z 5f80ecc2 f   winctrl2.obj
 0001:0000dd43       ?GetItemState@CTreeCtrl@@QBEIPAU_TREEITEM@@I@Z 5f80ed43 f   winctrl2.obj
 0001:0000ddd6       ?GetItemData@CTreeCtrl@@QBEKPAU_TREEITEM@@@Z 5f80edd6 f   winctrl2.obj
 0001:0000de5c       ?ItemHasChildren@CTreeCtrl@@QBEHPAU_TREEITEM@@@Z 5f80ee5c f   winctrl2.obj
 0001:0000dec4       ?SetItem@CTreeCtrl@@QAEHPAU_TREEITEM@@IPBGHHIIJ@Z 5f80eec4 f   winctrl2.obj
 0001:0000df4c       ?InsertItem@CTreeCtrl@@QAEPAU_TREEITEM@@IPBGHHIIJPAU2@1@Z 5f80ef4c f   winctrl2.obj
 0001:0000dfda       ?HitTest@CTreeCtrl@@QBEPAU_TREEITEM@@VCPoint@@PAI@Z 5f80efda f   winctrl2.obj
 0001:0000e052       ?RemoveImageList@CTreeCtrl@@IAEXH@Z 5f80f052 f   winctrl2.obj
 0001:0000e097       ?OnDestroy@CTreeCtrl@@QAEXXZ 5f80f097 f   winctrl2.obj
 0001:0000e0be       ?CreateDragImage@CTreeCtrl@@QAEPAVCImageList@@PAU_TREEITEM@@@Z 5f80f0be f   winctrl2.obj
 0001:0000e1b7       ?GetCheck@CTreeCtrl@@QBEHPAU_TREEITEM@@@Z 5f80f1b7 f   winctrl2.obj
 0001:0000e24a       ?SetCheck@CTreeCtrl@@QAEHPAU_TREEITEM@@H@Z 5f80f24a f   winctrl2.obj
 0001:0000e2c6       ?Create@CSpinButtonCtrl@@QAEHKABUtagRECT@@PAVCWnd@@I@Z 5f80f2c6 f   winctrl2.obj
 0001:0000e32a       ??1CSpinButtonCtrl@@UAE@XZ 5f80f32a f   winctrl2.obj
 0001:0000e37b       ?GetRange@CSpinButtonCtrl@@QBEXAAH0@Z 5f80f37b f   winctrl2.obj
 0001:0000e3f1       ?Create@CSliderCtrl@@QAEHKABUtagRECT@@PAVCWnd@@I@Z 5f80f3f1 f   winctrl2.obj
 0001:0000e458       ??1CSliderCtrl@@UAE@XZ     5f80f458 f   winctrl2.obj
 0001:0000e4a9       ?GetRange@CSliderCtrl@@QBEXAAH0@Z 5f80f4a9 f   winctrl2.obj
 0001:0000e501       ?SetRange@CSliderCtrl@@QAEXHHH@Z 5f80f501 f   winctrl2.obj
 0001:0000e52e       ?GetSelection@CSliderCtrl@@QBEXAAH0@Z 5f80f52e f   winctrl2.obj
 0001:0000e5a2       ?SetSelection@CSliderCtrl@@QAEXHH@Z 5f80f5a2 f   winctrl2.obj
 0001:0000e610       ?Create@CProgressCtrl@@QAEHKABUtagRECT@@PAVCWnd@@I@Z 5f80f610 f   winctrl2.obj
 0001:0000e677       ??1CProgressCtrl@@UAE@XZ   5f80f677 f   winctrl2.obj
 0001:0000e6c8       ?Create@CHeaderCtrl@@QAEHKABUtagRECT@@PAVCWnd@@I@Z 5f80f6c8 f   winctrl2.obj
 0001:0000e72f       ??1CHeaderCtrl@@UAE@XZ     5f80f72f f   winctrl2.obj
 0001:0000e780       ?DrawItem@CHeaderCtrl@@UAEXPAUtagDRAWITEMSTRUCT@@@Z 5f80f780 f   winctrl2.obj
 0001:0000e7b6       ?OnChildNotify@CHeaderCtrl@@MAEHIIJPAJ@Z 5f80f7b6 f   winctrl2.obj
 0001:0000e820       ?Create@CHotKeyCtrl@@QAEHKABUtagRECT@@PAVCWnd@@I@Z 5f80f820 f   winctrl2.obj
 0001:0000e887       ??1CHotKeyCtrl@@UAE@XZ     5f80f887 f   winctrl2.obj
 0001:0000e8d8       ?GetHotKey@CHotKeyCtrl@@QBEXAAG0@Z 5f80f8d8 f   winctrl2.obj
 0001:0000e959       ?_GetBaseMessageMap@CTabCtrl@@KGPBUAFX_MSGMAP@@XZ 5f80f959 f   winctrl2.obj
 0001:0000e963       ?GetMessageMap@CTabCtrl@@MBEPBUAFX_MSGMAP@@XZ 5f80f963 f   winctrl2.obj
 0001:0000e973       ?Create@CTabCtrl@@QAEHKABUtagRECT@@PAVCWnd@@I@Z 5f80f973 f   winctrl2.obj
 0001:0000e9da       ??1CTabCtrl@@UAE@XZ        5f80f9da f   winctrl2.obj
 0001:0000ea2b       ?DrawItem@CTabCtrl@@UAEXPAUtagDRAWITEMSTRUCT@@@Z 5f80fa2b f   winctrl2.obj
 0001:0000ea61       ?OnChildNotify@CTabCtrl@@MAEHIIJPAJ@Z 5f80fa61 f   winctrl2.obj
 0001:0000eacb       ?OnDestroy@CTabCtrl@@IAEXXZ 5f80facb f   winctrl2.obj
 0001:0000eb12       ?GetItemState@CTabCtrl@@QBEKHK@Z 5f80fb12 f   winctrl2.obj
 0001:0000eb9a       ?SetItemState@CTabCtrl@@QAEHHKK@Z 5f80fb9a f   winctrl2.obj
 0001:0000ec07       ?InsertItem@CTabCtrl@@QAEHIHPBGHJ@Z 5f80fc07 f   winctrl2.obj
 0001:0000ec79       ?InsertItem@CTabCtrl@@QAEHIHPBGHJKK@Z 5f80fc79 f   winctrl2.obj
 0001:0000ecf7       ?Create@CAnimateCtrl@@QAEHKABUtagRECT@@PAVCWnd@@I@Z 5f80fcf7 f   winctrl2.obj
 0001:0000ed5e       ??1CAnimateCtrl@@UAE@XZ    5f80fd5e f   winctrl2.obj
 0001:0000edaf       ??1CRichEditCtrl@@UAE@XZ   5f80fdaf f   winctrl2.obj
 0001:0000ee00       ?afxMapHIMAGELIST@@YGPAVCHandleMap@@H@Z 5f80fe00 f   winctrl2.obj
 0001:0000eed0       ??0CImageList@@QAE@XZ      5f80fed0 f   winctrl2.obj
 0001:0000eef9       ??1CImageList@@UAE@XZ      5f80fef9 f   winctrl2.obj
 0001:0000ef4a       ?Detach@CImageList@@QAEPAU_IMAGELIST@@XZ 5f80ff4a f   winctrl2.obj
 0001:0000ef92       ?DeleteImageList@CImageList@@QAEHXZ 5f80ff92 f   winctrl2.obj
 0001:0000efb9       ?FromHandle@CImageList@@SGPAV1@PAU_IMAGELIST@@@Z 5f80ffb9 f   winctrl2.obj
 0001:0000f032       ?FromHandlePermanent@CImageList@@SGPAV1@PAU_IMAGELIST@@@Z 5f810032 f   winctrl2.obj
 0001:0000f098       ?Create@CImageList@@QAEHHHIHH@Z 5f810098 f   winctrl2.obj
 0001:0000f0c8       ?Create@CImageList@@QAEHIHHK@Z 5f8100c8 f   winctrl2.obj
 0001:0000f160       ?Create@CImageList@@QAEHPBGHHK@Z 5f810160 f   winctrl2.obj
 0001:0000f1ca       ?Create@CImageList@@QAEHAAV1@H0HHH@Z 5f8101ca f   winctrl2.obj
 0001:0000f204       ?Attach@CImageList@@QAEHPAU_IMAGELIST@@@Z 5f810204 f   winctrl2.obj
 0001:0000f2b5       ?Read@CImageList@@QAEHPAVCArchive@@@Z 5f8102b5 f   winctrl2.obj
 0001:0000f35a       ?Write@CImageList@@QAEHPAVCArchive@@@Z 5f81035a f   winctrl2.obj
 0001:0000f3f4       ?Dump@CImageList@@UBEXAAVCDumpContext@@@Z 5f8103f4 f   winctrl2.obj
 0001:0000f435       ?AssertValid@CImageList@@UBEXXZ 5f810435 f   winctrl2.obj
 0001:0000f4f4       ??0CDragListBox@@QAE@XZ    5f8104f4 f   winctrl2.obj
 0001:0000f51d       ?ItemFromPt@CDragListBox@@QBEHVCPoint@@H@Z 5f81051d f   winctrl2.obj
 0001:0000f57f       ??0CToolBarCtrl@@QAE@XZ    5f81057f f   winctrl2.obj
 0001:0000f59e       ?EnableButton@CToolBarCtrl@@QAEHHH@Z 5f81059e f   winctrl2.obj
 0001:0000f5f8       ?CheckButton@CToolBarCtrl@@QAEHHH@Z 5f8105f8 f   winctrl2.obj
 0001:0000f652       ?PressButton@CToolBarCtrl@@QAEHHH@Z 5f810652 f   winctrl2.obj
 0001:0000f6ac       ?HideButton@CToolBarCtrl@@QAEHHH@Z 5f8106ac f   winctrl2.obj
 0001:0000f706       ?Indeterminate@CToolBarCtrl@@QAEHHH@Z 5f810706 f   winctrl2.obj
 0001:0000f760       ?IsButtonEnabled@CToolBarCtrl@@QBEHH@Z 5f810760 f   winctrl2.obj
 0001:0000f7b3       ?IsButtonChecked@CToolBarCtrl@@QBEHH@Z 5f8107b3 f   winctrl2.obj
 0001:0000f806       ?IsButtonPressed@CToolBarCtrl@@QBEHH@Z 5f810806 f   winctrl2.obj
 0001:0000f859       ?IsButtonHidden@CToolBarCtrl@@QBEHH@Z 5f810859 f   winctrl2.obj
 0001:0000f8ac       ?IsButtonIndeterminate@CToolBarCtrl@@QBEHH@Z 5f8108ac f   winctrl2.obj
 0001:0000f8ff       ?SetState@CToolBarCtrl@@QAEHHI@Z 5f8108ff f   winctrl2.obj
 0001:0000f959       ?GetState@CToolBarCtrl@@QBEHH@Z 5f810959 f   winctrl2.obj
 0001:0000f9ac       ?AddButtons@CToolBarCtrl@@QAEHHPAU_TBBUTTON@@@Z 5f8109ac f   winctrl2.obj
 0001:0000fa01       ?InsertButton@CToolBarCtrl@@QAEHHPAU_TBBUTTON@@@Z 5f810a01 f   winctrl2.obj
 0001:0000fa56       ?DeleteButton@CToolBarCtrl@@QAEHH@Z 5f810a56 f   winctrl2.obj
 0001:0000faa9       ?GetButton@CToolBarCtrl@@QBEHHPAU_TBBUTTON@@@Z 5f810aa9 f   winctrl2.obj
 0001:0000fafe       ?GetButtonCount@CToolBarCtrl@@QBEHXZ 5f810afe f   winctrl2.obj
 0001:0000fb4d       ?CommandToIndex@CToolBarCtrl@@QBEII@Z 5f810b4d f   winctrl2.obj
 0001:0000fba0       ?Customize@CToolBarCtrl@@QAEXXZ 5f810ba0 f   winctrl2.obj
 0001:0000fbef       ?AddStrings@CToolBarCtrl@@QAEHPBG@Z 5f810bef f   winctrl2.obj
 0001:0000fc42       ?GetItemRect@CToolBarCtrl@@QBEHHPAUtagRECT@@@Z 5f810c42 f   winctrl2.obj
 0001:0000fc97       ?SetButtonStructSize@CToolBarCtrl@@QAEXH@Z 5f810c97 f   winctrl2.obj
 0001:0000fcea       ?SetButtonSize@CToolBarCtrl@@QAEHVCSize@@@Z 5f810cea f   winctrl2.obj
 0001:0000fd50       ?SetBitmapSize@CToolBarCtrl@@QAEHVCSize@@@Z 5f810d50 f   winctrl2.obj
 0001:0000fdb6       ?AutoSize@CToolBarCtrl@@QAEXXZ 5f810db6 f   winctrl2.obj
 0001:0000fe05       ?GetToolTips@CToolBarCtrl@@QBEPAVCToolTipCtrl@@XZ 5f810e05 f   winctrl2.obj
 0001:0000fe5a       ?SetToolTips@CToolBarCtrl@@QAEXPAVCToolTipCtrl@@@Z 5f810e5a f   winctrl2.obj
 0001:0000feb2       ?SetOwner@CToolBarCtrl@@QAEXPAVCWnd@@@Z 5f810eb2 f   winctrl2.obj
 0001:0000ff0a       ?SetRows@CToolBarCtrl@@QAEXHHPAUtagRECT@@@Z 5f810f0a f   winctrl2.obj
 0001:0000ff73       ?GetRows@CToolBarCtrl@@QBEHXZ 5f810f73 f   winctrl2.obj
 0001:0000ffc2       ?SetCmdID@CToolBarCtrl@@QAEHHI@Z 5f810fc2 f   winctrl2.obj
 0001:00010017       ?GetBitmapFlags@CToolBarCtrl@@QBEIXZ 5f811017 f   winctrl2.obj
 0001:00010066       ?HitTest@CToolBarCtrl@@QBEHPAUtagPOINT@@@Z 5f811066 f   winctrl2.obj
 0001:000100b9       ?GetExtendedStyle@CToolBarCtrl@@QBEKXZ 5f8110b9 f   winctrl2.obj
 0001:00010108       ?SetExtendedStyle@CToolBarCtrl@@QAEKK@Z 5f811108 f   winctrl2.obj
 0001:0001015b       ?GetInsertMarkColor@CToolBarCtrl@@QBEKXZ 5f81115b f   winctrl2.obj
 0001:000101aa       ?SetInsertMarkColor@CToolBarCtrl@@QAEKK@Z 5f8111aa f   winctrl2.obj
 0001:000101fd       ??0CStatusBarCtrl@@QAE@XZ  5f8111fd f   winctrl2.obj
 0001:0001021c       ?SetText@CStatusBarCtrl@@QAEHPBGHH@Z 5f81121c f   winctrl2.obj
 0001:00010294       ?SetParts@CStatusBarCtrl@@QAEHHPAH@Z 5f811294 f   winctrl2.obj
 0001:000102e9       ?GetParts@CStatusBarCtrl@@QBEHHPAH@Z 5f8112e9 f   winctrl2.obj
 0001:0001033e       ?GetBorders@CStatusBarCtrl@@QBEHPAH@Z 5f81133e f   winctrl2.obj
 0001:00010391       ?SetMinHeight@CStatusBarCtrl@@QAEXH@Z 5f811391 f   winctrl2.obj
 0001:000103e4       ?SetSimple@CStatusBarCtrl@@QAEHH@Z 5f8113e4 f   winctrl2.obj
 0001:00010437       ?GetRect@CStatusBarCtrl@@QBEHHPAUtagRECT@@@Z 5f811437 f   winctrl2.obj
 0001:0001048c       ??0CListCtrl@@QAE@XZ       5f81148c f   winctrl2.obj
 0001:000104ab       ?GetBkColor@CListCtrl@@QBEKXZ 5f8114ab f   winctrl2.obj
 0001:000104fa       ?SetBkColor@CListCtrl@@QAEHK@Z 5f8114fa f   winctrl2.obj
 0001:0001054d       ?GetImageList@CListCtrl@@QBEPAVCImageList@@H@Z 5f81154d f   winctrl2.obj
 0001:000105a9       ?SetImageList@CListCtrl@@QAEPAVCImageList@@PAV2@H@Z 5f8115a9 f   winctrl2.obj
 0001:0001060c       ?GetItemCount@CListCtrl@@QBEHXZ 5f81160c f   winctrl2.obj
 0001:0001065e       ?GetItem@CListCtrl@@QBEHPAUtagLVITEMW@@@Z 5f81165e f   winctrl2.obj
 0001:000106b4       ?SetItem@CListCtrl@@QAEHPBUtagLVITEMW@@@Z 5f8116b4 f   winctrl2.obj
 0001:0001070a       ?SetItemData@CListCtrl@@QAEHHK@Z 5f81170a f   winctrl2.obj
 0001:00010764       ?InsertItem@CListCtrl@@QAEHPBUtagLVITEMW@@@Z 5f811764 f   winctrl2.obj
 0001:000107ba       ?InsertItem@CListCtrl@@QAEHHPBG@Z 5f8117ba f   winctrl2.obj
 0001:00010812       ?InsertItem@CListCtrl@@QAEHHPBGH@Z 5f811812 f   winctrl2.obj
 0001:0001086c       ?DeleteItem@CListCtrl@@QAEHH@Z 5f81186c f   winctrl2.obj
 0001:000108c2       ?DeleteAllItems@CListCtrl@@QAEHXZ 5f8118c2 f   winctrl2.obj
 0001:00010914       ?GetCallbackMask@CListCtrl@@QBEIXZ 5f811914 f   winctrl2.obj
 0001:00010966       ?SetCallbackMask@CListCtrl@@QAEHI@Z 5f811966 f   winctrl2.obj
 0001:000109bc       ?GetNextItem@CListCtrl@@QBEHHH@Z 5f8119bc f   winctrl2.obj
 0001:00010a19       ?GetFirstSelectedItemPosition@CListCtrl@@QBEPAU__POSITION@@XZ 5f811a19 f   winctrl2.obj
 0001:00010a64       ?GetNextSelectedItem@CListCtrl@@QBEHAAPAU__POSITION@@@Z 5f811a64 f   winctrl2.obj
 0001:00010ac8       ?FindItem@CListCtrl@@QBEHPAUtagLVFINDINFOW@@H@Z 5f811ac8 f   winctrl2.obj
 0001:00010b20       ?HitTest@CListCtrl@@QBEHPAUtagLVHITTESTINFO@@@Z 5f811b20 f   winctrl2.obj
 0001:00010b76       ?SetItemPosition@CListCtrl@@QAEHHUtagPOINT@@@Z 5f811b76 f   winctrl2.obj
 0001:00010bf9       ?GetItemPosition@CListCtrl@@QBEHHPAUtagPOINT@@@Z 5f811bf9 f   winctrl2.obj
 0001:00010c51       ?GetStringWidth@CListCtrl@@QBEHPBG@Z 5f811c51 f   winctrl2.obj
 0001:00010ca7       ?EnsureVisible@CListCtrl@@QAEHHH@Z 5f811ca7 f   winctrl2.obj
 0001:00010d04       ?Scroll@CListCtrl@@QAEHVCSize@@@Z 5f811d04 f   winctrl2.obj
 0001:00010d5c       ?RedrawItems@CListCtrl@@QAEHHH@Z 5f811d5c f   winctrl2.obj
 0001:00010db4       ?Arrange@CListCtrl@@QAEHI@Z 5f811db4 f   winctrl2.obj
 0001:00010e0a       ?EditLabel@CListCtrl@@QAEPAVCEdit@@H@Z 5f811e0a f   winctrl2.obj
 0001:00010e66       ?GetEditControl@CListCtrl@@QBEPAVCEdit@@XZ 5f811e66 f   winctrl2.obj
 0001:00010ebe       ?GetColumn@CListCtrl@@QBEHHPAUtagLVCOLUMNW@@@Z 5f811ebe f   winctrl2.obj
 0001:00010f16       ?SetColumn@CListCtrl@@QAEHHPBUtagLVCOLUMNW@@@Z 5f811f16 f   winctrl2.obj
 0001:00010f6e       ?InsertColumn@CListCtrl@@QAEHHPBUtagLVCOLUMNW@@@Z 5f811f6e f   winctrl2.obj
 0001:00010fc6       ?DeleteColumn@CListCtrl@@QAEHH@Z 5f811fc6 f   winctrl2.obj
 0001:0001101c       ?GetColumnWidth@CListCtrl@@QBEHH@Z 5f81201c f   winctrl2.obj
 0001:00011072       ?SetColumnWidth@CListCtrl@@QAEHHH@Z 5f812072 f   winctrl2.obj
 0001:000110cf       ?GetViewRect@CListCtrl@@QBEHPAUtagRECT@@@Z 5f8120cf f   winctrl2.obj
 0001:00011125       ?GetTextColor@CListCtrl@@QBEKXZ 5f812125 f   winctrl2.obj
 0001:00011177       ?SetTextColor@CListCtrl@@QAEHK@Z 5f812177 f   winctrl2.obj
 0001:000111cd       ?GetTextBkColor@CListCtrl@@QBEKXZ 5f8121cd f   winctrl2.obj
 0001:0001121f       ?SetTextBkColor@CListCtrl@@QAEHK@Z 5f81221f f   winctrl2.obj
 0001:00011275       ?GetTopIndex@CListCtrl@@QBEHXZ 5f812275 f   winctrl2.obj
 0001:000112c7       ?GetCountPerPage@CListCtrl@@QBEHXZ 5f8122c7 f   winctrl2.obj
 0001:00011319       ?GetOrigin@CListCtrl@@QBEHPAUtagPOINT@@@Z 5f812319 f   winctrl2.obj
 0001:0001136f       ?Update@CListCtrl@@QAEHH@Z 5f81236f f   winctrl2.obj
 0001:000113c5       ?SetItemState@CListCtrl@@QAEHHPAUtagLVITEMW@@@Z 5f8123c5 f   winctrl2.obj
 0001:0001141d       ?GetItemState@CListCtrl@@QBEIHI@Z 5f81241d f   winctrl2.obj
 0001:00011475       ?SetItemCount@CListCtrl@@QAEXH@Z 5f812475 f   winctrl2.obj
 0001:000114cb       ?SortItems@CListCtrl@@QAEHP6GHJJJ@ZK@Z 5f8124cb f   winctrl2.obj
 0001:0001154e       ?GetSelectedCount@CListCtrl@@QBEIXZ 5f81254e f   winctrl2.obj
 0001:000115a0       ??0CTreeCtrl@@QAE@XZ       5f8125a0 f   winctrl2.obj
 0001:000115bf       ?InsertItem@CTreeCtrl@@QAEPAU_TREEITEM@@PAUtagTVINSERTSTRUCTW@@@Z 5f8125bf f   winctrl2.obj
 0001:00011615       ?InsertItem@CTreeCtrl@@QAEPAU_TREEITEM@@PBGHHPAU2@1@Z 5f812615 f   winctrl2.obj
 0001:00011677       ?InsertItem@CTreeCtrl@@QAEPAU_TREEITEM@@PBGPAU2@1@Z 5f812677 f   winctrl2.obj
 0001:000116d5       ?DeleteItem@CTreeCtrl@@QAEHPAU_TREEITEM@@@Z 5f8126d5 f   winctrl2.obj
 0001:0001172b       ?DeleteAllItems@CTreeCtrl@@QAEHXZ 5f81272b f   winctrl2.obj
 0001:00011780       ?Expand@CTreeCtrl@@QAEHPAU_TREEITEM@@I@Z 5f812780 f   winctrl2.obj
 0001:000117d8       ?GetCount@CTreeCtrl@@QBEIXZ 5f8127d8 f   winctrl2.obj
 0001:0001182a       ?GetIndent@CTreeCtrl@@QBEIXZ 5f81282a f   winctrl2.obj
 0001:0001187c       ?SetIndent@CTreeCtrl@@QAEXI@Z 5f81287c f   winctrl2.obj
 0001:000118d2       ?GetImageList@CTreeCtrl@@QBEPAVCImageList@@I@Z 5f8128d2 f   winctrl2.obj
 0001:0001192e       ?SetImageList@CTreeCtrl@@QAEPAVCImageList@@PAV2@H@Z 5f81292e f   winctrl2.obj
 0001:00011991       ?GetNextItem@CTreeCtrl@@QBEPAU_TREEITEM@@PAU2@I@Z 5f812991 f   winctrl2.obj
 0001:000119e9       ?GetChildItem@CTreeCtrl@@QBEPAU_TREEITEM@@PAU2@@Z 5f8129e9 f   winctrl2.obj
 0001:00011a3f       ?GetNextSiblingItem@CTreeCtrl@@QBEPAU_TREEITEM@@PAU2@@Z 5f812a3f f   winctrl2.obj
 0001:00011a95       ?GetPrevSiblingItem@CTreeCtrl@@QBEPAU_TREEITEM@@PAU2@@Z 5f812a95 f   winctrl2.obj
 0001:00011aeb       ?GetParentItem@CTreeCtrl@@QBEPAU_TREEITEM@@PAU2@@Z 5f812aeb f   winctrl2.obj
 0001:00011b41       ?GetFirstVisibleItem@CTreeCtrl@@QBEPAU_TREEITEM@@XZ 5f812b41 f   winctrl2.obj
 0001:00011b93       ?GetNextVisibleItem@CTreeCtrl@@QBEPAU_TREEITEM@@PAU2@@Z 5f812b93 f   winctrl2.obj
 0001:00011be9       ?GetPrevVisibleItem@CTreeCtrl@@QBEPAU_TREEITEM@@PAU2@@Z 5f812be9 f   winctrl2.obj
 0001:00011c3f       ?GetSelectedItem@CTreeCtrl@@QBEPAU_TREEITEM@@XZ 5f812c3f f   winctrl2.obj
 0001:00011c91       ?GetDropHilightItem@CTreeCtrl@@QBEPAU_TREEITEM@@XZ 5f812c91 f   winctrl2.obj
 0001:00011ce3       ?GetRootItem@CTreeCtrl@@QBEPAU_TREEITEM@@XZ 5f812ce3 f   winctrl2.obj
 0001:00011d35       ?Select@CTreeCtrl@@QAEHPAU_TREEITEM@@I@Z 5f812d35 f   winctrl2.obj
 0001:00011d8d       ?SelectItem@CTreeCtrl@@QAEHPAU_TREEITEM@@@Z 5f812d8d f   winctrl2.obj
 0001:00011de3       ?SelectDropTarget@CTreeCtrl@@QAEHPAU_TREEITEM@@@Z 5f812de3 f   winctrl2.obj
 0001:00011e39       ?SelectSetFirstVisible@CTreeCtrl@@QAEHPAU_TREEITEM@@@Z 5f812e39 f   winctrl2.obj
 0001:00011e8f       ?GetItem@CTreeCtrl@@QBEHPAUtagTVITEMW@@@Z 5f812e8f f   winctrl2.obj
 0001:00011ee5       ?SetItem@CTreeCtrl@@QAEHPAUtagTVITEMW@@@Z 5f812ee5 f   winctrl2.obj
 0001:00011f3b       ?SetItemText@CTreeCtrl@@QAEHPAU_TREEITEM@@PBG@Z 5f812f3b f   winctrl2.obj
 0001:00011f95       ?SetItemImage@CTreeCtrl@@QAEHPAU_TREEITEM@@HH@Z 5f812f95 f   winctrl2.obj
 0001:00011ff1       ?SetItemState@CTreeCtrl@@QAEHPAU_TREEITEM@@II@Z 5f812ff1 f   winctrl2.obj
 0001:0001204d       ?SetItemData@CTreeCtrl@@QAEHPAU_TREEITEM@@K@Z 5f81304d f   winctrl2.obj
 0001:000120a7       ?EditLabel@CTreeCtrl@@QAEPAVCEdit@@PAU_TREEITEM@@@Z 5f8130a7 f   winctrl2.obj
 0001:00012103       ?HitTest@CTreeCtrl@@QBEPAU_TREEITEM@@PAUtagTVHITTESTINFO@@@Z 5f813103 f   winctrl2.obj
 0001:00012159       ?GetEditControl@CTreeCtrl@@QBEPAVCEdit@@XZ 5f813159 f   winctrl2.obj
 0001:000121b1       ?GetVisibleCount@CTreeCtrl@@QBEIXZ 5f8131b1 f   winctrl2.obj
 0001:00012203       ?SortChildren@CTreeCtrl@@QAEHPAU_TREEITEM@@@Z 5f813203 f   winctrl2.obj
 0001:00012259       ?EnsureVisible@CTreeCtrl@@QAEHPAU_TREEITEM@@@Z 5f813259 f   winctrl2.obj
 0001:000122af       ?SortChildrenCB@CTreeCtrl@@QAEHPAUtagTVSORTCB@@@Z 5f8132af f   winctrl2.obj
 0001:00012305       ?GetToolTips@CTreeCtrl@@QBEPAVCToolTipCtrl@@XZ 5f813305 f   winctrl2.obj
 0001:0001235d       ?SetToolTips@CTreeCtrl@@QAEPAVCToolTipCtrl@@PAV2@@Z 5f81335d f   winctrl2.obj
 0001:000123be       ?GetBkColor@CTreeCtrl@@QBEKXZ 5f8133be f   winctrl2.obj
 0001:00012410       ?SetBkColor@CTreeCtrl@@QAEKK@Z 5f813410 f   winctrl2.obj
 0001:00012466       ?GetItemHeight@CTreeCtrl@@QBEFXZ 5f813466 f   winctrl2.obj
 0001:000124b8       ?SetItemHeight@CTreeCtrl@@QAEFF@Z 5f8134b8 f   winctrl2.obj
 0001:0001250f       ?GetTextColor@CTreeCtrl@@QBEKXZ 5f81350f f   winctrl2.obj
 0001:00012561       ?SetTextColor@CTreeCtrl@@QAEKK@Z 5f813561 f   winctrl2.obj
 0001:000125b7       ?SetInsertMark@CTreeCtrl@@QAEHPAU_TREEITEM@@H@Z 5f8135b7 f   winctrl2.obj
 0001:0001260f       ?GetInsertMarkColor@CTreeCtrl@@QBEKXZ 5f81360f f   winctrl2.obj
 0001:00012661       ?SetInsertMarkColor@CTreeCtrl@@QAEKK@Z 5f813661 f   winctrl2.obj
 0001:000126b7       ??0CHotKeyCtrl@@QAE@XZ     5f8136b7 f   winctrl2.obj
 0001:000126d6       ?SetHotKey@CHotKeyCtrl@@QAEXGG@Z 5f8136d6 f   winctrl2.obj
 0001:00012744       ?GetHotKey@CHotKeyCtrl@@QBEKXZ 5f813744 f   winctrl2.obj
 0001:00012796       ?SetRules@CHotKeyCtrl@@QAEXGG@Z 5f813796 f   winctrl2.obj
 0001:000127f9       ?Activate@CToolTipCtrl@@QAEXH@Z 5f8137f9 f   winctrl2.obj
 0001:0001284f       ?SetToolInfo@CToolTipCtrl@@QAEXPAUtagTOOLINFOW@@@Z 5f81384f f   winctrl2.obj
 0001:000128a5       ?RelayEvent@CToolTipCtrl@@QAEXPAUtagMSG@@@Z 5f8138a5 f   winctrl2.obj
 0001:000128fb       ?GetToolCount@CToolTipCtrl@@QBEHXZ 5f8138fb f   winctrl2.obj
 0001:0001294d       ??0CSpinButtonCtrl@@QAE@XZ 5f81394d f   winctrl2.obj
 0001:0001296c       ?GetAccel@CSpinButtonCtrl@@QBEIHPAU_UDACCEL@@@Z 5f81396c f   winctrl2.obj
 0001:000129c9       ?GetBase@CSpinButtonCtrl@@QBEIXZ 5f8139c9 f   winctrl2.obj
 0001:00012a20       ?GetBuddy@CSpinButtonCtrl@@QBEPAVCWnd@@XZ 5f813a20 f   winctrl2.obj
 0001:00012a78       ?GetPos@CSpinButtonCtrl@@QBEHXZ 5f813a78 f   winctrl2.obj
 0001:00012aca       ?GetRange@CSpinButtonCtrl@@QBEKXZ 5f813aca f   winctrl2.obj
 0001:00012b1c       ?SetAccel@CSpinButtonCtrl@@QAEHHPAU_UDACCEL@@@Z 5f813b1c f   winctrl2.obj
 0001:00012b79       ?SetBase@CSpinButtonCtrl@@QAEHH@Z 5f813b79 f   winctrl2.obj
 0001:00012bcf       ?SetBuddy@CSpinButtonCtrl@@QAEPAVCWnd@@PAV2@@Z 5f813bcf f   winctrl2.obj
 0001:00012c30       ?SetPos@CSpinButtonCtrl@@QAEHH@Z 5f813c30 f   winctrl2.obj
 0001:00012c8e       ?SetRange@CSpinButtonCtrl@@QAEXHH@Z 5f813c8e f   winctrl2.obj
 0001:00012cf7       ??0CSliderCtrl@@QAE@XZ     5f813cf7 f   winctrl2.obj
 0001:00012d16       ?GetLineSize@CSliderCtrl@@QBEHXZ 5f813d16 f   winctrl2.obj
 0001:00012d68       ?SetLineSize@CSliderCtrl@@QAEHH@Z 5f813d68 f   winctrl2.obj
 0001:00012dbe       ?GetPageSize@CSliderCtrl@@QBEHXZ 5f813dbe f   winctrl2.obj
 0001:00012e10       ?SetPageSize@CSliderCtrl@@QAEHH@Z 5f813e10 f   winctrl2.obj
 0001:00012e66       ?GetRangeMax@CSliderCtrl@@QBEHXZ 5f813e66 f   winctrl2.obj
 0001:00012eb8       ?GetRangeMin@CSliderCtrl@@QBEHXZ 5f813eb8 f   winctrl2.obj
 0001:00012f0a       ?SetRangeMin@CSliderCtrl@@QAEXHH@Z 5f813f0a f   winctrl2.obj
 0001:00012f62       ?SetRangeMax@CSliderCtrl@@QAEXHH@Z 5f813f62 f   winctrl2.obj
 0001:00012fba       ?ClearSel@CSliderCtrl@@QAEXH@Z 5f813fba f   winctrl2.obj
 0001:00013010       ?GetChannelRect@CSliderCtrl@@QBEXPAUtagRECT@@@Z 5f814010 f   winctrl2.obj
 0001:00013066       ?GetThumbRect@CSliderCtrl@@QBEXPAUtagRECT@@@Z 5f814066 f   winctrl2.obj
 0001:000130bc       ?GetPos@CSliderCtrl@@QBEHXZ 5f8140bc f   winctrl2.obj
 0001:0001310e       ?SetPos@CSliderCtrl@@QAEXH@Z 5f81410e f   winctrl2.obj
 0001:00013164       ?VerifyPos@CSliderCtrl@@QAEXXZ 5f814164 f   winctrl2.obj
 0001:000131b6       ?ClearTics@CSliderCtrl@@QAEXH@Z 5f8141b6 f   winctrl2.obj
 0001:0001320c       ?GetNumTics@CSliderCtrl@@QBEIXZ 5f81420c f   winctrl2.obj
 0001:0001325e       ?GetTicArray@CSliderCtrl@@QBEPAKXZ 5f81425e f   winctrl2.obj
 0001:000132b0       ?GetTic@CSliderCtrl@@QBEHH@Z 5f8142b0 f   winctrl2.obj
 0001:00013306       ?GetTicPos@CSliderCtrl@@QBEHH@Z 5f814306 f   winctrl2.obj
 0001:0001335c       ?SetTic@CSliderCtrl@@QAEHH@Z 5f81435c f   winctrl2.obj
 0001:000133b2       ?SetTicFreq@CSliderCtrl@@QAEXH@Z 5f8143b2 f   winctrl2.obj
 0001:00013408       ?GetBuddy@CSliderCtrl@@QBEPAVCWnd@@H@Z 5f814408 f   winctrl2.obj
 0001:00013464       ?SetBuddy@CSliderCtrl@@QAEPAVCWnd@@PAV2@H@Z 5f814464 f   winctrl2.obj
 0001:000134c7       ?GetToolTips@CSliderCtrl@@QBEPAVCToolTipCtrl@@XZ 5f8144c7 f   winctrl2.obj
 0001:0001351f       ?SetToolTips@CSliderCtrl@@QAEXPAVCToolTipCtrl@@@Z 5f81451f f   winctrl2.obj
 0001:0001357a       ?SetTipSide@CSliderCtrl@@QAEHH@Z 5f81457a f   winctrl2.obj
 0001:000135d0       ??0CProgressCtrl@@QAE@XZ   5f8145d0 f   winctrl2.obj
 0001:000135ef       ?SetRange@CProgressCtrl@@QAEXFF@Z 5f8145ef f   winctrl2.obj
 0001:00013658       ?SetRange32@CProgressCtrl@@QAEXHH@Z 5f814658 f   winctrl2.obj
 0001:000136b0       ?GetPos@CProgressCtrl@@QAEHXZ 5f8146b0 f   winctrl2.obj
 0001:00013702       ?OffsetPos@CProgressCtrl@@QAEHH@Z 5f814702 f   winctrl2.obj
 0001:00013758       ?SetStep@CProgressCtrl@@QAEHH@Z 5f814758 f   winctrl2.obj
 0001:000137ae       ?StepIt@CProgressCtrl@@QAEHXZ 5f8147ae f   winctrl2.obj
 0001:00013800       ??0CHeaderCtrl@@QAE@XZ     5f814800 f   winctrl2.obj
 0001:0001381f       ?GetItemCount@CHeaderCtrl@@QBEHXZ 5f81481f f   winctrl2.obj
 0001:00013871       ?InsertItem@CHeaderCtrl@@QAEHHPAU_HD_ITEMW@@@Z 5f814871 f   winctrl2.obj
 0001:000138c9       ?DeleteItem@CHeaderCtrl@@QAEHH@Z 5f8148c9 f   winctrl2.obj
 0001:0001391f       ?GetItem@CHeaderCtrl@@QBEHHPAU_HD_ITEMW@@@Z 5f81491f f   winctrl2.obj
 0001:00013977       ?SetItem@CHeaderCtrl@@QAEHHPAU_HD_ITEMW@@@Z 5f814977 f   winctrl2.obj
 0001:000139cf       ?Layout@CHeaderCtrl@@QAEHPAU_HD_LAYOUT@@@Z 5f8149cf f   winctrl2.obj
 0001:00013a25       ??BCImageList@@QBEPAU_IMAGELIST@@XZ 5f814a25 f   winctrl2.obj
 0001:00013a36       ?GetSafeHandle@CImageList@@QBEPAU_IMAGELIST@@XZ 5f814a36 f   winctrl2.obj
 0001:00013a5e       ?GetImageCount@CImageList@@QBEHXZ 5f814a5e f   winctrl2.obj
 0001:00013a9f       ?Add@CImageList@@QAEHPAVCBitmap@@0@Z 5f814a9f f   winctrl2.obj
 0001:00013af4       ?Add@CImageList@@QAEHPAVCBitmap@@K@Z 5f814af4 f   winctrl2.obj
 0001:00013b44       ?Remove@CImageList@@QAEHH@Z 5f814b44 f   winctrl2.obj
 0001:00013b8b       ?Replace@CImageList@@QAEHHPAVCBitmap@@0@Z 5f814b8b f   winctrl2.obj
 0001:00013be4       ?Add@CImageList@@QAEHPAUHICON__@@@Z 5f814be4 f   winctrl2.obj
 0001:00013c2d       ?Replace@CImageList@@QAEHHPAUHICON__@@@Z 5f814c2d f   winctrl2.obj
 0001:00013c78       ?ExtractIconW@CImageList@@QAEPAUHICON__@@H@Z 5f814c78 f   winctrl2.obj
 0001:00013cc1       ?Draw@CImageList@@QAEHPAVCDC@@HUtagPOINT@@I@Z 5f814cc1 f   winctrl2.obj
 0001:00013d3d       ?SetBkColor@CImageList@@QAEKK@Z 5f814d3d f   winctrl2.obj
 0001:00013d84       ?GetBkColor@CImageList@@QBEKXZ 5f814d84 f   winctrl2.obj
 0001:00013dc5       ?SetOverlayImage@CImageList@@QAEHHH@Z 5f814dc5 f   winctrl2.obj
 0001:00013e10       ?GetImageInfo@CImageList@@QBEHHPAU_IMAGEINFO@@@Z 5f814e10 f   winctrl2.obj
 0001:00013e5b       ?BeginDrag@CImageList@@QAEHHVCPoint@@@Z 5f814e5b f   winctrl2.obj
 0001:00013eaa       ?EndDrag@CImageList@@SGXXZ 5f814eaa f   winctrl2.obj
 0001:00013eb5       ?DragMove@CImageList@@SGHVCPoint@@@Z 5f814eb5 f   winctrl2.obj
 0001:00013eca       ?SetDragCursorImage@CImageList@@QAEHHVCPoint@@@Z 5f814eca f   winctrl2.obj
 0001:00013f19       ?DragShowNolock@CImageList@@SGHH@Z 5f814f19 f   winctrl2.obj
 0001:00013f2a       ?GetDragImage@CImageList@@SGPAV1@PAUtagPOINT@@0@Z 5f814f2a f   winctrl2.obj
 0001:00013f45       ?DragEnter@CImageList@@SGHPAVCWnd@@VCPoint@@@Z 5f814f45 f   winctrl2.obj
 0001:00013f63       ?DragLeave@CImageList@@SGHPAVCWnd@@@Z 5f814f63 f   winctrl2.obj
 0001:00013f79       ??0CTabCtrl@@QAE@XZ        5f814f79 f   winctrl2.obj
 0001:00013f98       ?GetImageList@CTabCtrl@@QBEPAVCImageList@@XZ 5f814f98 f   winctrl2.obj
 0001:00013ff0       ?SetImageList@CTabCtrl@@QAEPAVCImageList@@PAV2@@Z 5f814ff0 f   winctrl2.obj
 0001:00014051       ?GetItemCount@CTabCtrl@@QBEHXZ 5f815051 f   winctrl2.obj
 0001:000140a3       ?GetItem@CTabCtrl@@QBEHHPAUtagTCITEMW@@@Z 5f8150a3 f   winctrl2.obj
 0001:000140fb       ?SetItem@CTabCtrl@@QAEHHPAUtagTCITEMW@@@Z 5f8150fb f   winctrl2.obj
 0001:00014153       ?SetItemExtra@CTabCtrl@@QAEHH@Z 5f815153 f   winctrl2.obj
 0001:000141a9       ?SetCurFocus@CTabCtrl@@QAEXH@Z 5f8151a9 f   winctrl2.obj
 0001:000141ff       ?InsertItem@CTabCtrl@@QAEHHPAUtagTCITEMW@@@Z 5f8151ff f   winctrl2.obj
 0001:00014257       ?InsertItem@CTabCtrl@@QAEHHPBG@Z 5f815257 f   winctrl2.obj
 0001:000142ab       ?InsertItem@CTabCtrl@@QAEHHPBGH@Z 5f8152ab f   winctrl2.obj
 0001:00014301       ?DeleteItem@CTabCtrl@@QAEHH@Z 5f815301 f   winctrl2.obj
 0001:00014357       ?DeleteAllItems@CTabCtrl@@QAEHXZ 5f815357 f   winctrl2.obj
 0001:000143a9       ?GetItemRect@CTabCtrl@@QBEHHPAUtagRECT@@@Z 5f8153a9 f   winctrl2.obj
 0001:00014401       ?GetCurSel@CTabCtrl@@QBEHXZ 5f815401 f   winctrl2.obj
 0001:00014453       ?SetCurSel@CTabCtrl@@QAEHH@Z 5f815453 f   winctrl2.obj
 0001:000144a9       ?HitTest@CTabCtrl@@QBEHPAUtagTCHITTESTINFO@@@Z 5f8154a9 f   winctrl2.obj
 0001:000144ff       ?AdjustRect@CTabCtrl@@QAEXHPAUtagRECT@@@Z 5f8154ff f   winctrl2.obj
 0001:00014557       ?SetItemSize@CTabCtrl@@QAE?AVCSize@@V2@@Z 5f815557 f   winctrl2.obj
 0001:000145db       ?RemoveImage@CTabCtrl@@QAEXH@Z 5f8155db f   winctrl2.obj
 0001:00014631       ?SetPadding@CTabCtrl@@QAEXVCSize@@@Z 5f815631 f   winctrl2.obj
 0001:0001469a       ?GetRowCount@CTabCtrl@@QBEHXZ 5f81569a f   winctrl2.obj
 0001:000146ec       ?GetToolTips@CTabCtrl@@QBEPAVCToolTipCtrl@@XZ 5f8156ec f   winctrl2.obj
 0001:00014744       ?SetToolTips@CTabCtrl@@QAEXPAVCToolTipCtrl@@@Z 5f815744 f   winctrl2.obj
 0001:0001479f       ?GetCurFocus@CTabCtrl@@QBEHXZ 5f81579f f   winctrl2.obj
 0001:000147f1       ?SetMinTabWidth@CTabCtrl@@QAEHH@Z 5f8157f1 f   winctrl2.obj
 0001:00014847       ?DeselectAll@CTabCtrl@@QAEXH@Z 5f815847 f   winctrl2.obj
 0001:0001489d       ?HighlightItem@CTabCtrl@@QAEHHH@Z 5f81589d f   winctrl2.obj
 0001:000148fa       ?GetExtendedStyle@CTabCtrl@@QAEKXZ 5f8158fa f   winctrl2.obj
 0001:0001494c       ?SetExtendedStyle@CTabCtrl@@QAEKKK@Z 5f81594c f   winctrl2.obj
 0001:000149a4       ??0CAnimateCtrl@@QAE@XZ    5f8159a4 f   winctrl2.obj
 0001:000149c3       ?Open@CAnimateCtrl@@QAEHPBG@Z 5f8159c3 f   winctrl2.obj
 0001:00014a19       ?Open@CAnimateCtrl@@QAEHI@Z 5f815a19 f   winctrl2.obj
 0001:00014a6f       ?Play@CAnimateCtrl@@QAEHIII@Z 5f815a6f f   winctrl2.obj
 0001:00014ada       ?Stop@CAnimateCtrl@@QAEHXZ 5f815ada f   winctrl2.obj
 0001:00014b2c       ?Close@CAnimateCtrl@@QAEHXZ 5f815b2c f   winctrl2.obj
 0001:00014b7e       ?Seek@CAnimateCtrl@@QAEHI@Z 5f815b7e f   winctrl2.obj
 0001:00014be7       ??0CRichEditCtrl@@QAE@XZ   5f815be7 f   winctrl2.obj
 0001:00014c06       ?CanUndo@CRichEditCtrl@@QBEHXZ 5f815c06 f   winctrl2.obj
 0001:00014c58       ?GetLineCount@CRichEditCtrl@@QBEHXZ 5f815c58 f   winctrl2.obj
 0001:00014caa       ?GetModify@CRichEditCtrl@@QBEHXZ 5f815caa f   winctrl2.obj
 0001:00014cfc       ?SetModify@CRichEditCtrl@@QAEXH@Z 5f815cfc f   winctrl2.obj
 0001:00014d52       ?GetRect@CRichEditCtrl@@QBEXPAUtagRECT@@@Z 5f815d52 f   winctrl2.obj
 0001:00014da8       ?GetCharPos@CRichEditCtrl@@QBE?AVCPoint@@J@Z 5f815da8 f   winctrl2.obj
 0001:00014e1b       ?SetOptions@CRichEditCtrl@@QAEXGK@Z 5f815e1b f   winctrl2.obj
 0001:00014e79       ?EmptyUndoBuffer@CRichEditCtrl@@QAEXXZ 5f815e79 f   winctrl2.obj
 0001:00014ecb       ?ReplaceSel@CRichEditCtrl@@QAEXPBGH@Z 5f815ecb f   winctrl2.obj
 0001:00014f23       ?SetRect@CRichEditCtrl@@QAEXPBUtagRECT@@@Z 5f815f23 f   winctrl2.obj
 0001:00014f79       ?Undo@CRichEditCtrl@@QAEHXZ 5f815f79 f   winctrl2.obj
 0001:00014fcb       ?Clear@CRichEditCtrl@@QAEXXZ 5f815fcb f   winctrl2.obj
 0001:0001501d       ?Copy@CRichEditCtrl@@QAEXXZ 5f81601d f   winctrl2.obj
 0001:0001506f       ?Cut@CRichEditCtrl@@QAEXXZ 5f81606f f   winctrl2.obj
 0001:000150c1       ?Paste@CRichEditCtrl@@QAEXXZ 5f8160c1 f   winctrl2.obj
 0001:00015113       ?SetReadOnly@CRichEditCtrl@@QAEHH@Z 5f816113 f   winctrl2.obj
 0001:00015169       ?GetFirstVisibleLine@CRichEditCtrl@@QBEHXZ 5f816169 f   winctrl2.obj
 0001:000151bb       ?DisplayBand@CRichEditCtrl@@QAEHPAUtagRECT@@@Z 5f8161bb f   winctrl2.obj
 0001:00015211       ?GetSel@CRichEditCtrl@@QBEXAAU_charrange@@@Z 5f816211 f   winctrl2.obj
 0001:00015267       ?LimitText@CRichEditCtrl@@QAEXJ@Z 5f816267 f   winctrl2.obj
 0001:000152bd       ?LineFromChar@CRichEditCtrl@@QBEJJ@Z 5f8162bd f   winctrl2.obj
 0001:00015313       ?SetSel@CRichEditCtrl@@QAEXAAU_charrange@@@Z 5f816313 f   winctrl2.obj
 0001:00015369       ?FindTextW@CRichEditCtrl@@QBEJKPAU_findtextexa@@@Z 5f816369 f   winctrl2.obj
 0001:000153c1       ?FormatRange@CRichEditCtrl@@QAEJPAU_formatrange@@H@Z 5f8163c1 f   winctrl2.obj
 0001:00015419       ?GetEventMask@CRichEditCtrl@@QBEJXZ 5f816419 f   winctrl2.obj
 0001:0001546b       ?GetLimitText@CRichEditCtrl@@QBEJXZ 5f81646b f   winctrl2.obj
 0001:000154bd       ?GetSelText@CRichEditCtrl@@QBEJPAD@Z 5f8164bd f   winctrl2.obj
 0001:00015513       ?HideSelection@CRichEditCtrl@@QAEXHH@Z 5f816513 f   winctrl2.obj
 0001:0001556b       ?RequestResize@CRichEditCtrl@@QAEXXZ 5f81656b f   winctrl2.obj
 0001:000155bd       ?GetSelectionType@CRichEditCtrl@@QBEGXZ 5f8165bd f   winctrl2.obj
 0001:0001560f       ?SetBackgroundColor@CRichEditCtrl@@QAEKHK@Z 5f81660f f   winctrl2.obj
 0001:00015667       ?SetEventMask@CRichEditCtrl@@QAEKK@Z 5f816667 f   winctrl2.obj
 0001:000156bd       ?SetOLECallback@CRichEditCtrl@@QAEHPAUIRichEditOleCallback@@@Z 5f8166bd f   winctrl2.obj
 0001:00015713       ?SetTargetDevice@CRichEditCtrl@@QAEHPAUHDC__@@J@Z 5f816713 f   winctrl2.obj
 0001:0001576b       ?SetTargetDevice@CRichEditCtrl@@QAEHAAVCDC@@J@Z 5f81676b f   winctrl2.obj
 0001:000157c6       ?StreamIn@CRichEditCtrl@@QAEJHAAU_editstream@@@Z 5f8167c6 f   winctrl2.obj
 0001:0001581e       ?StreamOut@CRichEditCtrl@@QAEJHAAU_editstream@@@Z 5f81681e f   winctrl2.obj
 0001:00015876       ?GetTextLength@CRichEditCtrl@@QBEJXZ 5f816876 f   winctrl2.obj
 0001:000158d0       ??1_AFX_RICHEDIT_STATE@@UAE@XZ 5f8168d0 f   winctrl4.obj
 0001:00015902       ?AfxGetRichEditState@@YAPAV_AFX_RICHEDIT_STATE@@XZ 5f816902 f   winctrl4.obj
 0001:00015911       ?AfxInitRichEdit@@YGHXZ    5f816911 f   winctrl4.obj
 0001:0001594c       ?Create@CRichEditCtrl@@QAEHKABUtagRECT@@PAVCWnd@@I@Z 5f81694c f   winctrl4.obj
 0001:00015992       ?GetLine@CRichEditCtrl@@QBEHHPAG@Z 5f816992 f   winctrl4.obj
 0001:000159e7       ?LineIndex@CRichEditCtrl@@QBEHH@Z 5f8169e7 f   winctrl4.obj
 0001:00015a3a       ?LineLength@CRichEditCtrl@@QBEHH@Z 5f816a3a f   winctrl4.obj
 0001:00015a8d       ?LineScroll@CRichEditCtrl@@QAEXHH@Z 5f816a8d f   winctrl4.obj
 0001:00015ae2       ?SetSel@CRichEditCtrl@@QAEXJJ@Z 5f816ae2 f   winctrl4.obj
 0001:00015b43       ?CanPaste@CRichEditCtrl@@QBEHI@Z 5f816b43 f   winctrl4.obj
 0001:00015bc8       ?PasteSpecial@CRichEditCtrl@@QAEXIKPAUHMETAFILE__@@@Z 5f816bc8 f   winctrl4.obj
 0001:00015c2b       ?GetLine@CRichEditCtrl@@QBEHHPAGH@Z 5f816c2b f   winctrl4.obj
 0001:00015c88       ?GetSel@CRichEditCtrl@@QBEXAAJ0@Z 5f816c88 f   winctrl4.obj
 0001:00015ced       ?GetSelText@CRichEditCtrl@@QBE?AVCString@@XZ 5f816ced f   winctrl4.obj
 0001:00015daf       ?GetIRichEditOle@CRichEditCtrl@@QBEPAUIRichEditOle@@XZ 5f816daf f   winctrl4.obj
 0001:00015e0f       ?SetDefaultCharFormat@CRichEditCtrl@@QAEHAAU_charformat@@@Z 5f816e0f f   winctrl4.obj
 0001:00015e6e       ?SetSelectionCharFormat@CRichEditCtrl@@QAEHAAU_charformat@@@Z 5f816e6e f   winctrl4.obj
 0001:00015ecd       ?SetWordCharFormat@CRichEditCtrl@@QAEHAAU_charformat@@@Z 5f816ecd f   winctrl4.obj
 0001:00015f2c       ?GetDefaultCharFormat@CRichEditCtrl@@QBEKAAU_charformat@@@Z 5f816f2c f   winctrl4.obj
 0001:00015f8b       ?GetSelectionCharFormat@CRichEditCtrl@@QBEKAAU_charformat@@@Z 5f816f8b f   winctrl4.obj
 0001:00015fea       ?GetParaFormat@CRichEditCtrl@@QBEKAAU_paraformat@@@Z 5f816fea f   winctrl4.obj
 0001:00016049       ?SetParaFormat@CRichEditCtrl@@QAEHAAU_paraformat@@@Z 5f817049 f   winctrl4.obj
 0001:000160e0       ??_G_AFX_RICHEDIT_STATE@@UAEPAXI@Z 5f8170e0 f i winctrl4.obj
 0001:000160e0       ??_E_AFX_RICHEDIT_STATE@@UAEPAXI@Z 5f8170e0 f i winctrl4.obj
 0001:00016110       ??1?$CProcessLocal@V_AFX_RICHEDIT_STATE@@@@QAE@XZ 5f817110 f i winctrl4.obj
 0001:00016130       ?GetData@?$CProcessLocal@V_AFX_RICHEDIT_STATE@@@@QAEPAV_AFX_RICHEDIT_STATE@@XZ 5f817130 f i winctrl4.obj
 0001:00016180       ??B?$CProcessLocal@V_AFX_RICHEDIT_STATE@@@@QAEPAV_AFX_RICHEDIT_STATE@@XZ 5f817180 f i winctrl4.obj
 0001:000161a0       ?CreateObject@?$CProcessLocal@V_AFX_RICHEDIT_STATE@@@@SGPAVCNoTrackObject@@XZ 5f8171a0 f i winctrl4.obj
 0001:00016210       ??0_AFX_RICHEDIT_STATE@@QAE@XZ 5f817210 f i winctrl4.obj
 0001:00016230       ?Create@CComboBoxEx@@QAEHKABUtagRECT@@PAVCWnd@@I@Z 5f817230 f   winctrl6.obj
 0001:00016294       ?DeleteItem@CComboBoxEx@@QAEHH@Z 5f817294 f   winctrl6.obj
 0001:000162e7       ?GetItem@CComboBoxEx@@QAEHPAUtagCOMBOBOXEXITEMW@@@Z 5f8172e7 f   winctrl6.obj
 0001:0001637f       ?InsertItem@CComboBoxEx@@QAEHPBUtagCOMBOBOXEXITEMW@@@Z 5f81737f f   winctrl6.obj
 0001:00016417       ?SetItem@CComboBoxEx@@QAEHPBUtagCOMBOBOXEXITEMW@@@Z 5f817417 f   winctrl6.obj
 0001:000164af       ??1CComboBoxEx@@UAE@XZ     5f8174af f   winctrl6.obj
 0001:00016500       ?Create@CReBarCtrl@@QAEHKABUtagRECT@@PAVCWnd@@I@Z 5f817500 f   winctrl6.obj
 0001:00016564       ?GetImageList@CReBarCtrl@@QBEPAVCImageList@@XZ 5f817564 f   winctrl6.obj
 0001:000165a7       ?SetImageList@CReBarCtrl@@QAEHPAVCImageList@@@Z 5f8175a7 f   winctrl6.obj
 0001:000165db       ?GetColorScheme@CReBarCtrl@@QAEHPAUtagCOLORSCHEME@@@Z 5f8175db f   winctrl6.obj
 0001:00016604       ?SetColorScheme@CReBarCtrl@@QAEXPBUtagCOLORSCHEME@@@Z 5f817604 f   winctrl6.obj
 0001:0001662d       ?SetColumnOrderArray@CListCtrl@@QAEHHPAH@Z 5f81762d f   winctrl6.obj
 0001:000166b5       ?GetColumnOrderArray@CListCtrl@@QAEHPAHH@Z 5f8176b5 f   winctrl6.obj
 0001:00016791       ?SetBkImage@CListCtrl@@QAEHPAUHBITMAP__@@HHH@Z 5f817791 f   winctrl6.obj
 0001:000167db       ?SetBkImage@CListCtrl@@QAEHPAGHHH@Z 5f8177db f   winctrl6.obj
 0001:00016825       ?GetCheck@CListCtrl@@QBEHH@Z 5f817825 f   winctrl6.obj
 0001:0001688c       ?SetCheck@CListCtrl@@QAEHHH@Z 5f81788c f   winctrl6.obj
 0001:000168fd       ?GetHeaderCtrl@CListCtrl@@QAEPAVCHeaderCtrl@@XZ 5f8178fd f   winctrl6.obj
 0001:00016967       ?SetOrderArray@CHeaderCtrl@@QAEHHPAH@Z 5f817967 f   winctrl6.obj
 0001:000169ef       ?GetOrderArray@CHeaderCtrl@@QAEHPAHH@Z 5f8179ef f   winctrl6.obj
 0001:00016a9a       ?GetRange@CProgressCtrl@@QAEXAAH0@Z 5f817a9a f   winctrl6.obj
 0001:00016b02       ?IsSimple@CStatusBarCtrl@@QBEHXZ 5f817b02 f   winctrl6.obj
 0001:00016b51       ?SetTipText@CStatusBarCtrl@@QAEXHPBG@Z 5f817b51 f   winctrl6.obj
 0001:00016ba6       ?SetBkColor@CStatusBarCtrl@@QAEKK@Z 5f817ba6 f   winctrl6.obj
 0001:00016bf9       ?SetIcon@CStatusBarCtrl@@QAEHHPAUHICON__@@@Z 5f817bf9 f   winctrl6.obj
 0001:00016c4e       ?SetRange32@CSpinButtonCtrl@@QAEXHH@Z 5f817c4e f   winctrl6.obj
 0001:00016ca3       ?GetRange32@CSpinButtonCtrl@@QBEXAAH0@Z 5f817ca3 f   winctrl6.obj
 0001:00016cf8       ?GetButtonSize@CToolBarCtrl@@QBEKXZ 5f817cf8 f   winctrl6.obj
 0001:00016d47       ?GetDisabledImageList@CToolBarCtrl@@QBEPAVCImageList@@XZ 5f817d47 f   winctrl6.obj
 0001:00016d9c       ?GetHotImageList@CToolBarCtrl@@QBEPAVCImageList@@XZ 5f817d9c f   winctrl6.obj
 0001:00016df1       ?GetImageList@CToolBarCtrl@@QBEPAVCImageList@@XZ 5f817df1 f   winctrl6.obj
 0001:00016e46       ?GetStyle@CToolBarCtrl@@QBEKXZ 5f817e46 f   winctrl6.obj
 0001:00016e95       ?GetMaxTextRows@CToolBarCtrl@@QBEHXZ 5f817e95 f   winctrl6.obj
 0001:00016ee4       ?GetRect@CToolBarCtrl@@QBEHHPAUtagRECT@@@Z 5f817ee4 f   winctrl6.obj
 0001:00016f39       ?IsButtonHighlighted@CToolBarCtrl@@QBEHH@Z 5f817f39 f   winctrl6.obj
 0001:00016f8c       ?LoadImages@CToolBarCtrl@@QAEXHPAUHINSTANCE__@@@Z 5f817f8c f   winctrl6.obj
 0001:00016fe1       ?SetButtonWidth@CToolBarCtrl@@QAEHHH@Z 5f817fe1 f   winctrl6.obj
 0001:00017047       ?SetDisabledImageList@CToolBarCtrl@@QAEPAVCImageList@@PAV2@@Z 5f818047 f   winctrl6.obj
 0001:000170a5       ?SetHotImageList@CToolBarCtrl@@QAEPAVCImageList@@PAV2@@Z 5f8180a5 f   winctrl6.obj
 0001:00017103       ?SetImageList@CToolBarCtrl@@QAEPAVCImageList@@PAV2@@Z 5f818103 f   winctrl6.obj
 0001:00017161       ?SetIndent@CToolBarCtrl@@QAEHH@Z 5f818161 f   winctrl6.obj
 0001:000171b4       ?SetMaxTextRows@CToolBarCtrl@@QAEHH@Z 5f8181b4 f   winctrl6.obj
 0001:00017207       ?SetStyle@CToolBarCtrl@@QAEXK@Z 5f818207 f   winctrl6.obj
 0001:0001725a       ?GetButtonInfo@CToolBarCtrl@@QBEHHPAUTBBUTTONINFOW@@@Z 5f81825a f   winctrl6.obj
 0001:000172af       ?SetButtonInfo@CToolBarCtrl@@QAEHHPAUTBBUTTONINFOW@@@Z 5f8182af f   winctrl6.obj
 0001:00017304       ?SetDrawTextFlags@CToolBarCtrl@@QAEKKK@Z 5f818304 f   winctrl6.obj
 0001:00017359       ?GetAnchorHighlight@CToolBarCtrl@@QBEHXZ 5f818359 f   winctrl6.obj
 0001:000173a8       ?SetAnchorHighlight@CToolBarCtrl@@QAEHH@Z 5f8183a8 f   winctrl6.obj
 0001:000173fb       ?GetHotItem@CToolBarCtrl@@QBEHXZ 5f8183fb f   winctrl6.obj
 0001:0001744a       ?SetHotItem@CToolBarCtrl@@QAEHH@Z 5f81844a f   winctrl6.obj
 0001:0001749d       ?GetInsertMark@CToolBarCtrl@@QBEXPAUTBINSERTMARK@@@Z 5f81849d f   winctrl6.obj
 0001:000174f0       ?SetInsertMark@CToolBarCtrl@@QAEXPAUTBINSERTMARK@@@Z 5f8184f0 f   winctrl6.obj
 0001:00017543       ?GetMaxSize@CToolBarCtrl@@QBEHPAUtagSIZE@@@Z 5f818543 f   winctrl6.obj
 0001:00017596       ?InsertMarkHitTest@CToolBarCtrl@@QBEHPAUtagPOINT@@PAUTBINSERTMARK@@@Z 5f818596 f   winctrl6.obj
 0001:000175eb       ?MapAccelerator@CToolBarCtrl@@QAEHGPAI@Z 5f8185eb f   winctrl6.obj
 0001:00017646       ?MarkButton@CToolBarCtrl@@QAEHHH@Z 5f818646 f   winctrl6.obj
 0001:000176a0       ?MoveButton@CToolBarCtrl@@QAEHII@Z 5f8186a0 f   winctrl6.obj
 0001:000176f5       ?SetExtendedStyle@CListCtrl@@QAEKK@Z 5f8186f5 f   winctrl6.obj
 0001:00017748       ?SetHotCursor@CListCtrl@@QAEPAUHICON__@@PAU2@@Z 5f818748 f   winctrl6.obj
 0001:000177a1       ?SetHotItem@CListCtrl@@QAEHH@Z 5f8187a1 f   winctrl6.obj
 0001:000177f4       ?SetWorkAreas@CListCtrl@@QAEXHPAUtagRECT@@@Z 5f8187f4 f   winctrl6.obj
 0001:00017849       ?SubItemHitTest@CListCtrl@@QAEHPAUtagLVHITTESTINFO@@@Z 5f818849 f   winctrl6.obj
 0001:0001789c       ?GetHotCursor@CListCtrl@@QAEPAUHICON__@@XZ 5f81889c f   winctrl6.obj
 0001:000178eb       ?GetHotItem@CListCtrl@@QAEHXZ 5f8188eb f   winctrl6.obj
 0001:0001793a       ?GetExtendedStyle@CListCtrl@@QAEKXZ 5f81893a f   winctrl6.obj
 0001:00017989       ?ApproximateViewRect@CListCtrl@@QBE?AVCSize@@V2@H@Z 5f818989 f   winctrl6.obj
 0001:00017a0c       ?GetBkImage@CListCtrl@@QBEHPAUtagLVBKIMAGEW@@@Z 5f818a0c f   winctrl6.obj
 0001:00017a5f       ?GetHoverTime@CListCtrl@@QBEKXZ 5f818a5f f   winctrl6.obj
 0001:00017aae       ?GetWorkAreas@CListCtrl@@QBEXHPAUtagRECT@@@Z 5f818aae f   winctrl6.obj
 0001:00017b03       ?SetBkImage@CListCtrl@@QAEHPAUtagLVBKIMAGEW@@@Z 5f818b03 f   winctrl6.obj
 0001:00017b56       ?SetHoverTime@CListCtrl@@QAEKK@Z 5f818b56 f   winctrl6.obj
 0001:00017ba9       ?GetNumberOfWorkAreas@CListCtrl@@QBEIXZ 5f818ba9 f   winctrl6.obj
 0001:00017bff       ?SetSelectionMark@CListCtrl@@QAEHH@Z 5f818bff f   winctrl6.obj
 0001:00017c55       ?GetSelectionMark@CListCtrl@@QAEHXZ 5f818c55 f   winctrl6.obj
 0001:00017ca7       ?GetItemRect@CHeaderCtrl@@QBEHHPAUtagRECT@@@Z 5f818ca7 f   winctrl6.obj
 0001:00017d1f       ?OrderToIndex@CHeaderCtrl@@QBEHH@Z 5f818d1f f   winctrl6.obj
 0001:00017d75       ?SetHotDivider@CHeaderCtrl@@QAEHVCPoint@@@Z 5f818d75 f   winctrl6.obj
 0001:00017dde       ?SetHotDivider@CHeaderCtrl@@QAEHH@Z 5f818dde f   winctrl6.obj
 0001:00017e34       ?GetImageList@CHeaderCtrl@@QBEPAVCImageList@@XZ 5f818e34 f   winctrl6.obj
 0001:00017e8c       ?SetImageList@CHeaderCtrl@@QAEPAVCImageList@@PAV2@@Z 5f818e8c f   winctrl6.obj
 0001:00017eed       ?CreateDragImage@CHeaderCtrl@@QAEPAVCImageList@@H@Z 5f818eed f   winctrl6.obj
 0001:00017f49       ??0CReBarCtrl@@QAE@XZ      5f818f49 f   winctrl6.obj
 0001:00017f68       ?GetBandCount@CReBarCtrl@@QBEIXZ 5f818f68 f   winctrl6.obj
 0001:00017fba       ?GetBandInfo@CReBarCtrl@@QBEHIPAUtagREBARBANDINFOW@@@Z 5f818fba f   winctrl6.obj
 0001:00018012       ?GetBarHeight@CReBarCtrl@@QBEIXZ 5f819012 f   winctrl6.obj
 0001:00018064       ?GetBarInfo@CReBarCtrl@@QBEHPAUtagREBARINFO@@@Z 5f819064 f   winctrl6.obj
 0001:000180ba       ?GetBkColor@CReBarCtrl@@QBEKXZ 5f8190ba f   winctrl6.obj
 0001:0001810c       ?GetDropTarget@CReBarCtrl@@QBEPAUIDropTarget@@XZ 5f81910c f   winctrl6.obj
 0001:00018165       ?GetRect@CReBarCtrl@@QBEHIPAUtagRECT@@@Z 5f819165 f   winctrl6.obj
 0001:000181bd       ?GetRowCount@CReBarCtrl@@QBEIXZ 5f8191bd f   winctrl6.obj
 0001:0001820f       ?GetRowHeight@CReBarCtrl@@QBEII@Z 5f81920f f   winctrl6.obj
 0001:00018265       ?GetTextColor@CReBarCtrl@@QBEKXZ 5f819265 f   winctrl6.obj
 0001:000182b7       ?GetToolTips@CReBarCtrl@@QBEPAVCToolTipCtrl@@XZ 5f8192b7 f   winctrl6.obj
 0001:0001830f       ?IDToIndex@CReBarCtrl@@QBEHI@Z 5f81930f f   winctrl6.obj
 0001:00018365       ?SetBandInfo@CReBarCtrl@@QAEHIPAUtagREBARBANDINFOW@@@Z 5f819365 f   winctrl6.obj
 0001:000183bd       ?SetBarInfo@CReBarCtrl@@QAEHPAUtagREBARINFO@@@Z 5f8193bd f   winctrl6.obj
 0001:00018413       ?SetBkColor@CReBarCtrl@@QAEKK@Z 5f819413 f   winctrl6.obj
 0001:00018469       ?SetOwner@CReBarCtrl@@QAEPAVCWnd@@PAV2@@Z 5f819469 f   winctrl6.obj
 0001:000184c8       ?SetTextColor@CReBarCtrl@@QAEKK@Z 5f8194c8 f   winctrl6.obj
 0001:0001851e       ?SetToolTips@CReBarCtrl@@QAEXPAVCToolTipCtrl@@@Z 5f81951e f   winctrl6.obj
 0001:00018577       ?BeginDrag@CReBarCtrl@@QAEXIK@Z 5f819577 f   winctrl6.obj
 0001:000185cf       ?DeleteBand@CReBarCtrl@@QAEHI@Z 5f8195cf f   winctrl6.obj
 0001:00018625       ?DragMove@CReBarCtrl@@QAEXK@Z 5f819625 f   winctrl6.obj
 0001:0001867b       ?EndDrag@CReBarCtrl@@QAEXXZ 5f81967b f   winctrl6.obj
 0001:000186cd       ?HitTest@CReBarCtrl@@QAEHPAU_RB_HITTESTINFO@@@Z 5f8196cd f   winctrl6.obj
 0001:00018723       ?InsertBand@CReBarCtrl@@QAEHIPAUtagREBARBANDINFOW@@@Z 5f819723 f   winctrl6.obj
 0001:0001877b       ?MaximizeBand@CReBarCtrl@@QAEXI@Z 5f81977b f   winctrl6.obj
 0001:000187d1       ?MinimizeBand@CReBarCtrl@@QAEXI@Z 5f8197d1 f   winctrl6.obj
 0001:00018827       ?SizeToRect@CReBarCtrl@@QAEHAAVCRect@@@Z 5f819827 f   winctrl6.obj
 0001:0001887d       ?ShowBand@CReBarCtrl@@QAEHIH@Z 5f81987d f   winctrl6.obj
 0001:000188d5       ?GetBandBorders@CReBarCtrl@@QBEXIPAUtagRECT@@@Z 5f8198d5 f   winctrl6.obj
 0001:0001892d       ?GetPalette@CReBarCtrl@@QBEPAVCPalette@@XZ 5f81992d f   winctrl6.obj
 0001:00018985       ?SetPalette@CReBarCtrl@@QAEPAVCPalette@@PAUHPALETTE__@@@Z 5f819985 f   winctrl6.obj
 0001:000189e1       ?MoveBand@CReBarCtrl@@QAEHII@Z 5f8199e1 f   winctrl6.obj
 0001:00018a39       ?SetDelayTime@CToolTipCtrl@@QAEXI@Z 5f819a39 f   winctrl6.obj
 0001:00018a8f       ?GetDelayTime@CToolTipCtrl@@QBEHK@Z 5f819a8f f   winctrl6.obj
 0001:00018ae5       ?GetMargin@CToolTipCtrl@@QBEXPAUtagRECT@@@Z 5f819ae5 f   winctrl6.obj
 0001:00018b3b       ?GetMaxTipWidth@CToolTipCtrl@@QBEHXZ 5f819b3b f   winctrl6.obj
 0001:00018b8d       ?GetTipBkColor@CToolTipCtrl@@QBEKXZ 5f819b8d f   winctrl6.obj
 0001:00018bdf       ?GetTipTextColor@CToolTipCtrl@@QBEKXZ 5f819bdf f   winctrl6.obj
 0001:00018c31       ?Pop@CToolTipCtrl@@QAEXXZ  5f819c31 f   winctrl6.obj
 0001:00018c83       ?SetDelayTime@CToolTipCtrl@@QAEXKH@Z 5f819c83 f   winctrl6.obj
 0001:00018ce0       ?SetMargin@CToolTipCtrl@@QAEXPAUtagRECT@@@Z 5f819ce0 f   winctrl6.obj
 0001:00018d36       ?SetMaxTipWidth@CToolTipCtrl@@QAEHH@Z 5f819d36 f   winctrl6.obj
 0001:00018d8c       ?SetTipBkColor@CToolTipCtrl@@QAEXK@Z 5f819d8c f   winctrl6.obj
 0001:00018de2       ?SetTipTextColor@CToolTipCtrl@@QAEXK@Z 5f819de2 f   winctrl6.obj
 0001:00018e38       ?Update@CToolTipCtrl@@QAEXXZ 5f819e38 f   winctrl6.obj
 0001:00018e8a       ??0CComboBoxEx@@QAE@XZ     5f819e8a f   winctrl6.obj
 0001:00018ea9       ?GetExtendedStyle@CComboBoxEx@@QBEKXZ 5f819ea9 f   winctrl6.obj
 0001:00018efb       ?SetExtendedStyle@CComboBoxEx@@QAEKKK@Z 5f819efb f   winctrl6.obj
 0001:00018f53       ?HasEditChanged@CComboBoxEx@@QAEHXZ 5f819f53 f   winctrl6.obj
 0001:00018fa5       ?GetEditCtrl@CComboBoxEx@@QAEPAVCEdit@@XZ 5f819fa5 f   winctrl6.obj
 0001:00018ffd       ?GetComboBoxCtrl@CComboBoxEx@@QAEPAVCComboBox@@XZ 5f819ffd f   winctrl6.obj
 0001:00019055       ?SetImageList@CComboBoxEx@@QAEPAVCImageList@@PAV2@@Z 5f81a055 f   winctrl6.obj
 0001:000190b6       ?GetImageList@CComboBoxEx@@QBEPAVCImageList@@XZ 5f81a0b6 f   winctrl6.obj
 0001:0001910e       ?Dir@CComboBoxEx@@QAEHIPBG@Z 5f81a10e f   winctrl6.obj
 0001:00019147       ?FindString@CComboBoxEx@@QBEHHPBG@Z 5f81a147 f   winctrl6.obj
 0001:00019180       ?AddString@CComboBoxEx@@QAEHPBG@Z 5f81a180 f   winctrl6.obj
 0001:000191b9       ?SetEditSel@CComboBoxEx@@QAEHHH@Z 5f81a1b9 f   winctrl6.obj
 0001:000191f1       ?InsertString@CComboBoxEx@@QAEHHPBG@Z 5f81a1f1 f   winctrl6.obj
 0001:0001922a       ?SetPos@CProgressCtrl@@QAEHH@Z 5f81a22a f   winctrl6.obj
 0001:00019280       ??0CIPAddressCtrl@@QAE@XZ  5f81a280 f   winctrl6.obj
 0001:0001929f       ?ClearAddress@CIPAddressCtrl@@QAEXXZ 5f81a29f f   winctrl6.obj
 0001:000192f1       ?IsBlank@CIPAddressCtrl@@QBEHXZ 5f81a2f1 f   winctrl6.obj
 0001:00019343       ?GetAddress@CIPAddressCtrl@@QAEHAAK@Z 5f81a343 f   winctrl6.obj
 0001:00019399       ?SetAddress@CIPAddressCtrl@@QAEXK@Z 5f81a399 f   winctrl6.obj
 0001:000193ef       ?SetAddress@CIPAddressCtrl@@QAEXEEEE@Z 5f81a3ef f   winctrl6.obj
 0001:00019474       ?SetFieldFocus@CIPAddressCtrl@@QAEXG@Z 5f81a474 f   winctrl6.obj
 0001:000194cf       ?SetFieldRange@CIPAddressCtrl@@QAEXHEE@Z 5f81a4cf f   winctrl6.obj
 0001:0001953f       ?SetImageCount@CImageList@@QAEHI@Z 5f81a53f f   winctrl6.obj
 0001:00019586       ?Copy@CImageList@@QAEHHHI@Z 5f81a586 f   winctrl6.obj
 0001:000195dc       ?Copy@CImageList@@QAEHHPAV1@HI@Z 5f81a5dc f   winctrl6.obj
 0001:00019660       ??_ECComboBoxEx@@UAEPAXI@Z 5f81a660 f i winctrl6.obj
 0001:00019660       ??_GCComboBoxEx@@UAEPAXI@Z 5f81a660 f i winctrl6.obj
 0001:00019690       ??_GCReBarCtrl@@UAEPAXI@Z  5f81a690 f i winctrl6.obj
 0001:00019690       ??_ECReBarCtrl@@UAEPAXI@Z  5f81a690 f i winctrl6.obj
 0001:000196c0       ??1CReBarCtrl@@UAE@XZ      5f81a6c0 f i winctrl6.obj
 0001:000196e0       ?DrawIndirect@CImageList@@QAEHPAU_IMAGELISTDRAWPARAMS@@@Z 5f81a6e0 f   winctrl7.obj
 0001:00019760       ?DrawIndirect@CImageList@@QAEHPAVCDC@@HUtagPOINT@@UtagSIZE@@1IKKK@Z 5f81a760 f   winctrl7.obj
 0001:0001981a       ?Create@CImageList@@QAEHPAV1@@Z 5f81a81a f   winctrl7.obj
 0001:00019860       ??0CByteArray@@QAE@XZ      5f81a860 f   array_b.obj
 0001:000198a7       ??1CByteArray@@UAE@XZ      5f81a8a7 f   array_b.obj
 0001:00019917       ?SetSize@CByteArray@@QAEXHH@Z 5f81a917 f   array_b.obj
 0001:00019bee       ?Append@CByteArray@@QAEHABV1@@Z 5f81abee f   array_b.obj
 0001:00019c7b       ?Copy@CByteArray@@QAEXABV1@@Z 5f81ac7b f   array_b.obj
 0001:00019cf1       ?FreeExtra@CByteArray@@QAEXXZ 5f81acf1 f   array_b.obj
 0001:00019dc2       ?SetAtGrow@CByteArray@@QAEXHE@Z 5f81adc2 f   array_b.obj
 0001:00019e33       ?InsertAt@CByteArray@@QAEXHEH@Z 5f81ae33 f   array_b.obj
 0001:00019f69       ?RemoveAt@CByteArray@@QAEXHH@Z 5f81af69 f   array_b.obj
 0001:0001a045       ?InsertAt@CByteArray@@QAEXHPAV1@@Z 5f81b045 f   array_b.obj
 0001:0001a154       ?Serialize@CByteArray@@UAEXAAVCArchive@@@Z 5f81b154 f   array_b.obj
 0001:0001a1e4       ?Dump@CByteArray@@UBEXAAVCDumpContext@@@Z 5f81b1e4 f   array_b.obj
 0001:0001a296       ?AssertValid@CByteArray@@UBEXXZ 5f81b296 f   array_b.obj
 0001:0001a3b0       ??0CDWordArray@@QAE@XZ     5f81b3b0 f   array_d.obj
 0001:0001a3f7       ??1CDWordArray@@UAE@XZ     5f81b3f7 f   array_d.obj
 0001:0001a467       ?SetSize@CDWordArray@@QAEXHH@Z 5f81b467 f   array_d.obj
 0001:0001a75c       ?Append@CDWordArray@@QAEHABV1@@Z 5f81b75c f   array_d.obj
 0001:0001a7ef       ?Copy@CDWordArray@@QAEXABV1@@Z 5f81b7ef f   array_d.obj
 0001:0001a868       ?FreeExtra@CDWordArray@@QAEXXZ 5f81b868 f   array_d.obj
 0001:0001a942       ?SetAtGrow@CDWordArray@@QAEXHK@Z 5f81b942 f   array_d.obj
 0001:0001a9b3       ?InsertAt@CDWordArray@@QAEXHKH@Z 5f81b9b3 f   array_d.obj
 0001:0001aaf6       ?RemoveAt@CDWordArray@@QAEXHH@Z 5f81baf6 f   array_d.obj
 0001:0001abd9       ?InsertAt@CDWordArray@@QAEXHPAV1@@Z 5f81bbd9 f   array_d.obj
 0001:0001ace8       ?Serialize@CDWordArray@@UAEXAAVCArchive@@@Z 5f81bce8 f   array_d.obj
 0001:0001ad7e       ?Dump@CDWordArray@@UBEXAAVCDumpContext@@@Z 5f81bd7e f   array_d.obj
 0001:0001ae30       ?AssertValid@CDWordArray@@UBEXXZ 5f81be30 f   array_d.obj
 0001:0001af50       ??0CPtrArray@@QAE@XZ       5f81bf50 f   array_p.obj
 0001:0001af97       ??1CPtrArray@@UAE@XZ       5f81bf97 f   array_p.obj
 0001:0001b007       ?SetSize@CPtrArray@@QAEXHH@Z 5f81c007 f   array_p.obj
 0001:0001b2fc       ?Append@CPtrArray@@QAEHABV1@@Z 5f81c2fc f   array_p.obj
 0001:0001b38f       ?Copy@CPtrArray@@QAEXABV1@@Z 5f81c38f f   array_p.obj
 0001:0001b408       ?FreeExtra@CPtrArray@@QAEXXZ 5f81c408 f   array_p.obj
 0001:0001b4e2       ?SetAtGrow@CPtrArray@@QAEXHPAX@Z 5f81c4e2 f   array_p.obj
 0001:0001b553       ?InsertAt@CPtrArray@@QAEXHPAXH@Z 5f81c553 f   array_p.obj
 0001:0001b696       ?RemoveAt@CPtrArray@@QAEXHH@Z 5f81c696 f   array_p.obj
 0001:0001b779       ?InsertAt@CPtrArray@@QAEXHPAV1@@Z 5f81c779 f   array_p.obj
 0001:0001b888       ?Dump@CPtrArray@@UBEXAAVCDumpContext@@@Z 5f81c888 f   array_p.obj
 0001:0001b93a       ?AssertValid@CPtrArray@@UBEXXZ 5f81c93a f   array_p.obj
 0001:0001ba50       ??0CObArray@@QAE@XZ        5f81ca50 f   array_o.obj
 0001:0001ba97       ??1CObArray@@UAE@XZ        5f81ca97 f   array_o.obj
 0001:0001bb07       ?SetSize@CObArray@@QAEXHH@Z 5f81cb07 f   array_o.obj
 0001:0001bdfc       ?Append@CObArray@@QAEHABV1@@Z 5f81cdfc f   array_o.obj
 0001:0001be8f       ?Copy@CObArray@@QAEXABV1@@Z 5f81ce8f f   array_o.obj
 0001:0001bf08       ?FreeExtra@CObArray@@QAEXXZ 5f81cf08 f   array_o.obj
 0001:0001bfe2       ?SetAtGrow@CObArray@@QAEXHPAVCObject@@@Z 5f81cfe2 f   array_o.obj
 0001:0001c053       ?InsertAt@CObArray@@QAEXHPAVCObject@@H@Z 5f81d053 f   array_o.obj
 0001:0001c196       ?RemoveAt@CObArray@@QAEXHH@Z 5f81d196 f   array_o.obj
 0001:0001c279       ?InsertAt@CObArray@@QAEXHPAV1@@Z 5f81d279 f   array_o.obj
 0001:0001c388       ?Serialize@CObArray@@UAEXAAVCArchive@@@Z 5f81d388 f   array_o.obj
 0001:0001c456       ?Dump@CObArray@@UBEXAAVCDumpContext@@@Z 5f81d456 f   array_o.obj
 0001:0001c508       ?AssertValid@CObArray@@UBEXXZ 5f81d508 f   array_o.obj
 0001:0001c620       ??0CStringArray@@QAE@XZ    5f81d620 f   array_s.obj
 0001:0001c667       ??1CStringArray@@UAE@XZ    5f81d667 f   array_s.obj
 0001:0001c74b       ?SetSize@CStringArray@@QAEXHH@Z 5f81d74b f   array_s.obj
 0001:0001cae7       ?Append@CStringArray@@QAEHABV1@@Z 5f81dae7 f   array_s.obj
 0001:0001cbcf       ?Copy@CStringArray@@QAEXABV1@@Z 5f81dbcf f   array_s.obj
 0001:0001cc45       ?FreeExtra@CStringArray@@QAEXXZ 5f81dc45 f   array_s.obj
 0001:0001cd1f       ?SetAtGrow@CStringArray@@QAEXHPBG@Z 5f81dd1f f   array_s.obj
 0001:0001cd96       ?SetAtGrow@CStringArray@@QAEXHABVCString@@@Z 5f81dd96 f   array_s.obj
 0001:0001ce0d       ?InsertEmpty@CStringArray@@IAEXHH@Z 5f81de0d f   array_s.obj
 0001:0001cf21       ?InsertAt@CStringArray@@QAEXHPBGH@Z 5f81df21 f   array_s.obj
 0001:0001cfb7       ?InsertAt@CStringArray@@QAEXHABVCString@@H@Z 5f81dfb7 f   array_s.obj
 0001:0001d00c       ?RemoveAt@CStringArray@@QAEXHH@Z 5f81e00c f   array_s.obj
 0001:0001d108       ?InsertAt@CStringArray@@QAEXHPAV1@@Z 5f81e108 f   array_s.obj
 0001:0001d286       ?Serialize@CStringArray@@UAEXAAVCArchive@@@Z 5f81e286 f   array_s.obj
 0001:0001d354       ?Dump@CStringArray@@UBEXAAVCDumpContext@@@Z 5f81e354 f   array_s.obj
 0001:0001d405       ?AssertValid@CStringArray@@UBEXXZ 5f81e405 f   array_s.obj
 0001:0001d520       ??_GCString@@QAEPAXI@Z     5f81e520 f i array_s.obj
 0001:0001d550       ??0CUIntArray@@QAE@XZ      5f81e550 f   array_u.obj
 0001:0001d597       ??1CUIntArray@@UAE@XZ      5f81e597 f   array_u.obj
 0001:0001d607       ?SetSize@CUIntArray@@QAEXHH@Z 5f81e607 f   array_u.obj
 0001:0001d8fc       ?Append@CUIntArray@@QAEHABV1@@Z 5f81e8fc f   array_u.obj
 0001:0001d98f       ?Copy@CUIntArray@@QAEXABV1@@Z 5f81e98f f   array_u.obj
 0001:0001da08       ?FreeExtra@CUIntArray@@QAEXXZ 5f81ea08 f   array_u.obj
 0001:0001dae2       ?SetAtGrow@CUIntArray@@QAEXHI@Z 5f81eae2 f   array_u.obj
 0001:0001db53       ?InsertAt@CUIntArray@@QAEXHIH@Z 5f81eb53 f   array_u.obj
 0001:0001dc96       ?RemoveAt@CUIntArray@@QAEXHH@Z 5f81ec96 f   array_u.obj
 0001:0001dd79       ?InsertAt@CUIntArray@@QAEXHPAV1@@Z 5f81ed79 f   array_u.obj
 0001:0001de88       ?Dump@CUIntArray@@UBEXAAVCDumpContext@@@Z 5f81ee88 f   array_u.obj
 0001:0001df3a       ?AssertValid@CUIntArray@@UBEXXZ 5f81ef3a f   array_u.obj
 0001:0001e050       ??0CWordArray@@QAE@XZ      5f81f050 f   array_w.obj
 0001:0001e097       ??1CWordArray@@UAE@XZ      5f81f097 f   array_w.obj
 0001:0001e107       ?SetSize@CWordArray@@QAEXHH@Z 5f81f107 f   array_w.obj
 0001:0001e3f6       ?Append@CWordArray@@QAEHABV1@@Z 5f81f3f6 f   array_w.obj
 0001:0001e488       ?Copy@CWordArray@@QAEXABV1@@Z 5f81f488 f   array_w.obj
 0001:0001e500       ?FreeExtra@CWordArray@@QAEXXZ 5f81f500 f   array_w.obj
 0001:0001e5d8       ?SetAtGrow@CWordArray@@QAEXHG@Z 5f81f5d8 f   array_w.obj
 0001:0001e64b       ?InsertAt@CWordArray@@QAEXHGH@Z 5f81f64b f   array_w.obj
 0001:0001e78e       ?RemoveAt@CWordArray@@QAEXHH@Z 5f81f78e f   array_w.obj
 0001:0001e870       ?InsertAt@CWordArray@@QAEXHPAV1@@Z 5f81f870 f   array_w.obj
 0001:0001e97f       ?Serialize@CWordArray@@UAEXAAVCArchive@@@Z 5f81f97f f   array_w.obj
 0001:0001ea13       ?Dump@CWordArray@@UBEXAAVCDumpContext@@@Z 5f81fa13 f   array_w.obj
 0001:0001eac6       ?AssertValid@CWordArray@@UBEXXZ 5f81fac6 f   array_w.obj
 0001:0001ebe0       ??0CObList@@QAE@H@Z        5f81fbe0 f   list_o.obj
 0001:0001ec8c       ?RemoveAll@CObList@@QAEXXZ 5f81fc8c f   list_o.obj
 0001:0001ece4       ??1CObList@@UAE@XZ         5f81fce4 f   list_o.obj
 0001:0001ed5b       ?NewNode@CObList@@IAEPAUCNode@1@PAU21@0@Z 5f81fd5b f   list_o.obj
 0001:0001ee70       ?FreeNode@CObList@@IAEXPAUCNode@1@@Z 5f81fe70 f   list_o.obj
 0001:0001eed7       ?AddHead@CObList@@QAEPAU__POSITION@@PAVCObject@@@Z 5f81fed7 f   list_o.obj
 0001:0001ef42       ?AddTail@CObList@@QAEPAU__POSITION@@PAVCObject@@@Z 5f81ff42 f   list_o.obj
 0001:0001efac       ?AddHead@CObList@@QAEXPAV1@@Z 5f81ffac f   list_o.obj
 0001:0001f05c       ?AddTail@CObList@@QAEXPAV1@@Z 5f82005c f   list_o.obj
 0001:0001f10c       ?RemoveHead@CObList@@QAEPAVCObject@@XZ 5f82010c f   list_o.obj
 0001:0001f1d1       ?RemoveTail@CObList@@QAEPAVCObject@@XZ 5f8201d1 f   list_o.obj
 0001:0001f296       ?InsertBefore@CObList@@QAEPAU__POSITION@@PAU2@PAVCObject@@@Z 5f820296 f   list_o.obj
 0001:0001f378       ?InsertAfter@CObList@@QAEPAU__POSITION@@PAU2@PAVCObject@@@Z 5f820378 f   list_o.obj
 0001:0001f481       ?RemoveAt@CObList@@QAEXPAU__POSITION@@@Z 5f820481 f   list_o.obj
 0001:0001f58d       ?FindIndex@CObList@@QBEPAU__POSITION@@H@Z 5f82058d f   list_o.obj
 0001:0001f61b       ?Find@CObList@@QBEPAU__POSITION@@PAVCObject@@PAU2@@Z 5f82061b f   list_o.obj
 0001:0001f6b1       ?Serialize@CObList@@UAEXAAVCArchive@@@Z 5f8206b1 f   list_o.obj
 0001:0001f78e       ?Dump@CObList@@UBEXAAVCDumpContext@@@Z 5f82078e f   list_o.obj
 0001:0001f81d       ?AssertValid@CObList@@UBEXXZ 5f82081d f   list_o.obj
 0001:0001f8f0       ?data@CPlex@@QAEPAXXZ      5f8208f0 f i list_o.obj
 0001:0001f910       ??0CPtrList@@QAE@H@Z       5f820910 f   list_p.obj
 0001:0001f9bc       ?RemoveAll@CPtrList@@QAEXXZ 5f8209bc f   list_p.obj
 0001:0001fa14       ??1CPtrList@@UAE@XZ        5f820a14 f   list_p.obj
 0001:0001fa8b       ?NewNode@CPtrList@@IAEPAUCNode@1@PAU21@0@Z 5f820a8b f   list_p.obj
 0001:0001fba0       ?FreeNode@CPtrList@@IAEXPAUCNode@1@@Z 5f820ba0 f   list_p.obj
 0001:0001fc07       ?AddHead@CPtrList@@QAEPAU__POSITION@@PAX@Z 5f820c07 f   list_p.obj
 0001:0001fc72       ?AddTail@CPtrList@@QAEPAU__POSITION@@PAX@Z 5f820c72 f   list_p.obj
 0001:0001fcdc       ?AddHead@CPtrList@@QAEXPAV1@@Z 5f820cdc f   list_p.obj
 0001:0001fd8c       ?AddTail@CPtrList@@QAEXPAV1@@Z 5f820d8c f   list_p.obj
 0001:0001fe3c       ?RemoveHead@CPtrList@@QAEPAXXZ 5f820e3c f   list_p.obj
 0001:0001ff01       ?RemoveTail@CPtrList@@QAEPAXXZ 5f820f01 f   list_p.obj
 0001:0001ffc6       ?InsertBefore@CPtrList@@QAEPAU__POSITION@@PAU2@PAX@Z 5f820fc6 f   list_p.obj
 0001:000200a8       ?InsertAfter@CPtrList@@QAEPAU__POSITION@@PAU2@PAX@Z 5f8210a8 f   list_p.obj
 0001:000201b1       ?RemoveAt@CPtrList@@QAEXPAU__POSITION@@@Z 5f8211b1 f   list_p.obj
 0001:000202bd       ?FindIndex@CPtrList@@QBEPAU__POSITION@@H@Z 5f8212bd f   list_p.obj
 0001:0002034b       ?Find@CPtrList@@QBEPAU__POSITION@@PAXPAU2@@Z 5f82134b f   list_p.obj
 0001:000203e1       ?Dump@CPtrList@@UBEXAAVCDumpContext@@@Z 5f8213e1 f   list_p.obj
 0001:00020470       ?AssertValid@CPtrList@@UBEXXZ 5f821470 f   list_p.obj
 0001:00020540       ??0CStringList@@QAE@H@Z    5f821540 f   list_s.obj
 0001:000205ec       ?RemoveAll@CStringList@@QAEXXZ 5f8215ec f   list_s.obj
 0001:0002067f       ??1CStringList@@UAE@XZ     5f82167f f   list_s.obj
 0001:000206f6       ?NewNode@CStringList@@IAEPAUCNode@1@PAU21@0@Z 5f8216f6 f   list_s.obj
 0001:00020829       ?FreeNode@CStringList@@IAEXPAUCNode@1@@Z 5f821829 f   list_s.obj
 0001:000208a2       ?AddHead@CStringList@@QAEPAU__POSITION@@PBG@Z 5f8218a2 f   list_s.obj
 0001:0002090d       ?AddHead@CStringList@@QAEPAU__POSITION@@ABVCString@@@Z 5f82190d f   list_s.obj
 0001:0002097e       ?AddTail@CStringList@@QAEPAU__POSITION@@PBG@Z 5f82197e f   list_s.obj
 0001:000209e9       ?AddTail@CStringList@@QAEPAU__POSITION@@ABVCString@@@Z 5f8219e9 f   list_s.obj
 0001:00020a59       ?AddHead@CStringList@@QAEXPAV1@@Z 5f821a59 f   list_s.obj
 0001:00020b07       ?AddTail@CStringList@@QAEXPAV1@@Z 5f821b07 f   list_s.obj
 0001:00020bb5       ?RemoveHead@CStringList@@QAE?AVCString@@XZ 5f821bb5 f   list_s.obj
 0001:00020ccf       ?RemoveTail@CStringList@@QAE?AVCString@@XZ 5f821ccf f   list_s.obj
 0001:00020de9       ?InsertBefore@CStringList@@QAEPAU__POSITION@@PAU2@PBG@Z 5f821de9 f   list_s.obj
 0001:00020e58       ?InsertBefore@CStringList@@QAEPAU__POSITION@@PAU2@ABVCString@@@Z 5f821e58 f   list_s.obj
 0001:00020f40       ?InsertAfter@CStringList@@QAEPAU__POSITION@@PAU2@PBG@Z 5f821f40 f   list_s.obj
 0001:00020faf       ?InsertAfter@CStringList@@QAEPAU__POSITION@@PAU2@ABVCString@@@Z 5f821faf f   list_s.obj
 0001:000210be       ?RemoveAt@CStringList@@QAEXPAU__POSITION@@@Z 5f8220be f   list_s.obj
 0001:000211ca       ?FindIndex@CStringList@@QBEPAU__POSITION@@H@Z 5f8221ca f   list_s.obj
 0001:00021258       ?Find@CStringList@@QBEPAU__POSITION@@PBGPAU2@@Z 5f822258 f   list_s.obj
 0001:000212fc       ?Serialize@CStringList@@UAEXAAVCArchive@@@Z 5f8222fc f   list_s.obj
 0001:00021416       ?Dump@CStringList@@UBEXAAVCDumpContext@@@Z 5f822416 f   list_s.obj
 0001:000214e9       ?AssertValid@CStringList@@UBEXXZ 5f8224e9 f   list_s.obj
 0001:000215b0       ?Create@CPlex@@SGPAU1@AAPAU1@II@Z 5f8225b0 f   plex.obj
 0001:0002161d       ?FreeDataChain@CPlex@@QAEXXZ 5f82261d f   plex.obj
 0001:00021660       ??0CMapPtrToPtr@@QAE@H@Z   5f822660 f   map_pp.obj
 0001:0002170c       ?InitHashTable@CMapPtrToPtr@@QAEXIH@Z 5f82270c f   map_pp.obj
 0001:000217df       ?RemoveAll@CMapPtrToPtr@@QAEXXZ 5f8227df f   map_pp.obj
 0001:0002184d       ??1CMapPtrToPtr@@UAE@XZ    5f82284d f   map_pp.obj
 0001:000218c4       ?NewAssoc@CMapPtrToPtr@@IAEPAUCAssoc@1@XZ 5f8228c4 f   map_pp.obj
 0001:000219d3       ?FreeAssoc@CMapPtrToPtr@@IAEXPAUCAssoc@1@@Z 5f8229d3 f   map_pp.obj
 0001:00021a3d       ?GetAssocAt@CMapPtrToPtr@@IBEPAUCAssoc@1@PAXAAI@Z 5f822a3d f   map_pp.obj
 0001:00021aa7       ?GetValueAt@CMapPtrToPtr@@QBEPAXPAX@Z 5f822aa7 f   map_pp.obj
 0001:00021b10       ?Lookup@CMapPtrToPtr@@QBEHPAXAAPAX@Z 5f822b10 f   map_pp.obj
 0001:00021b5f       ??ACMapPtrToPtr@@QAEAAPAXPAX@Z 5f822b5f f   map_pp.obj
 0001:00021bee       ?RemoveKey@CMapPtrToPtr@@QAEHPAX@Z 5f822bee f   map_pp.obj
 0001:00021c87       ?GetNextAssoc@CMapPtrToPtr@@QBEXAAPAU__POSITION@@AAPAX1@Z 5f822c87 f   map_pp.obj
 0001:00021df9       ?Dump@CMapPtrToPtr@@UBEXAAVCDumpContext@@@Z 5f822df9 f   map_pp.obj
 0001:00021eaa       ?AssertValid@CMapPtrToPtr@@UBEXXZ 5f822eaa f   map_pp.obj
 0001:00021f20       ??0CMapPtrToWord@@QAE@H@Z  5f822f20 f   map_pw.obj
 0001:00021fcc       ?InitHashTable@CMapPtrToWord@@QAEXIH@Z 5f822fcc f   map_pw.obj
 0001:0002209f       ?RemoveAll@CMapPtrToWord@@QAEXXZ 5f82309f f   map_pw.obj
 0001:0002210d       ??1CMapPtrToWord@@UAE@XZ   5f82310d f   map_pw.obj
 0001:00022184       ?NewAssoc@CMapPtrToWord@@IAEPAUCAssoc@1@XZ 5f823184 f   map_pw.obj
 0001:00022292       ?FreeAssoc@CMapPtrToWord@@IAEXPAUCAssoc@1@@Z 5f823292 f   map_pw.obj
 0001:000222fc       ?GetAssocAt@CMapPtrToWord@@IBEPAUCAssoc@1@PAXAAI@Z 5f8232fc f   map_pw.obj
 0001:00022366       ?Lookup@CMapPtrToWord@@QBEHPAXAAG@Z 5f823366 f   map_pw.obj
 0001:000223b7       ??ACMapPtrToWord@@QAEAAGPAX@Z 5f8233b7 f   map_pw.obj
 0001:00022446       ?RemoveKey@CMapPtrToWord@@QAEHPAX@Z 5f823446 f   map_pw.obj
 0001:000224df       ?GetNextAssoc@CMapPtrToWord@@QBEXAAPAU__POSITION@@AAPAXAAG@Z 5f8234df f   map_pw.obj
 0001:00022653       ?Dump@CMapPtrToWord@@UBEXAAVCDumpContext@@@Z 5f823653 f   map_pw.obj
 0001:00022705       ?AssertValid@CMapPtrToWord@@UBEXXZ 5f823705 f   map_pw.obj
 0001:00022770       ?HashKey@CMapPtrToPtr@@QBEIPAX@Z 5f823770 f i map_pw.obj
 0001:00022770       ?HashKey@CMapPtrToWord@@QBEIPAX@Z 5f823770 f i map_pw.obj
 0001:00022790       ??0CMapStringToOb@@QAE@H@Z 5f823790 f   map_so.obj
 0001:0002283c       ?InitHashTable@CMapStringToOb@@QAEXIH@Z 5f82383c f   map_so.obj
 0001:0002290f       ?RemoveAll@CMapStringToOb@@QAEXXZ 5f82390f f   map_so.obj
 0001:000229db       ??1CMapStringToOb@@UAE@XZ  5f8239db f   map_so.obj
 0001:00022a52       ?NewAssoc@CMapStringToOb@@IAEPAUCAssoc@1@XZ 5f823a52 f   map_so.obj
 0001:00022b71       ?FreeAssoc@CMapStringToOb@@IAEXPAUCAssoc@1@@Z 5f823b71 f   map_so.obj
 0001:00022bea       ?GetAssocAt@CMapStringToOb@@IBEPAUCAssoc@1@PBGAAI@Z 5f823bea f   map_so.obj
 0001:00022c62       ?Lookup@CMapStringToOb@@QBEHPBGAAPAVCObject@@@Z 5f823c62 f   map_so.obj
 0001:00022cb1       ?LookupKey@CMapStringToOb@@QBEHPBGAAPBG@Z 5f823cb1 f   map_so.obj
 0001:00022d05       ??ACMapStringToOb@@QAEAAPAVCObject@@PBG@Z 5f823d05 f   map_so.obj
 0001:00022da3       ?RemoveKey@CMapStringToOb@@QAEHPBG@Z 5f823da3 f   map_so.obj
 0001:00022e4a       ?GetNextAssoc@CMapStringToOb@@QBEXAAPAU__POSITION@@AAVCString@@AAPAVCObject@@@Z 5f823e4a f   map_so.obj
 0001:00022faf       ?Serialize@CMapStringToOb@@UAEXAAVCArchive@@@Z 5f823faf f   map_so.obj
 0001:0002311e       ?Dump@CMapStringToOb@@UBEXAAVCDumpContext@@@Z 5f82411e f   map_so.obj
 0001:0002320b       ?AssertValid@CMapStringToOb@@UBEXXZ 5f82420b f   map_so.obj
 0001:00023280       ??0CMapStringToPtr@@QAE@H@Z 5f824280 f   map_sp.obj
 0001:0002332c       ?InitHashTable@CMapStringToPtr@@QAEXIH@Z 5f82432c f   map_sp.obj
 0001:000233ff       ?RemoveAll@CMapStringToPtr@@QAEXXZ 5f8243ff f   map_sp.obj
 0001:000234cb       ??1CMapStringToPtr@@UAE@XZ 5f8244cb f   map_sp.obj
 0001:00023542       ?NewAssoc@CMapStringToPtr@@IAEPAUCAssoc@1@XZ 5f824542 f   map_sp.obj
 0001:00023661       ?FreeAssoc@CMapStringToPtr@@IAEXPAUCAssoc@1@@Z 5f824661 f   map_sp.obj
 0001:000236da       ?GetAssocAt@CMapStringToPtr@@IBEPAUCAssoc@1@PBGAAI@Z 5f8246da f   map_sp.obj
 0001:00023752       ?Lookup@CMapStringToPtr@@QBEHPBGAAPAX@Z 5f824752 f   map_sp.obj
 0001:000237a1       ?LookupKey@CMapStringToPtr@@QBEHPBGAAPBG@Z 5f8247a1 f   map_sp.obj
 0001:000237f5       ??ACMapStringToPtr@@QAEAAPAXPBG@Z 5f8247f5 f   map_sp.obj
 0001:00023893       ?RemoveKey@CMapStringToPtr@@QAEHPBG@Z 5f824893 f   map_sp.obj
 0001:0002393a       ?GetNextAssoc@CMapStringToPtr@@QBEXAAPAU__POSITION@@AAVCString@@AAPAX@Z 5f82493a f   map_sp.obj
 0001:00023a9f       ?Dump@CMapStringToPtr@@UBEXAAVCDumpContext@@@Z 5f824a9f f   map_sp.obj
 0001:00023b8c       ?AssertValid@CMapStringToPtr@@UBEXXZ 5f824b8c f   map_sp.obj
 0001:00023c00       ??0CMapStringToString@@QAE@H@Z 5f824c00 f   map_ss.obj
 0001:00023cac       ?InitHashTable@CMapStringToString@@QAEXIH@Z 5f824cac f   map_ss.obj
 0001:00023d7f       ?RemoveAll@CMapStringToString@@QAEXXZ 5f824d7f f   map_ss.obj
 0001:00023e5a       ??1CMapStringToString@@UAE@XZ 5f824e5a f   map_ss.obj
 0001:00023ed1       ?NewAssoc@CMapStringToString@@IAEPAUCAssoc@1@XZ 5f824ed1 f   map_ss.obj
 0001:0002400e       ?FreeAssoc@CMapStringToString@@IAEXPAUCAssoc@1@@Z 5f82500e f   map_ss.obj
 0001:00024096       ?GetAssocAt@CMapStringToString@@IBEPAUCAssoc@1@PBGAAI@Z 5f825096 f   map_ss.obj
 0001:0002410e       ?Lookup@CMapStringToString@@QBEHPBGAAVCString@@@Z 5f82510e f   map_ss.obj
 0001:00024161       ?LookupKey@CMapStringToString@@QBEHPBGAAPBG@Z 5f825161 f   map_ss.obj
 0001:000241b5       ??ACMapStringToString@@QAEAAVCString@@PBG@Z 5f8251b5 f   map_ss.obj
 0001:00024253       ?RemoveKey@CMapStringToString@@QAEHPBG@Z 5f825253 f   map_ss.obj
 0001:000242fa       ?GetNextAssoc@CMapStringToString@@QBEXAAPAU__POSITION@@AAVCString@@1@Z 5f8252fa f   map_ss.obj
 0001:00024463       ?Serialize@CMapStringToString@@UAEXAAVCArchive@@@Z 5f825463 f   map_ss.obj
 0001:000245f2       ?Dump@CMapStringToString@@UBEXAAVCDumpContext@@@Z 5f8255f2 f   map_ss.obj
 0001:000246fa       ?AssertValid@CMapStringToString@@UBEXXZ 5f8256fa f   map_ss.obj
 0001:00024770       ?HashKey@CMapStringToPtr@@QBEIPBG@Z 5f825770 f i map_ss.obj
 0001:00024770       ?HashKey@CMapStringToString@@QBEIPBG@Z 5f825770 f i map_ss.obj
 0001:00024770       ?HashKey@CMapStringToOb@@QBEIPBG@Z 5f825770 f i map_ss.obj
 0001:000247c0       ??0CMapWordToOb@@QAE@H@Z   5f8257c0 f   map_wo.obj
 0001:0002486c       ?InitHashTable@CMapWordToOb@@QAEXIH@Z 5f82586c f   map_wo.obj
 0001:0002493f       ?RemoveAll@CMapWordToOb@@QAEXXZ 5f82593f f   map_wo.obj
 0001:000249ad       ??1CMapWordToOb@@UAE@XZ    5f8259ad f   map_wo.obj
 0001:00024a24       ?NewAssoc@CMapWordToOb@@IAEPAUCAssoc@1@XZ 5f825a24 f   map_wo.obj
 0001:00024b32       ?FreeAssoc@CMapWordToOb@@IAEXPAUCAssoc@1@@Z 5f825b32 f   map_wo.obj
 0001:00024b9c       ?GetAssocAt@CMapWordToOb@@IBEPAUCAssoc@1@GAAI@Z 5f825b9c f   map_wo.obj
 0001:00024c12       ?Lookup@CMapWordToOb@@QBEHGAAPAVCObject@@@Z 5f825c12 f   map_wo.obj
 0001:00024c62       ??ACMapWordToOb@@QAEAAPAVCObject@@G@Z 5f825c62 f   map_wo.obj
 0001:00024cf4       ?RemoveKey@CMapWordToOb@@QAEHG@Z 5f825cf4 f   map_wo.obj
 0001:00024d98       ?GetNextAssoc@CMapWordToOb@@QBEXAAPAU__POSITION@@AAGAAPAVCObject@@@Z 5f825d98 f   map_wo.obj
 0001:00024f0d       ?Serialize@CMapWordToOb@@UAEXAAVCArchive@@@Z 5f825f0d f   map_wo.obj
 0001:0002503a       ?Dump@CMapWordToOb@@UBEXAAVCDumpContext@@@Z 5f82603a f   map_wo.obj
 0001:000250ec       ?AssertValid@CMapWordToOb@@UBEXXZ 5f8260ec f   map_wo.obj
 0001:00025160       ??0CMapWordToPtr@@QAE@H@Z  5f826160 f   map_wp.obj
 0001:0002520c       ?InitHashTable@CMapWordToPtr@@QAEXIH@Z 5f82620c f   map_wp.obj
 0001:000252df       ?RemoveAll@CMapWordToPtr@@QAEXXZ 5f8262df f   map_wp.obj
 0001:0002534d       ??1CMapWordToPtr@@UAE@XZ   5f82634d f   map_wp.obj
 0001:000253c4       ?NewAssoc@CMapWordToPtr@@IAEPAUCAssoc@1@XZ 5f8263c4 f   map_wp.obj
 0001:000254d2       ?FreeAssoc@CMapWordToPtr@@IAEXPAUCAssoc@1@@Z 5f8264d2 f   map_wp.obj
 0001:0002553c       ?GetAssocAt@CMapWordToPtr@@IBEPAUCAssoc@1@GAAI@Z 5f82653c f   map_wp.obj
 0001:000255b2       ?Lookup@CMapWordToPtr@@QBEHGAAPAX@Z 5f8265b2 f   map_wp.obj
 0001:00025602       ??ACMapWordToPtr@@QAEAAPAXG@Z 5f826602 f   map_wp.obj
 0001:00025694       ?RemoveKey@CMapWordToPtr@@QAEHG@Z 5f826694 f   map_wp.obj
 0001:00025738       ?GetNextAssoc@CMapWordToPtr@@QBEXAAPAU__POSITION@@AAGAAPAX@Z 5f826738 f   map_wp.obj
 0001:000258ad       ?Dump@CMapWordToPtr@@UBEXAAVCDumpContext@@@Z 5f8268ad f   map_wp.obj
 0001:0002595f       ?AssertValid@CMapWordToPtr@@UBEXXZ 5f82695f f   map_wp.obj
 0001:000259d0       ?HashKey@CMapWordToOb@@QBEIG@Z 5f8269d0 f i map_wp.obj
 0001:000259d0       ?HashKey@CMapWordToPtr@@QBEIG@Z 5f8269d0 f i map_wp.obj
 0001:000259f0       ?_GetBaseClass@CObject@@SGPAUCRuntimeClass@@XZ 5f8269f0 f   objcore.obj
 0001:000259f7       ?GetRuntimeClass@CObject@@UBEPAUCRuntimeClass@@XZ 5f8269f7 f   objcore.obj
 0001:00025a07       ?IsKindOf@CObject@@QBEHPBUCRuntimeClass@@@Z 5f826a07 f   objcore.obj
 0001:00025a7a       ?AfxDynamicDownCast@@YAPAVCObject@@PAUCRuntimeClass@@PAV1@@Z 5f826a7a f   objcore.obj
 0001:00025a9c       ?AfxStaticDownCast@@YAPAVCObject@@PAUCRuntimeClass@@PAV1@@Z 5f826a9c f   objcore.obj
 0001:00025ad7       ?AfxAssertValidObject@@YGXPBVCObject@@PBDH@Z 5f826ad7 f   objcore.obj
 0001:00025be1       ?AssertValid@CObject@@UBEXXZ 5f826be1 f   objcore.obj
 0001:00025c0f       ?Dump@CObject@@UBEXAAVCDumpContext@@@Z 5f826c0f f   objcore.obj
 0001:00025c60       ?CreateObject@CRuntimeClass@@QAEPAVCObject@@XZ 5f826c60 f   objcore.obj
 0001:00025d18       ?IsSerializable@CObject@@QBEHXZ 5f826d18 f   objcore.obj
 0001:00025d3b       ?AfxClassInit@@YGXPAUCRuntimeClass@@@Z 5f826d3b f   objcore.obj
 0001:00025d6a       ??0AFX_CLASSINIT_COMPAT@@QAE@PAUCRuntimeClass@@@Z 5f826d6a f   objcore.obj
 0001:00025da1       ?IsDerivedFrom@CRuntimeClass@@QBEHPBU1@@Z 5f826da1 f   objcore.obj
 0001:00025e74       ?AfxDoForAllClasses@@YGXP6AXPBUCRuntimeClass@@PAX@Z1@Z 5f826e74 f   objcore.obj
 0001:00025f30       ?AddHead@?$CTypedSimpleList@PAUCRuntimeClass@@@@QAEXPAUCRuntimeClass@@@Z 5f826f30 f i objcore.obj
 0001:00025f50       ??B?$CTypedSimpleList@PAVCDynLinkLibrary@@@@QAEPAVCDynLinkLibrary@@XZ 5f826f50 f i objcore.obj
 0001:00025f50       ??B?$CTypedSimpleList@PAUCRuntimeClass@@@@QAEPAUCRuntimeClass@@XZ 5f826f50 f i objcore.obj
 0001:00025f70       ??3CException@@SGXPAX@Z    5f826f70 f   except.obj
 0001:00025fe1       ??3CException@@SGXPAXPBDH@Z 5f826fe1 f   except.obj
 0001:00025ff1       ??0CException@@QAE@XZ      5f826ff1 f   except.obj
 0001:00026024       ??0CException@@QAE@H@Z     5f827024 f   except.obj
 0001:00026058       ?Delete@CException@@QAEXXZ 5f827058 f   except.obj
 0001:000260a3       ?GetErrorMessage@CException@@UAEHPAGIPAI@Z 5f8270a3 f   except.obj
 0001:000260d5       ?ReportError@CException@@UAEHII@Z 5f8270d5 f   except.obj
 0001:00026155       ??0AFX_EXCEPTION_LINK@@QAE@XZ 5f827155 f   except.obj
 0001:00026189       ?AfxTryCleanup@@YGXXZ      5f827189 f   except.obj
 0001:000261e7       ?AfxThrowLastCleanup@@YGXXZ 5f8271e7 f   except.obj
 0001:00026220       ??_GCException@@UAEPAXI@Z  5f827220 f i except.obj
 0001:00026220       ??_ECException@@UAEPAXI@Z  5f827220 f i except.obj
 0001:00026250       ?AfxGetExceptionContext@@YAPAUAFX_EXCEPTION_CONTEXT@@XZ 5f827250 f i except.obj
 0001:00026280       ??2CObject@@SGPAXI@Z       5f827280 f   afxmem.obj
 0001:00026299       ??3CObject@@SGXPAX@Z       5f827299 f   afxmem.obj
 0001:000262af       ??3CObject@@SGXPAX0@Z      5f8272af f   afxmem.obj
 0001:000262c5       ??2@YAPAXIPBDH@Z           5f8272c5 f   afxmem.obj
 0001:000262e0       ??3@YAXPAXPBDH@Z           5f8272e0 f   afxmem.obj
 0001:000262f1       ??2CObject@@SGPAXIPBDH@Z   5f8272f1 f   afxmem.obj
 0001:0002630e       ??3CObject@@SGXPAXPBDH@Z   5f82730e f   afxmem.obj
 0001:00026324       ?AfxAllocMemoryDebug@@YGPAXIHPBDH@Z 5f827324 f   afxmem.obj
 0001:0002634e       ?AfxFreeMemoryDebug@@YGXPAXH@Z 5f82734e f   afxmem.obj
 0001:00026370       ?_AfxDefaultAllocHook@@YGHIHJ@Z 5f827370 f   afxmem.obj
 0001:0002637c       ?_AfxAllocHookProxy@@YAHHPAXIHJPBEH@Z 5f82737c f   afxmem.obj
 0001:000263fb       ?AfxSetAllocHook@@YGP6GHIHJ@ZP6GHIHJ@Z@Z 5f8273fb f   afxmem.obj
 0001:00026435       ?AfxEnableMemoryTracking@@YGHH@Z 5f827435 f   afxmem.obj
 0001:0002648a       ?AfxSetAllocStop@@YGXJ@Z   5f82748a f   afxmem.obj
 0001:0002649e       ?AfxCheckMemory@@YGHXZ     5f82749e f   afxmem.obj
 0001:000264a9       ?AfxIsMemoryBlock@@YGHPBXIPAJ@Z 5f8274a9 f   afxmem.obj
 0001:000264c9       ??0CMemoryState@@QAE@XZ    5f8274c9 f   afxmem.obj
 0001:000264e7       ?UpdateData@CMemoryState@@QAEXXZ 5f8274e7 f   afxmem.obj
 0001:00026550       ?Difference@CMemoryState@@QAEHABU1@0@Z 5f827550 f   afxmem.obj
 0001:00026588       ?DumpStatistics@CMemoryState@@QBEXXZ 5f827588 f   afxmem.obj
 0001:000265a0       ?Checkpoint@CMemoryState@@QAEXXZ 5f8275a0 f   afxmem.obj
 0001:000265c0       ?DumpAllObjectsSince@CMemoryState@@QBEXXZ 5f8275c0 f   afxmem.obj
 0001:000265d8       ?_AfxDoForAllObjectsProxy@@YAXPAX0@Z 5f8275d8 f   afxmem.obj
 0001:000265f9       ?AfxDoForAllObjects@@YGXP6AXPAVCObject@@PAX@Z1@Z 5f8275f9 f   afxmem.obj
 0001:00026623       ?AfxDumpMemoryLeaks@@YGHXZ 5f827623 f   afxmem.obj
 0001:0002662e       ?AfxNewHandler@@YAHI@Z     5f82762e f   afxmem.obj
 0001:0002663a       ?AfxGetNewHandler@@YGP6AHI@ZXZ 5f82763a f   afxmem.obj
 0001:00026650       ?AfxSetNewHandler@@YGP6AHI@ZP6AHI@Z@Z 5f827650 f   afxmem.obj
 0001:00026679       ??2@YAPAXI@Z               5f827679 f   afxmem.obj
 0001:000266e3       ??3@YAXPAX@Z               5f8276e3 f   afxmem.obj
 0001:000266f7       ??2@YAPAXIHPBDH@Z          5f8276f7 f   afxmem.obj
 0001:00026770       ?IsDirSep@@YAHG@Z          5f827770 f i filecore.obj
 0001:000267b0       ??0CFile@@QAE@XZ           5f8277b0 f   filecore.obj
 0001:0002681b       ??0CFile@@QAE@H@Z          5f82781b f   filecore.obj
 0001:00026887       ??0CFile@@QAE@PBGI@Z       5f827887 f   filecore.obj
 0001:0002695e       ??1CFile@@UAE@XZ           5f82795e f   filecore.obj
 0001:000269d0       ?Duplicate@CFile@@UBEPAV1@XZ 5f8279d0 f   filecore.obj
 0001:00026b13       ?Open@CFile@@UAEHPBGIPAVCFileException@@@Z 5f827b13 f   filecore.obj
 0001:00026e75       ?Read@CFile@@UAEIPAXI@Z    5f827e75 f   filecore.obj
 0001:00026f47       ?Write@CFile@@UAEXPBXI@Z   5f827f47 f   filecore.obj
 0001:0002703e       ?Seek@CFile@@UAEJJI@Z      5f82803e f   filecore.obj
 0001:000270f3       ?GetPosition@CFile@@UBEKXZ 5f8280f3 f   filecore.obj
 0001:00027169       ?Flush@CFile@@UAEXXZ       5f828169 f   filecore.obj
 0001:000271b1       ?Close@CFile@@UAEXXZ       5f8281b1 f   filecore.obj
 0001:00027252       ?Abort@CFile@@UAEXXZ       5f828252 f   filecore.obj
 0001:0002729b       ?LockRange@CFile@@UAEXKK@Z 5f82829b f   filecore.obj
 0001:0002730f       ?UnlockRange@CFile@@UAEXKK@Z 5f82830f f   filecore.obj
 0001:00027383       ?SetLength@CFile@@UAEXK@Z  5f828383 f   filecore.obj
 0001:000273fc       ?GetLength@CFile@@UBEKXZ   5f8283fc f   filecore.obj
 0001:00027478       ?GetBufferPtr@CFile@@UAEIIIPAPAX0@Z 5f828478 f   filecore.obj
 0001:000274ad       ?Rename@CFile@@SGXPBG0@Z   5f8284ad f   filecore.obj
 0001:000274d4       ?Remove@CFile@@SGXPBG@Z    5f8284d4 f   filecore.obj
 0001:000274f7       ?CreateInstance@AFX_COM@@QAEJABU_GUID@@PAUIUnknown@@0PAPAX@Z 5f8284f7 f   filecore.obj
 0001:00027580       ?GetClassObject@AFX_COM@@QAEJABU_GUID@@0PAPAX@Z 5f828580 f   filecore.obj
 0001:000276cc       ?AfxStringFromCLSID@@YG?AVCString@@ABU_GUID@@@Z 5f8286cc f   filecore.obj
 0001:0002777c       ?AfxGetInProcServer@@YGHPBGAAVCString@@@Z 5f82877c f   filecore.obj
 0001:0002785b       ?AfxResolveShortcut@@YGHPAVCWnd@@PBGPAGH@Z 5f82885b f   filecore.obj
 0001:00027991       ?AfxFullPath@@YGHPAGPBG@Z  5f828991 f   filecore.obj
 0001:00027b38       ?AfxGetRoot@@YGXPBGAAVCString@@@Z 5f828b38 f   filecore.obj
 0001:00027d49       ?AfxComparePath@@YGHPBG0@Z 5f828d49 f   filecore.obj
 0001:00027f90       ?AfxGetFileTitle@@YGIPBGPAGI@Z 5f828f90 f   filecore.obj
 0001:00028075       ?AfxGetModuleShortFileName@@YGXPAUHINSTANCE__@@AAVCString@@@Z 5f829075 f   filecore.obj
 0001:000280d7       ?AssertValid@CFile@@UBEXXZ 5f8290d7 f   filecore.obj
 0001:000280ea       ?Dump@CFile@@UBEXAAVCDumpContext@@@Z 5f8290ea f   filecore.obj
 0001:00028160       ??0CStdioFile@@QAE@XZ      5f829160 f   filetxt.obj
 0001:00028189       ??0CStdioFile@@QAE@PAU_iobuf@@@Z 5f829189 f   filetxt.obj
 0001:0002821e       ??0CStdioFile@@QAE@PBGI@Z  5f82921e f   filetxt.obj
 0001:00028303       ??1CStdioFile@@UAE@XZ      5f829303 f   filetxt.obj
 0001:00028376       ?Open@CStdioFile@@UAEHPBGIPAVCFileException@@@Z 5f829376 f   filetxt.obj
 0001:000285ef       ?Read@CStdioFile@@UAEIPAXI@Z 5f8295ef f   filetxt.obj
 0001:00028709       ?Write@CStdioFile@@UAEXPBXI@Z 5f829709 f   filetxt.obj
 0001:000287ba       ?WriteString@CStdioFile@@UAEXPBG@Z 5f8297ba f   filetxt.obj
 0001:00028847       ?ReadString@CStdioFile@@UAEPAGPAGI@Z 5f829847 f   filetxt.obj
 0001:0002892c       ?ReadString@CStdioFile@@UAEHAAVCString@@@Z 5f82992c f   filetxt.obj
 0001:00028a84       ?Seek@CStdioFile@@UAEJJI@Z 5f829a84 f   filetxt.obj
 0001:00028b49       ?GetPosition@CStdioFile@@UBEKXZ 5f829b49 f   filetxt.obj
 0001:00028bca       ?Flush@CStdioFile@@UAEXXZ  5f829bca f   filetxt.obj
 0001:00028c21       ?Close@CStdioFile@@UAEXXZ  5f829c21 f   filetxt.obj
 0001:00028ccd       ?Abort@CStdioFile@@UAEXXZ  5f829ccd f   filetxt.obj
 0001:00028d2b       ?Duplicate@CStdioFile@@UBEPAVCFile@@XZ 5f829d2b f   filetxt.obj
 0001:00028d79       ?LockRange@CStdioFile@@UAEXKK@Z 5f829d79 f   filetxt.obj
 0001:00028dc7       ?UnlockRange@CStdioFile@@UAEXKK@Z 5f829dc7 f   filetxt.obj
 0001:00028e15       ?Dump@CStdioFile@@UBEXAAVCDumpContext@@@Z 5f829e15 f   filetxt.obj
 0001:00028e60       ?ThrowOsError@CFileException@@SGXJPBG@Z 5f829e60 f   filex.obj
 0001:00028e84       ?ThrowErrno@CFileException@@SGXHPBG@Z 5f829e84 f   filex.obj
 0001:00028ead       ?GetErrorMessage@CFileException@@UAEHPAGIPAI@Z 5f829ead f   filex.obj
 0001:00028fbc       ?Dump@CFileException@@UBEXAAVCDumpContext@@@Z 5f829fbc f   filex.obj
 0001:00029041       ?AfxThrowFileException@@YGXHJPBG@Z 5f82a041 f   filex.obj
 0001:00029114       ?ErrnoToException@CFileException@@SGHH@Z 5f82a114 f   filex.obj
 0001:000291bf       ?OsErrorToException@CFileException@@SGHJ@Z 5f82a1bf f   filex.obj
 0001:00029720       ?Dump@CFileStatus@@QBEXAAVCDumpContext@@@Z 5f82a720 f   filest.obj
 0001:0002980a       ?GetFileName@CFile@@UBE?AVCString@@XZ 5f82a80a f   filest.obj
 0001:000298da       ?GetFileTitle@CFile@@UBE?AVCString@@XZ 5f82a8da f   filest.obj
 0001:000299aa       ?GetFilePath@CFile@@UBE?AVCString@@XZ 5f82a9aa f   filest.obj
 0001:00029a19       ?GetStatus@CFile@@QBEHAAUCFileStatus@@@Z 5f82aa19 f   filest.obj
 0001:00029bac       ?GetStatus@CFile@@SGHPBGAAUCFileStatus@@@Z 5f82abac f   filest.obj
 0001:00029d0a       ?AfxTimeToFileTime@@YAXABVCTime@@PAU_FILETIME@@@Z 5f82ad0a f   filest.obj
 0001:00029da2       ?SetStatus@CFile@@SGXPBGABUCFileStatus@@@Z 5f82ada2 f   filest.obj
 0001:00029f49       ?GetStatus@CMemFile@@QBEHAAUCFileStatus@@@Z 5f82af49 f   filest.obj
 0001:00029fb0       ??0CFileStatus@@QAE@XZ     5f82afb0 f i filest.obj
 0001:00029fe0       ?AfxGetEmptyString@@YGABVCString@@XZ 5f82afe0 f   strcore.obj
 0001:00029fea       ??0CString@@QAE@XZ         5f82afea f   strcore.obj
 0001:0002a000       ??0CString@@QAE@ABV0@@Z    5f82b000 f   strcore.obj
 0001:0002a09f       ?AllocBuffer@CString@@IAEXH@Z 5f82b09f f   strcore.obj
 0001:0002a15a       ?FreeData@CString@@KIXPAUCStringData@@@Z 5f82b15a f   strcore.obj
 0001:0002a179       ?Release@CString@@IAEXXZ   5f82b179 f   strcore.obj
 0001:0002a1eb       ?Release@CString@@KGXPAUCStringData@@@Z 5f82b1eb f   strcore.obj
 0001:0002a23b       ?Empty@CString@@QAEXXZ     5f82b23b f   strcore.obj
 0001:0002a2e0       ?CopyBeforeWrite@CString@@IAEXXZ 5f82b2e0 f   strcore.obj
 0001:0002a36b       ?AllocBeforeWrite@CString@@IAEXH@Z 5f82b36b f   strcore.obj
 0001:0002a3d6       ??1CString@@QAE@XZ         5f82b3d6 f   strcore.obj
 0001:0002a413       ?AllocCopy@CString@@IBEXAAV1@HHH@Z 5f82b413 f   strcore.obj
 0001:0002a467       ??0CString@@QAE@PBG@Z      5f82b467 f   strcore.obj
 0001:0002a500       ??0CString@@QAE@PBD@Z      5f82b500 f   strcore.obj
 0001:0002a571       ??6@YGAAVCDumpContext@@AAV0@ABVCString@@@Z 5f82b571 f   strcore.obj
 0001:0002a589       ?AssignCopy@CString@@IAEXHPBG@Z 5f82b589 f   strcore.obj
 0001:0002a5d6       ??4CString@@QAEABV0@ABV0@@Z 5f82b5d6 f   strcore.obj
 0001:0002a68d       ??4CString@@QAEABV0@PBG@Z  5f82b68d f   strcore.obj
 0001:0002a6e8       ??4CString@@QAEABV0@PBD@Z  5f82b6e8 f   strcore.obj
 0001:0002a74b       ?ConcatCopy@CString@@IAEXHPBGH0@Z 5f82b74b f   strcore.obj
 0001:0002a7ab       ??H@YG?AVCString@@ABV0@0@Z 5f82b7ab f   strcore.obj
 0001:0002a83c       ??H@YG?AVCString@@ABV0@PBG@Z 5f82b83c f   strcore.obj
 0001:0002a8fe       ??H@YG?AVCString@@PBGABV0@@Z 5f82b8fe f   strcore.obj
 0001:0002a9c0       ?ConcatInPlace@CString@@IAEXHPBG@Z 5f82b9c0 f   strcore.obj
 0001:0002aaee       ??YCString@@QAEABV0@PBG@Z  5f82baee f   strcore.obj
 0001:0002ab49       ??YCString@@QAEABV0@G@Z    5f82bb49 f   strcore.obj
 0001:0002ab67       ??YCString@@QAEABV0@ABV0@@Z 5f82bb67 f   strcore.obj
 0001:0002ab91       ?GetBuffer@CString@@QAEPAGH@Z 5f82bb91 f   strcore.obj
 0001:0002accd       ?ReleaseBuffer@CString@@QAEXH@Z 5f82bccd f   strcore.obj
 0001:0002ad43       ?GetBufferSetLength@CString@@QAEPAGH@Z 5f82bd43 f   strcore.obj
 0001:0002ada3       ?FreeExtra@CString@@QAEXXZ 5f82bda3 f   strcore.obj
 0001:0002aea6       ?LockBuffer@CString@@QAEPAGXZ 5f82bea6 f   strcore.obj
 0001:0002aed1       ?UnlockBuffer@CString@@QAEXXZ 5f82bed1 f   strcore.obj
 0001:0002af27       ?Find@CString@@QBEHG@Z     5f82bf27 f   strcore.obj
 0001:0002af43       ?Find@CString@@QBEHGH@Z    5f82bf43 f   strcore.obj
 0001:0002afa8       ?FindOneOf@CString@@QBEHPBG@Z 5f82bfa8 f   strcore.obj
 0001:0002b01a       ?MakeUpper@CString@@QAEXXZ 5f82c01a f   strcore.obj
 0001:0002b03c       ?MakeLower@CString@@QAEXXZ 5f82c03c f   strcore.obj
 0001:0002b05e       ?MakeReverse@CString@@QAEXXZ 5f82c05e f   strcore.obj
 0001:0002b080       ?SetAt@CString@@QAEXHG@Z   5f82c080 f   strcore.obj
 0001:0002b0f5       ?_wcstombsz@@YAHPADPBGI@Z  5f82c0f5 f   strcore.obj
 0001:0002b16d       ?_mbstowcsz@@YAHPAGPBDI@Z  5f82c16d f   strcore.obj
 0001:0002b1e4       ?AfxA2WHelper@@YGPAGPAGPBDH@Z 5f82c1e4 f   strcore.obj
 0001:0002b25c       ?AfxW2AHelper@@YGPADPADPBGH@Z 5f82c25c f   strcore.obj
 0001:0002b477       ??0CWnd@@QAE@XZ            5f82c477 f   wincore.obj
 0001:0002b4a9       ??0CWnd@@AAE@PAUHWND__@@@Z 5f82c4a9 f   wincore.obj
 0001:0002b4e6       ?_AfxModifyStyle@@YGHPAUHWND__@@HKKI@Z 5f82c4e6 f   wincore.obj
 0001:0002b579       ?ModifyStyle@CWnd@@SGHPAUHWND__@@KKI@Z 5f82c579 f   wincore.obj
 0001:0002b597       ?ModifyStyleEx@CWnd@@SGHPAUHWND__@@KKI@Z 5f82c597 f   wincore.obj
 0001:0002b5b5       ?_AfxPreInitDialog@@YGXPAVCWnd@@PAUtagRECT@@PAK@Z 5f82c5b5 f   wincore.obj
 0001:0002b615       ?_AfxPostInitDialog@@YGXPAVCWnd@@ABUtagRECT@@K@Z 5f82c615 f   wincore.obj
 0001:0002b6b4       ?_AfxHandleActivate@@YGXPAVCWnd@@I0@Z 5f82c6b4 f   wincore.obj
 0001:0002b738       ?_AfxHandleSetCursor@@YGHPAVCWnd@@II@Z 5f82c738 f   wincore.obj
 0001:0002b7ac       ?AfxCallWndProc@@YGJPAVCWnd@@PAUHWND__@@IIJ@Z 5f82c7ac f   wincore.obj
 0001:0002b95c       ?GetCurrentMessage@CWnd@@KGPBUtagMSG@@XZ 5f82c95c f   wincore.obj
 0001:0002b9a2       ?Default@CWnd@@IAEJXZ      5f82c9a2 f   wincore.obj
 0001:0002b9df       ?afxMapHWND@@YGPAVCHandleMap@@H@Z 5f82c9df f   wincore.obj
 0001:0002baaf       ?FromHandle@CWnd@@SGPAV1@PAUHWND__@@@Z 5f82caaf f   wincore.obj
 0001:0002bb34       ?FromHandlePermanent@CWnd@@SGPAV1@PAUHWND__@@@Z 5f82cb34 f   wincore.obj
 0001:0002bb9a       ?Attach@CWnd@@QAEHPAUHWND__@@@Z 5f82cb9a f   wincore.obj
 0001:0002bc57       ?Detach@CWnd@@QAEPAUHWND__@@XZ 5f82cc57 f   wincore.obj
 0001:0002bca9       ?PreSubclassWindow@CWnd@@UAEXXZ 5f82cca9 f   wincore.obj
 0001:0002bcb4       ?AfxWndProc@@YGJPAUHWND__@@IIJ@Z 5f82ccb4 f   wincore.obj
 0001:0002bd3e       ?AfxGetAfxWndProc@@YGP6GJPAUHWND__@@IIJ@ZXZ 5f82cd3e f   wincore.obj
 0001:0002bd4e       ?_AfxActivationWndProc@@YGJPAUHWND__@@IIJ@Z 5f82cd4e f   wincore.obj
 0001:0002bfc4       ?_AfxGrayBackgroundWndProc@@YGJPAUHWND__@@IIJ@Z 5f82cfc4 f   wincore.obj
 0001:0002c057       ?_AfxCbtFilterHook@@YGJHIJ@Z 5f82d057 f   wincore.obj
 0001:0002c485       ?AfxHookWindowCreate@@YGXPAVCWnd@@@Z 5f82d485 f   wincore.obj
 0001:0002c577       ?AfxUnhookWindowCreate@@YGHXZ 5f82d577 f   wincore.obj
 0001:0002c5a8       ?CreateEx@CWnd@@QAEHKPBG0KABUtagRECT@@PAV1@IPAX@Z 5f82d5a8 f   wincore.obj
 0001:0002c604       ?CreateEx@CWnd@@QAEHKPBG0KHHHHPAUHWND__@@PAUHMENU__@@PAX@Z 5f82d604 f   wincore.obj
 0001:0002c732       ?PreCreateWindow@CWnd@@UAEHAAUtagCREATESTRUCTW@@@Z 5f82d732 f   wincore.obj
 0001:0002c7ab       ?Create@CWnd@@UAEHPBG0KABUtagRECT@@PAV1@IPAUCCreateContext@@@Z 5f82d7ab f   wincore.obj
 0001:0002c857       ??1CWnd@@UAE@XZ            5f82d857 f   wincore.obj
 0001:0002c936       ?OnDestroy@CWnd@@IAEXXZ    5f82d936 f   wincore.obj
 0001:0002c983       ?OnNcDestroy@CWnd@@IAEXXZ  5f82d983 f   wincore.obj
 0001:0002cb4f       ?PostNcDestroy@CWnd@@MAEXXZ 5f82db4f f   wincore.obj
 0001:0002cb5a       ?OnFinalRelease@CWnd@@UAEXXZ 5f82db5a f   wincore.obj
 0001:0002cb89       ?AssertValid@CWnd@@UBEXXZ  5f82db89 f   wincore.obj
 0001:0002cd0b       ?Dump@CWnd@@UBEXAAVCDumpContext@@@Z 5f82dd0b f   wincore.obj
 0001:0002cf68       ?DestroyWindow@CWnd@@UAEHXZ 5f82df68 f   wincore.obj
 0001:0002d061       ?DefWindowProcW@CWnd@@MAEJIIJ@Z 5f82e061 f   wincore.obj
 0001:0002d0ec       ?GetSuperWndProcAddr@CWnd@@MAEPAP6GJPAUHWND__@@IIJ@ZXZ 5f82e0ec f   wincore.obj
 0001:0002d0fd       ?PreTranslateMessage@CWnd@@UAEHPAUtagMSG@@@Z 5f82e0fd f   wincore.obj
 0001:0002d134       ?CancelToolTips@CWnd@@SGXH@Z 5f82e134 f   wincore.obj
 0001:0002d1a8       ?OnToolHitTest@CWnd@@UBEHVCPoint@@PAUtagTOOLINFOW@@@Z 5f82e1a8 f   wincore.obj
 0001:0002d268       ?GetWindowTextW@CWnd@@QBEXAAVCString@@@Z 5f82e268 f   wincore.obj
 0001:0002d306       ?GetDlgItemTextW@CWnd@@QBEHHAAVCString@@@Z 5f82e306 f   wincore.obj
 0001:0002d3d6       ?GetWindowPlacement@CWnd@@QBEHPAUtagWINDOWPLACEMENT@@@Z 5f82e3d6 f   wincore.obj
 0001:0002d42e       ?SetWindowPlacement@CWnd@@QAEHPBUtagWINDOWPLACEMENT@@@Z 5f82e42e f   wincore.obj
 0001:0002d486       ?OnDrawItem@CWnd@@IAEXHPAUtagDRAWITEMSTRUCT@@@Z 5f82e486 f   wincore.obj
 0001:0002d4e1       ?OnCompareItem@CWnd@@IAEHHPAUtagCOMPAREITEMSTRUCT@@@Z 5f82e4e1 f   wincore.obj
 0001:0002d511       ?OnDeleteItem@CWnd@@IAEXHPAUtagDELETEITEMSTRUCT@@@Z 5f82e511 f   wincore.obj
 0001:0002d53a       ?OnCharToItem@CWnd@@IAEHIPAVCListBox@@I@Z 5f82e53a f   wincore.obj
 0001:0002d56c       ?OnVKeyToItem@CWnd@@IAEHIPAVCListBox@@I@Z 5f82e56c f   wincore.obj
 0001:0002d59e       ?TrackPopupMenu@CMenu@@QAEHIHHPAVCWnd@@PBUtagRECT@@@Z 5f82e59e f   wincore.obj
 0001:0002d648       ?_AfxFindPopupMenuFromID@@YGPAVCMenu@@PAV1@I@Z 5f82e648 f   wincore.obj
 0001:0002d6e7       ?OnMeasureItem@CWnd@@IAEXHPAUtagMEASUREITEMSTRUCT@@@Z 5f82e6e7 f   wincore.obj
 0001:0002d7d4       ?AfxRegisterClass@@YGHPAUtagWNDCLASSW@@@Z 5f82e7d4 f   wincore.obj
 0001:0002d953       ?AfxRegisterWndClass@@YGPBGIPAUHICON__@@PAUHBRUSH__@@0@Z 5f82e953 f   wincore.obj
 0001:0002da5e       ?OnNTCtlColor@CWnd@@IAEJIJ@Z 5f82ea5e f   wincore.obj
 0001:0002daf0       ?WinHelpW@CWnd@@UAEXKI@Z   5f82eaf0 f   wincore.obj
 0001:0002dc63       ?_GetBaseMessageMap@CWnd@@KGPBUAFX_MSGMAP@@XZ 5f82ec63 f   wincore.obj
 0001:0002dc6d       ?GetMessageMap@CWnd@@MBEPBUAFX_MSGMAP@@XZ 5f82ec6d f   wincore.obj
 0001:0002dc7d       ?AfxFindMessageEntry@@YGPBUAFX_MSGMAP_ENTRY@@PBU1@III@Z 5f82ec7d f   wincore.obj
 0001:0002dd02       ?AfxResetMsgCache@@YGXXZ   5f82ed02 f   wincore.obj
 0001:0002dd1b       ?WindowProc@CWnd@@MAEJIIJ@Z 5f82ed1b f   wincore.obj
 0001:0002dd73       ?OnWndMsg@CWnd@@MAEHIIJPAJ@Z 5f82ed73 f   wincore.obj
 0001:0002ea1c       ??0CTestCmdUI@@QAE@XZ      5f82fa1c f   wincore.obj
 0001:0002ea45       ?Enable@CTestCmdUI@@UAEXH@Z 5f82fa45 f   wincore.obj
 0001:0002ea65       ?SetCheck@CTestCmdUI@@UAEXH@Z 5f82fa65 f   wincore.obj
 0001:0002ea72       ?SetRadio@CTestCmdUI@@UAEXH@Z 5f82fa72 f   wincore.obj
 0001:0002ea7f       ?SetText@CTestCmdUI@@UAEXPBG@Z 5f82fa7f f   wincore.obj
 0001:0002ea8c       ?OnCommand@CWnd@@MAEHIJ@Z  5f82fa8c f   wincore.obj
 0001:0002ebcd       ?OnNotify@CWnd@@MAEHIJPAJ@Z 5f82fbcd f   wincore.obj
 0001:0002ecdb       ?GetParentFrame@CWnd@@QBEPAVCFrameWnd@@XZ 5f82fcdb f   wincore.obj
 0001:0002ed42       ?AfxGetParentOwner@@YGPAUHWND__@@PAU1@@Z 5f82fd42 f   wincore.obj
 0001:0002eda7       ?GetTopLevelParent@CWnd@@QBEPAV1@XZ 5f82fda7 f   wincore.obj
 0001:0002ee03       ?GetTopLevelOwner@CWnd@@QBEPAV1@XZ 5f82fe03 f   wincore.obj
 0001:0002ee62       ?GetParentOwner@CWnd@@QBEPAV1@XZ 5f82fe62 f   wincore.obj
 0001:0002eed4       ?IsTopParentActive@CWnd@@QBEHXZ 5f82fed4 f   wincore.obj
 0001:0002ef3a       ?ActivateTopParent@CWnd@@QAEXXZ 5f82ff3a f   wincore.obj
 0001:0002ef8e       ?GetTopLevelFrame@CWnd@@QBEPAVCFrameWnd@@XZ 5f82ff8e f   wincore.obj
 0001:0002f003       ?GetSafeOwner@CWnd@@SGPAV1@PAV1@PAPAUHWND__@@@Z 5f830003 f   wincore.obj
 0001:0002f02b       ?MessageBoxW@CWnd@@QAEHPBG0I@Z 5f83002b f   wincore.obj
 0001:0002f069       ?GetDescendantWindow@CWnd@@SGPAV1@PAUHWND__@@HH@Z 5f830069 f   wincore.obj
 0001:0002f12a       ?SendMessageToDescendants@CWnd@@SGXPAUHWND__@@IIJHH@Z 5f83012a f   wincore.obj
 0001:0002f1e2       ?GetScrollBarCtrl@CWnd@@UBEPAVCScrollBar@@H@Z 5f8301e2 f   wincore.obj
 0001:0002f1f1       ?SetScrollPos@CWnd@@QAEHHHH@Z 5f8301f1 f   wincore.obj
 0001:0002f243       ?GetScrollPos@CWnd@@QBEHH@Z 5f830243 f   wincore.obj
 0001:0002f285       ?SetScrollRange@CWnd@@QAEXHHHH@Z 5f830285 f   wincore.obj
 0001:0002f2df       ?GetScrollRange@CWnd@@QBEXHPAH0@Z 5f8302df f   wincore.obj
 0001:0002f331       ?EnableScrollBarCtrl@CWnd@@QAEXHH@Z 5f830331 f   wincore.obj
 0001:0002f39a       ?SetScrollInfo@CWnd@@QAEHHPAUtagSCROLLINFO@@H@Z 5f83039a f   wincore.obj
 0001:0002f43a       ?GetScrollInfo@CWnd@@QAEHHPAUtagSCROLLINFO@@I@Z 5f83043a f   wincore.obj
 0001:0002f4da       ?GetScrollLimit@CWnd@@QAEHH@Z 5f8304da f   wincore.obj
 0001:0002f53b       ?ScrollWindow@CWnd@@QAEXHHPBUtagRECT@@0@Z 5f83053b f   wincore.obj
 0001:0002f651       ?RepositionBars@CWnd@@QAEXIIIIPAUtagRECT@@PBU2@H@Z 5f830651 f   wincore.obj
 0001:0002f89b       ?AfxRepositionWindow@@YGXPAUAFX_SIZEPARENTPARAMS@@PAUHWND__@@PBUtagRECT@@@Z 5f83089b f   wincore.obj
 0001:0002fa02       ?CalcWindowRect@CWnd@@UAEXPAUtagRECT@@I@Z 5f830a02 f   wincore.obj
 0001:0002fa44       ?HandleFloatingSysCommand@CWnd@@QAEHIJ@Z 5f830a44 f   wincore.obj
 0001:0002fc11       ?WalkPreTranslateTree@CWnd@@SGHPAUHWND__@@PAUtagMSG@@@Z 5f830c11 f   wincore.obj
 0001:0002fccb       ?SendChildNotifyLastMsg@CWnd@@QAEHPAJ@Z 5f830ccb f   wincore.obj
 0001:0002fd0e       ?ReflectLastMsg@CWnd@@KGHPAUHWND__@@PAJ@Z 5f830d0e f   wincore.obj
 0001:0002fe53       ?OnChildNotify@CWnd@@MAEHIIJPAJ@Z 5f830e53 f   wincore.obj
 0001:0002fed0       ?ReflectChildNotify@CWnd@@IAEHIIJPAJ@Z 5f830ed0 f   wincore.obj
 0001:000300c8       ?OnParentNotify@CWnd@@IAEXIJ@Z 5f8310c8 f   wincore.obj
 0001:00030109       ?OnActivateTopLevel@CWnd@@IAEJIJ@Z 5f831109 f   wincore.obj
 0001:00030148       ?OnSysColorChange@CWnd@@IAEXXZ 5f831148 f   wincore.obj
 0001:000301e3       ?OnSettingChange@CWnd@@IAEXIPBG@Z 5f8311e3 f   wincore.obj
 0001:00030248       ?OnWinIniChange@CWnd@@IAEXPBG@Z 5f831248 f   wincore.obj
 0001:000302a3       ?OnDevModeChange@CWnd@@IAEXPAG@Z 5f8312a3 f   wincore.obj
 0001:00030311       ?OnHelpInfo@CWnd@@IAEHPAUtagHELPINFO@@@Z 5f831311 f   wincore.obj
 0001:0003038f       ?OnDisplayChange@CWnd@@IAEJIJ@Z 5f83138f f   wincore.obj
 0001:000303f4       ?OnDragList@CWnd@@IAEJIJ@Z 5f8313f4 f   wincore.obj
 0001:00030450       ?OnHScroll@CWnd@@IAEXIIPAVCScrollBar@@@Z 5f831450 f   wincore.obj
 0001:0003047b       ?OnVScroll@CWnd@@IAEXIIPAVCScrollBar@@@Z 5f83147b f   wincore.obj
 0001:000304a6       ?OnEnterIdle@CWnd@@IAEXIPAV1@@Z 5f8314a6 f   wincore.obj
 0001:000304e5       ?OnCtlColor@CWnd@@IAEPAUHBRUSH__@@PAVCDC@@PAV1@I@Z 5f8314e5 f   wincore.obj
 0001:00030540       ?OnGrayCtlColor@CWnd@@QAEPAUHBRUSH__@@PAVCDC@@PAV1@I@Z 5f831540 f   wincore.obj
 0001:000305ac       ?GrayCtlColor@CWnd@@SGHPAUHDC__@@PAUHWND__@@IPAUHBRUSH__@@K@Z 5f8315ac f   wincore.obj
 0001:00030672       ?OnQuery3dControls@CWnd@@IAEJIJ@Z 5f831672 f   wincore.obj
 0001:00030684       ?UpdateData@CWnd@@QAEHH@Z  5f831684 f   wincore.obj
 0001:00030843       ??0CDataExchange@@QAE@PAVCWnd@@H@Z 5f831843 f   wincore.obj
 0001:00030881       ?CenterWindow@CWnd@@QAEXPAV1@@Z 5f831881 f   wincore.obj
 0001:00030b69       ?CheckAutoCenter@CWnd@@UAEHXZ 5f831b69 f   wincore.obj
 0001:00030b79       ?ExecuteDlgInit@CWnd@@QAEHPBG@Z 5f831b79 f   wincore.obj
 0001:00030c48       ?ExecuteDlgInit@CWnd@@QAEHPAX@Z 5f831c48 f   wincore.obj
 0001:00030f4d       ?UpdateDialogControls@CWnd@@QAEXPAVCCmdTarget@@H@Z 5f831f4d f   wincore.obj
 0001:000310c6       ?PreTranslateInput@CWnd@@QAEHPAUtagMSG@@@Z 5f8320c6 f   wincore.obj
 0001:00031144       ?RunModalLoop@CWnd@@QAEHK@Z 5f832144 f   wincore.obj
 0001:0003140a       ?ContinueModal@CWnd@@UAEHXZ 5f83240a f   wincore.obj
 0001:0003141e       ?EndModalLoop@CWnd@@UAEXH@Z 5f83241e f   wincore.obj
 0001:0003148f       ?SetOccDialogInfo@CWnd@@MAEHPAU_AFX_OCC_DIALOG_INFO@@@Z 5f83248f f   wincore.obj
 0001:000314c7       ?_AfxRegisterWithIcon@@YGHPAUtagWNDCLASSW@@PBGI@Z 5f8324c7 f   wincore.obj
 0001:0003152c       ?_AfxInitCommonControls@@YGJPAUtagINITCOMMONCONTROLSEX@@J@Z 5f83252c f   wincore.obj
 0001:000315da       ?AfxEndDeferRegisterClass@@YGHJ@Z 5f8325da f   wincore.obj
 0001:000319a9       ?IsFrameWnd@CWnd@@UBEHXZ   5f8329a9 f   wincore.obj
 0001:000319b6       ?IsFrameWnd@CFrameWnd@@UBEHXZ 5f8329b6 f   wincore.obj
 0001:000319c6       ?IsTracking@CFrameWnd@@QBEHXZ 5f8329c6 f   wincore.obj
 0001:00031a10       ?SubclassCtl3d@CWnd@@QAEHH@Z 5f832a10 f   wincore.obj
 0001:00031acd       ?SubclassDlg3d@CWnd@@QAEHK@Z 5f832acd f   wincore.obj
 0001:00031b6a       ?DragAcceptFiles@CWnd@@QAEXH@Z 5f832b6a f   wincore.obj
 0001:00031bb9       ?SubclassWindow@CWnd@@QAEHPAUHWND__@@@Z 5f832bb9 f   wincore.obj
 0001:00031ce7       ?SubclassDlgItem@CWnd@@QAEHIPAV1@@Z 5f832ce7 f   wincore.obj
 0001:00031e17       ?UnsubclassWindow@CWnd@@QAEPAUHWND__@@XZ 5f832e17 f   wincore.obj
 0001:00031e90       ?AfxLockTempMaps@@YGXXZ    5f832e90 f   winhand.obj
 0001:00031eaf       ?AfxUnlockTempMaps@@YGHH@Z 5f832eaf f   winhand.obj
 0001:00032071       ??0CHandleMap@@QAE@PAUCRuntimeClass@@IH@Z 5f833071 f   winhand.obj
 0001:00032139       ?FromHandle@CHandleMap@@QAEPAVCObject@@PAX@Z 5f833139 f   winhand.obj
 0001:00032363       ?SetPermanent@CHandleMap@@QAEXPAXPAVCObject@@@Z 5f833363 f   winhand.obj
 0001:00032396       ?RemoveHandle@CHandleMap@@QAEXPAX@Z 5f833396 f   winhand.obj
 0001:00032477       ?DeleteTemp@CHandleMap@@QAEXXZ 5f833477 f   winhand.obj
 0001:000325ad       ?DeleteTempMap@CWnd@@SGXXZ 5f8335ad f   winhand.obj
 0001:000325c8       ?DeleteTempMap@CImageList@@SGXXZ 5f8335c8 f   winhand.obj
 0001:000325e3       ?DeleteTempMap@CDC@@SGXXZ  5f8335e3 f   winhand.obj
 0001:000325fe       ?DeleteTempMap@CGdiObject@@SGXXZ 5f8335fe f   winhand.obj
 0001:00032619       ?DeleteTempMap@CMenu@@SGXXZ 5f833619 f   winhand.obj
 0001:00032640       ?AfxWinMain@@YGHPAUHINSTANCE__@@0PAGH@Z 5f833640 f   winmain.obj
 0001:00032760       ?AfxDlgProc@@YGHPAUHWND__@@IIJ@Z 5f833760 f   dlgcore.obj
 0001:000327ac       ?_GetBaseMessageMap@CDialog@@KGPBUAFX_MSGMAP@@XZ 5f8337ac f   dlgcore.obj
 0001:000327b6       ?GetMessageMap@CDialog@@MBEPBUAFX_MSGMAP@@XZ 5f8337b6 f   dlgcore.obj
 0001:000327c6       ?PreTranslateMessage@CDialog@@UAEHPAUtagMSG@@@Z 5f8337c6 f   dlgcore.obj
 0001:000328c7       ?OnCmdMsg@CDialog@@UAEHIHPAXPAUAFX_CMDHANDLERINFO@@@Z 5f8338c7 f   dlgcore.obj
 0001:00032a1c       ??0CDialog@@QAE@XZ         5f833a1c f   dlgcore.obj
 0001:00032aa4       ??1CDialog@@UAE@XZ         5f833aa4 f   dlgcore.obj
 0001:00032b22       ?Create@CDialog@@QAEHPBGPAVCWnd@@@Z 5f833b22 f   dlgcore.obj
 0001:00032c46       ?CreateIndirect@CDialog@@QAEHPAXPAVCWnd@@@Z 5f833c46 f   dlgcore.obj
 0001:00032c65       ?CreateIndirect@CDialog@@IAEHPAXPAVCWnd@@PAUHINSTANCE__@@@Z 5f833c65 f   dlgcore.obj
 0001:00032ccc       ?CreateIndirect@CDialog@@QAEHPBUDLGTEMPLATE@@PAVCWnd@@PAX@Z 5f833ccc f   dlgcore.obj
 0001:00032cef       ?CreateIndirect@CDialog@@IAEHPBUDLGTEMPLATE@@PAVCWnd@@PAXPAUHINSTANCE__@@@Z 5f833cef f   dlgcore.obj
 0001:00032d4d       ?CreateDlg@CWnd@@IAEHPBGPAV1@@Z 5f833d4d f   dlgcore.obj
 0001:00032e02       ?CreateDlgIndirect@CWnd@@IAEHPBUDLGTEMPLATE@@PAV1@@Z 5f833e02 f   dlgcore.obj
 0001:00032e21       ?CreateDlgIndirect@CWnd@@IAEHPBUDLGTEMPLATE@@PAV1@PAUHINSTANCE__@@@Z 5f833e21 f   dlgcore.obj
 0001:00033252       ?SetOccDialogInfo@CDialog@@MAEHPAU_AFX_OCC_DIALOG_INFO@@@Z 5f834252 f   dlgcore.obj
 0001:0003326d       ??0CDialog@@QAE@PBGPAVCWnd@@@Z 5f83426d f   dlgcore.obj
 0001:0003334d       ??0CDialog@@QAE@IPAVCWnd@@@Z 5f83434d f   dlgcore.obj
 0001:000333a2       ?InitModalIndirect@CDialog@@QAEHPAXPAVCWnd@@@Z 5f8343a2 f   dlgcore.obj
 0001:0003343b       ?InitModalIndirect@CDialog@@QAEHPBUDLGTEMPLATE@@PAVCWnd@@PAX@Z 5f83443b f   dlgcore.obj
 0001:000334dd       ?PreModal@CDialog@@IAEPAUHWND__@@XZ 5f8344dd f   dlgcore.obj
 0001:00033552       ?PostModal@CDialog@@IAEXXZ 5f834552 f   dlgcore.obj
 0001:000335ae       ?DoModal@CDialog@@UAEHXZ   5f8345ae f   dlgcore.obj
 0001:00033866       ?EndDialog@CDialog@@QAEXH@Z 5f834866 f   dlgcore.obj
 0001:000338d1       ?HandleSetFont@CDialog@@IAEJIJ@Z 5f8348d1 f   dlgcore.obj
 0001:000338fe       ?PreInitDialog@CDialog@@MAEXXZ 5f8348fe f   dlgcore.obj
 0001:00033909       ?HandleInitDialog@CDialog@@IAEJIJ@Z 5f834909 f   dlgcore.obj
 0001:000339fc       ?AfxHelpEnabled@@YGHXZ     5f8349fc f   dlgcore.obj
 0001:00033a64       ?OnSetFont@CDialog@@UAEXPAVCFont@@@Z 5f834a64 f   dlgcore.obj
 0001:00033a71       ?OnInitDialog@CDialog@@UAEHXZ 5f834a71 f   dlgcore.obj
 0001:00033b31       ?OnOK@CDialog@@MAEXXZ      5f834b31 f   dlgcore.obj
 0001:00033b68       ?OnCancel@CDialog@@MAEXXZ  5f834b68 f   dlgcore.obj
 0001:00033b7d       ?CheckAutoCenter@CDialog@@UAEHXZ 5f834b7d f   dlgcore.obj
 0001:00033cb4       ?OnCtlColor@CDialog@@IAEPAUHBRUSH__@@PAVCDC@@PAVCWnd@@I@Z 5f834cb4 f   dlgcore.obj
 0001:00033cd5       ?OnCommandHelp@CDialog@@IAEJIJ@Z 5f834cd5 f   dlgcore.obj
 0001:00033d33       ?OnHelpHitTest@CDialog@@IAEJIJ@Z 5f834d33 f   dlgcore.obj
 0001:00033d58       ?AssertValid@CDialog@@UBEXXZ 5f834d58 f   dlgcore.obj
 0001:00033d6b       ?Dump@CDialog@@UBEXAAVCDumpContext@@@Z 5f834d6b f   dlgcore.obj
 0001:00033e46       ?_AfxCheckDialogTemplate@@YGHPBGH@Z 5f834e46 f   dlgcore.obj
 0001:00034020       ?_AfxConvertDialogUnitsToPixels@@YGXPBGGHHPAUtagSIZE@@@Z 5f835020 f   dlgtempl.obj
 0001:0003416c       ??0CDialogTemplate@@QAE@PBUDLGTEMPLATE@@@Z 5f83516c f   dlgtempl.obj
 0001:000341ba       ??0CDialogTemplate@@QAE@PAX@Z 5f8351ba f   dlgtempl.obj
 0001:00034221       ?SetTemplate@CDialogTemplate@@IAEHPBUDLGTEMPLATE@@I@Z 5f835221 f   dlgtempl.obj
 0001:000342aa       ??1CDialogTemplate@@QAE@XZ 5f8352aa f   dlgtempl.obj
 0001:000342c9       ?Load@CDialogTemplate@@QAEHPBG@Z 5f8352c9 f   dlgtempl.obj
 0001:0003435e       ?Detach@CDialogTemplate@@QAEPAXXZ 5f83535e f   dlgtempl.obj
 0001:0003437f       ?HasFont@CDialogTemplate@@QBEHXZ 5f83537f f   dlgtempl.obj
 0001:000343b9       ?GetFontSizeField@CDialogTemplate@@KAPAEPBUDLGTEMPLATE@@@Z 5f8353b9 f   dlgtempl.obj
 0001:0003446a       ?GetTemplateSize@CDialogTemplate@@KAIPBUDLGTEMPLATE@@@Z 5f83546a f   dlgtempl.obj
 0001:000345ac       ?GetFont@CDialogTemplate@@SAHPBUDLGTEMPLATE@@AAVCString@@AAG@Z 5f8355ac f   dlgtempl.obj
 0001:00034637       ?GetFont@CDialogTemplate@@QBEHAAVCString@@AAG@Z 5f835637 f   dlgtempl.obj
 0001:000346a3       ?SetFont@CDialogTemplate@@QAEHPBGG@Z 5f8356a3 f   dlgtempl.obj
 0001:0003486d       ?SetSystemFont@CDialogTemplate@@QAEHG@Z 5f83586d f   dlgtempl.obj
 0001:0003492d       ?GetSizeInDialogUnits@CDialogTemplate@@QBEXPAUtagSIZE@@@Z 5f83592d f   dlgtempl.obj
 0001:000349f4       ?GetSizeInPixels@CDialogTemplate@@QBEXPAUtagSIZE@@@Z 5f8359f4 f   dlgtempl.obj
 0001:00034b40       ?IsDialogEx@@YAHPBUDLGTEMPLATE@@@Z 5f835b40 f i dlgtempl.obj
 0001:00034b60       ?HasFont@@YAHPBUDLGTEMPLATE@@@Z 5f835b60 f i dlgtempl.obj
 0001:00034ba0       ?FontAttrSize@@YAHH@Z      5f835ba0 f i dlgtempl.obj
 0001:00034bc0       ?_SkipString@@YAPAGPAG@Z   5f835bc0 f i dlgtempl.obj
 0001:00034be0       ?LoadStringW@CString@@QAEHI@Z 5f835be0 f   winstr.obj
 0001:00034ca0       ?AfxExtractSubString@@YGHAAVCString@@PBGHG@Z 5f835ca0 f   winstr.obj
 0001:00034d80       ?afxMapHMENU@@YGPAVCHandleMap@@H@Z 5f835d80 f   winmenu.obj
 0001:00034e49       ?FromHandle@CMenu@@SGPAV1@PAUHMENU__@@@Z 5f835e49 f   winmenu.obj
 0001:00034ebc       ?FromHandlePermanent@CMenu@@SGPAV1@PAUHMENU__@@@Z 5f835ebc f   winmenu.obj
 0001:00034f1f       ?AssertValid@CMenu@@UBEXXZ 5f835f1f f   winmenu.obj
 0001:00034f69       ?Dump@CMenu@@UBEXAAVCDumpContext@@@Z 5f835f69 f   winmenu.obj
 0001:00034faa       ?Attach@CMenu@@QAEHPAUHMENU__@@@Z 5f835faa f   winmenu.obj
 0001:0003502e       ?Detach@CMenu@@QAEPAUHMENU__@@XZ 5f83602e f   winmenu.obj
 0001:00035076       ?DestroyMenu@CMenu@@QAEHXZ 5f836076 f   winmenu.obj
 0001:0003509d       ?DrawItem@CMenu@@UAEXPAUtagDRAWITEMSTRUCT@@@Z 5f83609d f   winmenu.obj
 0001:000350aa       ?MeasureItem@CMenu@@UAEXPAUtagMEASUREITEMSTRUCT@@@Z 5f8360aa f   winmenu.obj
 0001:000350c0       ?UpdateSysColors@AUX_DATA@@QAEXXZ 5f8360c0 f   auxdata.obj
 0001:00035173       ?UpdateSysMetrics@AUX_DATA@@QAEXXZ 5f836173 f   auxdata.obj
 0001:00035220       ?OnAmbientProperty@CWnd@@UAEHPAVCOleControlSite@@JPAUtagVARIANT@@@Z 5f836220 f   winocc.obj
 0001:00035270       ?GetControlUnknown@CWnd@@QAEPAUIUnknown@@XZ 5f836270 f   winocc.obj
 0001:00035291       ?CheckDlgButton@CWnd@@QAEXHI@Z 5f836291 f   winocc.obj
 0001:00035305       ?CheckRadioButton@CWnd@@QAEXHHH@Z 5f836305 f   winocc.obj
 0001:00035381       ?GetDlgItem@CWnd@@QBEPAV1@H@Z 5f836381 f   winocc.obj
 0001:000353f3       ?GetDlgItem@CWnd@@QBEXHPAPAUHWND__@@@Z 5f8363f3 f   winocc.obj
 0001:00035485       ?GetDlgItemInt@CWnd@@QBEIHPAHH@Z 5f836485 f   winocc.obj
 0001:00035501       ?GetDlgItemTextW@CWnd@@QBEHHPAGH@Z 5f836501 f   winocc.obj
 0001:00035580       ?SendDlgItemMessageW@CWnd@@QAEJHIIJ@Z 5f836580 f   winocc.obj
 0001:00035607       ?SetDlgItemInt@CWnd@@QAEXHIH@Z 5f836607 f   winocc.obj
 0001:00035689       ?SetDlgItemTextW@CWnd@@QAEXHPBG@Z 5f836689 f   winocc.obj
 0001:00035703       ?IsDlgButtonChecked@CWnd@@QBEIH@Z 5f836703 f   winocc.obj
 0001:00035775       ?ScrollWindowEx@CWnd@@QAEHHHPBUtagRECT@@0PAVCRgn@@PAU2@I@Z 5f836775 f   winocc.obj
 0001:0003581a       ?IsDialogMessageW@CWnd@@QAEHPAUtagMSG@@@Z 5f83681a f   winocc.obj
 0001:0003589e       ?GetStyle@CWnd@@QBEKXZ     5f83689e f   winocc.obj
 0001:00035905       ?GetExStyle@CWnd@@QBEKXZ   5f836905 f   winocc.obj
 0001:0003596c       ?ModifyStyle@CWnd@@QAEHKKI@Z 5f83696c f   winocc.obj
 0001:000359ed       ?ModifyStyleEx@CWnd@@QAEHKKI@Z 5f8369ed f   winocc.obj
 0001:00035a6e       ?SetWindowTextW@CWnd@@QAEXPBG@Z 5f836a6e f   winocc.obj
 0001:00035ae0       ?GetWindowTextW@CWnd@@QBEHPAGH@Z 5f836ae0 f   winocc.obj
 0001:00035b5a       ?GetWindowTextLengthW@CWnd@@QBEHXZ 5f836b5a f   winocc.obj
 0001:00035bc2       ?GetDlgCtrlID@CWnd@@QBEHXZ 5f836bc2 f   winocc.obj
 0001:00035c2a       ?SetDlgCtrlID@CWnd@@QAEHH@Z 5f836c2a f   winocc.obj
 0001:00035c9e       ?MoveWindow@CWnd@@QAEXHHHHH@Z 5f836c9e f   winocc.obj
 0001:00035d30       ?SetWindowPos@CWnd@@QAEHPBV1@HHHHI@Z 5f836d30 f   winocc.obj
 0001:00035dcf       ?ShowWindow@CWnd@@QAEHH@Z  5f836dcf f   winocc.obj
 0001:00035e41       ?IsWindowEnabled@CWnd@@QBEHXZ 5f836e41 f   winocc.obj
 0001:00035ea9       ?EnableWindow@CWnd@@QAEHH@Z 5f836ea9 f   winocc.obj
 0001:00035f1b       ?SetFocus@CWnd@@QAEPAV1@XZ 5f836f1b f   winocc.obj
 0001:00035f89       ?InvokeHelper@CWnd@@QAAXJGGPAXPBEZZ 5f836f89 f   winocc.obj
 0001:00035ffd       ?GetProperty@CWnd@@QBEXJGPAX@Z 5f836ffd f   winocc.obj
 0001:0003605b       ?SetProperty@CWnd@@QAAXJGZZ 5f83705b f   winocc.obj
 0001:000360c2       ?GetDSCCursor@CWnd@@QAEPAUIUnknown@@XZ 5f8370c2 f   winocc.obj
 0001:0003615b       ?BindDefaultProperty@CWnd@@QAEXJGPBGPAV1@@Z 5f83715b f   winocc.obj
 0001:000361b6       ?BindProperty@CWnd@@QAEXJPAV1@@Z 5f8371b6 f   winocc.obj
 0001:00036208       ?AttachControlSite@CWnd@@IAEXPAVCHandleMap@@@Z 5f837208 f   winocc.obj
 0001:0003625d       ?AttachControlSite@CWnd@@QAEXPAV1@@Z 5f83725d f   winocc.obj
 0001:000362d1       ?AttachControlSite@COleControlContainer@@QAEXPAVCWnd@@@Z 5f8372d1 f   winocc.obj
 0001:00036380       ??0CCmdTarget@@QAE@XZ      5f837380 f   cmdtarg.obj
 0001:00036439       ??1CCmdTarget@@UAE@XZ      5f837439 f   cmdtarg.obj
 0001:000364ca       ?_AfxDispatchCmdMsg@@YGHPAVCCmdTarget@@IHP81@AEXXZPAXIPAUAFX_CMDHANDLERINFO@@@Z 5f8374ca f   cmdtarg.obj
 0001:00036a27       ?OnCmdMsg@CCmdTarget@@UAEHIHPAXPAUAFX_CMDHANDLERINFO@@@Z 5f837a27 f   cmdtarg.obj
 0001:00036cad       ?IsInvokeAllowed@CCmdTarget@@UAEHJ@Z 5f837cad f   cmdtarg.obj
 0001:00036cbf       ?GetDispatchIID@CCmdTarget@@UAEHPAU_GUID@@@Z 5f837cbf f   cmdtarg.obj
 0001:00036cce       ?GetTypeInfoCount@CCmdTarget@@UAEIXZ 5f837cce f   cmdtarg.obj
 0001:00036cdb       ?GetTypeLibCache@CCmdTarget@@UAEPAVCTypeLibCache@@XZ 5f837cdb f   cmdtarg.obj
 0001:00036ce8       ?GetTypeLib@CCmdTarget@@UAEJKPAPAUITypeLib@@@Z 5f837ce8 f   cmdtarg.obj
 0001:00036cfa       ?BeginWaitCursor@CCmdTarget@@QAEXXZ 5f837cfa f   cmdtarg.obj
 0001:00036d1f       ?EndWaitCursor@CCmdTarget@@QAEXXZ 5f837d1f f   cmdtarg.obj
 0001:00036d44       ?RestoreWaitCursor@CCmdTarget@@QAEXXZ 5f837d44 f   cmdtarg.obj
 0001:00036d69       ?_GetBaseMessageMap@CCmdTarget@@KGPBUAFX_MSGMAP@@XZ 5f837d69 f   cmdtarg.obj
 0001:00036d70       ?GetMessageMap@CCmdTarget@@MBEPBUAFX_MSGMAP@@XZ 5f837d70 f   cmdtarg.obj
 0001:00036d80       ?_GetBaseDispatchMap@CCmdTarget@@KGPBUAFX_DISPMAP@@XZ 5f837d80 f   cmdtarg.obj
 0001:00036d87       ?GetDispatchMap@CCmdTarget@@MBEPBUAFX_DISPMAP@@XZ 5f837d87 f   cmdtarg.obj
 0001:00036d97       ?_GetBaseEventSinkMap@CCmdTarget@@KGPBUAFX_EVENTSINKMAP@@XZ 5f837d97 f   cmdtarg.obj
 0001:00036d9e       ?GetEventSinkMap@CCmdTarget@@MBEPBUAFX_EVENTSINKMAP@@XZ 5f837d9e f   cmdtarg.obj
 0001:00036dae       ?_GetBaseInterfaceMap@CCmdTarget@@KGPBUAFX_INTERFACEMAP@@XZ 5f837dae f   cmdtarg.obj
 0001:00036db5       ?GetInterfaceMap@CCmdTarget@@MBEPBUAFX_INTERFACEMAP@@XZ 5f837db5 f   cmdtarg.obj
 0001:00036dc5       ?OnFinalRelease@CCmdTarget@@UAEXXZ 5f837dc5 f   cmdtarg.obj
 0001:00036e27       ?OnCreateAggregates@CCmdTarget@@UAEHXZ 5f837e27 f   cmdtarg.obj
 0001:00036e37       ?GetInterfaceHook@CCmdTarget@@UAEPAUIUnknown@@PBX@Z 5f837e37 f   cmdtarg.obj
 0001:00036e46       ?_GetBaseConnectionMap@CCmdTarget@@KGPBUAFX_CONNECTIONMAP@@XZ 5f837e46 f   cmdtarg.obj
 0001:00036e4d       ?GetConnectionMap@CCmdTarget@@MBEPBUAFX_CONNECTIONMAP@@XZ 5f837e4d f   cmdtarg.obj
 0001:00036e5d       ?GetConnectionHook@CCmdTarget@@MAEPAUIConnectionPoint@@ABU_GUID@@@Z 5f837e5d f   cmdtarg.obj
 0001:00036e6c       ?GetExtraConnectionPoints@CCmdTarget@@MAEHPAVCPtrArray@@@Z 5f837e6c f   cmdtarg.obj
 0001:00036e7b       ?_GetBaseCommandMap@CCmdTarget@@KGPBUAFX_OLECMDMAP@@XZ 5f837e7b f   cmdtarg.obj
 0001:00036e82       ?GetCommandMap@CCmdTarget@@MBEPBUAFX_OLECMDMAP@@XZ 5f837e82 f   cmdtarg.obj
 0001:00036e92       ?GetRoutingView@CCmdTarget@@IAEPAVCView@@XZ 5f837e92 f   cmdtarg.obj
 0001:00036ea2       ?GetRoutingFrame@CCmdTarget@@IAEPAVCFrameWnd@@XZ 5f837ea2 f   cmdtarg.obj
 0001:00036eb2       ??0CCmdUI@@QAE@XZ          5f837eb2 f   cmdtarg.obj
 0001:00036f23       ?Enable@CCmdUI@@UAEXH@Z    5f837f23 f   cmdtarg.obj
 0001:0003700e       ?SetCheck@CCmdUI@@UAEXH@Z  5f83800e f   cmdtarg.obj
 0001:000370d8       ?SetRadio@CCmdUI@@UAEXH@Z  5f8380d8 f   cmdtarg.obj
 0001:00037177       ?SetText@CCmdUI@@UAEXPBG@Z 5f838177 f   cmdtarg.obj
 0001:000372b8       ?DoUpdate@CCmdUI@@QAEHPAVCCmdTarget@@H@Z 5f8382b8 f   cmdtarg.obj
 0001:000373c0       ?_AfxThreadEntry@@YGIPAX@Z 5f8383c0 f   thrdcore.obj
 0001:00037728       ?AfxGetThread@@YGPAVCWinThread@@XZ 5f838728 f   thrdcore.obj
 0001:00037754       ?AfxBeginThread@@YGPAVCWinThread@@P6AIPAX@Z0HIKPAU_SECURITY_ATTRIBUTES@@@Z 5f838754 f   thrdcore.obj
 0001:00037893       ?AfxBeginThread@@YGPAVCWinThread@@PAUCRuntimeClass@@HIKPAU_SECURITY_ATTRIBUTES@@@Z 5f838893 f   thrdcore.obj
 0001:000379ab       ?AfxEndThread@@YGXIH@Z     5f8389ab f   thrdcore.obj
 0001:00037a50       ?AfxInitThread@@YGXXZ      5f838a50 f   thrdcore.obj
 0001:00037ae4       ?AfxTermThread@@YGXPAUHINSTANCE__@@@Z 5f838ae4 f   thrdcore.obj
 0001:00037bb1       ?CreateThread@CWinThread@@QAEHKIPAU_SECURITY_ATTRIBUTES@@@Z 5f838bb1 f   thrdcore.obj
 0001:00037daa       ?Delete@CWinThread@@UAEXXZ 5f838daa f   thrdcore.obj
 0001:00037deb       ?InitInstance@CWinThread@@UAEHXZ 5f838deb f   thrdcore.obj
 0001:00037e0b       ?Run@CWinThread@@UAEHXZ    5f838e0b f   thrdcore.obj
 0001:00037f0a       ?IsIdleMessage@CWinThread@@UAEHPAUtagMSG@@@Z 5f838f0a f   thrdcore.obj
 0001:00037fba       ?ExitInstance@CWinThread@@UAEHXZ 5f838fba f   thrdcore.obj
 0001:00038010       ?OnIdle@CWinThread@@UAEHJ@Z 5f839010 f   thrdcore.obj
 0001:0003821a       ?DispatchThreadMessage@CWinThread@@IAEXPAUtagMSG@@@Z 5f83921a f   thrdcore.obj
 0001:00038233       ?DispatchThreadMessageEx@CWinThread@@IAEHPAUtagMSG@@@Z 5f839233 f   thrdcore.obj
 0001:0003835e       ?PreTranslateMessage@CWinThread@@UAEHPAUtagMSG@@@Z 5f83935e f   thrdcore.obj
 0001:000383fb       ?ProcessWndProcException@CWinThread@@UAEJPAVCException@@PBUtagMSG@@@Z 5f8393fb f   thrdcore.obj
 0001:00038433       ?_AfxMsgFilterHook@@YGJHIJ@Z 5f839433 f   thrdcore.obj
 0001:000384c3       ?IsHelpKey@@YGHPAUtagMSG@@@Z 5f8394c3 f   thrdcore.obj
 0001:0003853e       ?ProcessMessageFilter@CWinThread@@UAEHHPAUtagMSG@@@Z 5f83953e f   thrdcore.obj
 0001:00038706       ?GetMainWnd@CWinThread@@UAEPAVCWnd@@XZ 5f839706 f   thrdcore.obj
 0001:00038738       ?PumpMessage@CWinThread@@UAEHXZ 5f839738 f   thrdcore.obj
 0001:00038844       ?AssertValid@CWinThread@@UBEXXZ 5f839844 f   thrdcore.obj
 0001:00038857       ?Dump@CWinThread@@UBEXAAVCDumpContext@@@Z 5f839857 f   thrdcore.obj
 0001:00038aa0       ?IsEnterKey@@YAHPAUtagMSG@@@Z 5f839aa0 f i thrdcore.obj
 0001:00038ad0       ?IsButtonUp@@YAHPAUtagMSG@@@Z 5f839ad0 f i thrdcore.obj
 0001:00038af0       ?_GetBaseMessageMap@CWinApp@@KGPBUAFX_MSGMAP@@XZ 5f839af0 f   appcore.obj
 0001:00038afa       ?GetMessageMap@CWinApp@@MBEPBUAFX_MSGMAP@@XZ 5f839afa f   appcore.obj
 0001:00038b0a       ?Run@CWinApp@@UAEHXZ       5f839b0a f   appcore.obj
 0001:00038b48       ?WinHelpW@CWinApp@@UAEXKI@Z 5f839b48 f   appcore.obj
 0001:00038ba3       ?ProcessWndProcException@CWinApp@@UAEJPAVCException@@PBUtagMSG@@@Z 5f839ba3 f   appcore.obj
 0001:00038c58       ?OnIdle@CWinApp@@UAEHJ@Z   5f839c58 f   appcore.obj
 0001:00038d4a       ?DevModeChange@CWinApp@@QAEXPAG@Z 5f839d4a f   appcore.obj
 0001:00038e99       ?AssertValid@CWinApp@@UBEXXZ 5f839e99 f   appcore.obj
 0001:00038f34       ?Dump@CWinApp@@UBEXAAVCDumpContext@@@Z 5f839f34 f   appcore.obj
 0001:000392a0       ?_AfxAbbreviateName@@YGXPAGHH@Z 5f83a2a0 f   filelist.obj
 0001:00039504       ??0CRecentFileList@@QAE@IPBG0HH@Z 5f83a504 f   filelist.obj
 0001:00039643       ??1CRecentFileList@@UAE@XZ 5f83a643 f   filelist.obj
 0001:000396da       ?Add@CRecentFileList@@UAEXPBG@Z 5f83a6da f   filelist.obj
 0001:0003987c       ?Remove@CRecentFileList@@UAEXH@Z 5f83a87c f   filelist.obj
 0001:0003995d       ?GetDisplayName@CRecentFileList@@QBEHAAVCString@@HPBGHH@Z 5f83a95d f   filelist.obj
 0001:00039b59       ?UpdateMenu@CRecentFileList@@UAEXPAVCCmdUI@@@Z 5f83ab59 f   filelist.obj
 0001:00039fdc       ?WriteList@CRecentFileList@@UAEXXZ 5f83afdc f   filelist.obj
 0001:0003a135       ?ReadList@CRecentFileList@@UAEXXZ 5f83b135 f   filelist.obj
 0001:0003a2b0       ??_GCRecentFileList@@UAEPAXI@Z 5f83b2b0 f i filelist.obj
 0001:0003a2b0       ??_ECRecentFileList@@UAEPAXI@Z 5f83b2b0 f i filelist.obj
 0001:0003a2e0       ??_ECString@@QAEPAXI@Z     5f83b2e0 f i filelist.obj
 0001:0003a350       ??6@YGAAVCArchive@@AAV0@ABVCString@@@Z 5f83b350 f   arccore.obj
 0001:0003a41a       ?_AfxReadStringLength@@YGIAAVCArchive@@@Z 5f83b41a f   arccore.obj
 0001:0003a497       ??5@YGAAVCArchive@@AAV0@AAVCString@@@Z 5f83b497 f   arccore.obj
 0001:0003a5b6       ?SerializeElements@@YGXAAVCArchive@@PAVCString@@H@Z 5f83b5b6 f   arccore.obj
 0001:0003a65b       ?Load@CRuntimeClass@@SGPAU1@AAVCArchive@@PAI@Z 5f83b65b f   arccore.obj
 0001:0003a7b3       ?Store@CRuntimeClass@@QBEXAAVCArchive@@@Z 5f83b7b3 f   arccore.obj
 0001:0003a806       ??0CArchive@@QAE@PAVCFile@@IHPAX@Z 5f83b806 f   arccore.obj
 0001:0003aa54       ??1CArchive@@QAE@XZ        5f83ba54 f   arccore.obj
 0001:0003aabd       ?Abort@CArchive@@QAEXXZ    5f83babd f   arccore.obj
 0001:0003ac6b       ?Close@CArchive@@QAEXXZ    5f83bc6b f   arccore.obj
 0001:0003ac9e       ?Read@CArchive@@QAEIPAXI@Z 5f83bc9e f   arccore.obj
 0001:0003b0f4       ?Write@CArchive@@QAEXPBXI@Z 5f83c0f4 f   arccore.obj
 0001:0003b433       ?Flush@CArchive@@QAEXXZ    5f83c433 f   arccore.obj
 0001:0003b688       ?FillBuffer@CArchive@@QAEXI@Z 5f83c688 f   arccore.obj
 0001:0003b9fa       ?WriteCount@CArchive@@QAEXK@Z 5f83c9fa f   arccore.obj
 0001:0003ba38       ?ReadCount@CArchive@@QAEKXZ 5f83ca38 f   arccore.obj
 0001:0003ba7b       ?WriteString@CArchive@@QAEXPBG@Z 5f83ca7b f   arccore.obj
 0001:0003bad0       ?ReadString@CArchive@@QAEPAGPAGI@Z 5f83cad0 f   arccore.obj
 0001:0003bc6c       ?ReadString@CArchive@@QAEHAAVCString@@@Z 5f83cc6c f   arccore.obj
 0001:0003bd60       ?CheckCount@CArchive@@QAEXXZ 5f83cd60 f   arcobj.obj
 0001:0003bd8a       ?WriteObject@CArchive@@QAEXPBVCObject@@@Z 5f83cd8a f   arcobj.obj
 0001:0003beb8       ?ReadObject@CArchive@@QAEPAVCObject@@PBUCRuntimeClass@@@Z 5f83ceb8 f   arcobj.obj
 0001:0003c056       ?GetObjectSchema@CArchive@@QAEIXZ 5f83d056 f   arcobj.obj
 0001:0003c079       ?MapObject@CArchive@@QAEXPBVCObject@@@Z 5f83d079 f   arcobj.obj
 0001:0003c24b       ?WriteClass@CArchive@@QAEXPBUCRuntimeClass@@@Z 5f83d24b f   arcobj.obj
 0001:0003c36f       ?ReadClass@CArchive@@QAEPAUCRuntimeClass@@PBU2@PAIPAK@Z 5f83d36f f   arcobj.obj
 0001:0003c6e7       ?SerializeClass@CArchive@@QAEXPBUCRuntimeClass@@@Z 5f83d6e7 f   arcobj.obj
 0001:0003c720       ?GetErrorMessage@CArchiveException@@UAEHPAGIPAI@Z 5f83d720 f   arcex.obj
 0001:0003c82f       ?Dump@CArchiveException@@UBEXAAVCDumpContext@@@Z 5f83d82f f   arcex.obj
 0001:0003c899       ?AfxThrowArchiveException@@YGXHPBG@Z 5f83d899 f   arcex.obj
 0001:0003c960       ??6@YGAAVCDumpContext@@AAV0@UtagSIZE@@@Z 5f83d960 f   wingdi.obj
 0001:0003c9a2       ??6@YGAAVCDumpContext@@AAV0@UtagPOINT@@@Z 5f83d9a2 f   wingdi.obj
 0001:0003c9e4       ??6@YGAAVCDumpContext@@AAV0@ABUtagRECT@@@Z 5f83d9e4 f   wingdi.obj
 0001:0003ca5f       ??0CDC@@QAE@XZ             5f83da5f f   wingdi.obj
 0001:0003ca9c       ?AssertValid@CDC@@UBEXXZ   5f83da9c f   wingdi.obj
 0001:0003caaf       ?Dump@CDC@@UBEXAAVCDumpContext@@@Z 5f83daaf f   wingdi.obj
 0001:0003cb26       ?afxMapHDC@@YGPAVCHandleMap@@H@Z 5f83db26 f   wingdi.obj
 0001:0003cbe4       ?FromHandle@CDC@@SGPAV1@PAUHDC__@@@Z 5f83dbe4 f   wingdi.obj
 0001:0003cc57       ?Attach@CDC@@QAEHPAUHDC__@@@Z 5f83dc57 f   wingdi.obj
 0001:0003cd0d       ?Detach@CDC@@QAEPAUHDC__@@XZ 5f83dd0d f   wingdi.obj
 0001:0003cd60       ?DeleteDC@CDC@@QAEHXZ      5f83dd60 f   wingdi.obj
 0001:0003cd87       ??1CDC@@UAE@XZ             5f83dd87 f   wingdi.obj
 0001:0003cde8       ?SetAttribDC@CDC@@UAEXPAUHDC__@@@Z 5f83dde8 f   wingdi.obj
 0001:0003cdfe       ?SetOutputDC@CDC@@UAEXPAUHDC__@@@Z 5f83ddfe f   wingdi.obj
 0001:0003ce75       ?ReleaseAttribDC@CDC@@UAEXXZ 5f83de75 f   wingdi.obj
 0001:0003ce8a       ?ReleaseOutputDC@CDC@@UAEXXZ 5f83de8a f   wingdi.obj
 0001:0003cf00       ?StartDocW@CDC@@QAEHPBG@Z  5f83df00 f   wingdi.obj
 0001:0003cf38       ?SaveDC@CDC@@UAEHXZ        5f83df38 f   wingdi.obj
 0001:0003cfb7       ?RestoreDC@CDC@@UAEHH@Z    5f83dfb7 f   wingdi.obj
 0001:0003d083       ?SelectGdiObject@CDC@@KGPAVCGdiObject@@PAUHDC__@@PAX@Z 5f83e083 f   wingdi.obj
 0001:0003d09e       ?SelectStockObject@CDC@@UAEPAVCGdiObject@@H@Z 5f83e09e f   wingdi.obj
 0001:0003d152       ?SelectObject@CDC@@QAEPAVCPen@@PAV2@@Z 5f83e152 f   wingdi.obj
 0001:0003d1e3       ?SelectObject@CDC@@QAEPAVCBrush@@PAV2@@Z 5f83e1e3 f   wingdi.obj
 0001:0003d274       ?SelectObject@CDC@@UAEPAVCFont@@PAV2@@Z 5f83e274 f   wingdi.obj
 0001:0003d305       ?SelectObject@CDC@@QAEHPAVCRgn@@@Z 5f83e305 f   wingdi.obj
 0001:0003d390       ?SelectPalette@CDC@@QAEPAVCPalette@@PAV2@H@Z 5f83e390 f   wingdi.obj
 0001:0003d3e6       ?SetBkColor@CDC@@UAEKK@Z   5f83e3e6 f   wingdi.obj
 0001:0003d467       ?SetBkMode@CDC@@QAEHH@Z    5f83e467 f   wingdi.obj
 0001:0003d4e8       ?SetPolyFillMode@CDC@@QAEHH@Z 5f83e4e8 f   wingdi.obj
 0001:0003d569       ?SetROP2@CDC@@QAEHH@Z      5f83e569 f   wingdi.obj
 0001:0003d5ea       ?SetStretchBltMode@CDC@@QAEHH@Z 5f83e5ea f   wingdi.obj
 0001:0003d66b       ?SetTextColor@CDC@@UAEKK@Z 5f83e66b f   wingdi.obj
 0001:0003d6ec       ?SetMapMode@CDC@@UAEHH@Z   5f83e6ec f   wingdi.obj
 0001:0003d76d       ?SetViewportOrg@CDC@@UAE?AVCPoint@@HH@Z 5f83e76d f   wingdi.obj
 0001:0003d843       ?OffsetViewportOrg@CDC@@UAE?AVCPoint@@HH@Z 5f83e843 f   wingdi.obj
 0001:0003d919       ?SetViewportExt@CDC@@UAE?AVCSize@@HH@Z 5f83e919 f   wingdi.obj
 0001:0003d9ef       ?ScaleViewportExt@CDC@@UAE?AVCSize@@HHHH@Z 5f83e9ef f   wingdi.obj
 0001:0003dad5       ?SetWindowOrg@CDC@@QAE?AVCPoint@@HH@Z 5f83ead5 f   wingdi.obj
 0001:0003dbab       ?OffsetWindowOrg@CDC@@QAE?AVCPoint@@HH@Z 5f83ebab f   wingdi.obj
 0001:0003dc81       ?SetWindowExt@CDC@@UAE?AVCSize@@HH@Z 5f83ec81 f   wingdi.obj
 0001:0003dd57       ?ScaleWindowExt@CDC@@UAE?AVCSize@@HHHH@Z 5f83ed57 f   wingdi.obj
 0001:0003de3d       ?GetClipBox@CDC@@UBEHPAUtagRECT@@@Z 5f83ee3d f   wingdi.obj
 0001:0003de84       ?SelectClipRgn@CDC@@QAEHPAVCRgn@@@Z 5f83ee84 f   wingdi.obj
 0001:0003df0f       ?ExcludeClipRect@CDC@@QAEHHHHH@Z 5f83ef0f f   wingdi.obj
 0001:0003dfa8       ?ExcludeClipRect@CDC@@QAEHPBUtagRECT@@@Z 5f83efa8 f   wingdi.obj
 0001:0003e057       ?IntersectClipRect@CDC@@QAEHHHHH@Z 5f83f057 f   wingdi.obj
 0001:0003e0f0       ?IntersectClipRect@CDC@@QAEHPBUtagRECT@@@Z 5f83f0f0 f   wingdi.obj
 0001:0003e19f       ?OffsetClipRgn@CDC@@QAEHHH@Z 5f83f19f f   wingdi.obj
 0001:0003e228       ?OffsetClipRgn@CDC@@QAEHUtagSIZE@@@Z 5f83f228 f   wingdi.obj
 0001:0003e2b1       ?MoveTo@CDC@@QAE?AVCPoint@@HH@Z 5f83f2b1 f   wingdi.obj
 0001:0003e387       ?LineTo@CDC@@QAEHHH@Z      5f83f387 f   wingdi.obj
 0001:0003e400       ?SetTextAlign@CDC@@QAEII@Z 5f83f400 f   wingdi.obj
 0001:0003e47e       ?SetTextJustification@CDC@@QAEHHH@Z 5f83f47e f   wingdi.obj
 0001:0003e507       ?SetTextCharacterExtra@CDC@@QAEHH@Z 5f83f507 f   wingdi.obj
 0001:0003e588       ?SetMapperFlags@CDC@@QAEKK@Z 5f83f588 f   wingdi.obj
 0001:0003e609       ?GetLayout@CDC@@QBEKXZ     5f83f609 f   wingdi.obj
 0001:0003e6ad       ?SetLayout@CDC@@QAEKK@Z    5f83f6ad f   wingdi.obj
 0001:0003e75d       ?ScreenToClient@CWnd@@QBEXPAUtagRECT@@@Z 5f83f75d f   wingdi.obj
 0001:0003e7dd       ?ClientToScreen@CWnd@@QBEXPAUtagRECT@@@Z 5f83f7dd f   wingdi.obj
 0001:0003e85d       ?ArcTo@CDC@@QAEHHHHHHHHH@Z 5f83f85d f   wingdi.obj
 0001:0003e942       ?SetArcDirection@CDC@@QAEHH@Z 5f83f942 f   wingdi.obj
 0001:0003e9c3       ?PolyDraw@CDC@@QAEHPBUtagPOINT@@PBEH@Z 5f83f9c3 f   wingdi.obj
 0001:0003ea94       ?PolylineTo@CDC@@QAEHPBUtagPOINT@@H@Z 5f83fa94 f   wingdi.obj
 0001:0003eb61       ?SetColorAdjustment@CDC@@QAEHPBUtagCOLORADJUSTMENT@@@Z 5f83fb61 f   wingdi.obj
 0001:0003ebe2       ?PolyBezierTo@CDC@@QAEHPBUtagPOINT@@H@Z 5f83fbe2 f   wingdi.obj
 0001:0003ecaf       ?SelectClipPath@CDC@@QAEHH@Z 5f83fcaf f   wingdi.obj
 0001:0003ed76       ?SelectClipRgn@CDC@@QAEHPAVCRgn@@H@Z 5f83fd76 f   wingdi.obj
 0001:0003ee09       ?AfxEnumMetaFileProc@@YGHPAUHDC__@@PAUtagHANDLETABLE@@PAUtagMETARECORD@@HJ@Z 5f83fe09 f   wingdi.obj
 0001:0003f165       ?PlayMetaFile@CDC@@QAEHPAUHMETAFILE__@@@Z 5f840165 f   wingdi.obj
 0001:0003f1b3       ?LPtoDP@CDC@@QBEXPAUtagSIZE@@@Z 5f8401b3 f   wingdi.obj
 0001:0003f279       ?DPtoLP@CDC@@QBEXPAUtagSIZE@@@Z 5f840279 f   wingdi.obj
 0001:0003f33f       ?AssertValid@CClientDC@@UBEXXZ 5f84033f f   wingdi.obj
 0001:0003f38c       ?Dump@CClientDC@@UBEXAAVCDumpContext@@@Z 5f84038c f   wingdi.obj
 0001:0003f3cd       ??0CClientDC@@QAE@PAVCWnd@@@Z 5f8403cd f   wingdi.obj
 0001:0003f47f       ??1CClientDC@@UAE@XZ       5f84047f f   wingdi.obj
 0001:0003f507       ?AssertValid@CWindowDC@@UBEXXZ 5f840507 f   wingdi.obj
 0001:0003f554       ?Dump@CWindowDC@@UBEXAAVCDumpContext@@@Z 5f840554 f   wingdi.obj
 0001:0003f595       ??0CWindowDC@@QAE@PAVCWnd@@@Z 5f840595 f   wingdi.obj
 0001:0003f647       ??1CWindowDC@@UAE@XZ       5f840647 f   wingdi.obj
 0001:0003f6cf       ?AssertValid@CPaintDC@@UBEXXZ 5f8406cf f   wingdi.obj
 0001:0003f713       ?Dump@CPaintDC@@UBEXAAVCDumpContext@@@Z 5f840713 f   wingdi.obj
 0001:0003f7af       ??0CPaintDC@@QAE@PAVCWnd@@@Z 5f8407af f   wingdi.obj
 0001:0003f873       ??1CPaintDC@@UAE@XZ        5f840873 f   wingdi.obj
 0001:0003f92c       ?Dump@CGdiObject@@UBEXAAVCDumpContext@@@Z 5f84092c f   wingdi.obj
 0001:0003f96d       ?AssertValid@CGdiObject@@UBEXXZ 5f84096d f   wingdi.obj
 0001:0003f9c3       ?afxMapHGDIOBJ@@YGPAVCHandleMap@@H@Z 5f8409c3 f   wingdi.obj
 0001:0003fa81       ?FromHandle@CGdiObject@@SGPAV1@PAX@Z 5f840a81 f   wingdi.obj
 0001:0003fafa       ?Attach@CGdiObject@@QAEHPAX@Z 5f840afa f   wingdi.obj
 0001:0003fb84       ?Detach@CGdiObject@@QAEPAXXZ 5f840b84 f   wingdi.obj
 0001:0003fbcc       ?DeleteObject@CGdiObject@@QAEHXZ 5f840bcc f   wingdi.obj
 0001:0003fbf3       ??0CPen@@QAE@HHK@Z         5f840bf3 f   wingdi.obj
 0001:0003fc65       ??0CPen@@QAE@HHPBUtagLOGBRUSH@@HPBK@Z 5f840c65 f   wingdi.obj
 0001:0003fcdf       ?Dump@CPen@@UBEXAAVCDumpContext@@@Z 5f840cdf f   wingdi.obj
 0001:0003fdbc       ??0CBrush@@QAE@K@Z         5f840dbc f   wingdi.obj
 0001:0003fe26       ??0CBrush@@QAE@HK@Z        5f840e26 f   wingdi.obj
 0001:0003fe94       ??0CBrush@@QAE@PAVCBitmap@@@Z 5f840e94 f   wingdi.obj
 0001:0003ff14       ?CreateDIBPatternBrush@CBrush@@QAEHPAXI@Z 5f840f14 f   wingdi.obj
 0001:0003ff9d       ?Dump@CBrush@@UBEXAAVCDumpContext@@@Z 5f840f9d f   wingdi.obj
 0001:0004007a       ?Dump@CFont@@UBEXAAVCDumpContext@@@Z 5f84107a f   wingdi.obj
 0001:0004028c       ?Dump@CBitmap@@UBEXAAVCDumpContext@@@Z 5f84128c f   wingdi.obj
 0001:000403b3       ?AfxThrowResourceException@@YGXXZ 5f8413b3 f   wingdi.obj
 0001:000403d0       ?AfxThrowUserException@@YGXXZ 5f8413d0 f   wingdi.obj
 0001:000403f0       ??_ECClientDC@@UAEPAXI@Z   5f8413f0 f i wingdi.obj
 0001:000403f0       ??_GCClientDC@@UAEPAXI@Z   5f8413f0 f i wingdi.obj
 0001:00040420       ??_ECWindowDC@@UAEPAXI@Z   5f841420 f i wingdi.obj
 0001:00040420       ??_GCWindowDC@@UAEPAXI@Z   5f841420 f i wingdi.obj
 0001:00040450       ??_GCPaintDC@@UAEPAXI@Z    5f841450 f i wingdi.obj
 0001:00040450       ??_ECPaintDC@@UAEPAXI@Z    5f841450 f i wingdi.obj
 0001:00040480       ?AfxCustomLogFont@@YGHIPAUtagLOGFONTW@@@Z 5f841480 f   winutil.obj
 0001:00040564       ?_AfxIsComboBoxControl@@YGHPAUHWND__@@I@Z 5f841564 f   winutil.obj
 0001:000405b6       ?_AfxCompareClassName@@YGHPAUHWND__@@PBG@Z 5f8415b6 f   winutil.obj
 0001:00040610       ?_AfxChildWindowFromPoint@@YGPAUHWND__@@PAU1@UtagPOINT@@@Z 5f841610 f   winutil.obj
 0001:000406d6       ?AfxSetWindowText@@YGXPAUHWND__@@PBG@Z 5f8416d6 f   winutil.obj
 0001:00040739       ?AfxDeleteObject@@YGXPAPAX@Z 5f841739 f   winutil.obj
 0001:00040780       ?AfxCancelModes@@YGXPAUHWND__@@@Z 5f841780 f   winutil.obj
 0001:00040827       ?AfxGlobalFree@@YGXPAX@Z   5f841827 f   winutil.obj
 0001:000408a2       ?AfxCriticalNewHandler@@YAHI@Z 5f8418a2 f   winutil.obj
 0001:000409a0       ?_GetBaseMessageMap@CDocument@@KGPBUAFX_MSGMAP@@XZ 5f8419a0 f   doccore.obj
 0001:000409aa       ?GetMessageMap@CDocument@@MBEPBUAFX_MSGMAP@@XZ 5f8419aa f   doccore.obj
 0001:000409ba       ??0CDocument@@QAE@XZ       5f8419ba f   doccore.obj
 0001:00040a89       ??1CDocument@@UAE@XZ       5f841a89 f   doccore.obj
 0001:00040b8f       ?OnFinalRelease@CDocument@@UAEXXZ 5f841b8f f   doccore.obj
 0001:00040bb8       ?DisconnectViews@CDocument@@QAEXXZ 5f841bb8 f   doccore.obj
 0001:00040c2c       ?SetTitle@CDocument@@UAEXPBG@Z 5f841c2c f   doccore.obj
 0001:00040c56       ?DeleteContents@CDocument@@UAEXXZ 5f841c56 f   doccore.obj
 0001:00040c61       ?OnChangedViewList@CDocument@@UAEXXZ 5f841c61 f   doccore.obj
 0001:00040ca2       ?UpdateFrameCounts@CDocument@@UAEXXZ 5f841ca2 f   doccore.obj
 0001:00040ef8       ?CanCloseFrame@CDocument@@UAEHPAVCFrameWnd@@@Z 5f841ef8 f   doccore.obj
 0001:00040f97       ?PreCloseFrame@CDocument@@UAEXPAVCFrameWnd@@@Z 5f841f97 f   doccore.obj
 0001:00040fa4       ?SetPathName@CDocument@@UAEXPBGH@Z 5f841fa4 f   doccore.obj
 0001:000410b1       ?OnFileClose@CDocument@@IAEXXZ 5f8420b1 f   doccore.obj
 0001:000410de       ?OnFileSave@CDocument@@IAEXXZ 5f8420de f   doccore.obj
 0001:000410f7       ?OnFileSaveAs@CDocument@@IAEXXZ 5f8420f7 f   doccore.obj
 0001:0004112a       ?DoFileSave@CDocument@@UAEHXZ 5f84212a f   doccore.obj
 0001:000411bf       ?DoSave@CDocument@@UAEHPBGH@Z 5f8421bf f   doccore.obj
 0001:00041469       ?SaveModified@CDocument@@UAEHXZ 5f842469 f   doccore.obj
 0001:0004165e       ?GetDefaultMenu@CDocument@@UAEPAUHMENU__@@XZ 5f84265e f   doccore.obj
 0001:0004166b       ?GetDefaultAccelerator@CDocument@@UAEPAUHACCEL__@@XZ 5f84266b f   doccore.obj
 0001:00041678       ?ReportSaveLoadException@CDocument@@UAEXPBGPAVCException@@HI@Z 5f842678 f   doccore.obj
 0001:000418ea       ?GetTempName@CMirrorFile@@SA?AVCString@@PBGH@Z 5f8428ea f   doccore.obj
 0001:000419c0       ?Open@CMirrorFile@@UAEHPBGIPAVCFileException@@@Z 5f8429c0 f   doccore.obj
 0001:00041cda       ?Abort@CMirrorFile@@UAEXXZ 5f842cda f   doccore.obj
 0001:00041d0d       ?Close@CMirrorFile@@UAEXXZ 5f842d0d f   doccore.obj
 0001:00041f1c       ?GetFile@CDocument@@UAEPAVCFile@@PBGIPAVCFileException@@@Z 5f842f1c f   doccore.obj
 0001:00041ffe       ?ReleaseFile@CDocument@@UAEXPAVCFile@@H@Z 5f842ffe f   doccore.obj
 0001:00042087       ?OnNewDocument@CDocument@@UAEHXZ 5f843087 f   doccore.obj
 0001:000420db       ?OnOpenDocument@CDocument@@UAEHPBG@Z 5f8430db f   doccore.obj
 0001:000423ca       ?OnSaveDocument@CDocument@@UAEHPBG@Z 5f8433ca f   doccore.obj
 0001:0004264d       ?OnCloseDocument@CDocument@@UAEXXZ 5f84364d f   doccore.obj
 0001:00042724       ?OnIdle@CDocument@@UAEXXZ  5f843724 f   doccore.obj
 0001:0004272f       ?AddView@CDocument@@QAEXPAVCView@@@Z 5f84372f f   doccore.obj
 0001:000427ed       ?RemoveView@CDocument@@QAEXPAVCView@@@Z 5f8437ed f   doccore.obj
 0001:0004286a       ?GetFirstViewPosition@CDocument@@UBEPAU__POSITION@@XZ 5f84386a f   doccore.obj
 0001:00042880       ?GetNextView@CDocument@@UBEPAVCView@@AAPAU__POSITION@@@Z 5f843880 f   doccore.obj
 0001:00042903       ?UpdateAllViews@CDocument@@QAEXPAVCView@@JPAVCObject@@@Z 5f843903 f   doccore.obj
 0001:000429a4       ?SendInitialUpdate@CDocument@@QAEXXZ 5f8439a4 f   doccore.obj
 0001:000429fa       ?OnCmdMsg@CDocument@@UAEHIHPAXPAUAFX_CMDHANDLERINFO@@@Z 5f8439fa f   doccore.obj
 0001:00042a61       ?Dump@CDocument@@UBEXAAVCDumpContext@@@Z 5f843a61 f   doccore.obj
 0001:00042b3f       ?AssertValid@CDocument@@UBEXXZ 5f843b3f f   doccore.obj
 0001:00042b90       ??_ECDocument@@UAEPAXI@Z   5f843b90 f i doccore.obj
 0001:00042b90       ??_GCDocument@@UAEPAXI@Z   5f843b90 f i doccore.obj
 0001:00042bc0       ??0CMirrorFile@@QAE@XZ     5f843bc0 f i doccore.obj
 0001:00042c20       ??1CMirrorFile@@UAE@XZ     5f843c20 f i doccore.obj
 0001:00042c70       ??0CDocTemplate@@IAE@IPAUCRuntimeClass@@00@Z 5f843c70 f   doctempl.obj
 0001:00042ef2       ?LoadTemplate@CDocTemplate@@UAEXXZ 5f843ef2 f   doctempl.obj
 0001:00043046       ?SetServerInfo@CDocTemplate@@QAEXIIPAUCRuntimeClass@@0@Z 5f844046 f   doctempl.obj
 0001:0004313f       ?SetContainerInfo@CDocTemplate@@QAEXI@Z 5f84413f f   doctempl.obj
 0001:0004318f       ??1CDocTemplate@@UAE@XZ    5f84418f f   doctempl.obj
 0001:00043267       ?GetDocString@CDocTemplate@@UBEHAAVCString@@W4DocStringIndex@1@@Z 5f844267 f   doctempl.obj
 0001:0004328f       ?AddDocument@CDocTemplate@@UAEXPAVCDocument@@@Z 5f84428f f   doctempl.obj
 0001:000432e1       ?RemoveDocument@CDocTemplate@@UAEXPAVCDocument@@@Z 5f8442e1 f   doctempl.obj
 0001:00043336       ?MatchDocType@CDocTemplate@@UAE?AW4Confidence@1@PBGAAPAVCDocument@@@Z 5f844336 f   doctempl.obj
 0001:000434af       ?CreateNewDocument@CDocTemplate@@UAEPAVCDocument@@XZ 5f8444af f   doctempl.obj
 0001:0004356f       ?CreateNewFrame@CDocTemplate@@UAEPAVCFrameWnd@@PAVCDocument@@PAV2@@Z 5f84456f f   doctempl.obj
 0001:000436d9       ?CreateOleFrame@CDocTemplate@@QAEPAVCFrameWnd@@PAVCWnd@@PAVCDocument@@H@Z 5f8446d9 f   doctempl.obj
 0001:000437d9       ?InitialUpdateFrame@CDocTemplate@@UAEXPAVCFrameWnd@@PAVCDocument@@H@Z 5f8447d9 f   doctempl.obj
 0001:000437f6       ?SaveAllModified@CDocTemplate@@UAEHXZ 5f8447f6 f   doctempl.obj
 0001:00043846       ?CloseAllDocuments@CDocTemplate@@UAEXH@Z 5f844846 f   doctempl.obj
 0001:0004388b       ?OnIdle@CDocTemplate@@UAEXXZ 5f84488b f   doctempl.obj
 0001:00043912       ?OnCmdMsg@CDocTemplate@@UAEHIHPAXPAUAFX_CMDHANDLERINFO@@@Z 5f844912 f   doctempl.obj
 0001:00043982       ?Dump@CDocTemplate@@UBEXAAVCDumpContext@@@Z 5f844982 f   doctempl.obj
 0001:00043a7a       ?AssertValid@CDocTemplate@@UBEXXZ 5f844a7a f   doctempl.obj
 0001:00043ad0       ??_ECDocTemplate@@UAEPAXI@Z 5f844ad0 f i doctempl.obj
 0001:00043ad0       ??_GCDocTemplate@@UAEPAXI@Z 5f844ad0 f i doctempl.obj
 0001:00043b00       ??0CSingleDocTemplate@@QAE@IPAUCRuntimeClass@@00@Z 5f844b00 f   docsingl.obj
 0001:00043b3b       ??1CSingleDocTemplate@@UAE@XZ 5f844b3b f   docsingl.obj
 0001:00043b9f       ?GetFirstDocPosition@CSingleDocTemplate@@UBEPAU__POSITION@@XZ 5f844b9f f   docsingl.obj
 0001:00043bb4       ?GetNextDoc@CSingleDocTemplate@@UBEPAVCDocument@@AAPAU__POSITION@@@Z 5f844bb4 f   docsingl.obj
 0001:00043c0d       ?AddDocument@CSingleDocTemplate@@UAEXPAVCDocument@@@Z 5f844c0d f   docsingl.obj
 0001:00043c65       ?RemoveDocument@CSingleDocTemplate@@UAEXPAVCDocument@@@Z 5f844c65 f   docsingl.obj
 0001:00043cc0       ?OpenDocumentFile@CSingleDocTemplate@@UAEPAVCDocument@@PBGH@Z 5f844cc0 f   docsingl.obj
 0001:0004403e       ?SetDefaultTitle@CSingleDocTemplate@@UAEXPAVCDocument@@@Z 5f84503e f   docsingl.obj
 0001:000440f0       ?Dump@CSingleDocTemplate@@UBEXAAVCDumpContext@@@Z 5f8450f0 f   docsingl.obj
 0001:00044149       ?AssertValid@CSingleDocTemplate@@UBEXXZ 5f845149 f   docsingl.obj
 0001:00044180       ??_ECSingleDocTemplate@@UAEPAXI@Z 5f845180 f i docsingl.obj
 0001:00044180       ??_GCSingleDocTemplate@@UAEPAXI@Z 5f845180 f i docsingl.obj
 0001:000441b0       ??0CMultiDocTemplate@@QAE@IPAUCRuntimeClass@@00@Z 5f8451b0 f   docmulti.obj
 0001:0004427d       ?LoadTemplate@CMultiDocTemplate@@UAEXXZ 5f84527d f   docmulti.obj
 0001:00044309       ??1CMultiDocTemplate@@UAE@XZ 5f845309 f   docmulti.obj
 0001:000443b5       ?GetFirstDocPosition@CMultiDocTemplate@@UBEPAU__POSITION@@XZ 5f8453b5 f   docmulti.obj
 0001:000443cb       ?GetNextDoc@CMultiDocTemplate@@UBEPAVCDocument@@AAPAU__POSITION@@@Z 5f8453cb f   docmulti.obj
 0001:000443e7       ?AddDocument@CMultiDocTemplate@@UAEXPAVCDocument@@@Z 5f8453e7 f   docmulti.obj
 0001:00044451       ?RemoveDocument@CMultiDocTemplate@@UAEXPAVCDocument@@@Z 5f845451 f   docmulti.obj
 0001:00044497       ?OpenDocumentFile@CMultiDocTemplate@@UAEPAVCDocument@@PBGH@Z 5f845497 f   docmulti.obj
 0001:0004469f       ?SetDefaultTitle@CMultiDocTemplate@@UAEXPAVCDocument@@@Z 5f84569f f   docmulti.obj
 0001:0004477e       ?Dump@CMultiDocTemplate@@UBEXAAVCDumpContext@@@Z 5f84577e f   docmulti.obj
 0001:00044866       ?AssertValid@CMultiDocTemplate@@UBEXXZ 5f845866 f   docmulti.obj
 0001:000448c0       ??_GCMultiDocTemplate@@UAEPAXI@Z 5f8458c0 f i docmulti.obj
 0001:000448c0       ??_ECMultiDocTemplate@@UAEPAXI@Z 5f8458c0 f i docmulti.obj
 0001:000448f0       ?OpenDocumentFile@CDocManager@@UAEPAVCDocument@@PBG@Z 5f8458f0 f   docmgr.obj
 0001:00044c32       ?GetOpenDocumentCount@CDocManager@@UAEHXZ 5f845c32 f   docmgr.obj
 0001:00044cb0       ?_GetBaseMessageMap@CView@@KGPBUAFX_MSGMAP@@XZ 5f845cb0 f   viewcore.obj
 0001:00044cba       ?GetMessageMap@CView@@MBEPBUAFX_MSGMAP@@XZ 5f845cba f   viewcore.obj
 0001:00044cca       ??0CView@@IAE@XZ           5f845cca f   viewcore.obj
 0001:00044cf3       ??1CView@@UAE@XZ           5f845cf3 f   viewcore.obj
 0001:00044d54       ?PreCreateWindow@CView@@MAEHAAUtagCREATESTRUCTW@@@Z 5f845d54 f   viewcore.obj
 0001:00044e01       ?OnCreate@CView@@IAEHPAUtagCREATESTRUCTW@@@Z 5f845e01 f   viewcore.obj
 0001:00044ea8       ?OnDestroy@CView@@IAEXXZ   5f845ea8 f   viewcore.obj
 0001:00044ee7       ?PostNcDestroy@CView@@MAEXXZ 5f845ee7 f   viewcore.obj
 0001:00044f1f       ?CalcWindowRect@CView@@UAEXPAUtagRECT@@I@Z 5f845f1f f   viewcore.obj
 0001:00044fe0       ?OnCmdMsg@CView@@UAEHIHPAXPAUAFX_CMDHANDLERINFO@@@Z 5f845fe0 f   viewcore.obj
 0001:00045087       ?OnPaint@CView@@IAEXXZ     5f846087 f   viewcore.obj
 0001:000450fb       ?OnInitialUpdate@CView@@UAEXXZ 5f8460fb f   viewcore.obj
 0001:0004511a       ?OnUpdate@CView@@MAEXPAV1@JPAVCObject@@@Z 5f84611a f   viewcore.obj
 0001:00045159       ?OnPrint@CView@@MAEXPAVCDC@@PAUCPrintInfo@@@Z 5f846159 f   viewcore.obj
 0001:0004518b       ?OnDraw@CView@@MAEXPAVCDC@@@Z 5f84618b f   viewcore.obj
 0001:00045198       ?IsSelected@CView@@UBEHPBVCObject@@@Z 5f846198 f   viewcore.obj
 0001:000451ba       ?OnActivateView@CView@@MAEXHPAV1@0@Z 5f8461ba f   viewcore.obj
 0001:00045209       ?OnActivateFrame@CView@@MAEXIPAVCFrameWnd@@@Z 5f846209 f   viewcore.obj
 0001:00045216       ?OnMouseActivate@CView@@IAEHPAVCWnd@@II@Z 5f846216 f   viewcore.obj
 0001:00045304       ?OnScroll@CView@@UAEHIIH@Z 5f846304 f   viewcore.obj
 0001:00045313       ?OnScrollBy@CView@@UAEHVCSize@@H@Z 5f846313 f   viewcore.obj
 0001:00045322       ?OnDragScroll@CView@@UAEKKVCPoint@@@Z 5f846322 f   viewcore.obj
 0001:00045334       ?OnDragEnter@CView@@UAEKPAVCOleDataObject@@KVCPoint@@@Z 5f846334 f   viewcore.obj
 0001:00045343       ?OnDragOver@CView@@UAEKPAVCOleDataObject@@KVCPoint@@@Z 5f846343 f   viewcore.obj
 0001:00045352       ?OnDrop@CView@@UAEHPAVCOleDataObject@@KVCPoint@@@Z 5f846352 f   viewcore.obj
 0001:00045361       ?OnDropEx@CView@@UAEKPAVCOleDataObject@@KKVCPoint@@@Z 5f846361 f   viewcore.obj
 0001:00045371       ?OnDragLeave@CView@@UAEXXZ 5f846371 f   viewcore.obj
 0001:0004537c       ?GetParentSplitter@CView@@SGPAVCSplitterWnd@@PBVCWnd@@H@Z 5f84637c f   viewcore.obj
 0001:000453d2       ?GetScrollBarCtrl@CView@@UBEPAVCScrollBar@@H@Z 5f8463d2 f   viewcore.obj
 0001:000454bb       ?OnUpdateSplitCmd@CView@@IAEXPAVCCmdUI@@@Z 5f8464bb f   viewcore.obj
 0001:00045508       ?OnSplitCmd@CView@@IAEHI@Z 5f846508 f   viewcore.obj
 0001:0004556e       ?OnUpdateNextPaneMenu@CView@@IAEXPAVCCmdUI@@@Z 5f84656e f   viewcore.obj
 0001:00045609       ?OnNextPaneCmd@CView@@IAEHI@Z 5f846609 f   viewcore.obj
 0001:00045682       ?OnPrepareDC@CView@@UAEXPAVCDC@@PAUCPrintInfo@@@Z 5f846682 f   viewcore.obj
 0001:000456db       ?OnPreparePrinting@CView@@MAEHPAUCPrintInfo@@@Z 5f8466db f   viewcore.obj
 0001:000456ed       ?OnBeginPrinting@CView@@MAEXPAVCDC@@PAUCPrintInfo@@@Z 5f8466ed f   viewcore.obj
 0001:0004570d       ?OnEndPrinting@CView@@MAEXPAVCDC@@PAUCPrintInfo@@@Z 5f84670d f   viewcore.obj
 0001:0004572d       ?OnEndPrintPreview@CView@@MAEXPAVCDC@@PAUCPrintInfo@@UtagPOINT@@PAVCPreviewView@@@Z 5f84672d f   viewcore.obj
 0001:0004583d       ?Dump@CView@@UBEXAAVCDumpContext@@@Z 5f84683d f   viewcore.obj
 0001:00045889       ?AssertValid@CView@@UBEXXZ 5f846889 f   viewcore.obj
 0001:0004589c       ?_GetBaseMessageMap@CCtrlView@@KGPBUAFX_MSGMAP@@XZ 5f84689c f   viewcore.obj
 0001:000458a6       ?GetMessageMap@CCtrlView@@MBEPBUAFX_MSGMAP@@XZ 5f8468a6 f   viewcore.obj
 0001:000458b6       ??0CCtrlView@@QAE@PBGK@Z   5f8468b6 f   viewcore.obj
 0001:0004592b       ?PreCreateWindow@CCtrlView@@MAEHAAUtagCREATESTRUCTW@@@Z 5f84692b f   viewcore.obj
 0001:000459db       ?OnDraw@CCtrlView@@MAEXPAVCDC@@@Z 5f8469db f   viewcore.obj
 0001:00045a11       ?OnPaint@CCtrlView@@IAEXXZ 5f846a11 f   viewcore.obj
 0001:00045a24       ?Dump@CCtrlView@@UBEXAAVCDumpContext@@@Z 5f846a24 f   viewcore.obj
 0001:00045a72       ?AssertValid@CCtrlView@@UBEXXZ 5f846a72 f   viewcore.obj
 0001:00045ac0       ??_GCView@@UAEPAXI@Z       5f846ac0 f i viewcore.obj
 0001:00045ac0       ??_ECView@@UAEPAXI@Z       5f846ac0 f i viewcore.obj
 0001:00045af0       ??_ECCtrlView@@UAEPAXI@Z   5f846af0 f i viewcore.obj
 0001:00045af0       ??_GCCtrlView@@UAEPAXI@Z   5f846af0 f i viewcore.obj
 0001:00045b20       ??1CCtrlView@@UAE@XZ       5f846b20 f i viewcore.obj
 0001:00045b70       ?_GetBaseMessageMap@CScrollView@@KGPBUAFX_MSGMAP@@XZ 5f846b70 f   viewscrl.obj
 0001:00045b7a       ?GetMessageMap@CScrollView@@MBEPBUAFX_MSGMAP@@XZ 5f846b7a f   viewscrl.obj
 0001:00045b8a       ?_AfxGetMouseScrollLines@@YGIXZ 5f846b8a f   viewscrl.obj
 0001:00045cef       ??0CScrollView@@IAE@XZ     5f846cef f   viewscrl.obj
 0001:00045d84       ??1CScrollView@@UAE@XZ     5f846d84 f   viewscrl.obj
 0001:00045da0       ?OnPrepareDC@CScrollView@@UAEXPAVCDC@@PAUCPrintInfo@@@Z 5f846da0 f   viewscrl.obj
 0001:0004602c       ?SetScaleToFitSize@CScrollView@@QAEXUtagSIZE@@@Z 5f84702c f   viewscrl.obj
 0001:00046148       ?SetScrollSizes@CScrollView@@QAEXHUtagSIZE@@ABU2@1@Z 5f847148 f   viewscrl.obj
 0001:000463fd       ?GetScrollPosition@CScrollView@@QBE?AVCPoint@@XZ 5f8473fd f   viewscrl.obj
 0001:000464ec       ?ScrollToPosition@CScrollView@@QAEXUtagPOINT@@@Z 5f8474ec f   viewscrl.obj
 0001:000465ed       ?GetDeviceScrollPosition@CScrollView@@QBE?AVCPoint@@XZ 5f8475ed f   viewscrl.obj
 0001:000466c4       ?GetDeviceScrollSizes@CScrollView@@QBEXAAHAAUtagSIZE@@11@Z 5f8476c4 f   viewscrl.obj
 0001:0004672a       ?ScrollToDevicePosition@CScrollView@@IAEXUtagPOINT@@@Z 5f84772a f   viewscrl.obj
 0001:000467d3       ?FillOutsideRect@CScrollView@@QAEXPAVCDC@@PAVCBrush@@@Z 5f8477d3 f   viewscrl.obj
 0001:000468b1       ?ResizeParentToFit@CScrollView@@QAEXH@Z 5f8478b1 f   viewscrl.obj
 0001:00046ade       ?OnSize@CScrollView@@QAEXIHH@Z 5f847ade f   viewscrl.obj
 0001:00046b33       ?CenterOnPoint@CScrollView@@IAEXVCPoint@@@Z 5f847b33 f   viewscrl.obj
 0001:00046c5d       ?GetScrollBarSizes@CScrollView@@IAEXAAVCSize@@@Z 5f847c5d f   viewscrl.obj
 0001:00046cf8       ?GetTrueClientSize@CScrollView@@IAEHAAVCSize@@0@Z 5f847cf8 f   viewscrl.obj
 0001:00046de8       ?GetScrollBarState@CScrollView@@IAEXVCSize@@AAV2@1AAVCPoint@@H@Z 5f847de8 f   viewscrl.obj
 0001:00046f5e       ?UpdateBars@CScrollView@@IAEXXZ 5f847f5e f   viewscrl.obj
 0001:0004719a       ?CalcWindowRect@CScrollView@@UAEXPAUtagRECT@@I@Z 5f84819a f   viewscrl.obj
 0001:00047287       ?OnHScroll@CScrollView@@QAEXIIPAVCScrollBar@@@Z 5f848287 f   viewscrl.obj
 0001:000472e5       ?OnVScroll@CScrollView@@QAEXIIPAVCScrollBar@@@Z 5f8482e5 f   viewscrl.obj
 0001:00047346       ?OnMouseWheel@CScrollView@@QAEHIFVCPoint@@@Z 5f848346 f   viewscrl.obj
 0001:0004738d       ?DoMouseWheel@CScrollView@@QAEHIFVCPoint@@@Z 5f84838d f   viewscrl.obj
 0001:000475a4       ?OnScroll@CScrollView@@UAEHIIH@Z 5f8485a4 f   viewscrl.obj
 0001:00047749       ?OnScrollBy@CScrollView@@UAEHVCSize@@H@Z 5f848749 f   viewscrl.obj
 0001:000478d2       ?Dump@CScrollView@@UBEXAAVCDumpContext@@@Z 5f8488d2 f   viewscrl.obj
 0001:00047ab0       ?AssertValid@CScrollView@@UBEXXZ 5f848ab0 f   viewscrl.obj
 0001:00047b50       ??_ECScrollView@@UAEPAXI@Z 5f848b50 f i viewscrl.obj
 0001:00047b50       ??_GCScrollView@@UAEPAXI@Z 5f848b50 f i viewscrl.obj
 0001:00047b80       ?_GetBaseMessageMap@CFormView@@KGPBUAFX_MSGMAP@@XZ 5f848b80 f   viewform.obj
 0001:00047b8a       ?GetMessageMap@CFormView@@MBEPBUAFX_MSGMAP@@XZ 5f848b8a f   viewform.obj
 0001:00047b9a       ??0CFormView@@IAE@PBG@Z    5f848b9a f   viewform.obj
 0001:00047bd8       ??0CFormView@@IAE@I@Z      5f848bd8 f   viewform.obj
 0001:00047c75       ?Create@CFormView@@MAEHPBG0KABUtagRECT@@PAVCWnd@@IPAUCCreateContext@@@Z 5f848c75 f   viewform.obj
 0001:00047e96       ?OnInitialUpdate@CFormView@@UAEXXZ 5f848e96 f   viewform.obj
 0001:00047ed9       ?OnCreate@CFormView@@IAEHPAUtagCREATESTRUCTW@@@Z 5f848ed9 f   viewform.obj
 0001:00047efd       ?OnActivateView@CFormView@@MAEXHPAVCView@@0@Z 5f848efd f   viewform.obj
 0001:00047f2c       ?OnActivateFrame@CFormView@@MAEXIPAVCFrameWnd@@@Z 5f848f2c f   viewform.obj
 0001:00047f47       ?SaveFocusControl@CFormView@@IAEHXZ 5f848f47 f   viewform.obj
 0001:00047f8a       ?OnSetFocus@CFormView@@IAEXPAVCWnd@@@Z 5f848f8a f   viewform.obj
 0001:00047fe1       ?PreTranslateMessage@CFormView@@MAEHPAUtagMSG@@@Z 5f848fe1 f   viewform.obj
 0001:000480df       ?OnDraw@CFormView@@MAEXPAVCDC@@@Z 5f8490df f   viewform.obj
 0001:0004811d       ?HandleInitDialog@CFormView@@IAEJIJ@Z 5f84911d f   viewform.obj
 0001:0004818a       ?SetOccDialogInfo@CFormView@@MAEHPAU_AFX_OCC_DIALOG_INFO@@@Z 5f84918a f   viewform.obj
 0001:000481a5       ?Dump@CFormView@@UBEXAAVCDumpContext@@@Z 5f8491a5 f   viewform.obj
 0001:00048214       ?AssertValid@CFormView@@UBEXXZ 5f849214 f   viewform.obj
 0001:00048230       ??_ECFormView@@UAEPAXI@Z   5f849230 f i viewform.obj
 0001:00048230       ??_GCFormView@@UAEPAXI@Z   5f849230 f i viewform.obj
 0001:00048260       ??1CFormView@@UAE@XZ       5f849260 f i viewform.obj
 0001:00048280       ?OnAppExit@CWinApp@@IAEXXZ 5f849280 f   appui.obj
 0001:000482d0       ?GetOpenDocumentCount@CWinApp@@QAEHXZ 5f8492d0 f   appui2.obj
 0001:00048320       ?AfxFindResourceHandle@@YGPAUHINSTANCE__@@PBG0@Z 5f849320 f   dllinit.obj
 0001:000484eb       ?AfxLoadString@@YGHIPAGI@Z 5f8494eb f   dllinit.obj
 0001:00048750       ??0CMemFile@@QAE@I@Z       5f849750 f   filemem.obj
 0001:000487fc       ??0CMemFile@@QAE@PAEII@Z   5f8497fc f   filemem.obj
 0001:000488ae       ?Attach@CMemFile@@QAEXPAEII@Z 5f8498ae f   filemem.obj
 0001:00048922       ?Detach@CMemFile@@QAEPAEXZ 5f849922 f   filemem.obj
 0001:00048963       ??1CMemFile@@UAE@XZ        5f849963 f   filemem.obj
 0001:00048a0b       ?Alloc@CMemFile@@MAEPAEK@Z 5f849a0b f   filemem.obj
 0001:00048a25       ?Realloc@CMemFile@@MAEPAEPAEK@Z 5f849a25 f   filemem.obj
 0001:00048a43       ?Memcpy@CMemFile@@MAEPAEPAEPBEI@Z 5f849a43 f   filemem.obj
 0001:00048afd       ?Free@CMemFile@@MAEXPAE@Z  5f849afd f   filemem.obj
 0001:00048b3a       ?GetPosition@CMemFile@@UBEKXZ 5f849b3a f   filemem.obj
 0001:00048b5b       ?GrowFile@CMemFile@@MAEXK@Z 5f849b5b f   filemem.obj
 0001:00048c45       ?SetLength@CMemFile@@UAEXK@Z 5f849c45 f   filemem.obj
 0001:00048caf       ?Read@CMemFile@@UAEIPAXI@Z 5f849caf f   filemem.obj
 0001:00048db0       ?Write@CMemFile@@UAEXPBXI@Z 5f849db0 f   filemem.obj
 0001:00048edb       ?Seek@CMemFile@@UAEJJI@Z   5f849edb f   filemem.obj
 0001:00048fa3       ?Flush@CMemFile@@UAEXXZ    5f849fa3 f   filemem.obj
 0001:00048fc1       ?Close@CMemFile@@UAEXXZ    5f849fc1 f   filemem.obj
 0001:0004909e       ?Abort@CMemFile@@UAEXXZ    5f84a09e f   filemem.obj
 0001:000490c7       ?LockRange@CMemFile@@UAEXKK@Z 5f84a0c7 f   filemem.obj
 0001:000490ec       ?UnlockRange@CMemFile@@UAEXKK@Z 5f84a0ec f   filemem.obj
 0001:00049111       ?Duplicate@CMemFile@@UBEPAVCFile@@XZ 5f84a111 f   filemem.obj
 0001:00049136       ?GetBufferPtr@CMemFile@@UAEIIIPAPAX0@Z 5f84a136 f   filemem.obj
 0001:00049351       ?Dump@CMemFile@@UBEXAAVCDumpContext@@@Z 5f84a351 f   filemem.obj
 0001:000493e3       ?AssertValid@CMemFile@@UBEXXZ 5f84a3e3 f   filemem.obj
 0001:00049470       ?OnHelp@CWnd@@QAEXXZ       5f84a470 f   winfrmx.obj
 0001:0004954a       ?OnHelp@CFrameWnd@@IAEXXZ  5f84a54a f   winfrmx.obj
 0001:00049595       ?OnHelpIndex@CWnd@@QAEXXZ  5f84a595 f   winfrmx.obj
 0001:000495bc       ?OnHelpFinder@CWnd@@QAEXXZ 5f84a5bc f   winfrmx.obj
 0001:000495e3       ?OnHelpUsing@CWnd@@QAEXXZ  5f84a5e3 f   winfrmx.obj
 0001:0004960a       ?CanEnterHelpMode@CFrameWnd@@QAEHXZ 5f84a60a f   winfrmx.obj
 0001:000496a9       ?OnContextHelp@CFrameWnd@@QAEXXZ 5f84a6a9 f   winfrmx.obj
 0001:0004995a       ?SetHelpCapture@CFrameWnd@@IAEPAUHWND__@@UtagPOINT@@PAH@Z 5f84a95a f   winfrmx.obj
 0001:00049ab7       ?_AfxMapClientArea@@YGKPAUHWND__@@UtagPOINT@@@Z 5f84aab7 f   winfrmx.obj
 0001:00049b85       ?_AfxMapNonClientArea@@YGKH@Z 5f84ab85 f   winfrmx.obj
 0001:00049bcb       ?ProcessHelpMsg@CFrameWnd@@IAEHAAUtagMSG@@PAK@Z 5f84abcb f   winfrmx.obj
 0001:00049fc0       ?_GetBaseMessageMap@CControlBar@@KGPBUAFX_MSGMAP@@XZ 5f84afc0 f   barcore.obj
 0001:00049fca       ?GetMessageMap@CControlBar@@MBEPBUAFX_MSGMAP@@XZ 5f84afca f   barcore.obj
 0001:00049fda       ??1CControlBar@@UAE@XZ     5f84afda f   barcore.obj
 0001:0004a105       ?PostNcDestroy@CControlBar@@UAEXXZ 5f84b105 f   barcore.obj
 0001:0004a146       ?CalcFixedLayout@CControlBar@@UAE?AVCSize@@HH@Z 5f84b146 f   barcore.obj
 0001:0004a1b2       ?CalcDynamicLayout@CControlBar@@UAE?AVCSize@@HK@Z 5f84b1b2 f   barcore.obj
 0001:0004a1f1       ?IsDockBar@CControlBar@@UBEHXZ 5f84b1f1 f   barcore.obj
 0001:0004a1fe       ?ResetTimer@CControlBar@@QAEXII@Z 5f84b1fe f   barcore.obj
 0001:0004a25b       ?OnTimer@CControlBar@@QAEXI@Z 5f84b25b f   barcore.obj
 0001:0004a416       ?SetStatusText@CControlBar@@UAEHH@Z 5f84b416 f   barcore.obj
 0001:0004a4f5       ?PreTranslateMessage@CControlBar@@UAEHPAUtagMSG@@@Z 5f84b4f5 f   barcore.obj
 0001:0004a79b       ?WindowProc@CControlBar@@UAEJIIJ@Z 5f84b79b f   barcore.obj
 0001:0004a9d2       ?OnHelpHitTest@CControlBar@@QAEJIJ@Z 5f84b9d2 f   barcore.obj
 0001:0004aa55       ?OnWindowPosChanging@CControlBar@@QAEXPAUtagWINDOWPOS@@@Z 5f84ba55 f   barcore.obj
 0001:0004ab9f       ?OnCreate@CControlBar@@QAEHPAUtagCREATESTRUCTW@@@Z 5f84bb9f f   barcore.obj
 0001:0004ac12       ?OnDestroy@CControlBar@@QAEXXZ 5f84bc12 f   barcore.obj
 0001:0004ac9b       ?DestroyWindow@CControlBar@@UAEHXZ 5f84bc9b f   barcore.obj
 0001:0004acdd       ?OnMouseActivate@CControlBar@@QAEHPAVCWnd@@II@Z 5f84bcdd f   barcore.obj
 0001:0004ad19       ?OnPaint@CControlBar@@QAEXXZ 5f84bd19 f   barcore.obj
 0001:0004ad8b       ?EraseNonClient@CControlBar@@QAEXXZ 5f84bd8b f   barcore.obj
 0001:0004ae96       ?OnCtlColor@CControlBar@@QAEPAUHBRUSH__@@PAVCDC@@PAVCWnd@@I@Z 5f84be96 f   barcore.obj
 0001:0004aef4       ?OnLButtonDown@CControlBar@@QAEXIVCPoint@@@Z 5f84bef4 f   barcore.obj
 0001:0004af87       ?OnLButtonDblClk@CControlBar@@QAEXIVCPoint@@@Z 5f84bf87 f   barcore.obj
 0001:0004b007       ?OnIdleUpdateCmdUI@CControlBar@@QAEJIJ@Z 5f84c007 f   barcore.obj
 0001:0004b114       ?OnInitialUpdate@CControlBar@@QAEXXZ 5f84c114 f   barcore.obj
 0001:0004b12b       ?RecalcDelayShow@CControlBar@@UAEKPAUAFX_SIZEPARENTPARAMS@@@Z 5f84c12b f   barcore.obj
 0001:0004b288       ?OnSizeParent@CControlBar@@QAEJIJ@Z 5f84c288 f   barcore.obj
 0001:0004b518       ?DelayShow@CControlBar@@UAEXH@Z 5f84c518 f   barcore.obj
 0001:0004b582       ?IsVisible@CControlBar@@UBEHXZ 5f84c582 f   barcore.obj
 0001:0004b5c5       ?DoPaint@CControlBar@@UAEXPAVCDC@@@Z 5f84c5c5 f   barcore.obj
 0001:0004b633       ?DrawBorders@CControlBar@@QAEXPAVCDC@@AAVCRect@@@Z 5f84c633 f   barcore.obj
 0001:0004b946       ?DrawGripper@CControlBar@@QAEXPAVCDC@@ABVCRect@@@Z 5f84c946 f   barcore.obj
 0001:0004ba01       ?CalcInsideRect@CControlBar@@QBEXAAVCRect@@H@Z 5f84ca01 f   barcore.obj
 0001:0004bb78       ?AssertValid@CControlBar@@UBEXXZ 5f84cb78 f   barcore.obj
 0001:0004bbeb       ?Dump@CControlBar@@UBEXAAVCDumpContext@@@Z 5f84cbeb f   barcore.obj
 0001:0004bcd0       ??_GCDockContext@@QAEPAXI@Z 5f84ccd0 f i barcore.obj
 0001:0004bd00       ?AfxLoadSysColorBitmap@@YGPAUHBITMAP__@@PAUHINSTANCE__@@PAUHRSRC__@@H@Z 5f84cd00 f   bartool.obj
 0001:0004bf61       ?_GetButton@CToolBar@@IBEXHPAU_TBBUTTON@@@Z 5f84cf61 f   bartool.obj
 0001:0004bfc4       ?_SetButton@CToolBar@@IAEXHPAU_TBBUTTON@@@Z 5f84cfc4 f   bartool.obj
 0001:0004c16b       ?CommandToIndex@CToolBar@@QBEHI@Z 5f84d16b f   bartool.obj
 0001:0004c1dd       ?GetItemID@CToolBar@@QBEIH@Z 5f84d1dd f   bartool.obj
 0001:0004c243       ?GetItemRect@CToolBar@@UBEXHPAUtagRECT@@@Z 5f84d243 f   bartool.obj
 0001:0004c2d9       ?Layout@CToolBar@@IAEXXZ   5f84d2d9 f   bartool.obj
 0001:0004c39a       ?GetButtonStyle@CToolBar@@QBEIH@Z 5f84d39a f   bartool.obj
 0001:0004c413       ?SetButtonStyle@CToolBar@@QAEXHI@Z 5f84d413 f   bartool.obj
 0001:0004c4da       ?CalcSize@CToolBar@@IAE?AVCSize@@PAU_TBBUTTON@@H@Z 5f84d4da f   bartool.obj
 0001:0004c7bd       ?WrapToolBar@CToolBar@@IAEHPAU_TBBUTTON@@HH@Z 5f84d7bd f   bartool.obj
 0001:0004ca37       ?SizeToolBar@CToolBar@@IAEXPAU_TBBUTTON@@HHH@Z 5f84da37 f   bartool.obj
 0001:0004cc8d       ?CalcLayout@CToolBar@@IAE?AVCSize@@KH@Z 5f84dc8d f   bartool.obj
 0001:0004d479       ?CalcFixedLayout@CToolBar@@UAE?AVCSize@@HH@Z 5f84e479 f   bartool.obj
 0001:0004d4c8       ?CalcDynamicLayout@CToolBar@@UAE?AVCSize@@HK@Z 5f84e4c8 f   bartool.obj
 0001:0004d55b       ?GetButtonInfo@CToolBar@@QBEXHAAI0AAH@Z 5f84e55b f   bartool.obj
 0001:0004d5e9       ?SetButtonInfo@CToolBar@@QAEXHIIH@Z 5f84e5e9 f   bartool.obj
 0001:0004d681       ?OnToolHitTest@CToolBar@@UBEHVCPoint@@PAUtagTOOLINFOW@@@Z 5f84e681 f   bartool.obj
 0001:0004d845       ?SetButtonText@CToolBar@@QAEHHPBG@Z 5f84e845 f   bartool.obj
 0001:0004d9fc       ?GetButtonText@CToolBar@@QBE?AVCString@@H@Z 5f84e9fc f   bartool.obj
 0001:0004da73       ?GetButtonText@CToolBar@@QBEXHAAVCString@@@Z 5f84ea73 f   bartool.obj
 0001:0004db3f       ?_GetBaseMessageMap@CToolBar@@KGPBUAFX_MSGMAP@@XZ 5f84eb3f f   bartool.obj
 0001:0004db49       ?GetMessageMap@CToolBar@@MBEPBUAFX_MSGMAP@@XZ 5f84eb49 f   bartool.obj
 0001:0004db59       ?OnEraseBkgnd@CToolBar@@IAEHPAVCDC@@@Z 5f84eb59 f   bartool.obj
 0001:0004db6e       ?OnNcHitTest@CToolBar@@IAEIVCPoint@@@Z 5f84eb6e f   bartool.obj
 0001:0004db80       ?OnNcCalcSize@CToolBar@@IAEXHPAUtagNCCALCSIZE_PARAMS@@@Z 5f84eb80 f   bartool.obj
 0001:0004dc6e       ?OnBarStyleChange@CToolBar@@UAEXKK@Z 5f84ec6e f   bartool.obj
 0001:0004dd4d       ?OnNcPaint@CToolBar@@IAEXXZ 5f84ed4d f   bartool.obj
 0001:0004dd60       ?OnWindowPosChanging@CToolBar@@IAEXPAUtagWINDOWPOS@@@Z 5f84ed60 f   bartool.obj
 0001:0004ddbf       ?OnPaint@CToolBar@@IAEXXZ  5f84edbf f   bartool.obj
 0001:0004dde6       ?OnSetButtonSize@CToolBar@@IAEJIJ@Z 5f84ede6 f   bartool.obj
 0001:0004de09       ?OnSetBitmapSize@CToolBar@@IAEJIJ@Z 5f84ee09 f   bartool.obj
 0001:0004de2c       ?OnSetSizeHelper@CToolBar@@IAEJAAVCSize@@J@Z 5f84ee2c f   bartool.obj
 0001:0004dee4       ?OnPreserveZeroBorderHelper@CToolBar@@IAEJIJ@Z 5f84eee4 f   bartool.obj
 0001:0004df7c       ?OnSysColorChange@CToolBar@@IAEXXZ 5f84ef7c f   bartool.obj
 0001:0004dfce       ?Enable@CToolCmdUI@@UAEXH@Z 5f84efce f   bartool.obj
 0001:0004e0d4       ?SetCheck@CToolCmdUI@@UAEXH@Z 5f84f0d4 f   bartool.obj
 0001:0004e200       ?SetText@CToolCmdUI@@UAEXPBG@Z 5f84f200 f   bartool.obj
 0001:0004e20d       ?OnUpdateCmdUI@CToolBar@@UAEXPAVCFrameWnd@@H@Z 5f84f20d f   bartool.obj
 0001:0004e2db       ?AssertValid@CToolBar@@UBEXXZ 5f84f2db f   bartool.obj
 0001:0004e36b       ?Dump@CToolBar@@UBEXAAVCDumpContext@@@Z 5f84f36b f   bartool.obj
 0001:0004e570       ??0_AFX_CONTROLPOS@@QAE@XZ 5f84f570 f i bartool.obj
 0001:0004e590       ??_H@YGXPAXIHP6EX0@Z@Z     5f84f590 f i bartool.obj
 0001:0004e5c0       ??0CToolCmdUI@@QAE@XZ      5f84f5c0 f i bartool.obj
 0001:0004e5e0       ??0CDialogBar@@QAE@XZ      5f84f5e0 f   bardlg.obj
 0001:0004e651       ??1CDialogBar@@UAE@XZ      5f84f651 f   bardlg.obj
 0001:0004e6a2       ?Create@CDialogBar@@QAEHPAVCWnd@@PBGII@Z 5f84f6a2 f   bardlg.obj
 0001:0004e877       ?CalcFixedLayout@CDialogBar@@UAE?AVCSize@@HH@Z 5f84f877 f   bardlg.obj
 0001:0004e8f8       ?OnUpdateCmdUI@CDialogBar@@UAEXPAVCFrameWnd@@H@Z 5f84f8f8 f   bardlg.obj
 0001:0004e915       ?_GetBaseMessageMap@CDialogBar@@KGPBUAFX_MSGMAP@@XZ 5f84f915 f   bardlg.obj
 0001:0004e91f       ?GetMessageMap@CDialogBar@@MBEPBUAFX_MSGMAP@@XZ 5f84f91f f   bardlg.obj
 0001:0004e92f       ?HandleInitDialog@CDialogBar@@IAEJIJ@Z 5f84f92f f   bardlg.obj
 0001:0004e9a8       ?SetOccDialogInfo@CDialogBar@@MAEHPAU_AFX_OCC_DIALOG_INFO@@@Z 5f84f9a8 f   bardlg.obj
 0001:0004e9d0       ?_GetPanePtr@CStatusBar@@IBEPAUAFX_STATUSPANE@@H@Z 5f84f9d0 f i barstat.obj
 0001:0004ea30       ?CommandToIndex@CStatusBar@@QBEHI@Z 5f84fa30 f   barstat.obj
 0001:0004eaa7       ?GetItemID@CStatusBar@@QBEIH@Z 5f84faa7 f   barstat.obj
 0001:0004ead5       ?GetItemRect@CStatusBar@@QBEXHPAUtagRECT@@@Z 5f84fad5 f   barstat.obj
 0001:0004eb57       ?GetPaneStyle@CStatusBar@@QBEIH@Z 5f84fb57 f   barstat.obj
 0001:0004eb73       ?SetPaneStyle@CStatusBar@@QAEXHI@Z 5f84fb73 f   barstat.obj
 0001:0004ebf6       ?GetPaneInfo@CStatusBar@@QBEXHAAI0AAH@Z 5f84fbf6 f   barstat.obj
 0001:0004ec47       ?SetPaneInfo@CStatusBar@@QAEXHIIH@Z 5f84fc47 f   barstat.obj
 0001:0004ed16       ?GetPaneText@CStatusBar@@QBEXHAAVCString@@@Z 5f84fd16 f   barstat.obj
 0001:0004ed56       ?GetPaneText@CStatusBar@@QBE?AVCString@@H@Z 5f84fd56 f   barstat.obj
 0001:0004eda8       ?SetPaneText@CStatusBar@@QAEHHPBGH@Z 5f84fda8 f   barstat.obj
 0001:0004ef5f       ?CalcFixedLayout@CStatusBar@@UAE?AVCSize@@HH@Z 5f84ff5f f   barstat.obj
 0001:0004f125       ?_GetBaseMessageMap@CStatusBar@@KGPBUAFX_MSGMAP@@XZ 5f850125 f   barstat.obj
 0001:0004f12f       ?GetMessageMap@CStatusBar@@MBEPBUAFX_MSGMAP@@XZ 5f85012f f   barstat.obj
 0001:0004f13f       ?OnNcHitTest@CStatusBar@@IAEIVCPoint@@@Z 5f85013f f   barstat.obj
 0001:0004f16b       ?OnNcCalcSize@CStatusBar@@IAEXHPAUtagNCCALCSIZE_PARAMS@@@Z 5f85016b f   barstat.obj
 0001:0004f1fc       ?OnBarStyleChange@CStatusBar@@UAEXKK@Z 5f8501fc f   barstat.obj
 0001:0004f23c       ?OnNcPaint@CStatusBar@@IAEXXZ 5f85023c f   barstat.obj
 0001:0004f24f       ?DrawItem@CStatusBar@@UAEXPAUtagDRAWITEMSTRUCT@@@Z 5f85024f f   barstat.obj
 0001:0004f285       ?OnChildNotify@CStatusBar@@MAEHIIJPAJ@Z 5f850285 f   barstat.obj
 0001:0004f2ef       ?OnPaint@CStatusBar@@IAEXXZ 5f8502ef f   barstat.obj
 0001:0004f30e       ?OnSize@CStatusBar@@IAEXIHH@Z 5f85030e f   barstat.obj
 0001:0004f37f       ?OnWindowPosChanging@CStatusBar@@IAEXPAUtagWINDOWPOS@@@Z 5f85037f f   barstat.obj
 0001:0004f3bb       ?OnSetText@CStatusBar@@IAEJIJ@Z 5f8503bb f   barstat.obj
 0001:0004f43f       ?OnGetText@CStatusBar@@IAEJIJ@Z 5f85043f f   barstat.obj
 0001:0004f520       ?OnGetTextLength@CStatusBar@@IAEJIJ@Z 5f850520 f   barstat.obj
 0001:0004f5ad       ?OnSetMinHeight@CStatusBar@@IAEJIJ@Z 5f8505ad f   barstat.obj
 0001:0004f5d3       ?Enable@CStatusCmdUI@@UAEXH@Z 5f8505d3 f   barstat.obj
 0001:0004f6aa       ?SetCheck@CStatusCmdUI@@UAEXH@Z 5f8506aa f   barstat.obj
 0001:0004f772       ?SetText@CStatusCmdUI@@UAEXPBG@Z 5f850772 f   barstat.obj
 0001:0004f818       ?OnUpdateCmdUI@CStatusBar@@UAEXPAVCFrameWnd@@H@Z 5f850818 f   barstat.obj
 0001:0004f8a3       ?AssertValid@CStatusBar@@UBEXXZ 5f8508a3 f   barstat.obj
 0001:0004f8b6       ?Dump@CStatusBar@@UBEXAAVCDumpContext@@@Z 5f8508b6 f   barstat.obj
 0001:0004f9e0       ??0CStatusCmdUI@@QAE@XZ    5f8509e0 f i barstat.obj
 0001:0004fa00       ?_GetBaseMessageMap@CDockBar@@KGPBUAFX_MSGMAP@@XZ 5f850a00 f   bardock.obj
 0001:0004fa0a       ?GetMessageMap@CDockBar@@MBEPBUAFX_MSGMAP@@XZ 5f850a0a f   bardock.obj
 0001:0004fa1a       ??0CDockBar@@QAE@H@Z       5f850a1a f   bardock.obj
 0001:0004faee       ??1CDockBar@@UAE@XZ        5f850aee f   bardock.obj
 0001:0004fb9c       ?Create@CDockBar@@QAEHPAVCWnd@@KI@Z 5f850b9c f   bardock.obj
 0001:0004fc58       ?IsDockBar@CDockBar@@UBEHXZ 5f850c58 f   bardock.obj
 0001:0004fc68       ?GetDockedCount@CDockBar@@QBEHXZ 5f850c68 f   bardock.obj
 0001:0004fcbf       ?GetDockedVisibleCount@CDockBar@@UBEHXZ 5f850cbf f   bardock.obj
 0001:0004fd3b       ?DockControlBar@CDockBar@@QAEXPAVCControlBar@@PBUtagRECT@@@Z 5f850d3b f   bardock.obj
 0001:00050150       ?ReDockControlBar@CDockBar@@QAEXPAVCControlBar@@PBUtagRECT@@@Z 5f851150 f   bardock.obj
 0001:000504fc       ?RemovePlaceHolder@CDockBar@@QAEXPAVCControlBar@@@Z 5f8514fc f   bardock.obj
 0001:000505a4       ?RemoveControlBar@CDockBar@@QAEHPAVCControlBar@@HH@Z 5f8515a4 f   bardock.obj
 0001:000507d7       ?CalcFixedLayout@CDockBar@@UAE?AVCSize@@HH@Z 5f8517d7 f   bardock.obj
 0001:00051049       ?OnSizeParent@CDockBar@@IAEJIJ@Z 5f852049 f   bardock.obj
 0001:000510f4       ?OnNcCalcSize@CDockBar@@IAEXHPAUtagNCCALCSIZE_PARAMS@@@Z 5f8520f4 f   bardock.obj
 0001:00051166       ?OnNcPaint@CDockBar@@IAEXXZ 5f852166 f   bardock.obj
 0001:00051179       ?DoPaint@CDockBar@@UAEXPAVCDC@@@Z 5f852179 f   bardock.obj
 0001:00051186       ?OnPaint@CDockBar@@IAEXXZ  5f852186 f   bardock.obj
 0001:0005120a       ?OnWindowPosChanging@CDockBar@@IAEXPAUtagWINDOWPOS@@@Z 5f85220a f   bardock.obj
 0001:00051246       ?FindBar@CDockBar@@QAEHPAVCControlBar@@H@Z 5f852246 f   bardock.obj
 0001:000512a5       ?ShowAll@CDockBar@@QAEXH@Z 5f8522a5 f   bardock.obj
 0001:0005130d       ?GetDockedControlBar@CDockBar@@IBEPAVCControlBar@@H@Z 5f85230d f   bardock.obj
 0001:0005134e       ?Insert@CDockBar@@IAEHPAVCControlBar@@VCRect@@VCPoint@@@Z 5f85234e f   bardock.obj
 0001:0005159d       ?OnUpdateCmdUI@CDockBar@@MAEXPAVCFrameWnd@@H@Z 5f85259d f   bardock.obj
 0001:000515aa       ?AssertValid@CDockBar@@UBEXXZ 5f8525aa f   bardock.obj
 0001:00051658       ?Dump@CDockBar@@UBEXAAVCDumpContext@@@Z 5f852658 f   bardock.obj
 0001:000516b7       ?EnableDocking@CControlBar@@QAEXK@Z 5f8526b7 f   bardock.obj
 0001:000517c5       ?_GetBaseMessageMap@CMiniDockFrameWnd@@KGPBUAFX_MSGMAP@@XZ 5f8527c5 f   bardock.obj
 0001:000517cf       ?GetMessageMap@CMiniDockFrameWnd@@MBEPBUAFX_MSGMAP@@XZ 5f8527cf f   bardock.obj
 0001:000517df       ?OnMouseActivate@CMiniDockFrameWnd@@QAEHPAVCWnd@@II@Z 5f8527df f   bardock.obj
 0001:00051813       ??0CMiniDockFrameWnd@@QAE@XZ 5f852813 f   bardock.obj
 0001:0005187c       ?Create@CMiniDockFrameWnd@@UAEHPAVCWnd@@K@Z 5f85287c f   bardock.obj
 0001:00051a51       ?RecalcLayout@CMiniDockFrameWnd@@UAEXH@Z 5f852a51 f   bardock.obj
 0001:00051ab7       ?OnClose@CMiniDockFrameWnd@@QAEXXZ 5f852ab7 f   bardock.obj
 0001:00051ad2       ?OnNcLButtonDown@CMiniDockFrameWnd@@QAEXIVCPoint@@@Z 5f852ad2 f   bardock.obj
 0001:00051d1e       ?OnNcLButtonDblClk@CMiniDockFrameWnd@@QAEXIVCPoint@@@Z 5f852d1e f   bardock.obj
 0001:00051e40       ??_ECDockBar@@UAEPAXI@Z    5f852e40 f i bardock.obj
 0001:00051e40       ??_GCDockBar@@UAEPAXI@Z    5f852e40 f i bardock.obj
 0001:00051e70       ??_ECMiniDockFrameWnd@@UAEPAXI@Z 5f852e70 f i bardock.obj
 0001:00051e70       ??_GCMiniDockFrameWnd@@UAEPAXI@Z 5f852e70 f i bardock.obj
 0001:00051ea0       ??1CMiniDockFrameWnd@@UAE@XZ 5f852ea0 f i bardock.obj
 0001:00051ef0       ?_AfxAdjustRectangle@@YGXAAVCRect@@VCPoint@@@Z 5f852ef0 f   dockcont.obj
 0001:00051f94       ??0CDockContext@@QAE@PAVCControlBar@@@Z 5f852f94 f   dockcont.obj
 0001:0005213c       ??1CDockContext@@QAE@XZ    5f85313c f   dockcont.obj
 0001:0005219b       ?StartDrag@CDockContext@@UAEXVCPoint@@@Z 5f85319b f   dockcont.obj
 0001:00052a8b       ?Move@CDockContext@@QAEXVCPoint@@@Z 5f853a8b f   dockcont.obj
 0001:00052b96       ?OnKey@CDockContext@@QAEXHH@Z 5f853b96 f   dockcont.obj
 0001:00052bd8       ?EndDrag@CDockContext@@QAEXXZ 5f853bd8 f   dockcont.obj
 0001:00052e11       ?StartResize@CDockContext@@UAEXHVCPoint@@@Z 5f853e11 f   dockcont.obj
 0001:00053155       ?Stretch@CDockContext@@QAEXVCPoint@@@Z 5f854155 f   dockcont.obj
 0001:00053407       ?EndResize@CDockContext@@QAEXXZ 5f854407 f   dockcont.obj
 0001:00053476       ?ToggleDocking@CDockContext@@UAEXXZ 5f854476 f   dockcont.obj
 0001:000535f3       ?InitLoop@CDockContext@@QAEXXZ 5f8545f3 f   dockcont.obj
 0001:00053756       ?CancelLoop@CDockContext@@QAEXXZ 5f854756 f   dockcont.obj
 0001:000537ae       ?DrawFocusRect@CDockContext@@QAEXH@Z 5f8547ae f   dockcont.obj
 0001:000539f6       ?UpdateState@CDockContext@@QAEXPAHH@Z 5f8549f6 f   dockcont.obj
 0001:00053a8c       ?CanDock@CDockContext@@QAEKXZ 5f854a8c f   dockcont.obj
 0001:00053cf8       ?GetDockBar@CDockContext@@QAEPAVCDockBar@@K@Z 5f854cf8 f   dockcont.obj
 0001:00053e34       ?Track@CDockContext@@QAEHXZ 5f854e34 f   dockcont.obj
 0001:00053ff0       ??0CControlBarInfo@@QAE@XZ 5f854ff0 f   dockstat.obj
 0001:00054108       ?Serialize@CControlBarInfo@@QAEXAAVCArchive@@PAVCDockState@@@Z 5f855108 f   dockstat.obj
 0001:000543e0       ?LoadState@CControlBarInfo@@QAEHPBGHPAVCDockState@@@Z 5f8553e0 f   dockstat.obj
 0001:00054758       ?SaveState@CControlBarInfo@@QAEHPBGH@Z 5f855758 f   dockstat.obj
 0001:00054b21       ??0CDockState@@QAE@XZ      5f855b21 f   dockstat.obj
 0001:00054c2f       ??1CDockState@@UAE@XZ      5f855c2f f   dockstat.obj
 0001:00054ce3       ?Serialize@CDockState@@UAEXAAVCArchive@@@Z 5f855ce3 f   dockstat.obj
 0001:00054efa       ?LoadState@CDockState@@QAEXPBG@Z 5f855efa f   dockstat.obj
 0001:00055075       ?SaveState@CDockState@@QAEXPBG@Z 5f856075 f   dockstat.obj
 0001:000551bf       ?Clear@CDockState@@QAEXXZ  5f8561bf f   dockstat.obj
 0001:00055231       ?GetVersion@CDockState@@QAEKXZ 5f856231 f   dockstat.obj
 0001:00055242       ?ScalePoint@CDockState@@QAEXAAVCPoint@@@Z 5f856242 f   dockstat.obj
 0001:000552e0       ?ScaleRectPos@CDockState@@QAEXAAVCRect@@@Z 5f8562e0 f   dockstat.obj
 0001:000553f5       ?GetScreenSize@CDockState@@QAE?AVCSize@@XZ 5f8563f5 f   dockstat.obj
 0001:00055423       ?SetScreenSize@CDockState@@QAEXAAVCSize@@@Z 5f856423 f   dockstat.obj
 0001:00055473       ?LoadBarState@CFrameWnd@@QAEXPBG@Z 5f856473 f   dockstat.obj
 0001:000554d7       ?SaveBarState@CFrameWnd@@QBEXPBG@Z 5f8564d7 f   dockstat.obj
 0001:0005553b       ?SetDockState@CFrameWnd@@QAEXABVCDockState@@@Z 5f85653b f   dockstat.obj
 0001:00055882       ?GetDockState@CFrameWnd@@QBEXAAVCDockState@@@Z 5f856882 f   dockstat.obj
 0001:00055973       ?GetBarInfo@CControlBar@@QAEXPAVCControlBarInfo@@@Z 5f856973 f   dockstat.obj
 0001:00055ad2       ?SetBarInfo@CControlBar@@QAEXPAVCControlBarInfo@@PAVCFrameWnd@@@Z 5f856ad2 f   dockstat.obj
 0001:00055c12       ?GetBarInfo@CDockBar@@QAEXPAVCControlBarInfo@@@Z 5f856c12 f   dockstat.obj
 0001:00055d52       ?SetBarInfo@CDockBar@@QAEXPAVCControlBarInfo@@PAVCFrameWnd@@@Z 5f856d52 f   dockstat.obj
 0001:000560f0       ??_GCControlBarInfo@@QAEPAXI@Z 5f8570f0 f i dockstat.obj
 0001:00056120       ??1CControlBarInfo@@QAE@XZ 5f857120 f i dockstat.obj
 0001:00056140       ?_GetBaseMessageMap@CReBar@@KGPBUAFX_MSGMAP@@XZ 5f857140 f   barcool.obj
 0001:0005614a       ?GetMessageMap@CReBar@@MBEPBUAFX_MSGMAP@@XZ 5f85714a f   barcool.obj
 0001:0005615a       ??0CReBar@@QAE@XZ          5f85715a f   barcool.obj
 0001:000561b6       ?OnRecalcParent@CReBar@@IAEXXZ 5f8571b6 f   barcool.obj
 0001:00056201       ?OnHeightChange@CReBar@@IAEXPAUtagNMHDR@@PAJ@Z 5f857201 f   barcool.obj
 0001:00056259       ?OnShowBand@CReBar@@IAEJIJ@Z 5f857259 f   barcool.obj
 0001:0005635d       ?_AddBar@CReBar@@IAEHPAVCWnd@@PAUtagREBARBANDINFOW@@@Z 5f85735d f   barcool.obj
 0001:00056515       ?AddBar@CReBar@@QAEHPAVCWnd@@PBGPAVCBitmap@@K@Z 5f857515 f   barcool.obj
 0001:0005656f       ?AddBar@CReBar@@QAEHPAVCWnd@@KKPBGK@Z 5f85756f f   barcool.obj
 0001:000565bb       ?CalcFixedLayout@CReBar@@UAE?AVCSize@@HH@Z 5f8575bb f   barcool.obj
 0001:000568f6       ?CalcDynamicLayout@CReBar@@UAE?AVCSize@@HK@Z 5f8578f6 f   barcool.obj
 0001:00056969       ?Create@CReBar@@QAEHPAVCWnd@@KKI@Z 5f857969 f   barcool.obj
 0001:00056a94       ?OnUpdateCmdUI@CReBar@@UAEXPAVCFrameWnd@@H@Z 5f857a94 f   barcool.obj
 0001:00056ab1       ?OnNcCreate@CReBar@@IAEHPAUtagCREATESTRUCTW@@@Z 5f857ab1 f   barcool.obj
 0001:00056afc       ?OnEraseBkgnd@CReBar@@IAEHPAVCDC@@@Z 5f857afc f   barcool.obj
 0001:00056b11       ?OnNcCalcSize@CReBar@@IAEXHPAUtagNCCALCSIZE_PARAMS@@@Z 5f857b11 f   barcool.obj
 0001:00056b8f       ?OnNcPaint@CReBar@@IAEXXZ  5f857b8f f   barcool.obj
 0001:00056ba2       ?OnPaint@CReBar@@IAEXXZ    5f857ba2 f   barcool.obj
 0001:00056bb5       ?OnToolHitTest@CReBar@@UBEHVCPoint@@PAUtagTOOLINFOW@@@Z 5f857bb5 f   barcool.obj
 0001:00056c8f       ?WindowProc@CReBar@@MAEJIIJ@Z 5f857c8f f   barcool.obj
 0001:00056cf0       ??_GCReBar@@UAEPAXI@Z      5f857cf0 f i barcool.obj
 0001:00056cf0       ??_ECReBar@@UAEPAXI@Z      5f857cf0 f i barcool.obj
 0001:00056d20       ??1CReBar@@UAE@XZ          5f857d20 f i barcool.obj
 0001:00056d40       ?PrepareEditCtrl@CDataExchange@@QAEPAUHWND__@@H@Z 5f857d40 f   dlgdata.obj
 0001:00056d8e       ?PrepareCtrl@CDataExchange@@QAEPAUHWND__@@H@Z 5f857d8e f   dlgdata.obj
 0001:00056e5f       ?Fail@CDataExchange@@QAEXXZ 5f857e5f f   dlgdata.obj
 0001:00056ed4       ?_AfxSimpleScanf@@YGHPBG0PAD@Z 5f857ed4 f   dlgdata.obj
 0001:00057139       ?_Afx_DDX_TextWithFormat@@YAXPAVCDataExchange@@HPBGIZZ 5f858139 f   dlgdata.obj
 0001:000571c2       ?DDX_Text@@YGXPAVCDataExchange@@HAAE@Z 5f8581c2 f   dlgdata.obj
 0001:00057243       ?DDX_Text@@YGXPAVCDataExchange@@HAAF@Z 5f858243 f   dlgdata.obj
 0001:00057293       ?DDX_Text@@YGXPAVCDataExchange@@HAAH@Z 5f858293 f   dlgdata.obj
 0001:000572e2       ?DDX_Text@@YGXPAVCDataExchange@@HAAI@Z 5f8582e2 f   dlgdata.obj
 0001:00057331       ?DDX_Text@@YGXPAVCDataExchange@@HAAJ@Z 5f858331 f   dlgdata.obj
 0001:00057380       ?DDX_Text@@YGXPAVCDataExchange@@HAAK@Z 5f858380 f   dlgdata.obj
 0001:000573cf       ?DDX_Text@@YGXPAVCDataExchange@@HAAVCString@@@Z 5f8583cf f   dlgdata.obj
 0001:0005743b       ?DDX_Text@@YGXPAVCDataExchange@@HPAGH@Z 5f85843b f   dlgdata.obj
 0001:000574ce       ?DDX_Check@@YGXPAVCDataExchange@@HAAH@Z 5f8584ce f   dlgdata.obj
 0001:0005757c       ?DDX_Radio@@YGXPAVCDataExchange@@HAAH@Z 5f85857c f   dlgdata.obj
 0001:000576e7       ?DDX_LBString@@YGXPAVCDataExchange@@HAAVCString@@@Z 5f8586e7 f   dlgdata.obj
 0001:000577a5       ?DDX_LBStringExact@@YGXPAVCDataExchange@@HAAVCString@@@Z 5f8587a5 f   dlgdata.obj
 0001:00057827       ?DDX_CBString@@YGXPAVCDataExchange@@HAAVCString@@@Z 5f858827 f   dlgdata.obj
 0001:000578d7       ?DDX_CBStringExact@@YGXPAVCDataExchange@@HAAVCString@@@Z 5f8588d7 f   dlgdata.obj
 0001:00057959       ?DDX_LBIndex@@YGXPAVCDataExchange@@HAAH@Z 5f858959 f   dlgdata.obj
 0001:000579ab       ?DDX_CBIndex@@YGXPAVCDataExchange@@HAAH@Z 5f8589ab f   dlgdata.obj
 0001:000579fd       ?DDX_Scroll@@YGXPAVCDataExchange@@HAAH@Z 5f8589fd f   dlgdata.obj
 0001:00057a45       ?DDX_Slider@@YGXPAVCDataExchange@@HAAH@Z 5f858a45 f   dlgdata.obj
 0001:00057a97       ?_AfxFailMinMaxWithFormat@@YGXPAVCDataExchange@@JJPBGI@Z 5f858a97 f   dlgdata.obj
 0001:00057ba0       ?DDV_MinMaxByte@@YGXPAVCDataExchange@@EEE@Z 5f858ba0 f   dlgdata.obj
 0001:00057c2d       ?DDV_MinMaxShort@@YGXPAVCDataExchange@@FFF@Z 5f858c2d f   dlgdata.obj
 0001:00057c95       ?DDV_MinMaxInt@@YGXPAVCDataExchange@@HHH@Z 5f858c95 f   dlgdata.obj
 0001:00057cef       ?DDV_MinMaxLong@@YGXPAVCDataExchange@@JJJ@Z 5f858cef f   dlgdata.obj
 0001:00057d49       ?DDV_MinMaxUInt@@YGXPAVCDataExchange@@III@Z 5f858d49 f   dlgdata.obj
 0001:00057da3       ?DDV_MinMaxDWord@@YGXPAVCDataExchange@@KKK@Z 5f858da3 f   dlgdata.obj
 0001:00057dfd       ?DDV_MinMaxSlider@@YGXPAVCDataExchange@@KKK@Z 5f858dfd f   dlgdata.obj
 0001:00057e9c       ?DDV_MaxChars@@YGXPAVCDataExchange@@ABVCString@@H@Z 5f858e9c f   dlgdata.obj
 0001:00057f99       ?DDX_Control@@YGXPAVCDataExchange@@HAAVCWnd@@@Z 5f858f99 f   dlgdata.obj
 0001:00058048       ?AfxFailMaxChars@@YGXPAVCDataExchange@@H@Z 5f859048 f   dlgdata.obj
 0001:000580de       ?AfxFailRadio@@YGXPAVCDataExchange@@@Z 5f8590de f   dlgdata.obj
 0001:00058160       ?_AfxSimpleFloatParse@@YGHPBGAAN@Z 5f859160 f   dlgfloat.obj
 0001:0005822f       ?AfxTextFloatFormat@@YGXPAVCDataExchange@@HPAXNH@Z 5f85922f f   dlgfloat.obj
 0001:000582f7       ?DDX_Text@@YGXPAVCDataExchange@@HAAM@Z 5f8592f7 f   dlgfloat.obj
 0001:0005831c       ?DDX_Text@@YGXPAVCDataExchange@@HAAN@Z 5f85931c f   dlgfloat.obj
 0001:00058340       ?_AfxFailMinMaxReal@@YGXPAVCDataExchange@@NNHI@Z 5f859340 f   dlgfloat.obj
 0001:00058435       ?DDV_MinMaxFloat@@YGXPAVCDataExchange@@ABMMM@Z 5f859435 f   dlgfloat.obj
 0001:000584a6       ?DDV_MinMaxDouble@@YGXPAVCDataExchange@@ABNNN@Z 5f8594a6 f   dlgfloat.obj
 0001:00058520       ?_AfxAppendFilterSuffix@@YGXAAVCString@@AAUtagOFNW@@PAVCDocTemplate@@PAV1@@Z 5f859520 f   docmgr.obj
 0001:000586e7       ?_GetBaseMessageMap@CNewTypeDlg@@KGPBUAFX_MSGMAP@@XZ 5f8596e7 f   docmgr.obj
 0001:000586f1       ?GetMessageMap@CNewTypeDlg@@MBEPBUAFX_MSGMAP@@XZ 5f8596f1 f   docmgr.obj
 0001:00058701       ?OnInitDialog@CNewTypeDlg@@MAEHXZ 5f859701 f   docmgr.obj
 0001:000588fc       ?OnOK@CNewTypeDlg@@MAEXXZ  5f8598fc f   docmgr.obj
 0001:000589b7       ?AddDocTemplate@CDocManager@@UAEXPAVCDocTemplate@@@Z 5f8599b7 f   docmgr.obj
 0001:00058ab7       ?GetFirstDocTemplatePosition@CDocManager@@UBEPAU__POSITION@@XZ 5f859ab7 f   docmgr.obj
 0001:00058acd       ?GetNextDocTemplate@CDocManager@@UBEPAVCDocTemplate@@AAPAU__POSITION@@@Z 5f859acd f   docmgr.obj
 0001:00058ae9       ?SaveAllModified@CDocManager@@UAEHXZ 5f859ae9 f   docmgr.obj
 0001:00058b6c       ?CloseAllDocuments@CDocManager@@UAEXH@Z 5f859b6c f   docmgr.obj
 0001:00058be8       ?DoPromptFileName@CDocManager@@UAEHAAVCString@@IKHPAVCDocTemplate@@@Z 5f859be8 f   docmgr.obj
 0001:00058e93       ?GetDocumentCount@CDocManager@@IAEHXZ 5f859e93 f   docmgr.obj
 0001:00058f02       ?OnDDECommand@CDocManager@@UAEHPAG@Z 5f859f02 f   docmgr.obj
 0001:00059875       ?OnFileNew@CDocManager@@UAEXXZ 5f85a875 f   docmgr.obj
 0001:000599a7       ?OnFileOpen@CDocManager@@UAEXXZ 5f85a9a7 f   docmgr.obj
 0001:00059a42       ?AssertValid@CDocManager@@UBEXXZ 5f85aa42 f   docmgr.obj
 0001:00059a92       ?Dump@CDocManager@@UBEXAAVCDumpContext@@@Z 5f85aa92 f   docmgr.obj
 0001:00059b20       ??0CNewTypeDlg@@QAE@PAVCPtrList@@@Z 5f85ab20 f i docmgr.obj
 0001:00059b60       ??1CNewTypeDlg@@UAE@XZ     5f85ab60 f i docmgr.obj
 0001:00059b80       ??_GCNewTypeDlg@@UAEPAXI@Z 5f85ab80 f i docmgr.obj
 0001:00059b80       ??_ECNewTypeDlg@@UAEPAXI@Z 5f85ab80 f i docmgr.obj
 0001:00059bb0       ?_GetBaseMessageMap@CSplitterWnd@@KGPBUAFX_MSGMAP@@XZ 5f85abb0 f   winsplit.obj
 0001:00059bba       ?GetMessageMap@CSplitterWnd@@MBEPBUAFX_MSGMAP@@XZ 5f85abba f   winsplit.obj
 0001:00059bca       ??0CSplitterWnd@@QAE@XZ    5f85abca f   winsplit.obj
 0001:00059d56       ??1CSplitterWnd@@UAE@XZ    5f85ad56 f   winsplit.obj
 0001:00059dce       ?Create@CSplitterWnd@@QAEHPAVCWnd@@HHUtagSIZE@@PAUCCreateContext@@KI@Z 5f85adce f   winsplit.obj
 0001:0005a03a       ?CreateStatic@CSplitterWnd@@QAEHPAVCWnd@@HHKI@Z 5f85b03a f   winsplit.obj
 0001:0005a1bc       ?CreateCommon@CSplitterWnd@@IAEHPAVCWnd@@UtagSIZE@@KI@Z 5f85b1bc f   winsplit.obj
 0001:0005a4c3       ?OnNcCreate@CSplitterWnd@@IAEHPAUtagCREATESTRUCTW@@@Z 5f85b4c3 f   winsplit.obj
 0001:0005a51a       ?CreateView@CSplitterWnd@@UAEHHHPAUCRuntimeClass@@UtagSIZE@@PAUCCreateContext@@@Z 5f85b51a f   winsplit.obj
 0001:0005a905       ?CreateScrollBarCtrl@CSplitterWnd@@UAEHKI@Z 5f85b905 f   winsplit.obj
 0001:0005a9ae       ?IdFromRowCol@CSplitterWnd@@QBEHHH@Z 5f85b9ae f   winsplit.obj
 0001:0005aa6e       ?GetPane@CSplitterWnd@@QBEPAVCWnd@@HH@Z 5f85ba6e f   winsplit.obj
 0001:0005aad5       ?IsChildPane@CSplitterWnd@@QAEHPAVCWnd@@PAH1@Z 5f85bad5 f   winsplit.obj
 0001:0005ac07       ?GetRowInfo@CSplitterWnd@@QBEXHAAH0@Z 5f85bc07 f   winsplit.obj
 0001:0005ac87       ?SetRowInfo@CSplitterWnd@@QAEXHHH@Z 5f85bc87 f   winsplit.obj
 0001:0005ad43       ?GetColumnInfo@CSplitterWnd@@QBEXHAAH0@Z 5f85bd43 f   winsplit.obj
 0001:0005adbd       ?SetColumnInfo@CSplitterWnd@@QAEXHHH@Z 5f85bdbd f   winsplit.obj
 0001:0005ae73       ?GetScrollStyle@CSplitterWnd@@QBEKXZ 5f85be73 f   winsplit.obj
 0001:0005aeb3       ?SetScrollStyle@CSplitterWnd@@QAEXK@Z 5f85beb3 f   winsplit.obj
 0001:0005b09b       ?DeleteView@CSplitterWnd@@UAEXHH@Z 5f85c09b f   winsplit.obj
 0001:0005b133       ?OnDrawSplitter@CSplitterWnd@@MAEXPAVCDC@@W4ESplitType@1@ABVCRect@@@Z 5f85c133 f   winsplit.obj
 0001:0005b32e       ?_AfxCanSplitRowCol@@YGHPAUCRowColInfo@CSplitterWnd@@HH@Z 5f85c32e f   winsplit.obj
 0001:0005b41e       ?SplitRow@CSplitterWnd@@UAEHH@Z 5f85c41e f   winsplit.obj
 0001:0005b6ac       ?SplitColumn@CSplitterWnd@@UAEHH@Z 5f85c6ac f   winsplit.obj
 0001:0005b934       ?DeleteRow@CSplitterWnd@@UAEXH@Z 5f85c934 f   winsplit.obj
 0001:0005bb74       ?DeleteColumn@CSplitterWnd@@UAEXH@Z 5f85cb74 f   winsplit.obj
 0001:0005bdb4       ?GetInsideRect@CSplitterWnd@@MBEXAAVCRect@@@Z 5f85cdb4 f   winsplit.obj
 0001:0005be6f       ?StartTracking@CSplitterWnd@@MAEXH@Z 5f85ce6f f   winsplit.obj
 0001:0005c11e       ?TrackRowSize@CSplitterWnd@@MAEXHH@Z 5f85d11e f   winsplit.obj
 0001:0005c26c       ?TrackColumnSize@CSplitterWnd@@MAEXHH@Z 5f85d26c f   winsplit.obj
 0001:0005c3a8       ?StopTracking@CSplitterWnd@@MAEXH@Z 5f85d3a8 f   winsplit.obj
 0001:0005c687       ?GetHitRect@CSplitterWnd@@MAEXHAAVCRect@@@Z 5f85d687 f   winsplit.obj
 0001:0005c9f6       ?HitTest@CSplitterWnd@@MBEHVCPoint@@@Z 5f85d9f6 f   winsplit.obj
 0001:0005cc8b       ?OnInvertTracker@CSplitterWnd@@MAEXABVCRect@@@Z 5f85dc8b f   winsplit.obj
 0001:0005cd8a       ?DoKeyboardSplit@CSplitterWnd@@UAEHXZ 5f85dd8a f   winsplit.obj
 0001:0005cf04       ?OnDisplayChange@CSplitterWnd@@IAEXXZ 5f85df04 f   winsplit.obj
 0001:0005cf35       ?OnSize@CSplitterWnd@@IAEXIHH@Z 5f85df35 f   winsplit.obj
 0001:0005cf76       ?_AfxLayoutRowCol@@YGXPAUCRowColInfo@CSplitterWnd@@HHH@Z 5f85df76 f   winsplit.obj
 0001:0005d261       ?_AfxDeferClientPos@@YGXPAUAFX_SIZEPARENTPARAMS@@PAVCWnd@@HHHHH@Z 5f85e261 f   winsplit.obj
 0001:0005d3e3       ?GetSizingParent@CSplitterWnd@@IAEPAVCWnd@@XZ 5f85e3e3 f   winsplit.obj
 0001:0005d4e5       ?RecalcLayout@CSplitterWnd@@UAEXXZ 5f85e4e5 f   winsplit.obj
 0001:0005daa2       ?DrawAllSplitBars@CSplitterWnd@@MAEXPAVCDC@@HH@Z 5f85eaa2 f   winsplit.obj
 0001:0005dd64       ?OnPaint@CSplitterWnd@@IAEXXZ 5f85ed64 f   winsplit.obj
 0001:0005e0a3       ?OnSetCursor@CSplitterWnd@@IAEHPAVCWnd@@II@Z 5f85f0a3 f   winsplit.obj
 0001:0005e0e5       ?SetSplitCursor@CSplitterWnd@@MAEXH@Z 5f85f0e5 f   winsplit.obj
 0001:0005e2d2       ?OnMouseMove@CSplitterWnd@@IAEXIVCPoint@@@Z 5f85f2d2 f   winsplit.obj
 0001:0005e5be       ?OnLButtonDown@CSplitterWnd@@IAEXIVCPoint@@@Z 5f85f5be f   winsplit.obj
 0001:0005e5fe       ?OnLButtonDblClk@CSplitterWnd@@IAEXIVCPoint@@@Z 5f85f5fe f   winsplit.obj
 0001:0005e7f7       ?OnLButtonUp@CSplitterWnd@@IAEXIVCPoint@@@Z 5f85f7f7 f   winsplit.obj
 0001:0005e814       ?OnCancelMode@CSplitterWnd@@IAEXXZ 5f85f814 f   winsplit.obj
 0001:0005e82f       ?OnKeyDown@CSplitterWnd@@IAEXIII@Z 5f85f82f f   winsplit.obj
 0001:0005ea40       ?OnSysCommand@CSplitterWnd@@IAEXIJ@Z 5f85fa40 f   winsplit.obj
 0001:0005ea96       ?OnCommand@CSplitterWnd@@MAEHIJ@Z 5f85fa96 f   winsplit.obj
 0001:0005eada       ?OnNotify@CSplitterWnd@@MAEHIJPAJ@Z 5f85fada f   winsplit.obj
 0001:0005eb29       ?OnMouseWheel@CSplitterWnd@@IAEHIFVCPoint@@@Z 5f85fb29 f   winsplit.obj
 0001:0005ec36       ?OnHScroll@CSplitterWnd@@IAEXIIPAVCScrollBar@@@Z 5f85fc36 f   winsplit.obj
 0001:0005ed8b       ?OnVScroll@CSplitterWnd@@IAEXIIPAVCScrollBar@@@Z 5f85fd8b f   winsplit.obj
 0001:0005eee0       ?DoScroll@CSplitterWnd@@UAEHPAVCView@@IH@Z 5f85fee0 f   winsplit.obj
 0001:0005f1b9       ?DoScrollBy@CSplitterWnd@@UAEHPAVCView@@VCSize@@H@Z 5f8601b9 f   winsplit.obj
 0001:0005f474       ?CanActivateNext@CSplitterWnd@@UAEHH@Z 5f860474 f   winsplit.obj
 0001:0005f533       ?ActivateNext@CSplitterWnd@@UAEXH@Z 5f860533 f   winsplit.obj
 0001:0005f66e       ?SetActivePane@CSplitterWnd@@UAEXHHPAVCWnd@@@Z 5f86066e f   winsplit.obj
 0001:0005f6fd       ?GetActivePane@CSplitterWnd@@UAEPAVCWnd@@PAH0@Z 5f8606fd f   winsplit.obj
 0001:0005f785       ?AssertValid@CSplitterWnd@@UBEXXZ 5f860785 f   winsplit.obj
 0001:0005f8a6       ?Dump@CSplitterWnd@@UBEXAAVCDumpContext@@@Z 5f8608a6 f   winsplit.obj
 0001:0005fa90       ?HideApplication@CWinApp@@QAEXXZ 5f860a90 f   appui.obj
 0001:0005fae2       ?DoWaitCursor@CWinApp@@UAEXH@Z 5f860ae2 f   appui.obj
 0001:0005fbbb       ?SaveAllModified@CWinApp@@UAEHXZ 5f860bbb f   appui.obj
 0001:0005fbf0       ?AddToRecentFileList@CWinApp@@UAEXPBG@Z 5f860bf0 f   appui.obj
 0001:0005fc7d       ?OpenDocumentFile@CWinApp@@UAEPAVCDocument@@PBG@Z 5f860c7d f   appui.obj
 0001:0005fcce       ?CloseAllDocuments@CWinApp@@QAEXH@Z 5f860cce f   appui.obj
 0001:0005fd02       ?OnUpdateRecentFileMenu@CWinApp@@IAEXPAVCCmdUI@@@Z 5f860d02 f   appui.obj
 0001:0005fd54       ?OnDDECommand@CWinApp@@UAEHPAG@Z 5f860d54 f   appui.obj
 0001:0005fd8c       ?OnOpenRecentFile@CWinApp@@IAEHI@Z 5f860d8c f   appui.obj
 0001:0005fef0       ?EnableModeless@CWinApp@@QAEXH@Z 5f860ef0 f   appui1.obj
 0001:0005ff73       ?DoMessageBox@CWinApp@@UAEHPBGII@Z 5f860f73 f   appui1.obj
 0001:00060154       ?AfxMessageBox@@YGHPBGII@Z 5f861154 f   appui1.obj
 0001:0006019c       ?AfxMessageBox@@YGHIII@Z   5f86119c f   appui1.obj
 0001:00060257       ?GetSafeOwner_@CWnd@@SGPAUHWND__@@PAU2@PAPAU2@@Z 5f861257 f   appui1.obj
 0001:00060349       ?GetRoutingView_@CCmdTarget@@KGPAVCView@@XZ 5f861349 f   appui1.obj
 0001:0006037b       ?GetRoutingFrame_@CCmdTarget@@KGPAVCFrameWnd@@XZ 5f86137b f   appui1.obj
 0001:000603b0       ?AddDocTemplate@CWinApp@@QAEXPAVCDocTemplate@@@Z 5f8613b0 f   appui2.obj
 0001:00060449       ?GetFirstDocTemplatePosition@CWinApp@@QBEPAU__POSITION@@XZ 5f861449 f   appui2.obj
 0001:0006047b       ?GetNextDocTemplate@CWinApp@@QBEPAVCDocTemplate@@AAPAU__POSITION@@@Z 5f86147b f   appui2.obj
 0001:000604d0       ?WriteProfileInt@CWinApp@@QAEHPBG0H@Z 5f8614d0 f   appui3.obj
 0001:000605d5       ?WriteProfileStringW@CWinApp@@QAEHPBG00@Z 5f8615d5 f   appui3.obj
 0001:00060763       ?WriteProfileBinary@CWinApp@@QAEHPBG0PAEI@Z 5f861763 f   appui3.obj
 0001:000608d0       ?OnFileNew@CWinApp@@IAEXXZ 5f8618d0 f   appdlg.obj
 0001:000608fe       ?OnFileOpen@CWinApp@@IAEXXZ 5f8618fe f   appdlg.obj
 0001:00060949       ?DoPromptFileName@CWinApp@@QAEHAAVCString@@IKHPAVCDocTemplate@@@Z 5f861949 f   appdlg.obj
 0001:000609b0       ?AfxFormatStrings@@YGXAAVCString@@IPBQBGH@Z 5f8619b0 f   apphelp.obj
 0001:00060a2e       ?AfxFormatStrings@@YGXAAVCString@@PBGPBQBGH@Z 5f861a2e f   apphelp.obj
 0001:00060cac       ?AfxFormatString1@@YGXAAVCString@@IPBG@Z 5f861cac f   apphelp.obj
 0001:00060cc6       ?AfxFormatString2@@YGXAAVCString@@IPBG1@Z 5f861cc6 f   apphelp.obj
 0001:00060d00       ?OnHelp@CWinApp@@IAEXXZ    5f861d00 f   apphelpx.obj
 0001:00060d80       ?OnHelpIndex@CWinApp@@IAEXXZ 5f861d80 f   apphelpx.obj
 0001:00060d9d       ?OnHelpFinder@CWinApp@@IAEXXZ 5f861d9d f   apphelpx.obj
 0001:00060dba       ?OnHelpUsing@CWinApp@@IAEXXZ 5f861dba f   apphelpx.obj
 0001:00060dd7       ?OnContextHelp@CWinApp@@IAEXXZ 5f861dd7 f   apphelpx.obj
 0001:00060e60       ??0CSharedFile@@QAE@II@Z   5f861e60 f   fileshrd.obj
 0001:00060ea2       ??1CSharedFile@@UAE@XZ     5f861ea2 f   fileshrd.obj
 0001:00060f22       ?SetHandle@CSharedFile@@QAEXPAXH@Z 5f861f22 f   fileshrd.obj
 0001:00060fd9       ?Alloc@CSharedFile@@MAEPAEK@Z 5f861fd9 f   fileshrd.obj
 0001:0006103d       ?Realloc@CSharedFile@@MAEPAEPAEK@Z 5f86203d f   fileshrd.obj
 0001:000610c7       ?Free@CSharedFile@@MAEXPAE@Z 5f8620c7 f   fileshrd.obj
 0001:00061114       ?Detach@CSharedFile@@QAEPAXXZ 5f862114 f   fileshrd.obj
 0001:00061230       ?_GetBaseMessageMap@CFrameWnd@@KGPBUAFX_MSGMAP@@XZ 5f862230 f   winfrm.obj
 0001:0006123a       ?GetMessageMap@CFrameWnd@@MBEPBUAFX_MSGMAP@@XZ 5f86223a f   winfrm.obj
 0001:0006124a       ??0CFrameWnd@@QAE@XZ       5f86224a f   winfrm.obj
 0001:000613e9       ??1CFrameWnd@@UAE@XZ       5f8623e9 f   winfrm.obj
 0001:00061481       ?AddFrameWnd@CFrameWnd@@IAEXXZ 5f862481 f   winfrm.obj
 0001:000614b1       ?RemoveFrameWnd@CFrameWnd@@IAEXXZ 5f8624b1 f   winfrm.obj
 0001:000614e1       ?LoadAccelTable@CFrameWnd@@QAEHPBG@Z 5f8624e1 f   winfrm.obj
 0001:00061567       ?GetDefaultAccelerator@CFrameWnd@@UAEPAUHACCEL__@@XZ 5f862567 f   winfrm.obj
 0001:000615b4       ?PreTranslateMessage@CFrameWnd@@UAEHPAUtagMSG@@@Z 5f8625b4 f   winfrm.obj
 0001:00061688       ?PostNcDestroy@CFrameWnd@@MAEXXZ 5f862688 f   winfrm.obj
 0001:000616c0       ?OnPaletteChanged@CFrameWnd@@IAEXPAVCWnd@@@Z 5f8626c0 f   winfrm.obj
 0001:000616f7       ?OnQueryNewPalette@CFrameWnd@@IAEHXZ 5f8626f7 f   winfrm.obj
 0001:0006172f       ?ExitHelpMode@CFrameWnd@@UAEXXZ 5f86272f f   winfrm.obj
 0001:000617fc       ?OnSetCursor@CFrameWnd@@IAEHPAVCWnd@@II@Z 5f8627fc f   winfrm.obj
 0001:0006185a       ?OnCommandHelp@CFrameWnd@@IAEJIJ@Z 5f86285a f   winfrm.obj
 0001:000618d1       ?OnHelpHitTest@CFrameWnd@@IAEJIJ@Z 5f8628d1 f   winfrm.obj
 0001:000618fc       ?OnCommand@CFrameWnd@@MAEHIJ@Z 5f8628fc f   winfrm.obj
 0001:000619ad       ?AfxIsDescendant@@YGHPAUHWND__@@0@Z 5f8629ad f   winfrm.obj
 0001:00061a2d       ?BeginModalState@CFrameWnd@@UAEXXZ 5f862a2d f   winfrm.obj
 0001:00061c77       ?EndModalState@CFrameWnd@@UAEXXZ 5f862c77 f   winfrm.obj
 0001:00061d95       ?ShowOwnedWindows@CFrameWnd@@QAEXH@Z 5f862d95 f   winfrm.obj
 0001:00061e8a       ?OnEnable@CFrameWnd@@IAEXH@Z 5f862e8a f   winfrm.obj
 0001:00061fba       ?NotifyFloatingWindows@CFrameWnd@@QAEXK@Z 5f862fba f   winfrm.obj
 0001:0006211a       ?PreCreateWindow@CFrameWnd@@MAEHAAUtagCREATESTRUCTW@@@Z 5f86311a f   winfrm.obj
 0001:000621aa       ?Create@CFrameWnd@@QAEHPBG0KABUtagRECT@@PAVCWnd@@0KPAUCCreateContext@@@Z 5f8631aa f   winfrm.obj
 0001:000622a2       ?CreateView@CFrameWnd@@QAEPAVCWnd@@PAUCCreateContext@@I@Z 5f8632a2 f   winfrm.obj
 0001:0006241a       ?OnCreateClient@CFrameWnd@@MAEHPAUtagCREATESTRUCTW@@PAUCCreateContext@@@Z 5f86341a f   winfrm.obj
 0001:00062453       ?OnCreate@CFrameWnd@@IAEHPAUtagCREATESTRUCTW@@@Z 5f863453 f   winfrm.obj
 0001:0006247a       ?OnCreateHelper@CFrameWnd@@IAEHPAUtagCREATESTRUCTW@@PAUCCreateContext@@@Z 5f86347a f   winfrm.obj
 0001:000624f4       ?GetIconWndClass@CFrameWnd@@IAEPBGKI@Z 5f8634f4 f   winfrm.obj
 0001:000625c7       ?LoadFrame@CFrameWnd@@UAEHIKPAVCWnd@@PAUCCreateContext@@@Z 5f8635c7 f   winfrm.obj
 0001:000627b0       ?OnUpdateFrameMenu@CFrameWnd@@UAEXPAUHMENU__@@@Z 5f8637b0 f   winfrm.obj
 0001:0006280d       ?InitialUpdateFrame@CFrameWnd@@QAEXPAVCDocument@@H@Z 5f86380d f   winfrm.obj
 0001:0006292c       ?OnClose@CFrameWnd@@IAEXXZ 5f86392c f   winfrm.obj
 0001:00062aaf       ?OnDestroy@CFrameWnd@@IAEXXZ 5f863aaf f   winfrm.obj
 0001:00062b5f       ?RemoveControlBar@CFrameWnd@@QAEXPAVCControlBar@@@Z 5f863b5f f   winfrm.obj
 0001:00062b97       ?OnCmdMsg@CFrameWnd@@UAEHIHPAXPAUAFX_CMDHANDLERINFO@@@Z 5f863b97 f   winfrm.obj
 0001:00062cbe       ?OnHScroll@CFrameWnd@@IAEXIIPAVCScrollBar@@@Z 5f863cbe f   winfrm.obj
 0001:00062d01       ?OnVScroll@CFrameWnd@@IAEXIIPAVCScrollBar@@@Z 5f863d01 f   winfrm.obj
 0001:00062d44       ?OnActivateTopLevel@CFrameWnd@@IAEJIJ@Z 5f863d44 f   winfrm.obj
 0001:00062e27       ?OnActivate@CFrameWnd@@IAEXIPAVCWnd@@H@Z 5f863e27 f   winfrm.obj
 0001:00062f9e       ?OnNcActivate@CFrameWnd@@IAEHH@Z 5f863f9e f   winfrm.obj
 0001:00062feb       ?OnSysCommand@CFrameWnd@@IAEXIJ@Z 5f863feb f   winfrm.obj
 0001:00063202       ?OnDropFiles@CFrameWnd@@IAEXPAUHDROP__@@@Z 5f864202 f   winfrm.obj
 0001:000632b8       ?OnQueryEndSession@CFrameWnd@@IAEHXZ 5f8642b8 f   winfrm.obj
 0001:000632f3       ?OnEndSession@CFrameWnd@@IAEXH@Z 5f8642f3 f   winfrm.obj
 0001:0006333f       ?OnDDEInitiate@CFrameWnd@@IAEJIJ@Z 5f86433f f   winfrm.obj
 0001:00063500       ?OnDDEExecute@CFrameWnd@@IAEJIJ@Z 5f864500 f   winfrm.obj
 0001:00063628       ?OnDDETerminate@CFrameWnd@@IAEJIJ@Z 5f864628 f   winfrm.obj
 0001:00063651       ?GetActiveView@CFrameWnd@@QBEPAVCView@@XZ 5f864651 f   winfrm.obj
 0001:000636a8       ?SetActiveView@CFrameWnd@@QAEXPAVCView@@H@Z 5f8646a8 f   winfrm.obj
 0001:00063797       ?OnSetFocus@CFrameWnd@@IAEXPAVCWnd@@@Z 5f864797 f   winfrm.obj
 0001:000637cc       ?GetActiveDocument@CFrameWnd@@UAEPAVCDocument@@XZ 5f8647cc f   winfrm.obj
 0001:00063809       ?ShowControlBar@CFrameWnd@@QAEXPAVCControlBar@@HH@Z 5f864809 f   winfrm.obj
 0001:000639ec       ?OnInitMenu@CFrameWnd@@IAEXPAVCMenu@@@Z 5f8649ec f   winfrm.obj
 0001:00063a5d       ?OnInitMenuPopup@CFrameWnd@@IAEXPAVCMenu@@IH@Z 5f864a5d f   winfrm.obj
 0001:00063d52       ?OnMenuSelect@CFrameWnd@@IAEXIIPAUHMENU__@@@Z 5f864d52 f   winfrm.obj
 0001:00063f87       ?GetMessageString@CFrameWnd@@UBEXIAAVCString@@@Z 5f864f87 f   winfrm.obj
 0001:00063ff8       ?OnPopMessageString@CFrameWnd@@IAEJIJ@Z 5f864ff8 f   winfrm.obj
 0001:0006402b       ?OnSetMessageString@CFrameWnd@@IAEJIJ@Z 5f86502b f   winfrm.obj
 0001:0006417a       ?OnHelpPromptAddr@CFrameWnd@@IAEJIJ@Z 5f86517a f   winfrm.obj
 0001:0006418d       ?GetMessageBar@CFrameWnd@@UAEPAVCWnd@@XZ 5f86518d f   winfrm.obj
 0001:000641a7       ?OnEnterIdle@CFrameWnd@@IAEXIPAVCWnd@@@Z 5f8651a7 f   winfrm.obj
 0001:00064226       ?SetMessageText@CFrameWnd@@QAEXPBG@Z 5f865226 f   winfrm.obj
 0001:00064246       ?SetMessageText@CFrameWnd@@QAEXI@Z 5f865246 f   winfrm.obj
 0001:00064266       ?DestroyDockBars@CFrameWnd@@QAEXXZ 5f865266 f   winfrm.obj
 0001:00064383       ?GetControlBar@CFrameWnd@@QAEPAVCControlBar@@I@Z 5f865383 f   winfrm.obj
 0001:0006443f       ?OnUpdateControlBarMenu@CFrameWnd@@QAEXPAVCCmdUI@@@Z 5f86543f f   winfrm.obj
 0001:000644bc       ?OnBarCheck@CFrameWnd@@QAEHI@Z 5f8654bc f   winfrm.obj
 0001:00064537       ?OnToolTipText@CFrameWnd@@IAEHIPAUtagNMHDR@@PAJ@Z 5f865537 f   winfrm.obj
 0001:00064703       ?OnUpdateKeyIndicator@CFrameWnd@@IAEXPAVCCmdUI@@@Z 5f865703 f   winfrm.obj
 0001:000647ec       ?OnUpdateContextHelp@CFrameWnd@@IAEXPAVCCmdUI@@@Z 5f8657ec f   winfrm.obj
 0001:00064825       ?OnUpdateFrameTitle@CFrameWnd@@UAEXH@Z 5f865825 f   winfrm.obj
 0001:000648a8       ?UpdateFrameTitleForDocument@CFrameWnd@@QAEXPBG@Z 5f8658a8 f   winfrm.obj
 0001:000649fb       ?OnSetPreviewMode@CFrameWnd@@UAEXHPAUCPrintPreviewState@@@Z 5f8659fb f   winfrm.obj
 0001:00064da6       ?DelayUpdateFrameMenu@CFrameWnd@@UAEXPAUHMENU__@@@Z 5f865da6 f   winfrm.obj
 0001:00064dd3       ?OnIdleUpdateCmdUI@CFrameWnd@@IAEXXZ 5f865dd3 f   winfrm.obj
 0001:00064ec0       ?GetActiveFrame@CFrameWnd@@UAEPAV1@XZ 5f865ec0 f   winfrm.obj
 0001:00064ece       ?RecalcLayout@CFrameWnd@@UAEXH@Z 5f865ece f   winfrm.obj
 0001:00065018       ?NegotiateBorderSpace@CFrameWnd@@UAEHIPAUtagRECT@@@Z 5f866018 f   winfrm.obj
 0001:0006512e       ?OnSize@CFrameWnd@@IAEXIHH@Z 5f86612e f   winfrm.obj
 0001:00065165       ?OnEraseBkgnd@CFrameWnd@@IAEHPAVCDC@@@Z 5f866165 f   winfrm.obj
 0001:00065191       ?OnRegisteredMouseWheel@CFrameWnd@@IAEJIJ@Z 5f866191 f   winfrm.obj
 0001:00065274       ?ActivateFrame@CFrameWnd@@UAEXH@Z 5f866274 f   winfrm.obj
 0001:000652d9       ?BringToTop@CFrameWnd@@IAEXH@Z 5f8662d9 f   winfrm.obj
 0001:00065320       ?AssertValid@CFrameWnd@@UBEXXZ 5f866320 f   winfrm.obj
 0001:00065358       ?Dump@CFrameWnd@@UBEXAAVCDumpContext@@@Z 5f866358 f   winfrm.obj
 0001:00065447       ?GetDockingFrame@CControlBar@@QBEPAVCFrameWnd@@XZ 5f866447 f   winfrm.obj
 0001:000654c2       ?IsFloating@CControlBar@@QBEHXZ 5f8664c2 f   winfrm.obj
 0001:00065520       ?CreateFloatingFrame@CFrameWnd@@QAEPAVCMiniDockFrameWnd@@K@Z 5f866520 f   winfrm2.obj
 0001:000655c5       ?EnableDocking@CFrameWnd@@QAEXK@Z 5f8665c5 f   winfrm2.obj
 0001:000656fc       ?DockControlBar@CFrameWnd@@QAEXPAVCControlBar@@IPBUtagRECT@@@Z 5f8666fc f   winfrm2.obj
 0001:00065743       ?DockControlBar@CFrameWnd@@QAEXPAVCControlBar@@PAVCDockBar@@PBUtagRECT@@@Z 5f866743 f   winfrm2.obj
 0001:00065885       ?ReDockControlBar@CFrameWnd@@QAEXPAVCControlBar@@PAVCDockBar@@PBUtagRECT@@@Z 5f866885 f   winfrm2.obj
 0001:00065a33       ?FloatControlBar@CFrameWnd@@QAEXPAVCControlBar@@VCPoint@@K@Z 5f866a33 f   winfrm2.obj
 0001:00065cce       ?CanDock@CFrameWnd@@QAEKVCRect@@KPAPAVCDockBar@@@Z 5f866cce f   winfrm2.obj
 0001:00065e00       ?_GetBaseMessageMap@CMDIFrameWnd@@KGPBUAFX_MSGMAP@@XZ 5f866e00 f   winmdi.obj
 0001:00065e0a       ?GetMessageMap@CMDIFrameWnd@@MBEPBUAFX_MSGMAP@@XZ 5f866e0a f   winmdi.obj
 0001:00065e1a       ??0CMDIFrameWnd@@QAE@XZ    5f866e1a f   winmdi.obj
 0001:00065e46       ?OnCommand@CMDIFrameWnd@@MAEHIJ@Z 5f866e46 f   winmdi.obj
 0001:00065f05       ?OnCmdMsg@CMDIFrameWnd@@UAEHIHPAXPAUAFX_CMDHANDLERINFO@@@Z 5f866f05 f   winmdi.obj
 0001:00065fba       ?OnCommandHelp@CMDIFrameWnd@@IAEJIJ@Z 5f866fba f   winmdi.obj
 0001:0006607c       ?OnCreateClient@CMDIFrameWnd@@UAEHPAUtagCREATESTRUCTW@@PAUCCreateContext@@@Z 5f86707c f   winmdi.obj
 0001:00066143       ?CreateClient@CMDIFrameWnd@@UAEHPAUtagCREATESTRUCTW@@PAVCMenu@@@Z 5f867143 f   winmdi.obj
 0001:00066286       ?DefWindowProcW@CMDIFrameWnd@@MAEJIIJ@Z 5f867286 f   winmdi.obj
 0001:000662b6       ?PreTranslateMessage@CMDIFrameWnd@@UAEHPAUtagMSG@@@Z 5f8672b6 f   winmdi.obj
 0001:000663ea       ?DelayUpdateFrameMenu@CMDIFrameWnd@@UAEXPAUHMENU__@@@Z 5f8673ea f   winmdi.obj
 0001:0006641e       ?OnIdleUpdateCmdUI@CMDIFrameWnd@@IAEXXZ 5f86741e f   winmdi.obj
 0001:0006645d       ?GetActiveFrame@CMDIFrameWnd@@UAEPAVCFrameWnd@@XZ 5f86745d f   winmdi.obj
 0001:00066485       ?PreCreateWindow@CMDIFrameWnd@@UAEHAAUtagCREATESTRUCTW@@@Z 5f867485 f   winmdi.obj
 0001:000664d5       ?LoadFrame@CMDIFrameWnd@@UAEHIKPAVCWnd@@PAUCCreateContext@@@Z 5f8674d5 f   winmdi.obj
 0001:0006655e       ?OnDestroy@CMDIFrameWnd@@IAEXXZ 5f86755e f   winmdi.obj
 0001:000665e2       ?OnSize@CMDIFrameWnd@@IAEXIHH@Z 5f8675e2 f   winmdi.obj
 0001:00066605       ?OnMenuChar@CMDIFrameWnd@@IAEJIIPAVCMenu@@@Z 5f867605 f   winmdi.obj
 0001:00066630       ?MDIGetActive@CMDIFrameWnd@@QBEPAVCMDIChildWnd@@PAH@Z 5f867630 f   winmdi.obj
 0001:000666fe       ?CreateNewChild@CMDIFrameWnd@@QAEPAVCMDIChildWnd@@PAUCRuntimeClass@@IPAUHMENU__@@PAUHACCEL__@@@Z 5f8676fe f   winmdi.obj
 0001:0006688d       ?AssertValid@CMDIFrameWnd@@UBEXXZ 5f86788d f   winmdi.obj
 0001:00066914       ?Dump@CMDIFrameWnd@@UBEXAAVCDumpContext@@@Z 5f867914 f   winmdi.obj
 0001:00066973       ?_GetBaseMessageMap@CMDIChildWnd@@KGPBUAFX_MSGMAP@@XZ 5f867973 f   winmdi.obj
 0001:0006697d       ?GetMessageMap@CMDIChildWnd@@MBEPBUAFX_MSGMAP@@XZ 5f86797d f   winmdi.obj
 0001:0006698d       ??0CMDIChildWnd@@QAE@XZ    5f86798d f   winmdi.obj
 0001:000669c6       ?DefWindowProcW@CMDIChildWnd@@MAEJIIJ@Z 5f8679c6 f   winmdi.obj
 0001:000669ec       ?DestroyWindow@CMDIChildWnd@@UAEHXZ 5f8679ec f   winmdi.obj
 0001:00066aca       ?PreTranslateMessage@CMDIChildWnd@@UAEHPAUtagMSG@@@Z 5f867aca f   winmdi.obj
 0001:00066b77       ?PreCreateWindow@CMDIChildWnd@@UAEHAAUtagCREATESTRUCTW@@@Z 5f867b77 f   winmdi.obj
 0001:00066bc0       ?Create@CMDIChildWnd@@UAEHPBG0KABUtagRECT@@PAVCMDIFrameWnd@@PAUCCreateContext@@@Z 5f867bc0 f   winmdi.obj
 0001:00066e78       ?LoadFrame@CMDIChildWnd@@UAEHIKPAVCWnd@@PAUCCreateContext@@@Z 5f867e78 f   winmdi.obj
 0001:00067120       ?OnSize@CMDIChildWnd@@IAEXIHH@Z 5f868120 f   winmdi.obj
 0001:0006715e       ?UpdateClientEdge@CMDIChildWnd@@IAEHPAUtagRECT@@@Z 5f86815e f   winmdi.obj
 0001:00067277       ?OnWindowPosChanging@CMDIChildWnd@@IAEXPAUtagWINDOWPOS@@@Z 5f868277 f   winmdi.obj
 0001:0006732b       ?OnDestroy@CMDIChildWnd@@IAEXXZ 5f86832b f   winmdi.obj
 0001:00067348       ?OnNcActivate@CMDIChildWnd@@IAEHH@Z 5f868348 f   winmdi.obj
 0001:00067361       ?OnMouseActivate@CMDIChildWnd@@IAEHPAVCWnd@@II@Z 5f868361 f   winmdi.obj
 0001:000673d6       ?OnToolTipText@CMDIChildWnd@@IAEHIPAUtagNMHDR@@PAJ@Z 5f8683d6 f   winmdi.obj
 0001:0006744a       ?ActivateFrame@CMDIChildWnd@@UAEXH@Z 5f86844a f   winmdi.obj
 0001:0006765e       ?SetHandles@CMDIChildWnd@@QAEXPAUHMENU__@@PAUHACCEL__@@@Z 5f86865e f   winmdi.obj
 0001:00067680       ?AssertValid@CMDIChildWnd@@UBEXXZ 5f868680 f   winmdi.obj
 0001:000676d3       ?Dump@CMDIChildWnd@@UBEXAAVCDumpContext@@@Z 5f8686d3 f   winmdi.obj
 0001:00067717       ?GetWindowMenuPopup@CMDIFrameWnd@@UAEPAUHMENU__@@PAU2@@Z 5f868717 f   winmdi.obj
 0001:000677fc       ?OnUpdateFrameMenu@CMDIFrameWnd@@UAEXPAUHMENU__@@@Z 5f8687fc f   winmdi.obj
 0001:00067862       ?GetMDIFrame@CMDIChildWnd@@QAEPAVCMDIFrameWnd@@XZ 5f868862 f   winmdi.obj
 0001:0006798f       ?GetMessageBar@CMDIChildWnd@@MAEPAVCWnd@@XZ 5f86898f f   winmdi.obj
 0001:000679b5       ?OnUpdateFrameTitle@CMDIChildWnd@@MAEXH@Z 5f8689b5 f   winmdi.obj
 0001:00067ac0       ?OnMDIActivate@CMDIChildWnd@@IAEXHPAVCWnd@@0@Z 5f868ac0 f   winmdi.obj
 0001:00067bdf       ?OnUpdateFrameMenu@CMDIChildWnd@@UAEXHPAVCWnd@@PAUHMENU__@@@Z 5f868bdf f   winmdi.obj
 0001:00067cf5       ?OnNcCreate@CMDIChildWnd@@IAEHPAUtagCREATESTRUCTW@@@Z 5f868cf5 f   winmdi.obj
 0001:00067d64       ?OnCreate@CMDIChildWnd@@IAEHPAUtagCREATESTRUCTW@@@Z 5f868d64 f   winmdi.obj
 0001:00067d94       ?OnUpdateFrameTitle@CMDIFrameWnd@@UAEXH@Z 5f868d94 f   winmdi.obj
 0001:00067ef3       ?OnUpdateMDIWindowCmd@CMDIFrameWnd@@IAEXPAVCCmdUI@@@Z 5f868ef3 f   winmdi.obj
 0001:00067f47       ?OnMDIWindowCmd@CMDIFrameWnd@@IAEHI@Z 5f868f47 f   winmdi.obj
 0001:0006800a       ?OnWindowNew@CMDIFrameWnd@@IAEXXZ 5f86900a f   winmdi.obj
 0001:000680d0       ??1CMDIChildWnd@@UAE@XZ    5f8690d0 f i winmdi.obj
 0001:000680d0       ??1CMDIFrameWnd@@UAE@XZ    5f8690d0 f i winmdi.obj
 0001:000680f0       ??_ECMDIChildWnd@@UAEPAXI@Z 5f8690f0 f i winmdi.obj
 0001:000680f0       ??_ECMDIFrameWnd@@UAEPAXI@Z 5f8690f0 f i winmdi.obj
 0001:000680f0       ??_GCMDIFrameWnd@@UAEPAXI@Z 5f8690f0 f i winmdi.obj
 0001:000680f0       ??_GCMDIChildWnd@@UAEPAXI@Z 5f8690f0 f i winmdi.obj
 0001:00068120       ?_AfxWinminiTerm@@YAXXZ    5f869120 f   winmini.obj
 0001:0006815a       ?_GetBaseMessageMap@CMiniFrameWnd@@KGPBUAFX_MSGMAP@@XZ 5f86915a f   winmini.obj
 0001:00068164       ?GetMessageMap@CMiniFrameWnd@@MBEPBUAFX_MSGMAP@@XZ 5f869164 f   winmini.obj
 0001:00068174       ??0CMiniFrameWnd@@QAE@XZ   5f869174 f   winmini.obj
 0001:000681e4       ?Initialize@CMiniFrameWnd@@SAXXZ 5f8691e4 f   winmini.obj
 0001:000683d4       ??1CMiniFrameWnd@@UAE@XZ   5f8693d4 f   winmini.obj
 0001:00068437       ?Create@CMiniFrameWnd@@QAEHPBG0KABUtagRECT@@PAVCWnd@@I@Z 5f869437 f   winmini.obj
 0001:00068466       ?CreateEx@CMiniFrameWnd@@QAEHKPBG0KABUtagRECT@@PAVCWnd@@I@Z 5f869466 f   winmini.obj
 0001:000684fe       ?OnNcCreate@CMiniFrameWnd@@QAEHPAUtagCREATESTRUCTW@@@Z 5f8694fe f   winmini.obj
 0001:000685d4       ?PreCreateWindow@CMiniFrameWnd@@MAEHAAUtagCREATESTRUCTW@@@Z 5f8695d4 f   winmini.obj
 0001:0006866d       ?OnGetMinMaxInfo@CMiniFrameWnd@@QAEXPAUtagMINMAXINFO@@@Z 5f86966d f   winmini.obj
 0001:000686dc       ?OnNcActivate@CMiniFrameWnd@@QAEHH@Z 5f8696dc f   winmini.obj
 0001:00068753       ?OnNcCalcSize@CMiniFrameWnd@@QAEXHPAUtagNCCALCSIZE_PARAMS@@@Z 5f869753 f   winmini.obj
 0001:000687ec       ?OnNcHitTest@CMiniFrameWnd@@QAEIVCPoint@@@Z 5f8697ec f   winmini.obj
 0001:00068c99       ?OnNcLButtonDown@CMiniFrameWnd@@QAEXIVCPoint@@@Z 5f869c99 f   winmini.obj
 0001:00068cf5       ?OnMouseMove@CMiniFrameWnd@@QAEXIVCPoint@@@Z 5f869cf5 f   winmini.obj
 0001:00068d91       ?OnLButtonUp@CMiniFrameWnd@@QAEXIVCPoint@@@Z 5f869d91 f   winmini.obj
 0001:00068dfe       ?InvertSysMenu@CMiniFrameWnd@@IAEXXZ 5f869dfe f   winmini.obj
 0001:00068eae       ?_AfxDrawFrame@@YGXPAVCDC@@PBUtagRECT@@HHAAVCBrush@@@Z 5f869eae f   winmini.obj
 0001:00068f76       ?OnNcPaint@CMiniFrameWnd@@QAEXXZ 5f869f76 f   winmini.obj
 0001:0006961b       ?OnSysCommand@CMiniFrameWnd@@QAEXIJ@Z 5f86a61b f   winmini.obj
 0001:000696a3       ?CalcWindowRect@CMiniFrameWnd@@UAEXPAUtagRECT@@I@Z 5f86a6a3 f   winmini.obj
 0001:0006973e       ?CalcBorders@CMiniFrameWnd@@SGXPAUtagRECT@@KK@Z 5f86a73e f   winmini.obj
 0001:000697d0       ?OnGetText@CMiniFrameWnd@@QAEJIJ@Z 5f86a7d0 f   winmini.obj
 0001:00069834       ?OnGetTextLength@CMiniFrameWnd@@QAEJIJ@Z 5f86a834 f   winmini.obj
 0001:00069862       ?OnSetText@CMiniFrameWnd@@QAEJIJ@Z 5f86a862 f   winmini.obj
 0001:00069953       ?OnFloatStatus@CMiniFrameWnd@@QAEJIJ@Z 5f86a953 f   winmini.obj
 0001:00069ad2       ?OnQueryCenterWnd@CMiniFrameWnd@@QAEJIJ@Z 5f86aad2 f   winmini.obj
 0001:00069b20       ??_GCMiniFrameWnd@@UAEPAXI@Z 5f86ab20 f i winmini.obj
 0001:00069b20       ??_ECMiniFrameWnd@@UAEPAXI@Z 5f86ab20 f i winmini.obj
 0001:00069b50       ?AfxTrackerTerm@@YAXXZ     5f86ab50 f   trckrect.obj
 0001:00069b8a       ??0CRectTracker@@QAE@PBUtagRECT@@I@Z 5f86ab8a f   trckrect.obj
 0001:00069c1d       ?Construct@CRectTracker@@IAEXXZ 5f86ac1d f   trckrect.obj
 0001:00069e8c       ??1CRectTracker@@UAE@XZ    5f86ae8c f   trckrect.obj
 0001:00069ea0       ?Draw@CRectTracker@@QBEXPAVCDC@@@Z 5f86aea0 f   trckrect.obj
 0001:0006a223       ?SetCursor@CRectTracker@@QBEHPAVCWnd@@I@Z 5f86b223 f   trckrect.obj
 0001:0006a305       ?HitTest@CRectTracker@@QBEHVCPoint@@@Z 5f86b305 f   trckrect.obj
 0001:0006a3c5       ?NormalizeHit@CRectTracker@@QBEHH@Z 5f86b3c5 f   trckrect.obj
 0001:0006a462       ?Track@CRectTracker@@QAEHPAVCWnd@@VCPoint@@H0@Z 5f86b462 f   trckrect.obj
 0001:0006a4b3       ?TrackRubberBand@CRectTracker@@QAEHPAVCWnd@@VCPoint@@H@Z 5f86b4b3 f   trckrect.obj
 0001:0006a4fc       ?DrawTrackerRect@CRectTracker@@UAEXPBUtagRECT@@PAVCWnd@@PAVCDC@@1@Z 5f86b4fc f   trckrect.obj
 0001:0006a664       ?AdjustRect@CRectTracker@@UAEXHPAUtagRECT@@@Z 5f86b664 f   trckrect.obj
 0001:0006a84e       ?GetTrueRect@CRectTracker@@QBEXPAUtagRECT@@@Z 5f86b84e f   trckrect.obj
 0001:0006a91e       ?OnChangedRect@CRectTracker@@UAEXABVCRect@@@Z 5f86b91e f   trckrect.obj
 0001:0006a92b       ?GetHandleRect@CRectTracker@@IBEXHPAVCRect@@@Z 5f86b92b f   trckrect.obj
 0001:0006aaae       ?GetHandleSize@CRectTracker@@MBEHPBUtagRECT@@@Z 5f86baae f   trckrect.obj
 0001:0006ab62       ?HitTestHandles@CRectTracker@@IBEHVCPoint@@@Z 5f86bb62 f   trckrect.obj
 0001:0006ac95       ?TrackHandle@CRectTracker@@IAEHHPAVCWnd@@VCPoint@@0@Z 5f86bc95 f   trckrect.obj
 0001:0006b0c6       ?GetModifyPointers@CRectTracker@@IAEXHPAPAH0PAH1@Z 5f86c0c6 f   trckrect.obj
 0001:0006b202       ?GetHandleMask@CRectTracker@@UBEIXZ 5f86c202 f   trckrect.obj
 0001:0006b270       ?Create@CStatic@@QAEHPBGKABUtagRECT@@PAVCWnd@@I@Z 5f86c270 f   winctrl1.obj
 0001:0006b2ab       ??1CStatic@@UAE@XZ         5f86c2ab f   winctrl1.obj
 0001:0006b2fc       ?Create@CButton@@QAEHPBGKABUtagRECT@@PAVCWnd@@I@Z 5f86c2fc f   winctrl1.obj
 0001:0006b337       ??1CButton@@UAE@XZ         5f86c337 f   winctrl1.obj
 0001:0006b388       ?GetCheckedRadioButton@CWnd@@QAEHHH@Z 5f86c388 f   winctrl1.obj
 0001:0006b3c9       ?DrawItem@CButton@@UAEXPAUtagDRAWITEMSTRUCT@@@Z 5f86c3c9 f   winctrl1.obj
 0001:0006b3fc       ?OnChildNotify@CButton@@MAEHIIJPAJ@Z 5f86c3fc f   winctrl1.obj
 0001:0006b463       ?Create@CListBox@@QAEHKABUtagRECT@@PAVCWnd@@I@Z 5f86c463 f   winctrl1.obj
 0001:0006b49c       ??1CListBox@@UAE@XZ        5f86c49c f   winctrl1.obj
 0001:0006b4ed       ?DrawItem@CListBox@@UAEXPAUtagDRAWITEMSTRUCT@@@Z 5f86c4ed f   winctrl1.obj
 0001:0006b520       ?MeasureItem@CListBox@@UAEXPAUtagMEASUREITEMSTRUCT@@@Z 5f86c520 f   winctrl1.obj
 0001:0006b553       ?CompareItem@CListBox@@UAEHPAUtagCOMPAREITEMSTRUCT@@@Z 5f86c553 f   winctrl1.obj
 0001:0006b588       ?DeleteItem@CListBox@@UAEXPAUtagDELETEITEMSTRUCT@@@Z 5f86c588 f   winctrl1.obj
 0001:0006b595       ?VKeyToItem@CListBox@@UAEHII@Z 5f86c595 f   winctrl1.obj
 0001:0006b5aa       ?CharToItem@CListBox@@UAEHII@Z 5f86c5aa f   winctrl1.obj
 0001:0006b5bf       ?OnChildNotify@CListBox@@MAEHIIJPAJ@Z 5f86c5bf f   winctrl1.obj
 0001:0006b782       ?GetText@CListBox@@QBEXHAAVCString@@@Z 5f86c782 f   winctrl1.obj
 0001:0006b7ec       ?ItemFromPoint@CListBox@@QBEIVCPoint@@AAH@Z 5f86c7ec f   winctrl1.obj
 0001:0006b87f       ?Create@CComboBox@@QAEHKABUtagRECT@@PAVCWnd@@I@Z 5f86c87f f   winctrl1.obj
 0001:0006b8b8       ??1CComboBox@@UAE@XZ       5f86c8b8 f   winctrl1.obj
 0001:0006b909       ?DrawItem@CComboBox@@UAEXPAUtagDRAWITEMSTRUCT@@@Z 5f86c909 f   winctrl1.obj
 0001:0006b93f       ?MeasureItem@CComboBox@@UAEXPAUtagMEASUREITEMSTRUCT@@@Z 5f86c93f f   winctrl1.obj
 0001:0006b975       ?CompareItem@CComboBox@@UAEHPAUtagCOMPAREITEMSTRUCT@@@Z 5f86c975 f   winctrl1.obj
 0001:0006b9ad       ?DeleteItem@CComboBox@@UAEXPAUtagDELETEITEMSTRUCT@@@Z 5f86c9ad f   winctrl1.obj
 0001:0006b9ba       ?OnChildNotify@CComboBox@@MAEHIIJPAJ@Z 5f86c9ba f   winctrl1.obj
 0001:0006bb17       ?GetLBText@CComboBox@@QBEXHAAVCString@@@Z 5f86cb17 f   winctrl1.obj
 0001:0006bb81       ?Create@CEdit@@QAEHKABUtagRECT@@PAVCWnd@@I@Z 5f86cb81 f   winctrl1.obj
 0001:0006bbba       ??1CEdit@@UAE@XZ           5f86cbba f   winctrl1.obj
 0001:0006bc0b       ?Create@CScrollBar@@QAEHKABUtagRECT@@PAVCWnd@@I@Z 5f86cc0b f   winctrl1.obj
 0001:0006bc44       ??1CScrollBar@@UAE@XZ      5f86cc44 f   winctrl1.obj
 0001:0006bca0       ??0_AFX_CHECKLIST_STATE@@QAE@XZ 5f86cca0 f   winctrl3.obj
 0001:0006bdb3       ??1_AFX_CHECKLIST_STATE@@UAE@XZ 5f86cdb3 f   winctrl3.obj
 0001:0006bde5       ?_GetBaseMessageMap@CCheckListBox@@KGPBUAFX_MSGMAP@@XZ 5f86cde5 f   winctrl3.obj
 0001:0006bdef       ?GetMessageMap@CCheckListBox@@MBEPBUAFX_MSGMAP@@XZ 5f86cdef f   winctrl3.obj
 0001:0006bdff       ?Create@CCheckListBox@@QAEHKABUtagRECT@@PAVCWnd@@I@Z 5f86cdff f   winctrl3.obj
 0001:0006be37       ?SetCheckStyle@CCheckListBox@@QAEXI@Z 5f86ce37 f   winctrl3.obj
 0001:0006be88       ?SetCheck@CCheckListBox@@QAEXHH@Z 5f86ce88 f   winctrl3.obj
 0001:0006bfcc       ?GetCheck@CCheckListBox@@QAEHH@Z 5f86cfcc f   winctrl3.obj
 0001:0006c043       ?Enable@CCheckListBox@@QAEXHH@Z 5f86d043 f   winctrl3.obj
 0001:0006c16e       ?IsEnabled@CCheckListBox@@QAEHH@Z 5f86d16e f   winctrl3.obj
 0001:0006c1e9       ?OnGetCheckPosition@CCheckListBox@@UAE?AVCRect@@V2@0@Z 5f86d1e9 f   winctrl3.obj
 0001:0006c213       ?DrawItem@CCheckListBox@@UAEXPAUtagDRAWITEMSTRUCT@@@Z 5f86d213 f   winctrl3.obj
 0001:0006c480       ?MeasureItem@CCheckListBox@@UAEXPAUtagMEASUREITEMSTRUCT@@@Z 5f86d480 f   winctrl3.obj
 0001:0006c4bd       ?PreDrawItem@CCheckListBox@@IAEXPAUtagDRAWITEMSTRUCT@@@Z 5f86d4bd f   winctrl3.obj
 0001:0006c8b8       ?PreMeasureItem@CCheckListBox@@IAEXPAUtagMEASUREITEMSTRUCT@@@Z 5f86d8b8 f   winctrl3.obj
 0001:0006c986       ?PreCompareItem@CCheckListBox@@IAEHPAUtagCOMPAREITEMSTRUCT@@@Z 5f86d986 f   winctrl3.obj
 0001:0006c9ef       ?PreDeleteItem@CCheckListBox@@IAEXPAUtagDELETEITEMSTRUCT@@@Z 5f86d9ef f   winctrl3.obj
 0001:0006ca7d       ?OnChildNotify@CCheckListBox@@MAEHIIJPAJ@Z 5f86da7d f   winctrl3.obj
 0001:0006cbbf       ?PreSubclassWindow@CCheckListBox@@MAEXXZ 5f86dbbf f   winctrl3.obj
 0001:0006cc01       ?CalcMinimumItemHeight@CCheckListBox@@IAEHXZ 5f86dc01 f   winctrl3.obj
 0001:0006cd08       ?InvalidateCheck@CCheckListBox@@IAEXH@Z 5f86dd08 f   winctrl3.obj
 0001:0006cd64       ?InvalidateItem@CCheckListBox@@IAEXH@Z 5f86dd64 f   winctrl3.obj
 0001:0006cda3       ?CheckFromPoint@CCheckListBox@@IAEHVCPoint@@AAH@Z 5f86dda3 f   winctrl3.obj
 0001:0006cebe       ?SetSelectionCheck@CCheckListBox@@IAEXH@Z 5f86debe f   winctrl3.obj
 0001:0006cf68       ?OnLButtonDown@CCheckListBox@@IAEXIVCPoint@@@Z 5f86df68 f   winctrl3.obj
 0001:0006d0d6       ?OnLButtonDblClk@CCheckListBox@@IAEXIVCPoint@@@Z 5f86e0d6 f   winctrl3.obj
 0001:0006d129       ?OnKeyDown@CCheckListBox@@IAEXIII@Z 5f86e129 f   winctrl3.obj
 0001:0006d35b       ?OnCreate@CCheckListBox@@IAEHPAUtagCREATESTRUCTW@@@Z 5f86e35b f   winctrl3.obj
 0001:0006d3a3       ?OnSetFont@CCheckListBox@@IAEJIJ@Z 5f86e3a3 f   winctrl3.obj
 0001:0006d3dd       ?OnLBAddString@CCheckListBox@@IAEJIJ@Z 5f86e3dd f   winctrl3.obj
 0001:0006d4ba       ?OnLBFindString@CCheckListBox@@IAEJIJ@Z 5f86e4ba f   winctrl3.obj
 0001:0006d53b       ?OnLBFindStringExact@CCheckListBox@@IAEJIJ@Z 5f86e53b f   winctrl3.obj
 0001:0006d5bc       ?OnLBGetItemData@CCheckListBox@@IAEJIJ@Z 5f86e5bc f   winctrl3.obj
 0001:0006d60b       ?OnLBGetText@CCheckListBox@@IAEJIJ@Z 5f86e60b f   winctrl3.obj
 0001:0006d66a       ?OnLBInsertString@CCheckListBox@@IAEJIJ@Z 5f86e66a f   winctrl3.obj
 0001:0006d747       ?OnLBSelectString@CCheckListBox@@IAEJIJ@Z 5f86e747 f   winctrl3.obj
 0001:0006d7d4       ?OnLBSetItemData@CCheckListBox@@IAEJIJ@Z 5f86e7d4 f   winctrl3.obj
 0001:0006d8c1       ?OnLBSetItemHeight@CCheckListBox@@IAEJIJ@Z 5f86e8c1 f   winctrl3.obj
 0001:0006d930       ??_E_AFX_CHECKLIST_STATE@@UAEPAXI@Z 5f86e930 f i winctrl3.obj
 0001:0006d930       ??_G_AFX_CHECKLIST_STATE@@UAEPAXI@Z 5f86e930 f i winctrl3.obj
 0001:0006d960       ??0AFX_CHECK_DATA@@QAE@XZ  5f86e960 f i winctrl3.obj
 0001:0006d990       ?AfxPropPageCallback@@YGIPAUHWND__@@IPAU_PROPSHEETPAGEW@@@Z 5f86e990 f   dlgprop.obj
 0001:0006dabc       ?_GetBaseMessageMap@CPropertyPage@@KGPBUAFX_MSGMAP@@XZ 5f86eabc f   dlgprop.obj
 0001:0006dac6       ?GetMessageMap@CPropertyPage@@MBEPBUAFX_MSGMAP@@XZ 5f86eac6 f   dlgprop.obj
 0001:0006dad6       ??0CPropertyPage@@QAE@II@Z 5f86ead6 f   dlgprop.obj
 0001:0006db6e       ??0CPropertyPage@@QAE@PBGI@Z 5f86eb6e f   dlgprop.obj
 0001:0006dc0a       ?Construct@CPropertyPage@@QAEXII@Z 5f86ec0a f   dlgprop.obj
 0001:0006dc50       ?Construct@CPropertyPage@@QAEXPBGI@Z 5f86ec50 f   dlgprop.obj
 0001:0006dcad       ??0CPropertyPage@@QAE@XZ   5f86ecad f   dlgprop.obj
 0001:0006dd17       ?CommonConstruct@CPropertyPage@@IAEXPBGI@Z 5f86ed17 f   dlgprop.obj
 0001:0006de3a       ??1CPropertyPage@@UAE@XZ   5f86ee3a f   dlgprop.obj
 0001:0006deb3       ?Cleanup@CPropertyPage@@IAEXXZ 5f86eeb3 f   dlgprop.obj
 0001:0006df09       ?_AfxChangePropPageFont@@YGPAUDLGTEMPLATE@@PBU1@H@Z 5f86ef09 f   dlgprop.obj
 0001:0006e047       ?InitDialogInfo@CPropertyPage@@IAEPBUDLGTEMPLATE@@PBU2@@Z 5f86f047 f   dlgprop.obj
 0001:0006e093       ?PreProcessPageTemplate@CPropertyPage@@IAEXAAU_PROPSHEETPAGEW@@H@Z 5f86f093 f   dlgprop.obj
 0001:0006e269       ?CancelToClose@CPropertyPage@@QAEXXZ 5f86f269 f   dlgprop.obj
 0001:0006e2e3       ?SetModified@CPropertyPage@@QAEXH@Z 5f86f2e3 f   dlgprop.obj
 0001:0006e396       ?QuerySiblings@CPropertyPage@@QAEJIJ@Z 5f86f396 f   dlgprop.obj
 0001:0006e416       ?OnApply@CPropertyPage@@UAEHXZ 5f86f416 f   dlgprop.obj
 0001:0006e447       ?OnReset@CPropertyPage@@UAEXXZ 5f86f447 f   dlgprop.obj
 0001:0006e473       ?OnOK@CPropertyPage@@UAEXXZ 5f86f473 f   dlgprop.obj
 0001:0006e491       ?OnCancel@CPropertyPage@@UAEXXZ 5f86f491 f   dlgprop.obj
 0001:0006e4af       ?OnSetActive@CPropertyPage@@UAEHXZ 5f86f4af f   dlgprop.obj
 0001:0006e4f7       ?OnKillActive@CPropertyPage@@UAEHXZ 5f86f4f7 f   dlgprop.obj
 0001:0006e53e       ?OnQueryCancel@CPropertyPage@@UAEHXZ 5f86f53e f   dlgprop.obj
 0001:0006e54e       ?OnWizardBack@CPropertyPage@@UAEJXZ 5f86f54e f   dlgprop.obj
 0001:0006e55b       ?OnWizardNext@CPropertyPage@@UAEJXZ 5f86f55b f   dlgprop.obj
 0001:0006e568       ?OnWizardFinish@CPropertyPage@@UAEHXZ 5f86f568 f   dlgprop.obj
 0001:0006e578       ?MapWizardResult@CPropertyPage@@IAEJJ@Z 5f86f578 f   dlgprop.obj
 0001:0006e649       ?IsButtonEnabled@CPropertyPage@@IAEHH@Z 5f86f649 f   dlgprop.obj
 0001:0006e687       ?OnNotify@CPropertyPage@@MAEHIJPAJ@Z 5f86f687 f   dlgprop.obj
 0001:0006e8c4       ?PreTranslateMessage@CPropertyPage@@MAEHPAUtagMSG@@@Z 5f86f8c4 f   dlgprop.obj
 0001:0006e903       ?OnCtlColor@CPropertyPage@@IAEPAUHBRUSH__@@PAVCDC@@PAVCWnd@@I@Z 5f86f903 f   dlgprop.obj
 0001:0006e980       ?AssertValid@CPropertyPage@@UBEXXZ 5f86f980 f   dlgprop.obj
 0001:0006ea30       ?Dump@CPropertyPage@@UBEXAAVCDumpContext@@@Z 5f86fa30 f   dlgprop.obj
 0001:0006ea99       ?EndDialog@CPropertyPage@@QAEXH@Z 5f86fa99 f   dlgprop.obj
 0001:0006ead3       ?_GetBaseMessageMap@CPropertySheet@@KGPBUAFX_MSGMAP@@XZ 5f86fad3 f   dlgprop.obj
 0001:0006eadd       ?GetMessageMap@CPropertySheet@@MBEPBUAFX_MSGMAP@@XZ 5f86fadd f   dlgprop.obj
 0001:0006eaed       ?GetPropSheetHeader@CPropertySheet@@QAEPAU_AFX_OLDPROPSHEETHEADER@@XZ 5f86faed f   dlgprop.obj
 0001:0006eb24       ?OnSetDefID@CPropertySheet@@IAEJIJ@Z 5f86fb24 f   dlgprop.obj
 0001:0006ec30       ??0CPropertySheet@@QAE@XZ  5f86fc30 f   dlgprop.obj
 0001:0006eca6       ??0CPropertySheet@@QAE@IPAVCWnd@@I@Z 5f86fca6 f   dlgprop.obj
 0001:0006ed75       ??0CPropertySheet@@QAE@PBGPAVCWnd@@I@Z 5f86fd75 f   dlgprop.obj
 0001:0006ee26       ?Construct@CPropertySheet@@QAEXIPAVCWnd@@I@Z 5f86fe26 f   dlgprop.obj
 0001:0006ee96       ?Construct@CPropertySheet@@QAEXPBGPAVCWnd@@I@Z 5f86fe96 f   dlgprop.obj
 0001:0006eee8       ?CommonConstruct@CPropertySheet@@QAEXPAVCWnd@@I@Z 5f86fee8 f   dlgprop.obj
 0001:0006ef74       ?EnableStackedTabs@CPropertySheet@@QAEXH@Z 5f86ff74 f   dlgprop.obj
 0001:0006ef8d       ?SetTitle@CPropertySheet@@QAEXPBGI@Z 5f86ff8d f   dlgprop.obj
 0001:0006f05c       ??1CPropertySheet@@UAE@XZ  5f87005c f   dlgprop.obj
 0001:0006f0da       ?PreTranslateMessage@CPropertySheet@@UAEHPAUtagMSG@@@Z 5f8700da f   dlgprop.obj
 0001:0006f171       ?OnCmdMsg@CPropertySheet@@UAEHIHPAXPAUAFX_CMDHANDLERINFO@@@Z 5f870171 f   dlgprop.obj
 0001:0006f2c9       ?GetActivePage@CPropertySheet@@QBEPAVCPropertyPage@@XZ 5f8702c9 f   dlgprop.obj
 0001:0006f338       ?ContinueModal@CPropertySheet@@UAEHXZ 5f870338 f   dlgprop.obj
 0001:0006f39d       ?DoModal@CPropertySheet@@UAEHXZ 5f87039d f   dlgprop.obj
 0001:0006f612       ?AfxPropSheetCallback@@YGHPAUHWND__@@IJ@Z 5f870612 f   dlgprop.obj
 0001:0006f6ad       ?Create@CPropertySheet@@QAEHPAVCWnd@@KK@Z 5f8706ad f   dlgprop.obj
 0001:0006f83f       ?BuildPropPageArray@CPropertySheet@@UAEXXZ 5f87083f f   dlgprop.obj
 0001:0006f926       ?GetPageCount@CPropertySheet@@QBEHXZ 5f870926 f   dlgprop.obj
 0001:0006f982       ?GetActiveIndex@CPropertySheet@@QBEHXZ 5f870982 f   dlgprop.obj
 0001:0006f9cb       ?SetActivePage@CPropertySheet@@QAEHH@Z 5f8709cb f   dlgprop.obj
 0001:0006fa09       ?GetPageIndex@CPropertySheet@@QAEHPAVCPropertyPage@@@Z 5f870a09 f   dlgprop.obj
 0001:0006fa52       ?SetActivePage@CPropertySheet@@QAEHPAVCPropertyPage@@@Z 5f870a52 f   dlgprop.obj
 0001:0006fb00       ?AddPage@CPropertySheet@@QAEXPAVCPropertyPage@@@Z 5f870b00 f   dlgprop.obj
 0001:0006fc90       ?RemovePage@CPropertySheet@@QAEXPAVCPropertyPage@@@Z 5f870c90 f   dlgprop.obj
 0001:0006fd3e       ?RemovePage@CPropertySheet@@QAEXH@Z 5f870d3e f   dlgprop.obj
 0001:0006fd8b       ?EndDialog@CPropertySheet@@QAEXH@Z 5f870d8b f   dlgprop.obj
 0001:0006fde1       ?OnClose@CPropertySheet@@IAEXXZ 5f870de1 f   dlgprop.obj
 0001:0006fe17       ?OnSysCommand@CPropertySheet@@IAEXIJ@Z 5f870e17 f   dlgprop.obj
 0001:0006fe6b       ?OnInitDialog@CPropertySheet@@UAEHXZ 5f870e6b f   dlgprop.obj
 0001:00070142       ?OnNcCreate@CPropertySheet@@IAEHPAUtagCREATESTRUCTW@@@Z 5f871142 f   dlgprop.obj
 0001:00070168       ?HandleInitDialog@CPropertySheet@@IAEJIJ@Z 5f871168 f   dlgprop.obj
 0001:0007018b       ?OnCommand@CPropertySheet@@UAEHIJ@Z 5f87118b f   dlgprop.obj
 0001:0007023c       ?OnCommandHelp@CPropertySheet@@IAEJIJ@Z 5f87123c f   dlgprop.obj
 0001:00070299       ?OnCtlColor@CPropertySheet@@IAEPAUHBRUSH__@@PAVCDC@@PAVCWnd@@I@Z 5f871299 f   dlgprop.obj
 0001:00070316       ?AssertValid@CPropertySheet@@UBEXXZ 5f871316 f   dlgprop.obj
 0001:00070389       ?Dump@CPropertySheet@@UBEXAAVCDumpContext@@@Z 5f871389 f   dlgprop.obj
 0001:00070448       ??0CPropertyPageEx@@QAE@IIII@Z 5f871448 f   dlgprop.obj
 0001:000704fe       ??0CPropertyPageEx@@QAE@PBGIII@Z 5f8714fe f   dlgprop.obj
 0001:000705b7       ?Construct@CPropertyPageEx@@QAEXIIII@Z 5f8715b7 f   dlgprop.obj
 0001:00070608       ?Construct@CPropertyPageEx@@QAEXPBGIII@Z 5f871608 f   dlgprop.obj
 0001:00070670       ??0CPropertyPageEx@@QAE@XZ 5f871670 f   dlgprop.obj
 0001:000706f0       ?CommonConstruct@CPropertyPageEx@@IAEXPBGIII@Z 5f8716f0 f   dlgprop.obj
 0001:00070882       ?AssertValid@CPropertyPageEx@@UBEXXZ 5f871882 f   dlgprop.obj
 0001:00070932       ?Dump@CPropertyPageEx@@UBEXAAVCDumpContext@@@Z 5f871932 f   dlgprop.obj
 0001:000709ed       ??0CPropertySheetEx@@QAE@XZ 5f8719ed f   dlgprop.obj
 0001:00070a4b       ??0CPropertySheetEx@@QAE@IPAVCWnd@@IPAUHBITMAP__@@PAUHPALETTE__@@1@Z 5f871a4b f   dlgprop.obj
 0001:00070b08       ??0CPropertySheetEx@@QAE@PBGPAVCWnd@@IPAUHBITMAP__@@PAUHPALETTE__@@2@Z 5f871b08 f   dlgprop.obj
 0001:00070ba7       ?Construct@CPropertySheetEx@@QAEXIPAVCWnd@@IPAUHBITMAP__@@PAUHPALETTE__@@1@Z 5f871ba7 f   dlgprop.obj
 0001:00070c23       ?Construct@CPropertySheetEx@@QAEXPBGPAVCWnd@@IPAUHBITMAP__@@PAUHPALETTE__@@2@Z 5f871c23 f   dlgprop.obj
 0001:00070c81       ?CommonConstruct@CPropertySheetEx@@QAEXPAVCWnd@@IPAUHBITMAP__@@PAUHPALETTE__@@1@Z 5f871c81 f   dlgprop.obj
 0001:00070d9e       ?BuildPropPageArray@CPropertySheetEx@@UAEXXZ 5f871d9e f   dlgprop.obj
 0001:00070f5a       ??1CPropertySheetEx@@UAE@XZ 5f871f5a f   dlgprop.obj
 0001:00070fbd       ?AddPage@CPropertySheetEx@@QAEXPAVCPropertyPageEx@@@Z 5f871fbd f   dlgprop.obj
 0001:000711c0       ?AssertValid@CPropertySheetEx@@UBEXXZ 5f8721c0 f   dlgprop.obj
 0001:00071239       ?Dump@CPropertySheetEx@@UBEXAAVCDumpContext@@@Z 5f872239 f   dlgprop.obj
 0001:00071300       ??_ECPropertyPage@@UAEPAXI@Z 5f872300 f i dlgprop.obj
 0001:00071300       ??_GCPropertyPage@@UAEPAXI@Z 5f872300 f i dlgprop.obj
 0001:00071330       ??_ECPropertySheet@@UAEPAXI@Z 5f872330 f i dlgprop.obj
 0001:00071330       ??_GCPropertySheet@@UAEPAXI@Z 5f872330 f i dlgprop.obj
 0001:00071360       ??_GCPropertyPageEx@@UAEPAXI@Z 5f872360 f i dlgprop.obj
 0001:00071360       ??_ECPropertyPageEx@@UAEPAXI@Z 5f872360 f i dlgprop.obj
 0001:00071390       ??1CPropertyPageEx@@UAE@XZ 5f872390 f i dlgprop.obj
 0001:000713f0       ??_GCPropertySheetEx@@UAEPAXI@Z 5f8723f0 f i dlgprop.obj
 0001:000713f0       ??_ECPropertySheetEx@@UAEPAXI@Z 5f8723f0 f i dlgprop.obj
 0001:00071420       ?AfxWingdixTerm@@YAXXZ     5f872420 f   wingdix.obj
 0001:00071450       ?DPtoHIMETRIC@CDC@@QBEXPAUtagSIZE@@@Z 5f872450 f   wingdix.obj
 0001:00071593       ?HIMETRICtoDP@CDC@@QBEXPAUtagSIZE@@@Z 5f872593 f   wingdix.obj
 0001:000716d6       ?LPtoHIMETRIC@CDC@@QBEXPAUtagSIZE@@@Z 5f8726d6 f   wingdix.obj
 0001:00071729       ?HIMETRICtoLP@CDC@@QBEXPAUtagSIZE@@@Z 5f872729 f   wingdix.obj
 0001:0007177c       ?GetHalftoneBrush@CDC@@SGPAVCBrush@@XZ 5f87277c f   wingdix.obj
 0001:0007180c       ?DrawDragRect@CDC@@QAEXPBUtagRECT@@UtagSIZE@@01PAVCBrush@@2@Z 5f87280c f   wingdix.obj
 0001:00071b56       ?FillSolidRect@CDC@@QAEXPBUtagRECT@@K@Z 5f872b56 f   wingdix.obj
 0001:00071bcd       ?FillSolidRect@CDC@@QAEXHHHHK@Z 5f872bcd f   wingdix.obj
 0001:00071c64       ?Draw3dRect@CDC@@QAEXPBUtagRECT@@KK@Z 5f872c64 f   wingdix.obj
 0001:00071ca7       ?Draw3dRect@CDC@@QAEXHHHHKK@Z 5f872ca7 f   wingdix.obj
 0001:00071d28       ?CreatePointFont@CFont@@QAEHHPBGPAVCDC@@@Z 5f872d28 f   wingdix.obj
 0001:00071da0       ?CreatePointFontIndirect@CFont@@QAEHPBUtagLOGFONTW@@PAVCDC@@@Z 5f872da0 f   wingdix.obj
 0001:00071ec0       ?NormalizeRect@CRect@@QAEXXZ 5f872ec0 f   wingdix.obj
 0001:00071f22       ?InflateRect@CRect@@QAEXPBUtagRECT@@@Z 5f872f22 f   wingdix.obj
 0001:00071f74       ?InflateRect@CRect@@QAEXHHHH@Z 5f872f74 f   wingdix.obj
 0001:00071fbb       ?DeflateRect@CRect@@QAEXPBUtagRECT@@@Z 5f872fbb f   wingdix.obj
 0001:0007200d       ?DeflateRect@CRect@@QAEXHHHH@Z 5f87300d f   wingdix.obj
 0001:00072054       ?MulDiv@CRect@@QBE?AV1@HH@Z 5f873054 f   wingdix.obj
 0001:000720ff       ?AfxEditviewTerm@@YAXXZ    5f8730ff f   viewedit.obj
 0001:0007212f       ?_GetBaseMessageMap@CEditView@@KGPBUAFX_MSGMAP@@XZ 5f87312f f   viewedit.obj
 0001:00072139       ?GetMessageMap@CEditView@@MBEPBUAFX_MSGMAP@@XZ 5f873139 f   viewedit.obj
 0001:00072149       ??0_AFX_EDIT_STATE@@QAE@XZ 5f873149 f   viewedit.obj
 0001:000721b9       ??1_AFX_EDIT_STATE@@UAE@XZ 5f8731b9 f   viewedit.obj
 0001:0007221c       ??0CEditView@@QAE@XZ       5f87321c f   viewedit.obj
 0001:000722ac       ??1CEditView@@UAE@XZ       5f8732ac f   viewedit.obj
 0001:0007236a       ?PreCreateWindow@CEditView@@MAEHAAUtagCREATESTRUCTW@@@Z 5f87336a f   viewedit.obj
 0001:0007238d       ?OnCreate@CEditView@@IAEHPAUtagCREATESTRUCTW@@@Z 5f87338d f   viewedit.obj
 0001:000724e0       ?OnDestroy@CEditView@@IAEXXZ 5f8734e0 f   viewedit.obj
 0001:0007250c       ?CalcWindowRect@CEditView@@MAEXPAUtagRECT@@I@Z 5f87350c f   viewedit.obj
 0001:00072596       ?DeleteContents@CEditView@@UAEXXZ 5f873596 f   viewedit.obj
 0001:000725fa       ?Serialize@CEditView@@UAEXAAVCArchive@@@Z 5f8735fa f   viewedit.obj
 0001:000726bd       ?ReadFromArchive@CEditView@@QAEXAAVCArchive@@I@Z 5f8736bd f   viewedit.obj
 0001:000727ea       ?WriteToArchive@CEditView@@QAEXAAVCArchive@@@Z 5f8737ea f   viewedit.obj
 0001:000728e4       ?SerializeRaw@CEditView@@QAEXAAVCArchive@@@Z 5f8738e4 f   viewedit.obj
 0001:000729ad       ?_AfxEndOfLine@@YGIPBGII@Z 5f8739ad f   viewedit.obj
 0001:00072a2c       ?_AfxNextLine@@YGIPBGII@Z  5f873a2c f   viewedit.obj
 0001:00072ac9       ?_AfxClipLine@@YGIPAVCDC@@QAHHHPBGII@Z 5f873ac9 f   viewedit.obj
 0001:00072d2c       ?OnPreparePrinting@CEditView@@MAEHPAUCPrintInfo@@@Z 5f873d2c f   viewedit.obj
 0001:00072d45       ?OnBeginPrinting@CEditView@@MAEXPAVCDC@@PAUCPrintInfo@@@Z 5f873d45 f   viewedit.obj
 0001:00072f4a       ?PaginateTo@CEditView@@IAEHPAVCDC@@PAUCPrintInfo@@@Z 5f873f4a f   viewedit.obj
 0001:00073181       ?OnPrepareDC@CEditView@@UAEXPAVCDC@@PAUCPrintInfo@@@Z 5f874181 f   viewedit.obj
 0001:0007321e       ?PrintInsideRect@CEditView@@QAEIPAVCDC@@AAUtagRECT@@II@Z 5f87421e f   viewedit.obj
 0001:00073780       ?OnPrint@CEditView@@MAEXPAVCDC@@PAUCPrintInfo@@@Z 5f874780 f   viewedit.obj
 0001:00073942       ?OnEndPrinting@CEditView@@MAEXPAVCDC@@PAUCPrintInfo@@@Z 5f874942 f   viewedit.obj
 0001:0007399a       ?OnUpdateNeedSel@CEditView@@IAEXPAVCCmdUI@@@Z 5f87499a f   viewedit.obj
 0001:000739fc       ?OnUpdateNeedClip@CEditView@@IAEXPAVCCmdUI@@@Z 5f8749fc f   viewedit.obj
 0001:00073a42       ?OnUpdateNeedText@CEditView@@IAEXPAVCCmdUI@@@Z 5f874a42 f   viewedit.obj
 0001:00073a8e       ?OnUpdateNeedFind@CEditView@@IAEXPAVCCmdUI@@@Z 5f874a8e f   viewedit.obj
 0001:00073b09       ?OnUpdateEditUndo@CEditView@@IAEXPAVCCmdUI@@@Z 5f874b09 f   viewedit.obj
 0001:00073b56       ?OnEditChange@CEditView@@IAEHXZ 5f874b56 f   viewedit.obj
 0001:00073ba3       ?OnEditCut@CEditView@@IAEXXZ 5f874ba3 f   viewedit.obj
 0001:00073be3       ?OnEditCopy@CEditView@@IAEXXZ 5f874be3 f   viewedit.obj
 0001:00073c23       ?OnEditPaste@CEditView@@IAEXXZ 5f874c23 f   viewedit.obj
 0001:00073c63       ?OnEditClear@CEditView@@IAEXXZ 5f874c63 f   viewedit.obj
 0001:00073ca3       ?OnEditUndo@CEditView@@IAEXXZ 5f874ca3 f   viewedit.obj
 0001:00073ce3       ?OnEditSelectAll@CEditView@@IAEXXZ 5f874ce3 f   viewedit.obj
 0001:00073d29       ?OnSetFont@CEditView@@IAEJIJ@Z 5f874d29 f   viewedit.obj
 0001:00073d7c       ?SetPrinterFont@CEditView@@QAEXPAVCFont@@@Z 5f874d7c f   viewedit.obj
 0001:00073dbd       ?GetPrinterFont@CEditView@@QBEPAVCFont@@XZ 5f874dbd f   viewedit.obj
 0001:00073de7       ?LockBuffer@CEditView@@QBEPBGXZ 5f874de7 f   viewedit.obj
 0001:00073ea5       ?UnlockBuffer@CEditView@@QBEXXZ 5f874ea5 f   viewedit.obj
 0001:00073f2a       ?GetBufferLength@CEditView@@QBEIXZ 5f874f2a f   viewedit.obj
 0001:00073f96       ?GetSelectedText@CEditView@@QBEXAAVCString@@@Z 5f874f96 f   viewedit.obj
 0001:0007406a       ?OnEditFind@CEditView@@IAEXXZ 5f87506a f   viewedit.obj
 0001:000740a5       ?OnEditReplace@CEditView@@IAEXXZ 5f8750a5 f   viewedit.obj
 0001:000740e0       ?OnEditRepeat@CEditView@@IAEXXZ 5f8750e0 f   viewedit.obj
 0001:00074160       ?OnEditFindReplace@CEditView@@IAEXH@Z 5f875160 f   viewedit.obj
 0001:0007440c       ?OnFindNext@CEditView@@MAEXPBGHH@Z 5f87540c f   viewedit.obj
 0001:000744a9       ?OnReplaceSel@CEditView@@MAEXPBGHH0@Z 5f8754a9 f   viewedit.obj
 0001:00074562       ?OnReplaceAll@CEditView@@MAEXPBG0H@Z 5f875562 f   viewedit.obj
 0001:0007463d       ?InitializeReplace@CEditView@@IAEHXZ 5f87563d f   viewedit.obj
 0001:00074748       ?OnFindReplaceCmd@CEditView@@IAEJIJ@Z 5f875748 f   viewedit.obj
 0001:000749e8       ?SameAsSelected@CEditView@@IAEHPBGH@Z 5f8759e8 f   viewedit.obj
 0001:00074ac6       ?FindTextW@CEditView@@QAEHPBGHH@Z 5f875ac6 f   viewedit.obj
 0001:00074fbe       ?OnTextNotFound@CEditView@@MAEXPBG@Z 5f875fbe f   viewedit.obj
 0001:00074fe6       ?SetTabStops@CEditView@@QAEXH@Z 5f875fe6 f   viewedit.obj
 0001:00075042       ?AssertValid@CEditView@@UBEXXZ 5f876042 f   viewedit.obj
 0001:000750e3       ?Dump@CEditView@@UBEXAAVCDumpContext@@@Z 5f8760e3 f   viewedit.obj
 0001:00075250       ??_E_AFX_EDIT_STATE@@UAEPAXI@Z 5f876250 f i viewedit.obj
 0001:00075250       ??_G_AFX_EDIT_STATE@@UAEPAXI@Z 5f876250 f i viewedit.obj
 0001:00075280       ??_ECEditView@@UAEPAXI@Z   5f876280 f i viewedit.obj
 0001:00075280       ??_GCEditView@@UAEPAXI@Z   5f876280 f i viewedit.obj
 0001:000752b0       ?_GetBaseMessageMap@CListView@@KGPBUAFX_MSGMAP@@XZ 5f8762b0 f   viewcmn.obj
 0001:000752ba       ?GetMessageMap@CListView@@MBEPBUAFX_MSGMAP@@XZ 5f8762ba f   viewcmn.obj
 0001:000752ca       ?PreCreateWindow@CListView@@UAEHAAUtagCREATESTRUCTW@@@Z 5f8762ca f   viewcmn.obj
 0001:000752e3       ?DrawItem@CListView@@UAEXPAUtagDRAWITEMSTRUCT@@@Z 5f8762e3 f   viewcmn.obj
 0001:00075316       ?OnChildNotify@CListView@@MAEHIIJPAJ@Z 5f876316 f   viewcmn.obj
 0001:0007537d       ?RemoveImageList@CListView@@IAEXH@Z 5f87637d f   viewcmn.obj
 0001:000753c2       ?OnNcDestroy@CListView@@QAEXXZ 5f8763c2 f   viewcmn.obj
 0001:000753f3       ?_GetBaseMessageMap@CTreeView@@KGPBUAFX_MSGMAP@@XZ 5f8763f3 f   viewcmn.obj
 0001:000753fd       ?GetMessageMap@CTreeView@@MBEPBUAFX_MSGMAP@@XZ 5f8763fd f   viewcmn.obj
 0001:0007540d       ?PreCreateWindow@CTreeView@@UAEHAAUtagCREATESTRUCTW@@@Z 5f87640d f   viewcmn.obj
 0001:00075426       ?RemoveImageList@CTreeView@@IAEXH@Z 5f876426 f   viewcmn.obj
 0001:0007546b       ?OnDestroy@CTreeView@@QAEXXZ 5f87646b f   viewcmn.obj
 0001:00075492       ??0CListView@@QAE@XZ       5f876492 f   viewcmn.obj
 0001:000754bb       ?GetListCtrl@CListView@@QBEAAVCListCtrl@@XZ 5f8764bb f   viewcmn.obj
 0001:000754c9       ??0CTreeView@@QAE@XZ       5f8764c9 f   viewcmn.obj
 0001:000754f2       ?GetTreeCtrl@CTreeView@@QBEAAVCTreeCtrl@@XZ 5f8764f2 f   viewcmn.obj
 0001:00075500       ??1CTreeView@@UAE@XZ       5f876500 f i viewcmn.obj
 0001:00075500       ??1CListView@@UAE@XZ       5f876500 f i viewcmn.obj
 0001:00075520       ?AfxOleOnReleaseAllObjects@@YGXXZ 5f876520 f   olelock.obj
 0001:00075588       ?AfxOleCanExitApp@@YGHXZ   5f876588 f   olelock.obj
 0001:000755a6       ?AfxOleLockApp@@YGXXZ      5f8765a6 f   olelock.obj
 0001:000755c3       ?AfxOleUnlockApp@@YGXXZ    5f8765c3 f   olelock.obj
 0001:0007560f       ?AfxOleSetUserCtrl@@YGXH@Z 5f87660f f   olelock.obj
 0001:00075673       ?AfxOleGetUserCtrl@@YGHXZ  5f876673 f   olelock.obj
 0001:00075690       ?OutputString@CDumpContext@@IAEXPBG@Z 5f876690 f   dumpcont.obj
 0001:0007577d       ??0CDumpContext@@QAE@PAVCFile@@@Z 5f87677d f   dumpcont.obj
 0001:000757b5       ?Flush@CDumpContext@@QAEXXZ 5f8767b5 f   dumpcont.obj
 0001:000757da       ??6CDumpContext@@QAEAAV0@PBG@Z 5f8767da f   dumpcont.obj
 0001:0007592a       ??6CDumpContext@@QAEAAV0@E@Z 5f87692a f   dumpcont.obj
 0001:00075963       ??6CDumpContext@@QAEAAV0@G@Z 5f876963 f   dumpcont.obj
 0001:0007599c       ??6CDumpContext@@QAEAAV0@I@Z 5f87699c f   dumpcont.obj
 0001:000759d0       ??6CDumpContext@@QAEAAV0@J@Z 5f8769d0 f   dumpcont.obj
 0001:00075a04       ??6CDumpContext@@QAEAAV0@K@Z 5f876a04 f   dumpcont.obj
 0001:00075a38       ??6CDumpContext@@QAEAAV0@H@Z 5f876a38 f   dumpcont.obj
 0001:00075a6c       ??6CDumpContext@@QAEAAV0@PBVCObject@@@Z 5f876a6c f   dumpcont.obj
 0001:00075aae       ??6CDumpContext@@QAEAAV0@ABVCObject@@@Z 5f876aae f   dumpcont.obj
 0001:00075ac7       ??6CDumpContext@@QAEAAV0@PBX@Z 5f876ac7 f   dumpcont.obj
 0001:00075afb       ?HexDump@CDumpContext@@QAEXPBGPAEHH@Z 5f876afb f   dumpcont.obj
 0001:00075c68       ??6CDumpContext@@QAEAAV0@PBD@Z 5f876c68 f   dumpcont.obj
 0001:00075ce0       ??6CDumpContext@@QAEAAV0@M@Z 5f876ce0 f   dumpflt.obj
 0001:00075d16       ??6CDumpContext@@QAEAAV0@N@Z 5f876d16 f   dumpflt.obj
 0001:00075d50       ?AfxAssertFailedLine@@YGHPBDH@Z 5f876d50 f   afxasert.obj
 0001:00075da0       ??0CObject@@IAE@XZ         5f876da0 f   afxinl1.obj
 0001:00075db7       ??1CObject@@UAE@XZ         5f876db7 f   afxinl1.obj
 0001:00075dcb       ?Serialize@CObject@@UAEXAAVCArchive@@@Z 5f876dcb f   afxinl1.obj
 0001:00075dd8       ??2CObject@@SGPAXIPAX@Z    5f876dd8 f   afxinl1.obj
 0001:00075de2       ?AfxDynamicDownCast@@YAPBVCObject@@PAUCRuntimeClass@@PBV1@@Z 5f876de2 f   afxinl1.obj
 0001:00075df7       ?AfxStaticDownCast@@YAPBVCObject@@PAUCRuntimeClass@@PBV1@@Z 5f876df7 f   afxinl1.obj
 0001:00075e0c       ??1CException@@UAE@XZ      5f876e0c f   afxinl1.obj
 0001:00075e28       ??0CSimpleException@@QAE@XZ 5f876e28 f   afxinl1.obj
 0001:00075e5b       ??0CSimpleException@@QAE@H@Z 5f876e5b f   afxinl1.obj
 0001:00075e94       ??1CSimpleException@@UAE@XZ 5f876e94 f   afxinl1.obj
 0001:00075eb0       ??0CMemoryException@@QAE@XZ 5f876eb0 f   afxinl1.obj
 0001:00075ecf       ??0CMemoryException@@QAE@HI@Z 5f876ecf f   afxinl1.obj
 0001:00075f00       ??1CMemoryException@@UAE@XZ 5f876f00 f   afxinl1.obj
 0001:00075f1c       ??0CNotSupportedException@@QAE@XZ 5f876f1c f   afxinl1.obj
 0001:00075f3b       ??0CNotSupportedException@@QAE@HI@Z 5f876f3b f   afxinl1.obj
 0001:00075f6c       ??1CNotSupportedException@@UAE@XZ 5f876f6c f   afxinl1.obj
 0001:00075f88       ??0CArchiveException@@QAE@HPBG@Z 5f876f88 f   afxinl1.obj
 0001:00075ffd       ??1CArchiveException@@UAE@XZ 5f876ffd f   afxinl1.obj
 0001:00076051       ??0CFileException@@QAE@HJPBG@Z 5f877051 f   afxinl1.obj
 0001:000760cf       ??1CFileException@@UAE@XZ  5f8770cf f   afxinl1.obj
 0001:00076123       ??BCFile@@QBEHXZ           5f877123 f   afxinl1.obj
 0001:00076134       ?ReadHuge@CFile@@QAEKPAXK@Z 5f877134 f   afxinl1.obj
 0001:00076154       ?WriteHuge@CFile@@QAEXPBXK@Z 5f877154 f   afxinl1.obj
 0001:00076174       ?SeekToEnd@CFile@@QAEKXZ   5f877174 f   afxinl1.obj
 0001:0007618e       ?SeekToBegin@CFile@@QAEXXZ 5f87718e f   afxinl1.obj
 0001:000761a8       ?SetFilePath@CFile@@UAEXPBG@Z 5f8771a8 f   afxinl1.obj
 0001:00076200       ?IsReadOnly@CFileFind@@QBEHXZ 5f877200 f   afxinl1.obj
 0001:00076218       ?IsDirectory@CFileFind@@QBEHXZ 5f877218 f   afxinl1.obj
 0001:00076230       ?IsCompressed@CFileFind@@QBEHXZ 5f877230 f   afxinl1.obj
 0001:0007624b       ?IsSystem@CFileFind@@QBEHXZ 5f87724b f   afxinl1.obj
 0001:00076263       ?IsHidden@CFileFind@@QBEHXZ 5f877263 f   afxinl1.obj
 0001:0007627b       ?IsTemporary@CFileFind@@QBEHXZ 5f87727b f   afxinl1.obj
 0001:00076296       ?IsNormal@CFileFind@@QBEHXZ 5f877296 f   afxinl1.obj
 0001:000762b1       ?IsArchived@CFileFind@@QBEHXZ 5f8772b1 f   afxinl1.obj
 0001:000762c9       ?GetData@CString@@IBEPAUCStringData@@XZ 5f8772c9 f   afxinl1.obj
 0001:00076301       ?Init@CString@@IAEXXZ      5f877301 f   afxinl1.obj
 0001:00076318       ??0CString@@QAE@PBE@Z      5f877318 f   afxinl1.obj
 0001:0007633c       ??4CString@@QAEABV0@PBE@Z  5f87733c f   afxinl1.obj
 0001:00076358       ??YCString@@QAEABV0@D@Z    5f877358 f   afxinl1.obj
 0001:00076376       ??4CString@@QAEABV0@D@Z    5f877376 f   afxinl1.obj
 0001:00076394       ??H@YG?AVCString@@ABV0@D@Z 5f877394 f   afxinl1.obj
 0001:000763c3       ??H@YG?AVCString@@DABV0@@Z 5f8773c3 f   afxinl1.obj
 0001:000763f2       ?GetLength@CString@@QBEHXZ 5f8773f2 f   afxinl1.obj
 0001:00076408       ?GetAllocLength@CString@@QBEHXZ 5f877408 f   afxinl1.obj
 0001:0007641e       ?IsEmpty@CString@@QBEHXZ   5f87741e f   afxinl1.obj
 0001:0007643c       ??BCString@@QBEPBGXZ       5f87743c f   afxinl1.obj
 0001:0007644c       ?SafeStrlen@CString@@KGHPBG@Z 5f87744c f   afxinl1.obj
 0001:00076475       ?Compare@CString@@QBEHPBG@Z 5f877475 f   afxinl1.obj
 0001:000764c4       ?CompareNoCase@CString@@QBEHPBG@Z 5f8774c4 f   afxinl1.obj
 0001:00076513       ?Collate@CString@@QBEHPBG@Z 5f877513 f   afxinl1.obj
 0001:00076562       ?CollateNoCase@CString@@QBEHPBG@Z 5f877562 f   afxinl1.obj
 0001:000765b1       ?GetAt@CString@@QBEGH@Z    5f8775b1 f   afxinl1.obj
 0001:0007661a       ??ACString@@QBEGH@Z        5f87761a f   afxinl1.obj
 0001:00076683       ??8@YG_NABVCString@@0@Z    5f877683 f   afxinl1.obj
 0001:000766a0       ??8@YG_NABVCString@@PBG@Z  5f8776a0 f   afxinl1.obj
 0001:000766b8       ??8@YG_NPBGABVCString@@@Z  5f8776b8 f   afxinl1.obj
 0001:000766d0       ??9@YG_NABVCString@@0@Z    5f8776d0 f   afxinl1.obj
 0001:000766ee       ??9@YG_NABVCString@@PBG@Z  5f8776ee f   afxinl1.obj
 0001:00076707       ??9@YG_NPBGABVCString@@@Z  5f877707 f   afxinl1.obj
 0001:00076720       ??M@YG_NABVCString@@0@Z    5f877720 f   afxinl1.obj
 0001:00076741       ??M@YG_NABVCString@@PBG@Z  5f877741 f   afxinl1.obj
 0001:0007675d       ??M@YG_NPBGABVCString@@@Z  5f87775d f   afxinl1.obj
 0001:00076779       ??O@YG_NABVCString@@0@Z    5f877779 f   afxinl1.obj
 0001:0007679a       ??O@YG_NABVCString@@PBG@Z  5f87779a f   afxinl1.obj
 0001:000767b6       ??O@YG_NPBGABVCString@@@Z  5f8777b6 f   afxinl1.obj
 0001:000767d2       ??N@YG_NABVCString@@0@Z    5f8777d2 f   afxinl1.obj
 0001:000767f3       ??N@YG_NABVCString@@PBG@Z  5f8777f3 f   afxinl1.obj
 0001:0007680f       ??N@YG_NPBGABVCString@@@Z  5f87780f f   afxinl1.obj
 0001:0007682b       ??P@YG_NABVCString@@0@Z    5f87782b f   afxinl1.obj
 0001:0007684c       ??P@YG_NABVCString@@PBG@Z  5f87784c f   afxinl1.obj
 0001:00076868       ??P@YG_NPBGABVCString@@@Z  5f877868 f   afxinl1.obj
 0001:00076884       ??0CTimeSpan@@QAE@XZ       5f877884 f   afxinl1.obj
 0001:00076892       ??0CTimeSpan@@QAE@J@Z      5f877892 f   afxinl1.obj
 0001:000768aa       ??0CTimeSpan@@QAE@JHHH@Z   5f8778aa f   afxinl1.obj
 0001:000768da       ??0CTimeSpan@@QAE@ABV0@@Z  5f8778da f   afxinl1.obj
 0001:000768f4       ??4CTimeSpan@@QAEABV0@ABV0@@Z 5f8778f4 f   afxinl1.obj
 0001:0007690e       ?GetDays@CTimeSpan@@QBEJXZ 5f87790e f   afxinl1.obj
 0001:00076926       ?GetTotalHours@CTimeSpan@@QBEJXZ 5f877926 f   afxinl1.obj
 0001:0007693e       ?GetHours@CTimeSpan@@QBEHXZ 5f87793e f   afxinl1.obj
 0001:00076964       ?GetTotalMinutes@CTimeSpan@@QBEJXZ 5f877964 f   afxinl1.obj
 0001:0007697c       ?GetMinutes@CTimeSpan@@QBEHXZ 5f87797c f   afxinl1.obj
 0001:000769a2       ?GetTotalSeconds@CTimeSpan@@QBEJXZ 5f8779a2 f   afxinl1.obj
 0001:000769b2       ?GetSeconds@CTimeSpan@@QBEHXZ 5f8779b2 f   afxinl1.obj
 0001:000769d8       ??GCTimeSpan@@QBE?AV0@V0@@Z 5f8779d8 f   afxinl1.obj
 0001:00076a04       ??HCTimeSpan@@QBE?AV0@V0@@Z 5f877a04 f   afxinl1.obj
 0001:00076a30       ??YCTimeSpan@@QAEABV0@V0@@Z 5f877a30 f   afxinl1.obj
 0001:00076a4d       ??ZCTimeSpan@@QAEABV0@V0@@Z 5f877a4d f   afxinl1.obj
 0001:00076a6a       ??8CTimeSpan@@QBEHV0@@Z    5f877a6a f   afxinl1.obj
 0001:00076a84       ??9CTimeSpan@@QBEHV0@@Z    5f877a84 f   afxinl1.obj
 0001:00076a9e       ??MCTimeSpan@@QBEHV0@@Z    5f877a9e f   afxinl1.obj
 0001:00076ab8       ??OCTimeSpan@@QBEHV0@@Z    5f877ab8 f   afxinl1.obj
 0001:00076ad2       ??NCTimeSpan@@QBEHV0@@Z    5f877ad2 f   afxinl1.obj
 0001:00076aec       ??PCTimeSpan@@QBEHV0@@Z    5f877aec f   afxinl1.obj
 0001:00076b06       ??0CTime@@QAE@XZ           5f877b06 f   afxinl1.obj
 0001:00076b14       ??0CTime@@QAE@J@Z          5f877b14 f   afxinl1.obj
 0001:00076b2c       ??0CTime@@QAE@ABV0@@Z      5f877b2c f   afxinl1.obj
 0001:00076b46       ??4CTime@@QAEABV0@ABV0@@Z  5f877b46 f   afxinl1.obj
 0001:00076b60       ??4CTime@@QAEABV0@J@Z      5f877b60 f   afxinl1.obj
 0001:00076b78       ?GetTime@CTime@@QBEJXZ     5f877b78 f   afxinl1.obj
 0001:00076b88       ?GetYear@CTime@@QBEHXZ     5f877b88 f   afxinl1.obj
 0001:00076ba5       ?GetMonth@CTime@@QBEHXZ    5f877ba5 f   afxinl1.obj
 0001:00076bc0       ?GetDay@CTime@@QBEHXZ      5f877bc0 f   afxinl1.obj
 0001:00076bd8       ?GetHour@CTime@@QBEHXZ     5f877bd8 f   afxinl1.obj
 0001:00076bf0       ?GetMinute@CTime@@QBEHXZ   5f877bf0 f   afxinl1.obj
 0001:00076c08       ?GetSecond@CTime@@QBEHXZ   5f877c08 f   afxinl1.obj
 0001:00076c1f       ?GetDayOfWeek@CTime@@QBEHXZ 5f877c1f f   afxinl1.obj
 0001:00076c3a       ??GCTime@@QBE?AVCTimeSpan@@V0@@Z 5f877c3a f   afxinl1.obj
 0001:00076c66       ??GCTime@@QBE?AV0@VCTimeSpan@@@Z 5f877c66 f   afxinl1.obj
 0001:00076c92       ??HCTime@@QBE?AV0@VCTimeSpan@@@Z 5f877c92 f   afxinl1.obj
 0001:00076cbe       ??YCTime@@QAEABV0@VCTimeSpan@@@Z 5f877cbe f   afxinl1.obj
 0001:00076cdb       ??ZCTime@@QAEABV0@VCTimeSpan@@@Z 5f877cdb f   afxinl1.obj
 0001:00076cf8       ??8CTime@@QBEHV0@@Z        5f877cf8 f   afxinl1.obj
 0001:00076d12       ??9CTime@@QBEHV0@@Z        5f877d12 f   afxinl1.obj
 0001:00076d2c       ??MCTime@@QBEHV0@@Z        5f877d2c f   afxinl1.obj
 0001:00076d46       ??OCTime@@QBEHV0@@Z        5f877d46 f   afxinl1.obj
 0001:00076d60       ??NCTime@@QBEHV0@@Z        5f877d60 f   afxinl1.obj
 0001:00076d7a       ??PCTime@@QBEHV0@@Z        5f877d7a f   afxinl1.obj
 0001:00076d94       ?IsLoading@CArchive@@QBEHXZ 5f877d94 f   afxinl1.obj
 0001:00076dae       ?IsStoring@CArchive@@QBEHXZ 5f877dae f   afxinl1.obj
 0001:00076dc7       ?IsByteSwapping@CArchive@@QBEHXZ 5f877dc7 f   afxinl1.obj
 0001:00076de0       ?IsBufferEmpty@CArchive@@QBEHXZ 5f877de0 f   afxinl1.obj
 0001:00076dfc       ?GetFile@CArchive@@QBEPAVCFile@@XZ 5f877dfc f   afxinl1.obj
 0001:00076e0d       ?SetObjectSchema@CArchive@@QAEXI@Z 5f877e0d f   afxinl1.obj
 0001:00076e23       ?SetStoreParams@CArchive@@QAEXII@Z 5f877e23 f   afxinl1.obj
 0001:00076e91       ?SetLoadParams@CArchive@@QAEXI@Z 5f877e91 f   afxinl1.obj
 0001:00076ef6       ??6CArchive@@QAEAAV0@H@Z   5f877ef6 f   afxinl1.obj
 0001:00076f0f       ??6CArchive@@QAEAAV0@I@Z   5f877f0f f   afxinl1.obj
 0001:00076f28       ??6CArchive@@QAEAAV0@F@Z   5f877f28 f   afxinl1.obj
 0001:00076f42       ??6CArchive@@QAEAAV0@D@Z   5f877f42 f   afxinl1.obj
 0001:00076f5b       ??6CArchive@@QAEAAV0@E@Z   5f877f5b f   afxinl1.obj
 0001:00076f9e       ??6CArchive@@QAEAAV0@G@Z   5f877f9e f   afxinl1.obj
 0001:00076fe3       ??6CArchive@@QAEAAV0@J@Z   5f877fe3 f   afxinl1.obj
 0001:00077026       ??6CArchive@@QAEAAV0@K@Z   5f878026 f   afxinl1.obj
 0001:00077069       ??6CArchive@@QAEAAV0@M@Z   5f878069 f   afxinl1.obj
 0001:000770ac       ??6CArchive@@QAEAAV0@N@Z   5f8780ac f   afxinl1.obj
 0001:000770f5       ??5CArchive@@QAEAAV0@AAH@Z 5f8780f5 f   afxinl1.obj
 0001:0007710e       ??5CArchive@@QAEAAV0@AAI@Z 5f87810e f   afxinl1.obj
 0001:00077127       ??5CArchive@@QAEAAV0@AAF@Z 5f878127 f   afxinl1.obj
 0001:00077140       ??5CArchive@@QAEAAV0@AAD@Z 5f878140 f   afxinl1.obj
 0001:00077159       ??5CArchive@@QAEAAV0@AAE@Z 5f878159 f   afxinl1.obj
 0001:000771b2       ??5CArchive@@QAEAAV0@AAG@Z 5f8781b2 f   afxinl1.obj
 0001:0007720d       ??5CArchive@@QAEAAV0@AAK@Z 5f87820d f   afxinl1.obj
 0001:00077266       ??5CArchive@@QAEAAV0@AAM@Z 5f878266 f   afxinl1.obj
 0001:000772bf       ??5CArchive@@QAEAAV0@AAN@Z 5f8782bf f   afxinl1.obj
 0001:0007731e       ??5CArchive@@QAEAAV0@AAJ@Z 5f87831e f   afxinl1.obj
 0001:00077377       ??0CArchive@@IAE@ABV0@@Z   5f878377 f   afxinl1.obj
 0001:00077392       ??4CArchive@@IAEXABV0@@Z   5f878392 f   afxinl1.obj
 0001:0007739f       ??6@YGAAVCArchive@@AAV0@PBVCObject@@@Z 5f87839f f   afxinl1.obj
 0001:000773b5       ??5@YGAAVCArchive@@AAV0@AAPAVCObject@@@Z 5f8783b5 f   afxinl1.obj
 0001:000773ce       ??5@YGAAVCArchive@@AAV0@AAPBVCObject@@@Z 5f8783ce f   afxinl1.obj
 0001:000773e7       ?GetDepth@CDumpContext@@QBEHXZ 5f8783e7 f   afxinl1.obj
 0001:000773f7       ?SetDepth@CDumpContext@@QAEXH@Z 5f8783f7 f   afxinl1.obj
 0001:0007740c       ??0CDumpContext@@IAE@ABV0@@Z 5f87840c f   afxinl1.obj
 0001:0007741c       ??4CDumpContext@@IAEXABV0@@Z 5f87841c f   afxinl1.obj
 0001:00077429       ?GetSize@CByteArray@@QBEHXZ 5f878429 f   afxinl1.obj
 0001:0007743a       ?GetUpperBound@CByteArray@@QBEHXZ 5f87843a f   afxinl1.obj
 0001:0007744e       ?RemoveAll@CByteArray@@QAEXXZ 5f87844e f   afxinl1.obj
 0001:00077465       ?GetAt@CByteArray@@QBEEH@Z 5f878465 f   afxinl1.obj
 0001:000774ac       ?SetAt@CByteArray@@QAEXHE@Z 5f8784ac f   afxinl1.obj
 0001:000774f6       ?ElementAt@CByteArray@@QAEAAEH@Z 5f8784f6 f   afxinl1.obj
 0001:0007753a       ?GetData@CByteArray@@QBEPBEXZ 5f87853a f   afxinl1.obj
 0001:0007754b       ?GetData@CByteArray@@QAEPAEXZ 5f87854b f   afxinl1.obj
 0001:0007755c       ?Add@CByteArray@@QAEHE@Z   5f87855c f   afxinl1.obj
 0001:00077587       ??ACByteArray@@QBEEH@Z     5f878587 f   afxinl1.obj
 0001:000775a0       ??ACByteArray@@QAEAAEH@Z   5f8785a0 f   afxinl1.obj
 0001:000775b9       ?GetSize@CWordArray@@QBEHXZ 5f8785b9 f   afxinl1.obj
 0001:000775ca       ?GetUpperBound@CWordArray@@QBEHXZ 5f8785ca f   afxinl1.obj
 0001:000775de       ?RemoveAll@CWordArray@@QAEXXZ 5f8785de f   afxinl1.obj
 0001:000775f5       ?GetAt@CWordArray@@QBEGH@Z 5f8785f5 f   afxinl1.obj
 0001:0007763d       ?SetAt@CWordArray@@QAEXHG@Z 5f87863d f   afxinl1.obj
 0001:00077689       ?ElementAt@CWordArray@@QAEAAGH@Z 5f878689 f   afxinl1.obj
 0001:000776d0       ?GetData@CWordArray@@QBEPBGXZ 5f8786d0 f   afxinl1.obj
 0001:000776e1       ?GetData@CWordArray@@QAEPAGXZ 5f8786e1 f   afxinl1.obj
 0001:000776f2       ?Add@CWordArray@@QAEHG@Z   5f8786f2 f   afxinl1.obj
 0001:0007771e       ??ACWordArray@@QBEGH@Z     5f87871e f   afxinl1.obj
 0001:00077737       ??ACWordArray@@QAEAAGH@Z   5f878737 f   afxinl1.obj
 0001:00077750       ?GetSize@CDWordArray@@QBEHXZ 5f878750 f   afxinl1.obj
 0001:00077761       ?GetUpperBound@CDWordArray@@QBEHXZ 5f878761 f   afxinl1.obj
 0001:00077775       ?RemoveAll@CDWordArray@@QAEXXZ 5f878775 f   afxinl1.obj
 0001:0007778c       ?GetAt@CDWordArray@@QBEKH@Z 5f87878c f   afxinl1.obj
 0001:000777d3       ?SetAt@CDWordArray@@QAEXHK@Z 5f8787d3 f   afxinl1.obj
 0001:0007781d       ?ElementAt@CDWordArray@@QAEAAKH@Z 5f87881d f   afxinl1.obj
 0001:00077864       ?GetData@CDWordArray@@QBEPBKXZ 5f878864 f   afxinl1.obj
 0001:00077875       ?GetData@CDWordArray@@QAEPAKXZ 5f878875 f   afxinl1.obj
 0001:00077886       ?Add@CDWordArray@@QAEHK@Z  5f878886 f   afxinl1.obj
 0001:000778b1       ??ACDWordArray@@QBEKH@Z    5f8788b1 f   afxinl1.obj
 0001:000778ca       ??ACDWordArray@@QAEAAKH@Z  5f8788ca f   afxinl1.obj
 0001:000778e3       ?GetSize@CUIntArray@@QBEHXZ 5f8788e3 f   afxinl1.obj
 0001:000778f4       ?GetUpperBound@CUIntArray@@QBEHXZ 5f8788f4 f   afxinl1.obj
 0001:00077908       ?RemoveAll@CUIntArray@@QAEXXZ 5f878908 f   afxinl1.obj
 0001:0007791f       ?GetAt@CUIntArray@@QBEIH@Z 5f87891f f   afxinl1.obj
 0001:00077966       ?SetAt@CUIntArray@@QAEXHI@Z 5f878966 f   afxinl1.obj
 0001:000779b0       ?ElementAt@CUIntArray@@QAEAAIH@Z 5f8789b0 f   afxinl1.obj
 0001:000779fa       ?GetData@CUIntArray@@QBEPBIXZ 5f8789fa f   afxinl1.obj
 0001:00077a0b       ?GetData@CUIntArray@@QAEPAIXZ 5f878a0b f   afxinl1.obj
 0001:00077a1c       ?Add@CUIntArray@@QAEHI@Z   5f878a1c f   afxinl1.obj
 0001:00077a47       ??ACUIntArray@@QBEIH@Z     5f878a47 f   afxinl1.obj
 0001:00077a60       ??ACUIntArray@@QAEAAIH@Z   5f878a60 f   afxinl1.obj
 0001:00077a79       ?GetSize@CPtrArray@@QBEHXZ 5f878a79 f   afxinl1.obj
 0001:00077a8a       ?GetUpperBound@CPtrArray@@QBEHXZ 5f878a8a f   afxinl1.obj
 0001:00077a9e       ?RemoveAll@CPtrArray@@QAEXXZ 5f878a9e f   afxinl1.obj
 0001:00077ab5       ?GetAt@CPtrArray@@QBEPAXH@Z 5f878ab5 f   afxinl1.obj
 0001:00077aff       ?SetAt@CPtrArray@@QAEXHPAX@Z 5f878aff f   afxinl1.obj
 0001:00077b4c       ?ElementAt@CPtrArray@@QAEAAPAXH@Z 5f878b4c f   afxinl1.obj
 0001:00077b96       ?GetData@CPtrArray@@QBEPAPBXXZ 5f878b96 f   afxinl1.obj
 0001:00077ba7       ?GetData@CPtrArray@@QAEPAPAXXZ 5f878ba7 f   afxinl1.obj
 0001:00077bb8       ?Add@CPtrArray@@QAEHPAX@Z  5f878bb8 f   afxinl1.obj
 0001:00077be3       ??ACPtrArray@@QBEPAXH@Z    5f878be3 f   afxinl1.obj
 0001:00077bfc       ??ACPtrArray@@QAEAAPAXH@Z  5f878bfc f   afxinl1.obj
 0001:00077c15       ?GetSize@CObArray@@QBEHXZ  5f878c15 f   afxinl1.obj
 0001:00077c26       ?GetUpperBound@CObArray@@QBEHXZ 5f878c26 f   afxinl1.obj
 0001:00077c3a       ?RemoveAll@CObArray@@QAEXXZ 5f878c3a f   afxinl1.obj
 0001:00077c51       ?GetAt@CObArray@@QBEPAVCObject@@H@Z 5f878c51 f   afxinl1.obj
 0001:00077c9b       ?SetAt@CObArray@@QAEXHPAVCObject@@@Z 5f878c9b f   afxinl1.obj
 0001:00077ce8       ?ElementAt@CObArray@@QAEAAPAVCObject@@H@Z 5f878ce8 f   afxinl1.obj
 0001:00077d32       ?GetData@CObArray@@QBEPAPBVCObject@@XZ 5f878d32 f   afxinl1.obj
 0001:00077d43       ?GetData@CObArray@@QAEPAPAVCObject@@XZ 5f878d43 f   afxinl1.obj
 0001:00077d54       ?Add@CObArray@@QAEHPAVCObject@@@Z 5f878d54 f   afxinl1.obj
 0001:00077d7f       ??ACObArray@@QBEPAVCObject@@H@Z 5f878d7f f   afxinl1.obj
 0001:00077d98       ??ACObArray@@QAEAAPAVCObject@@H@Z 5f878d98 f   afxinl1.obj
 0001:00077db1       ?GetSize@CStringArray@@QBEHXZ 5f878db1 f   afxinl1.obj
 0001:00077dc2       ?GetUpperBound@CStringArray@@QBEHXZ 5f878dc2 f   afxinl1.obj
 0001:00077dd6       ?RemoveAll@CStringArray@@QAEXXZ 5f878dd6 f   afxinl1.obj
 0001:00077ded       ?GetAt@CStringArray@@QBE?AVCString@@H@Z 5f878ded f   afxinl1.obj
 0001:00077e55       ?SetAt@CStringArray@@QAEXHPBG@Z 5f878e55 f   afxinl1.obj
 0001:00077ea8       ?SetAt@CStringArray@@QAEXHABVCString@@@Z 5f878ea8 f   afxinl1.obj
 0001:00077efb       ?ElementAt@CStringArray@@QAEAAVCString@@H@Z 5f878efb f   afxinl1.obj
 0001:00077f45       ?GetData@CStringArray@@QBEPBVCString@@XZ 5f878f45 f   afxinl1.obj
 0001:00077f56       ?GetData@CStringArray@@QAEPAVCString@@XZ 5f878f56 f   afxinl1.obj
 0001:00077f67       ?Add@CStringArray@@QAEHPBG@Z 5f878f67 f   afxinl1.obj
 0001:00077f92       ?Add@CStringArray@@QAEHABVCString@@@Z 5f878f92 f   afxinl1.obj
 0001:00077fbd       ??ACStringArray@@QBE?AVCString@@H@Z 5f878fbd f   afxinl1.obj
 0001:00077fef       ??ACStringArray@@QAEAAVCString@@H@Z 5f878fef f   afxinl1.obj
 0001:00078008       ?GetCount@CPtrList@@QBEHXZ 5f879008 f   afxinl1.obj
 0001:00078019       ?IsEmpty@CPtrList@@QBEHXZ  5f879019 f   afxinl1.obj
 0001:00078032       ?GetHead@CPtrList@@QAEAAPAXXZ 5f879032 f   afxinl1.obj
 0001:0007806f       ?GetHead@CPtrList@@QBEPAXXZ 5f87906f f   afxinl1.obj
 0001:000780ac       ?GetTail@CPtrList@@QAEAAPAXXZ 5f8790ac f   afxinl1.obj
 0001:000780e9       ?GetTail@CPtrList@@QBEPAXXZ 5f8790e9 f   afxinl1.obj
 0001:00078126       ?GetHeadPosition@CPtrList@@QBEPAU__POSITION@@XZ 5f879126 f   afxinl1.obj
 0001:00078137       ?GetTailPosition@CPtrList@@QBEPAU__POSITION@@XZ 5f879137 f   afxinl1.obj
 0001:00078148       ?GetNext@CPtrList@@QAEAAPAXAAPAU__POSITION@@@Z 5f879148 f   afxinl1.obj
 0001:000781a0       ?GetNext@CPtrList@@QBEPAXAAPAU__POSITION@@@Z 5f8791a0 f   afxinl1.obj
 0001:000781f8       ?GetPrev@CPtrList@@QAEAAPAXAAPAU__POSITION@@@Z 5f8791f8 f   afxinl1.obj
 0001:00078251       ?GetPrev@CPtrList@@QBEPAXAAPAU__POSITION@@@Z 5f879251 f   afxinl1.obj
 0001:000782aa       ?GetAt@CPtrList@@QAEAAPAXPAU__POSITION@@@Z 5f8792aa f   afxinl1.obj
 0001:000782f6       ?GetAt@CPtrList@@QBEPAXPAU__POSITION@@@Z 5f8792f6 f   afxinl1.obj
 0001:00078342       ?SetAt@CPtrList@@QAEXPAU__POSITION@@PAX@Z 5f879342 f   afxinl1.obj
 0001:00078391       ?GetCount@CObList@@QBEHXZ  5f879391 f   afxinl1.obj
 0001:000783a2       ?IsEmpty@CObList@@QBEHXZ   5f8793a2 f   afxinl1.obj
 0001:000783bb       ?GetHead@CObList@@QAEAAPAVCObject@@XZ 5f8793bb f   afxinl1.obj
 0001:000783f8       ?GetHead@CObList@@QBEPAVCObject@@XZ 5f8793f8 f   afxinl1.obj
 0001:00078435       ?GetTail@CObList@@QAEAAPAVCObject@@XZ 5f879435 f   afxinl1.obj
 0001:00078472       ?GetTail@CObList@@QBEPAVCObject@@XZ 5f879472 f   afxinl1.obj
 0001:000784af       ?GetHeadPosition@CObList@@QBEPAU__POSITION@@XZ 5f8794af f   afxinl1.obj
 0001:000784c0       ?GetTailPosition@CObList@@QBEPAU__POSITION@@XZ 5f8794c0 f   afxinl1.obj
 0001:000784d1       ?GetNext@CObList@@QAEAAPAVCObject@@AAPAU__POSITION@@@Z 5f8794d1 f   afxinl1.obj
 0001:00078529       ?GetNext@CObList@@QBEPAVCObject@@AAPAU__POSITION@@@Z 5f879529 f   afxinl1.obj
 0001:00078581       ?GetPrev@CObList@@QAEAAPAVCObject@@AAPAU__POSITION@@@Z 5f879581 f   afxinl1.obj
 0001:000785da       ?GetPrev@CObList@@QBEPAVCObject@@AAPAU__POSITION@@@Z 5f8795da f   afxinl1.obj
 0001:00078633       ?GetAt@CObList@@QAEAAPAVCObject@@PAU__POSITION@@@Z 5f879633 f   afxinl1.obj
 0001:0007867f       ?GetAt@CObList@@QBEPAVCObject@@PAU__POSITION@@@Z 5f87967f f   afxinl1.obj
 0001:000786cb       ?SetAt@CObList@@QAEXPAU__POSITION@@PAVCObject@@@Z 5f8796cb f   afxinl1.obj
 0001:0007871a       ?GetCount@CStringList@@QBEHXZ 5f87971a f   afxinl1.obj
 0001:0007872b       ?IsEmpty@CStringList@@QBEHXZ 5f87972b f   afxinl1.obj
 0001:00078744       ?GetHead@CStringList@@QAEAAVCString@@XZ 5f879744 f   afxinl1.obj
 0001:00078781       ?GetHead@CStringList@@QBE?AVCString@@XZ 5f879781 f   afxinl1.obj
 0001:000787de       ?GetTail@CStringList@@QAEAAVCString@@XZ 5f8797de f   afxinl1.obj
 0001:0007881b       ?GetTail@CStringList@@QBE?AVCString@@XZ 5f87981b f   afxinl1.obj
 0001:00078878       ?GetHeadPosition@CStringList@@QBEPAU__POSITION@@XZ 5f879878 f   afxinl1.obj
 0001:00078889       ?GetTailPosition@CStringList@@QBEPAU__POSITION@@XZ 5f879889 f   afxinl1.obj
 0001:0007889a       ?GetNext@CStringList@@QAEAAVCString@@AAPAU__POSITION@@@Z 5f87989a f   afxinl1.obj
 0001:000788f2       ?GetNext@CStringList@@QBE?AVCString@@AAPAU__POSITION@@@Z 5f8798f2 f   afxinl1.obj
 0001:00078966       ?GetPrev@CStringList@@QAEAAVCString@@AAPAU__POSITION@@@Z 5f879966 f   afxinl1.obj
 0001:000789bf       ?GetPrev@CStringList@@QBE?AVCString@@AAPAU__POSITION@@@Z 5f8799bf f   afxinl1.obj
 0001:00078a34       ?GetAt@CStringList@@QAEAAVCString@@PAU__POSITION@@@Z 5f879a34 f   afxinl1.obj
 0001:00078a80       ?GetAt@CStringList@@QBE?AVCString@@PAU__POSITION@@@Z 5f879a80 f   afxinl1.obj
 0001:00078ae8       ?SetAt@CStringList@@QAEXPAU__POSITION@@PBG@Z 5f879ae8 f   afxinl1.obj
 0001:00078b3d       ?SetAt@CStringList@@QAEXPAU__POSITION@@ABVCString@@@Z 5f879b3d f   afxinl1.obj
 0001:00078b92       ?GetCount@CMapWordToPtr@@QBEHXZ 5f879b92 f   afxinl1.obj
 0001:00078ba3       ?IsEmpty@CMapWordToPtr@@QBEHXZ 5f879ba3 f   afxinl1.obj
 0001:00078bbc       ?SetAt@CMapWordToPtr@@QAEXGPAX@Z 5f879bbc f   afxinl1.obj
 0001:00078bdb       ?GetStartPosition@CMapWordToPtr@@QBEPAU__POSITION@@XZ 5f879bdb f   afxinl1.obj
 0001:00078bf0       ?GetHashTableSize@CMapWordToPtr@@QBEIXZ 5f879bf0 f   afxinl1.obj
 0001:00078c01       ?GetCount@CMapPtrToWord@@QBEHXZ 5f879c01 f   afxinl1.obj
 0001:00078c12       ?IsEmpty@CMapPtrToWord@@QBEHXZ 5f879c12 f   afxinl1.obj
 0001:00078c2b       ?SetAt@CMapPtrToWord@@QAEXPAXG@Z 5f879c2b f   afxinl1.obj
 0001:00078c4b       ?GetStartPosition@CMapPtrToWord@@QBEPAU__POSITION@@XZ 5f879c4b f   afxinl1.obj
 0001:00078c60       ?GetHashTableSize@CMapPtrToWord@@QBEIXZ 5f879c60 f   afxinl1.obj
 0001:00078c71       ?GetCount@CMapPtrToPtr@@QBEHXZ 5f879c71 f   afxinl1.obj
 0001:00078c82       ?IsEmpty@CMapPtrToPtr@@QBEHXZ 5f879c82 f   afxinl1.obj
 0001:00078c9b       ?SetAt@CMapPtrToPtr@@QAEXPAX0@Z 5f879c9b f   afxinl1.obj
 0001:00078cb9       ?GetStartPosition@CMapPtrToPtr@@QBEPAU__POSITION@@XZ 5f879cb9 f   afxinl1.obj
 0001:00078cce       ?GetHashTableSize@CMapPtrToPtr@@QBEIXZ 5f879cce f   afxinl1.obj
 0001:00078cdf       ?GetCount@CMapWordToOb@@QBEHXZ 5f879cdf f   afxinl1.obj
 0001:00078cf0       ?IsEmpty@CMapWordToOb@@QBEHXZ 5f879cf0 f   afxinl1.obj
 0001:00078d09       ?SetAt@CMapWordToOb@@QAEXGPAVCObject@@@Z 5f879d09 f   afxinl1.obj
 0001:00078d28       ?GetStartPosition@CMapWordToOb@@QBEPAU__POSITION@@XZ 5f879d28 f   afxinl1.obj
 0001:00078d3d       ?GetHashTableSize@CMapWordToOb@@QBEIXZ 5f879d3d f   afxinl1.obj
 0001:00078d4e       ?GetCount@CMapStringToPtr@@QBEHXZ 5f879d4e f   afxinl1.obj
 0001:00078d5f       ?IsEmpty@CMapStringToPtr@@QBEHXZ 5f879d5f f   afxinl1.obj
 0001:00078d78       ?SetAt@CMapStringToPtr@@QAEXPBGPAX@Z 5f879d78 f   afxinl1.obj
 0001:00078d96       ?GetStartPosition@CMapStringToPtr@@QBEPAU__POSITION@@XZ 5f879d96 f   afxinl1.obj
 0001:00078dab       ?GetHashTableSize@CMapStringToPtr@@QBEIXZ 5f879dab f   afxinl1.obj
 0001:00078dbc       ?GetCount@CMapStringToOb@@QBEHXZ 5f879dbc f   afxinl1.obj
 0001:00078dcd       ?IsEmpty@CMapStringToOb@@QBEHXZ 5f879dcd f   afxinl1.obj
 0001:00078de6       ?SetAt@CMapStringToOb@@QAEXPBGPAVCObject@@@Z 5f879de6 f   afxinl1.obj
 0001:00078e04       ?GetStartPosition@CMapStringToOb@@QBEPAU__POSITION@@XZ 5f879e04 f   afxinl1.obj
 0001:00078e19       ?GetHashTableSize@CMapStringToOb@@QBEIXZ 5f879e19 f   afxinl1.obj
 0001:00078e2a       ?GetCount@CMapStringToString@@QBEHXZ 5f879e2a f   afxinl1.obj
 0001:00078e3b       ?IsEmpty@CMapStringToString@@QBEHXZ 5f879e3b f   afxinl1.obj
 0001:00078e54       ?SetAt@CMapStringToString@@QAEXPBG0@Z 5f879e54 f   afxinl1.obj
 0001:00078e78       ?GetStartPosition@CMapStringToString@@QBEPAU__POSITION@@XZ 5f879e78 f   afxinl1.obj
 0001:00078e8d       ?GetHashTableSize@CMapStringToString@@QBEIXZ 5f879e8d f   afxinl1.obj
 0001:00078e9e       ??0CCommonDialog@@QAE@PAVCWnd@@@Z 5f879e9e f   afxinl1.obj
 0001:00078ec5       ?GetReadOnlyPref@CFileDialog@@QBEHXZ 5f879ec5 f   afxinl1.obj
 0001:00078ee2       ?SetTemplate@CFileDialog@@QAEXII@Z 5f879ee2 f   afxinl1.obj
 0001:00078f0a       ?GetStartPosition@CFileDialog@@QBEPAU__POSITION@@XZ 5f879f0a f   afxinl1.obj
 0001:00078f1b       ?GetFaceName@CFontDialog@@QBE?AVCString@@XZ 5f879f1b f   afxinl1.obj
 0001:00078f4f       ?GetStyleName@CFontDialog@@QBE?AVCString@@XZ 5f879f4f f   afxinl1.obj
 0001:00078f83       ?GetSize@CFontDialog@@QBEHXZ 5f879f83 f   afxinl1.obj
 0001:00078f94       ?GetWeight@CFontDialog@@QBEHXZ 5f879f94 f   afxinl1.obj
 0001:00078fa8       ?IsItalic@CFontDialog@@QBEHXZ 5f879fa8 f   afxinl1.obj
 0001:00078fc6       ?IsStrikeOut@CFontDialog@@QBEHXZ 5f879fc6 f   afxinl1.obj
 0001:00078fe4       ?IsBold@CFontDialog@@QBEHXZ 5f879fe4 f   afxinl1.obj
 0001:00079001       ?IsUnderline@CFontDialog@@QBEHXZ 5f87a001 f   afxinl1.obj
 0001:0007901f       ?GetColor@CFontDialog@@QBEKXZ 5f87a01f f   afxinl1.obj
 0001:00079030       ?GetColor@CColorDialog@@QBEKXZ 5f87a030 f   afxinl1.obj
 0001:00079041       ?PrintSelection@CPrintDialog@@QBEHXZ 5f87a041 f   afxinl1.obj
 0001:0007905e       ?PrintRange@CPrintDialog@@QBEHXZ 5f87a05e f   afxinl1.obj
 0001:0007907b       ?PrintAll@CPrintDialog@@QBEHXZ 5f87a07b f   afxinl1.obj
 0001:000790b3       ?PrintCollate@CPrintDialog@@QBEHXZ 5f87a0b3 f   afxinl1.obj
 0001:000790d0       ?GetFromPage@CPrintDialog@@QBEHXZ 5f87a0d0 f   afxinl1.obj
 0001:00079104       ?GetToPage@CPrintDialog@@QBEHXZ 5f87a104 f   afxinl1.obj
 0001:00079138       ?GetPrinterDC@CPrintDialog@@QBEPAUHDC__@@XZ 5f87a138 f   afxinl1.obj
 0001:0007918b       ?IsTerminating@CFindReplaceDialog@@QBEHXZ 5f87a18b f   afxinl1.obj
 0001:000791a5       ?GetReplaceString@CFindReplaceDialog@@QBE?AVCString@@XZ 5f87a1a5 f   afxinl1.obj
 0001:000791d6       ?GetFindString@CFindReplaceDialog@@QBE?AVCString@@XZ 5f87a1d6 f   afxinl1.obj
 0001:00079207       ?SearchDown@CFindReplaceDialog@@QBEHXZ 5f87a207 f   afxinl1.obj
 0001:00079221       ?FindNext@CFindReplaceDialog@@QBEHXZ 5f87a221 f   afxinl1.obj
 0001:0007923b       ?MatchCase@CFindReplaceDialog@@QBEHXZ 5f87a23b f   afxinl1.obj
 0001:00079255       ?MatchWholeWord@CFindReplaceDialog@@QBEHXZ 5f87a255 f   afxinl1.obj
 0001:0007926f       ?ReplaceCurrent@CFindReplaceDialog@@QBEHXZ 5f87a26f f   afxinl1.obj
 0001:00079289       ?ReplaceAll@CFindReplaceDialog@@QBEHXZ 5f87a289 f   afxinl1.obj
 0001:000792a3       ?GetPage@CPropertySheet@@QBEPAVCPropertyPage@@H@Z 5f87a2a3 f   afxinl1.obj
 0001:000792cd       ?SetWizardMode@CPropertySheet@@QAEXXZ 5f87a2cd f   afxinl1.obj
 0001:000792e7       ?SetFinishText@CPropertySheet@@QAEXPBG@Z 5f87a2e7 f   afxinl1.obj
 0001:0007933a       ?SetWizardButtons@CPropertySheet@@QAEXK@Z 5f87a33a f   afxinl1.obj
 0001:0007938d       ?GetTabControl@CPropertySheet@@QBEPAVCTabCtrl@@XZ 5f87a38d f   afxinl1.obj
 0001:000793e2       ?PressButton@CPropertySheet@@QAEHH@Z 5f87a3e2 f   afxinl1.obj
 0001:00079435       ?IsWizard@CPropertySheet@@QBEHXZ 5f87a435 f   afxinl1.obj
 0001:00079456       ?SetWizardMode@CPropertySheetEx@@QAEXXZ 5f87a456 f   afxinl1.obj
 0001:00079476       ?GetPaperSize@CPageSetupDialog@@QBE?AVCSize@@XZ 5f87a476 f   afxinl1.obj
 0001:000794ab       ??0CCreateContext@@QAE@XZ  5f87a4ab f   afxinl1.obj
 0001:000794c9       ?Create@CMetaFileDC@@QAEHPBG@Z 5f87a4c9 f   afxinl1.obj
 0001:000794e9       ?Close@CMetaFileDC@@QAEPAUHMETAFILE__@@XZ 5f87a4e9 f   afxinl1.obj
 0001:00079503       ?CreateEnhanced@CMetaFileDC@@QAEHPAVCDC@@PBGPBUtagRECT@@1@Z 5f87a503 f   afxinl1.obj
 0001:00079534       ?CloseEnhanced@CMetaFileDC@@QAEPAUHENHMETAFILE__@@XZ 5f87a534 f   afxinl1.obj
 0001:0007954e       ?SetViewportOrg@CMetaFileDC@@QAE?AVCPoint@@UtagPOINT@@@Z 5f87a54e f   afxinl1.obj
 0001:000795aa       ?SetViewportExt@CMetaFileDC@@QAE?AVCSize@@UtagSIZE@@@Z 5f87a5aa f   afxinl1.obj
 0001:00079606       ?TextOutW@CMetaFileDC@@QAEHHHABVCString@@@Z 5f87a606 f   afxinl1.obj
 0001:0007965e       ?ExtTextOutW@CMetaFileDC@@QAEHHHIPBUtagRECT@@ABVCString@@PAH@Z 5f87a65e f   afxinl1.obj
 0001:000796c4       ?TabbedTextOutW@CMetaFileDC@@QAE?AVCSize@@HHABVCString@@HPAHH@Z 5f87a6c4 f   afxinl1.obj
 0001:00079736       ?DrawTextW@CMetaFileDC@@QAEHABVCString@@PAUtagRECT@@I@Z 5f87a736 f   afxinl1.obj
 0001:0007978e       ?PtVisible@CMetaFileDC@@QBEHUtagPOINT@@@Z 5f87a78e f   afxinl1.obj
 0001:000797d4       ?GetRowCount@CSplitterWnd@@QBEHXZ 5f87a7d4 f   afxinl1.obj
 0001:000797e5       ?GetColumnCount@CSplitterWnd@@QBEHXZ 5f87a7e5 f   afxinl1.obj
 0001:000797f6       ?IsChildPane@CSplitterWnd@@QAEHPAVCWnd@@AAH1@Z 5f87a7f6 f   afxinl1.obj
 0001:00079817       ?GetActivePane@CSplitterWnd@@IAEPAVCWnd@@AAH0@Z 5f87a817 f   afxinl1.obj
 0001:0007983a       ?IsTracking@CSplitterWnd@@QAEHXZ 5f87a83a f   afxinl1.obj
 0001:0007984e       ?GetCount@CControlBar@@QBEHXZ 5f87a84e f   afxinl1.obj
 0001:0007985f       ?GetBarStyle@CControlBar@@QAEKXZ 5f87a85f f   afxinl1.obj
 0001:00079870       ?SetBorders@CControlBar@@QAEXPBUtagRECT@@@Z 5f87a870 f   afxinl1.obj
 0001:000798a0       ?GetBorders@CControlBar@@QBE?AVCRect@@XZ 5f87a8a0 f   afxinl1.obj
 0001:000798ef       ?LoadToolBar@CToolBar@@QAEHI@Z 5f87a8ef f   afxinl1.obj
 0001:0007990d       ?LoadBitmapW@CToolBar@@QAEHI@Z 5f87a90d f   afxinl1.obj
 0001:0007992b       ?GetToolBarCtrl@CToolBar@@QBEAAVCToolBarCtrl@@XZ 5f87a92b f   afxinl1.obj
 0001:00079939       ?Create@CDialogBar@@QAEHPAVCWnd@@III@Z 5f87a939 f   afxinl1.obj
 0001:00079964       ?GetStatusBarCtrl@CStatusBar@@QBEAAVCStatusBarCtrl@@XZ 5f87a964 f   afxinl1.obj
 0001:00079972       ?SetBorders@CStatusBar@@QAEXPBUtagRECT@@@Z 5f87a972 f   afxinl1.obj
 0001:000799a2       ?SetBorders@CStatusBar@@QAEXHHHH@Z 5f87a9a2 f   afxinl1.obj
 0001:000799ea       ?EnableDocking@CStatusBar@@QAEXK@Z 5f87a9ea f   afxinl1.obj
 0001:00079a1d       ?GetReBarCtrl@CReBar@@QBEAAVCReBarCtrl@@XZ 5f87aa1d f   afxinl1.obj
 0001:00079a2b       ?EnableDocking@CReBar@@QAEXK@Z 5f87aa2b f   afxinl1.obj
 0001:00079a5e       ??0CRectTracker@@QAE@XZ    5f87aa5e f   afxinl1.obj
 0001:00079aa9       ??0CBitmapButton@@QAE@XZ   5f87aaa9 f   afxinl1.obj
 0001:00079b2d       ?LoadBitmaps@CBitmapButton@@QAEHIIII@Z 5f87ab2d f   afxinl1.obj
 0001:00079b68       ?SetMinPage@CPrintInfo@@QAEXI@Z 5f87ab68 f   afxinl1.obj
 0001:00079b85       ?SetMaxPage@CPrintInfo@@QAEXI@Z 5f87ab85 f   afxinl1.obj
 0001:00079ba2       ?GetMinPage@CPrintInfo@@QBEIXZ 5f87aba2 f   afxinl1.obj
 0001:00079bbb       ?GetMaxPage@CPrintInfo@@QBEIXZ 5f87abbb f   afxinl1.obj
 0001:00079bd4       ?GetFromPage@CPrintInfo@@QBEIXZ 5f87abd4 f   afxinl1.obj
 0001:00079bed       ?GetToPage@CPrintInfo@@QBEIXZ 5f87abed f   afxinl1.obj
 0001:00079c06       ?GetEditCtrl@CEditView@@QBEAAVCEdit@@XZ 5f87ac06 f   afxinl1.obj
 0001:00079c20       ??_GCObject@@UAEPAXI@Z     5f87ac20 f i afxinl1.obj
 0001:00079c20       ??_ECObject@@UAEPAXI@Z     5f87ac20 f i afxinl1.obj
 0001:00079c50       ??_ECSimpleException@@UAEPAXI@Z 5f87ac50 f i afxinl1.obj
 0001:00079c50       ??_GCSimpleException@@UAEPAXI@Z 5f87ac50 f i afxinl1.obj
 0001:00079c80       ??_ECMemoryException@@UAEPAXI@Z 5f87ac80 f i afxinl1.obj
 0001:00079c80       ??_GCMemoryException@@UAEPAXI@Z 5f87ac80 f i afxinl1.obj
 0001:00079cb0       ??_GCNotSupportedException@@UAEPAXI@Z 5f87acb0 f i afxinl1.obj
 0001:00079cb0       ??_ECNotSupportedException@@UAEPAXI@Z 5f87acb0 f i afxinl1.obj
 0001:00079ce0       ??_ECArchiveException@@UAEPAXI@Z 5f87ace0 f i afxinl1.obj
 0001:00079ce0       ??_GCArchiveException@@UAEPAXI@Z 5f87ace0 f i afxinl1.obj
 0001:00079d10       ??_ECFileException@@UAEPAXI@Z 5f87ad10 f i afxinl1.obj
 0001:00079d10       ??_GCFileException@@UAEPAXI@Z 5f87ad10 f i afxinl1.obj
 0001:00079d40       ??_ECCommonDialog@@UAEPAXI@Z 5f87ad40 f i afxinl1.obj
 0001:00079d40       ??_GCCommonDialog@@UAEPAXI@Z 5f87ad40 f i afxinl1.obj
 0001:00079d70       ??1CCommonDialog@@UAE@XZ   5f87ad70 f i afxinl1.obj
 0001:00079d90       ??1CBitmapButton@@UAE@XZ   5f87ad90 f i afxinl1.obj
 0001:00079e10       ?_AfxTraceMsg@@YGXPBGPBUtagMSG@@@Z 5f87ae10 f   afxtrace.obj
 0001:0007a290       ?AfxGetApp@@YGPAVCWinApp@@XZ 5f87b290 f   afxinl2.obj
 0001:0007a29d       ?AfxGetInstanceHandle@@YGPAUHINSTANCE__@@XZ 5f87b29d f   afxinl2.obj
 0001:0007a2d2       ?AfxGetResourceHandle@@YGPAUHINSTANCE__@@XZ 5f87b2d2 f   afxinl2.obj
 0001:0007a307       ?AfxSetResourceHandle@@YGXPAUHINSTANCE__@@@Z 5f87b307 f   afxinl2.obj
 0001:0007a33c       ?AfxGetAppName@@YGPBGXZ    5f87b33c f   afxinl2.obj
 0001:0007a371       ?AfxOleGetMessageFilter@@YGPAVCOleMessageFilter@@XZ 5f87b371 f   afxinl2.obj
 0001:0007a390       ?AfxGetMainWnd@@YGPAVCWnd@@XZ 5f87b390 f   afxinl2.obj
 0001:0007a3c2       ??0AFX_MAINTAIN_STATE@@QAE@PAVAFX_MODULE_STATE@@@Z 5f87b3c2 f   afxinl2.obj
 0001:0007a3e0       ??1AFX_MAINTAIN_STATE2@@QAE@XZ 5f87b3e0 f   afxinl2.obj
 0001:0007a3f9       ??0CSize@@QAE@XZ           5f87b3f9 f   afxinl2.obj
 0001:0007a407       ??0CSize@@QAE@HH@Z         5f87b407 f   afxinl2.obj
 0001:0007a428       ??0CSize@@QAE@UtagSIZE@@@Z 5f87b428 f   afxinl2.obj
 0001:0007a446       ??0CSize@@QAE@UtagPOINT@@@Z 5f87b446 f   afxinl2.obj
 0001:0007a464       ??0CSize@@QAE@K@Z          5f87b464 f   afxinl2.obj
 0001:0007a492       ??8CSize@@QBEHUtagSIZE@@@Z 5f87b492 f   afxinl2.obj
 0001:0007a4c9       ??9CSize@@QBEHUtagSIZE@@@Z 5f87b4c9 f   afxinl2.obj
 0001:0007a500       ??YCSize@@QAEXUtagSIZE@@@Z 5f87b500 f   afxinl2.obj
 0001:0007a529       ??ZCSize@@QAEXUtagSIZE@@@Z 5f87b529 f   afxinl2.obj
 0001:0007a552       ??HCSize@@QBE?AV0@UtagSIZE@@@Z 5f87b552 f   afxinl2.obj
 0001:0007a58c       ??GCSize@@QBE?AV0@UtagSIZE@@@Z 5f87b58c f   afxinl2.obj
 0001:0007a5c6       ??GCSize@@QBE?AV0@XZ       5f87b5c6 f   afxinl2.obj
 0001:0007a5fe       ??HCSize@@QBE?AVCPoint@@UtagPOINT@@@Z 5f87b5fe f   afxinl2.obj
 0001:0007a638       ??GCSize@@QBE?AVCPoint@@UtagPOINT@@@Z 5f87b638 f   afxinl2.obj
 0001:0007a672       ??HCSize@@QBE?AVCRect@@PBUtagRECT@@@Z 5f87b672 f   afxinl2.obj
 0001:0007a6ca       ??GCSize@@QBE?AVCRect@@PBUtagRECT@@@Z 5f87b6ca f   afxinl2.obj
 0001:0007a722       ??0CPoint@@QAE@XZ          5f87b722 f   afxinl2.obj
 0001:0007a730       ??0CPoint@@QAE@HH@Z        5f87b730 f   afxinl2.obj
 0001:0007a751       ??0CPoint@@QAE@UtagPOINT@@@Z 5f87b751 f   afxinl2.obj
 0001:0007a76f       ??0CPoint@@QAE@UtagSIZE@@@Z 5f87b76f f   afxinl2.obj
 0001:0007a78d       ??0CPoint@@QAE@K@Z         5f87b78d f   afxinl2.obj
 0001:0007a7bb       ?Offset@CPoint@@QAEXHH@Z   5f87b7bb f   afxinl2.obj
 0001:0007a7e4       ?Offset@CPoint@@QAEXUtagPOINT@@@Z 5f87b7e4 f   afxinl2.obj
 0001:0007a80d       ?Offset@CPoint@@QAEXUtagSIZE@@@Z 5f87b80d f   afxinl2.obj
 0001:0007a836       ??8CPoint@@QBEHUtagPOINT@@@Z 5f87b836 f   afxinl2.obj
 0001:0007a86d       ??9CPoint@@QBEHUtagPOINT@@@Z 5f87b86d f   afxinl2.obj
 0001:0007a8a4       ??YCPoint@@QAEXUtagSIZE@@@Z 5f87b8a4 f   afxinl2.obj
 0001:0007a8cd       ??ZCPoint@@QAEXUtagSIZE@@@Z 5f87b8cd f   afxinl2.obj
 0001:0007a8f6       ??YCPoint@@QAEXUtagPOINT@@@Z 5f87b8f6 f   afxinl2.obj
 0001:0007a91f       ??ZCPoint@@QAEXUtagPOINT@@@Z 5f87b91f f   afxinl2.obj
 0001:0007a948       ??HCPoint@@QBE?AV0@UtagSIZE@@@Z 5f87b948 f   afxinl2.obj
 0001:0007a982       ??GCPoint@@QBE?AV0@UtagSIZE@@@Z 5f87b982 f   afxinl2.obj
 0001:0007a9bc       ??GCPoint@@QBE?AV0@XZ      5f87b9bc f   afxinl2.obj
 0001:0007a9f4       ??HCPoint@@QBE?AV0@UtagPOINT@@@Z 5f87b9f4 f   afxinl2.obj
 0001:0007aa2e       ??GCPoint@@QBE?AVCSize@@UtagPOINT@@@Z 5f87ba2e f   afxinl2.obj
 0001:0007aa68       ??HCPoint@@QBE?AVCRect@@PBUtagRECT@@@Z 5f87ba68 f   afxinl2.obj
 0001:0007aac0       ??GCPoint@@QBE?AVCRect@@PBUtagRECT@@@Z 5f87bac0 f   afxinl2.obj
 0001:0007ab18       ??0CRect@@QAE@XZ           5f87bb18 f   afxinl2.obj
 0001:0007ab26       ??0CRect@@QAE@HHHH@Z       5f87bb26 f   afxinl2.obj
 0001:0007ab59       ??0CRect@@QAE@ABUtagRECT@@@Z 5f87bb59 f   afxinl2.obj
 0001:0007ab77       ??0CRect@@QAE@PBUtagRECT@@@Z 5f87bb77 f   afxinl2.obj
 0001:0007ab95       ??0CRect@@QAE@UtagPOINT@@UtagSIZE@@@Z 5f87bb95 f   afxinl2.obj
 0001:0007abce       ??0CRect@@QAE@UtagPOINT@@0@Z 5f87bbce f   afxinl2.obj
 0001:0007ac01       ?Width@CRect@@QBEHXZ       5f87bc01 f   afxinl2.obj
 0001:0007ac17       ?Height@CRect@@QBEHXZ      5f87bc17 f   afxinl2.obj
 0001:0007ac2e       ?Size@CRect@@QBE?AVCSize@@XZ 5f87bc2e f   afxinl2.obj
 0001:0007ac6e       ?TopLeft@CRect@@QAEAAVCPoint@@XZ 5f87bc6e f   afxinl2.obj
 0001:0007ac7c       ?BottomRight@CRect@@QAEAAVCPoint@@XZ 5f87bc7c f   afxinl2.obj
 0001:0007ac8d       ?TopLeft@CRect@@QBEABVCPoint@@XZ 5f87bc8d f   afxinl2.obj
 0001:0007ac9b       ?BottomRight@CRect@@QBEABVCPoint@@XZ 5f87bc9b f   afxinl2.obj
 0001:0007acac       ?CenterPoint@CRect@@QBE?AVCPoint@@XZ 5f87bcac f   afxinl2.obj
 0001:0007acf6       ?SwapLeftRight@CRect@@QAEXXZ 5f87bcf6 f   afxinl2.obj
 0001:0007ad0d       ?SwapLeftRight@CRect@@SAXPAUtagRECT@@@Z 5f87bd0d f   afxinl2.obj
 0001:0007ad31       ??BCRect@@QAEPAUtagRECT@@XZ 5f87bd31 f   afxinl2.obj
 0001:0007ad3f       ??BCRect@@QBEPBUtagRECT@@XZ 5f87bd3f f   afxinl2.obj
 0001:0007ad4d       ?IsRectEmpty@CRect@@QBEHXZ 5f87bd4d f   afxinl2.obj
 0001:0007ad62       ?IsRectNull@CRect@@QBEHXZ  5f87bd62 f   afxinl2.obj
 0001:0007ada5       ?PtInRect@CRect@@QBEHUtagPOINT@@@Z 5f87bda5 f   afxinl2.obj
 0001:0007adc4       ?SetRect@CRect@@QAEXHHHH@Z 5f87bdc4 f   afxinl2.obj
 0001:0007adeb       ?SetRect@CRect@@QAEXUtagPOINT@@0@Z 5f87bdeb f   afxinl2.obj
 0001:0007ae12       ?SetRectEmpty@CRect@@QAEXXZ 5f87be12 f   afxinl2.obj
 0001:0007ae27       ?CopyRect@CRect@@QAEXPBUtagRECT@@@Z 5f87be27 f   afxinl2.obj
 0001:0007ae42       ?EqualRect@CRect@@QBEHPBUtagRECT@@@Z 5f87be42 f   afxinl2.obj
 0001:0007ae5d       ?InflateRect@CRect@@QAEXHH@Z 5f87be5d f   afxinl2.obj
 0001:0007ae7c       ?InflateRect@CRect@@QAEXUtagSIZE@@@Z 5f87be7c f   afxinl2.obj
 0001:0007ae9b       ?DeflateRect@CRect@@QAEXHH@Z 5f87be9b f   afxinl2.obj
 0001:0007aebe       ?DeflateRect@CRect@@QAEXUtagSIZE@@@Z 5f87bebe f   afxinl2.obj
 0001:0007aee1       ?OffsetRect@CRect@@QAEXHH@Z 5f87bee1 f   afxinl2.obj
 0001:0007af00       ?OffsetRect@CRect@@QAEXUtagPOINT@@@Z 5f87bf00 f   afxinl2.obj
 0001:0007af1f       ?OffsetRect@CRect@@QAEXUtagSIZE@@@Z 5f87bf1f f   afxinl2.obj
 0001:0007af3e       ?IntersectRect@CRect@@QAEHPBUtagRECT@@0@Z 5f87bf3e f   afxinl2.obj
 0001:0007af5d       ?UnionRect@CRect@@QAEHPBUtagRECT@@0@Z 5f87bf5d f   afxinl2.obj
 0001:0007af7c       ??4CRect@@QAEXABUtagRECT@@@Z 5f87bf7c f   afxinl2.obj
 0001:0007af97       ??8CRect@@QBEHABUtagRECT@@@Z 5f87bf97 f   afxinl2.obj
 0001:0007afb2       ??9CRect@@QBEHABUtagRECT@@@Z 5f87bfb2 f   afxinl2.obj
 0001:0007afd2       ??YCRect@@QAEXUtagPOINT@@@Z 5f87bfd2 f   afxinl2.obj
 0001:0007aff1       ??YCRect@@QAEXUtagSIZE@@@Z 5f87bff1 f   afxinl2.obj
 0001:0007b010       ??YCRect@@QAEXPBUtagRECT@@@Z 5f87c010 f   afxinl2.obj
 0001:0007b029       ??ZCRect@@QAEXUtagPOINT@@@Z 5f87c029 f   afxinl2.obj
 0001:0007b04c       ??ZCRect@@QAEXUtagSIZE@@@Z 5f87c04c f   afxinl2.obj
 0001:0007b06f       ??ZCRect@@QAEXPBUtagRECT@@@Z 5f87c06f f   afxinl2.obj
 0001:0007b088       ??_4CRect@@QAEXABUtagRECT@@@Z 5f87c088 f   afxinl2.obj
 0001:0007b0a7       ??_5CRect@@QAEXABUtagRECT@@@Z 5f87c0a7 f   afxinl2.obj
 0001:0007b0c6       ??HCRect@@QBE?AV0@UtagPOINT@@@Z 5f87c0c6 f   afxinl2.obj
 0001:0007b11e       ??GCRect@@QBE?AV0@UtagPOINT@@@Z 5f87c11e f   afxinl2.obj
 0001:0007b17a       ??HCRect@@QBE?AV0@UtagSIZE@@@Z 5f87c17a f   afxinl2.obj
 0001:0007b1d2       ??GCRect@@QBE?AV0@UtagSIZE@@@Z 5f87c1d2 f   afxinl2.obj
 0001:0007b22e       ??HCRect@@QBE?AV0@PBUtagRECT@@@Z 5f87c22e f   afxinl2.obj
 0001:0007b272       ??GCRect@@QBE?AV0@PBUtagRECT@@@Z 5f87c272 f   afxinl2.obj
 0001:0007b2b6       ??ICRect@@QBE?AV0@ABUtagRECT@@@Z 5f87c2b6 f   afxinl2.obj
 0001:0007b2fc       ??UCRect@@QBE?AV0@ABUtagRECT@@@Z 5f87c2fc f   afxinl2.obj
 0001:0007b342       ?SubtractRect@CRect@@QAEHPBUtagRECT@@0@Z 5f87c342 f   afxinl2.obj
 0001:0007b361       ??6@YGAAVCArchive@@AAV0@UtagSIZE@@@Z 5f87c361 f   afxinl2.obj
 0001:0007b379       ??6@YGAAVCArchive@@AAV0@UtagPOINT@@@Z 5f87c379 f   afxinl2.obj
 0001:0007b391       ??6@YGAAVCArchive@@AAV0@ABUtagRECT@@@Z 5f87c391 f   afxinl2.obj
 0001:0007b3a9       ??5@YGAAVCArchive@@AAV0@AAUtagSIZE@@@Z 5f87c3a9 f   afxinl2.obj
 0001:0007b3c1       ??5@YGAAVCArchive@@AAV0@AAUtagPOINT@@@Z 5f87c3c1 f   afxinl2.obj
 0001:0007b3d9       ??5@YGAAVCArchive@@AAV0@AAUtagRECT@@@Z 5f87c3d9 f   afxinl2.obj
 0001:0007b3f1       ??0CResourceException@@QAE@XZ 5f87c3f1 f   afxinl2.obj
 0001:0007b410       ??0CResourceException@@QAE@HI@Z 5f87c410 f   afxinl2.obj
 0001:0007b441       ??1CResourceException@@UAE@XZ 5f87c441 f   afxinl2.obj
 0001:0007b45d       ??0CUserException@@QAE@XZ  5f87c45d f   afxinl2.obj
 0001:0007b47c       ??0CUserException@@QAE@HI@Z 5f87c47c f   afxinl2.obj
 0001:0007b4ad       ??1CUserException@@UAE@XZ  5f87c4ad f   afxinl2.obj
 0001:0007b4c9       ??BCGdiObject@@QBEPAXXZ    5f87c4c9 f   afxinl2.obj
 0001:0007b4f1       ?GetSafeHandle@CGdiObject@@QBEPAXXZ 5f87c4f1 f   afxinl2.obj
 0001:0007b519       ??0CGdiObject@@QAE@XZ      5f87c519 f   afxinl2.obj
 0001:0007b542       ??1CGdiObject@@UAE@XZ      5f87c542 f   afxinl2.obj
 0001:0007b593       ?GetObjectW@CGdiObject@@QBEHHPAX@Z 5f87c593 f   afxinl2.obj
 0001:0007b5de       ?CreateStockObject@CGdiObject@@QAEHH@Z 5f87c5de f   afxinl2.obj
 0001:0007b607       ?UnrealizeObject@CGdiObject@@QAEHXZ 5f87c607 f   afxinl2.obj
 0001:0007b648       ?GetObjectType@CGdiObject@@QBEIXZ 5f87c648 f   afxinl2.obj
 0001:0007b660       ??8CGdiObject@@QBEHABV0@@Z 5f87c660 f   afxinl2.obj
 0001:0007b682       ??9CGdiObject@@QBEHABV0@@Z 5f87c682 f   afxinl2.obj
 0001:0007b6a4       ??BCPen@@QBEPAUHPEN__@@XZ  5f87c6a4 f   afxinl2.obj
 0001:0007b6cc       ?FromHandle@CPen@@SGPAV1@PAUHPEN__@@@Z 5f87c6cc f   afxinl2.obj
 0001:0007b6dc       ??0CPen@@QAE@XZ            5f87c6dc f   afxinl2.obj
 0001:0007b6fb       ??1CPen@@UAE@XZ            5f87c6fb f   afxinl2.obj
 0001:0007b717       ?CreatePen@CPen@@QAEHHHK@Z 5f87c717 f   afxinl2.obj
 0001:0007b73f       ?CreatePenIndirect@CPen@@QAEHPAUtagLOGPEN@@@Z 5f87c73f f   afxinl2.obj
 0001:0007b75f       ?CreatePen@CPen@@QAEHHHPBUtagLOGBRUSH@@HPBK@Z 5f87c75f f   afxinl2.obj
 0001:0007b78f       ?GetExtLogPen@CPen@@QAEHPAUtagEXTLOGPEN@@@Z 5f87c78f f   afxinl2.obj
 0001:0007b7d8       ?GetLogPen@CPen@@QAEHPAUtagLOGPEN@@@Z 5f87c7d8 f   afxinl2.obj
 0001:0007b821       ??BCBrush@@QBEPAUHBRUSH__@@XZ 5f87c821 f   afxinl2.obj
 0001:0007b849       ?FromHandle@CBrush@@SGPAV1@PAUHBRUSH__@@@Z 5f87c849 f   afxinl2.obj
 0001:0007b859       ??0CBrush@@QAE@XZ          5f87c859 f   afxinl2.obj
 0001:0007b878       ??1CBrush@@UAE@XZ          5f87c878 f   afxinl2.obj
 0001:0007b894       ?CreateSolidBrush@CBrush@@QAEHK@Z 5f87c894 f   afxinl2.obj
 0001:0007b8b4       ?CreateHatchBrush@CBrush@@QAEHHK@Z 5f87c8b4 f   afxinl2.obj
 0001:0007b8d8       ?CreateBrushIndirect@CBrush@@QAEHPBUtagLOGBRUSH@@@Z 5f87c8d8 f   afxinl2.obj
 0001:0007b8f8       ?CreatePatternBrush@CBrush@@QAEHPAVCBitmap@@@Z 5f87c8f8 f   afxinl2.obj
 0001:0007b91d       ?CreateDIBPatternBrush@CBrush@@QAEHPBXI@Z 5f87c91d f   afxinl2.obj
 0001:0007b941       ?CreateSysColorBrush@CBrush@@QAEHH@Z 5f87c941 f   afxinl2.obj
 0001:0007b961       ?GetLogBrush@CBrush@@QAEHPAUtagLOGBRUSH@@@Z 5f87c961 f   afxinl2.obj
 0001:0007b9aa       ??BCFont@@QBEPAUHFONT__@@XZ 5f87c9aa f   afxinl2.obj
 0001:0007b9d2       ?FromHandle@CFont@@SGPAV1@PAUHFONT__@@@Z 5f87c9d2 f   afxinl2.obj
 0001:0007b9e2       ??0CFont@@QAE@XZ           5f87c9e2 f   afxinl2.obj
 0001:0007ba01       ??1CFont@@UAE@XZ           5f87ca01 f   afxinl2.obj
 0001:0007ba1d       ?CreateFontIndirectW@CFont@@QAEHPBUtagLOGFONTW@@@Z 5f87ca1d f   afxinl2.obj
 0001:0007ba3d       ?CreateFontW@CFont@@QAEHHHHHHEEEEEEEEPBG@Z 5f87ca3d f   afxinl2.obj
 0001:0007babf       ?GetLogFont@CFont@@QAEHPAUtagLOGFONTW@@@Z 5f87cabf f   afxinl2.obj
 0001:0007bb08       ??BCBitmap@@QBEPAUHBITMAP__@@XZ 5f87cb08 f   afxinl2.obj
 0001:0007bb30       ?FromHandle@CBitmap@@SGPAV1@PAUHBITMAP__@@@Z 5f87cb30 f   afxinl2.obj
 0001:0007bb40       ??0CBitmap@@QAE@XZ         5f87cb40 f   afxinl2.obj
 0001:0007bb5f       ??1CBitmap@@UAE@XZ         5f87cb5f f   afxinl2.obj
 0001:0007bb7b       ?CreateBitmap@CBitmap@@QAEHHHIIPBX@Z 5f87cb7b f   afxinl2.obj
 0001:0007bbab       ?CreateBitmapIndirect@CBitmap@@QAEHPAUtagBITMAP@@@Z 5f87cbab f   afxinl2.obj
 0001:0007bbcb       ?SetBitmapBits@CBitmap@@QAEKKPBX@Z 5f87cbcb f   afxinl2.obj
 0001:0007bbed       ?GetBitmapBits@CBitmap@@QBEKKPAX@Z 5f87cbed f   afxinl2.obj
 0001:0007bc0f       ?LoadBitmapW@CBitmap@@QAEHPBG@Z 5f87cc0f f   afxinl2.obj
 0001:0007bc3b       ?LoadMappedBitmap@CBitmap@@QAEHIIPAU_COLORMAP@@H@Z 5f87cc3b f   afxinl2.obj
 0001:0007bc7f       ?SetBitmapDimension@CBitmap@@QAE?AVCSize@@HH@Z 5f87cc7f f   afxinl2.obj
 0001:0007bcde       ?GetBitmapDimension@CBitmap@@QBE?AVCSize@@XZ 5f87ccde f   afxinl2.obj
 0001:0007bd35       ?LoadBitmapW@CBitmap@@QAEHI@Z 5f87cd35 f   afxinl2.obj
 0001:0007bd6c       ?LoadOEMBitmap@CBitmap@@QAEHI@Z 5f87cd6c f   afxinl2.obj
 0001:0007bd93       ?CreateCompatibleBitmap@CBitmap@@QAEHPAVCDC@@HH@Z 5f87cd93 f   afxinl2.obj
 0001:0007bdbe       ?CreateDiscardableBitmap@CBitmap@@QAEHPAVCDC@@HH@Z 5f87cdbe f   afxinl2.obj
 0001:0007bde9       ?GetBitmap@CBitmap@@QAEHPAUtagBITMAP@@@Z 5f87cde9 f   afxinl2.obj
 0001:0007be32       ??BCPalette@@QBEPAUHPALETTE__@@XZ 5f87ce32 f   afxinl2.obj
 0001:0007be5a       ?FromHandle@CPalette@@SGPAV1@PAUHPALETTE__@@@Z 5f87ce5a f   afxinl2.obj
 0001:0007be6a       ??0CPalette@@QAE@XZ        5f87ce6a f   afxinl2.obj
 0001:0007be89       ??1CPalette@@UAE@XZ        5f87ce89 f   afxinl2.obj
 0001:0007bea5       ?CreatePalette@CPalette@@QAEHPAUtagLOGPALETTE@@@Z 5f87cea5 f   afxinl2.obj
 0001:0007bec5       ?CreateHalftonePalette@CPalette@@QAEHPAVCDC@@@Z 5f87cec5 f   afxinl2.obj
 0001:0007bf17       ?GetPaletteEntries@CPalette@@QBEIIIPAUtagPALETTEENTRY@@@Z 5f87cf17 f   afxinl2.obj
 0001:0007bf66       ?SetPaletteEntries@CPalette@@QAEIIIPAUtagPALETTEENTRY@@@Z 5f87cf66 f   afxinl2.obj
 0001:0007bfb5       ?AnimatePalette@CPalette@@QAEXIIPAUtagPALETTEENTRY@@@Z 5f87cfb5 f   afxinl2.obj
 0001:0007c004       ?GetNearestPaletteIndex@CPalette@@QBEIK@Z 5f87d004 f   afxinl2.obj
 0001:0007c04b       ?ResizePalette@CPalette@@QAEHI@Z 5f87d04b f   afxinl2.obj
 0001:0007c092       ?GetEntryCount@CPalette@@QAEHXZ 5f87d092 f   afxinl2.obj
 0001:0007c0e3       ??BCRgn@@QBEPAUHRGN__@@XZ  5f87d0e3 f   afxinl2.obj
 0001:0007c10b       ?FromHandle@CRgn@@SGPAV1@PAUHRGN__@@@Z 5f87d10b f   afxinl2.obj
 0001:0007c11b       ??0CRgn@@QAE@XZ            5f87d11b f   afxinl2.obj
 0001:0007c13a       ??1CRgn@@UAE@XZ            5f87d13a f   afxinl2.obj
 0001:0007c156       ?CreateRectRgn@CRgn@@QAEHHHHH@Z 5f87d156 f   afxinl2.obj
 0001:0007c182       ?CreateRectRgnIndirect@CRgn@@QAEHPBUtagRECT@@@Z 5f87d182 f   afxinl2.obj
 0001:0007c1a2       ?CreateEllipticRgn@CRgn@@QAEHHHHH@Z 5f87d1a2 f   afxinl2.obj
 0001:0007c1ce       ?CreateEllipticRgnIndirect@CRgn@@QAEHPBUtagRECT@@@Z 5f87d1ce f   afxinl2.obj
 0001:0007c1ee       ?CreatePolygonRgn@CRgn@@QAEHPAUtagPOINT@@HH@Z 5f87d1ee f   afxinl2.obj
 0001:0007c216       ?CreatePolyPolygonRgn@CRgn@@QAEHPAUtagPOINT@@PAHHH@Z 5f87d216 f   afxinl2.obj
 0001:0007c242       ?CreateRoundRectRgn@CRgn@@QAEHHHHHHH@Z 5f87d242 f   afxinl2.obj
 0001:0007c276       ?CreateFromPath@CRgn@@QAEHPAVCDC@@@Z 5f87d276 f   afxinl2.obj
 0001:0007c2bf       ?CreateFromData@CRgn@@QAEHPBUtagXFORM@@HPBU_RGNDATA@@@Z 5f87d2bf f   afxinl2.obj
 0001:0007c2e7       ?GetRegionData@CRgn@@QBEHPAU_RGNDATA@@H@Z 5f87d2e7 f   afxinl2.obj
 0001:0007c332       ?SetRectRgn@CRgn@@QAEXHHHH@Z 5f87d332 f   afxinl2.obj
 0001:0007c385       ?SetRectRgn@CRgn@@QAEXPBUtagRECT@@@Z 5f87d385 f   afxinl2.obj
 0001:0007c3e3       ?CombineRgn@CRgn@@QAEHPAV1@0H@Z 5f87d3e3 f   afxinl2.obj
 0001:0007c43c       ?CopyRgn@CRgn@@QAEHPAV1@@Z 5f87d43c f   afxinl2.obj
 0001:0007c48c       ?EqualRgn@CRgn@@QBEHPAV1@@Z 5f87d48c f   afxinl2.obj
 0001:0007c4d8       ?OffsetRgn@CRgn@@QAEHHH@Z  5f87d4d8 f   afxinl2.obj
 0001:0007c523       ?OffsetRgn@CRgn@@QAEHUtagPOINT@@@Z 5f87d523 f   afxinl2.obj
 0001:0007c56e       ?GetRgnBox@CRgn@@QBEHPAUtagRECT@@@Z 5f87d56e f   afxinl2.obj
 0001:0007c5b5       ?PtInRegion@CRgn@@QBEHHH@Z 5f87d5b5 f   afxinl2.obj
 0001:0007c600       ?PtInRegion@CRgn@@QBEHUtagPOINT@@@Z 5f87d600 f   afxinl2.obj
 0001:0007c64b       ?RectInRegion@CRgn@@QBEHPBUtagRECT@@@Z 5f87d64b f   afxinl2.obj
 0001:0007c692       ??BCDC@@QBEPAUHDC__@@XZ    5f87d692 f   afxinl2.obj
 0001:0007c6ba       ?GetSafeHdc@CDC@@QBEPAUHDC__@@XZ 5f87d6ba f   afxinl2.obj
 0001:0007c6e2       ?GetWindow@CDC@@QBEPAVCWnd@@XZ 5f87d6e2 f   afxinl2.obj
 0001:0007c729       ?IsPrinting@CDC@@QBEHXZ    5f87d729 f   afxinl2.obj
 0001:0007c73a       ?CreateDCW@CDC@@QAEHPBG00PBX@Z 5f87d73a f   afxinl2.obj
 0001:0007c766       ?CreateICW@CDC@@QAEHPBG00PBX@Z 5f87d766 f   afxinl2.obj
 0001:0007c792       ?CreateCompatibleDC@CDC@@QAEHPAV1@@Z 5f87d792 f   afxinl2.obj
 0001:0007c7b7       ?ExcludeUpdateRgn@CDC@@QAEHPAVCWnd@@@Z 5f87d7b7 f   afxinl2.obj
 0001:0007c801       ?GetDeviceCaps@CDC@@QBEHH@Z 5f87d801 f   afxinl2.obj
 0001:0007c848       ?GetBrushOrg@CDC@@QBE?AVCPoint@@XZ 5f87d848 f   afxinl2.obj
 0001:0007c8c2       ?SetBrushOrg@CDC@@QAE?AVCPoint@@HH@Z 5f87d8c2 f   afxinl2.obj
 0001:0007c944       ?SetBrushOrg@CDC@@QAE?AVCPoint@@UtagPOINT@@@Z 5f87d944 f   afxinl2.obj
 0001:0007c9c4       ?EnumObjects@CDC@@QAEHHP6GHPAXJ@ZJ@Z 5f87d9c4 f   afxinl2.obj
 0001:0007ca13       ?SelectObject@CDC@@QAEPAVCBitmap@@PAV2@@Z 5f87da13 f   afxinl2.obj
 0001:0007ca5e       ?SelectObject@CDC@@QAEPAVCGdiObject@@PAV2@@Z 5f87da5e f   afxinl2.obj
 0001:0007caa9       ?SelectObject@CDC@@QAEPAXPAX@Z 5f87daa9 f   afxinl2.obj
 0001:0007cb0c       ?GetNearestColor@CDC@@QBEKK@Z 5f87db0c f   afxinl2.obj
 0001:0007cb53       ?RealizePalette@CDC@@QAEIXZ 5f87db53 f   afxinl2.obj
 0001:0007cb94       ?UpdateColors@CDC@@QAEXXZ  5f87db94 f   afxinl2.obj
 0001:0007cbd5       ?GetBkColor@CDC@@QBEKXZ    5f87dbd5 f   afxinl2.obj
 0001:0007cc16       ?GetBkMode@CDC@@QBEHXZ     5f87dc16 f   afxinl2.obj
 0001:0007cc57       ?GetPolyFillMode@CDC@@QBEHXZ 5f87dc57 f   afxinl2.obj
 0001:0007cc98       ?GetROP2@CDC@@QBEHXZ       5f87dc98 f   afxinl2.obj
 0001:0007ccd9       ?GetStretchBltMode@CDC@@QBEHXZ 5f87dcd9 f   afxinl2.obj
 0001:0007cd1a       ?GetTextColor@CDC@@QBEKXZ  5f87dd1a f   afxinl2.obj
 0001:0007cd5b       ?GetMapMode@CDC@@QBEHXZ    5f87dd5b f   afxinl2.obj
 0001:0007cd9c       ?GetViewportOrg@CDC@@QBE?AVCPoint@@XZ 5f87dd9c f   afxinl2.obj
 0001:0007ce16       ?GetViewportExt@CDC@@QBE?AVCSize@@XZ 5f87de16 f   afxinl2.obj
 0001:0007ce90       ?GetWindowOrg@CDC@@QBE?AVCPoint@@XZ 5f87de90 f   afxinl2.obj
 0001:0007cf0a       ?GetWindowExt@CDC@@QBE?AVCSize@@XZ 5f87df0a f   afxinl2.obj
 0001:0007cf84       ?SetViewportOrg@CDC@@QAE?AVCPoint@@UtagPOINT@@@Z 5f87df84 f   afxinl2.obj
 0001:0007cfe3       ?SetViewportExt@CDC@@QAE?AVCSize@@UtagSIZE@@@Z 5f87dfe3 f   afxinl2.obj
 0001:0007d042       ?SetWindowOrg@CDC@@QAE?AVCPoint@@UtagPOINT@@@Z 5f87e042 f   afxinl2.obj
 0001:0007d09e       ?SetWindowExt@CDC@@QAE?AVCSize@@UtagSIZE@@@Z 5f87e09e f   afxinl2.obj
 0001:0007d0fd       ?DPtoLP@CDC@@QBEXPAUtagPOINT@@H@Z 5f87e0fd f   afxinl2.obj
 0001:0007d166       ?DPtoLP@CDC@@QBEXPAUtagRECT@@@Z 5f87e166 f   afxinl2.obj
 0001:0007d1cd       ?LPtoDP@CDC@@QBEXPAUtagPOINT@@H@Z 5f87e1cd f   afxinl2.obj
 0001:0007d236       ?LPtoDP@CDC@@QBEXPAUtagRECT@@@Z 5f87e236 f   afxinl2.obj
 0001:0007d29d       ?FillRgn@CDC@@QAEHPAVCRgn@@PAVCBrush@@@Z 5f87e29d f   afxinl2.obj
 0001:0007d2f2       ?FrameRgn@CDC@@QAEHPAVCRgn@@PAVCBrush@@HH@Z 5f87e2f2 f   afxinl2.obj
 0001:0007d34f       ?InvertRgn@CDC@@QAEHPAVCRgn@@@Z 5f87e34f f   afxinl2.obj
 0001:0007d39b       ?PaintRgn@CDC@@QAEHPAVCRgn@@@Z 5f87e39b f   afxinl2.obj
 0001:0007d3e7       ?PtVisible@CDC@@UBEHHH@Z   5f87e3e7 f   afxinl2.obj
 0001:0007d432       ?PtVisible@CDC@@QBEHUtagPOINT@@@Z 5f87e432 f   afxinl2.obj
 0001:0007d47b       ?RectVisible@CDC@@UBEHPBUtagRECT@@@Z 5f87e47b f   afxinl2.obj
 0001:0007d4c2       ?GetCurrentPosition@CDC@@QBE?AVCPoint@@XZ 5f87e4c2 f   afxinl2.obj
 0001:0007d53c       ?MoveTo@CDC@@QAE?AVCPoint@@UtagPOINT@@@Z 5f87e53c f   afxinl2.obj
 0001:0007d598       ?LineTo@CDC@@QAEHUtagPOINT@@@Z 5f87e598 f   afxinl2.obj
 0001:0007d5de       ?Arc@CDC@@QAEHHHHHHHHH@Z   5f87e5de f   afxinl2.obj
 0001:0007d641       ?Arc@CDC@@QAEHPBUtagRECT@@UtagPOINT@@1@Z 5f87e641 f   afxinl2.obj
 0001:0007d6af       ?Polyline@CDC@@QAEHPAUtagPOINT@@H@Z 5f87e6af f   afxinl2.obj
 0001:0007d6fa       ?FillRect@CDC@@QAEXPBUtagRECT@@PAVCBrush@@@Z 5f87e6fa f   afxinl2.obj
 0001:0007d74a       ?FrameRect@CDC@@QAEXPBUtagRECT@@PAVCBrush@@@Z 5f87e74a f   afxinl2.obj
 0001:0007d79a       ?InvertRect@CDC@@QAEXPBUtagRECT@@@Z 5f87e79a f   afxinl2.obj
 0001:0007d7e1       ?DrawIcon@CDC@@QAEHHHPAUHICON__@@@Z 5f87e7e1 f   afxinl2.obj
 0001:0007d830       ?DrawIcon@CDC@@QAEHUtagPOINT@@PAUHICON__@@@Z 5f87e830 f   afxinl2.obj
 0001:0007d87f       ?DrawState@CDC@@QAEHVCPoint@@VCSize@@PAUHBITMAP__@@IPAUHBRUSH__@@@Z 5f87e87f f   afxinl2.obj
 0001:0007d8e4       ?DrawState@CDC@@QAEHVCPoint@@VCSize@@PAVCBitmap@@IPAVCBrush@@@Z 5f87e8e4 f   afxinl2.obj
 0001:0007d953       ?DrawState@CDC@@QAEHVCPoint@@VCSize@@PAUHICON__@@IPAUHBRUSH__@@@Z 5f87e953 f   afxinl2.obj
 0001:0007d9b8       ?DrawState@CDC@@QAEHVCPoint@@VCSize@@PAUHICON__@@IPAVCBrush@@@Z 5f87e9b8 f   afxinl2.obj
 0001:0007da22       ?DrawState@CDC@@QAEHVCPoint@@VCSize@@PBGIHHPAUHBRUSH__@@@Z 5f87ea22 f   afxinl2.obj
 0001:0007da92       ?DrawState@CDC@@QAEHVCPoint@@VCSize@@PBGIHHPAVCBrush@@@Z 5f87ea92 f   afxinl2.obj
 0001:0007db07       ?DrawState@CDC@@QAEHVCPoint@@VCSize@@P6GHPAUHDC__@@JIHH@ZJIPAUHBRUSH__@@@Z 5f87eb07 f   afxinl2.obj
 0001:0007db6b       ?DrawState@CDC@@QAEHVCPoint@@VCSize@@P6GHPAUHDC__@@JIHH@ZJIPAVCBrush@@@Z 5f87eb6b f   afxinl2.obj
 0001:0007dbd4       ?DrawEdge@CDC@@QAEHPAUtagRECT@@II@Z 5f87ebd4 f   afxinl2.obj
 0001:0007dc23       ?DrawFrameControl@CDC@@QAEHPAUtagRECT@@II@Z 5f87ec23 f   afxinl2.obj
 0001:0007dc72       ?Chord@CDC@@QAEHHHHHHHHH@Z 5f87ec72 f   afxinl2.obj
 0001:0007dcd5       ?Chord@CDC@@QAEHPBUtagRECT@@UtagPOINT@@1@Z 5f87ecd5 f   afxinl2.obj
 0001:0007dd43       ?DrawFocusRect@CDC@@QAEXPBUtagRECT@@@Z 5f87ed43 f   afxinl2.obj
 0001:0007dd8a       ?Ellipse@CDC@@QAEHHHHH@Z   5f87ed8a f   afxinl2.obj
 0001:0007dddd       ?Ellipse@CDC@@QAEHPBUtagRECT@@@Z 5f87eddd f   afxinl2.obj
 0001:0007de3b       ?Pie@CDC@@QAEHHHHHHHHH@Z   5f87ee3b f   afxinl2.obj
 0001:0007de9e       ?Pie@CDC@@QAEHPBUtagRECT@@UtagPOINT@@1@Z 5f87ee9e f   afxinl2.obj
 0001:0007df0c       ?Polygon@CDC@@QAEHPAUtagPOINT@@H@Z 5f87ef0c f   afxinl2.obj
 0001:0007df57       ?PolyPolygon@CDC@@QAEHPAUtagPOINT@@PAHH@Z 5f87ef57 f   afxinl2.obj
 0001:0007dfa6       ?Rectangle@CDC@@QAEHHHHH@Z 5f87efa6 f   afxinl2.obj
 0001:0007dff9       ?Rectangle@CDC@@QAEHPBUtagRECT@@@Z 5f87eff9 f   afxinl2.obj
 0001:0007e057       ?RoundRect@CDC@@QAEHHHHHHH@Z 5f87f057 f   afxinl2.obj
 0001:0007e0b2       ?RoundRect@CDC@@QAEHPBUtagRECT@@UtagPOINT@@@Z 5f87f0b2 f   afxinl2.obj
 0001:0007e118       ?PatBlt@CDC@@QAEHHHHHK@Z   5f87f118 f   afxinl2.obj
 0001:0007e16f       ?BitBlt@CDC@@QAEHHHHHPAV1@HHK@Z 5f87f16f f   afxinl2.obj
 0001:0007e1d7       ?StretchBlt@CDC@@QAEHHHHHPAV1@HHHHK@Z 5f87f1d7 f   afxinl2.obj
 0001:0007e247       ?GetPixel@CDC@@QBEKHH@Z    5f87f247 f   afxinl2.obj
 0001:0007e292       ?GetPixel@CDC@@QBEKUtagPOINT@@@Z 5f87f292 f   afxinl2.obj
 0001:0007e2dd       ?SetPixel@CDC@@QAEKHHK@Z   5f87f2dd f   afxinl2.obj
 0001:0007e32c       ?SetPixel@CDC@@QAEKUtagPOINT@@K@Z 5f87f32c f   afxinl2.obj
 0001:0007e37b       ?FloodFill@CDC@@QAEHHHK@Z  5f87f37b f   afxinl2.obj
 0001:0007e3ca       ?ExtFloodFill@CDC@@QAEHHHKI@Z 5f87f3ca f   afxinl2.obj
 0001:0007e41d       ?TextOutW@CDC@@UAEHHHPBGH@Z 5f87f41d f   afxinl2.obj
 0001:0007e470       ?TextOutW@CDC@@QAEHHHABVCString@@@Z 5f87f470 f   afxinl2.obj
 0001:0007e4cb       ?ExtTextOutW@CDC@@UAEHHHIPBUtagRECT@@PBGIPAH@Z 5f87f4cb f   afxinl2.obj
 0001:0007e52a       ?ExtTextOutW@CDC@@QAEHHHIPBUtagRECT@@ABVCString@@PAH@Z 5f87f52a f   afxinl2.obj
 0001:0007e593       ?TabbedTextOutW@CDC@@UAE?AVCSize@@HHPBGHHPAHH@Z 5f87f593 f   afxinl2.obj
 0001:0007e5fe       ?TabbedTextOutW@CDC@@QAE?AVCSize@@HHABVCString@@HPAHH@Z 5f87f5fe f   afxinl2.obj
 0001:0007e673       ?DrawTextW@CDC@@UAEHPBGHPAUtagRECT@@I@Z 5f87f673 f   afxinl2.obj
 0001:0007e6c6       ?DrawTextW@CDC@@QAEHABVCString@@PAUtagRECT@@I@Z 5f87f6c6 f   afxinl2.obj
 0001:0007e777       ?GetTextExtent@CDC@@QBE?AVCSize@@PBGH@Z 5f87f777 f   afxinl2.obj
 0001:0007e7f9       ?GetTextExtent@CDC@@QBE?AVCSize@@ABVCString@@@Z 5f87f7f9 f   afxinl2.obj
 0001:0007e885       ?GetOutputTextExtent@CDC@@QBE?AVCSize@@PBGH@Z 5f87f885 f   afxinl2.obj
 0001:0007e907       ?GetOutputTextExtent@CDC@@QBE?AVCSize@@ABVCString@@@Z 5f87f907 f   afxinl2.obj
 0001:0007e993       ?GetTabbedTextExtentW@CDC@@QBE?AVCSize@@PBGHHPAH@Z 5f87f993 f   afxinl2.obj
 0001:0007e9f2       ?GetTabbedTextExtentW@CDC@@QBE?AVCSize@@ABVCString@@HPAH@Z 5f87f9f2 f   afxinl2.obj
 0001:0007ea5b       ?GetOutputTabbedTextExtent@CDC@@QBE?AVCSize@@PBGHHPAH@Z 5f87fa5b f   afxinl2.obj
 0001:0007eaba       ?GetOutputTabbedTextExtent@CDC@@QBE?AVCSize@@ABVCString@@HPAH@Z 5f87faba f   afxinl2.obj
 0001:0007eb23       ?GrayStringW@CDC@@UAEHPAVCBrush@@P6GHPAUHDC__@@JH@ZJHHHHH@Z 5f87fb23 f   afxinl2.obj
 0001:0007eb8b       ?GetTextAlign@CDC@@QBEIXZ  5f87fb8b f   afxinl2.obj
 0001:0007ebcc       ?GetTextFaceW@CDC@@QBEHHPAG@Z 5f87fbcc f   afxinl2.obj
 0001:0007ec17       ?GetTextFaceW@CDC@@QBEHAAVCString@@@Z 5f87fc17 f   afxinl2.obj
 0001:0007ec7f       ?GetTextMetricsW@CDC@@QBEHPAUtagTEXTMETRICW@@@Z 5f87fc7f f   afxinl2.obj
 0001:0007ecc6       ?GetOutputTextMetrics@CDC@@QBEHPAUtagTEXTMETRICW@@@Z 5f87fcc6 f   afxinl2.obj
 0001:0007ed0d       ?GetTextCharacterExtra@CDC@@QBEHXZ 5f87fd0d f   afxinl2.obj
 0001:0007ed4e       ?GetCharWidthW@CDC@@QBEHIIPAH@Z 5f87fd4e f   afxinl2.obj
 0001:0007ed9d       ?GetOutputCharWidth@CDC@@QBEHIIPAH@Z 5f87fd9d f   afxinl2.obj
 0001:0007edec       ?GetAspectRatioFilter@CDC@@QBE?AVCSize@@XZ 5f87fdec f   afxinl2.obj
 0001:0007ee66       ?ScrollDC@CDC@@QAEHHHPBUtagRECT@@0PAVCRgn@@PAU2@@Z 5f87fe66 f   afxinl2.obj
 0001:0007eec6       ?Escape@CDC@@UAEHHHPBDPAX@Z 5f87fec6 f   afxinl2.obj
 0001:0007ef19       ?SetBoundsRect@CDC@@QAEIPBUtagRECT@@I@Z 5f87ff19 f   afxinl2.obj
 0001:0007ef64       ?GetBoundsRect@CDC@@QAEIPAUtagRECT@@I@Z 5f87ff64 f   afxinl2.obj
 0001:0007efaf       ?ResetDCW@CDC@@QAEHPBU_devicemodeW@@@Z 5f87ffaf f   afxinl2.obj
 0001:0007effc       ?GetOutlineTextMetricsW@CDC@@QBEIIPAU_OUTLINETEXTMETRICW@@@Z 5f87fffc f   afxinl2.obj
 0001:0007f047       ?GetCharABCWidthsW@CDC@@QBEHIIPAU_ABC@@@Z 5f880047 f   afxinl2.obj
 0001:0007f096       ?GetFontData@CDC@@QBEKKKPAXK@Z 5f880096 f   afxinl2.obj
 0001:0007f0e9       ?GetKerningPairsW@CDC@@QBEHHPAUtagKERNINGPAIR@@@Z 5f8800e9 f   afxinl2.obj
 0001:0007f134       ?GetGlyphOutlineW@CDC@@QBEKIIPAU_GLYPHMETRICS@@KPAXPBU_MAT2@@@Z 5f880134 f   afxinl2.obj
 0001:0007f18f       ?StartDocW@CDC@@QAEHPAU_DOCINFOW@@@Z 5f88018f f   afxinl2.obj
 0001:0007f1d6       ?StartPage@CDC@@QAEHXZ     5f8801d6 f   afxinl2.obj
 0001:0007f217       ?EndPage@CDC@@QAEHXZ       5f880217 f   afxinl2.obj
 0001:0007f258       ?SetAbortProc@CDC@@QAEHP6GHPAUHDC__@@H@Z@Z 5f880258 f   afxinl2.obj
 0001:0007f29f       ?AbortDoc@CDC@@QAEHXZ      5f88029f f   afxinl2.obj
 0001:0007f2e0       ?EndDoc@CDC@@QAEHXZ        5f8802e0 f   afxinl2.obj
 0001:0007f321       ?MaskBlt@CDC@@QAEHHHHHPAV1@HHAAVCBitmap@@HHK@Z 5f880321 f   afxinl2.obj
 0001:0007f398       ?PlgBlt@CDC@@QAEHPAUtagPOINT@@PAV1@HHHHAAVCBitmap@@HH@Z 5f880398 f   afxinl2.obj
 0001:0007f407       ?SetPixelV@CDC@@QAEHHHK@Z  5f880407 f   afxinl2.obj
 0001:0007f456       ?SetPixelV@CDC@@QAEHUtagPOINT@@K@Z 5f880456 f   afxinl2.obj
 0001:0007f4a5       ?AngleArc@CDC@@QAEHHHHMM@Z 5f8804a5 f   afxinl2.obj
 0001:0007f4fc       ?ArcTo@CDC@@QAEHPBUtagRECT@@UtagPOINT@@1@Z 5f8804fc f   afxinl2.obj
 0001:0007f565       ?GetArcDirection@CDC@@QBEHXZ 5f880565 f   afxinl2.obj
 0001:0007f5a6       ?PolyPolyline@CDC@@QAEHPBUtagPOINT@@PBKH@Z 5f8805a6 f   afxinl2.obj
 0001:0007f5f5       ?GetColorAdjustment@CDC@@QBEHPAUtagCOLORADJUSTMENT@@@Z 5f8805f5 f   afxinl2.obj
 0001:0007f63c       ?GetCurrentPen@CDC@@QBEPAVCPen@@XZ 5f88063c f   afxinl2.obj
 0001:0007f685       ?GetCurrentBrush@CDC@@QBEPAVCBrush@@XZ 5f880685 f   afxinl2.obj
 0001:0007f6ce       ?GetCurrentPalette@CDC@@QBEPAVCPalette@@XZ 5f8806ce f   afxinl2.obj
 0001:0007f717       ?GetCurrentFont@CDC@@QBEPAVCFont@@XZ 5f880717 f   afxinl2.obj
 0001:0007f760       ?GetCurrentBitmap@CDC@@QBEPAVCBitmap@@XZ 5f880760 f   afxinl2.obj
 0001:0007f7a9       ?PolyBezier@CDC@@QAEHPBUtagPOINT@@H@Z 5f8807a9 f   afxinl2.obj
 0001:0007f7f4       ?DrawEscape@CDC@@QAEHHHPBD@Z 5f8807f4 f   afxinl2.obj
 0001:0007f843       ?Escape@CDC@@QAEHHHPBDHPAD@Z 5f880843 f   afxinl2.obj
 0001:0007f89a       ?GetCharABCWidthsW@CDC@@QBEHIIPAU_ABCFLOAT@@@Z 5f88089a f   afxinl2.obj
 0001:0007f8e9       ?GetCharWidthW@CDC@@QBEHIIPAM@Z 5f8808e9 f   afxinl2.obj
 0001:0007f938       ?AbortPath@CDC@@QAEHXZ     5f880938 f   afxinl2.obj
 0001:0007f979       ?BeginPath@CDC@@QAEHXZ     5f880979 f   afxinl2.obj
 0001:0007f9ba       ?CloseFigure@CDC@@QAEHXZ   5f8809ba f   afxinl2.obj
 0001:0007f9fb       ?EndPath@CDC@@QAEHXZ       5f8809fb f   afxinl2.obj
 0001:0007fa3c       ?FillPath@CDC@@QAEHXZ      5f880a3c f   afxinl2.obj
 0001:0007fa7d       ?FlattenPath@CDC@@QAEHXZ   5f880a7d f   afxinl2.obj
 0001:0007fabe       ?GetMiterLimit@CDC@@QBEMXZ 5f880abe f   afxinl2.obj
 0001:0007fb26       ?GetPath@CDC@@QBEHPAUtagPOINT@@PAEH@Z 5f880b26 f   afxinl2.obj
 0001:0007fb75       ?SetMiterLimit@CDC@@QAEHM@Z 5f880b75 f   afxinl2.obj
 0001:0007fbbe       ?StrokeAndFillPath@CDC@@QAEHXZ 5f880bbe f   afxinl2.obj
 0001:0007fbff       ?StrokePath@CDC@@QAEHXZ    5f880bff f   afxinl2.obj
 0001:0007fc40       ?WidenPath@CDC@@QAEHXZ     5f880c40 f   afxinl2.obj
 0001:0007fc81       ?AddMetaFileComment@CDC@@QAEHIPBE@Z 5f880c81 f   afxinl2.obj
 0001:0007fccc       ?PlayMetaFile@CDC@@QAEHPAUHENHMETAFILE__@@PBUtagRECT@@@Z 5f880ccc f   afxinl2.obj
 0001:0007fd17       ??0CMenu@@QAE@XZ           5f880d17 f   afxinl2.obj
 0001:0007fd40       ??1CMenu@@UAE@XZ           5f880d40 f   afxinl2.obj
 0001:0007fd91       ?CreateMenu@CMenu@@QAEHXZ  5f880d91 f   afxinl2.obj
 0001:0007fdab       ?CreatePopupMenu@CMenu@@QAEHXZ 5f880dab f   afxinl2.obj
 0001:0007fdc5       ??BCMenu@@QBEPAUHMENU__@@XZ 5f880dc5 f   afxinl2.obj
 0001:0007fe2d       ??8CMenu@@QBEHABV0@@Z      5f880e2d f   afxinl2.obj
 0001:0007fe4f       ??9CMenu@@QBEHABV0@@Z      5f880e4f f   afxinl2.obj
 0001:0007fe71       ?GetSafeHmenu@CMenu@@QBEPAUHMENU__@@XZ 5f880e71 f   afxinl2.obj
 0001:0007fed9       ?DeleteMenu@CMenu@@QAEHII@Z 5f880ed9 f   afxinl2.obj
 0001:0007ff2c       ?AppendMenuW@CMenu@@QAEHIIPBG@Z 5f880f2c f   afxinl2.obj
 0001:0007ff83       ?AppendMenuW@CMenu@@QAEHIIPBVCBitmap@@@Z 5f880f83 f   afxinl2.obj
 0001:0007ffe2       ?CheckMenuItem@CMenu@@QAEIII@Z 5f880fe2 f   afxinl2.obj
 0001:00080035       ?EnableMenuItem@CMenu@@QAEIII@Z 5f881035 f   afxinl2.obj
 0001:00080088       ?SetDefaultItem@CMenu@@QAEHIH@Z 5f881088 f   afxinl2.obj
 0001:000800db       ?GetDefaultItem@CMenu@@QAEIIH@Z 5f8810db f   afxinl2.obj
 0001:0008012e       ?GetMenuItemCount@CMenu@@QBEIXZ 5f88112e f   afxinl2.obj
 0001:00080177       ?GetMenuItemID@CMenu@@QBEIH@Z 5f881177 f   afxinl2.obj
 0001:000801c6       ?GetMenuState@CMenu@@QBEIII@Z 5f8811c6 f   afxinl2.obj
 0001:00080219       ?GetMenuStringW@CMenu@@QBEHIPAGHI@Z 5f881219 f   afxinl2.obj
 0001:00080274       ?GetMenuStringW@CMenu@@QBEHIAAVCString@@I@Z 5f881274 f   afxinl2.obj
 0001:000802ec       ?GetMenuItemInfoW@CMenu@@QAEHIPAUtagMENUITEMINFOW@@H@Z 5f8812ec f   afxinl2.obj
 0001:00080374       ?GetSubMenu@CMenu@@QBEPAV1@H@Z 5f881374 f   afxinl2.obj
 0001:000803c9       ?InsertMenuW@CMenu@@QAEHIIIPBG@Z 5f8813c9 f   afxinl2.obj
 0001:00080424       ?InsertMenuW@CMenu@@QAEHIIIPBVCBitmap@@@Z 5f881424 f   afxinl2.obj
 0001:00080487       ?ModifyMenuW@CMenu@@QAEHIIIPBG@Z 5f881487 f   afxinl2.obj
 0001:000804e2       ?ModifyMenuW@CMenu@@QAEHIIIPBVCBitmap@@@Z 5f8814e2 f   afxinl2.obj
 0001:00080545       ?RemoveMenu@CMenu@@QAEHII@Z 5f881545 f   afxinl2.obj
 0001:00080598       ?SetMenuItemBitmaps@CMenu@@QAEHIIPBVCBitmap@@0@Z 5f881598 f   afxinl2.obj
 0001:000805fd       ?LoadMenuW@CMenu@@QAEHPBG@Z 5f8815fd f   afxinl2.obj
 0001:00080629       ?LoadMenuW@CMenu@@QAEHI@Z  5f881629 f   afxinl2.obj
 0001:00080660       ?LoadMenuIndirectW@CMenu@@QAEHPBX@Z 5f881660 f   afxinl2.obj
 0001:00080680       ?SetMenuContextHelpId@CMenu@@QAEHK@Z 5f881680 f   afxinl2.obj
 0001:0008069e       ?GetMenuContextHelpId@CMenu@@QBEKXZ 5f88169e f   afxinl2.obj
 0001:000806b6       ?CheckMenuRadioItem@CMenu@@QAEHIIII@Z 5f8816b6 f   afxinl2.obj
 0001:000806e0       ?ContinueRouting@CCmdUI@@QAEXXZ 5f8816e0 f   afxinl2.obj
 0001:00080700       ??_GCResourceException@@UAEPAXI@Z 5f881700 f i afxinl2.obj
 0001:00080700       ??_ECResourceException@@UAEPAXI@Z 5f881700 f i afxinl2.obj
 0001:00080730       ??_ECUserException@@UAEPAXI@Z 5f881730 f i afxinl2.obj
 0001:00080730       ??_GCUserException@@UAEPAXI@Z 5f881730 f i afxinl2.obj
 0001:00080760       ??BCWnd@@QBEPAUHWND__@@XZ  5f881760 f   afxinl3.obj
 0001:00080788       ??8CWnd@@QBEHABV0@@Z       5f881788 f   afxinl3.obj
 0001:000807aa       ??9CWnd@@QBEHABV0@@Z       5f8817aa f   afxinl3.obj
 0001:000807cc       ?GetSafeHwnd@CWnd@@QBEPAUHWND__@@XZ 5f8817cc f   afxinl3.obj
 0001:000807f4       ?GetOwner@CWnd@@QBEPAV1@XZ 5f8817f4 f   afxinl3.obj
 0001:00080829       ?SetOwner@CWnd@@QAEXPAV1@@Z 5f881829 f   afxinl3.obj
 0001:00080859       ?SendMessageW@CWnd@@QAEJIIJ@Z 5f881859 f   afxinl3.obj
 0001:000808ad       ?PostMessageW@CWnd@@QAEHIIJ@Z 5f8818ad f   afxinl3.obj
 0001:00080901       ?SetFont@CWnd@@QAEXPAVCFont@@H@Z 5f881901 f   afxinl3.obj
 0001:00080958       ?GetFont@CWnd@@QBEPAVCFont@@XZ 5f881958 f   afxinl3.obj
 0001:000809aa       ?GetMenu@CWnd@@QBEPAVCMenu@@XZ 5f8819aa f   afxinl3.obj
 0001:000809f6       ?SetMenu@CWnd@@QAEHPAVCMenu@@@Z 5f8819f6 f   afxinl3.obj
 0001:00080a47       ?DrawMenuBar@CWnd@@QAEXXZ  5f881a47 f   afxinl3.obj
 0001:00080a8d       ?GetSystemMenu@CWnd@@QBEPAVCMenu@@H@Z 5f881a8d f   afxinl3.obj
 0001:00080adf       ?HiliteMenuItem@CWnd@@QAEHPAVCMenu@@II@Z 5f881adf f   afxinl3.obj
 0001:00080b36       ?IsIconic@CWnd@@QBEHXZ     5f881b36 f   afxinl3.obj
 0001:00080b7c       ?IsZoomed@CWnd@@QBEHXZ     5f881b7c f   afxinl3.obj
 0001:00080bc2       ?MoveWindow@CWnd@@QAEXPBUtagRECT@@H@Z 5f881bc2 f   afxinl3.obj
 0001:00080c01       ?ArrangeIconicWindows@CWnd@@QAEIXZ 5f881c01 f   afxinl3.obj
 0001:00080c47       ?SetWindowRgn@CWnd@@QAEHPAUHRGN__@@H@Z 5f881c47 f   afxinl3.obj
 0001:00080c97       ?GetWindowRgn@CWnd@@QBEHPAUHRGN__@@@Z 5f881c97 f   afxinl3.obj
 0001:00080ce9       ?BringWindowToTop@CWnd@@QAEXXZ 5f881ce9 f   afxinl3.obj
 0001:00080d2f       ?GetWindowRect@CWnd@@QBEXPAUtagRECT@@@Z 5f881d2f f   afxinl3.obj
 0001:00080d7b       ?GetClientRect@CWnd@@QBEXPAUtagRECT@@@Z 5f881d7b f   afxinl3.obj
 0001:00080dc7       ?MapWindowPoints@CWnd@@QBEXPAV1@PAUtagPOINT@@I@Z 5f881dc7 f   afxinl3.obj
 0001:00080e20       ?MapWindowPoints@CWnd@@QBEXPAV1@PAUtagRECT@@@Z 5f881e20 f   afxinl3.obj
 0001:00080e77       ?ClientToScreen@CWnd@@QBEXPAUtagPOINT@@@Z 5f881e77 f   afxinl3.obj
 0001:00080ec3       ?ScreenToClient@CWnd@@QBEXPAUtagPOINT@@@Z 5f881ec3 f   afxinl3.obj
 0001:00080f0f       ?BeginPaint@CWnd@@QAEPAVCDC@@PAUtagPAINTSTRUCT@@@Z 5f881f0f f   afxinl3.obj
 0001:00080f61       ?EndPaint@CWnd@@QAEXPAUtagPAINTSTRUCT@@@Z 5f881f61 f   afxinl3.obj
 0001:00080fad       ?GetDC@CWnd@@QAEPAVCDC@@XZ 5f881fad f   afxinl3.obj
 0001:00080ff9       ?GetWindowDC@CWnd@@QAEPAVCDC@@XZ 5f881ff9 f   afxinl3.obj
 0001:00081045       ?ReleaseDC@CWnd@@QAEHPAVCDC@@@Z 5f882045 f   afxinl3.obj
 0001:00081094       ?UpdateWindow@CWnd@@QAEXXZ 5f882094 f   afxinl3.obj
 0001:000810da       ?SetRedraw@CWnd@@QAEXH@Z   5f8820da f   afxinl3.obj
 0001:0008112a       ?GetUpdateRect@CWnd@@QAEHPAUtagRECT@@H@Z 5f88212a f   afxinl3.obj
 0001:0008117a       ?GetUpdateRgn@CWnd@@QAEHPAVCRgn@@H@Z 5f88217a f   afxinl3.obj
 0001:000811cf       ?Invalidate@CWnd@@QAEXH@Z  5f8821cf f   afxinl3.obj
 0001:0008121d       ?InvalidateRect@CWnd@@QAEXPBUtagRECT@@H@Z 5f88221d f   afxinl3.obj
 0001:00081270       ?InvalidateRgn@CWnd@@QAEXPAVCRgn@@H@Z 5f882270 f   afxinl3.obj
 0001:000812c8       ?ValidateRect@CWnd@@QAEXPBUtagRECT@@@Z 5f8822c8 f   afxinl3.obj
 0001:00081317       ?ValidateRgn@CWnd@@QAEXPAVCRgn@@@Z 5f882317 f   afxinl3.obj
 0001:0008136b       ?IsWindowVisible@CWnd@@QBEHXZ 5f88236b f   afxinl3.obj
 0001:000813b4       ?ShowOwnedPopups@CWnd@@QAEXH@Z 5f8823b4 f   afxinl3.obj
 0001:00081403       ?SendMessageToDescendants@CWnd@@QAEXIIJHH@Z 5f882403 f   afxinl3.obj
 0001:00081461       ?GetDescendantWindow@CWnd@@QBEPAV1@HH@Z 5f882461 f   afxinl3.obj
 0001:000814b3       ?GetDCEx@CWnd@@QAEPAVCDC@@PAVCRgn@@K@Z 5f8824b3 f   afxinl3.obj
 0001:00081511       ?LockWindowUpdate@CWnd@@QAEHXZ 5f882511 f   afxinl3.obj
 0001:0008155a       ?UnlockWindowUpdate@CWnd@@QAEXXZ 5f88255a f   afxinl3.obj
 0001:0008159e       ?RedrawWindow@CWnd@@QAEHPBUtagRECT@@PAVCRgn@@I@Z 5f88259e f   afxinl3.obj
 0001:000815fa       ?EnableScrollBar@CWnd@@QAEHHI@Z 5f8825fa f   afxinl3.obj
 0001:0008164d       ?SetTimer@CWnd@@QAEIIIP6GXPAUHWND__@@IIK@Z@Z 5f88264d f   afxinl3.obj
 0001:000816a4       ?KillTimer@CWnd@@QAEHH@Z   5f8826a4 f   afxinl3.obj
 0001:000816f3       ?GetActiveWindow@CWnd@@SGPAV1@XZ 5f8826f3 f   afxinl3.obj
 0001:00081704       ?SetActiveWindow@CWnd@@QAEPAV1@XZ 5f882704 f   afxinl3.obj
 0001:00081753       ?GetCapture@CWnd@@SGPAV1@XZ 5f882753 f   afxinl3.obj
 0001:00081764       ?SetCapture@CWnd@@QAEPAV1@XZ 5f882764 f   afxinl3.obj
 0001:000817b3       ?GetFocus@CWnd@@SGPAV1@XZ  5f8827b3 f   afxinl3.obj
 0001:000817c4       ?GetDesktopWindow@CWnd@@SGPAV1@XZ 5f8827c4 f   afxinl3.obj
 0001:000817d5       ?DlgDirListW@CWnd@@QAEHPAGHHI@Z 5f8827d5 f   afxinl3.obj
 0001:00081830       ?DlgDirListComboBoxW@CWnd@@QAEHPAGHHI@Z 5f882830 f   afxinl3.obj
 0001:0008188b       ?DlgDirSelect@CWnd@@QAEHPAGH@Z 5f88288b f   afxinl3.obj
 0001:000818e3       ?DlgDirSelectComboBox@CWnd@@QAEHPAGH@Z 5f8828e3 f   afxinl3.obj
 0001:0008193b       ?GetNextDlgGroupItem@CWnd@@QBEPAV1@PAV1@H@Z 5f88293b f   afxinl3.obj
 0001:00081999       ?GetNextDlgTabItem@CWnd@@QBEPAV1@PAV1@H@Z 5f882999 f   afxinl3.obj
 0001:000819f7       ?ShowScrollBar@CWnd@@QAEXIH@Z 5f8829f7 f   afxinl3.obj
 0001:00081a4a       ?ChildWindowFromPoint@CWnd@@QBEPAV1@UtagPOINT@@@Z 5f882a4a f   afxinl3.obj
 0001:00081aa3       ?ChildWindowFromPoint@CWnd@@QBEPAV1@UtagPOINT@@I@Z 5f882aa3 f   afxinl3.obj
 0001:00081b00       ?FindWindowW@CWnd@@SGPAV1@PBG0@Z 5f882b00 f   afxinl3.obj
 0001:00081b1b       ?GetNextWindow@CWnd@@QBEPAV1@I@Z 5f882b1b f   afxinl3.obj
 0001:00081b72       ?GetTopWindow@CWnd@@QBEPAV1@XZ 5f882b72 f   afxinl3.obj
 0001:00081bc1       ?GetWindow@CWnd@@QBEPAV1@I@Z 5f882bc1 f   afxinl3.obj
 0001:00081c16       ?GetLastActivePopup@CWnd@@QBEPAV1@XZ 5f882c16 f   afxinl3.obj
 0001:00081c65       ?IsChild@CWnd@@QBEHPBV1@@Z 5f882c65 f   afxinl3.obj
 0001:00081cb9       ?GetParent@CWnd@@QBEPAV1@XZ 5f882cb9 f   afxinl3.obj
 0001:00081d08       ?SetParent@CWnd@@QAEPAV1@PAV1@@Z 5f882d08 f   afxinl3.obj
 0001:00081d62       ?WindowFromPoint@CWnd@@SGPAV1@UtagPOINT@@@Z 5f882d62 f   afxinl3.obj
 0001:00081d7d       ?FlashWindow@CWnd@@QAEHH@Z 5f882d7d f   afxinl3.obj
 0001:00081dcc       ?ChangeClipboardChain@CWnd@@QAEHPAUHWND__@@@Z 5f882dcc f   afxinl3.obj
 0001:00081e1b       ?SetClipboardViewer@CWnd@@QAEPAUHWND__@@XZ 5f882e1b f   afxinl3.obj
 0001:00081e64       ?OpenClipboard@CWnd@@QAEHXZ 5f882e64 f   afxinl3.obj
 0001:00081ead       ?GetOpenClipboardWindow@CWnd@@SGPAV1@XZ 5f882ead f   afxinl3.obj
 0001:00081ebe       ?GetClipboardOwner@CWnd@@SGPAV1@XZ 5f882ebe f   afxinl3.obj
 0001:00081ecf       ?GetClipboardViewer@CWnd@@SGPAV1@XZ 5f882ecf f   afxinl3.obj
 0001:00081ee0       ?CreateCaret@CWnd@@QAEXPAVCBitmap@@@Z 5f882ee0 f   afxinl3.obj
 0001:00081f38       ?CreateSolidCaret@CWnd@@QAEXHH@Z 5f882f38 f   afxinl3.obj
 0001:00081f8d       ?CreateGrayCaret@CWnd@@QAEXHH@Z 5f882f8d f   afxinl3.obj
 0001:00081fe2       ?GetCaretPos@CWnd@@SG?AVCPoint@@XZ 5f882fe2 f   afxinl3.obj
 0001:00082011       ?SetCaretPos@CWnd@@SGXUtagPOINT@@@Z 5f883011 f   afxinl3.obj
 0001:00082026       ?HideCaret@CWnd@@QAEXXZ    5f883026 f   afxinl3.obj
 0001:0008206f       ?ShowCaret@CWnd@@QAEXXZ    5f88306f f   afxinl3.obj
 0001:000820b8       ?SetForegroundWindow@CWnd@@QAEHXZ 5f8830b8 f   afxinl3.obj
 0001:00082101       ?GetForegroundWindow@CWnd@@SGPAV1@XZ 5f883101 f   afxinl3.obj
 0001:00082112       ?SendNotifyMessageW@CWnd@@QAEHIIJ@Z 5f883112 f   afxinl3.obj
 0001:00082169       ?SetIcon@CWnd@@QAEPAUHICON__@@PAU2@H@Z 5f883169 f   afxinl3.obj
 0001:000821c1       ?GetIcon@CWnd@@QBEPAUHICON__@@H@Z 5f8831c1 f   afxinl3.obj
 0001:00082214       ?Print@CWnd@@QBEXPAVCDC@@K@Z 5f883214 f   afxinl3.obj
 0001:00082271       ?PrintClient@CWnd@@QBEXPAVCDC@@K@Z 5f883271 f   afxinl3.obj
 0001:000822ce       ?SetWindowContextHelpId@CWnd@@QAEHK@Z 5f8832ce f   afxinl3.obj
 0001:0008231d       ?GetWindowContextHelpId@CWnd@@QBEKXZ 5f88331d f   afxinl3.obj
 0001:00082366       ?OnActivateApp@CWnd@@IAEXHPAUHTASK__@@@Z 5f883366 f   afxinl3.obj
 0001:0008237b       ?OnActivate@CWnd@@IAEXIPAV1@H@Z 5f88337b f   afxinl3.obj
 0001:00082390       ?OnCancelMode@CWnd@@IAEXXZ 5f883390 f   afxinl3.obj
 0001:000823a3       ?OnChildActivate@CWnd@@IAEXXZ 5f8833a3 f   afxinl3.obj
 0001:000823b6       ?OnClose@CWnd@@IAEXXZ      5f8833b6 f   afxinl3.obj
 0001:000823c9       ?OnContextMenu@CWnd@@IAEXPAV1@VCPoint@@@Z 5f8833c9 f   afxinl3.obj
 0001:000823de       ?OnCopyData@CWnd@@IAEHPAV1@PAUtagCOPYDATASTRUCT@@@Z 5f8833de f   afxinl3.obj
 0001:000823f3       ?OnCreate@CWnd@@IAEHPAUtagCREATESTRUCTW@@@Z 5f8833f3 f   afxinl3.obj
 0001:00082408       ?OnEnable@CWnd@@IAEXH@Z    5f883408 f   afxinl3.obj
 0001:0008241d       ?OnEndSession@CWnd@@IAEXH@Z 5f88341d f   afxinl3.obj
 0001:00082432       ?OnEraseBkgnd@CWnd@@IAEHPAVCDC@@@Z 5f883432 f   afxinl3.obj
 0001:00082447       ?OnGetMinMaxInfo@CWnd@@IAEXPAUtagMINMAXINFO@@@Z 5f883447 f   afxinl3.obj
 0001:0008245c       ?OnIconEraseBkgnd@CWnd@@IAEXPAVCDC@@@Z 5f88345c f   afxinl3.obj
 0001:00082471       ?OnKillFocus@CWnd@@IAEXPAV1@@Z 5f883471 f   afxinl3.obj
 0001:00082486       ?OnMenuChar@CWnd@@IAEJIIPAVCMenu@@@Z 5f883486 f   afxinl3.obj
 0001:0008249b       ?OnMenuSelect@CWnd@@IAEXIIPAUHMENU__@@@Z 5f88349b f   afxinl3.obj
 0001:000824b0       ?OnMove@CWnd@@IAEXHH@Z     5f8834b0 f   afxinl3.obj
 0001:000824c5       ?OnPaint@CWnd@@IAEXXZ      5f8834c5 f   afxinl3.obj
 0001:000824d8       ?OnQueryDragIcon@CWnd@@IAEPAUHICON__@@XZ 5f8834d8 f   afxinl3.obj
 0001:000824eb       ?OnQueryEndSession@CWnd@@IAEHXZ 5f8834eb f   afxinl3.obj
 0001:000824fe       ?OnQueryNewPalette@CWnd@@IAEHXZ 5f8834fe f   afxinl3.obj
 0001:00082511       ?OnQueryOpen@CWnd@@IAEHXZ  5f883511 f   afxinl3.obj
 0001:00082524       ?OnSetCursor@CWnd@@IAEHPAV1@II@Z 5f883524 f   afxinl3.obj
 0001:00082539       ?OnSetFocus@CWnd@@IAEXPAV1@@Z 5f883539 f   afxinl3.obj
 0001:0008254e       ?OnShowWindow@CWnd@@IAEXHI@Z 5f88354e f   afxinl3.obj
 0001:00082563       ?OnSize@CWnd@@IAEXIHH@Z    5f883563 f   afxinl3.obj
 0001:00082578       ?OnTCard@CWnd@@IAEXIK@Z    5f883578 f   afxinl3.obj
 0001:0008258d       ?OnWindowPosChanging@CWnd@@IAEXPAUtagWINDOWPOS@@@Z 5f88358d f   afxinl3.obj
 0001:000825a2       ?OnWindowPosChanged@CWnd@@IAEXPAUtagWINDOWPOS@@@Z 5f8835a2 f   afxinl3.obj
 0001:000825b7       ?OnDropFiles@CWnd@@IAEXPAUHDROP__@@@Z 5f8835b7 f   afxinl3.obj
 0001:000825cc       ?OnPaletteIsChanging@CWnd@@IAEXPAV1@@Z 5f8835cc f   afxinl3.obj
 0001:000825e1       ?OnNcActivate@CWnd@@IAEHH@Z 5f8835e1 f   afxinl3.obj
 0001:000825f6       ?OnNcCalcSize@CWnd@@IAEXHPAUtagNCCALCSIZE_PARAMS@@@Z 5f8835f6 f   afxinl3.obj
 0001:0008260b       ?OnNcCreate@CWnd@@IAEHPAUtagCREATESTRUCTW@@@Z 5f88360b f   afxinl3.obj
 0001:00082620       ?OnNcHitTest@CWnd@@IAEIVCPoint@@@Z 5f883620 f   afxinl3.obj
 0001:00082635       ?OnNcLButtonDblClk@CWnd@@IAEXIVCPoint@@@Z 5f883635 f   afxinl3.obj
 0001:0008264a       ?OnNcLButtonDown@CWnd@@IAEXIVCPoint@@@Z 5f88364a f   afxinl3.obj
 0001:0008265f       ?OnNcLButtonUp@CWnd@@IAEXIVCPoint@@@Z 5f88365f f   afxinl3.obj
 0001:00082674       ?OnNcMButtonDblClk@CWnd@@IAEXIVCPoint@@@Z 5f883674 f   afxinl3.obj
 0001:00082689       ?OnNcMButtonDown@CWnd@@IAEXIVCPoint@@@Z 5f883689 f   afxinl3.obj
 0001:0008269e       ?OnNcMButtonUp@CWnd@@IAEXIVCPoint@@@Z 5f88369e f   afxinl3.obj
 0001:000826b3       ?OnNcMouseMove@CWnd@@IAEXIVCPoint@@@Z 5f8836b3 f   afxinl3.obj
 0001:000826c8       ?OnNcPaint@CWnd@@IAEXXZ    5f8836c8 f   afxinl3.obj
 0001:000826db       ?OnNcRButtonDblClk@CWnd@@IAEXIVCPoint@@@Z 5f8836db f   afxinl3.obj
 0001:000826f0       ?OnNcRButtonDown@CWnd@@IAEXIVCPoint@@@Z 5f8836f0 f   afxinl3.obj
 0001:00082705       ?OnNcRButtonUp@CWnd@@IAEXIVCPoint@@@Z 5f883705 f   afxinl3.obj
 0001:0008271a       ?OnSysChar@CWnd@@IAEXIII@Z 5f88371a f   afxinl3.obj
 0001:0008272f       ?OnSysCommand@CWnd@@IAEXIJ@Z 5f88372f f   afxinl3.obj
 0001:00082744       ?OnSysDeadChar@CWnd@@IAEXIII@Z 5f883744 f   afxinl3.obj
 0001:00082759       ?OnSysKeyDown@CWnd@@IAEXIII@Z 5f883759 f   afxinl3.obj
 0001:0008276e       ?OnSysKeyUp@CWnd@@IAEXIII@Z 5f88376e f   afxinl3.obj
 0001:00082783       ?OnCompacting@CWnd@@IAEXI@Z 5f883783 f   afxinl3.obj
 0001:00082798       ?OnFontChange@CWnd@@IAEXXZ 5f883798 f   afxinl3.obj
 0001:000827ab       ?OnPaletteChanged@CWnd@@IAEXPAV1@@Z 5f8837ab f   afxinl3.obj
 0001:000827c0       ?OnSpoolerStatus@CWnd@@IAEXII@Z 5f8837c0 f   afxinl3.obj
 0001:000827d5       ?OnTimeChange@CWnd@@IAEXXZ 5f8837d5 f   afxinl3.obj
 0001:000827e8       ?OnChar@CWnd@@IAEXIII@Z    5f8837e8 f   afxinl3.obj
 0001:000827fd       ?OnDeadChar@CWnd@@IAEXIII@Z 5f8837fd f   afxinl3.obj
 0001:00082812       ?OnKeyDown@CWnd@@IAEXIII@Z 5f883812 f   afxinl3.obj
 0001:00082827       ?OnKeyUp@CWnd@@IAEXIII@Z   5f883827 f   afxinl3.obj
 0001:0008283c       ?OnLButtonDblClk@CWnd@@IAEXIVCPoint@@@Z 5f88383c f   afxinl3.obj
 0001:00082851       ?OnLButtonDown@CWnd@@IAEXIVCPoint@@@Z 5f883851 f   afxinl3.obj
 0001:00082866       ?OnLButtonUp@CWnd@@IAEXIVCPoint@@@Z 5f883866 f   afxinl3.obj
 0001:0008287b       ?OnMButtonDblClk@CWnd@@IAEXIVCPoint@@@Z 5f88387b f   afxinl3.obj
 0001:00082890       ?OnMButtonDown@CWnd@@IAEXIVCPoint@@@Z 5f883890 f   afxinl3.obj
 0001:000828a5       ?OnMButtonUp@CWnd@@IAEXIVCPoint@@@Z 5f8838a5 f   afxinl3.obj
 0001:000828ba       ?OnMouseActivate@CWnd@@IAEHPAV1@II@Z 5f8838ba f   afxinl3.obj
 0001:000828cf       ?OnMouseMove@CWnd@@IAEXIVCPoint@@@Z 5f8838cf f   afxinl3.obj
 0001:000828e4       ?OnMouseWheel@CWnd@@IAEHIFVCPoint@@@Z 5f8838e4 f   afxinl3.obj
 0001:000828f9       ?OnRegisteredMouseWheel@CWnd@@IAEJIJ@Z 5f8838f9 f   afxinl3.obj
 0001:0008290e       ?OnRButtonDblClk@CWnd@@IAEXIVCPoint@@@Z 5f88390e f   afxinl3.obj
 0001:00082923       ?OnRButtonDown@CWnd@@IAEXIVCPoint@@@Z 5f883923 f   afxinl3.obj
 0001:00082938       ?OnRButtonUp@CWnd@@IAEXIVCPoint@@@Z 5f883938 f   afxinl3.obj
 0001:0008294d       ?OnTimer@CWnd@@IAEXI@Z     5f88394d f   afxinl3.obj
 0001:00082962       ?OnInitMenu@CWnd@@IAEXPAVCMenu@@@Z 5f883962 f   afxinl3.obj
 0001:00082977       ?OnInitMenuPopup@CWnd@@IAEXPAVCMenu@@IH@Z 5f883977 f   afxinl3.obj
 0001:0008298c       ?OnAskCbFormatName@CWnd@@IAEXIPAG@Z 5f88398c f   afxinl3.obj
 0001:000829a1       ?OnChangeCbChain@CWnd@@IAEXPAUHWND__@@0@Z 5f8839a1 f   afxinl3.obj
 0001:000829b6       ?OnDestroyClipboard@CWnd@@IAEXXZ 5f8839b6 f   afxinl3.obj
 0001:000829c9       ?OnDrawClipboard@CWnd@@IAEXXZ 5f8839c9 f   afxinl3.obj
 0001:000829dc       ?OnHScrollClipboard@CWnd@@IAEXPAV1@II@Z 5f8839dc f   afxinl3.obj
 0001:000829f1       ?OnPaintClipboard@CWnd@@IAEXPAV1@PAX@Z 5f8839f1 f   afxinl3.obj
 0001:00082a06       ?OnRenderAllFormats@CWnd@@IAEXXZ 5f883a06 f   afxinl3.obj
 0001:00082a19       ?OnRenderFormat@CWnd@@IAEXI@Z 5f883a19 f   afxinl3.obj
 0001:00082a2e       ?OnSizeClipboard@CWnd@@IAEXPAV1@PAX@Z 5f883a2e f   afxinl3.obj
 0001:00082a43       ?OnVScrollClipboard@CWnd@@IAEXPAV1@II@Z 5f883a43 f   afxinl3.obj
 0001:00082a58       ?OnGetDlgCode@CWnd@@IAEIXZ 5f883a58 f   afxinl3.obj
 0001:00082a6b       ?OnMDIActivate@CWnd@@IAEXHPAV1@0@Z 5f883a6b f   afxinl3.obj
 0001:00082a80       ?OnEnterMenuLoop@CWnd@@IAEXH@Z 5f883a80 f   afxinl3.obj
 0001:00082a95       ?OnExitMenuLoop@CWnd@@IAEXH@Z 5f883a95 f   afxinl3.obj
 0001:00082aaa       ?OnStyleChanged@CWnd@@IAEXHPAUtagSTYLESTRUCT@@@Z 5f883aaa f   afxinl3.obj
 0001:00082abf       ?OnStyleChanging@CWnd@@IAEXHPAUtagSTYLESTRUCT@@@Z 5f883abf f   afxinl3.obj
 0001:00082ad4       ?OnSizing@CWnd@@IAEXIPAUtagRECT@@@Z 5f883ad4 f   afxinl3.obj
 0001:00082ae9       ?OnMoving@CWnd@@IAEXIPAUtagRECT@@@Z 5f883ae9 f   afxinl3.obj
 0001:00082afe       ?OnCaptureChanged@CWnd@@IAEXPAV1@@Z 5f883afe f   afxinl3.obj
 0001:00082b13       ?OnDeviceChange@CWnd@@IAEHIK@Z 5f883b13 f   afxinl3.obj
 0001:00082b28       ?DoDataExchange@CWnd@@MAEXPAVCDataExchange@@@Z 5f883b28 f   afxinl3.obj
 0001:00082b35       ?BeginModalState@CWnd@@UAEXXZ 5f883b35 f   afxinl3.obj
 0001:00082b4f       ?EndModalState@CWnd@@UAEXXZ 5f883b4f f   afxinl3.obj
 0001:00082b69       ?DelayUpdateFrameTitle@CFrameWnd@@QAEXXZ 5f883b69 f   afxinl3.obj
 0001:00082b89       ?DelayRecalcLayout@CFrameWnd@@QAEXH@Z 5f883b89 f   afxinl3.obj
 0001:00082bb6       ?InModalState@CFrameWnd@@QBEHXZ 5f883bb6 f   afxinl3.obj
 0001:00082bd2       ?AddControlBar@CFrameWnd@@QAEXPAVCControlBar@@@Z 5f883bd2 f   afxinl3.obj
 0001:00082bee       ?SetTitle@CFrameWnd@@QAEXPBG@Z 5f883bee f   afxinl3.obj
 0001:00082c0d       ?GetTitle@CFrameWnd@@QBE?AVCString@@XZ 5f883c0d f   afxinl3.obj
 0001:00082c40       ?Create@CDialog@@QAEHIPAVCWnd@@@Z 5f883c40 f   afxinl3.obj
 0001:00082c63       ?MapDialogRect@CDialog@@QBEXPAUtagRECT@@@Z 5f883c63 f   afxinl3.obj
 0001:00082cb2       ?SetHelpID@CDialog@@QAEXI@Z 5f883cb2 f   afxinl3.obj
 0001:00082cc8       ?NextDlgCtrl@CDialog@@QBEXXZ 5f883cc8 f   afxinl3.obj
 0001:00082d17       ?PrevDlgCtrl@CDialog@@QBEXXZ 5f883d17 f   afxinl3.obj
 0001:00082d66       ?GotoDlgCtrl@CDialog@@QAEXPAVCWnd@@@Z 5f883d66 f   afxinl3.obj
 0001:00082dbc       ?SetDefID@CDialog@@QAEXI@Z 5f883dbc f   afxinl3.obj
 0001:00082e12       ?GetDefID@CDialog@@QBEKXZ  5f883e12 f   afxinl3.obj
 0001:00082e64       ??0CStatic@@QAE@XZ         5f883e64 f   afxinl3.obj
 0001:00082e83       ?SetIcon@CStatic@@QAEPAUHICON__@@PAU2@@Z 5f883e83 f   afxinl3.obj
 0001:00082ed9       ?GetIcon@CStatic@@QBEPAUHICON__@@XZ 5f883ed9 f   afxinl3.obj
 0001:00082f2b       ?SetEnhMetaFile@CStatic@@QAEPAUHENHMETAFILE__@@PAU2@@Z 5f883f2b f   afxinl3.obj
 0001:00082f81       ?GetEnhMetaFileW@CStatic@@QBEPAUHENHMETAFILE__@@XZ 5f883f81 f   afxinl3.obj
 0001:00082fd3       ?SetBitmap@CStatic@@QAEPAUHBITMAP__@@PAU2@@Z 5f883fd3 f   afxinl3.obj
 0001:00083029       ?GetBitmap@CStatic@@QBEPAUHBITMAP__@@XZ 5f884029 f   afxinl3.obj
 0001:0008307b       ?SetCursor@CStatic@@QAEPAUHICON__@@PAU2@@Z 5f88407b f   afxinl3.obj
 0001:000830d1       ?GetCursor@CStatic@@QAEPAUHICON__@@XZ 5f8840d1 f   afxinl3.obj
 0001:00083123       ??0CButton@@QAE@XZ         5f884123 f   afxinl3.obj
 0001:00083142       ?GetState@CButton@@QBEIXZ  5f884142 f   afxinl3.obj
 0001:00083194       ?SetState@CButton@@QAEXH@Z 5f884194 f   afxinl3.obj
 0001:000831b9       ?GetCheck@CButton@@QBEHXZ  5f8841b9 f   afxinl3.obj
 0001:0008320b       ?SetCheck@CButton@@QAEXH@Z 5f88420b f   afxinl3.obj
 0001:00083261       ?GetButtonStyle@CButton@@QBEIXZ 5f884261 f   afxinl3.obj
 0001:000832b1       ?SetButtonStyle@CButton@@QAEXIH@Z 5f8842b1 f   afxinl3.obj
 0001:00083309       ?SetIcon@CButton@@QAEPAUHICON__@@PAU2@@Z 5f884309 f   afxinl3.obj
 0001:0008335f       ?GetIcon@CButton@@QBEPAUHICON__@@XZ 5f88435f f   afxinl3.obj
 0001:000833b1       ?SetBitmap@CButton@@QAEPAUHBITMAP__@@PAU2@@Z 5f8843b1 f   afxinl3.obj
 0001:00083407       ?GetBitmap@CButton@@QBEPAUHBITMAP__@@XZ 5f884407 f   afxinl3.obj
 0001:00083459       ?SetCursor@CButton@@QAEPAUHICON__@@PAU2@@Z 5f884459 f   afxinl3.obj
 0001:000834af       ?GetCursor@CButton@@QAEPAUHICON__@@XZ 5f8844af f   afxinl3.obj
 0001:00083501       ??0CListBox@@QAE@XZ        5f884501 f   afxinl3.obj
 0001:00083520       ?GetCount@CListBox@@QBEHXZ 5f884520 f   afxinl3.obj
 0001:00083572       ?GetCurSel@CListBox@@QBEHXZ 5f884572 f   afxinl3.obj
 0001:000835c4       ?SetCurSel@CListBox@@QAEHH@Z 5f8845c4 f   afxinl3.obj
 0001:0008361a       ?GetHorizontalExtent@CListBox@@QBEHXZ 5f88461a f   afxinl3.obj
 0001:0008366c       ?SetHorizontalExtent@CListBox@@QAEXH@Z 5f88466c f   afxinl3.obj
 0001:000836c2       ?GetSelCount@CListBox@@QBEHXZ 5f8846c2 f   afxinl3.obj
 0001:00083714       ?GetSelItems@CListBox@@QBEHHPAH@Z 5f884714 f   afxinl3.obj
 0001:0008376c       ?GetTopIndex@CListBox@@QBEHXZ 5f88476c f   afxinl3.obj
 0001:000837be       ?SetTopIndex@CListBox@@QAEHH@Z 5f8847be f   afxinl3.obj
 0001:00083814       ?GetItemData@CListBox@@QBEKH@Z 5f884814 f   afxinl3.obj
 0001:0008386a       ?SetItemData@CListBox@@QAEHHK@Z 5f88486a f   afxinl3.obj
 0001:000838c2       ?GetItemDataPtr@CListBox@@QBEPAXH@Z 5f8848c2 f   afxinl3.obj
 0001:00083918       ?SetItemDataPtr@CListBox@@QAEHHPAX@Z 5f884918 f   afxinl3.obj
 0001:00083966       ?GetItemRect@CListBox@@QBEHHPAUtagRECT@@@Z 5f884966 f   afxinl3.obj
 0001:000839be       ?GetSel@CListBox@@QBEHH@Z  5f8849be f   afxinl3.obj
 0001:00083a14       ?SetSel@CListBox@@QAEHHH@Z 5f884a14 f   afxinl3.obj
 0001:00083a6c       ?GetText@CListBox@@QBEHHPAG@Z 5f884a6c f   afxinl3.obj
 0001:00083ac4       ?GetTextLen@CListBox@@QBEHH@Z 5f884ac4 f   afxinl3.obj
 0001:00083b1a       ?SetColumnWidth@CListBox@@QAEXH@Z 5f884b1a f   afxinl3.obj
 0001:00083b70       ?SetTabStops@CListBox@@QAEHHPAH@Z 5f884b70 f   afxinl3.obj
 0001:00083bc8       ?SetTabStops@CListBox@@QAEXXZ 5f884bc8 f   afxinl3.obj
 0001:00083c38       ?SetTabStops@CListBox@@QAEHABH@Z 5f884c38 f   afxinl3.obj
 0001:00083c8e       ?SetItemHeight@CListBox@@QAEHHI@Z 5f884c8e f   afxinl3.obj
 0001:00083ceb       ?GetItemHeight@CListBox@@QBEHH@Z 5f884ceb f   afxinl3.obj
 0001:00083d41       ?FindStringExact@CListBox@@QBEHHPBG@Z 5f884d41 f   afxinl3.obj
 0001:00083d99       ?GetCaretIndex@CListBox@@QBEHXZ 5f884d99 f   afxinl3.obj
 0001:00083deb       ?SetCaretIndex@CListBox@@QAEHHH@Z 5f884deb f   afxinl3.obj
 0001:00083e48       ?AddString@CListBox@@QAEHPBG@Z 5f884e48 f   afxinl3.obj
 0001:00083e9e       ?DeleteString@CListBox@@QAEHI@Z 5f884e9e f   afxinl3.obj
 0001:00083ef4       ?InsertString@CListBox@@QAEHHPBG@Z 5f884ef4 f   afxinl3.obj
 0001:00083f4c       ?ResetContent@CListBox@@QAEXXZ 5f884f4c f   afxinl3.obj
 0001:00083f9e       ?Dir@CListBox@@QAEHIPBG@Z  5f884f9e f   afxinl3.obj
 0001:00083ff6       ?FindString@CListBox@@QBEHHPBG@Z 5f884ff6 f   afxinl3.obj
 0001:0008404e       ?SelectString@CListBox@@QAEHHPBG@Z 5f88504e f   afxinl3.obj
 0001:000840a6       ?SelItemRange@CListBox@@QAEHHHH@Z 5f8850a6 f   afxinl3.obj
 0001:0008412b       ?SetAnchorIndex@CListBox@@QAEXH@Z 5f88512b f   afxinl3.obj
 0001:00084181       ?GetAnchorIndex@CListBox@@QBEHXZ 5f885181 f   afxinl3.obj
 0001:000841d3       ?GetLocale@CListBox@@QBEKXZ 5f8851d3 f   afxinl3.obj
 0001:00084225       ?SetLocale@CListBox@@QAEKK@Z 5f885225 f   afxinl3.obj
 0001:0008427b       ?InitStorage@CListBox@@QAEHHI@Z 5f88527b f   afxinl3.obj
 0001:000842d3       ??0CCheckListBox@@QAE@XZ   5f8852d3 f   afxinl3.obj
 0001:00084306       ?GetCheckStyle@CCheckListBox@@QAEIXZ 5f885306 f   afxinl3.obj
 0001:00084317       ??0CComboBox@@QAE@XZ       5f885317 f   afxinl3.obj
 0001:00084336       ?GetCount@CComboBox@@QBEHXZ 5f885336 f   afxinl3.obj
 0001:00084388       ?GetCurSel@CComboBox@@QBEHXZ 5f885388 f   afxinl3.obj
 0001:000843da       ?SetCurSel@CComboBox@@QAEHH@Z 5f8853da f   afxinl3.obj
 0001:00084430       ?GetEditSel@CComboBox@@QBEKXZ 5f885430 f   afxinl3.obj
 0001:00084482       ?LimitText@CComboBox@@QAEHH@Z 5f885482 f   afxinl3.obj
 0001:000844d8       ?SetEditSel@CComboBox@@QAEHHH@Z 5f8854d8 f   afxinl3.obj
 0001:00084541       ?GetItemData@CComboBox@@QBEKH@Z 5f885541 f   afxinl3.obj
 0001:00084597       ?SetItemData@CComboBox@@QAEHHK@Z 5f885597 f   afxinl3.obj
 0001:000845ef       ?GetItemDataPtr@CComboBox@@QBEPAXH@Z 5f8855ef f   afxinl3.obj
 0001:00084639       ?SetItemDataPtr@CComboBox@@QAEHHPAX@Z 5f885639 f   afxinl3.obj
 0001:00084687       ?GetLBText@CComboBox@@QBEHHPAG@Z 5f885687 f   afxinl3.obj
 0001:000846df       ?GetLBTextLen@CComboBox@@QBEHH@Z 5f8856df f   afxinl3.obj
 0001:00084735       ?ShowDropDown@CComboBox@@QAEXH@Z 5f885735 f   afxinl3.obj
 0001:0008478b       ?AddString@CComboBox@@QAEHPBG@Z 5f88578b f   afxinl3.obj
 0001:000847e1       ?DeleteString@CComboBox@@QAEHI@Z 5f8857e1 f   afxinl3.obj
 0001:00084837       ?InsertString@CComboBox@@QAEHHPBG@Z 5f885837 f   afxinl3.obj
 0001:0008488f       ?ResetContent@CComboBox@@QAEXXZ 5f88588f f   afxinl3.obj
 0001:000848e1       ?Dir@CComboBox@@QAEHIPBG@Z 5f8858e1 f   afxinl3.obj
 0001:00084939       ?FindString@CComboBox@@QBEHHPBG@Z 5f885939 f   afxinl3.obj
 0001:00084991       ?SelectString@CComboBox@@QAEHHPBG@Z 5f885991 f   afxinl3.obj
 0001:000849e9       ?Clear@CComboBox@@QAEXXZ   5f8859e9 f   afxinl3.obj
 0001:00084a3b       ?Copy@CComboBox@@QAEXXZ    5f885a3b f   afxinl3.obj
 0001:00084a8d       ?Cut@CComboBox@@QAEXXZ     5f885a8d f   afxinl3.obj
 0001:00084adf       ?Paste@CComboBox@@QAEXXZ   5f885adf f   afxinl3.obj
 0001:00084b31       ?SetItemHeight@CComboBox@@QAEHHI@Z 5f885b31 f   afxinl3.obj
 0001:00084b8e       ?GetItemHeight@CComboBox@@QBEHH@Z 5f885b8e f   afxinl3.obj
 0001:00084be4       ?FindStringExact@CComboBox@@QBEHHPBG@Z 5f885be4 f   afxinl3.obj
 0001:00084c3c       ?SetExtendedUI@CComboBox@@QAEHH@Z 5f885c3c f   afxinl3.obj
 0001:00084c92       ?GetExtendedUI@CComboBox@@QBEHXZ 5f885c92 f   afxinl3.obj
 0001:00084ce4       ?GetDroppedControlRect@CComboBox@@QBEXPAUtagRECT@@@Z 5f885ce4 f   afxinl3.obj
 0001:00084d3a       ?GetDroppedState@CComboBox@@QBEHXZ 5f885d3a f   afxinl3.obj
 0001:00084d8c       ?GetLocale@CComboBox@@QBEKXZ 5f885d8c f   afxinl3.obj
 0001:00084dde       ?SetLocale@CComboBox@@QAEKK@Z 5f885dde f   afxinl3.obj
 0001:00084e34       ?GetTopIndex@CComboBox@@QBEHXZ 5f885e34 f   afxinl3.obj
 0001:00084e86       ?SetTopIndex@CComboBox@@QAEHH@Z 5f885e86 f   afxinl3.obj
 0001:00084edc       ?InitStorage@CComboBox@@QAEHHI@Z 5f885edc f   afxinl3.obj
 0001:00084f34       ?SetHorizontalExtent@CComboBox@@QAEXI@Z 5f885f34 f   afxinl3.obj
 0001:00084f8a       ?GetHorizontalExtent@CComboBox@@QBEIXZ 5f885f8a f   afxinl3.obj
 0001:00084fdc       ?SetDroppedWidth@CComboBox@@QAEHI@Z 5f885fdc f   afxinl3.obj
 0001:00085032       ?GetDroppedWidth@CComboBox@@QBEHXZ 5f886032 f   afxinl3.obj
 0001:00085084       ??0CEdit@@QAE@XZ           5f886084 f   afxinl3.obj
 0001:000850a3       ?CanUndo@CEdit@@QBEHXZ     5f8860a3 f   afxinl3.obj
 0001:000850f5       ?GetLineCount@CEdit@@QBEHXZ 5f8860f5 f   afxinl3.obj
 0001:00085147       ?GetModify@CEdit@@QBEHXZ   5f886147 f   afxinl3.obj
 0001:00085199       ?SetModify@CEdit@@QAEXH@Z  5f886199 f   afxinl3.obj
 0001:000851ef       ?GetRect@CEdit@@QBEXPAUtagRECT@@@Z 5f8861ef f   afxinl3.obj
 0001:00085245       ?GetSel@CEdit@@QBEXAAH0@Z  5f886245 f   afxinl3.obj
 0001:0008529d       ?GetSel@CEdit@@QBEKXZ      5f88629d f   afxinl3.obj
 0001:000852ef       ?GetHandle@CEdit@@QBEPAXXZ 5f8862ef f   afxinl3.obj
 0001:00085341       ?SetHandle@CEdit@@QAEXPAX@Z 5f886341 f   afxinl3.obj
 0001:00085397       ?GetLine@CEdit@@QBEHHPAG@Z 5f886397 f   afxinl3.obj
 0001:000853ef       ?GetLine@CEdit@@QBEHHPAGH@Z 5f8863ef f   afxinl3.obj
 0001:00085451       ?EmptyUndoBuffer@CEdit@@QAEXXZ 5f886451 f   afxinl3.obj
 0001:000854a3       ?FmtLines@CEdit@@QAEHH@Z   5f8864a3 f   afxinl3.obj
 0001:000854f9       ?LimitText@CEdit@@QAEXH@Z  5f8864f9 f   afxinl3.obj
 0001:0008554f       ?LineFromChar@CEdit@@QBEHH@Z 5f88654f f   afxinl3.obj
 0001:000855a5       ?LineIndex@CEdit@@QBEHH@Z  5f8865a5 f   afxinl3.obj
 0001:000855fb       ?LineLength@CEdit@@QBEHH@Z 5f8865fb f   afxinl3.obj
 0001:00085651       ?LineScroll@CEdit@@QAEXHH@Z 5f886651 f   afxinl3.obj
 0001:000856a9       ?ReplaceSel@CEdit@@QAEXPBGH@Z 5f8866a9 f   afxinl3.obj
 0001:00085701       ?SetPasswordChar@CEdit@@QAEXG@Z 5f886701 f   afxinl3.obj
 0001:0008575c       ?SetRect@CEdit@@QAEXPBUtagRECT@@@Z 5f88675c f   afxinl3.obj
 0001:000857b2       ?SetRectNP@CEdit@@QAEXPBUtagRECT@@@Z 5f8867b2 f   afxinl3.obj
 0001:00085808       ?SetSel@CEdit@@QAEXKH@Z    5f886808 f   afxinl3.obj
 0001:0008588f       ?SetSel@CEdit@@QAEXHHH@Z   5f88688f f   afxinl3.obj
 0001:00085903       ?SetTabStops@CEdit@@QAEHHPAH@Z 5f886903 f   afxinl3.obj
 0001:0008595b       ?SetTabStops@CEdit@@QAEXXZ 5f88695b f   afxinl3.obj
 0001:000859cb       ?SetTabStops@CEdit@@QAEHABH@Z 5f8869cb f   afxinl3.obj
 0001:00085a21       ?Undo@CEdit@@QAEHXZ        5f886a21 f   afxinl3.obj
 0001:00085a73       ?Clear@CEdit@@QAEXXZ       5f886a73 f   afxinl3.obj
 0001:00085ac5       ?Copy@CEdit@@QAEXXZ        5f886ac5 f   afxinl3.obj
 0001:00085b17       ?Cut@CEdit@@QAEXXZ         5f886b17 f   afxinl3.obj
 0001:00085b69       ?Paste@CEdit@@QAEXXZ       5f886b69 f   afxinl3.obj
 0001:00085bbb       ?SetReadOnly@CEdit@@QAEHH@Z 5f886bbb f   afxinl3.obj
 0001:00085c11       ?GetFirstVisibleLine@CEdit@@QBEHXZ 5f886c11 f   afxinl3.obj
 0001:00085c63       ?GetPasswordChar@CEdit@@QBEGXZ 5f886c63 f   afxinl3.obj
 0001:00085cb5       ?SetMargins@CEdit@@QAEXII@Z 5f886cb5 f   afxinl3.obj
 0001:00085d1e       ?GetMargins@CEdit@@QBEKXZ  5f886d1e f   afxinl3.obj
 0001:00085d70       ?SetLimitText@CEdit@@QAEXI@Z 5f886d70 f   afxinl3.obj
 0001:00085dc6       ?GetLimitText@CEdit@@QBEIXZ 5f886dc6 f   afxinl3.obj
 0001:00085e18       ?PosFromChar@CEdit@@QBE?AVCPoint@@I@Z 5f886e18 f   afxinl3.obj
 0001:00085e89       ?CharFromPos@CEdit@@QBEHVCPoint@@@Z 5f886e89 f   afxinl3.obj
 0001:00085ef2       ??0CScrollBar@@QAE@XZ      5f886ef2 f   afxinl3.obj
 0001:00085f11       ?GetScrollPos@CScrollBar@@QBEHXZ 5f886f11 f   afxinl3.obj
 0001:00085f5c       ?SetScrollPos@CScrollBar@@QAEHHH@Z 5f886f5c f   afxinl3.obj
 0001:00085fb1       ?GetScrollRange@CScrollBar@@QBEXPAH0@Z 5f886fb1 f   afxinl3.obj
 0001:00086006       ?SetScrollRange@CScrollBar@@QAEXHHH@Z 5f887006 f   afxinl3.obj
 0001:0008605f       ?ShowScrollBar@CScrollBar@@QAEXH@Z 5f88705f f   afxinl3.obj
 0001:000860b0       ?EnableScrollBar@CScrollBar@@QAEHI@Z 5f8870b0 f   afxinl3.obj
 0001:00086101       ?SetScrollInfo@CScrollBar@@QAEHPAUtagSCROLLINFO@@H@Z 5f887101 f   afxinl3.obj
 0001:00086120       ?GetScrollInfo@CScrollBar@@QAEHPAUtagSCROLLINFO@@I@Z 5f887120 f   afxinl3.obj
 0001:0008613f       ?GetScrollLimit@CScrollBar@@QAEHXZ 5f88713f f   afxinl3.obj
 0001:00086154       ?MDIActivate@CMDIFrameWnd@@QAEXPAVCWnd@@@Z 5f887154 f   afxinl3.obj
 0001:000861b0       ?MDIIconArrange@CMDIFrameWnd@@QAEXXZ 5f8871b0 f   afxinl3.obj
 0001:00086205       ?MDIMaximize@CMDIFrameWnd@@QAEXPAVCWnd@@@Z 5f887205 f   afxinl3.obj
 0001:00086261       ?MDINext@CMDIFrameWnd@@QAEXXZ 5f887261 f   afxinl3.obj
 0001:000862b6       ?MDIRestore@CMDIFrameWnd@@QAEXPAVCWnd@@@Z 5f8872b6 f   afxinl3.obj
 0001:00086312       ?MDISetMenu@CMDIFrameWnd@@QAEPAVCMenu@@PAV2@0@Z 5f887312 f   afxinl3.obj
 0001:0008637d       ?MDITile@CMDIFrameWnd@@QAEXXZ 5f88737d f   afxinl3.obj
 0001:000863d2       ?MDICascade@CMDIFrameWnd@@QAEXXZ 5f8873d2 f   afxinl3.obj
 0001:00086427       ?MDICascade@CMDIFrameWnd@@QAEXH@Z 5f887427 f   afxinl3.obj
 0001:00086480       ?MDITile@CMDIFrameWnd@@QAEXH@Z 5f887480 f   afxinl3.obj
 0001:000864d9       ?MDIDestroy@CMDIChildWnd@@QAEXXZ 5f8874d9 f   afxinl3.obj
 0001:00086535       ?MDIActivate@CMDIChildWnd@@QAEXXZ 5f887535 f   afxinl3.obj
 0001:00086591       ?MDIMaximize@CMDIChildWnd@@QAEXXZ 5f887591 f   afxinl3.obj
 0001:000865ed       ?MDIRestore@CMDIChildWnd@@QAEXXZ 5f8875ed f   afxinl3.obj
 0001:00086649       ?GetDocument@CView@@QBEPAVCDocument@@XZ 5f887649 f   afxinl3.obj
 0001:00086680       ?GetTotalSize@CScrollView@@QBE?AVCSize@@XZ 5f887680 f   afxinl3.obj
 0001:000866c7       ?GetTitle@CDocument@@QBEABVCString@@XZ 5f8876c7 f   afxinl3.obj
 0001:000866fe       ?GetPathName@CDocument@@QBEABVCString@@XZ 5f8876fe f   afxinl3.obj
 0001:00086735       ?GetDocTemplate@CDocument@@QBEPAVCDocTemplate@@XZ 5f887735 f   afxinl3.obj
 0001:0008676c       ?IsModified@CDocument@@UAEHXZ 5f88776c f   afxinl3.obj
 0001:000867a3       ?SetModifiedFlag@CDocument@@UAEXH@Z 5f8877a3 f   afxinl3.obj
 0001:000867df       ??BCWinThread@@QBEPAXXZ    5f8877df f   afxinl3.obj
 0001:00086807       ?SetThreadPriority@CWinThread@@QAEHH@Z 5f887807 f   afxinl3.obj
 0001:0008684e       ?GetThreadPriority@CWinThread@@QAEHXZ 5f88784e f   afxinl3.obj
 0001:0008688f       ?ResumeThread@CWinThread@@QAEKXZ 5f88788f f   afxinl3.obj
 0001:000868d0       ?SuspendThread@CWinThread@@QAEKXZ 5f8878d0 f   afxinl3.obj
 0001:00086911       ?PostThreadMessageW@CWinThread@@QAEHIIJ@Z 5f887911 f   afxinl3.obj
 0001:00086960       ?LoadCursorW@CWinApp@@QBEPAUHICON__@@PBG@Z 5f887960 f   afxinl3.obj
 0001:00086983       ?LoadCursorW@CWinApp@@QBEPAUHICON__@@I@Z 5f887983 f   afxinl3.obj
 0001:000869b1       ?LoadStandardCursor@CWinApp@@QBEPAUHICON__@@PBG@Z 5f8879b1 f   afxinl3.obj
 0001:000869ca       ?LoadOEMCursor@CWinApp@@QBEPAUHICON__@@I@Z 5f8879ca f   afxinl3.obj
 0001:000869e8       ?LoadIconW@CWinApp@@QBEPAUHICON__@@PBG@Z 5f8879e8 f   afxinl3.obj
 0001:00086a0b       ?LoadIconW@CWinApp@@QBEPAUHICON__@@I@Z 5f887a0b f   afxinl3.obj
 0001:00086a39       ?LoadStandardIcon@CWinApp@@QBEPAUHICON__@@PBG@Z 5f887a39 f   afxinl3.obj
 0001:00086a52       ?LoadOEMIcon@CWinApp@@QBEPAUHICON__@@I@Z 5f887a52 f   afxinl3.obj
 0001:00086a70       ??0CWaitCursor@@QAE@XZ     5f887a70 f   afxinl3.obj
 0001:00086a8a       ??1CWaitCursor@@QAE@XZ     5f887a8a f   afxinl3.obj
 0001:00086aa1       ?Restore@CWaitCursor@@QAEXXZ 5f887aa1 f   afxinl3.obj
 0001:00086ab8       ?CloseWindow@CWnd@@QAEXXZ  5f887ab8 f   afxinl3.obj
 0001:00086b01       ?OpenIcon@CWnd@@QAEHXZ     5f887b01 f   afxinl3.obj
 0001:00086b50       ??1CCheckListBox@@UAE@XZ   5f887b50 f i afxinl3.obj
 0001:00086b70       ??1CIPAddressCtrl@@UAE@XZ  5f887b70 f   winctrl6.obj
 0001:00086bc1       ?Create@CIPAddressCtrl@@QAEHKABUtagRECT@@PAVCWnd@@I@Z 5f887bc1 f   winctrl6.obj
 0001:00086c49       ?GetAddress@CIPAddressCtrl@@QAEHAAE000@Z 5f887c49 f   winctrl6.obj
 0001:00086cf0       ??_ECIPAddressCtrl@@UAEPAXI@Z 5f887cf0 f i winctrl6.obj
 0001:00086cf0       ??_GCIPAddressCtrl@@UAEPAXI@Z 5f887cf0 f i winctrl6.obj
 0001:00086d20       ?_AfxParseURLWorker@@YGHPBGPAUURL_COMPONENTSW@@AAKAAGK@Z 5f887d20 f   inet.obj
 0001:0008703e       ?AfxParseURLEx@@YGHPBGAAKAAVCString@@2AAG22K@Z 5f88803e f   inet.obj
 0001:00087140       ?AfxParseURL@@YGHPBGAAKAAVCString@@2AAG@Z 5f888140 f   inet.obj
 0001:000871fe       ?AfxGetInternetHandleType@@YGKPAX@Z 5f8881fe f   inet.obj
 0001:00087239       ?_AfxQueryCStringInternetOption@@YGHPAXKAAVCString@@@Z 5f888239 f   inet.obj
 0001:000872ba       ?AfxInternetStatusCallbackDebug@@YGXPAXKK0K@Z 5f8882ba f   inet.obj
 0001:000874ef       ?AfxInternetStatusCallback@@YGXPAXKK0K@Z 5f8884ef f   inet.obj
 0001:0008754f       ??1CInternetSession@@UAE@XZ 5f88854f f   inet.obj
 0001:000875a0       ??0CInternetSession@@QAE@PBGKK00K@Z 5f8885a0 f   inet.obj
 0001:00087694       ?Close@CInternetSession@@UAEXXZ 5f888694 f   inet.obj
 0001:000876e3       ?GetGopherConnection@CInternetSession@@QAEPAVCGopherConnection@@PBG00G@Z 5f8886e3 f   inet.obj
 0001:000877a7       ?GetFtpConnection@CInternetSession@@QAEPAVCFtpConnection@@PBG00GH@Z 5f8887a7 f   inet.obj
 0001:0008786f       ?GetHttpConnection@CInternetSession@@QAEPAVCHttpConnection@@PBGG00@Z 5f88886f f   inet.obj
 0001:00087933       ?GetHttpConnection@CInternetSession@@QAEPAVCHttpConnection@@PBGKG00@Z 5f888933 f   inet.obj
 0001:00087a22       ?OpenURL@CInternetSession@@QAEPAVCStdioFile@@PBGKK0K@Z 5f888a22 f   inet.obj
 0001:00087e2c       ?SetOption@CInternetSession@@QAEHKPAXKK@Z 5f888e2c f   inet.obj
 0001:00087f21       ?QueryOption@CInternetSession@@QBEHKPAXPAK@Z 5f888f21 f   inet.obj
 0001:00087ff5       ?QueryOption@CInternetSession@@QBEHKAAK@Z 5f888ff5 f   inet.obj
 0001:00088024       ?QueryOption@CInternetSession@@QBEHKAAVCString@@@Z 5f889024 f   inet.obj
 0001:00088071       ?OnStatusCallback@CInternetSession@@UAEXKKPAXK@Z 5f889071 f   inet.obj
 0001:000880cd       ?EnableStatusCallback@CInternetSession@@QAEHH@Z 5f8890cd f   inet.obj
 0001:000881dc       ?SetCookie@CInternetSession@@SAHPBDPBG1@Z 5f8891dc f   inet.obj
 0001:0008824b       ?GetCookie@CInternetSession@@SAHPBDPBGPAGK@Z 5f88924b f   inet.obj
 0001:000882de       ?GetCookieLength@CInternetSession@@SAKPBDPBG@Z 5f8892de f   inet.obj
 0001:00088360       ?GetCookie@CInternetSession@@SAHPBDPBGAAVCString@@@Z 5f889360 f   inet.obj
 0001:0008841d       ?Dump@CInternetSession@@UBEXAAVCDumpContext@@@Z 5f88941d f   inet.obj
 0001:0008846c       ??0CInternetFile@@IAE@PAX0PBG1KH@Z 5f88946c f   inet.obj
 0001:000885c0       ??0CInternetFile@@IAE@PAXPBGPAVCInternetConnection@@H@Z 5f8895c0 f   inet.obj
 0001:00088761       ?QueryOption@CInternetFile@@QBEHKPAXPAK@Z 5f889761 f   inet.obj
 0001:00088858       ?QueryOption@CInternetFile@@QBEHKAAK@Z 5f889858 f   inet.obj
 0001:000888b0       ?QueryOption@CInternetFile@@QBEHKAAVCString@@@Z 5f8898b0 f   inet.obj
 0001:00088920       ?SetOption@CInternetFile@@QAEHKPAXKK@Z 5f889920 f   inet.obj
 0001:00088a15       ?SetReadBufferSize@CInternetFile@@QAEHI@Z 5f889a15 f   inet.obj
 0001:00088b74       ?SetWriteBufferSize@CInternetFile@@QAEHI@Z 5f889b74 f   inet.obj
 0001:00088c86       ?Seek@CInternetFile@@UAEJJI@Z 5f889c86 f   inet.obj
 0001:00088dd5       ??1CInternetFile@@UAE@XZ   5f889dd5 f   inet.obj
 0001:00088f0f       ?Abort@CInternetFile@@UAEXXZ 5f889f0f f   inet.obj
 0001:00088f4c       ?Flush@CInternetFile@@UAEXXZ 5f889f4c f   inet.obj
 0001:00088fbf       ?Close@CInternetFile@@UAEXXZ 5f889fbf f   inet.obj
 0001:0008905c       ?Read@CInternetFile@@UAEIPAXI@Z 5f88a05c f   inet.obj
 0001:00089323       ?Write@CInternetFile@@UAEXPBXI@Z 5f88a323 f   inet.obj
 0001:000894e6       ?WriteString@CInternetFile@@UAEXPBG@Z 5f88a4e6 f   inet.obj
 0001:000895b5       ?ReadString@CInternetFile@@UAEPAGPAGI@Z 5f88a5b5 f   inet.obj
 0001:00089792       ?ReadString@CInternetFile@@UAEHAAVCString@@@Z 5f88a792 f   inet.obj
 0001:000898ce       ?GetLength@CInternetFile@@UBEKXZ 5f88a8ce f   inet.obj
 0001:0008994a       ?LockRange@CInternetFile@@UAEXKK@Z 5f88a94a f   inet.obj
 0001:00089998       ?UnlockRange@CInternetFile@@UAEXKK@Z 5f88a998 f   inet.obj
 0001:000899e6       ?SetLength@CInternetFile@@UAEXK@Z 5f88a9e6 f   inet.obj
 0001:00089a34       ?Duplicate@CInternetFile@@UBEPAVCFile@@XZ 5f88aa34 f   inet.obj
 0001:00089a82       ?AssertValid@CInternetFile@@MBEXXZ 5f88aa82 f   inet.obj
 0001:00089bbf       ?Dump@CInternetFile@@MBEXAAVCDumpContext@@@Z 5f88abbf f   inet.obj
 0001:00089c14       ??0CInternetConnection@@QAE@PAVCInternetSession@@PBGGK@Z 5f88ac14 f   inet.obj
 0001:00089d06       ??1CInternetConnection@@UAE@XZ 5f88ad06 f   inet.obj
 0001:00089e0b       ?SetOption@CInternetConnection@@QAEHKPAXKK@Z 5f88ae0b f   inet.obj
 0001:00089f00       ?QueryOption@CInternetConnection@@QBEHKPAXPAK@Z 5f88af00 f   inet.obj
 0001:00089fd4       ?QueryOption@CInternetConnection@@QBEHKAAK@Z 5f88afd4 f   inet.obj
 0001:0008a003       ?QueryOption@CInternetConnection@@QBEHKAAVCString@@@Z 5f88b003 f   inet.obj
 0001:0008a050       ?Close@CInternetConnection@@MAEXXZ 5f88b050 f   inet.obj
 0001:0008a08c       ?Dump@CInternetConnection@@UBEXAAVCDumpContext@@@Z 5f88b08c f   inet.obj
 0001:0008a0c0       ?AssertValid@CInternetConnection@@UBEXXZ 5f88b0c0 f   inet.obj
 0001:0008a0d3       ??1CFtpConnection@@UAE@XZ  5f88b0d3 f   inet.obj
 0001:0008a127       ??0CFtpConnection@@QAE@PAVCInternetSession@@PAXPBGK@Z 5f88b127 f   inet.obj
 0001:0008a271       ??0CFtpConnection@@QAE@PAVCInternetSession@@PBG11KGH@Z 5f88b271 f   inet.obj
 0001:0008a3da       ?Close@CFtpConnection@@UAEXXZ 5f88b3da f   inet.obj
 0001:0008a3ed       ?Remove@CFtpConnection@@QAEHPBG@Z 5f88b3ed f   inet.obj
 0001:0008a470       ?Rename@CFtpConnection@@QAEHPBG0@Z 5f88b470 f   inet.obj
 0001:0008a520       ?CreateDirectoryW@CFtpConnection@@QAEHPBG@Z 5f88b520 f   inet.obj
 0001:0008a5a3       ?RemoveDirectoryW@CFtpConnection@@QAEHPBG@Z 5f88b5a3 f   inet.obj
 0001:0008a626       ?SetCurrentDirectoryW@CFtpConnection@@QAEHPBG@Z 5f88b626 f   inet.obj
 0001:0008a6a9       ?GetCurrentDirectoryW@CFtpConnection@@QBEHPAGPAK@Z 5f88b6a9 f   inet.obj
 0001:0008a756       ?GetCurrentDirectoryAsURL@CFtpConnection@@QBEHAAVCString@@@Z 5f88b756 f   inet.obj
 0001:0008a842       ?GetCurrentDirectoryAsURL@CFtpConnection@@QBEHPAGPAK@Z 5f88b842 f   inet.obj
 0001:0008a9bd       ?GetCurrentDirectoryW@CFtpConnection@@QBEHAAVCString@@@Z 5f88b9bd f   inet.obj
 0001:0008aa57       ?OpenFile@CFtpConnection@@QAEPAVCInternetFile@@PBGKKK@Z 5f88ba57 f   inet.obj
 0001:0008abdd       ?PutFile@CFtpConnection@@QAEHPBG0KK@Z 5f88bbdd f   inet.obj
 0001:0008accb       ?GetFile@CFtpConnection@@QAEHPBG0HKKK@Z 5f88bccb f   inet.obj
 0001:0008ade4       ?Dump@CFtpConnection@@UBEXAAVCDumpContext@@@Z 5f88bde4 f   inet.obj
 0001:0008ae17       ?AssertValid@CFtpConnection@@UBEXXZ 5f88be17 f   inet.obj
 0001:0008ae7f       ??1CGopherConnection@@UAE@XZ 5f88be7f f   inet.obj
 0001:0008ae9b       ??0CGopherConnection@@QAE@PAVCInternetSession@@PBG11KG@Z 5f88be9b f   inet.obj
 0001:0008afd6       ??0CGopherConnection@@QAE@PAVCInternetSession@@PAXPBGK@Z 5f88bfd6 f   inet.obj
 0001:0008b102       ?CreateLocator@CGopherConnection@@SA?AVCGopherLocator@@PBG@Z 5f88c102 f   inet.obj
 0001:0008b173       ?CreateLocator@CGopherConnection@@SA?AVCGopherLocator@@PBG00KG@Z 5f88c173 f   inet.obj
 0001:0008b2a8       ?CreateLocator@CGopherConnection@@QAE?AVCGopherLocator@@PBG0K@Z 5f88c2a8 f   inet.obj
 0001:0008b3d5       ?GetAttribute@CGopherConnection@@QAEHAAVCGopherLocator@@VCString@@AAV3@@Z 5f88c3d5 f   inet.obj
 0001:0008b48f       ?OpenFile@CGopherConnection@@QAEPAVCGopherFile@@AAVCGopherLocator@@KPBGK@Z 5f88c48f f   inet.obj
 0001:0008b595       ?Close@CGopherConnection@@UAEXXZ 5f88c595 f   inet.obj
 0001:0008b5a8       ?Dump@CGopherConnection@@UBEXAAVCDumpContext@@@Z 5f88c5a8 f   inet.obj
 0001:0008b5db       ?AssertValid@CGopherConnection@@UBEXXZ 5f88c5db f   inet.obj
 0001:0008b643       ??1CHttpConnection@@UAE@XZ 5f88c643 f   inet.obj
 0001:0008b697       ??0CHttpConnection@@QAE@PAVCInternetSession@@PAXPBGK@Z 5f88c697 f   inet.obj
 0001:0008b7d2       ??0CHttpConnection@@QAE@PAVCInternetSession@@PBGG11K@Z 5f88c7d2 f   inet.obj
 0001:0008b91c       ??0CHttpConnection@@QAE@PAVCInternetSession@@PBGKG11K@Z 5f88c91c f   inet.obj
 0001:0008ba8f       ?Close@CHttpConnection@@UAEXXZ 5f88ca8f f   inet.obj
 0001:0008baa2       ?OpenRequest@CHttpConnection@@QAEPAVCHttpFile@@PBG00KPAPBG0K@Z 5f88caa2 f   inet.obj
 0001:0008bbde       ?OpenRequest@CHttpConnection@@QAEPAVCHttpFile@@HPBG0KPAPBG0K@Z 5f88cbde f   inet.obj
 0001:0008bce4       ?Dump@CHttpConnection@@UBEXAAVCDumpContext@@@Z 5f88cce4 f   inet.obj
 0001:0008bd17       ?AssertValid@CHttpConnection@@UBEXXZ 5f88cd17 f   inet.obj
 0001:0008bd7f       ??0CHttpFile@@IAE@PAX0PBG11K@Z 5f88cd7f f   inet.obj
 0001:0008be38       ??0CHttpFile@@IAE@PAXPBG1PAVCHttpConnection@@@Z 5f88ce38 f   inet.obj
 0001:0008bf33       ??1CHttpFile@@UAE@XZ       5f88cf33 f   inet.obj
 0001:0008bf96       ?Close@CHttpFile@@UAEXXZ   5f88cf96 f   inet.obj
 0001:0008bfa9       ?ErrorDlg@CHttpFile@@QAEKPAVCWnd@@KKPAPAX@Z 5f88cfa9 f   inet.obj
 0001:0008c03f       ?GetVerb@CHttpFile@@QBE?AVCString@@XZ 5f88d03f f   inet.obj
 0001:0008c0ac       ?GetObjectW@CHttpFile@@QBE?AVCString@@XZ 5f88d0ac f   inet.obj
 0001:0008c119       ?GetFileURL@CHttpFile@@UBE?AVCString@@XZ 5f88d119 f   inet.obj
 0001:0008c235       ?AddRequestHeaders@CHttpFile@@QAEHPBGKH@Z 5f88d235 f   inet.obj
 0001:0008c308       ?AddRequestHeaders@CHttpFile@@QAEHAAVCString@@K@Z 5f88d308 f   inet.obj
 0001:0008c333       ?SendRequest@CHttpFile@@QAEHPBGKPAXK@Z 5f88d333 f   inet.obj
 0001:0008c401       ?EndRequest@CHttpFile@@QAEHKPAU_INTERNET_BUFFERSW@@K@Z 5f88d401 f   inet.obj
 0001:0008c49e       ?SendRequestEx@CHttpFile@@QAEHKKK@Z 5f88d49e f   inet.obj
 0001:0008c518       ?SendRequestEx@CHttpFile@@QAEHPAU_INTERNET_BUFFERSW@@0KK@Z 5f88d518 f   inet.obj
 0001:0008c602       ?SendRequest@CHttpFile@@QAEHAAVCString@@PAXK@Z 5f88d602 f   inet.obj
 0001:0008c693       ?QueryInfo@CHttpFile@@QBEHKPAXPAK1@Z 5f88d693 f   inet.obj
 0001:0008c74e       ?QueryInfo@CHttpFile@@QBEHKAAKPAK@Z 5f88d74e f   inet.obj
 0001:0008c787       ?QueryInfo@CHttpFile@@QBEHKPAU_SYSTEMTIME@@PAK@Z 5f88d787 f   inet.obj
 0001:0008c7c0       ?QueryInfoStatusCode@CHttpFile@@QBEHAAK@Z 5f88d7c0 f   inet.obj
 0001:0008c85e       ?QueryInfo@CHttpFile@@QBEHKAAVCString@@PAK@Z 5f88d85e f   inet.obj
 0001:0008c954       ?Dump@CHttpFile@@MBEXAAVCDumpContext@@@Z 5f88d954 f   inet.obj
 0001:0008c995       ?AssertValid@CHttpFile@@MBEXXZ 5f88d995 f   inet.obj
 0001:0008c9a8       ??0CGopherFile@@IAE@PAXAAVCGopherLocator@@PAVCGopherConnection@@@Z 5f88d9a8 f   inet.obj
 0001:0008ca51       ??0CGopherFile@@IAE@PAX0PBGKK@Z 5f88da51 f   inet.obj
 0001:0008caca       ??1CGopherFile@@UAE@XZ     5f88daca f   inet.obj
 0001:0008cb1e       ?Close@CGopherFile@@UAEXXZ 5f88db1e f   inet.obj
 0001:0008cb31       ?Write@CGopherFile@@UAEXPBXI@Z 5f88db31 f   inet.obj
 0001:0008cb6c       ?WriteString@CGopherFile@@UAEXPBG@Z 5f88db6c f   inet.obj
 0001:0008cba7       ?Dump@CGopherFile@@UBEXAAVCDumpContext@@@Z 5f88dba7 f   inet.obj
 0001:0008cbc0       ?AssertValid@CGopherFile@@UBEXXZ 5f88dbc0 f   inet.obj
 0001:0008cbd3       ??0CFtpFileFind@@QAE@PAVCFtpConnection@@K@Z 5f88dbd3 f   inet.obj
 0001:0008cc9e       ??1CFtpFileFind@@UAE@XZ    5f88dc9e f   inet.obj
 0001:0008ccba       ?FindFile@CFtpFileFind@@UAEHPBGK@Z 5f88dcba f   inet.obj
 0001:0008cf4f       ?FindNextFileW@CFtpFileFind@@UAEHXZ 5f88df4f f   inet.obj
 0001:0008d003       ?CloseContext@CFtpFileFind@@MAEXXZ 5f88e003 f   inet.obj
 0001:0008d037       ?GetFileURL@CFtpFileFind@@UBE?AVCString@@XZ 5f88e037 f   inet.obj
 0001:0008d158       ?Dump@CFtpFileFind@@UBEXAAVCDumpContext@@@Z 5f88e158 f   inet.obj
 0001:0008d18c       ?AssertValid@CFtpFileFind@@UBEXXZ 5f88e18c f   inet.obj
 0001:0008d19f       ??0CGopherFileFind@@QAE@PAVCGopherConnection@@K@Z 5f88e19f f   inet.obj
 0001:0008d261       ??1CGopherFileFind@@UAE@XZ 5f88e261 f   inet.obj
 0001:0008d27d       ?FindFile@CGopherFileFind@@UAEHPBGK@Z 5f88e27d f   inet.obj
 0001:0008d33c       ?FindFile@CGopherFileFind@@UAEHAAVCGopherLocator@@PBGK@Z 5f88e33c f   inet.obj
 0001:0008d423       ?FindNextFileW@CGopherFileFind@@UAEHXZ 5f88e423 f   inet.obj
 0001:0008d4d7       ?CloseContext@CGopherFileFind@@MAEXXZ 5f88e4d7 f   inet.obj
 0001:0008d50b       ?GetFileName@CGopherFileFind@@UBE?AVCString@@XZ 5f88e50b f   inet.obj
 0001:0008d539       ?GetFilePath@CGopherFileFind@@UBE?AVCString@@XZ 5f88e539 f   inet.obj
 0001:0008d567       ?GetFileTitle@CGopherFileFind@@UBE?AVCString@@XZ 5f88e567 f   inet.obj
 0001:0008d595       ?IsDots@CGopherFileFind@@UBEHXZ 5f88e595 f   inet.obj
 0001:0008d5a2       ?GetLastWriteTime@CGopherFileFind@@UBEHPAU_FILETIME@@@Z 5f88e5a2 f   inet.obj
 0001:0008d64e       ?GetLastAccessTime@CGopherFileFind@@UBEHPAU_FILETIME@@@Z 5f88e64e f   inet.obj
 0001:0008d6a1       ?GetCreationTime@CGopherFileFind@@UBEHPAU_FILETIME@@@Z 5f88e6a1 f   inet.obj
 0001:0008d6f4       ?GetLastWriteTime@CGopherFileFind@@UBEHAAVCTime@@@Z 5f88e6f4 f   inet.obj
 0001:0008d771       ?GetCreationTime@CGopherFileFind@@UBEHAAVCTime@@@Z 5f88e771 f   inet.obj
 0001:0008d78d       ?GetLastAccessTime@CGopherFileFind@@UBEHAAVCTime@@@Z 5f88e78d f   inet.obj
 0001:0008d7a9       ?GetFileURL@CGopherFileFind@@UBE?AVCString@@XZ 5f88e7a9 f   inet.obj
 0001:0008d7d7       ?GetRoot@CGopherFileFind@@UBE?AVCString@@XZ 5f88e7d7 f   inet.obj
 0001:0008d805       ?GetLocator@CGopherFileFind@@QBE?AVCGopherLocator@@XZ 5f88e805 f   inet.obj
 0001:0008d885       ?GetScreenName@CGopherFileFind@@QBE?AVCString@@XZ 5f88e885 f   inet.obj
 0001:0008d941       ?GetLength@CGopherFileFind@@UBEKXZ 5f88e941 f   inet.obj
 0001:0008d978       ?GetLength64@CGopherFileFind@@UBE_JXZ 5f88e978 f   inet.obj
 0001:0008d9c6       ?Dump@CGopherFileFind@@UBEXAAVCDumpContext@@@Z 5f88e9c6 f   inet.obj
 0001:0008d9fa       ?AssertValid@CGopherFileFind@@UBEXXZ 5f88e9fa f   inet.obj
 0001:0008da0d       ??0CGopherLocator@@AAE@PBGK@Z 5f88ea0d f   inet.obj
 0001:0008dad9       ??1CGopherLocator@@UAE@XZ  5f88ead9 f   inet.obj
 0001:0008db2d       ?AfxThrowInternetException@@YGXKK@Z 5f88eb2d f   inet.obj
 0001:0008dbe1       ?GetErrorMessage@CInternetException@@UAEHPAGIPAI@Z 5f88ebe1 f   inet.obj
 0001:0008dd87       ??0CInternetException@@QAE@K@Z 5f88ed87 f   inet.obj
 0001:0008ddb1       ??1CInternetException@@UAE@XZ 5f88edb1 f   inet.obj
 0001:0008ddcd       ?Dump@CInternetException@@UBEXAAVCDumpContext@@@Z 5f88edcd f   inet.obj
 0001:0008de1c       ?GetContext@CInternetSession@@QBEKXZ 5f88ee1c f   inet.obj
 0001:0008de2d       ?GetServerName@CInternetConnection@@QBE?AVCString@@XZ 5f88ee2d f   inet.obj
 0001:0008de5e       ?GetSession@CInternetConnection@@QBEPAVCInternetSession@@XZ 5f88ee5e f   inet.obj
 0001:0008de6f       ??BCInternetSession@@QBEPAXXZ 5f88ee6f f   inet.obj
 0001:0008de80       ?SetOption@CInternetSession@@QAEHKKK@Z 5f88ee80 f   inet.obj
 0001:0008decc       ??BCGopherLocator@@QBEPBGXZ 5f88eecc f   inet.obj
 0001:0008dee2       ?GetLocatorType@CGopherLocator@@QBEHAAK@Z 5f88eee2 f   inet.obj
 0001:0008df05       ??0CGopherLocator@@QAE@ABV0@@Z 5f88ef05 f   inet.obj
 0001:0008df80       ??BCInternetConnection@@QBEPAXXZ 5f88ef80 f   inet.obj
 0001:0008df91       ?GetContext@CInternetConnection@@QBEKXZ 5f88ef91 f   inet.obj
 0001:0008dfa2       ?SetOption@CInternetConnection@@QAEHKKK@Z 5f88efa2 f   inet.obj
 0001:0008dfc5       ?GetContext@CInternetFile@@QBEKXZ 5f88efc5 f   inet.obj
 0001:0008dfd6       ??BCInternetFile@@QBEPAXXZ 5f88efd6 f   inet.obj
 0001:0008dfe7       ?SetOption@CInternetFile@@QAEHKKK@Z 5f88efe7 f   inet.obj
 0001:0008e040       ?Lookup@CSessionMapPtrToPtr@@QAEHPAXAAPAVCInternetSession@@@Z 5f88f040 f i inet.obj
 0001:0008e080       ?SetAt@CSessionMapPtrToPtr@@QAEXPAXPAVCInternetSession@@@Z 5f88f080 f i inet.obj
 0001:0008e0c0       ?RemoveKey@CSessionMapPtrToPtr@@QAEXPAX@Z 5f88f0c0 f i inet.obj
 0001:0008e100       ??_ECInternetFile@@UAEPAXI@Z 5f88f100 f i inet.obj
 0001:0008e100       ??_GCInternetFile@@UAEPAXI@Z 5f88f100 f i inet.obj
 0001:0008e130       ??_GCInternetConnection@@UAEPAXI@Z 5f88f130 f i inet.obj
 0001:0008e130       ??_ECInternetConnection@@UAEPAXI@Z 5f88f130 f i inet.obj
 0001:0008e160       ??_ECFtpConnection@@UAEPAXI@Z 5f88f160 f i inet.obj
 0001:0008e160       ??_GCFtpConnection@@UAEPAXI@Z 5f88f160 f i inet.obj
 0001:0008e190       ??_GCGopherConnection@@UAEPAXI@Z 5f88f190 f i inet.obj
 0001:0008e190       ??_ECGopherConnection@@UAEPAXI@Z 5f88f190 f i inet.obj
 0001:0008e1c0       ??_GCHttpConnection@@UAEPAXI@Z 5f88f1c0 f i inet.obj
 0001:0008e1c0       ??_ECHttpConnection@@UAEPAXI@Z 5f88f1c0 f i inet.obj
 0001:0008e1f0       ??_ECHttpFile@@UAEPAXI@Z   5f88f1f0 f i inet.obj
 0001:0008e1f0       ??_GCHttpFile@@UAEPAXI@Z   5f88f1f0 f i inet.obj
 0001:0008e220       ??_ECGopherFile@@UAEPAXI@Z 5f88f220 f i inet.obj
 0001:0008e220       ??_GCGopherFile@@UAEPAXI@Z 5f88f220 f i inet.obj
 0001:0008e250       ??_ECFtpFileFind@@UAEPAXI@Z 5f88f250 f i inet.obj
 0001:0008e250       ??_GCFtpFileFind@@UAEPAXI@Z 5f88f250 f i inet.obj
 0001:0008e280       ??_GCGopherFileFind@@UAEPAXI@Z 5f88f280 f i inet.obj
 0001:0008e280       ??_ECGopherFileFind@@UAEPAXI@Z 5f88f280 f i inet.obj
 0001:0008e2b0       ??_GCGopherLocator@@UAEPAXI@Z 5f88f2b0 f i inet.obj
 0001:0008e2b0       ??_ECGopherLocator@@UAEPAXI@Z 5f88f2b0 f i inet.obj
 0001:0008e2e0       ??_ECInternetException@@UAEPAXI@Z 5f88f2e0 f i inet.obj
 0001:0008e2e0       ??_GCInternetException@@UAEPAXI@Z 5f88f2e0 f i inet.obj
 0001:0008e310       ??0CSessionMapPtrToPtr@@QAE@XZ 5f88f310 f i inet.obj
 0001:0008e370       ??_ECSessionMapPtrToPtr@@UAEPAXI@Z 5f88f370 f i inet.obj
 0001:0008e370       ??_GCSessionMapPtrToPtr@@UAEPAXI@Z 5f88f370 f i inet.obj
 0001:0008e3a0       ??1CSessionMapPtrToPtr@@UAE@XZ 5f88f3a0 f i inet.obj
 0001:0008e400       ?_GetBaseClass@CException@@KGPAUCRuntimeClass@@XZ 5f88f400 f   except.obj
 0001:0008e40a       ?GetRuntimeClass@CException@@UBEPAUCRuntimeClass@@XZ 5f88f40a f   except.obj
 0001:0008e41a       ?_GetBaseClass@CMemoryException@@KGPAUCRuntimeClass@@XZ 5f88f41a f   except.obj
 0001:0008e424       ?GetRuntimeClass@CMemoryException@@UBEPAUCRuntimeClass@@XZ 5f88f424 f   except.obj
 0001:0008e47a       ?_GetBaseClass@CNotSupportedException@@KGPAUCRuntimeClass@@XZ 5f88f47a f   except.obj
 0001:0008e484       ?GetRuntimeClass@CNotSupportedException@@UBEPAUCRuntimeClass@@XZ 5f88f484 f   except.obj
 0001:0008e4e0       ??B?$CThreadLocal@V_AFX_THREAD_STATE@@@@QAEPAV_AFX_THREAD_STATE@@XZ 5f88f4e0 f i except.obj
 0001:0008e4e0       ??C?$CThreadLocal@V_AFX_THREAD_STATE@@@@QAEPAV_AFX_THREAD_STATE@@XZ 5f88f4e0 f i except.obj
 0001:0008e500       ?GetData@?$CThreadLocal@V_AFX_THREAD_STATE@@@@QAEPAV_AFX_THREAD_STATE@@XZ 5f88f500 f i except.obj
 0001:0008e550       ?CreateObject@?$CThreadLocal@V_AFX_THREAD_STATE@@@@SGPAVCNoTrackObject@@XZ 5f88f550 f i except.obj
 0001:0008e5c0       ?_GetBaseClass@CArchiveException@@KGPAUCRuntimeClass@@XZ 5f88f5c0 f   arcex.obj
 0001:0008e5ca       ?GetRuntimeClass@CArchiveException@@UBEPAUCRuntimeClass@@XZ 5f88f5ca f   arcex.obj
 0001:0008e5e0       ?_GetBaseClass@CFile@@KGPAUCRuntimeClass@@XZ 5f88f5e0 f   filecore.obj
 0001:0008e5ea       ?GetRuntimeClass@CFile@@UBEPAUCRuntimeClass@@XZ 5f88f5ea f   filecore.obj
 0001:0008e600       ?_GetBaseClass@CStdioFile@@KGPAUCRuntimeClass@@XZ 5f88f600 f   filetxt.obj
 0001:0008e60a       ?GetRuntimeClass@CStdioFile@@UBEPAUCRuntimeClass@@XZ 5f88f60a f   filetxt.obj
 0001:0008e620       ?_GetBaseClass@CMemFile@@KGPAUCRuntimeClass@@XZ 5f88f620 f   filemem.obj
 0001:0008e62a       ?GetRuntimeClass@CMemFile@@UBEPAUCRuntimeClass@@XZ 5f88f62a f   filemem.obj
 0001:0008e640       ?_GetBaseClass@CSharedFile@@KGPAUCRuntimeClass@@XZ 5f88f640 f   fileshrd.obj
 0001:0008e64a       ?GetRuntimeClass@CSharedFile@@UBEPAUCRuntimeClass@@XZ 5f88f64a f   fileshrd.obj
 0001:0008e660       ?_GetBaseClass@CFileException@@KGPAUCRuntimeClass@@XZ 5f88f660 f   filex.obj
 0001:0008e66a       ?GetRuntimeClass@CFileException@@UBEPAUCRuntimeClass@@XZ 5f88f66a f   filex.obj
 0001:0008e680       ?CreateObject@CByteArray@@SGPAVCObject@@XZ 5f88f680 f   array_b.obj
 0001:0008e6ee       ?_GetBaseClass@CByteArray@@KGPAUCRuntimeClass@@XZ 5f88f6ee f   array_b.obj
 0001:0008e6f8       ?GetRuntimeClass@CByteArray@@UBEPAUCRuntimeClass@@XZ 5f88f6f8 f   array_b.obj
 0001:0008e726       ??5@YGAAVCArchive@@AAV0@AAPAVCByteArray@@@Z 5f88f726 f   array_b.obj
 0001:0008e750       ?CreateObject@CDWordArray@@SGPAVCObject@@XZ 5f88f750 f   array_d.obj
 0001:0008e7be       ?_GetBaseClass@CDWordArray@@KGPAUCRuntimeClass@@XZ 5f88f7be f   array_d.obj
 0001:0008e7c8       ?GetRuntimeClass@CDWordArray@@UBEPAUCRuntimeClass@@XZ 5f88f7c8 f   array_d.obj
 0001:0008e7f6       ??5@YGAAVCArchive@@AAV0@AAPAVCDWordArray@@@Z 5f88f7f6 f   array_d.obj
 0001:0008e820       ?_GetBaseClass@CPtrArray@@KGPAUCRuntimeClass@@XZ 5f88f820 f   array_p.obj
 0001:0008e82a       ?GetRuntimeClass@CPtrArray@@UBEPAUCRuntimeClass@@XZ 5f88f82a f   array_p.obj
 0001:0008e840       ?CreateObject@CObArray@@SGPAVCObject@@XZ 5f88f840 f   array_o.obj
 0001:0008e8ae       ?_GetBaseClass@CObArray@@KGPAUCRuntimeClass@@XZ 5f88f8ae f   array_o.obj
 0001:0008e8b8       ?GetRuntimeClass@CObArray@@UBEPAUCRuntimeClass@@XZ 5f88f8b8 f   array_o.obj
 0001:0008e8e6       ??5@YGAAVCArchive@@AAV0@AAPAVCObArray@@@Z 5f88f8e6 f   array_o.obj
 0001:0008e910       ?CreateObject@CStringArray@@SGPAVCObject@@XZ 5f88f910 f   array_s.obj
 0001:0008e97e       ?_GetBaseClass@CStringArray@@KGPAUCRuntimeClass@@XZ 5f88f97e f   array_s.obj
 0001:0008e988       ?GetRuntimeClass@CStringArray@@UBEPAUCRuntimeClass@@XZ 5f88f988 f   array_s.obj
 0001:0008e9b6       ??5@YGAAVCArchive@@AAV0@AAPAVCStringArray@@@Z 5f88f9b6 f   array_s.obj
 0001:0008e9e0       ?_GetBaseClass@CUIntArray@@KGPAUCRuntimeClass@@XZ 5f88f9e0 f   array_u.obj
 0001:0008e9ea       ?GetRuntimeClass@CUIntArray@@UBEPAUCRuntimeClass@@XZ 5f88f9ea f   array_u.obj
 0001:0008ea00       ?CreateObject@CWordArray@@SGPAVCObject@@XZ 5f88fa00 f   array_w.obj
 0001:0008ea6e       ?_GetBaseClass@CWordArray@@KGPAUCRuntimeClass@@XZ 5f88fa6e f   array_w.obj
 0001:0008ea78       ?GetRuntimeClass@CWordArray@@UBEPAUCRuntimeClass@@XZ 5f88fa78 f   array_w.obj
 0001:0008eaa6       ??5@YGAAVCArchive@@AAV0@AAPAVCWordArray@@@Z 5f88faa6 f   array_w.obj
 0001:0008ead0       ?CreateObject@CObList@@SGPAVCObject@@XZ 5f88fad0 f   list_o.obj
 0001:0008eb40       ?_GetBaseClass@CObList@@KGPAUCRuntimeClass@@XZ 5f88fb40 f   list_o.obj
 0001:0008eb4a       ?GetRuntimeClass@CObList@@UBEPAUCRuntimeClass@@XZ 5f88fb4a f   list_o.obj
 0001:0008eb78       ??5@YGAAVCArchive@@AAV0@AAPAVCObList@@@Z 5f88fb78 f   list_o.obj
 0001:0008eba0       ?_GetBaseClass@CPtrList@@KGPAUCRuntimeClass@@XZ 5f88fba0 f   list_p.obj
 0001:0008ebaa       ?GetRuntimeClass@CPtrList@@UBEPAUCRuntimeClass@@XZ 5f88fbaa f   list_p.obj
 0001:0008ebc0       ?CreateObject@CStringList@@SGPAVCObject@@XZ 5f88fbc0 f   list_s.obj
 0001:0008ec30       ?_GetBaseClass@CStringList@@KGPAUCRuntimeClass@@XZ 5f88fc30 f   list_s.obj
 0001:0008ec3a       ?GetRuntimeClass@CStringList@@UBEPAUCRuntimeClass@@XZ 5f88fc3a f   list_s.obj
 0001:0008ec68       ??5@YGAAVCArchive@@AAV0@AAPAVCStringList@@@Z 5f88fc68 f   list_s.obj
 0001:0008ec90       ?_GetBaseClass@CMapPtrToPtr@@KGPAUCRuntimeClass@@XZ 5f88fc90 f   map_pp.obj
 0001:0008ec9a       ?GetRuntimeClass@CMapPtrToPtr@@UBEPAUCRuntimeClass@@XZ 5f88fc9a f   map_pp.obj
 0001:0008ecb0       ?_GetBaseClass@CMapPtrToWord@@KGPAUCRuntimeClass@@XZ 5f88fcb0 f   map_pw.obj
 0001:0008ecba       ?GetRuntimeClass@CMapPtrToWord@@UBEPAUCRuntimeClass@@XZ 5f88fcba f   map_pw.obj
 0001:0008ecd0       ?CreateObject@CMapStringToOb@@SGPAVCObject@@XZ 5f88fcd0 f   map_so.obj
 0001:0008ed40       ?_GetBaseClass@CMapStringToOb@@KGPAUCRuntimeClass@@XZ 5f88fd40 f   map_so.obj
 0001:0008ed4a       ?GetRuntimeClass@CMapStringToOb@@UBEPAUCRuntimeClass@@XZ 5f88fd4a f   map_so.obj
 0001:0008ed78       ??5@YGAAVCArchive@@AAV0@AAPAVCMapStringToOb@@@Z 5f88fd78 f   map_so.obj
 0001:0008eda0       ?_GetBaseClass@CMapStringToPtr@@KGPAUCRuntimeClass@@XZ 5f88fda0 f   map_sp.obj
 0001:0008edaa       ?GetRuntimeClass@CMapStringToPtr@@UBEPAUCRuntimeClass@@XZ 5f88fdaa f   map_sp.obj
 0001:0008edc0       ?CreateObject@CMapStringToString@@SGPAVCObject@@XZ 5f88fdc0 f   map_ss.obj
 0001:0008ee30       ?_GetBaseClass@CMapStringToString@@KGPAUCRuntimeClass@@XZ 5f88fe30 f   map_ss.obj
 0001:0008ee3a       ?GetRuntimeClass@CMapStringToString@@UBEPAUCRuntimeClass@@XZ 5f88fe3a f   map_ss.obj
 0001:0008ee68       ??5@YGAAVCArchive@@AAV0@AAPAVCMapStringToString@@@Z 5f88fe68 f   map_ss.obj
 0001:0008ee90       ?CreateObject@CMapWordToOb@@SGPAVCObject@@XZ 5f88fe90 f   map_wo.obj
 0001:0008ef00       ?_GetBaseClass@CMapWordToOb@@KGPAUCRuntimeClass@@XZ 5f88ff00 f   map_wo.obj
 0001:0008ef0a       ?GetRuntimeClass@CMapWordToOb@@UBEPAUCRuntimeClass@@XZ 5f88ff0a f   map_wo.obj
 0001:0008ef38       ??5@YGAAVCArchive@@AAV0@AAPAVCMapWordToOb@@@Z 5f88ff38 f   map_wo.obj
 0001:0008ef60       ?_GetBaseClass@CMapWordToPtr@@KGPAUCRuntimeClass@@XZ 5f88ff60 f   map_wp.obj
 0001:0008ef6a       ?GetRuntimeClass@CMapWordToPtr@@UBEPAUCRuntimeClass@@XZ 5f88ff6a f   map_wp.obj
 0001:0008ef80       ?AfxSetModuleState@@YGPAVAFX_MODULE_STATE@@PAV1@@Z 5f88ff80 f   afxstate.obj
 0001:0008efae       ??1AFX_MAINTAIN_STATE@@QAE@XZ 5f88ffae f   afxstate.obj
 0001:0008efd3       ??0AFX_MAINTAIN_STATE2@@QAE@PAVAFX_MODULE_STATE@@@Z 5f88ffd3 f   afxstate.obj
 0001:0008f00d       ??0_AFX_THREAD_STATE@@QAE@XZ 5f89000d f   afxstate.obj
 0001:0008f046       ??1_AFX_THREAD_STATE@@UAE@XZ 5f890046 f   afxstate.obj
 0001:0008f153       ?AfxGetThreadState@@YGPAV_AFX_THREAD_STATE@@XZ 5f890153 f   afxstate.obj
 0001:0008f197       ??0AFX_MODULE_STATE@@QAE@HP6GJPAUHWND__@@IIJ@ZKH@Z 5f890197 f   afxstate.obj
 0001:0008f2a9       ??0AFX_MODULE_STATE@@QAE@HP6GJPAUHWND__@@IIJ@ZK@Z 5f8902a9 f   afxstate.obj
 0001:0008f38f       ??1AFX_MODULE_STATE@@UAE@XZ 5f89038f f   afxstate.obj
 0001:0008f47a       ?RemoveAll@CTypeLibCacheMap@@UAEXPAX@Z 5f89047a f   afxstate.obj
 0001:0008f4ca       ??0AFX_MODULE_THREAD_STATE@@QAE@XZ 5f8904ca f   afxstate.obj
 0001:0008f567       ??1AFX_MODULE_THREAD_STATE@@UAE@XZ 5f890567 f   afxstate.obj
 0001:0008f733       ?AfxWndProcBase@@YGJPAUHWND__@@IIJ@Z 5f890733 f   afxstate.obj
 0001:0008f7a2       ?AfxGetAppModuleState@@YGPAVAFX_MODULE_STATE@@XZ 5f8907a2 f   afxstate.obj
 0001:0008f7b1       ?AfxGetModuleState@@YGPAVAFX_MODULE_STATE@@XZ 5f8907b1 f   afxstate.obj
 0001:0008f812       ?AfxGetModuleThreadState@@YGPAVAFX_MODULE_THREAD_STATE@@XZ 5f890812 f   afxstate.obj
 0001:0008f829       ?Unlock@CTypeLibCache@@QAEXXZ 5f890829 f   afxstate.obj
 0001:0008f8c0       ??_E_AFX_THREAD_STATE@@UAEPAXI@Z 5f8908c0 f i afxstate.obj
 0001:0008f8c0       ??_G_AFX_THREAD_STATE@@UAEPAXI@Z 5f8908c0 f i afxstate.obj
 0001:0008f8f0       ??_EAFX_MODULE_STATE@@UAEPAXI@Z 5f8908f0 f i afxstate.obj
 0001:0008f8f0       ??_GAFX_MODULE_STATE@@UAEPAXI@Z 5f8908f0 f i afxstate.obj
 0001:0008f920       ??1?$CThreadLocal@V_AFX_THREAD_STATE@@@@QAE@XZ 5f890920 f i afxstate.obj
 0001:0008f920       ??1?$CThreadLocal@VAFX_MODULE_THREAD_STATE@@@@QAE@XZ 5f890920 f i afxstate.obj
 0001:0008f920       ??1?$CThreadLocal@V_AFX_CTL3D_THREAD@@@@QAE@XZ 5f890920 f i afxstate.obj
 0001:0008f940       ??_EAFX_MODULE_THREAD_STATE@@UAEPAXI@Z 5f890940 f i afxstate.obj
 0001:0008f940       ??_GAFX_MODULE_THREAD_STATE@@UAEPAXI@Z 5f890940 f i afxstate.obj
 0001:0008f970       ??0?$CEmbeddedButActsLikePtr@VCMapPtrToPtr@@@@QAE@XZ 5f890970 f i afxstate.obj
 0001:0008f990       ??1?$CEmbeddedButActsLikePtr@VCMapPtrToPtr@@@@QAE@XZ 5f890990 f i afxstate.obj
 0001:0008f9b0       ??0?$CEmbeddedButActsLikePtr@VCPtrList@@@@QAE@XZ 5f8909b0 f i afxstate.obj
 0001:0008f9d0       ??1?$CEmbeddedButActsLikePtr@VCPtrList@@@@QAE@XZ 5f8909d0 f i afxstate.obj
 0001:0008f9f0       ??_GCHandleMap@@QAEPAXI@Z  5f8909f0 f i afxstate.obj
 0001:0008fa20       ??0?$CTypedSimpleList@PAVCDynLinkLibrary@@@@QAE@H@Z 5f890a20 f i afxstate.obj
 0001:0008fa20       ??0?$CTypedSimpleList@PAUCThreadData@@@@QAE@H@Z 5f890a20 f i afxstate.obj
 0001:0008fa20       ??0?$CTypedSimpleList@PAVCOleControlLock@@@@QAE@H@Z 5f890a20 f i afxstate.obj
 0001:0008fa20       ??0?$CTypedSimpleList@PAVCOleObjectFactory@@@@QAE@H@Z 5f890a20 f i afxstate.obj
 0001:0008fa20       ??0?$CTypedSimpleList@PAVCFrameWnd@@@@QAE@H@Z 5f890a20 f i afxstate.obj
 0001:0008fa20       ??0?$CTypedSimpleList@PAUCRuntimeClass@@@@QAE@H@Z 5f890a20 f i afxstate.obj
 0001:0008fa40       ??C?$CEmbeddedButActsLikePtr@VCPtrList@@@@QAEPAVCPtrList@@XZ 5f890a40 f i afxstate.obj
 0001:0008fa40       ??B?$CEmbeddedButActsLikePtr@VCPtrList@@@@QAEPAVCPtrList@@XZ 5f890a40 f i afxstate.obj
 0001:0008fa50       ?GetData@?$CThreadLocal@VAFX_MODULE_THREAD_STATE@@@@QAEPAVAFX_MODULE_THREAD_STATE@@XZ 5f890a50 f i afxstate.obj
 0001:0008faa0       ?GetData@?$CProcessLocal@V_AFX_BASE_MODULE_STATE@@@@QAEPAV_AFX_BASE_MODULE_STATE@@XZ 5f890aa0 f i afxstate.obj
 0001:0008faf0       ?CreateObject@?$CThreadLocal@VAFX_MODULE_THREAD_STATE@@@@SGPAVCNoTrackObject@@XZ 5f890af0 f i afxstate.obj
 0001:0008fb60       ?CreateObject@?$CProcessLocal@V_AFX_BASE_MODULE_STATE@@@@SGPAVCNoTrackObject@@XZ 5f890b60 f i afxstate.obj
 0001:0008fbd0       ??0_AFX_BASE_MODULE_STATE@@QAE@XZ 5f890bd0 f i afxstate.obj
 0001:0008fc00       ??_E_AFX_BASE_MODULE_STATE@@UAEPAXI@Z 5f890c00 f i afxstate.obj
 0001:0008fc00       ??_G_AFX_BASE_MODULE_STATE@@UAEPAXI@Z 5f890c00 f i afxstate.obj
 0001:0008fc30       ??1_AFX_BASE_MODULE_STATE@@UAE@XZ 5f890c30 f i afxstate.obj
 0001:0008fc50       ?AddHead@CSimpleList@@QAEXPAX@Z 5f890c50 f   afxtls.obj
 0001:0008fcc3       ?Remove@CSimpleList@@QAEHPAX@Z 5f890cc3 f   afxtls.obj
 0001:0008fdb7       ??2CNoTrackObject@@SGPAXIPBDH@Z 5f890db7 f   afxtls.obj
 0001:0008fdc7       ??3CNoTrackObject@@SGXPAXPBDH@Z 5f890dc7 f   afxtls.obj
 0001:0008fdde       ??2CNoTrackObject@@SGPAXI@Z 5f890dde f   afxtls.obj
 0001:0008fe05       ??3CNoTrackObject@@SGXPAX@Z 5f890e05 f   afxtls.obj
 0001:0008fe1c       ??0CThreadSlotData@@QAE@XZ 5f890e1c f   afxtls.obj
 0001:0008fe91       ??1CThreadSlotData@@QAE@XZ 5f890e91 f   afxtls.obj
 0001:0008ff32       ?AllocSlot@CThreadSlotData@@QAEHXZ 5f890f32 f   afxtls.obj
 0001:00090127       ?FreeSlot@CThreadSlotData@@QAEXH@Z 5f891127 f   afxtls.obj
 0001:00090259       ?SetValue@CThreadSlotData@@QAEXHPAX@Z 5f891259 f   afxtls.obj
 0001:00090498       ?AssignInstance@CThreadSlotData@@QAEXPAUHINSTANCE__@@@Z 5f891498 f   afxtls.obj
 0001:0009055c       ?DeleteValues@CThreadSlotData@@QAEXPAUCThreadData@@PAUHINSTANCE__@@@Z 5f89155c f   afxtls.obj
 0001:000906a1       ?DeleteValues@CThreadSlotData@@QAEXPAUHINSTANCE__@@H@Z 5f8916a1 f   afxtls.obj
 0001:0009072c       ?GetData@CThreadLocalObject@@QAEPAVCNoTrackObject@@P6GPAV2@XZ@Z 5f89172c f   afxtls.obj
 0001:00090845       ?GetDataNA@CThreadLocalObject@@QAEPAVCNoTrackObject@@XZ 5f891845 f   afxtls.obj
 0001:0009087e       ??1CThreadLocalObject@@QAE@XZ 5f89187e f   afxtls.obj
 0001:000908b4       ?GetData@CProcessLocalObject@@QAEPAVCNoTrackObject@@P6GPAV2@XZ@Z 5f8918b4 f   afxtls.obj
 0001:00090968       ??1CProcessLocalObject@@QAE@XZ 5f891968 f   afxtls.obj
 0001:000909af       ?AfxInitLocalData@@YGXPAUHINSTANCE__@@@Z 5f8919af f   afxtls.obj
 0001:000909ce       ?AfxTermLocalData@@YGXPAUHINSTANCE__@@H@Z 5f8919ce f   afxtls.obj
 0001:000909f1       ?AfxTlsAddRef@@YGXXZ       5f8919f1 f   afxtls.obj
 0001:00090a03       ?AfxTlsRelease@@YGXXZ      5f891a03 f   afxtls.obj
 0001:00090a50       ??0CThreadData@@QAE@XZ     5f891a50 f i afxtls.obj
 0001:00090a70       ??_GCThreadData@@UAEPAXI@Z 5f891a70 f i afxtls.obj
 0001:00090a70       ??_ECThreadData@@UAEPAXI@Z 5f891a70 f i afxtls.obj
 0001:00090aa0       ??1CThreadData@@UAE@XZ     5f891aa0 f i afxtls.obj
 0001:00090ac0       ?GetThreadValue@CThreadSlotData@@QAEPAXH@Z 5f891ac0 f i afxtls.obj
 0001:00090bb0       ??_GCThreadSlotData@@QAEPAXI@Z 5f891bb0 f i afxtls.obj
 0001:00090be0       ??B?$CTypedSimpleList@PAUCThreadData@@@@QAEPAUCThreadData@@XZ 5f891be0 f i afxtls.obj
 0001:00090be0       ??B?$CTypedSimpleList@PAVCFrameWnd@@@@QAEPAVCFrameWnd@@XZ 5f891be0 f i afxtls.obj
 0001:00090c00       ?_GetBaseClass@CCriticalSection@@KGPAUCRuntimeClass@@XZ 5f891c00 f   mtcore.obj
 0001:00090c0a       ?GetRuntimeClass@CCriticalSection@@UBEPAUCRuntimeClass@@XZ 5f891c0a f   mtcore.obj
 0001:00090c1a       ?_GetBaseClass@CSyncObject@@KGPAUCRuntimeClass@@XZ 5f891c1a f   mtcore.obj
 0001:00090c24       ?GetRuntimeClass@CSyncObject@@UBEPAUCRuntimeClass@@XZ 5f891c24 f   mtcore.obj
 0001:00090c40       ?_GetBaseClass@CEvent@@KGPAUCRuntimeClass@@XZ 5f891c40 f   mtex.obj
 0001:00090c4a       ?GetRuntimeClass@CEvent@@UBEPAUCRuntimeClass@@XZ 5f891c4a f   mtex.obj
 0001:00090c5a       ?_GetBaseClass@CSemaphore@@KGPAUCRuntimeClass@@XZ 5f891c5a f   mtex.obj
 0001:00090c64       ?GetRuntimeClass@CSemaphore@@UBEPAUCRuntimeClass@@XZ 5f891c64 f   mtex.obj
 0001:00090c74       ?_GetBaseClass@CMutex@@KGPAUCRuntimeClass@@XZ 5f891c74 f   mtex.obj
 0001:00090c7e       ?GetRuntimeClass@CMutex@@UBEPAUCRuntimeClass@@XZ 5f891c7e f   mtex.obj
 0001:00090c90       ?CreateObject@CWnd@@SGPAVCObject@@XZ 5f891c90 f   wincore.obj
 0001:00090cfe       ?_GetBaseClass@CWnd@@KGPAUCRuntimeClass@@XZ 5f891cfe f   wincore.obj
 0001:00090d08       ?GetRuntimeClass@CWnd@@UBEPAUCRuntimeClass@@XZ 5f891d08 f   wincore.obj
 0001:00090d18       ?CreateObject@CTempWnd@@SGPAVCObject@@XZ 5f891d18 f   wincore.obj
 0001:00090d86       ?_GetBaseClass@CTempWnd@@KGPAUCRuntimeClass@@XZ 5f891d86 f   wincore.obj
 0001:00090d90       ?GetRuntimeClass@CTempWnd@@UBEPAUCRuntimeClass@@XZ 5f891d90 f   wincore.obj
 0001:00090da0       ??0CTempWnd@@QAE@XZ        5f891da0 f i wincore.obj
 0001:00090dc0       ??_GCTempWnd@@UAEPAXI@Z    5f891dc0 f i wincore.obj
 0001:00090dc0       ??_ECTempWnd@@UAEPAXI@Z    5f891dc0 f i wincore.obj
 0001:00090df0       ??1CTempWnd@@UAE@XZ        5f891df0 f i wincore.obj
 0001:00090e10       ??B?$CProcessLocal@V_AFX_WIN_STATE@@@@QAEPAV_AFX_WIN_STATE@@XZ 5f891e10 f i wincore.obj
 0001:00090e30       ?GetDataNA@?$CProcessLocal@V_AFX_CTL3D_STATE@@@@QAEPAV_AFX_CTL3D_STATE@@XZ 5f891e30 f i wincore.obj
 0001:00090e40       ??B?$CProcessLocal@V_AFX_CTL3D_STATE@@@@QAEPAV_AFX_CTL3D_STATE@@XZ 5f891e40 f i wincore.obj
 0001:00090e60       ?GetData@?$CProcessLocal@V_AFX_WIN_STATE@@@@QAEPAV_AFX_WIN_STATE@@XZ 5f891e60 f i wincore.obj
 0001:00090eb0       ?GetData@?$CProcessLocal@V_AFX_CTL3D_STATE@@@@QAEPAV_AFX_CTL3D_STATE@@XZ 5f891eb0 f i wincore.obj
 0001:00090f00       ?CreateObject@?$CProcessLocal@V_AFX_WIN_STATE@@@@SGPAVCNoTrackObject@@XZ 5f891f00 f i wincore.obj
 0001:00090f70       ?CreateObject@?$CProcessLocal@V_AFX_CTL3D_STATE@@@@SGPAVCNoTrackObject@@XZ 5f891f70 f i wincore.obj
 0001:00090fe0       ??0_AFX_CTL3D_STATE@@QAE@XZ 5f891fe0 f i wincore.obj
 0001:00091000       ??_E_AFX_CTL3D_STATE@@UAEPAXI@Z 5f892000 f i wincore.obj
 0001:00091000       ??_G_AFX_CTL3D_STATE@@UAEPAXI@Z 5f892000 f i wincore.obj
 0001:00091030       ?CreateObject@CFrameWnd@@SGPAVCObject@@XZ 5f892030 f   winfrm.obj
 0001:000910a1       ?_GetBaseClass@CFrameWnd@@KGPAUCRuntimeClass@@XZ 5f8920a1 f   winfrm.obj
 0001:000910ab       ?GetRuntimeClass@CFrameWnd@@UBEPAUCRuntimeClass@@XZ 5f8920ab f   winfrm.obj
 0001:000910bb       ?_GetBaseClass@CView@@KGPAUCRuntimeClass@@XZ 5f8920bb f   winfrm.obj
 0001:000910c5       ?GetRuntimeClass@CView@@UBEPAUCRuntimeClass@@XZ 5f8920c5 f   winfrm.obj
 0001:000910d5       ?_GetBaseClass@CControlBar@@KGPAUCRuntimeClass@@XZ 5f8920d5 f   winfrm.obj
 0001:000910df       ?GetRuntimeClass@CControlBar@@UBEPAUCRuntimeClass@@XZ 5f8920df f   winfrm.obj
 0001:000910f0       ?AddHead@?$CTypedSimpleList@PAUCThreadData@@@@QAEXPAUCThreadData@@@Z 5f8920f0 f i winfrm.obj
 0001:000910f0       ?AddHead@?$CTypedSimpleList@PAVCFrameWnd@@@@QAEXPAVCFrameWnd@@@Z 5f8920f0 f i winfrm.obj
 0001:00091110       ?Remove@?$CTypedSimpleList@PAUCThreadData@@@@QAEHPAUCThreadData@@@Z 5f892110 f i winfrm.obj
 0001:00091110       ?Remove@?$CTypedSimpleList@PAVCFrameWnd@@@@QAEHPAVCFrameWnd@@@Z 5f892110 f i winfrm.obj
 0001:00091130       ??B?$CThreadLocal@VAFX_MODULE_THREAD_STATE@@@@QAEPAVAFX_MODULE_THREAD_STATE@@XZ 5f892130 f i winfrm.obj
 0001:00091150       ?CreateObject@CMDIFrameWnd@@SGPAVCObject@@XZ 5f892150 f   winmdi.obj
 0001:000911b7       ?_GetBaseClass@CMDIFrameWnd@@KGPAUCRuntimeClass@@XZ 5f8921b7 f   winmdi.obj
 0001:000911c1       ?GetRuntimeClass@CMDIFrameWnd@@UBEPAUCRuntimeClass@@XZ 5f8921c1 f   winmdi.obj
 0001:000911d1       ?CreateObject@CMDIChildWnd@@SGPAVCObject@@XZ 5f8921d1 f   winmdi.obj
 0001:00091238       ?_GetBaseClass@CMDIChildWnd@@KGPAUCRuntimeClass@@XZ 5f892238 f   winmdi.obj
 0001:00091242       ?GetRuntimeClass@CMDIChildWnd@@UBEPAUCRuntimeClass@@XZ 5f892242 f   winmdi.obj
 0001:00091260       ?_GetBaseClass@CToolTipCtrl@@KGPAUCRuntimeClass@@XZ 5f892260 f   tooltip.obj
 0001:0009126a       ?GetRuntimeClass@CToolTipCtrl@@UBEPAUCRuntimeClass@@XZ 5f89226a f   tooltip.obj
 0001:00091280       ?CreateObject@CMiniFrameWnd@@SGPAVCObject@@XZ 5f892280 f   winmini.obj
 0001:000912f1       ?_GetBaseClass@CMiniFrameWnd@@KGPAUCRuntimeClass@@XZ 5f8922f1 f   winmini.obj
 0001:000912fb       ?GetRuntimeClass@CMiniFrameWnd@@UBEPAUCRuntimeClass@@XZ 5f8922fb f   winmini.obj
 0001:00091310       ??0CControlBar@@IAE@XZ     5f892310 f   barcore.obj
 0001:000913cf       ?SetBorders@CControlBar@@QAEXHHHH@Z 5f8923cf f   barcore.obj
 0001:0009147a       ?PreCreateWindow@CControlBar@@UAEHAAUtagCREATESTRUCTW@@@Z 5f89247a f   barcore.obj
 0001:0009156a       ?SetBarStyle@CControlBar@@QAEXK@Z 5f89256a f   barcore.obj
 0001:000915e8       ?OnBarStyleChange@CControlBar@@UAEXKK@Z 5f8925e8 f   barcore.obj
 0001:000915f5       ?AllocElements@CControlBar@@QAEHHH@Z 5f8925f5 f   barcore.obj
 0001:000916f0       ??_ECControlBar@@UAEPAXI@Z 5f8926f0 f i barcore.obj
 0001:000916f0       ??_GCControlBar@@UAEPAXI@Z 5f8926f0 f i barcore.obj
 0001:00091720       ?_AfxGetComCtlVersion@@YGKXZ 5f892720 f   bartool.obj
 0001:00091826       ?_AfxGetDropDownWidth@@YGHXZ 5f892826 f   bartool.obj
 0001:00091940       ??0CToolBar@@QAE@XZ        5f892940 f   bartool.obj
 0001:00091a2e       ??1CToolBar@@UAE@XZ        5f892a2e f   bartool.obj
 0001:00091ac3       ?Create@CToolBar@@QAEHPAVCWnd@@KI@Z 5f892ac3 f   bartool.obj
 0001:00091b27       ?CreateEx@CToolBar@@QAEHPAVCWnd@@KKVCRect@@I@Z 5f892b27 f   bartool.obj
 0001:00091cca       ?OnNcCreate@CToolBar@@IAEHPAUtagCREATESTRUCTW@@@Z 5f892cca f   bartool.obj
 0001:00091d2c       ?SetOwner@CToolBar@@QAEXPAVCWnd@@@Z 5f892d2c f   bartool.obj
 0001:00091db0       ?SetSizes@CToolBar@@QAEXUtagSIZE@@0@Z 5f892db0 f   bartool.obj
 0001:00091f61       ?SetHeight@CToolBar@@QAEXH@Z 5f892f61 f   bartool.obj
 0001:00092042       ?LoadToolBar@CToolBar@@QAEHPBG@Z 5f893042 f   bartool.obj
 0001:00092245       ?LoadBitmapW@CToolBar@@QAEHPBG@Z 5f893245 f   bartool.obj
 0001:000922f8       ?SetBitmap@CToolBar@@QAEHPAUHBITMAP__@@@Z 5f8932f8 f   bartool.obj
 0001:00092361       ?AddReplaceBitmap@CToolBar@@QAEHPAUHBITMAP__@@@Z 5f893361 f   bartool.obj
 0001:0009245b       ?SetButtons@CToolBar@@QAEHPBIH@Z 5f89345b f   bartool.obj
 0001:000926c7       ?_GetBaseClass@CToolBar@@KGPAUCRuntimeClass@@XZ 5f8936c7 f   bartool.obj
 0001:000926d1       ?GetRuntimeClass@CToolBar@@UBEPAUCRuntimeClass@@XZ 5f8936d1 f   bartool.obj
 0001:000926f0       ?items@CToolBarData@@QAEPAGXZ 5f8936f0 f i bartool.obj
 0001:00092710       ?_GetBaseClass@CDialogBar@@KGPAUCRuntimeClass@@XZ 5f893710 f   bardlg.obj
 0001:0009271a       ?GetRuntimeClass@CDialogBar@@UBEPAUCRuntimeClass@@XZ 5f89371a f   bardlg.obj
 0001:00092730       ??0CStatusBar@@QAE@XZ      5f893730 f   barstat.obj
 0001:000927aa       ??1CStatusBar@@UAE@XZ      5f8937aa f   barstat.obj
 0001:000927ff       ?Create@CStatusBar@@QAEHPAVCWnd@@KI@Z 5f8937ff f   barstat.obj
 0001:00092822       ?CreateEx@CStatusBar@@QAEHPAVCWnd@@KKI@Z 5f893822 f   barstat.obj
 0001:000928e3       ?PreCreateWindow@CStatusBar@@UAEHAAUtagCREATESTRUCTW@@@Z 5f8938e3 f   barstat.obj
 0001:0009292a       ?SetIndicators@CStatusBar@@QAEHPBIH@Z 5f89392a f   barstat.obj
 0001:00092bd0       ?AllocElements@CStatusBar@@QAEHHH@Z 5f893bd0 f   barstat.obj
 0001:00092c8a       ?CalcInsideRect@CStatusBar@@QBEXAAVCRect@@H@Z 5f893c8a f   barstat.obj
 0001:00092d7b       ?UpdateAllPanes@CStatusBar@@IAEXHH@Z 5f893d7b f   barstat.obj
 0001:00093044       ?_GetBaseClass@CStatusBar@@KGPAUCRuntimeClass@@XZ 5f894044 f   barstat.obj
 0001:0009304e       ?GetRuntimeClass@CStatusBar@@UBEPAUCRuntimeClass@@XZ 5f89404e f   barstat.obj
 0001:00093060       ?_GetBaseClass@CDockBar@@KGPAUCRuntimeClass@@XZ 5f894060 f   bardock.obj
 0001:0009306a       ?GetRuntimeClass@CDockBar@@UBEPAUCRuntimeClass@@XZ 5f89406a f   bardock.obj
 0001:0009307a       ?CreateObject@CMiniDockFrameWnd@@SGPAVCObject@@XZ 5f89407a f   bardock.obj
 0001:000930eb       ?_GetBaseClass@CMiniDockFrameWnd@@KGPAUCRuntimeClass@@XZ 5f8940eb f   bardock.obj
 0001:000930f5       ?GetRuntimeClass@CMiniDockFrameWnd@@UBEPAUCRuntimeClass@@XZ 5f8940f5 f   bardock.obj
 0001:00093110       ?CreateObject@CDockState@@SGPAVCObject@@XZ 5f894110 f   dockstat.obj
 0001:0009317e       ?_GetBaseClass@CDockState@@KGPAUCRuntimeClass@@XZ 5f89417e f   dockstat.obj
 0001:00093188       ?GetRuntimeClass@CDockState@@UBEPAUCRuntimeClass@@XZ 5f894188 f   dockstat.obj
 0001:000931b6       ??5@YGAAVCArchive@@AAV0@AAPAVCDockState@@@Z 5f8941b6 f   dockstat.obj
 0001:000931e0       ?_GetBaseClass@CPreviewDC@@KGPAUCRuntimeClass@@XZ 5f8941e0 f   dcprev.obj
 0001:000931ea       ?GetRuntimeClass@CPreviewDC@@UBEPAUCRuntimeClass@@XZ 5f8941ea f   dcprev.obj
 0001:00093200       ?_GetBaseClass@CMetaFileDC@@KGPAUCRuntimeClass@@XZ 5f894200 f   dcmeta.obj
 0001:0009320a       ?GetRuntimeClass@CMetaFileDC@@UBEPAUCRuntimeClass@@XZ 5f89420a f   dcmeta.obj
 0001:00093220       ?_GetBaseClass@CReBar@@KGPAUCRuntimeClass@@XZ 5f894220 f   barcool.obj
 0001:0009322a       ?GetRuntimeClass@CReBar@@UBEPAUCRuntimeClass@@XZ 5f89422a f   barcool.obj
 0001:00093240       ?_GetBaseClass@CStatic@@KGPAUCRuntimeClass@@XZ 5f894240 f   winctrl1.obj
 0001:0009324a       ?GetRuntimeClass@CStatic@@UBEPAUCRuntimeClass@@XZ 5f89424a f   winctrl1.obj
 0001:0009325a       ?_GetBaseClass@CButton@@KGPAUCRuntimeClass@@XZ 5f89425a f   winctrl1.obj
 0001:00093264       ?GetRuntimeClass@CButton@@UBEPAUCRuntimeClass@@XZ 5f894264 f   winctrl1.obj
 0001:00093274       ?_GetBaseClass@CListBox@@KGPAUCRuntimeClass@@XZ 5f894274 f   winctrl1.obj
 0001:0009327e       ?GetRuntimeClass@CListBox@@UBEPAUCRuntimeClass@@XZ 5f89427e f   winctrl1.obj
 0001:0009328e       ?_GetBaseClass@CComboBox@@KGPAUCRuntimeClass@@XZ 5f89428e f   winctrl1.obj
 0001:00093298       ?GetRuntimeClass@CComboBox@@UBEPAUCRuntimeClass@@XZ 5f894298 f   winctrl1.obj
 0001:000932a8       ?_GetBaseClass@CEdit@@KGPAUCRuntimeClass@@XZ 5f8942a8 f   winctrl1.obj
 0001:000932b2       ?GetRuntimeClass@CEdit@@UBEPAUCRuntimeClass@@XZ 5f8942b2 f   winctrl1.obj
 0001:000932c2       ?_GetBaseClass@CScrollBar@@KGPAUCRuntimeClass@@XZ 5f8942c2 f   winctrl1.obj
 0001:000932cc       ?GetRuntimeClass@CScrollBar@@UBEPAUCRuntimeClass@@XZ 5f8942cc f   winctrl1.obj
 0001:000932e0       ?_GetBaseClass@CDragListBox@@KGPAUCRuntimeClass@@XZ 5f8942e0 f   winctrl2.obj
 0001:000932ea       ?GetRuntimeClass@CDragListBox@@UBEPAUCRuntimeClass@@XZ 5f8942ea f   winctrl2.obj
 0001:000932fa       ?_GetBaseClass@CSpinButtonCtrl@@KGPAUCRuntimeClass@@XZ 5f8942fa f   winctrl2.obj
 0001:00093304       ?GetRuntimeClass@CSpinButtonCtrl@@UBEPAUCRuntimeClass@@XZ 5f894304 f   winctrl2.obj
 0001:00093314       ?_GetBaseClass@CSliderCtrl@@KGPAUCRuntimeClass@@XZ 5f894314 f   winctrl2.obj
 0001:0009331e       ?GetRuntimeClass@CSliderCtrl@@UBEPAUCRuntimeClass@@XZ 5f89431e f   winctrl2.obj
 0001:0009332e       ?_GetBaseClass@CProgressCtrl@@KGPAUCRuntimeClass@@XZ 5f89432e f   winctrl2.obj
 0001:00093338       ?GetRuntimeClass@CProgressCtrl@@UBEPAUCRuntimeClass@@XZ 5f894338 f   winctrl2.obj
 0001:00093348       ?_GetBaseClass@CComboBoxEx@@KGPAUCRuntimeClass@@XZ 5f894348 f   winctrl2.obj
 0001:00093352       ?GetRuntimeClass@CComboBoxEx@@UBEPAUCRuntimeClass@@XZ 5f894352 f   winctrl2.obj
 0001:00093362       ?_GetBaseClass@CHeaderCtrl@@KGPAUCRuntimeClass@@XZ 5f894362 f   winctrl2.obj
 0001:0009336c       ?GetRuntimeClass@CHeaderCtrl@@UBEPAUCRuntimeClass@@XZ 5f89436c f   winctrl2.obj
 0001:0009337c       ?_GetBaseClass@CHotKeyCtrl@@KGPAUCRuntimeClass@@XZ 5f89437c f   winctrl2.obj
 0001:00093386       ?GetRuntimeClass@CHotKeyCtrl@@UBEPAUCRuntimeClass@@XZ 5f894386 f   winctrl2.obj
 0001:00093396       ?_GetBaseClass@CAnimateCtrl@@KGPAUCRuntimeClass@@XZ 5f894396 f   winctrl2.obj
 0001:000933a0       ?GetRuntimeClass@CAnimateCtrl@@UBEPAUCRuntimeClass@@XZ 5f8943a0 f   winctrl2.obj
 0001:000933b0       ?_GetBaseClass@CTabCtrl@@KGPAUCRuntimeClass@@XZ 5f8943b0 f   winctrl2.obj
 0001:000933ba       ?GetRuntimeClass@CTabCtrl@@UBEPAUCRuntimeClass@@XZ 5f8943ba f   winctrl2.obj
 0001:000933ca       ?_GetBaseClass@CTreeCtrl@@KGPAUCRuntimeClass@@XZ 5f8943ca f   winctrl2.obj
 0001:000933d4       ?GetRuntimeClass@CTreeCtrl@@UBEPAUCRuntimeClass@@XZ 5f8943d4 f   winctrl2.obj
 0001:000933e4       ?_GetBaseClass@CListCtrl@@KGPAUCRuntimeClass@@XZ 5f8943e4 f   winctrl2.obj
 0001:000933ee       ?GetRuntimeClass@CListCtrl@@UBEPAUCRuntimeClass@@XZ 5f8943ee f   winctrl2.obj
 0001:000933fe       ?_GetBaseClass@CToolBarCtrl@@KGPAUCRuntimeClass@@XZ 5f8943fe f   winctrl2.obj
 0001:00093408       ?GetRuntimeClass@CToolBarCtrl@@UBEPAUCRuntimeClass@@XZ 5f894408 f   winctrl2.obj
 0001:00093418       ?_GetBaseClass@CStatusBarCtrl@@KGPAUCRuntimeClass@@XZ 5f894418 f   winctrl2.obj
 0001:00093422       ?GetRuntimeClass@CStatusBarCtrl@@UBEPAUCRuntimeClass@@XZ 5f894422 f   winctrl2.obj
 0001:00093432       ?CreateObject@CImageList@@SGPAVCObject@@XZ 5f894432 f   winctrl2.obj
 0001:000934a0       ?_GetBaseClass@CImageList@@KGPAUCRuntimeClass@@XZ 5f8944a0 f   winctrl2.obj
 0001:000934aa       ?GetRuntimeClass@CImageList@@UBEPAUCRuntimeClass@@XZ 5f8944aa f   winctrl2.obj
 0001:000934ba       ?CreateObject@CTempImageList@@SGPAVCObject@@XZ 5f8944ba f   winctrl2.obj
 0001:00093528       ?_GetBaseClass@CTempImageList@@KGPAUCRuntimeClass@@XZ 5f894528 f   winctrl2.obj
 0001:00093532       ?GetRuntimeClass@CTempImageList@@UBEPAUCRuntimeClass@@XZ 5f894532 f   winctrl2.obj
 0001:00093542       ?_GetBaseClass@CRichEditCtrl@@KGPAUCRuntimeClass@@XZ 5f894542 f   winctrl2.obj
 0001:0009354c       ?GetRuntimeClass@CRichEditCtrl@@UBEPAUCRuntimeClass@@XZ 5f89454c f   winctrl2.obj
 0001:00093560       ??0CTempImageList@@QAE@XZ  5f894560 f i winctrl2.obj
 0001:00093580       ??_ECTempImageList@@UAEPAXI@Z 5f894580 f i winctrl2.obj
 0001:00093580       ??_GCTempImageList@@UAEPAXI@Z 5f894580 f i winctrl2.obj
 0001:000935b0       ??1CTempImageList@@UAE@XZ  5f8945b0 f i winctrl2.obj
 0001:000935d0       ?_GetBaseClass@CCheckListBox@@KGPAUCRuntimeClass@@XZ 5f8945d0 f   winctrl3.obj
 0001:000935da       ?GetRuntimeClass@CCheckListBox@@UBEPAUCRuntimeClass@@XZ 5f8945da f   winctrl3.obj
 0001:00093620       ??B?$CProcessLocal@V_AFX_CHECKLIST_STATE@@@@QAEPAV_AFX_CHECKLIST_STATE@@XZ 5f894620 f i winctrl3.obj
 0001:00093640       ?GetData@?$CProcessLocal@V_AFX_CHECKLIST_STATE@@@@QAEPAV_AFX_CHECKLIST_STATE@@XZ 5f894640 f i winctrl3.obj
 0001:00093690       ?CreateObject@?$CProcessLocal@V_AFX_CHECKLIST_STATE@@@@SGPAVCNoTrackObject@@XZ 5f894690 f i winctrl3.obj
 0001:00093700       ?_GetBaseClass@CBitmapButton@@KGPAUCRuntimeClass@@XZ 5f894700 f   winbtn.obj
 0001:0009370a       ?GetRuntimeClass@CBitmapButton@@UBEPAUCRuntimeClass@@XZ 5f89470a f   winbtn.obj
 0001:00093720       ?_GetBaseClass@CDialog@@KGPAUCRuntimeClass@@XZ 5f894720 f   dlgcore.obj
 0001:0009372a       ?GetRuntimeClass@CDialog@@UBEPAUCRuntimeClass@@XZ 5f89472a f   dlgcore.obj
 0001:00093740       ?_GetBaseClass@CPropertyPage@@KGPAUCRuntimeClass@@XZ 5f894740 f   dlgprop.obj
 0001:0009374a       ?GetRuntimeClass@CPropertyPage@@UBEPAUCRuntimeClass@@XZ 5f89474a f   dlgprop.obj
 0001:0009375a       ?_GetBaseClass@CPropertySheet@@KGPAUCRuntimeClass@@XZ 5f89475a f   dlgprop.obj
 0001:00093764       ?GetRuntimeClass@CPropertySheet@@UBEPAUCRuntimeClass@@XZ 5f894764 f   dlgprop.obj
 0001:00093774       ?_GetBaseClass@CPropertyPageEx@@KGPAUCRuntimeClass@@XZ 5f894774 f   dlgprop.obj
 0001:0009377e       ?GetRuntimeClass@CPropertyPageEx@@UBEPAUCRuntimeClass@@XZ 5f89477e f   dlgprop.obj
 0001:0009378e       ?_GetBaseClass@CPropertySheetEx@@KGPAUCRuntimeClass@@XZ 5f89478e f   dlgprop.obj
 0001:00093798       ?GetRuntimeClass@CPropertySheetEx@@UBEPAUCRuntimeClass@@XZ 5f894798 f   dlgprop.obj
 0001:000937b0       ?_GetBaseClass@CFileDialog@@KGPAUCRuntimeClass@@XZ 5f8947b0 f   dlgfile.obj
 0001:000937ba       ?GetRuntimeClass@CFileDialog@@UBEPAUCRuntimeClass@@XZ 5f8947ba f   dlgfile.obj
 0001:000937d0       ?_GetBaseClass@CPrintDialog@@KGPAUCRuntimeClass@@XZ 5f8947d0 f   dlgprnt.obj
 0001:000937da       ?GetRuntimeClass@CPrintDialog@@UBEPAUCRuntimeClass@@XZ 5f8947da f   dlgprnt.obj
 0001:000937ea       ?_GetBaseClass@CPageSetupDialog@@KGPAUCRuntimeClass@@XZ 5f8947ea f   dlgprnt.obj
 0001:000937f4       ?GetRuntimeClass@CPageSetupDialog@@UBEPAUCRuntimeClass@@XZ 5f8947f4 f   dlgprnt.obj
 0001:00093810       ?_GetBaseClass@CColorDialog@@KGPAUCRuntimeClass@@XZ 5f894810 f   dlgclr.obj
 0001:0009381a       ?GetRuntimeClass@CColorDialog@@UBEPAUCRuntimeClass@@XZ 5f89481a f   dlgclr.obj
 0001:00093860       ??1?$CProcessLocal@V_AFX_CHECKLIST_STATE@@@@QAE@XZ 5f894860 f i dlgclr.obj
 0001:00093860       ??1?$CProcessLocal@V_AFX_MAIL_STATE@@@@QAE@XZ 5f894860 f i dlgclr.obj
 0001:00093860       ??1?$CProcessLocal@U_AFX_PROPPAGEFONTINFO@@@@QAE@XZ 5f894860 f i dlgclr.obj
 0001:00093860       ??1?$CProcessLocal@V_AFX_WIN_STATE@@@@QAE@XZ 5f894860 f i dlgclr.obj
 0001:00093860       ??1?$CProcessLocal@V_AFX_EDIT_STATE@@@@QAE@XZ 5f894860 f i dlgclr.obj
 0001:00093860       ??1?$CProcessLocal@V_AFX_CTL3D_STATE@@@@QAE@XZ 5f894860 f i dlgclr.obj
 0001:00093860       ??1?$CProcessLocal@V_AFX_BASE_MODULE_STATE@@@@QAE@XZ 5f894860 f i dlgclr.obj
 0001:00093860       ??1?$CProcessLocal@V_AFX_COLOR_STATE@@@@QAE@XZ 5f894860 f i dlgclr.obj
 0001:00093880       ??C?$CProcessLocal@V_AFX_COLOR_STATE@@@@QAEPAV_AFX_COLOR_STATE@@XZ 5f894880 f i dlgclr.obj
 0001:000938a0       ?GetData@?$CProcessLocal@V_AFX_COLOR_STATE@@@@QAEPAV_AFX_COLOR_STATE@@XZ 5f8948a0 f i dlgclr.obj
 0001:000938f0       ?CreateObject@?$CProcessLocal@V_AFX_COLOR_STATE@@@@SGPAVCNoTrackObject@@XZ 5f8948f0 f i dlgclr.obj
 0001:00093960       ?_GetBaseClass@CFontDialog@@KGPAUCRuntimeClass@@XZ 5f894960 f   dlgfnt.obj
 0001:0009396a       ?GetRuntimeClass@CFontDialog@@UBEPAUCRuntimeClass@@XZ 5f89496a f   dlgfnt.obj
 0001:00093980       ?_GetBaseClass@CFindReplaceDialog@@KGPAUCRuntimeClass@@XZ 5f894980 f   dlgfr.obj
 0001:0009398a       ?GetRuntimeClass@CFindReplaceDialog@@UBEPAUCRuntimeClass@@XZ 5f89498a f   dlgfr.obj
 0001:000939d5       ?AfxGetPropSheetFont@@YGHAAVCString@@AAGH@Z 5f8949d5 f   ccdata.obj
 0001:00093b00       ?GetData@?$CProcessLocal@U_AFX_PROPPAGEFONTINFO@@@@QAEPAU_AFX_PROPPAGEFONTINFO@@XZ 5f894b00 f i ccdata.obj
 0001:00093b50       ?CreateObject@?$CProcessLocal@U_AFX_PROPPAGEFONTINFO@@@@SGPAVCNoTrackObject@@XZ 5f894b50 f i ccdata.obj
 0001:00093bc0       ??0_AFX_PROPPAGEFONTINFO@@QAE@XZ 5f894bc0 f i ccdata.obj
 0001:00093c00       ??_E_AFX_PROPPAGEFONTINFO@@UAEPAXI@Z 5f894c00 f i ccdata.obj
 0001:00093c00       ??_G_AFX_PROPPAGEFONTINFO@@UAEPAXI@Z 5f894c00 f i ccdata.obj
 0001:00093c30       ??1_AFX_PROPPAGEFONTINFO@@UAE@XZ 5f894c30 f i ccdata.obj
 0001:00093c60       ?_GetBaseClass@CIPAddressCtrl@@KGPAUCRuntimeClass@@XZ 5f894c60 f   winctrl6.obj
 0001:00093c6a       ?GetRuntimeClass@CIPAddressCtrl@@UBEPAUCRuntimeClass@@XZ 5f894c6a f   winctrl6.obj
 0001:00093c7a       ?_GetBaseClass@CReBarCtrl@@KGPAUCRuntimeClass@@XZ 5f894c7a f   winctrl6.obj
 0001:00093c84       ?GetRuntimeClass@CReBarCtrl@@UBEPAUCRuntimeClass@@XZ 5f894c84 f   winctrl6.obj
 0001:00093ca0       ?_GetBaseClass@CResourceException@@KGPAUCRuntimeClass@@XZ 5f894ca0 f   wingdi.obj
 0001:00093caa       ?GetRuntimeClass@CResourceException@@UBEPAUCRuntimeClass@@XZ 5f894caa f   wingdi.obj
 0001:00093d00       ?_GetBaseClass@CUserException@@KGPAUCRuntimeClass@@XZ 5f894d00 f   wingdi.obj
 0001:00093d0a       ?GetRuntimeClass@CUserException@@UBEPAUCRuntimeClass@@XZ 5f894d0a f   wingdi.obj
 0001:00093d60       ?CreateObject@CDC@@SGPAVCObject@@XZ 5f894d60 f   wingdi.obj
 0001:00093dc4       ?_GetBaseClass@CDC@@KGPAUCRuntimeClass@@XZ 5f894dc4 f   wingdi.obj
 0001:00093dce       ?GetRuntimeClass@CDC@@UBEPAUCRuntimeClass@@XZ 5f894dce f   wingdi.obj
 0001:00093dde       ?_GetBaseClass@CClientDC@@KGPAUCRuntimeClass@@XZ 5f894dde f   wingdi.obj
 0001:00093de8       ?GetRuntimeClass@CClientDC@@UBEPAUCRuntimeClass@@XZ 5f894de8 f   wingdi.obj
 0001:00093df8       ?_GetBaseClass@CWindowDC@@KGPAUCRuntimeClass@@XZ 5f894df8 f   wingdi.obj
 0001:00093e02       ?GetRuntimeClass@CWindowDC@@UBEPAUCRuntimeClass@@XZ 5f894e02 f   wingdi.obj
 0001:00093e12       ?_GetBaseClass@CPaintDC@@KGPAUCRuntimeClass@@XZ 5f894e12 f   wingdi.obj
 0001:00093e1c       ?GetRuntimeClass@CPaintDC@@UBEPAUCRuntimeClass@@XZ 5f894e1c f   wingdi.obj
 0001:00093e2c       ?CreateObject@CGdiObject@@SGPAVCObject@@XZ 5f894e2c f   wingdi.obj
 0001:00093e90       ?_GetBaseClass@CGdiObject@@KGPAUCRuntimeClass@@XZ 5f894e90 f   wingdi.obj
 0001:00093e9a       ?GetRuntimeClass@CGdiObject@@UBEPAUCRuntimeClass@@XZ 5f894e9a f   wingdi.obj
 0001:00093eaa       ?_GetBaseClass@CPen@@KGPAUCRuntimeClass@@XZ 5f894eaa f   wingdi.obj
 0001:00093eb4       ?GetRuntimeClass@CPen@@UBEPAUCRuntimeClass@@XZ 5f894eb4 f   wingdi.obj
 0001:00093ec4       ?_GetBaseClass@CBrush@@KGPAUCRuntimeClass@@XZ 5f894ec4 f   wingdi.obj
 0001:00093ece       ?GetRuntimeClass@CBrush@@UBEPAUCRuntimeClass@@XZ 5f894ece f   wingdi.obj
 0001:00093ede       ?_GetBaseClass@CFont@@KGPAUCRuntimeClass@@XZ 5f894ede f   wingdi.obj
 0001:00093ee8       ?GetRuntimeClass@CFont@@UBEPAUCRuntimeClass@@XZ 5f894ee8 f   wingdi.obj
 0001:00093ef8       ?_GetBaseClass@CBitmap@@KGPAUCRuntimeClass@@XZ 5f894ef8 f   wingdi.obj
 0001:00093f02       ?GetRuntimeClass@CBitmap@@UBEPAUCRuntimeClass@@XZ 5f894f02 f   wingdi.obj
 0001:00093f12       ?_GetBaseClass@CPalette@@KGPAUCRuntimeClass@@XZ 5f894f12 f   wingdi.obj
 0001:00093f1c       ?GetRuntimeClass@CPalette@@UBEPAUCRuntimeClass@@XZ 5f894f1c f   wingdi.obj
 0001:00093f2c       ?_GetBaseClass@CRgn@@KGPAUCRuntimeClass@@XZ 5f894f2c f   wingdi.obj
 0001:00093f36       ?GetRuntimeClass@CRgn@@UBEPAUCRuntimeClass@@XZ 5f894f36 f   wingdi.obj
 0001:00093f46       ?CreateObject@CTempDC@@SGPAVCObject@@XZ 5f894f46 f   wingdi.obj
 0001:00093faa       ?_GetBaseClass@CTempDC@@KGPAUCRuntimeClass@@XZ 5f894faa f   wingdi.obj
 0001:00093fb4       ?GetRuntimeClass@CTempDC@@UBEPAUCRuntimeClass@@XZ 5f894fb4 f   wingdi.obj
 0001:00093fc4       ?CreateObject@CTempGdiObject@@SGPAVCObject@@XZ 5f894fc4 f   wingdi.obj
 0001:00094028       ?_GetBaseClass@CTempGdiObject@@KGPAUCRuntimeClass@@XZ 5f895028 f   wingdi.obj
 0001:00094032       ?GetRuntimeClass@CTempGdiObject@@UBEPAUCRuntimeClass@@XZ 5f895032 f   wingdi.obj
 0001:00094050       ??0CTempDC@@QAE@XZ         5f895050 f i wingdi.obj
 0001:00094070       ??_ECTempDC@@UAEPAXI@Z     5f895070 f i wingdi.obj
 0001:00094070       ??_GCTempDC@@UAEPAXI@Z     5f895070 f i wingdi.obj
 0001:000940a0       ??1CTempDC@@UAE@XZ         5f8950a0 f i wingdi.obj
 0001:000940c0       ??0CTempGdiObject@@QAE@XZ  5f8950c0 f i wingdi.obj
 0001:000940e0       ??_ECTempGdiObject@@UAEPAXI@Z 5f8950e0 f i wingdi.obj
 0001:000940e0       ??_GCTempGdiObject@@UAEPAXI@Z 5f8950e0 f i wingdi.obj
 0001:00094110       ??1CTempGdiObject@@UAE@XZ  5f895110 f i wingdi.obj
 0001:00094130       ?CreateObject@CMenu@@SGPAVCObject@@XZ 5f895130 f   winmenu.obj
 0001:0009419e       ?_GetBaseClass@CMenu@@KGPAUCRuntimeClass@@XZ 5f89519e f   winmenu.obj
 0001:000941a8       ?GetRuntimeClass@CMenu@@UBEPAUCRuntimeClass@@XZ 5f8951a8 f   winmenu.obj
 0001:000941b8       ?CreateObject@CTempMenu@@SGPAVCObject@@XZ 5f8951b8 f   winmenu.obj
 0001:00094226       ?_GetBaseClass@CTempMenu@@KGPAUCRuntimeClass@@XZ 5f895226 f   winmenu.obj
 0001:00094230       ?GetRuntimeClass@CTempMenu@@UBEPAUCRuntimeClass@@XZ 5f895230 f   winmenu.obj
 0001:00094240       ??0CTempMenu@@QAE@XZ       5f895240 f i winmenu.obj
 0001:00094260       ??_GCTempMenu@@UAEPAXI@Z   5f895260 f i winmenu.obj
 0001:00094260       ??_ECTempMenu@@UAEPAXI@Z   5f895260 f i winmenu.obj
 0001:00094290       ??1CTempMenu@@UAE@XZ       5f895290 f i winmenu.obj
 0001:000942ef       ?AfxEnableWin40Compatibility@@YGXXZ 5f8952ef f   auxdata.obj
 0001:00094327       ?AfxEnableWin31Compatibility@@YGXXZ 5f895327 f   auxdata.obj
 0001:00094350       ??0AUX_DATA@@QAE@XZ        5f895350 f   auxdata.obj
 0001:000944d0       ?AfxCriticalInit@@YGHXZ    5f8954d0 f   afxcrit.obj
 0001:0009456b       ?AfxCriticalTerm@@YGXXZ    5f89556b f   afxcrit.obj
 0001:0009466a       ?AfxLockGlobals@@YGXH@Z    5f89566a f   afxcrit.obj
 0001:0009479c       ?AfxUnlockGlobals@@YGXH@Z  5f89579c f   afxcrit.obj
 0001:00094870       ?_AfxLoadDotBitmap@@YGXXZ  5f895870 f   cmdtarg.obj
 0001:00094a3a       ?Dump@CCmdTarget@@UBEXAAVCDumpContext@@@Z 5f895a3a f   cmdtarg.obj
 0001:00094b1e       ?AssertValid@CCmdTarget@@UBEXXZ 5f895b1e f   cmdtarg.obj
 0001:00094b31       ?_GetBaseClass@CCmdTarget@@KGPAUCRuntimeClass@@XZ 5f895b31 f   cmdtarg.obj
 0001:00094b3b       ?GetRuntimeClass@CCmdTarget@@UBEPAUCRuntimeClass@@XZ 5f895b3b f   cmdtarg.obj
 0001:00094b50       ?_GetBaseClass@CDocument@@KGPAUCRuntimeClass@@XZ 5f895b50 f   doccore.obj
 0001:00094b5a       ?GetRuntimeClass@CDocument@@UBEPAUCRuntimeClass@@XZ 5f895b5a f   doccore.obj
 0001:00094b70       ?_GetBaseClass@CDocTemplate@@KGPAUCRuntimeClass@@XZ 5f895b70 f   doctempl.obj
 0001:00094b7a       ?GetRuntimeClass@CDocTemplate@@UBEPAUCRuntimeClass@@XZ 5f895b7a f   doctempl.obj
 0001:00094b90       ?_GetBaseClass@CSingleDocTemplate@@KGPAUCRuntimeClass@@XZ 5f895b90 f   docsingl.obj
 0001:00094b9a       ?GetRuntimeClass@CSingleDocTemplate@@UBEPAUCRuntimeClass@@XZ 5f895b9a f   docsingl.obj
 0001:00094bb0       ?_GetBaseClass@CMultiDocTemplate@@KGPAUCRuntimeClass@@XZ 5f895bb0 f   docmulti.obj
 0001:00094bba       ?GetRuntimeClass@CMultiDocTemplate@@UBEPAUCRuntimeClass@@XZ 5f895bba f   docmulti.obj
 0001:00094bd0       ?_AfxDeleteRegKey@@YGHPBG@Z 5f895bd0 f   docmgr.obj
 0001:00094cc2       ?_AfxSetRegKey@@YGHPBG00@Z 5f895cc2 f   docmgr.obj
 0001:00094d83       ??0CDocManager@@QAE@XZ     5f895d83 f   docmgr.obj
 0001:00094ddc       ?UnregisterShellFileTypes@CDocManager@@QAEXXZ 5f895ddc f   docmgr.obj
 0001:000951b8       ?RegisterShellFileTypes@CDocManager@@UAEXH@Z 5f8961b8 f   docmgr.obj
 0001:00095aca       ?_GetBaseClass@CDocManager@@KGPAUCRuntimeClass@@XZ 5f896aca f   docmgr.obj
 0001:00095ad4       ?GetRuntimeClass@CDocManager@@UBEPAUCRuntimeClass@@XZ 5f896ad4 f   docmgr.obj
 0001:00095af0       ?_GetBaseClass@CSplitterWnd@@KGPAUCRuntimeClass@@XZ 5f896af0 f   viewcore.obj
 0001:00095afa       ?GetRuntimeClass@CSplitterWnd@@UBEPAUCRuntimeClass@@XZ 5f896afa f   viewcore.obj
 0001:00095b0a       ?_GetBaseClass@CCtrlView@@KGPAUCRuntimeClass@@XZ 5f896b0a f   viewcore.obj
 0001:00095b14       ?GetRuntimeClass@CCtrlView@@UBEPAUCRuntimeClass@@XZ 5f896b14 f   viewcore.obj
 0001:00095b30       ?_GetBaseClass@CScrollView@@KGPAUCRuntimeClass@@XZ 5f896b30 f   viewscrl.obj
 0001:00095b3a       ?GetRuntimeClass@CScrollView@@UBEPAUCRuntimeClass@@XZ 5f896b3a f   viewscrl.obj
 0001:00095b50       ?_GetBaseClass@CFormView@@KGPAUCRuntimeClass@@XZ 5f896b50 f   viewform.obj
 0001:00095b5a       ?GetRuntimeClass@CFormView@@UBEPAUCRuntimeClass@@XZ 5f896b5a f   viewform.obj
 0001:00095b70       ?CreateObject@CEditView@@SGPAVCObject@@XZ 5f896b70 f   viewedit.obj
 0001:00095bde       ?_GetBaseClass@CEditView@@KGPAUCRuntimeClass@@XZ 5f896bde f   viewedit.obj
 0001:00095be8       ?GetRuntimeClass@CEditView@@UBEPAUCRuntimeClass@@XZ 5f896be8 f   viewedit.obj
 0001:00095c30       ??B?$CProcessLocal@V_AFX_EDIT_STATE@@@@QAEPAV_AFX_EDIT_STATE@@XZ 5f896c30 f i viewedit.obj
 0001:00095c50       ?GetData@?$CProcessLocal@V_AFX_EDIT_STATE@@@@QAEPAV_AFX_EDIT_STATE@@XZ 5f896c50 f i viewedit.obj
 0001:00095ca0       ?CreateObject@?$CProcessLocal@V_AFX_EDIT_STATE@@@@SGPAVCNoTrackObject@@XZ 5f896ca0 f i viewedit.obj
 0001:00095d10       ?CreateObject@CPreviewView@@SGPAVCObject@@XZ 5f896d10 f   viewprev.obj
 0001:00095d77       ?_GetBaseClass@CPreviewView@@KGPAUCRuntimeClass@@XZ 5f896d77 f   viewprev.obj
 0001:00095d81       ?GetRuntimeClass@CPreviewView@@UBEPAUCRuntimeClass@@XZ 5f896d81 f   viewprev.obj
 0001:00095da0       ?CreateObject@CListView@@SGPAVCObject@@XZ 5f896da0 f   viewcmn.obj
 0001:00095e0b       ?_GetBaseClass@CListView@@KGPAUCRuntimeClass@@XZ 5f896e0b f   viewcmn.obj
 0001:00095e15       ?GetRuntimeClass@CListView@@UBEPAUCRuntimeClass@@XZ 5f896e15 f   viewcmn.obj
 0001:00095e25       ?CreateObject@CTreeView@@SGPAVCObject@@XZ 5f896e25 f   viewcmn.obj
 0001:00095e90       ?_GetBaseClass@CTreeView@@KGPAUCRuntimeClass@@XZ 5f896e90 f   viewcmn.obj
 0001:00095e9a       ?GetRuntimeClass@CTreeView@@UBEPAUCRuntimeClass@@XZ 5f896e9a f   viewcmn.obj
 0001:00095ef0       ??B?$CProcessLocal@V_AFX_MAIL_STATE@@@@QAEPAV_AFX_MAIL_STATE@@XZ 5f896ef0 f i docmapi.obj
 0001:00095f10       ?GetData@?$CProcessLocal@V_AFX_MAIL_STATE@@@@QAEPAV_AFX_MAIL_STATE@@XZ 5f896f10 f i docmapi.obj
 0001:00095f60       ?CreateObject@?$CProcessLocal@V_AFX_MAIL_STATE@@@@SGPAVCNoTrackObject@@XZ 5f896f60 f i docmapi.obj
 0001:00095fd0       ??0_AFX_MAIL_STATE@@QAE@XZ 5f896fd0 f i docmapi.obj
 0001:00095ff0       ??0CWinThread@@QAE@P6AIPAX@Z0@Z 5f896ff0 f   thrdcore.obj
 0001:00096063       ??0CWinThread@@QAE@XZ      5f897063 f   thrdcore.obj
 0001:000960d6       ?CommonConstruct@CWinThread@@QAEXXZ 5f8970d6 f   thrdcore.obj
 0001:00096152       ?_GetBaseClass@CWinThread@@KGPAUCRuntimeClass@@XZ 5f897152 f   thrdcore.obj
 0001:0009615c       ?GetRuntimeClass@CWinThread@@UBEPAUCRuntimeClass@@XZ 5f89715c f   thrdcore.obj
 0001:00096170       ??_GCWinThread@@UAEPAXI@Z  5f897170 f i thrdcore.obj
 0001:00096170       ??_ECWinThread@@UAEPAXI@Z  5f897170 f i thrdcore.obj
 0001:000961a0       ?GetDataNA@?$CThreadLocal@V_AFX_THREAD_STATE@@@@QAEPAV_AFX_THREAD_STATE@@XZ 5f8971a0 f i thrdcore.obj
 0001:000961c0       ??B?$CThreadLocal@V_AFX_CTL3D_THREAD@@@@QAEPAV_AFX_CTL3D_THREAD@@XZ 5f8971c0 f i thrdcore.obj
 0001:000961e0       ?GetData@?$CThreadLocal@V_AFX_CTL3D_THREAD@@@@QAEPAV_AFX_CTL3D_THREAD@@XZ 5f8971e0 f i thrdcore.obj
 0001:00096230       ?CreateObject@?$CThreadLocal@V_AFX_CTL3D_THREAD@@@@SGPAVCNoTrackObject@@XZ 5f897230 f i thrdcore.obj
 0001:000962a0       ??0_AFX_CTL3D_THREAD@@QAE@XZ 5f8972a0 f i thrdcore.obj
 0001:000962c0       ??_G_AFX_CTL3D_THREAD@@UAEPAXI@Z 5f8972c0 f i thrdcore.obj
 0001:000962c0       ??_E_AFX_CTL3D_THREAD@@UAEPAXI@Z 5f8972c0 f i thrdcore.obj
 0001:000962f0       ??0_AFX_WIN_STATE@@QAE@XZ  5f8972f0 f   appcore.obj
 0001:0009630f       ??0CWinApp@@QAE@PBG@Z      5f89730f f   appcore.obj
 0001:00096547       ?InitApplication@CWinApp@@UAEHXZ 5f897547 f   appcore.obj
 0001:000965b6       ?InitInstance@CWinApp@@UAEHXZ 5f8975b6 f   appcore.obj
 0001:000965c6       ?LoadStdProfileSettings@CWinApp@@IAEXI@Z 5f8975c6 f   appcore.obj
 0001:000966c6       ?ParseCommandLine@CWinApp@@QAEXAAVCCommandLineInfo@@@Z 5f8976c6 f   appcore.obj
 0001:0009676a       ??0CCommandLineInfo@@QAE@XZ 5f89776a f   appcore.obj
 0001:00096816       ??1CCommandLineInfo@@UAE@XZ 5f897816 f   appcore.obj
 0001:00096897       ?ParseParam@CCommandLineInfo@@UAEXPBGHH@Z 5f897897 f   appcore.obj
 0001:0009693b       ?ParseParam@CCommandLineInfo@@UAEXPBDHH@Z 5f89793b f   appcore.obj
 0001:00096974       ?ParseParamFlag@CCommandLineInfo@@IAEXPBD@Z 5f897974 f   appcore.obj
 0001:00096a7e       ?ParseParamNotFlag@CCommandLineInfo@@IAEXPBG@Z 5f897a7e f   appcore.obj
 0001:00096b24       ?ParseParamNotFlag@CCommandLineInfo@@IAEXPBD@Z 5f897b24 f   appcore.obj
 0001:00096bca       ?ParseLast@CCommandLineInfo@@IAEXH@Z 5f897bca f   appcore.obj
 0001:00096c2c       ??1CWinApp@@UAE@XZ         5f897c2c f   appcore.obj
 0001:00096edb       ?SaveStdProfileSettings@CWinApp@@IAEXXZ 5f897edb f   appcore.obj
 0001:00096f44       ?ExitInstance@CWinApp@@UAEHXZ 5f897f44 f   appcore.obj
 0001:00096fc9       ?_GetBaseClass@CWinApp@@KGPAUCRuntimeClass@@XZ 5f897fc9 f   appcore.obj
 0001:00096fd3       ?GetRuntimeClass@CWinApp@@UBEPAUCRuntimeClass@@XZ 5f897fd3 f   appcore.obj
 0001:00097020       ??_E_AFX_WIN_STATE@@UAEPAXI@Z 5f898020 f i appcore.obj
 0001:00097020       ??_G_AFX_WIN_STATE@@UAEPAXI@Z 5f898020 f i appcore.obj
 0001:00097050       ??_ECWinApp@@UAEPAXI@Z     5f898050 f i appcore.obj
 0001:00097050       ??_GCWinApp@@UAEPAXI@Z     5f898050 f i appcore.obj
 0001:00097080       ?AfxWinInit@@YGHPAUHINSTANCE__@@0PAGH@Z 5f898080 f   appinit.obj
 0001:0009712f       ?SetCurrentHandles@CWinApp@@QAEXXZ 5f89812f f   appinit.obj
 0001:0009743f       ?AfxGetFileName@@YGIPBGPAGI@Z 5f89843f f   appinit.obj
 0001:00097540       ?ProcessShellCommand@CWinApp@@QAEHAAVCCommandLineInfo@@@Z 5f898540 f   appui2.obj
 0001:00097764       ?Unregister@CWinApp@@QAEHXZ 5f898764 f   appui2.obj
 0001:000979a6       ?DelRegTree@CWinApp@@QAEJPAUHKEY__@@ABVCString@@@Z 5f8989a6 f   appui2.obj
 0001:000979c0       ?AfxDelRegTreeHelper@@YGJPAUHKEY__@@ABVCString@@@Z 5f8989c0 f   appui2.obj
 0001:00097acc       ?EnableShellOpen@CWinApp@@IAEXXZ 5f898acc f   appui2.obj
 0001:00097b46       ?RegisterShellFileTypes@CWinApp@@IAEXH@Z 5f898b46 f   appui2.obj
 0001:00097b9a       ?RegisterShellFileTypesCompat@CWinApp@@IAEXXZ 5f898b9a f   appui2.obj
 0001:00097bea       ?UnregisterShellFileTypes@CWinApp@@IAEXXZ 5f898bea f   appui2.obj
 0001:00097c30       ?SetRegistryKey@CWinApp@@IAEXPBG@Z 5f898c30 f   appui3.obj
 0001:00097d13       ?SetRegistryKey@CWinApp@@IAEXI@Z 5f898d13 f   appui3.obj
 0001:00097d96       ?GetAppRegistryKey@CWinApp@@QAEPAUHKEY__@@XZ 5f898d96 f   appui3.obj
 0001:00097e9c       ?GetSectionKey@CWinApp@@QAEPAUHKEY__@@PBG@Z 5f898e9c f   appui3.obj
 0001:00097f1a       ?GetProfileIntW@CWinApp@@QAEIPBG0H@Z 5f898f1a f   appui3.obj
 0001:00098052       ?GetProfileStringW@CWinApp@@QAE?AVCString@@PBG00@Z 5f899052 f   appui3.obj
 0001:000982ef       ?GetProfileBinary@CWinApp@@QAEHPBG0PAPAEPAI@Z 5f8992ef f   appui3.obj
 0001:00098610       ?SetDialogBkColor@CWinApp@@IAEXKK@Z 5f899610 f   appgray.obj
 0001:000986b0       ??1_AFX_CTL3D_STATE@@UAE@XZ 5f8996b0 f   app3d.obj
 0001:00098720       ??1_AFX_CTL3D_THREAD@@UAE@XZ 5f899720 f   app3d.obj
 0001:0009878d       ?Enable3dControls@CWinApp@@IAEHXZ 5f89978d f   app3d.obj
 0001:000989a7       ?AfxGetCtl3dState@@YGPAV_AFX_CTL3D_STATE@@XZ 5f8999a7 f   app3d.obj
 0001:00098a20       ?_GetBaseClass@CInternetException@@KGPAUCRuntimeClass@@XZ 5f899a20 f   inet.obj
 0001:00098a2a       ?GetRuntimeClass@CInternetException@@UBEPAUCRuntimeClass@@XZ 5f899a2a f   inet.obj
 0001:00098a3a       ?_GetBaseClass@CInternetFile@@KGPAUCRuntimeClass@@XZ 5f899a3a f   inet.obj
 0001:00098a44       ?GetRuntimeClass@CInternetFile@@UBEPAUCRuntimeClass@@XZ 5f899a44 f   inet.obj
 0001:00098a54       ?_GetBaseClass@CHttpFile@@KGPAUCRuntimeClass@@XZ 5f899a54 f   inet.obj
 0001:00098a5e       ?GetRuntimeClass@CHttpFile@@UBEPAUCRuntimeClass@@XZ 5f899a5e f   inet.obj
 0001:00098a6e       ?_GetBaseClass@CGopherFile@@KGPAUCRuntimeClass@@XZ 5f899a6e f   inet.obj
 0001:00098a78       ?GetRuntimeClass@CGopherFile@@UBEPAUCRuntimeClass@@XZ 5f899a78 f   inet.obj
 0001:00098a88       ?_GetBaseClass@CInternetSession@@KGPAUCRuntimeClass@@XZ 5f899a88 f   inet.obj
 0001:00098a92       ?GetRuntimeClass@CInternetSession@@UBEPAUCRuntimeClass@@XZ 5f899a92 f   inet.obj
 0001:00098aa2       ?_GetBaseClass@CInternetConnection@@KGPAUCRuntimeClass@@XZ 5f899aa2 f   inet.obj
 0001:00098aac       ?GetRuntimeClass@CInternetConnection@@UBEPAUCRuntimeClass@@XZ 5f899aac f   inet.obj
 0001:00098abc       ?_GetBaseClass@CFtpConnection@@KGPAUCRuntimeClass@@XZ 5f899abc f   inet.obj
 0001:00098ac6       ?GetRuntimeClass@CFtpConnection@@UBEPAUCRuntimeClass@@XZ 5f899ac6 f   inet.obj
 0001:00098ad6       ?_GetBaseClass@CHttpConnection@@KGPAUCRuntimeClass@@XZ 5f899ad6 f   inet.obj
 0001:00098ae0       ?GetRuntimeClass@CHttpConnection@@UBEPAUCRuntimeClass@@XZ 5f899ae0 f   inet.obj
 0001:00098af0       ?_GetBaseClass@CGopherConnection@@KGPAUCRuntimeClass@@XZ 5f899af0 f   inet.obj
 0001:00098afa       ?GetRuntimeClass@CGopherConnection@@UBEPAUCRuntimeClass@@XZ 5f899afa f   inet.obj
 0001:00098b0a       ?_GetBaseClass@CFtpFileFind@@KGPAUCRuntimeClass@@XZ 5f899b0a f   inet.obj
 0001:00098b14       ?GetRuntimeClass@CFtpFileFind@@UBEPAUCRuntimeClass@@XZ 5f899b14 f   inet.obj
 0001:00098b24       ?_GetBaseClass@CGopherFileFind@@KGPAUCRuntimeClass@@XZ 5f899b24 f   inet.obj
 0001:00098b2e       ?GetRuntimeClass@CGopherFileFind@@UBEPAUCRuntimeClass@@XZ 5f899b2e f   inet.obj
 0001:00098b80       ?_GetBaseClass@CFileFind@@KGPAUCRuntimeClass@@XZ 5f899b80 f   filefind.obj
 0001:00098b8a       ?GetRuntimeClass@CFileFind@@UBEPAUCRuntimeClass@@XZ 5f899b8a f   filefind.obj
 0001:00098ba0       ?_GetBaseClass@CDynLinkLibrary@@KGPAUCRuntimeClass@@XZ 5f899ba0 f   dllinit.obj
 0001:00098baa       ?GetRuntimeClass@CDynLinkLibrary@@UBEPAUCRuntimeClass@@XZ 5f899baa f   dllinit.obj
 0001:00098bba       ??0CDynLinkLibrary@@QAE@AAUAFX_EXTENSION_MODULE@@H@Z 5f899bba f   dllinit.obj
 0001:00098cc8       ??0CDynLinkLibrary@@QAE@PAUHINSTANCE__@@0@Z 5f899cc8 f   dllinit.obj
 0001:00098da7       ?AfxInitExtensionModule@@YGHAAUAFX_EXTENSION_MODULE@@PAUHINSTANCE__@@@Z 5f899da7 f   dllinit.obj
 0001:00098e54       _RawDllMain@12             5f899e54 f   dllinit.obj
 0001:00098f09       _DllMain@12                5f899f09 f   dllinit.obj
 0001:00099157       ?AfxCoreInitModule@@YGXXZ  5f89a157 f   dllinit.obj
 0001:00099250       ??_GCDynLinkLibrary@@UAEPAXI@Z 5f89a250 f i dllinit.obj
 0001:00099250       ??_ECDynLinkLibrary@@UAEPAXI@Z 5f89a250 f i dllinit.obj
 0001:00099280       ??1_AFX_MAIL_STATE@@UAE@XZ 5f89a280 f   docmapi.obj
 0001:000992b2       ?OnFileSendMail@CDocument@@IAEXXZ 5f89a2b2 f   docmapi.obj
 0001:000997f1       ?OnUpdateFileSendMail@CDocument@@IAEXPAVCCmdUI@@@Z 5f89a7f1 f   docmapi.obj
 0001:00099926       ?OnFileSendMail@COleDocument@@IAEXXZ 5f89a926 f   docmapi.obj
 0001:00099a30       ??_E_AFX_MAIL_STATE@@UAEPAXI@Z 5f89aa30 f i docmapi.obj
 0001:00099a30       ??_G_AFX_MAIL_STATE@@UAEPAXI@Z 5f89aa30 f i docmapi.obj
 0001:00099a60       ?_AfxMultMultDivDiv@@YGJHHHHH@Z 5f89aa60 f   dcprev.obj
 0001:00099cca       ??0CPreviewDC@@QAE@XZ      5f89acca f   dcprev.obj
 0001:00099d73       ?SetOutputDC@CPreviewDC@@UAEXPAUHDC__@@@Z 5f89ad73 f   dcprev.obj
 0001:00099e01       ?ReleaseOutputDC@CPreviewDC@@UAEXXZ 5f89ae01 f   dcprev.obj
 0001:00099e51       ?SetAttribDC@CPreviewDC@@UAEXPAUHDC__@@@Z 5f89ae51 f   dcprev.obj
 0001:00099eaa       ??1CPreviewDC@@UAE@XZ      5f89aeaa f   dcprev.obj
 0001:00099f28       ?SetScaleRatio@CPreviewDC@@QAEXHH@Z 5f89af28 f   dcprev.obj
 0001:00099f62       ?AssertValid@CPreviewDC@@UBEXXZ 5f89af62 f   dcprev.obj
 0001:00099f75       ?Dump@CPreviewDC@@UBEXAAVCDumpContext@@@Z 5f89af75 f   dcprev.obj
 0001:00099fd0       ?SaveDC@CPreviewDC@@UAEHXZ 5f89afd0 f   dcprev.obj
 0001:0009a06e       ?RestoreDC@CPreviewDC@@UAEHH@Z 5f89b06e f   dcprev.obj
 0001:0009a149       ?MirrorAttributes@CPreviewDC@@IAEXXZ 5f89b149 f   dcprev.obj
 0001:0009a291       ?SelectStockObject@CPreviewDC@@UAEPAVCGdiObject@@H@Z 5f89b291 f   dcprev.obj
 0001:0009a3a1       ?MirrorFont@CPreviewDC@@IAEXXZ 5f89b3a1 f   dcprev.obj
 0001:0009a6ab       ?SelectObject@CPreviewDC@@UAEPAVCFont@@PAV2@@Z 5f89b6ab f   dcprev.obj
 0001:0009a742       ?SetBkColor@CPreviewDC@@UAEKK@Z 5f89b742 f   dcprev.obj
 0001:0009a7b1       ?SetTextColor@CPreviewDC@@UAEKK@Z 5f89b7b1 f   dcprev.obj
 0001:0009a820       ?SetMapMode@CPreviewDC@@UAEHH@Z 5f89b820 f   dcprev.obj
 0001:0009a879       ?SetViewportOrg@CPreviewDC@@UAE?AVCPoint@@HH@Z 5f89b879 f   dcprev.obj
 0001:0009a909       ?OffsetViewportOrg@CPreviewDC@@UAE?AVCPoint@@HH@Z 5f89b909 f   dcprev.obj
 0001:0009a999       ?SetViewportExt@CPreviewDC@@UAE?AVCSize@@HH@Z 5f89b999 f   dcprev.obj
 0001:0009aa2b       ?ScaleViewportExt@CPreviewDC@@UAE?AVCSize@@HHHH@Z 5f89ba2b f   dcprev.obj
 0001:0009aac5       ?SetWindowExt@CPreviewDC@@UAE?AVCSize@@HH@Z 5f89bac5 f   dcprev.obj
 0001:0009ab57       ?ScaleWindowExt@CPreviewDC@@UAE?AVCSize@@HHHH@Z 5f89bb57 f   dcprev.obj
 0001:0009abf1       ?_AfxComputeNextTab@@YGHHIPAHHH@Z 5f89bbf1 f   dcprev.obj
 0001:0009ac4e       ?ComputeDeltas@CPreviewDC@@IAE?AVCSize@@AAHPBGAAIHIPAHHPAG30@Z 5f89bc4e f   dcprev.obj
 0001:0009b0d2       ?TextOutW@CPreviewDC@@UAEHHHPBGH@Z 5f89c0d2 f   dcprev.obj
 0001:0009b100       ?ExtTextOutW@CPreviewDC@@UAEHHHIPBUtagRECT@@PBGIPAH@Z 5f89c100 f   dcprev.obj
 0001:0009b3b7       ?TabbedTextOutW@CPreviewDC@@UAE?AVCSize@@HHPBGHHPAHH@Z 5f89c3b7 f   dcprev.obj
 0001:0009b675       ?DrawTextW@CPreviewDC@@UAEHPBGHPAUtagRECT@@I@Z 5f89c675 f   dcprev.obj
 0001:0009b7d6       ?GrayStringW@CPreviewDC@@UAEHPAVCBrush@@P6GHPAUHDC__@@JH@ZJHHHHH@Z 5f89c7d6 f   dcprev.obj
 0001:0009b810       ?Escape@CPreviewDC@@UAEHHHPBDPAX@Z 5f89c810 f   dcprev.obj
 0001:0009b910       ?MirrorMappingMode@CPreviewDC@@IAEXH@Z 5f89c910 f   dcprev.obj
 0001:0009bb6c       ?MirrorViewportOrg@CPreviewDC@@IAEXXZ 5f89cb6c f   dcprev.obj
 0001:0009bc5d       ?SetTopLeftOffset@CPreviewDC@@QAEXVCSize@@@Z 5f89cc5d f   dcprev.obj
 0001:0009bcaa       ?ClipToPage@CPreviewDC@@QAEXXZ 5f89ccaa f   dcprev.obj
 0001:0009bd9f       ?PrinterDPtoScreenDP@CPreviewDC@@QBEXPAUtagPOINT@@@Z 5f89cd9f f   dcprev.obj
 0001:0009bea0       ??_GCPreviewDC@@UAEPAXI@Z  5f89cea0 f i dcprev.obj
 0001:0009bea0       ??_ECPreviewDC@@UAEPAXI@Z  5f89cea0 f i dcprev.obj
 0001:0009bed0       ??0CMetaFileDC@@QAE@XZ     5f89ced0 f   dcmeta.obj
 0001:0009beef       ?SetOutputDC@CMetaFileDC@@MAEXPAUHDC__@@@Z 5f89ceef f   dcmeta.obj
 0001:0009bf34       ?ReleaseOutputDC@CMetaFileDC@@MAEXXZ 5f89cf34 f   dcmeta.obj
 0001:0009bf77       ?SetAttribDC@CMetaFileDC@@UAEXPAUHDC__@@@Z 5f89cf77 f   dcmeta.obj
 0001:0009bfb4       ??1CMetaFileDC@@UAE@XZ     5f89cfb4 f   dcmeta.obj
 0001:0009c02f       ?GetClipBox@CMetaFileDC@@UBEHPAUtagRECT@@@Z 5f89d02f f   dcmeta.obj
 0001:0009c0b8       ?PtVisible@CMetaFileDC@@UBEHHH@Z 5f89d0b8 f   dcmeta.obj
 0001:0009c100       ?RectVisible@CMetaFileDC@@UBEHPBUtagRECT@@@Z 5f89d100 f   dcmeta.obj
 0001:0009c138       ?TextOutW@CMetaFileDC@@UAEHHHPBGH@Z 5f89d138 f   dcmeta.obj
 0001:0009c254       ?ExtTextOutW@CMetaFileDC@@UAEHHHIPBUtagRECT@@PBGIPAH@Z 5f89d254 f   dcmeta.obj
 0001:0009c3b8       ?TabbedTextOutW@CMetaFileDC@@UAE?AVCSize@@HHPBGHHPAHH@Z 5f89d3b8 f   dcmeta.obj
 0001:0009c68e       ?AdjustCP@CMetaFileDC@@IAEXH@Z 5f89d68e f   dcmeta.obj
 0001:0009c703       ?DrawTextW@CMetaFileDC@@UAEHPBGHPAUtagRECT@@I@Z 5f89d703 f   dcmeta.obj
 0001:0009c8a3       ?Escape@CMetaFileDC@@UAEHHHPBDPAX@Z 5f89d8a3 f   dcmeta.obj
 0001:0009c9fd       ?SetViewportOrg@CMetaFileDC@@UAE?AVCPoint@@HH@Z 5f89d9fd f   dcmeta.obj
 0001:0009ca8b       ?OffsetViewportOrg@CMetaFileDC@@UAE?AVCPoint@@HH@Z 5f89da8b f   dcmeta.obj
 0001:0009cb19       ?SetViewportExt@CMetaFileDC@@UAE?AVCSize@@HH@Z 5f89db19 f   dcmeta.obj
 0001:0009cba7       ?ScaleViewportExt@CMetaFileDC@@UAE?AVCSize@@HHHH@Z 5f89dba7 f   dcmeta.obj
 0001:0009cc50       ?_AfxAbortProc@@YGHPAUHDC__@@H@Z 5f89dc50 f   viewprnt.obj
 0001:0009ccb1       ?OnInitDialog@CPrintingDialog@@UAEHXZ 5f89dcb1 f   viewprnt.obj
 0001:0009ccdc       ?OnCancel@CPrintingDialog@@UAEXXZ 5f89dcdc f   viewprnt.obj
 0001:0009cd00       ?DoPreparePrinting@CView@@QAEHPAUCPrintInfo@@@Z 5f89dd00 f   viewprnt.obj
 0001:0009cf38       ?OnFilePrint@CView@@IAEXXZ 5f89df38 f   viewprnt.obj
 0001:0009d8ed       ??0CPrintInfo@@QAE@XZ      5f89e8ed f   viewprnt.obj
 0001:0009da1b       ??1CPrintInfo@@QAE@XZ      5f89ea1b f   viewprnt.obj
 0001:0009dad0       ??0CPrintingDialog@@QAE@PAVCWnd@@@Z 5f89ead0 f i viewprnt.obj
 0001:0009db40       ??1CPrintingDialog@@UAE@XZ 5f89eb40 f i viewprnt.obj
 0001:0009db60       ??_ECPrintingDialog@@UAEPAXI@Z 5f89eb60 f i viewprnt.obj
 0001:0009db60       ??_GCPrintingDialog@@UAEPAXI@Z 5f89eb60 f i viewprnt.obj
 0001:0009db90       ??C?$CProcessLocal@V_AFX_WIN_STATE@@@@QAEPAV_AFX_WIN_STATE@@XZ 5f89eb90 f i viewprnt.obj
 0001:0009dbb0       ??0CPrintPreviewState@@QAE@XZ 5f89ebb0 f   viewprev.obj
 0001:0009dbf9       ?OnFilePrintPreview@CView@@IAEXXZ 5f89ebf9 f   viewprev.obj
 0001:0009dcb6       ?DoPrintPreview@CView@@QAEHIPAV1@PAUCRuntimeClass@@PAUCPrintPreviewState@@@Z 5f89ecb6 f   viewprev.obj
 0001:0009e0a0       ?_AfxPreviewCloseProc@@YGHPAVCFrameWnd@@@Z 5f89f0a0 f   viewprev.obj
 0001:0009e108       ?_GetBaseMessageMap@CPreviewView@@KGPBUAFX_MSGMAP@@XZ 5f89f108 f   viewprev.obj
 0001:0009e112       ?GetMessageMap@CPreviewView@@MBEPBUAFX_MSGMAP@@XZ 5f89f112 f   viewprev.obj
 0001:0009e122       ??0CPreviewView@@QAE@XZ    5f89f122 f   viewprev.obj
 0001:0009e242       ??0PAGE_INFO@CPreviewView@@QAE@XZ 5f89f242 f   viewprev.obj
 0001:0009e279       ??1CPreviewView@@UAE@XZ    5f89f279 f   viewprev.obj
 0001:0009e382       ?OnCreate@CPreviewView@@IAEHPAUtagCREATESTRUCTW@@@Z 5f89f382 f   viewprev.obj
 0001:0009e419       ?SetPrintView@CPreviewView@@QAEHPAVCView@@@Z 5f89f419 f   viewprev.obj
 0001:0009e87b       ?OnSize@CPreviewView@@IAEXIHH@Z 5f89f87b f   viewprev.obj
 0001:0009e92d       ?OnActivateView@CPreviewView@@MAEXHPAVCView@@0@Z 5f89f92d f   viewprev.obj
 0001:0009e98c       ?OnPreviewClose@CPreviewView@@IAEXXZ 5f89f98c f   viewprev.obj
 0001:0009ea1a       ?CalcScaleRatio@CPreviewView@@MAE?AVCSize@@V2@0@Z 5f89fa1a f   viewprev.obj
 0001:0009ea79       ?PositionPage@CPreviewView@@MAEXI@Z 5f89fa79 f   viewprev.obj
 0001:0009eb94       ?CalcPageDisplaySize@CPreviewView@@IAE?AVCSize@@XZ 5f89fb94 f   viewprev.obj
 0001:0009ec6c       ?SetScaledSize@CPreviewView@@IAEXI@Z 5f89fc6c f   viewprev.obj
 0001:0009ef06       ?OnPrepareDC@CPreviewView@@UAEXPAVCDC@@PAUCPrintInfo@@@Z 5f89ff06 f   viewprev.obj
 0001:0009ef63       ?OnEraseBkgnd@CPreviewView@@IAEHPAVCDC@@@Z 5f89ff63 f   viewprev.obj
 0001:0009f02e       ?OnDraw@CPreviewView@@MAEXPAVCDC@@@Z 5f8a002e f   viewprev.obj
 0001:0009f6e7       ?OnHScroll@CPreviewView@@IAEXIIPAVCScrollBar@@@Z 5f8a06e7 f   viewprev.obj
 0001:0009f714       ?OnVScroll@CPreviewView@@IAEXIIPAVCScrollBar@@@Z 5f8a0714 f   viewprev.obj
 0001:0009f88f       ?OnNumPageChange@CPreviewView@@IAEXXZ 5f8a088f f   viewprev.obj
 0001:0009f923       ?OnNextPage@CPreviewView@@IAEXXZ 5f8a0923 f   viewprev.obj
 0001:0009f945       ?OnPrevPage@CPreviewView@@IAEXXZ 5f8a0945 f   viewprev.obj
 0001:0009f967       ?OnPreviewPrint@CPreviewView@@IAEXXZ 5f8a0967 f   viewprev.obj
 0001:0009f9ae       ?FindPageRect@CPreviewView@@IAEHAAVCPoint@@AAI@Z 5f8a09ae f   viewprev.obj
 0001:0009fb45       ?OnLButtonDown@CPreviewView@@IAEXIVCPoint@@@Z 5f8a0b45 f   viewprev.obj
 0001:0009fba6       ?SetZoomState@CPreviewView@@IAEXIIVCPoint@@@Z 5f8a0ba6 f   viewprev.obj
 0001:0009fbe1       ?OnZoomIn@CPreviewView@@IAEXXZ 5f8a0be1 f   viewprev.obj
 0001:0009fc24       ?OnZoomOut@CPreviewView@@IAEXXZ 5f8a0c24 f   viewprev.obj
 0001:0009fc67       ?DoZoom@CPreviewView@@IAEXIVCPoint@@@Z 5f8a0c67 f   viewprev.obj
 0001:0009fe96       ?SetCurrentPage@CPreviewView@@IAEXIH@Z 5f8a0e96 f   viewprev.obj
 0001:0009ff7c       ?OnDisplayPageNumber@CPreviewView@@MAEXII@Z 5f8a0f7c f   viewprev.obj
 0001:000a00cd       ?OnUpdateNumPageChange@CPreviewView@@IAEXPAVCCmdUI@@@Z 5f8a10cd f   viewprev.obj
 0001:000a01ea       ?OnUpdateNextPage@CPreviewView@@IAEXPAVCCmdUI@@@Z 5f8a11ea f   viewprev.obj
 0001:000a022e       ?OnUpdatePrevPage@CPreviewView@@IAEXPAVCCmdUI@@@Z 5f8a122e f   viewprev.obj
 0001:000a0261       ?OnUpdateZoomIn@CPreviewView@@IAEXPAVCCmdUI@@@Z 5f8a1261 f   viewprev.obj
 0001:000a0288       ?OnUpdateZoomOut@CPreviewView@@IAEXPAVCCmdUI@@@Z 5f8a1288 f   viewprev.obj
 0001:000a02af       ?OnSetCursor@CPreviewView@@IAEHPAVCWnd@@II@Z 5f8a12af f   viewprev.obj
 0001:000a0376       ?AssertValid@CPreviewView@@UBEXXZ 5f8a1376 f   viewprev.obj
 0001:000a0441       ?Dump@CPreviewView@@UBEXAAVCDumpContext@@@Z 5f8a1441 f   viewprev.obj
 0001:000a0730       ??_GCPreviewView@@UAEPAXI@Z 5f8a1730 f i viewprev.obj
 0001:000a0730       ??_ECPreviewView@@UAEPAXI@Z 5f8a1730 f i viewprev.obj
 0001:000a0760       ??_GCPrintInfo@@QAEPAXI@Z  5f8a1760 f i viewprev.obj
 0001:000a0790       ?GetPrinterDeviceDefaults@CWinApp@@QAEHPAUtagPDW@@@Z 5f8a1790 f   appprnt.obj
 0001:000a0808       ?UpdatePrinterSelection@CWinApp@@IAEXH@Z 5f8a1808 f   appprnt.obj
 0001:000a0bea       ?DoPrintDialog@CWinApp@@QAEHPAVCPrintDialog@@@Z 5f8a1bea f   appprnt.obj
 0001:000a0d85       ?OnFilePrintSetup@CWinApp@@IAEXXZ 5f8a1d85 f   appprnt.obj
 0001:000a0df6       ?SelectPrinter@CWinApp@@QAEXPAX0H@Z 5f8a1df6 f   appprnt.obj
 0001:000a0e79       ?CreatePrinterDC@CWinApp@@QAEHAAVCDC@@@Z 5f8a1e79 f   appprnt.obj
 0001:000a0ef0       ??1AUX_DATA@@QAE@XZ        5f8a1ef0 f   auxdata.obj
 0001:000a0f10       ??1CDocManager@@UAE@XZ     5f8a1f10 f   docmgr.obj
 0001:000a0fe0       ??1CWinThread@@UAE@XZ      5f8a1fe0 f   thrdcore.obj
 0001:000a1060       ??1_AFX_WIN_STATE@@UAE@XZ  5f8a2060 f   appcore.obj
 0001:000a10b5       ?AfxPostQuitMessage@@YGXH@Z 5f8a20b5 f   appcore.obj
 0001:000a10f0       ?AfxWinTerm@@YGXXZ         5f8a20f0 f   appterm.obj
 0001:000a1230       ??1CDynLinkLibrary@@UAE@XZ 5f8a2230 f   dllinit.obj
 0001:000a129c       ?AssertValid@CDynLinkLibrary@@UBEXXZ 5f8a229c f   dllinit.obj
 0001:000a12cd       ?Dump@CDynLinkLibrary@@UBEXAAVCDumpContext@@@Z 5f8a22cd f   dllinit.obj
 0001:000a138c       ?AfxTermExtensionModule@@YGXAAUAFX_EXTENSION_MODULE@@H@Z 5f8a238c f   dllinit.obj
 0001:000a145e       ?AfxLoadLibrary@@YGPAUHINSTANCE__@@PBG@Z 5f8a245e f   dllinit.obj
 0001:000a14ac       ?AfxFreeLibrary@@YGHPAUHINSTANCE__@@@Z 5f8a24ac f   dllinit.obj
 0001:000a39b0       ?_AfxBinaryCompatibleStubFunction@@YAXXZ 5f8a49b0 f   dllinit.obj
 0001:000a39e0       ??_ECBitmap@@UAEPAXI@Z     5f8a49e0 f i dllinit.obj
 0001:000a3a50       ??_ECBitmapButton@@UAEPAXI@Z 5f8a4a50 f i dllinit.obj
 0001:000a3ac0       ??_ECBrush@@UAEPAXI@Z      5f8a4ac0 f i dllinit.obj
 0001:000a3b30       ??_ECButton@@UAEPAXI@Z     5f8a4b30 f i dllinit.obj
 0001:000a3ba0       ??_ECByteArray@@UAEPAXI@Z  5f8a4ba0 f i dllinit.obj
 0001:000a3c10       ??_ECCmdTarget@@UAEPAXI@Z  5f8a4c10 f i dllinit.obj
 0001:000a3c80       ??_ECComboBox@@UAEPAXI@Z   5f8a4c80 f i dllinit.obj
 0001:000a3cf0       ??_ECDC@@UAEPAXI@Z         5f8a4cf0 f i dllinit.obj
 0001:000a3d60       ??_ECDWordArray@@UAEPAXI@Z 5f8a4d60 f i dllinit.obj
 0001:000a3dd0       ??_ECDialog@@UAEPAXI@Z     5f8a4dd0 f i dllinit.obj
 0001:000a3e40       ??_ECDialogBar@@UAEPAXI@Z  5f8a4e40 f i dllinit.obj
 0001:000a3eb0       ??_ECEdit@@UAEPAXI@Z       5f8a4eb0 f i dllinit.obj
 0001:000a3f20       ??_ECFile@@UAEPAXI@Z       5f8a4f20 f i dllinit.obj
 0001:000a3f90       ??_ECFont@@UAEPAXI@Z       5f8a4f90 f i dllinit.obj
 0001:000a4000       ??_ECFrameWnd@@UAEPAXI@Z   5f8a5000 f i dllinit.obj
 0001:000a4070       ??_ECGdiObject@@UAEPAXI@Z  5f8a5070 f i dllinit.obj
 0001:000a40e0       ??_ECListBox@@UAEPAXI@Z    5f8a50e0 f i dllinit.obj
 0001:000a4150       ??_ECCheckListBox@@UAEPAXI@Z 5f8a5150 f i dllinit.obj
 0001:000a41c0       ??_ECMapPtrToPtr@@UAEPAXI@Z 5f8a51c0 f i dllinit.obj
 0001:000a4230       ??_FCMapPtrToPtr@@QAEXXZ   5f8a5230 f i dllinit.obj
 0001:000a4250       ??_ECMapPtrToWord@@UAEPAXI@Z 5f8a5250 f i dllinit.obj
 0001:000a42c0       ??_FCMapPtrToWord@@QAEXXZ  5f8a52c0 f i dllinit.obj
 0001:000a42e0       ??_ECMapStringToOb@@UAEPAXI@Z 5f8a52e0 f i dllinit.obj
 0001:000a4350       ??_FCMapStringToOb@@QAEXXZ 5f8a5350 f i dllinit.obj
 0001:000a4370       ??_ECMapStringToPtr@@UAEPAXI@Z 5f8a5370 f i dllinit.obj
 0001:000a43e0       ??_FCMapStringToPtr@@QAEXXZ 5f8a53e0 f i dllinit.obj
 0001:000a4400       ??_ECMapStringToString@@UAEPAXI@Z 5f8a5400 f i dllinit.obj
 0001:000a4470       ??_FCMapStringToString@@QAEXXZ 5f8a5470 f i dllinit.obj
 0001:000a4490       ??_ECMapWordToOb@@UAEPAXI@Z 5f8a5490 f i dllinit.obj
 0001:000a4500       ??_FCMapWordToOb@@QAEXXZ   5f8a5500 f i dllinit.obj
 0001:000a4520       ??_ECMapWordToPtr@@UAEPAXI@Z 5f8a5520 f i dllinit.obj
 0001:000a4590       ??_FCMapWordToPtr@@QAEXXZ  5f8a5590 f i dllinit.obj
 0001:000a45b0       ??_ECMemFile@@UAEPAXI@Z    5f8a55b0 f i dllinit.obj
 0001:000a4620       ??_FCMemFile@@QAEXXZ       5f8a5620 f i dllinit.obj
 0001:000a4640       ??_ECMenu@@UAEPAXI@Z       5f8a5640 f i dllinit.obj
 0001:000a46b0       ??_ECMetaFileDC@@UAEPAXI@Z 5f8a56b0 f i dllinit.obj
 0001:000a4720       ??_ECObArray@@UAEPAXI@Z    5f8a5720 f i dllinit.obj
 0001:000a4790       ??_ECObList@@UAEPAXI@Z     5f8a5790 f i dllinit.obj
 0001:000a4800       ??_FCObList@@QAEXXZ        5f8a5800 f i dllinit.obj
 0001:000a4820       ??_ECPalette@@UAEPAXI@Z    5f8a5820 f i dllinit.obj
 0001:000a4890       ??_ECPen@@UAEPAXI@Z        5f8a5890 f i dllinit.obj
 0001:000a4900       ??_ECPtrArray@@UAEPAXI@Z   5f8a5900 f i dllinit.obj
 0001:000a4970       ??_ECPtrList@@UAEPAXI@Z    5f8a5970 f i dllinit.obj
 0001:000a49e0       ??_FCPtrList@@QAEXXZ       5f8a59e0 f i dllinit.obj
 0001:000a4a00       ??_ECRectTracker@@UAEPAXI@Z 5f8a5a00 f i dllinit.obj
 0001:000a4a70       ??_ECRgn@@UAEPAXI@Z        5f8a5a70 f i dllinit.obj
 0001:000a4ae0       ??_ECScrollBar@@UAEPAXI@Z  5f8a5ae0 f i dllinit.obj
 0001:000a4b50       ??_ECSharedFile@@UAEPAXI@Z 5f8a5b50 f i dllinit.obj
 0001:000a4bc0       ??_FCSharedFile@@QAEXXZ    5f8a5bc0 f i dllinit.obj
 0001:000a4be0       ??_ECSplitterWnd@@UAEPAXI@Z 5f8a5be0 f i dllinit.obj
 0001:000a4c50       ??_ECStatic@@UAEPAXI@Z     5f8a5c50 f i dllinit.obj
 0001:000a4cc0       ??_ECStatusBar@@UAEPAXI@Z  5f8a5cc0 f i dllinit.obj
 0001:000a4d30       ??_ECStdioFile@@UAEPAXI@Z  5f8a5d30 f i dllinit.obj
 0001:000a4da0       ??_ECStringArray@@UAEPAXI@Z 5f8a5da0 f i dllinit.obj
 0001:000a4e10       ??_ECStringList@@UAEPAXI@Z 5f8a5e10 f i dllinit.obj
 0001:000a4e80       ??_FCStringList@@QAEXXZ    5f8a5e80 f i dllinit.obj
 0001:000a4ea0       ??_ECToolBar@@UAEPAXI@Z    5f8a5ea0 f i dllinit.obj
 0001:000a4f10       ??_ECUIntArray@@UAEPAXI@Z  5f8a5f10 f i dllinit.obj
 0001:000a4f80       ??_ECWnd@@UAEPAXI@Z        5f8a5f80 f i dllinit.obj
 0001:000a4ff0       ??_ECWordArray@@UAEPAXI@Z  5f8a5ff0 f i dllinit.obj
 0001:000a5060       ??_ECFileFind@@UAEPAXI@Z   5f8a6060 f i dllinit.obj
 0001:000a50d0       ??_ECInternetSession@@UAEPAXI@Z 5f8a60d0 f i dllinit.obj
 0001:000a5140       ??_FCInternetSession@@QAEXXZ 5f8a6140 f i dllinit.obj
 0001:000a5160       ??_ECDragListBox@@UAEPAXI@Z 5f8a6160 f i dllinit.obj
 0001:000a51d0       ??_ECStatusBarCtrl@@UAEPAXI@Z 5f8a61d0 f i dllinit.obj
 0001:000a5240       ??_ECListCtrl@@UAEPAXI@Z   5f8a6240 f i dllinit.obj
 0001:000a52b0       ??_ECTreeCtrl@@UAEPAXI@Z   5f8a62b0 f i dllinit.obj
 0001:000a5320       ??_ECSpinButtonCtrl@@UAEPAXI@Z 5f8a6320 f i dllinit.obj
 0001:000a5390       ??_ECSliderCtrl@@UAEPAXI@Z 5f8a6390 f i dllinit.obj
 0001:000a5400       ??_ECProgressCtrl@@UAEPAXI@Z 5f8a6400 f i dllinit.obj
 0001:000a5470       ??_ECHeaderCtrl@@UAEPAXI@Z 5f8a6470 f i dllinit.obj
 0001:000a54e0       ??_ECHotKeyCtrl@@UAEPAXI@Z 5f8a64e0 f i dllinit.obj
 0001:000a5550       ??_ECToolTipCtrl@@UAEPAXI@Z 5f8a6550 f i dllinit.obj
 0001:000a55c0       ??_ECTabCtrl@@UAEPAXI@Z    5f8a65c0 f i dllinit.obj
 0001:000a5630       ??_ECAnimateCtrl@@UAEPAXI@Z 5f8a6630 f i dllinit.obj
 0001:000a56a0       ??_ECImageList@@UAEPAXI@Z  5f8a66a0 f i dllinit.obj
 0001:000a5710       ??_ECToolBarCtrl@@UAEPAXI@Z 5f8a6710 f i dllinit.obj
 0001:000a5780       ??_ECRichEditCtrl@@UAEPAXI@Z 5f8a6780 f i dllinit.obj
 0001:000a57f0       ??_ECMirrorFile@@UAEPAXI@Z 5f8a67f0 f i dllinit.obj
 0001:000a5860       ??_ECDockState@@UAEPAXI@Z  5f8a6860 f i dllinit.obj
 0001:000a58d0       ??_ECTreeView@@UAEPAXI@Z   5f8a68d0 f i dllinit.obj
 0001:000a58d0       ??_ECListView@@UAEPAXI@Z   5f8a68d0 f i dllinit.obj
 0001:000a5940       ??_ECCommandLineInfo@@UAEPAXI@Z 5f8a6940 f i dllinit.obj
 0001:000a59b0       ??_ECDocManager@@UAEPAXI@Z 5f8a69b0 f i dllinit.obj
 0001:000a5a20       ??_ECPageSetupDialog@@UAEPAXI@Z 5f8a6a20 f i dllinit.obj
 0001:000a5a90       ??_FCPageSetupDialog@@QAEXXZ 5f8a6a90 f i dllinit.obj
 0001:000a5ab0       ??_ECSemaphore@@UAEPAXI@Z  5f8a6ab0 f i dllinit.obj
 0001:000a5b20       ??_FCSemaphore@@QAEXXZ     5f8a6b20 f i dllinit.obj
 0001:000a5b40       ??_ECMutex@@UAEPAXI@Z      5f8a6b40 f i dllinit.obj
 0001:000a5bb0       ??_FCMutex@@QAEXXZ         5f8a6bb0 f i dllinit.obj
 0001:000a5bd0       ??_ECEvent@@UAEPAXI@Z      5f8a6bd0 f i dllinit.obj
 0001:000a5c40       ??_FCEvent@@QAEXXZ         5f8a6c40 f i dllinit.obj
 0001:000a5c60       ??_ECCriticalSection@@UAEPAXI@Z 5f8a6c60 f i dllinit.obj
 0001:000a5cd0       ?GetHead@?$CTypedSimpleList@PAVCOleObjectFactory@@@@QAEPAVCOleObjectFactory@@XZ 5f8a6cd0 f i dllinit.obj
 0001:000a5cd0       ?GetHead@?$CTypedSimpleList@PAUCRuntimeClass@@@@QAEPAUCRuntimeClass@@XZ 5f8a6cd0 f i dllinit.obj
 0001:000a5cf0       ?AddHead@?$CTypedSimpleList@PAVCDynLinkLibrary@@@@QAEXPAVCDynLinkLibrary@@@Z 5f8a6cf0 f i dllinit.obj
 0001:000a5d10       ?Remove@?$CTypedSimpleList@PAVCDynLinkLibrary@@@@QAEHPAVCDynLinkLibrary@@@Z 5f8a6d10 f i dllinit.obj
 0002:00000000       __imp__GetCharABCWidthsW@16 5f8ab000     gdi32:GDI32.dll
 0002:00000004       __imp__GetFontData@20      5f8ab004     gdi32:GDI32.dll
 0002:00000008       __imp__GetCharWidthW@16    5f8ab008     gdi32:GDI32.dll
 0002:0000000c       __imp__PlayMetaFile@8      5f8ab00c     gdi32:GDI32.dll
 0002:00000010       __imp__EnumMetaFile@16     5f8ab010     gdi32:GDI32.dll
 0002:00000014       __imp__PlayMetaFileRecord@16 5f8ab014     gdi32:GDI32.dll
 0002:00000018       __imp__ExtSelectClipRgn@12 5f8ab018     gdi32:GDI32.dll
 0002:0000001c       __imp__SelectClipPath@8    5f8ab01c     gdi32:GDI32.dll
 0002:00000020       __imp__GetClipRgn@8        5f8ab020     gdi32:GDI32.dll
 0002:00000024       __imp__PolyBezierTo@12     5f8ab024     gdi32:GDI32.dll
 0002:00000028       __imp__SetColorAdjustment@8 5f8ab028     gdi32:GDI32.dll
 0002:0000002c       __imp__PolylineTo@12       5f8ab02c     gdi32:GDI32.dll
 0002:00000030       __imp__PolyDraw@16         5f8ab030     gdi32:GDI32.dll
 0002:00000034       __imp__SetArcDirection@8   5f8ab034     gdi32:GDI32.dll
 0002:00000038       __imp__ArcTo@36            5f8ab038     gdi32:GDI32.dll
 0002:0000003c       __imp__SetMapperFlags@8    5f8ab03c     gdi32:GDI32.dll
 0002:00000040       __imp__SetTextCharacterExtra@8 5f8ab040     gdi32:GDI32.dll
 0002:00000044       __imp__SetTextJustification@12 5f8ab044     gdi32:GDI32.dll
 0002:00000048       __imp__SetTextAlign@8      5f8ab048     gdi32:GDI32.dll
 0002:0000004c       __imp__LineTo@12           5f8ab04c     gdi32:GDI32.dll
 0002:00000050       __imp__OffsetClipRgn@12    5f8ab050     gdi32:GDI32.dll
 0002:00000054       __imp__ExcludeClipRect@20  5f8ab054     gdi32:GDI32.dll
 0002:00000058       __imp__SelectClipRgn@8     5f8ab058     gdi32:GDI32.dll
 0002:0000005c       __imp__OffsetWindowOrgEx@16 5f8ab05c     gdi32:GDI32.dll
 0002:00000060       __imp__SetStretchBltMode@8 5f8ab060     gdi32:GDI32.dll
 0002:00000064       __imp__SetROP2@8           5f8ab064     gdi32:GDI32.dll
 0002:00000068       __imp__SetPolyFillMode@8   5f8ab068     gdi32:GDI32.dll
 0002:0000006c       __imp__SetBkMode@8         5f8ab06c     gdi32:GDI32.dll
 0002:00000070       __imp__SelectPalette@12    5f8ab070     gdi32:GDI32.dll
 0002:00000074       __imp__DeleteMetaFile@4    5f8ab074     gdi32:GDI32.dll
 0002:00000078       __imp__IntersectClipRect@20 5f8ab078     gdi32:GDI32.dll
 0002:0000007c       __imp__SetWindowOrgEx@16   5f8ab07c     gdi32:GDI32.dll
 0002:00000080       __imp__GetTextExtentPoint32A@16 5f8ab080     gdi32:GDI32.dll
 0002:00000084       __imp__MoveToEx@16         5f8ab084     gdi32:GDI32.dll
 0002:00000088       __imp__ScaleWindowExtEx@24 5f8ab088     gdi32:GDI32.dll
 0002:0000008c       __imp__SetWindowExtEx@16   5f8ab08c     gdi32:GDI32.dll
 0002:00000090       __imp__ScaleViewportExtEx@24 5f8ab090     gdi32:GDI32.dll
 0002:00000094       __imp__SetViewportExtEx@16 5f8ab094     gdi32:GDI32.dll
 0002:00000098       __imp__OffsetViewportOrgEx@16 5f8ab098     gdi32:GDI32.dll
 0002:0000009c       __imp__SetViewportOrgEx@16 5f8ab09c     gdi32:GDI32.dll
 0002:000000a0       __imp__SetMapMode@8        5f8ab0a0     gdi32:GDI32.dll
 0002:000000a4       __imp__RestoreDC@8         5f8ab0a4     gdi32:GDI32.dll
 0002:000000a8       __imp__SaveDC@4            5f8ab0a8     gdi32:GDI32.dll
 0002:000000ac       __imp__DeleteObject@4      5f8ab0ac     gdi32:GDI32.dll
 0002:000000b0       __imp__StretchDIBits@52    5f8ab0b0     gdi32:GDI32.dll
 0002:000000b4       __imp__DeleteDC@4          5f8ab0b4     gdi32:GDI32.dll
 0002:000000b8       __imp__SetBkColor@8        5f8ab0b8     gdi32:GDI32.dll
 0002:000000bc       __imp__SetTextColor@8      5f8ab0bc     gdi32:GDI32.dll
 0002:000000c0       __imp__GetClipBox@8        5f8ab0c0     gdi32:GDI32.dll
 0002:000000c4       __imp__GetDCOrgEx@8        5f8ab0c4     gdi32:GDI32.dll
 0002:000000c8       __imp__PlayEnhMetaFile@12  5f8ab0c8     gdi32:GDI32.dll
 0002:000000cc       __imp__GdiComment@12       5f8ab0cc     gdi32:GDI32.dll
 0002:000000d0       __imp__WidenPath@4         5f8ab0d0     gdi32:GDI32.dll
 0002:000000d4       __imp__StrokePath@4        5f8ab0d4     gdi32:GDI32.dll
 0002:000000d8       __imp__StrokeAndFillPath@4 5f8ab0d8     gdi32:GDI32.dll
 0002:000000dc       __imp__SetMiterLimit@12    5f8ab0dc     gdi32:GDI32.dll
 0002:000000e0       __imp__GetPath@16          5f8ab0e0     gdi32:GDI32.dll
 0002:000000e4       __imp__GetMiterLimit@8     5f8ab0e4     gdi32:GDI32.dll
 0002:000000e8       __imp__FlattenPath@4       5f8ab0e8     gdi32:GDI32.dll
 0002:000000ec       __imp__FillPath@4          5f8ab0ec     gdi32:GDI32.dll
 0002:000000f0       __imp__EndPath@4           5f8ab0f0     gdi32:GDI32.dll
 0002:000000f4       __imp__CloseFigure@4       5f8ab0f4     gdi32:GDI32.dll
 0002:000000f8       __imp__BeginPath@4         5f8ab0f8     gdi32:GDI32.dll
 0002:000000fc       __imp__AbortPath@4         5f8ab0fc     gdi32:GDI32.dll
 0002:00000100       __imp__GetCharWidthFloatW@16 5f8ab100     gdi32:GDI32.dll
 0002:00000104       __imp__GetCharABCWidthsFloatW@16 5f8ab104     gdi32:GDI32.dll
 0002:00000108       __imp__ExtEscape@24        5f8ab108     gdi32:GDI32.dll
 0002:0000010c       __imp__DrawEscape@16       5f8ab10c     gdi32:GDI32.dll
 0002:00000110       __imp__PolyBezier@12       5f8ab110     gdi32:GDI32.dll
 0002:00000114       __imp__GetCurrentObject@8  5f8ab114     gdi32:GDI32.dll
 0002:00000118       __imp__GetColorAdjustment@8 5f8ab118     gdi32:GDI32.dll
 0002:0000011c       __imp__PolyPolyline@16     5f8ab11c     gdi32:GDI32.dll
 0002:00000120       __imp__GetArcDirection@4   5f8ab120     gdi32:GDI32.dll
 0002:00000124       __imp__AngleArc@24         5f8ab124     gdi32:GDI32.dll
 0002:00000128       __imp__SetPixelV@16        5f8ab128     gdi32:GDI32.dll
 0002:0000012c       __imp__PlgBlt@40           5f8ab12c     gdi32:GDI32.dll
 0002:00000130       __imp__MaskBlt@48          5f8ab130     gdi32:GDI32.dll
 0002:00000134       __imp__EndDoc@4            5f8ab134     gdi32:GDI32.dll
 0002:00000138       __imp__AbortDoc@4          5f8ab138     gdi32:GDI32.dll
 0002:0000013c       __imp__SetAbortProc@8      5f8ab13c     gdi32:GDI32.dll
 0002:00000140       __imp__EndPage@4           5f8ab140     gdi32:GDI32.dll
 0002:00000144       __imp__StartPage@4         5f8ab144     gdi32:GDI32.dll
 0002:00000148       __imp__StartDocW@8         5f8ab148     gdi32:GDI32.dll
 0002:0000014c       __imp__GetGlyphOutlineW@28 5f8ab14c     gdi32:GDI32.dll
 0002:00000150       __imp__GetKerningPairsW@12 5f8ab150     gdi32:GDI32.dll
 0002:00000154       __imp__GetOutlineTextMetricsW@12 5f8ab154     gdi32:GDI32.dll
 0002:00000158       __imp__ResetDCW@8          5f8ab158     gdi32:GDI32.dll
 0002:0000015c       __imp__GetBoundsRect@12    5f8ab15c     gdi32:GDI32.dll
 0002:00000160       __imp__SetBoundsRect@12    5f8ab160     gdi32:GDI32.dll
 0002:00000164       __imp__Escape@20           5f8ab164     gdi32:GDI32.dll
 0002:00000168       __imp__GetAspectRatioFilterEx@8 5f8ab168     gdi32:GDI32.dll
 0002:0000016c       __imp__GetTextMetricsW@8   5f8ab16c     gdi32:GDI32.dll
 0002:00000170       __imp__GetTextFaceW@12     5f8ab170     gdi32:GDI32.dll
 0002:00000174       __imp__GetTextAlign@4      5f8ab174     gdi32:GDI32.dll
 0002:00000178       __imp__GetTextExtentPoint32W@16 5f8ab178     gdi32:GDI32.dll
 0002:0000017c       __imp__TextOutW@20         5f8ab17c     gdi32:GDI32.dll
 0002:00000180       __imp__ExtFloodFill@20     5f8ab180     gdi32:GDI32.dll
 0002:00000184       __imp__FloodFill@16        5f8ab184     gdi32:GDI32.dll
 0002:00000188       __imp__SetPixel@16         5f8ab188     gdi32:GDI32.dll
 0002:0000018c       __imp__GetPixel@12         5f8ab18c     gdi32:GDI32.dll
 0002:00000190       __imp__StretchBlt@44       5f8ab190     gdi32:GDI32.dll
 0002:00000194       __imp__BitBlt@36           5f8ab194     gdi32:GDI32.dll
 0002:00000198       __imp__PatBlt@24           5f8ab198     gdi32:GDI32.dll
 0002:0000019c       __imp__RoundRect@28        5f8ab19c     gdi32:GDI32.dll
 0002:000001a0       __imp__Rectangle@20        5f8ab1a0     gdi32:GDI32.dll
 0002:000001a4       __imp__PolyPolygon@16      5f8ab1a4     gdi32:GDI32.dll
 0002:000001a8       __imp__Polygon@12          5f8ab1a8     gdi32:GDI32.dll
 0002:000001ac       __imp__Pie@36              5f8ab1ac     gdi32:GDI32.dll
 0002:000001b0       __imp__Ellipse@20          5f8ab1b0     gdi32:GDI32.dll
 0002:000001b4       __imp__Chord@36            5f8ab1b4     gdi32:GDI32.dll
 0002:000001b8       __imp__Polyline@12         5f8ab1b8     gdi32:GDI32.dll
 0002:000001bc       __imp__Arc@36              5f8ab1bc     gdi32:GDI32.dll
 0002:000001c0       __imp__GetCurrentPositionEx@8 5f8ab1c0     gdi32:GDI32.dll
 0002:000001c4       __imp__RectVisible@8       5f8ab1c4     gdi32:GDI32.dll
 0002:000001c8       __imp__PtVisible@12        5f8ab1c8     gdi32:GDI32.dll
 0002:000001cc       __imp__PaintRgn@8          5f8ab1cc     gdi32:GDI32.dll
 0002:000001d0       __imp__InvertRgn@8         5f8ab1d0     gdi32:GDI32.dll
 0002:000001d4       __imp__FrameRgn@20         5f8ab1d4     gdi32:GDI32.dll
 0002:000001d8       __imp__FillRgn@12          5f8ab1d8     gdi32:GDI32.dll
 0002:000001dc       __imp__LPtoDP@12           5f8ab1dc     gdi32:GDI32.dll
 0002:000001e0       __imp__DPtoLP@12           5f8ab1e0     gdi32:GDI32.dll
 0002:000001e4       __imp__GetWindowExtEx@8    5f8ab1e4     gdi32:GDI32.dll
 0002:000001e8       __imp__GetWindowOrgEx@8    5f8ab1e8     gdi32:GDI32.dll
 0002:000001ec       __imp__GetViewportExtEx@8  5f8ab1ec     gdi32:GDI32.dll
 0002:000001f0       __imp__GetViewportOrgEx@8  5f8ab1f0     gdi32:GDI32.dll
 0002:000001f4       __imp__GetMapMode@4        5f8ab1f4     gdi32:GDI32.dll
 0002:000001f8       __imp__GetTextColor@4      5f8ab1f8     gdi32:GDI32.dll
 0002:000001fc       __imp__GetStretchBltMode@4 5f8ab1fc     gdi32:GDI32.dll
 0002:00000200       __imp__GetROP2@4           5f8ab200     gdi32:GDI32.dll
 0002:00000204       __imp__GetPolyFillMode@4   5f8ab204     gdi32:GDI32.dll
 0002:00000208       __imp__GetBkMode@4         5f8ab208     gdi32:GDI32.dll
 0002:0000020c       __imp__GetBkColor@4        5f8ab20c     gdi32:GDI32.dll
 0002:00000210       __imp__UpdateColors@4      5f8ab210     gdi32:GDI32.dll
 0002:00000214       __imp__RealizePalette@4    5f8ab214     gdi32:GDI32.dll
 0002:00000218       __imp__GetNearestColor@8   5f8ab218     gdi32:GDI32.dll
 0002:0000021c       __imp__SelectObject@8      5f8ab21c     gdi32:GDI32.dll
 0002:00000220       __imp__EnumObjects@16      5f8ab220     gdi32:GDI32.dll
 0002:00000224       __imp__SetBrushOrgEx@16    5f8ab224     gdi32:GDI32.dll
 0002:00000228       __imp__GetBrushOrgEx@8     5f8ab228     gdi32:GDI32.dll
 0002:0000022c       __imp__GetDeviceCaps@8     5f8ab22c     gdi32:GDI32.dll
 0002:00000230       __imp__CreateCompatibleDC@4 5f8ab230     gdi32:GDI32.dll
 0002:00000234       __imp__CreateICW@16        5f8ab234     gdi32:GDI32.dll
 0002:00000238       __imp__CreateDCW@16        5f8ab238     gdi32:GDI32.dll
 0002:0000023c       __imp__RectInRegion@8      5f8ab23c     gdi32:GDI32.dll
 0002:00000240       __imp__PtInRegion@12       5f8ab240     gdi32:GDI32.dll
 0002:00000244       __imp__GetRgnBox@8         5f8ab244     gdi32:GDI32.dll
 0002:00000248       __imp__OffsetRgn@12        5f8ab248     gdi32:GDI32.dll
 0002:0000024c       __imp__EqualRgn@8          5f8ab24c     gdi32:GDI32.dll
 0002:00000250       __imp__CombineRgn@16       5f8ab250     gdi32:GDI32.dll
 0002:00000254       __imp__SetRectRgn@20       5f8ab254     gdi32:GDI32.dll
 0002:00000258       __imp__GetRegionData@12    5f8ab258     gdi32:GDI32.dll
 0002:0000025c       __imp__ExtCreateRegion@12  5f8ab25c     gdi32:GDI32.dll
 0002:00000260       __imp__PathToRegion@4      5f8ab260     gdi32:GDI32.dll
 0002:00000264       __imp__CreateRoundRectRgn@24 5f8ab264     gdi32:GDI32.dll
 0002:00000268       __imp__CreatePolyPolygonRgn@16 5f8ab268     gdi32:GDI32.dll
 0002:0000026c       __imp__CreatePolygonRgn@12 5f8ab26c     gdi32:GDI32.dll
 0002:00000270       __imp__CreateEllipticRgnIndirect@4 5f8ab270     gdi32:GDI32.dll
 0002:00000274       __imp__CreateEllipticRgn@16 5f8ab274     gdi32:GDI32.dll
 0002:00000278       __imp__GetTextCharacterExtra@4 5f8ab278     gdi32:GDI32.dll
 0002:0000027c       __imp__CreateRectRgnIndirect@4 5f8ab27c     gdi32:GDI32.dll
 0002:00000280       __imp__CreateRectRgn@16    5f8ab280     gdi32:GDI32.dll
 0002:00000284       __imp__ResizePalette@8     5f8ab284     gdi32:GDI32.dll
 0002:00000288       __imp__GetNearestPaletteIndex@8 5f8ab288     gdi32:GDI32.dll
 0002:0000028c       __imp__AnimatePalette@16   5f8ab28c     gdi32:GDI32.dll
 0002:00000290       __imp__SetPaletteEntries@16 5f8ab290     gdi32:GDI32.dll
 0002:00000294       __imp__GetPaletteEntries@16 5f8ab294     gdi32:GDI32.dll
 0002:00000298       __imp__CreateHalftonePalette@4 5f8ab298     gdi32:GDI32.dll
 0002:0000029c       __imp__CreatePalette@4     5f8ab29c     gdi32:GDI32.dll
 0002:000002a0       __imp__CreateDiscardableBitmap@12 5f8ab2a0     gdi32:GDI32.dll
 0002:000002a4       __imp__CreateCompatibleBitmap@12 5f8ab2a4     gdi32:GDI32.dll
 0002:000002a8       __imp__GetBitmapDimensionEx@8 5f8ab2a8     gdi32:GDI32.dll
 0002:000002ac       __imp__SetBitmapDimensionEx@16 5f8ab2ac     gdi32:GDI32.dll
 0002:000002b0       __imp__GetBitmapBits@12    5f8ab2b0     gdi32:GDI32.dll
 0002:000002b4       __imp__SetBitmapBits@12    5f8ab2b4     gdi32:GDI32.dll
 0002:000002b8       __imp__CreateBitmapIndirect@4 5f8ab2b8     gdi32:GDI32.dll
 0002:000002bc       __imp__CreateBitmap@20     5f8ab2bc     gdi32:GDI32.dll
 0002:000002c0       __imp__CreateFontW@56      5f8ab2c0     gdi32:GDI32.dll
 0002:000002c4       __imp__CreateFontIndirectW@4 5f8ab2c4     gdi32:GDI32.dll
 0002:000002c8       __imp__CreateDIBPatternBrushPt@8 5f8ab2c8     gdi32:GDI32.dll
 0002:000002cc       __imp__CreatePatternBrush@4 5f8ab2cc     gdi32:GDI32.dll
 0002:000002d0       __imp__CreateBrushIndirect@4 5f8ab2d0     gdi32:GDI32.dll
 0002:000002d4       __imp__CreateHatchBrush@8  5f8ab2d4     gdi32:GDI32.dll
 0002:000002d8       __imp__CreateSolidBrush@4  5f8ab2d8     gdi32:GDI32.dll
 0002:000002dc       __imp__ExtCreatePen@20     5f8ab2dc     gdi32:GDI32.dll
 0002:000002e0       __imp__CreatePenIndirect@4 5f8ab2e0     gdi32:GDI32.dll
 0002:000002e4       __imp__CreatePen@12        5f8ab2e4     gdi32:GDI32.dll
 0002:000002e8       __imp__GetObjectType@4     5f8ab2e8     gdi32:GDI32.dll
 0002:000002ec       __imp__UnrealizeObject@4   5f8ab2ec     gdi32:GDI32.dll
 0002:000002f0       __imp__GetStockObject@4    5f8ab2f0     gdi32:GDI32.dll
 0002:000002f4       __imp__GetObjectW@12       5f8ab2f4     gdi32:GDI32.dll
 0002:000002f8       __imp__ExtTextOutW@32      5f8ab2f8     gdi32:GDI32.dll
 0002:000002fc       __imp__CloseEnhMetaFile@4  5f8ab2fc     gdi32:GDI32.dll
 0002:00000300       __imp__CreateEnhMetaFileW@16 5f8ab300     gdi32:GDI32.dll
 0002:00000304       __imp__CloseMetaFile@4     5f8ab304     gdi32:GDI32.dll
 0002:00000308       __imp__CreateMetaFileW@4   5f8ab308     gdi32:GDI32.dll
 0002:0000030c       \177GDI32_NULL_THUNK_DATA  5f8ab30c     gdi32:GDI32.dll
 0002:00000310       __imp__GetTempFileNameW@16 5f8ab310     kernel32:KERNEL32.dll
 0002:00000314       __imp__GetDiskFreeSpaceW@20 5f8ab314     kernel32:KERNEL32.dll
 0002:00000318       __imp__LocalUnlock@4       5f8ab318     kernel32:KERNEL32.dll
 0002:0000031c       __imp__LocalLock@4         5f8ab31c     kernel32:KERNEL32.dll
 0002:00000320       __imp__GetTempPathW@8      5f8ab320     kernel32:KERNEL32.dll
 0002:00000324       __imp__SearchPathW@24      5f8ab324     kernel32:KERNEL32.dll
 0002:00000328       __imp__GlobalFlags@4       5f8ab328     kernel32:KERNEL32.dll
 0002:0000032c       __imp__GetProcessVersion@4 5f8ab32c     kernel32:KERNEL32.dll
 0002:00000330       __imp__lstrcmpW@8          5f8ab330     kernel32:KERNEL32.dll
 0002:00000334       __imp__SetErrorMode@4      5f8ab334     kernel32:KERNEL32.dll
 0002:00000338       __imp__InterlockedExchange@8 5f8ab338     kernel32:KERNEL32.dll
 0002:0000033c       __imp__WritePrivateProfileStringW@16 5f8ab33c     kernel32:KERNEL32.dll
 0002:00000340       __imp__GetCurrentDirectoryW@8 5f8ab340     kernel32:KERNEL32.dll
 0002:00000344       __imp__FindNextFileW@8     5f8ab344     kernel32:KERNEL32.dll
 0002:00000348       __imp__lstrcatA@8          5f8ab348     kernel32:KERNEL32.dll
 0002:0000034c       __imp__GetSystemDirectoryA@8 5f8ab34c     kernel32:KERNEL32.dll
 0002:00000350       __imp__SizeofResource@8    5f8ab350     kernel32:KERNEL32.dll
 0002:00000354       __imp__lstrcpyA@8          5f8ab354     kernel32:KERNEL32.dll
 0002:00000358       __imp__VirtualProtect@16   5f8ab358     kernel32:KERNEL32.dll
 0002:0000035c       __imp__GetProfileIntW@12   5f8ab35c     kernel32:KERNEL32.dll
 0002:00000360       __imp__MulDiv@12           5f8ab360     kernel32:KERNEL32.dll
 0002:00000364       __imp__GetModuleHandleA@4  5f8ab364     kernel32:KERNEL32.dll
 0002:00000368       __imp__LoadLibraryA@4      5f8ab368     kernel32:KERNEL32.dll
 0002:0000036c       __imp__FreeLibrary@4       5f8ab36c     kernel32:KERNEL32.dll
 0002:00000370       __imp__FindResourceW@12    5f8ab370     kernel32:KERNEL32.dll
 0002:00000374       __imp__LoadResource@8      5f8ab374     kernel32:KERNEL32.dll
 0002:00000378       __imp__LockResource@4      5f8ab378     kernel32:KERNEL32.dll
 0002:0000037c       __imp__FreeResource@4      5f8ab37c     kernel32:KERNEL32.dll
 0002:00000380       __imp__GetVersion@0        5f8ab380     kernel32:KERNEL32.dll
 0002:00000384       __imp__lstrcatW@8          5f8ab384     kernel32:KERNEL32.dll
 0002:00000388       __imp__GetCurrentThreadId@0 5f8ab388     kernel32:KERNEL32.dll
 0002:0000038c       __imp__GlobalGetAtomNameW@12 5f8ab38c     kernel32:KERNEL32.dll
 0002:00000390       __imp__GlobalAddAtomW@4    5f8ab390     kernel32:KERNEL32.dll
 0002:00000394       __imp__GlobalFindAtomW@4   5f8ab394     kernel32:KERNEL32.dll
 0002:00000398       __imp__GlobalDeleteAtom@4  5f8ab398     kernel32:KERNEL32.dll
 0002:0000039c       __imp__GetModuleHandleW@4  5f8ab39c     kernel32:KERNEL32.dll
 0002:000003a0       __imp__WaitForMultipleObjects@16 5f8ab3a0     kernel32:KERNEL32.dll
 0002:000003a4       __imp__CreateEventW@16     5f8ab3a4     kernel32:KERNEL32.dll
 0002:000003a8       __imp__ReleaseMutex@4      5f8ab3a8     kernel32:KERNEL32.dll
 0002:000003ac       __imp__CreateMutexW@12     5f8ab3ac     kernel32:KERNEL32.dll
 0002:000003b0       __imp__ReleaseSemaphore@12 5f8ab3b0     kernel32:KERNEL32.dll
 0002:000003b4       __imp__CreateSemaphoreW@16 5f8ab3b4     kernel32:KERNEL32.dll
 0002:000003b8       __imp__ResetEvent@4        5f8ab3b8     kernel32:KERNEL32.dll
 0002:000003bc       __imp__PulseEvent@4        5f8ab3bc     kernel32:KERNEL32.dll
 0002:000003c0       __imp__SetEvent@4          5f8ab3c0     kernel32:KERNEL32.dll
 0002:000003c4       __imp__WaitForSingleObject@8 5f8ab3c4     kernel32:KERNEL32.dll
 0002:000003c8       __imp__TlsGetValue@4       5f8ab3c8     kernel32:KERNEL32.dll
 0002:000003cc       __imp__LocalReAlloc@12     5f8ab3cc     kernel32:KERNEL32.dll
 0002:000003d0       __imp__TlsSetValue@8       5f8ab3d0     kernel32:KERNEL32.dll
 0002:000003d4       __imp__EnterCriticalSection@4 5f8ab3d4     kernel32:KERNEL32.dll
 0002:000003d8       __imp__TlsFree@4           5f8ab3d8     kernel32:KERNEL32.dll
 0002:000003dc       __imp__GlobalHandle@4      5f8ab3dc     kernel32:KERNEL32.dll
 0002:000003e0       __imp__DeleteCriticalSection@4 5f8ab3e0     kernel32:KERNEL32.dll
 0002:000003e4       __imp__TlsAlloc@0          5f8ab3e4     kernel32:KERNEL32.dll
 0002:000003e8       __imp__InitializeCriticalSection@4 5f8ab3e8     kernel32:KERNEL32.dll
 0002:000003ec       __imp__LocalAlloc@8        5f8ab3ec     kernel32:KERNEL32.dll
 0002:000003f0       __imp__FileTimeToLocalFileTime@8 5f8ab3f0     kernel32:KERNEL32.dll
 0002:000003f4       __imp__FileTimeToSystemTime@8 5f8ab3f4     kernel32:KERNEL32.dll
 0002:000003f8       __imp__FormatMessageW@28   5f8ab3f8     kernel32:KERNEL32.dll
 0002:000003fc       __imp__LocalFree@4         5f8ab3fc     kernel32:KERNEL32.dll
 0002:00000400       __imp__MultiByteToWideChar@24 5f8ab400     kernel32:KERNEL32.dll
 0002:00000404       __imp__InterlockedDecrement@4 5f8ab404     kernel32:KERNEL32.dll
 0002:00000408       __imp__InterlockedIncrement@4 5f8ab408     kernel32:KERNEL32.dll
 0002:0000040c       __imp__SetFileAttributesW@8 5f8ab40c     kernel32:KERNEL32.dll
 0002:00000410       __imp__SetFileTime@16      5f8ab410     kernel32:KERNEL32.dll
 0002:00000414       __imp__SystemTimeToFileTime@8 5f8ab414     kernel32:KERNEL32.dll
 0002:00000418       __imp__LocalFileTimeToFileTime@8 5f8ab418     kernel32:KERNEL32.dll
 0002:0000041c       __imp__GetFileTime@16      5f8ab41c     kernel32:KERNEL32.dll
 0002:00000420       __imp__GetFileSize@8       5f8ab420     kernel32:KERNEL32.dll
 0002:00000424       __imp__GetFileAttributesW@4 5f8ab424     kernel32:KERNEL32.dll
 0002:00000428       __imp__GlobalFree@4        5f8ab428     kernel32:KERNEL32.dll
 0002:0000042c       __imp__GlobalUnlock@4      5f8ab42c     kernel32:KERNEL32.dll
 0002:00000430       __imp__GlobalReAlloc@12    5f8ab430     kernel32:KERNEL32.dll
 0002:00000434       __imp__GlobalAlloc@8       5f8ab434     kernel32:KERNEL32.dll
 0002:00000438       __imp__GlobalLock@4        5f8ab438     kernel32:KERNEL32.dll
 0002:0000043c       __imp__GlobalSize@4        5f8ab43c     kernel32:KERNEL32.dll
 0002:00000440       __imp__GetModuleFileNameW@12 5f8ab440     kernel32:KERNEL32.dll
 0002:00000444       __imp__GetShortPathNameW@12 5f8ab444     kernel32:KERNEL32.dll
 0002:00000448       __imp__lstrcmpiW@8         5f8ab448     kernel32:KERNEL32.dll
 0002:0000044c       __imp__GetThreadLocale@0   5f8ab44c     kernel32:KERNEL32.dll
 0002:00000450       __imp__GetStringTypeExW@20 5f8ab450     kernel32:KERNEL32.dll
 0002:00000454       __imp__GetFullPathNameW@16 5f8ab454     kernel32:KERNEL32.dll
 0002:00000458       __imp__GetVolumeInformationW@32 5f8ab458     kernel32:KERNEL32.dll
 0002:0000045c       __imp__FindFirstFileW@8    5f8ab45c     kernel32:KERNEL32.dll
 0002:00000460       __imp__FindClose@4         5f8ab460     kernel32:KERNEL32.dll
 0002:00000464       __imp__lstrcpyW@8          5f8ab464     kernel32:KERNEL32.dll
 0002:00000468       __imp__LoadLibraryW@4      5f8ab468     kernel32:KERNEL32.dll
 0002:0000046c       __imp__GetProcAddress@8    5f8ab46c     kernel32:KERNEL32.dll
 0002:00000470       __imp__DeleteFileW@4       5f8ab470     kernel32:KERNEL32.dll
 0002:00000474       __imp__MoveFileW@8         5f8ab474     kernel32:KERNEL32.dll
 0002:00000478       __imp__SetEndOfFile@4      5f8ab478     kernel32:KERNEL32.dll
 0002:0000047c       __imp__UnlockFile@20       5f8ab47c     kernel32:KERNEL32.dll
 0002:00000480       __imp__LockFile@20         5f8ab480     kernel32:KERNEL32.dll
 0002:00000484       __imp__CloseHandle@4       5f8ab484     kernel32:KERNEL32.dll
 0002:00000488       __imp__FlushFileBuffers@4  5f8ab488     kernel32:KERNEL32.dll
 0002:0000048c       __imp__SetFilePointer@16   5f8ab48c     kernel32:KERNEL32.dll
 0002:00000490       __imp__WriteFile@20        5f8ab490     kernel32:KERNEL32.dll
 0002:00000494       __imp__ReadFile@20         5f8ab494     kernel32:KERNEL32.dll
 0002:00000498       __imp__CreateFileW@28      5f8ab498     kernel32:KERNEL32.dll
 0002:0000049c       __imp__GetCurrentProcess@0 5f8ab49c     kernel32:KERNEL32.dll
 0002:000004a0       __imp__DuplicateHandle@28  5f8ab4a0     kernel32:KERNEL32.dll
 0002:000004a4       __imp__SuspendThread@4     5f8ab4a4     kernel32:KERNEL32.dll
 0002:000004a8       __imp__ResumeThread@4      5f8ab4a8     kernel32:KERNEL32.dll
 0002:000004ac       __imp__GetThreadPriority@4 5f8ab4ac     kernel32:KERNEL32.dll
 0002:000004b0       __imp__SetThreadPriority@8 5f8ab4b0     kernel32:KERNEL32.dll
 0002:000004b4       __imp__GetPrivateProfileIntW@16 5f8ab4b4     kernel32:KERNEL32.dll
 0002:000004b8       __imp__lstrlenA@4          5f8ab4b8     kernel32:KERNEL32.dll
 0002:000004bc       __imp__lstrcmpA@8          5f8ab4bc     kernel32:KERNEL32.dll
 0002:000004c0       __imp__WideCharToMultiByte@32 5f8ab4c0     kernel32:KERNEL32.dll
 0002:000004c4       __imp__lstrlenW@4          5f8ab4c4     kernel32:KERNEL32.dll
 0002:000004c8       __imp__IsBadReadPtr@8      5f8ab4c8     kernel32:KERNEL32.dll
 0002:000004cc       __imp__IsBadWritePtr@8     5f8ab4cc     kernel32:KERNEL32.dll
 0002:000004d0       __imp__IsBadStringPtrA@8   5f8ab4d0     kernel32:KERNEL32.dll
 0002:000004d4       __imp__IsBadStringPtrW@8   5f8ab4d4     kernel32:KERNEL32.dll
 0002:000004d8       __imp__lstrcpynW@12        5f8ab4d8     kernel32:KERNEL32.dll
 0002:000004dc       __imp__GetLastError@0      5f8ab4dc     kernel32:KERNEL32.dll
 0002:000004e0       __imp__SetLastError@4      5f8ab4e0     kernel32:KERNEL32.dll
 0002:000004e4       __imp__GetCurrentThread@0  5f8ab4e4     kernel32:KERNEL32.dll
 0002:000004e8       __imp__lstrcmpiA@8         5f8ab4e8     kernel32:KERNEL32.dll
 0002:000004ec       __imp__LeaveCriticalSection@4 5f8ab4ec     kernel32:KERNEL32.dll
 0002:000004f0       __imp__GetPrivateProfileStringW@24 5f8ab4f0     kernel32:KERNEL32.dll
 0002:000004f4       __imp__RaiseException@16   5f8ab4f4     kernel32:KERNEL32.dll
 0002:000004f8       \177KERNEL32_NULL_THUNK_DATA 5f8ab4f8     kernel32:KERNEL32.dll
 0002:000004fc       __imp___initterm           5f8ab4fc     msvcrtd:MSVCRTD.dll
 0002:00000500       __imp_?terminate@@YAXXZ    5f8ab500     msvcrtd:MSVCRTD.dll
 0002:00000504       __imp___onexit             5f8ab504     msvcrtd:MSVCRTD.dll
 0002:00000508       __imp___adjust_fdiv        5f8ab508     msvcrtd:MSVCRTD.dll
 0002:0000050c       __imp____dllonexit         5f8ab50c     msvcrtd:MSVCRTD.dll
 0002:00000510       __imp____CxxFrameHandler   5f8ab510     msvcrtd:MSVCRTD.dll
 0002:00000514       __imp___CrtDbgReport       5f8ab514     msvcrtd:MSVCRTD.dll
 0002:00000518       __imp_??1type_info@@UAE@XZ 5f8ab518     msvcrtd:MSVCRTD.dll
 0002:0000051c       __imp___wsplitpath         5f8ab51c     msvcrtd:MSVCRTD.dll
 0002:00000520       __imp___wfullpath          5f8ab520     msvcrtd:MSVCRTD.dll
 0002:00000524       __imp___wtol               5f8ab524     msvcrtd:MSVCRTD.dll
 0002:00000528       __imp____p___argc          5f8ab528     msvcrtd:MSVCRTD.dll
 0002:0000052c       __imp____p___wargv         5f8ab52c     msvcrtd:MSVCRTD.dll
 0002:00000530       __imp___beginthreadex      5f8ab530     msvcrtd:MSVCRTD.dll
 0002:00000534       __imp___endthreadex        5f8ab534     msvcrtd:MSVCRTD.dll
 0002:00000538       __imp___wcsdup             5f8ab538     msvcrtd:MSVCRTD.dll
 0002:0000053c       __imp___expand             5f8ab53c     msvcrtd:MSVCRTD.dll
 0002:00000540       __imp__swprintf            5f8ab540     msvcrtd:MSVCRTD.dll
 0002:00000544       __imp__wcstod              5f8ab544     msvcrtd:MSVCRTD.dll
 0002:00000548       __imp__wcstol              5f8ab548     msvcrtd:MSVCRTD.dll
 0002:0000054c       __imp__wcstoul             5f8ab54c     msvcrtd:MSVCRTD.dll
 0002:00000550       __imp__abs                 5f8ab550     msvcrtd:MSVCRTD.dll
 0002:00000554       __imp__calloc              5f8ab554     msvcrtd:MSVCRTD.dll
 0002:00000558       __imp___msize              5f8ab558     msvcrtd:MSVCRTD.dll
 0002:0000055c       __imp___purecall           5f8ab55c     msvcrtd:MSVCRTD.dll
 0002:00000560       __imp__wcsftime            5f8ab560     msvcrtd:MSVCRTD.dll
 0002:00000564       __imp__ctime               5f8ab564     msvcrtd:MSVCRTD.dll
 0002:00000568       __imp__localtime           5f8ab568     msvcrtd:MSVCRTD.dll
 0002:0000056c       __imp__gmtime              5f8ab56c     msvcrtd:MSVCRTD.dll
 0002:00000570       __imp__time                5f8ab570     msvcrtd:MSVCRTD.dll
 0002:00000574       __imp__mktime              5f8ab574     msvcrtd:MSVCRTD.dll
 0002:00000578       __imp__iswspace            5f8ab578     msvcrtd:MSVCRTD.dll
 0002:0000057c       __imp___wtoi               5f8ab57c     msvcrtd:MSVCRTD.dll
 0002:00000580       __imp__iswdigit            5f8ab580     msvcrtd:MSVCRTD.dll
 0002:00000584       __imp__wcsncmp             5f8ab584     msvcrtd:MSVCRTD.dll
 0002:00000588       __imp__wcslen              5f8ab588     msvcrtd:MSVCRTD.dll
 0002:0000058c       __imp__vswprintf           5f8ab58c     msvcrtd:MSVCRTD.dll
 0002:00000590       __imp__wcsrchr             5f8ab590     msvcrtd:MSVCRTD.dll
 0002:00000594       __imp__wcscspn             5f8ab594     msvcrtd:MSVCRTD.dll
 0002:00000598       __imp__wcsspn              5f8ab598     msvcrtd:MSVCRTD.dll
 0002:0000059c       __imp__wcsstr              5f8ab59c     msvcrtd:MSVCRTD.dll
 0002:000005a0       __imp___wcsrev             5f8ab5a0     msvcrtd:MSVCRTD.dll
 0002:000005a4       __imp___wcslwr             5f8ab5a4     msvcrtd:MSVCRTD.dll
 0002:000005a8       __imp___wcsupr             5f8ab5a8     msvcrtd:MSVCRTD.dll
 0002:000005ac       __imp__wcspbrk             5f8ab5ac     msvcrtd:MSVCRTD.dll
 0002:000005b0       __imp__free                5f8ab5b0     msvcrtd:MSVCRTD.dll
 0002:000005b4       __imp__realloc             5f8ab5b4     msvcrtd:MSVCRTD.dll
 0002:000005b8       __imp__malloc              5f8ab5b8     msvcrtd:MSVCRTD.dll
 0002:000005bc       __imp__fclose              5f8ab5bc     msvcrtd:MSVCRTD.dll
 0002:000005c0       __imp__fflush              5f8ab5c0     msvcrtd:MSVCRTD.dll
 0002:000005c4       __imp__fseek               5f8ab5c4     msvcrtd:MSVCRTD.dll
 0002:000005c8       __imp__ftell               5f8ab5c8     msvcrtd:MSVCRTD.dll
 0002:000005cc       __imp__fgetws              5f8ab5cc     msvcrtd:MSVCRTD.dll
 0002:000005d0       __imp__fputws              5f8ab5d0     msvcrtd:MSVCRTD.dll
 0002:000005d4       __imp__fwrite              5f8ab5d4     msvcrtd:MSVCRTD.dll
 0002:000005d8       __imp__fread               5f8ab5d8     msvcrtd:MSVCRTD.dll
 0002:000005dc       __imp__clearerr            5f8ab5dc     msvcrtd:MSVCRTD.dll
 0002:000005e0       __imp___open_osfhandle     5f8ab5e0     msvcrtd:MSVCRTD.dll
 0002:000005e4       __imp___fdopen             5f8ab5e4     msvcrtd:MSVCRTD.dll
 0002:000005e8       __imp____doserrno          5f8ab5e8     msvcrtd:MSVCRTD.dll
 0002:000005ec       __imp___get_osfhandle      5f8ab5ec     msvcrtd:MSVCRTD.dll
 0002:000005f0       __imp___wcsicoll           5f8ab5f0     msvcrtd:MSVCRTD.dll
 0002:000005f4       __imp__wcscoll             5f8ab5f4     msvcrtd:MSVCRTD.dll
 0002:000005f8       __imp___wcsicmp            5f8ab5f8     msvcrtd:MSVCRTD.dll
 0002:000005fc       __imp__wcscmp              5f8ab5fc     msvcrtd:MSVCRTD.dll
 0002:00000600       __imp__abort               5f8ab600     msvcrtd:MSVCRTD.dll
 0002:00000604       __imp___CrtDoForAllClientObjects 5f8ab604     msvcrtd:MSVCRTD.dll
 0002:00000608       __imp___CrtMemDumpAllObjectsSince 5f8ab608     msvcrtd:MSVCRTD.dll
 0002:0000060c       __imp___CrtMemCheckpoint   5f8ab60c     msvcrtd:MSVCRTD.dll
 0002:00000610       __imp___CrtMemDumpStatistics 5f8ab610     msvcrtd:MSVCRTD.dll
 0002:00000614       __imp___CrtMemDifference   5f8ab614     msvcrtd:MSVCRTD.dll
 0002:00000618       __imp__memset              5f8ab618     msvcrtd:MSVCRTD.dll
 0002:0000061c       __imp___CrtIsMemoryBlock   5f8ab61c     msvcrtd:MSVCRTD.dll
 0002:00000620       __imp___CrtCheckMemory     5f8ab620     msvcrtd:MSVCRTD.dll
 0002:00000624       __imp___CrtSetBreakAlloc   5f8ab624     msvcrtd:MSVCRTD.dll
 0002:00000628       __imp___CrtSetAllocHook    5f8ab628     msvcrtd:MSVCRTD.dll
 0002:0000062c       __imp___malloc_dbg         5f8ab62c     msvcrtd:MSVCRTD.dll
 0002:00000630       __imp___free_dbg           5f8ab630     msvcrtd:MSVCRTD.dll
 0002:00000634       __imp___vsnwprintf         5f8ab634     msvcrtd:MSVCRTD.dll
 0002:00000638       __imp___CrtDumpMemoryLeaks 5f8ab638     msvcrtd:MSVCRTD.dll
 0002:0000063c       __imp___CrtSetDbgFlag      5f8ab63c     msvcrtd:MSVCRTD.dll
 0002:00000640       __imp___CrtSetDumpClient   5f8ab640     msvcrtd:MSVCRTD.dll
 0002:00000644       __imp___CrtSetReportHook   5f8ab644     msvcrtd:MSVCRTD.dll
 0002:00000648       __imp___CrtSetReportMode   5f8ab648     msvcrtd:MSVCRTD.dll
 0002:0000064c       __imp___except_handler3    5f8ab64c     msvcrtd:MSVCRTD.dll
 0002:00000650       __imp__memcmp              5f8ab650     msvcrtd:MSVCRTD.dll
 0002:00000654       __imp__memmove             5f8ab654     msvcrtd:MSVCRTD.dll
 0002:00000658       __imp__memcpy              5f8ab658     msvcrtd:MSVCRTD.dll
 0002:0000065c       __imp___gcvt               5f8ab65c     msvcrtd:MSVCRTD.dll
 0002:00000660       __imp__wcschr              5f8ab660     msvcrtd:MSVCRTD.dll
 0002:00000664       __imp___CxxThrowException@8 5f8ab664     msvcrtd:MSVCRTD.dll
 0002:00000668       \177MSVCRTD_NULL_THUNK_DATA 5f8ab668     msvcrtd:MSVCRTD.dll
 0002:0000066c       __imp__OpenClipboard@4     5f8ab66c     user32:USER32.dll
 0002:00000670       __imp__PeekMessageW@20     5f8ab670     user32:USER32.dll
 0002:00000674       __imp__SendMessageW@16     5f8ab674     user32:USER32.dll
 0002:00000678       __imp__IsWindow@4          5f8ab678     user32:USER32.dll
 0002:0000067c       __imp__PostMessageW@16     5f8ab67c     user32:USER32.dll
 0002:00000680       __imp__TabbedTextOutW@32   5f8ab680     user32:USER32.dll
 0002:00000684       __imp__CopyRect@8          5f8ab684     user32:USER32.dll
 0002:00000688       __imp__IsRectEmpty@4       5f8ab688     user32:USER32.dll
 0002:0000068c       __imp__PtInRect@12         5f8ab68c     user32:USER32.dll
 0002:00000690       __imp__SetRect@20          5f8ab690     user32:USER32.dll
 0002:00000694       __imp__SetRectEmpty@4      5f8ab694     user32:USER32.dll
 0002:00000698       __imp__EqualRect@8         5f8ab698     user32:USER32.dll
 0002:0000069c       __imp__InflateRect@12      5f8ab69c     user32:USER32.dll
 0002:000006a0       __imp__OffsetRect@12       5f8ab6a0     user32:USER32.dll
 0002:000006a4       __imp__IntersectRect@12    5f8ab6a4     user32:USER32.dll
 0002:000006a8       __imp__UnionRect@12        5f8ab6a8     user32:USER32.dll
 0002:000006ac       __imp__SubtractRect@12     5f8ab6ac     user32:USER32.dll
 0002:000006b0       __imp__GetSysColorBrush@4  5f8ab6b0     user32:USER32.dll
 0002:000006b4       __imp__LoadBitmapW@8       5f8ab6b4     user32:USER32.dll
 0002:000006b8       __imp__WindowFromDC@4      5f8ab6b8     user32:USER32.dll
 0002:000006bc       __imp__ExcludeUpdateRgn@8  5f8ab6bc     user32:USER32.dll
 0002:000006c0       __imp__FillRect@12         5f8ab6c0     user32:USER32.dll
 0002:000006c4       __imp__FrameRect@12        5f8ab6c4     user32:USER32.dll
 0002:000006c8       __imp__InvertRect@8        5f8ab6c8     user32:USER32.dll
 0002:000006cc       __imp__DrawIcon@16         5f8ab6cc     user32:USER32.dll
 0002:000006d0       __imp__DrawStateW@40       5f8ab6d0     user32:USER32.dll
 0002:000006d4       __imp__DrawEdge@16         5f8ab6d4     user32:USER32.dll
 0002:000006d8       __imp__DrawFrameControl@16 5f8ab6d8     user32:USER32.dll
 0002:000006dc       __imp__DrawFocusRect@8     5f8ab6dc     user32:USER32.dll
 0002:000006e0       __imp__DrawTextW@20        5f8ab6e0     user32:USER32.dll
 0002:000006e4       __imp__GetTabbedTextExtentW@20 5f8ab6e4     user32:USER32.dll
 0002:000006e8       __imp__GrayStringW@36      5f8ab6e8     user32:USER32.dll
 0002:000006ec       __imp__ScrollDC@28         5f8ab6ec     user32:USER32.dll
 0002:000006f0       __imp__CreateMenu@0        5f8ab6f0     user32:USER32.dll
 0002:000006f4       __imp__CreatePopupMenu@0   5f8ab6f4     user32:USER32.dll
 0002:000006f8       __imp__IsMenu@4            5f8ab6f8     user32:USER32.dll
 0002:000006fc       __imp__DeleteMenu@12       5f8ab6fc     user32:USER32.dll
 0002:00000700       __imp__AppendMenuW@16      5f8ab700     user32:USER32.dll
 0002:00000704       __imp__CheckMenuItem@12    5f8ab704     user32:USER32.dll
 0002:00000708       __imp__EnableMenuItem@12   5f8ab708     user32:USER32.dll
 0002:0000070c       __imp__SetMenuDefaultItem@12 5f8ab70c     user32:USER32.dll
 0002:00000710       __imp__GetMenuDefaultItem@12 5f8ab710     user32:USER32.dll
 0002:00000714       __imp__GetMenuItemCount@4  5f8ab714     user32:USER32.dll
 0002:00000718       __imp__GetMenuItemID@8     5f8ab718     user32:USER32.dll
 0002:0000071c       __imp__GetMenuState@12     5f8ab71c     user32:USER32.dll
 0002:00000720       __imp__GetMenuStringW@20   5f8ab720     user32:USER32.dll
 0002:00000724       __imp__GetMenuItemInfoW@16 5f8ab724     user32:USER32.dll
 0002:00000728       __imp__GetSubMenu@8        5f8ab728     user32:USER32.dll
 0002:0000072c       __imp__InsertMenuW@20      5f8ab72c     user32:USER32.dll
 0002:00000730       __imp__ModifyMenuW@20      5f8ab730     user32:USER32.dll
 0002:00000734       __imp__RemoveMenu@12       5f8ab734     user32:USER32.dll
 0002:00000738       __imp__SetMenuItemBitmaps@20 5f8ab738     user32:USER32.dll
 0002:0000073c       __imp__LoadMenuW@8         5f8ab73c     user32:USER32.dll
 0002:00000740       __imp__LoadMenuIndirectW@4 5f8ab740     user32:USER32.dll
 0002:00000744       __imp__SetMenuContextHelpId@8 5f8ab744     user32:USER32.dll
 0002:00000748       __imp__GetMenuContextHelpId@4 5f8ab748     user32:USER32.dll
 0002:0000074c       __imp__CheckMenuRadioItem@20 5f8ab74c     user32:USER32.dll
 0002:00000750       __imp__GetMenu@4           5f8ab750     user32:USER32.dll
 0002:00000754       __imp__SetMenu@8           5f8ab754     user32:USER32.dll
 0002:00000758       __imp__DrawMenuBar@4       5f8ab758     user32:USER32.dll
 0002:0000075c       __imp__GetSystemMenu@8     5f8ab75c     user32:USER32.dll
 0002:00000760       __imp__HiliteMenuItem@16   5f8ab760     user32:USER32.dll
 0002:00000764       __imp__IsIconic@4          5f8ab764     user32:USER32.dll
 0002:00000768       __imp__IsZoomed@4          5f8ab768     user32:USER32.dll
 0002:0000076c       __imp__ArrangeIconicWindows@4 5f8ab76c     user32:USER32.dll
 0002:00000770       __imp__SetWindowRgn@12     5f8ab770     user32:USER32.dll
 0002:00000774       __imp__GetWindowRgn@8      5f8ab774     user32:USER32.dll
 0002:00000778       __imp__BringWindowToTop@4  5f8ab778     user32:USER32.dll
 0002:0000077c       __imp__GetWindowRect@8     5f8ab77c     user32:USER32.dll
 0002:00000780       __imp__GetClientRect@8     5f8ab780     user32:USER32.dll
 0002:00000784       __imp__MapWindowPoints@16  5f8ab784     user32:USER32.dll
 0002:00000788       __imp__ClientToScreen@8    5f8ab788     user32:USER32.dll
 0002:0000078c       __imp__ScreenToClient@8    5f8ab78c     user32:USER32.dll
 0002:00000790       __imp__BeginPaint@8        5f8ab790     user32:USER32.dll
 0002:00000794       __imp__EndPaint@8          5f8ab794     user32:USER32.dll
 0002:00000798       __imp__GetDC@4             5f8ab798     user32:USER32.dll
 0002:0000079c       __imp__GetWindowDC@4       5f8ab79c     user32:USER32.dll
 0002:000007a0       __imp__ReleaseDC@8         5f8ab7a0     user32:USER32.dll
 0002:000007a4       __imp__UpdateWindow@4      5f8ab7a4     user32:USER32.dll
 0002:000007a8       __imp__GetUpdateRect@12    5f8ab7a8     user32:USER32.dll
 0002:000007ac       __imp__GetUpdateRgn@12     5f8ab7ac     user32:USER32.dll
 0002:000007b0       __imp__InvalidateRect@12   5f8ab7b0     user32:USER32.dll
 0002:000007b4       __imp__InvalidateRgn@12    5f8ab7b4     user32:USER32.dll
 0002:000007b8       __imp__ValidateRect@8      5f8ab7b8     user32:USER32.dll
 0002:000007bc       __imp__ValidateRgn@8       5f8ab7bc     user32:USER32.dll
 0002:000007c0       __imp__IsWindowVisible@4   5f8ab7c0     user32:USER32.dll
 0002:000007c4       __imp__ShowOwnedPopups@8   5f8ab7c4     user32:USER32.dll
 0002:000007c8       __imp__GetDCEx@12          5f8ab7c8     user32:USER32.dll
 0002:000007cc       __imp__LockWindowUpdate@4  5f8ab7cc     user32:USER32.dll
 0002:000007d0       __imp__RedrawWindow@16     5f8ab7d0     user32:USER32.dll
 0002:000007d4       __imp__EnableScrollBar@12  5f8ab7d4     user32:USER32.dll
 0002:000007d8       __imp__SetTimer@16         5f8ab7d8     user32:USER32.dll
 0002:000007dc       __imp__KillTimer@8         5f8ab7dc     user32:USER32.dll
 0002:000007e0       __imp__GetActiveWindow@0   5f8ab7e0     user32:USER32.dll
 0002:000007e4       __imp__SetActiveWindow@4   5f8ab7e4     user32:USER32.dll
 0002:000007e8       __imp__GetCapture@0        5f8ab7e8     user32:USER32.dll
 0002:000007ec       __imp__SetCapture@4        5f8ab7ec     user32:USER32.dll
 0002:000007f0       __imp__GetFocus@0          5f8ab7f0     user32:USER32.dll
 0002:000007f4       __imp__GetDesktopWindow@0  5f8ab7f4     user32:USER32.dll
 0002:000007f8       __imp__DlgDirListW@20      5f8ab7f8     user32:USER32.dll
 0002:000007fc       __imp__DlgDirListComboBoxW@20 5f8ab7fc     user32:USER32.dll
 0002:00000800       __imp__DlgDirSelectExW@16  5f8ab800     user32:USER32.dll
 0002:00000804       __imp__DlgDirSelectComboBoxExW@16 5f8ab804     user32:USER32.dll
 0002:00000808       __imp__GetNextDlgGroupItem@12 5f8ab808     user32:USER32.dll
 0002:0000080c       __imp__GetNextDlgTabItem@12 5f8ab80c     user32:USER32.dll
 0002:00000810       __imp__ShowScrollBar@12    5f8ab810     user32:USER32.dll
 0002:00000814       __imp__ChildWindowFromPoint@12 5f8ab814     user32:USER32.dll
 0002:00000818       __imp__ChildWindowFromPointEx@16 5f8ab818     user32:USER32.dll
 0002:0000081c       __imp__FindWindowW@8       5f8ab81c     user32:USER32.dll
 0002:00000820       __imp__GetWindow@8         5f8ab820     user32:USER32.dll
 0002:00000824       __imp__GetTopWindow@4      5f8ab824     user32:USER32.dll
 0002:00000828       __imp__GetLastActivePopup@4 5f8ab828     user32:USER32.dll
 0002:0000082c       __imp__IsChild@8           5f8ab82c     user32:USER32.dll
 0002:00000830       __imp__GetParent@4         5f8ab830     user32:USER32.dll
 0002:00000834       __imp__SetParent@8         5f8ab834     user32:USER32.dll
 0002:00000838       __imp__WindowFromPoint@8   5f8ab838     user32:USER32.dll
 0002:0000083c       __imp__FlashWindow@8       5f8ab83c     user32:USER32.dll
 0002:00000840       __imp__ChangeClipboardChain@8 5f8ab840     user32:USER32.dll
 0002:00000844       __imp__SetClipboardViewer@4 5f8ab844     user32:USER32.dll
 0002:00000848       __imp__PostQuitMessage@4   5f8ab848     user32:USER32.dll
 0002:0000084c       __imp__GetOpenClipboardWindow@0 5f8ab84c     user32:USER32.dll
 0002:00000850       __imp__GetClipboardOwner@0 5f8ab850     user32:USER32.dll
 0002:00000854       __imp__GetClipboardViewer@0 5f8ab854     user32:USER32.dll
 0002:00000858       __imp__CreateCaret@16      5f8ab858     user32:USER32.dll
 0002:0000085c       __imp__GetCaretPos@4       5f8ab85c     user32:USER32.dll
 0002:00000860       __imp__SetCaretPos@8       5f8ab860     user32:USER32.dll
 0002:00000864       __imp__HideCaret@4         5f8ab864     user32:USER32.dll
 0002:00000868       __imp__ShowCaret@4         5f8ab868     user32:USER32.dll
 0002:0000086c       __imp__SetForegroundWindow@4 5f8ab86c     user32:USER32.dll
 0002:00000870       __imp__GetForegroundWindow@0 5f8ab870     user32:USER32.dll
 0002:00000874       __imp__SendNotifyMessageW@16 5f8ab874     user32:USER32.dll
 0002:00000878       __imp__SetWindowContextHelpId@8 5f8ab878     user32:USER32.dll
 0002:0000087c       __imp__GetWindowContextHelpId@4 5f8ab87c     user32:USER32.dll
 0002:00000880       __imp__EnableWindow@8      5f8ab880     user32:USER32.dll
 0002:00000884       __imp__MapDialogRect@8     5f8ab884     user32:USER32.dll
 0002:00000888       __imp__GetWindowLongW@8    5f8ab888     user32:USER32.dll
 0002:0000088c       __imp__GetScrollPos@8      5f8ab88c     user32:USER32.dll
 0002:00000890       __imp__SetScrollPos@16     5f8ab890     user32:USER32.dll
 0002:00000894       __imp__GetScrollRange@16   5f8ab894     user32:USER32.dll
 0002:00000898       __imp__SetScrollRange@20   5f8ab898     user32:USER32.dll
 0002:0000089c       __imp__PostThreadMessageW@16 5f8ab89c     user32:USER32.dll
 0002:000008a0       __imp__LoadCursorW@8       5f8ab8a0     user32:USER32.dll
 0002:000008a4       __imp__LoadIconW@8         5f8ab8a4     user32:USER32.dll
 0002:000008a8       __imp__CloseWindow@4       5f8ab8a8     user32:USER32.dll
 0002:000008ac       __imp__OpenIcon@4          5f8ab8ac     user32:USER32.dll
 0002:000008b0       __imp__CharUpperW@4        5f8ab8b0     user32:USER32.dll
 0002:000008b4       __imp__GetSystemMetrics@4  5f8ab8b4     user32:USER32.dll
 0002:000008b8       __imp__UnhookWindowsHookEx@4 5f8ab8b8     user32:USER32.dll
 0002:000008bc       __imp__MsgWaitForMultipleObjects@20 5f8ab8bc     user32:USER32.dll
 0002:000008c0       __imp__GetWindowPlacement@8 5f8ab8c0     user32:USER32.dll
 0002:000008c4       __imp__SystemParametersInfoW@16 5f8ab8c4     user32:USER32.dll
 0002:000008c8       __imp__RegisterWindowMessageW@4 5f8ab8c8     user32:USER32.dll
 0002:000008cc       __imp__SetWindowPos@28     5f8ab8cc     user32:USER32.dll
 0002:000008d0       __imp__SetWindowLongW@12   5f8ab8d0     user32:USER32.dll
 0002:000008d4       __imp__GetMessagePos@0     5f8ab8d4     user32:USER32.dll
 0002:000008d8       __imp__GetMessageTime@0    5f8ab8d8     user32:USER32.dll
 0002:000008dc       __imp__RemovePropW@8       5f8ab8dc     user32:USER32.dll
 0002:000008e0       __imp__CallWindowProcW@20  5f8ab8e0     user32:USER32.dll
 0002:000008e4       __imp__GetPropW@8          5f8ab8e4     user32:USER32.dll
 0002:000008e8       __imp__SetPropW@12         5f8ab8e8     user32:USER32.dll
 0002:000008ec       __imp__GetClassLongW@8     5f8ab8ec     user32:USER32.dll
 0002:000008f0       __imp__CallNextHookEx@16   5f8ab8f0     user32:USER32.dll
 0002:000008f4       __imp__SetWindowsHookExW@16 5f8ab8f4     user32:USER32.dll
 0002:000008f8       __imp__CreateWindowExW@48  5f8ab8f8     user32:USER32.dll
 0002:000008fc       __imp__GetDlgCtrlID@4      5f8ab8fc     user32:USER32.dll
 0002:00000900       __imp__GetClassNameW@12    5f8ab900     user32:USER32.dll
 0002:00000904       __imp__DefWindowProcW@16   5f8ab904     user32:USER32.dll
 0002:00000908       __imp__DestroyWindow@4     5f8ab908     user32:USER32.dll
 0002:0000090c       __imp__GetKeyState@4       5f8ab90c     user32:USER32.dll
 0002:00000910       __imp__GetWindowTextW@12   5f8ab910     user32:USER32.dll
 0002:00000914       __imp__GetWindowTextLengthW@4 5f8ab914     user32:USER32.dll
 0002:00000918       __imp__GetDlgItem@8        5f8ab918     user32:USER32.dll
 0002:0000091c       __imp__SetWindowPlacement@8 5f8ab91c     user32:USER32.dll
 0002:00000920       __imp__TrackPopupMenu@28   5f8ab920     user32:USER32.dll
 0002:00000924       __imp__RegisterClassW@4    5f8ab924     user32:USER32.dll
 0002:00000928       __imp__GetClassInfoW@12    5f8ab928     user32:USER32.dll
 0002:0000092c       __imp__WinHelpW@16         5f8ab92c     user32:USER32.dll
 0002:00000930       __imp__MessageBoxW@16      5f8ab930     user32:USER32.dll
 0002:00000934       __imp__SetScrollInfo@16    5f8ab934     user32:USER32.dll
 0002:00000938       __imp__GetScrollInfo@12    5f8ab938     user32:USER32.dll
 0002:0000093c       __imp__ScrollWindow@20     5f8ab93c     user32:USER32.dll
 0002:00000940       __imp__EndDeferWindowPos@4 5f8ab940     user32:USER32.dll
 0002:00000944       __imp__BeginDeferWindowPos@4 5f8ab944     user32:USER32.dll
 0002:00000948       __imp__DeferWindowPos@32   5f8ab948     user32:USER32.dll
 0002:0000094c       __imp__AdjustWindowRectEx@16 5f8ab94c     user32:USER32.dll
 0002:00000950       __imp__SetFocus@4          5f8ab950     user32:USER32.dll
 0002:00000954       __imp__DispatchMessageW@4  5f8ab954     user32:USER32.dll
 0002:00000958       __imp__GetSysColor@4       5f8ab958     user32:USER32.dll
 0002:0000095c       __imp__SendDlgItemMessageA@20 5f8ab95c     user32:USER32.dll
 0002:00000960       __imp__SendDlgItemMessageW@20 5f8ab960     user32:USER32.dll
 0002:00000964       __imp__LoadAcceleratorsW@8 5f8ab964     user32:USER32.dll
 0002:00000968       __imp__TranslateAcceleratorW@12 5f8ab968     user32:USER32.dll
 0002:0000096c       __imp__ReleaseCapture@0    5f8ab96c     user32:USER32.dll
 0002:00000970       __imp__SetCursor@4         5f8ab970     user32:USER32.dll
 0002:00000974       __imp__IsWindowEnabled@4   5f8ab974     user32:USER32.dll
 0002:00000978       __imp__ShowWindow@8        5f8ab978     user32:USER32.dll
 0002:0000097c       __imp__DestroyMenu@4       5f8ab97c     user32:USER32.dll
 0002:00000980       __imp__ReuseDDElParam@20   5f8ab980     user32:USER32.dll
 0002:00000984       __imp__UnpackDDElParam@16  5f8ab984     user32:USER32.dll
 0002:00000988       __imp__WaitMessage@0       5f8ab988     user32:USER32.dll
 0002:0000098c       __imp__GetCursorPos@4      5f8ab98c     user32:USER32.dll
 0002:00000990       __imp__GetWindowThreadProcessId@8 5f8ab990     user32:USER32.dll
 0002:00000994       __imp__TranslateMessage@4  5f8ab994     user32:USER32.dll
 0002:00000998       __imp__GetMessageW@16      5f8ab998     user32:USER32.dll
 0002:0000099c       __imp__DefFrameProcW@20    5f8ab99c     user32:USER32.dll
 0002:000009a0       __imp__TranslateMDISysAccel@8 5f8ab9a0     user32:USER32.dll
 0002:000009a4       __imp__DefMDIChildProcW@16 5f8ab9a4     user32:USER32.dll
 0002:000009a8       __imp__GetTabbedTextExtentA@20 5f8ab9a8     user32:USER32.dll
 0002:000009ac       __imp__CreateDialogIndirectParamW@20 5f8ab9ac     user32:USER32.dll
 0002:000009b0       __imp__EndDialog@8         5f8ab9b0     user32:USER32.dll
 0002:000009b4       __imp__wvsprintfW@12       5f8ab9b4     user32:USER32.dll
 0002:000009b8       __imp__GetAsyncKeyState@4  5f8ab9b8     user32:USER32.dll
 0002:000009bc       __imp__GetDialogBaseUnits@0 5f8ab9bc     user32:USER32.dll
 0002:000009c0       __imp__GetClipboardFormatNameA@12 5f8ab9c0     user32:USER32.dll
 0002:000009c4       __imp__GetClipboardFormatNameW@12 5f8ab9c4     user32:USER32.dll
 0002:000009c8       __imp__SetWindowTextW@8    5f8ab9c8     user32:USER32.dll
 0002:000009cc       __imp__CheckDlgButton@12   5f8ab9cc     user32:USER32.dll
 0002:000009d0       __imp__CheckRadioButton@16 5f8ab9d0     user32:USER32.dll
 0002:000009d4       __imp__GetDlgItemInt@16    5f8ab9d4     user32:USER32.dll
 0002:000009d8       __imp__GetDlgItemTextW@16  5f8ab9d8     user32:USER32.dll
 0002:000009dc       __imp__SetDlgItemInt@16    5f8ab9dc     user32:USER32.dll
 0002:000009e0       __imp__SetDlgItemTextW@12  5f8ab9e0     user32:USER32.dll
 0002:000009e4       __imp__IsDlgButtonChecked@8 5f8ab9e4     user32:USER32.dll
 0002:000009e8       __imp__ScrollWindowEx@32   5f8ab9e8     user32:USER32.dll
 0002:000009ec       __imp__IsDialogMessageW@8  5f8ab9ec     user32:USER32.dll
 0002:000009f0       __imp__MoveWindow@24       5f8ab9f0     user32:USER32.dll
 0002:000009f4       __imp__GetMenuCheckMarkDimensions@0 5f8ab9f4     user32:USER32.dll
 0002:000009f8       __imp__DestroyIcon@4       5f8ab9f8     user32:USER32.dll
 0002:000009fc       __imp__SetCursorPos@8      5f8ab9fc     user32:USER32.dll
 0002:00000a00       __imp__DestroyCursor@4     5f8aba00     user32:USER32.dll
 0002:00000a04       __imp__IsClipboardFormatAvailable@4 5f8aba04     user32:USER32.dll
 0002:00000a08       __imp__MessageBeep@4       5f8aba08     user32:USER32.dll
 0002:00000a0c       __imp__UnregisterClassW@8  5f8aba0c     user32:USER32.dll
 0002:00000a10       __imp__LoadStringW@16      5f8aba10     user32:USER32.dll
 0002:00000a14       __imp__MessageBoxA@16      5f8aba14     user32:USER32.dll
 0002:00000a18       __imp__wsprintfA           5f8aba18     user32:USER32.dll
 0002:00000a1c       __imp__wsprintfW           5f8aba1c     user32:USER32.dll
 0002:00000a20       \177USER32_NULL_THUNK_DATA 5f8aba20     user32:USER32.dll
 0002:00000a50       ?classCObject@CObject@@2UCRuntimeClass@@B 5f8aba50     objcore.obj
 0002:00000a68       ??_C@_07EFMO@CObject?$AA@  5f8aba68     objcore.obj
 0002:00000a70       ??_C@_1GC@OANJ@?$AAA?$AAS?$AAS?$AAE?$AAR?$AAT?$AA_?$AAV?$AAA?$AAL?$AAI?$AAD?$AA?5?$AAf?$AAa?$AAi?$AAl?$AAs?$AA?5?$AAw@ 5f8aba70     objcore.obj
 0002:00000ad4       ??_C@_1FE@IBFO@?$AAA?$AAS?$AAS?$AAE?$AAR?$AAT?$AA_?$AAV?$AAA?$AAL?$AAI?$AAD?$AA?5?$AAf?$AAa?$AAi?$AAl?$AAs?$AA?5?$AAw@ 5f8abad4     objcore.obj
 0002:00000b28       ??_C@_15DEDE@?$AA?$CF?$AAs?$AA?$AA@ 5f8abb28     objcore.obj
 0002:00000b30       ??_C@_1EO@MGBE@?$AAA?$AAS?$AAS?$AAE?$AAR?$AAT?$AA_?$AAV?$AAA?$AAL?$AAI?$AAD?$AA?5?$AAf?$AAa?$AAi?$AAl?$AAs?$AA?5?$AAw@ 5f8abb30     objcore.obj
 0002:00000b80       ??_C@_02DLLN@a?5?$AA@      5f8abb80     objcore.obj
 0002:00000b84       ??_C@_04CCDP@?5at?5?$AA@   5f8abb84     objcore.obj
 0002:00000b8c       ??_C@_01BJG@?6?$AA@        5f8abb8c     objcore.obj
 0002:00000b90       ??_C@_1LA@PGEA@?$AAE?$AAr?$AAr?$AAo?$AAr?$AA?3?$AA?5?$AAT?$AAr?$AAy?$AAi?$AAn?$AAg?$AA?5?$AAt?$AAo?$AA?5?$AAc?$AAr?$AAe@ 5f8abb90     objcore.obj
 0002:00000c40       ?classCNotSupportedException@CNotSupportedException@@2UCRuntimeClass@@B 5f8abc40     except.obj
 0002:00000c58       ??_C@_0BH@JODH@CNotSupportedException?$AA@ 5f8abc58     except.obj
 0002:00000c70       ?classCMemoryException@CMemoryException@@2UCRuntimeClass@@B 5f8abc70     except.obj
 0002:00000c88       ??_C@_0BB@NODM@CMemoryException?$AA@ 5f8abc88     except.obj
 0002:00000ca0       ?classCException@CException@@2UCRuntimeClass@@B 5f8abca0     except.obj
 0002:00000cb8       ??_C@_0L@CMNH@CException?$AA@ 5f8abcb8     except.obj
 0002:00000cc4       ??_C@_0L@EMID@except?4cpp?$AA@ 5f8abcc4     except.obj
 0002:00000cd4       ??_7CException@@6B@        5f8abcd4     except.obj
 0002:00000cf0       ??_C@_0CH@KFAI@E?3?28168?2vc98?2mfc?2mfc?2include?2afx@ 5f8abcf0     except.obj
 0002:00000d18       ??_C@_02DILL@?$CFs?$AA@    5f8abd18     dumpcont.obj
 0002:00000d1c       ??_C@_1O@DAJD@?$AA?$CI?$AAN?$AAU?$AAL?$AAL?$AA?$CJ?$AA?$AA@ 5f8abd1c     dumpcont.obj
 0002:00000d2c       ??_C@_15KLDP@?$AA?$CF?$AAd?$AA?$AA@ 5f8abd2c     dumpcont.obj
 0002:00000d34       ??_C@_15NIED@?$AA?$CF?$AAu?$AA?$AA@ 5f8abd34     dumpcont.obj
 0002:00000d3c       ??_C@_19JHMD@?$AA0?$AAx?$AA?$CF?$AAX?$AA?$AA@ 5f8abd3c     dumpcont.obj
 0002:00000d48       ??_C@_17EFBD@?$AA?$CF?$AAl?$AAd?$AA?$AA@ 5f8abd48     dumpcont.obj
 0002:00000d50       ??_C@_17DGGP@?$AA?$CF?$AAl?$AAu?$AA?$AA@ 5f8abd50     dumpcont.obj
 0002:00000d58       ??_C@_19KF@?$AAN?$AAU?$AAL?$AAL?$AA?$AA@ 5f8abd58     dumpcont.obj
 0002:00000d64       ??_C@_19LOGG@?$AA$?$AA?$CF?$AAl?$AAX?$AA?$AA@ 5f8abd64     dumpcont.obj
 0002:00000d70       ??_C@_13DEJI@?$AA?6?$AA?$AA@ 5f8abd70     dumpcont.obj
 0002:00000d74       ??_C@_1M@JKLL@?$AA?5?$AA?$CF?$AA0?$AA2?$AAX?$AA?$AA@ 5f8abd74     dumpcont.obj
 0002:00000d80       ??_C@_08PEKM@lpa?5?$CB?$DN?50?$AA@ 5f8abd80     dumpcont.obj
 0002:00000d8c       ??_C@_0CH@IIKL@E?3?28168?2vc98?2mfc?2atl?2include?2atl@ 5f8abd8c     dumpcont.obj
 0002:00000db4       ??_C@_08NDGO@lpw?5?$CB?$DN?50?$AA@ 5f8abdb4     dumpcont.obj
 0002:00000dc0       ??_C@_1HI@FMGH@?$AAW?$AAa?$AAr?$AAn?$AAi?$AAn?$AAg?$AA?3?$AA?5?$AAC?$AAa?$AAn?$AAn?$AAo?$AAt?$AA?5?$AAl?$AAo?$AAa?$AAd@ 5f8abdc0     arccore.obj
 0002:00000e38       ??_C@_1GM@INHD@?$AAW?$AAa?$AAr?$AAn?$AAi?$AAn?$AAg?$AA?3?$AA?5?$AAC?$AAa?$AAn?$AAn?$AAo?$AAt?$AA?5?$AAc?$AAa?$AAl?$AAl@ 5f8abe38     arcobj.obj
 0002:00000ea4       ??_C@_1GI@EPDB@?$AAW?$AAa?$AAr?$AAn?$AAi?$AAn?$AAg?$AA?3?$AA?5?$AAC?$AAa?$AAn?$AAn?$AAo?$AAt?$AA?5?$AAc?$AAa?$AAl?$AAl@ 5f8abea4     arcobj.obj
 0002:00000f10       ?classCArchiveException@CArchiveException@@2UCRuntimeClass@@B 5f8abf10     arcex.obj
 0002:00000f28       ??_C@_0BC@BIF@CArchiveException?$AA@ 5f8abf28     arcex.obj
 0002:00000f64       ??_C@_09GHEH@badSchema?$AA@ 5f8abf64     arcex.obj
 0002:00000f70       ??_C@_08PPOL@badClass?$AA@ 5f8abf70     arcex.obj
 0002:00000f7c       ??_C@_08FIDE@badIndex?$AA@ 5f8abf7c     arcex.obj
 0002:00000f88       ??_C@_09HDPC@writeOnly?$AA@ 5f8abf88     arcex.obj
 0002:00000f94       ??_C@_09CLBG@endOfFile?$AA@ 5f8abf94     arcex.obj
 0002:00000fa0       ??_C@_08DEHK@readOnly?$AA@ 5f8abfa0     arcex.obj
 0002:00000fac       ??_C@_07LFGH@generic?$AA@  5f8abfac     arcex.obj
 0002:00000fb4       ??_C@_04KIKH@none?$AA@     5f8abfb4     arcex.obj
 0002:00000fbc       ??_C@_0M@EBCL@?5m_cause?5?$DN?5?$AA@ 5f8abfbc     arcex.obj
 0002:00000fc8       ??_C@_1DE@DAPO@?$AAC?$AAA?$AAr?$AAc?$AAh?$AAi?$AAv?$AAe?$AA?5?$AAe?$AAx?$AAc?$AAe?$AAp?$AAt?$AAi?$AAo?$AAn?$AA?3?$AA?5@ 5f8abfc8     arcex.obj
 0002:00001000       ??_7CArchiveStream@@6B@    5f8ac000     arcstrm.obj
 0002:000010a4       ??_C@_0DH@ODEG@faulted?5while?5dumping?5object?5at?5@ 5f8ac0a4     dumpinit.obj
 0002:000010dc       ??_C@_0CH@OFAB@a?5?$CFhs?5object?5at?5$?$CF08lX?0?5?$CFu?5bytes@ 5f8ac0dc     dumpinit.obj
 0002:00001104       ??_C@_0CM@EDOO@an?5invalid?5object?5at?5$?$CF08lX?0?5?$CFu?5@ 5f8ac104     dumpinit.obj
 0002:00001130       ??_C@_0N@POFF@dumpinit?4cpp?$AA@ 5f8ac130     dumpinit.obj
 0002:00001144       ??_7_AFX_DEBUG_STATE@@6B@  5f8ac144     dumpinit.obj
 0002:0000114c       ??_7CNoTrackObject@@6B@    5f8ac14c     dumpinit.obj
 0002:00001150       ??_C@_02HFBK@?3?5?$AA@     5f8ac150     dumpout.obj
 0002:00001154       ?_pfnUninitialized@@3Q6AHI@ZA 5f8ac154     afxmem.obj
 0002:00001158       ??_C@_1CE@MDGC@?$AAA?$AAf?$AAx?$AAA?$AAb?$AAo?$AAr?$AAt?$AA?5?$AAc?$AAa?$AAl?$AAl?$AAe?$AAd?$AA?4?$AA?6?$AA?$AA@ 5f8ac158     afxabort.obj
 0002:000011ac       ??_7CObject@@6B@           5f8ac1ac     afxinl1.obj
 0002:000011c4       ??_7CSimpleException@@6B@  5f8ac1c4     afxinl1.obj
 0002:000011e4       ??_7CMemoryException@@6B@  5f8ac1e4     afxinl1.obj
 0002:00001204       ??_7CNotSupportedException@@6B@ 5f8ac204     afxinl1.obj
 0002:00001224       ??_7CArchiveException@@6B@ 5f8ac224     afxinl1.obj
 0002:00001244       ??_7CFileException@@6B@    5f8ac244     afxinl1.obj
 0002:00001264       ??_7CCommonDialog@@6B@     5f8ac264     afxinl1.obj
 0002:00001340       ??_7CRectTracker@@6B@      5f8ac340     afxinl1.obj
 0002:0000135c       ??_7CBitmapButton@@6B@     5f8ac35c     afxinl1.obj
 0002:00001430       ??_7CResourceException@@6B@ 5f8ac430     afxinl2.obj
 0002:00001450       ??_7CUserException@@6B@    5f8ac450     afxinl2.obj
 0002:00001470       ??_7CGdiObject@@6B@        5f8ac470     afxinl2.obj
 0002:00001488       ??_7CPen@@6B@              5f8ac488     afxinl2.obj
 0002:000014a0       ??_7CBrush@@6B@            5f8ac4a0     afxinl2.obj
 0002:000014b8       ??_7CFont@@6B@             5f8ac4b8     afxinl2.obj
 0002:000014d0       ??_7CBitmap@@6B@           5f8ac4d0     afxinl2.obj
 0002:000014e8       ??_7CPalette@@6B@          5f8ac4e8     afxinl2.obj
 0002:00001500       ??_7CRgn@@6B@              5f8ac500     afxinl2.obj
 0002:00001518       ??_7CMenu@@6B@             5f8ac518     afxinl2.obj
 0002:00001544       ??_7CStatic@@6B@           5f8ac544     afxinl3.obj
 0002:00001608       ??_7CButton@@6B@           5f8ac608     afxinl3.obj
 0002:000016d0       ??_7CListBox@@6B@          5f8ac6d0     afxinl3.obj
 0002:000017ac       ??_7CCheckListBox@@6B@     5f8ac7ac     afxinl3.obj
 0002:0000188c       ??_7CComboBox@@6B@         5f8ac88c     afxinl3.obj
 0002:00001960       ??_7CEdit@@6B@             5f8ac960     afxinl3.obj
 0002:00001a24       ??_7CScrollBar@@6B@        5f8aca24     afxinl3.obj
 0002:00001ae8       ?classCFile@CFile@@2UCRuntimeClass@@B 5f8acae8     filecore.obj
 0002:00001b00       ??_C@_05GM@CFile?$AA@      5f8acb00     filecore.obj
 0002:00001b08       _afxIID_IShellLinkW        5f8acb08     filecore.obj
 0002:00001b18       _afxCLSID_ShellLink        5f8acb18     filecore.obj
 0002:00001b2c       ??_7CFile@@6B@             5f8acb2c     filecore.obj
 0002:00001b88       ??_C@_0BC@KFKC@DllGetClassObject?$AA@ 5f8acb88     filecore.obj
 0002:00001b9c       ??_C@_1GG@OAL@?$AA?$HL?$AA?$CF?$AA0?$AA8?$AAX?$AA?9?$AA?$CF?$AA0?$AA4?$AAX?$AA?9?$AA?$CF?$AA0?$AA4?$AAX?$AA?9?$AA?$CF?$AA0?$AA2?$AAX@ 5f8acb9c     filecore.obj
 0002:00001c04       ??_C@_11A@?$AA?$AA@        5f8acc04     filecore.obj
 0002:00001c08       ??_C@_1BO@DEPG@?$AAI?$AAn?$AAP?$AAr?$AAo?$AAc?$AAS?$AAe?$AAr?$AAv?$AAe?$AAr?$AA3?$AA2?$AA?$AA@ 5f8acc08     filecore.obj
 0002:00001c28       ??_C@_1M@EPCN@?$AAC?$AAL?$AAS?$AAI?$AAD?$AA?$AA@ 5f8acc28     filecore.obj
 0002:00001c34       ??_C@_1GC@CEID@?$AAW?$AAa?$AAr?$AAn?$AAi?$AAn?$AAg?$AA?3?$AA?5?$AAc?$AAo?$AAu?$AAl?$AAd?$AA?5?$AAn?$AAo?$AAt?$AA?5?$AAg@ 5f8acc34     filecore.obj
 0002:00001c98       ??_C@_1FC@EIIJ@?$AAW?$AAa?$AAr?$AAn?$AAi?$AAn?$AAg?$AA?3?$AA?5?$AAc?$AAo?$AAu?$AAl?$AAd?$AA?5?$AAn?$AAo?$AAt?$AA?5?$AAp@ 5f8acc98     filecore.obj
 0002:00001cec       ??_C@_0M@KEJC@?5and?5name?5?$CC?$AA@ 5f8accec     filecore.obj
 0002:00001cf8       ??_C@_01HMO@?$CC?$AA@      5f8accf8     filecore.obj
 0002:00001cfc       ??_C@_0N@MAIC@with?5handle?5?$AA@ 5f8accfc     filecore.obj
 0002:00001d10       ?classCStdioFile@CStdioFile@@2UCRuntimeClass@@B 5f8acd10     filetxt.obj
 0002:00001d28       ??_C@_0L@JAPO@CStdioFile?$AA@ 5f8acd28     filetxt.obj
 0002:00001d38       ??_7CStdioFile@@6B@        5f8acd38     filetxt.obj
 0002:00001da0       ??_C@_0N@FDDN@m_pStream?5?$DN?5?$AA@ 5f8acda0     filetxt.obj
 0002:00001db0       ?classCMemFile@CMemFile@@2UCRuntimeClass@@B 5f8acdb0     filemem.obj
 0002:00001dc8       ??_C@_08EMMO@CMemFile?$AA@ 5f8acdc8     filemem.obj
 0002:00001dd8       ??_7CMemFile@@6B@          5f8acdd8     filemem.obj
 0002:00001e48       ??_C@_0BB@KJDL@?6m_nGrowBytes?5?$DN?5?$AA@ 5f8ace48     filemem.obj
 0002:00001e5c       ??_C@_0BA@IEDI@?6m_nPosition?5?$DN?5?$AA@ 5f8ace5c     filemem.obj
 0002:00001e6c       ??_C@_0BC@LAMI@?6m_nBufferSize?5?$DN?5?$AA@ 5f8ace6c     filemem.obj
 0002:00001e80       ??_C@_0P@IHAB@m_nFileSize?5?$DN?5?$AA@ 5f8ace80     filemem.obj
 0002:00001e90       ?classCSharedFile@CSharedFile@@2UCRuntimeClass@@B 5f8ace90     fileshrd.obj
 0002:00001ea8       ??_C@_0M@DHDK@CSharedFile?$AA@ 5f8acea8     fileshrd.obj
 0002:00001eb8       ??_7CSharedFile@@6B@       5f8aceb8     fileshrd.obj
 0002:00001f28       ?classCFileException@CFileException@@2UCRuntimeClass@@B 5f8acf28     filex.obj
 0002:00001f40       ??_C@_0P@HFKI@CFileException?$AA@ 5f8acf40     filex.obj
 0002:00001f94       ??_C@_08DJIA@diskFull?$AA@ 5f8acf94     filex.obj
 0002:00001fa0       ??_C@_0O@IKIP@lockViolation?$AA@ 5f8acfa0     filex.obj
 0002:00001fb0       ??_C@_0BB@KIFC@sharingViolation?$AA@ 5f8acfb0     filex.obj
 0002:00001fc4       ??_C@_06BPHG@hardIO?$AA@   5f8acfc4     filex.obj
 0002:00001fcc       ??_C@_07DCIG@badSeek?$AA@  5f8acfcc     filex.obj
 0002:00001fd4       ??_C@_0O@NHLK@directoryFull?$AA@ 5f8acfd4     filex.obj
 0002:00001fe4       ??_C@_0BB@OOOA@removeCurrentDir?$AA@ 5f8acfe4     filex.obj
 0002:00001ff8       ??_C@_0M@BHGP@invalidFile?$AA@ 5f8acff8     filex.obj
 0002:00002004       ??_C@_0N@CFIF@accessDenied?$AA@ 5f8ad004     filex.obj
 0002:00002014       ??_C@_0BB@KBLL@tooManyOpenFiles?$AA@ 5f8ad014     filex.obj
 0002:00002028       ??_C@_07JGJA@badPath?$AA@  5f8ad028     filex.obj
 0002:00002030       ??_C@_0N@KFOJ@fileNotFound?$AA@ 5f8ad030     filex.obj
 0002:00002040       ??_C@_0P@CDGG@?6m_lOsError?5?$DN?5?$AA@ 5f8ad040     filex.obj
 0002:00002050       ??_C@_0L@BAND@m_cause?5?$DN?5?$AA@ 5f8ad050     filex.obj
 0002:0000205c       ??_C@_1HI@GAHB@?$AAC?$AAF?$AAi?$AAl?$AAe?$AA?5?$AAe?$AAx?$AAc?$AAe?$AAp?$AAt?$AAi?$AAo?$AAn?$AA?3?$AA?5?$AA?$CF?$AAh?$AAs@ 5f8ad05c     filex.obj
 0002:000020d4       ??_C@_1BA@JDJI@?$AAU?$AAn?$AAk?$AAn?$AAo?$AAw?$AAn?$AA?$AA@ 5f8ad0d4     filex.obj
 0002:000020e4       ??_C@_0BB@FMKN@?6m_szFullName?5?$DN?5?$AA@ 5f8ad0e4     filest.obj
 0002:000020f8       ??_C@_0BA@MINE@?6m_attribute?5?$DN?5?$AA@ 5f8ad0f8     filest.obj
 0002:00002108       ??_C@_0L@MFI@?6m_size?5?$DN?5?$AA@ 5f8ad108     filest.obj
 0002:00002114       ??_C@_0M@BOFF@?6m_atime?5?$DN?5?$AA@ 5f8ad114     filest.obj
 0002:00002120       ??_C@_0M@HPJL@?6m_mtime?5?$DN?5?$AA@ 5f8ad120     filest.obj
 0002:0000212c       ??_C@_0M@IOAI@?6m_ctime?5?$DN?5?$AA@ 5f8ad12c     filest.obj
 0002:00002138       ??_C@_0BC@PLAF@a?5CFileStatus?5at?5?$AA@ 5f8ad138     filest.obj
 0002:0000214c       ??_C@_1JG@BKCB@?$AAW?$AAa?$AAr?$AAn?$AAi?$AAn?$AAg?$AA?3?$AA?5?$AAC?$AAF?$AAi?$AAl?$AAe?$AA?3?$AA?3?$AAG?$AAe?$AAt?$AAS@ 5f8ad14c     filest.obj
 0002:000021e4       ??_C@_0L@LFP@CByteArray?$AA@ 5f8ad1e4     array_b.obj
 0002:000021f4       ??_7CByteArray@@6B@        5f8ad1f4     array_b.obj
 0002:00002208       ??_C@_03DANH@?6?7?$FL?$AA@ 5f8ad208     array_b.obj
 0002:0000220c       ??_C@_04MNLE@?$FN?5?$DN?5?$AA@ 5f8ad20c     array_b.obj
 0002:00002214       ??_C@_05KIFI@with?5?$AA@   5f8ad214     array_b.obj
 0002:0000221c       ??_C@_09LOPF@?5elements?$AA@ 5f8ad21c     array_b.obj
 0002:00002228       ??_C@_0M@JHEJ@CDWordArray?$AA@ 5f8ad228     array_d.obj
 0002:00002238       ??_7CDWordArray@@6B@       5f8ad238     array_d.obj
 0002:00002250       ?classCPtrArray@CPtrArray@@2UCRuntimeClass@@B 5f8ad250     array_p.obj
 0002:00002268       ??_C@_09BHCJ@CPtrArray?$AA@ 5f8ad268     array_p.obj
 0002:00002278       ??_7CPtrArray@@6B@         5f8ad278     array_p.obj
 0002:0000228c       ??_C@_08PPJP@CObArray?$AA@ 5f8ad28c     array_o.obj
 0002:0000229c       ??_7CObArray@@6B@          5f8ad29c     array_o.obj
 0002:000022b0       ??_C@_0N@FMIP@CStringArray?$AA@ 5f8ad2b0     array_s.obj
 0002:000022c4       ??_7CStringArray@@6B@      5f8ad2c4     array_s.obj
 0002:000022d8       ?classCUIntArray@CUIntArray@@2UCRuntimeClass@@B 5f8ad2d8     array_u.obj
 0002:000022f0       ??_C@_0L@OIGA@CUIntArray?$AA@ 5f8ad2f0     array_u.obj
 0002:00002300       ??_7CUIntArray@@6B@        5f8ad300     array_u.obj
 0002:00002314       ??_C@_0L@KEGG@CWordArray?$AA@ 5f8ad314     array_w.obj
 0002:00002324       ??_7CWordArray@@6B@        5f8ad324     array_w.obj
 0002:00002338       ??_C@_07ICCG@CObList?$AA@  5f8ad338     list_o.obj
 0002:00002344       ??_7CObList@@6B@           5f8ad344     list_o.obj
 0002:00002358       ??_C@_02GGCO@?6?7?$AA@     5f8ad358     list_o.obj
 0002:00002360       ?classCPtrList@CPtrList@@2UCRuntimeClass@@B 5f8ad360     list_p.obj
 0002:00002378       ??_C@_08DEKG@CPtrList?$AA@ 5f8ad378     list_p.obj
 0002:00002388       ??_7CPtrList@@6B@          5f8ad388     list_p.obj
 0002:0000239c       ??_C@_0M@JCPP@CStringList?$AA@ 5f8ad39c     list_s.obj
 0002:000023ac       ??_7CStringList@@6B@       5f8ad3ac     list_s.obj
 0002:000023c0       ?classCMapPtrToPtr@CMapPtrToPtr@@2UCRuntimeClass@@B 5f8ad3c0     map_pp.obj
 0002:000023d8       ??_C@_0N@EGND@CMapPtrToPtr?$AA@ 5f8ad3d8     map_pp.obj
 0002:000023ec       ??_7CMapPtrToPtr@@6B@      5f8ad3ec     map_pp.obj
 0002:00002400       ?classCMapPtrToWord@CMapPtrToWord@@2UCRuntimeClass@@B 5f8ad400     map_pw.obj
 0002:00002418       ??_C@_0O@CNGA@CMapPtrToWord?$AA@ 5f8ad418     map_pw.obj
 0002:0000242c       ??_7CMapPtrToWord@@6B@     5f8ad42c     map_pw.obj
 0002:00002440       ??_C@_0P@FLNF@CMapStringToOb?$AA@ 5f8ad440     map_so.obj
 0002:00002454       ??_7CMapStringToOb@@6B@    5f8ad454     map_so.obj
 0002:00002468       ?classCMapStringToPtr@CMapStringToPtr@@2UCRuntimeClass@@B 5f8ad468     map_sp.obj
 0002:00002480       ??_C@_0BA@PAMN@CMapStringToPtr?$AA@ 5f8ad480     map_sp.obj
 0002:00002494       ??_7CMapStringToPtr@@6B@   5f8ad494     map_sp.obj
 0002:000024a8       ??_C@_0BD@HCIA@CMapStringToString?$AA@ 5f8ad4a8     map_ss.obj
 0002:000024c0       ??_7CMapStringToString@@6B@ 5f8ad4c0     map_ss.obj
 0002:000024d4       ??_C@_0N@DJOC@CMapWordToOb?$AA@ 5f8ad4d4     map_wo.obj
 0002:000024e8       ??_7CMapWordToOb@@6B@      5f8ad4e8     map_wo.obj
 0002:00002500       ?classCMapWordToPtr@CMapWordToPtr@@2UCRuntimeClass@@B 5f8ad500     map_wp.obj
 0002:00002518       ??_C@_0O@MJKP@CMapWordToPtr?$AA@ 5f8ad518     map_wp.obj
 0002:0000252c       ??_7CMapWordToPtr@@6B@     5f8ad52c     map_wp.obj
 0002:00002540       ??_C@_1FC@LHMI@?$AAW?$AAa?$AAr?$AAn?$AAi?$AAn?$AAg?$AA?3?$AA?5?$AAi?$AAm?$AAp?$AAl?$AAi?$AAc?$AAi?$AAt?$AA?5?$AAL?$AAo@ 5f8ad540     strcore.obj
 0002:00002594       ??_C@_1IA@OBOF@?$AAW?$AAa?$AAr?$AAn?$AAi?$AAn?$AAg?$AA?3?$AA?5?$AAG?$AAe?$AAt?$AAB?$AAu?$AAf?$AAf?$AAe?$AAr?$AA?5?$AAo@ 5f8ad594     strcore.obj
 0002:00002614       ??_C@_17BCJF@?$AAI?$AA6?$AA4?$AA?$AA@ 5f8ad614     strex.obj
 0002:0000261c       ??_C@_07MABK@CTime?$CI?$CC?$AA@ 5f8ad61c     timecore.obj
 0002:00002624       ??_C@_02FEMI@?$CC?$CJ?$AA@ 5f8ad624     timecore.obj
 0002:00002628       ??_C@_0BA@NLOD@CTime?$CIinvalid?5?$CD?$AA@ 5f8ad628     timecore.obj
 0002:00002638       ??_C@_01KMMP@?$CJ?$AA@     5f8ad638     timecore.obj
 0002:0000263c       ??_C@_0L@DOCK@CTimeSpan?$CI?$AA@ 5f8ad63c     timecore.obj
 0002:00002648       ??_C@_07CJKE@?5days?0?5?$AA@ 5f8ad648     timecore.obj
 0002:00002650       ??_C@_08CJPE@?5hours?0?5?$AA@ 5f8ad650     timecore.obj
 0002:0000265c       ??_C@_0O@BFOJ@?5minutes?5and?5?$AA@ 5f8ad65c     timecore.obj
 0002:0000266c       ??_C@_09PGME@?5seconds?$CJ?$AA@ 5f8ad66c     timecore.obj
 0002:00002678       ??_C@_19HABD@?$AA?$CF?$AA0?$AA2?$AAd?$AA?$AA@ 5f8ad678     timecore.obj
 0002:00002688       ??_7_AFX_THREAD_STATE@@6B@ 5f8ad688     afxstate.obj
 0002:00002690       ??_7AFX_MODULE_STATE@@6B@  5f8ad690     afxstate.obj
 0002:00002698       ??_7AFX_MODULE_THREAD_STATE@@6B@ 5f8ad698     afxstate.obj
 0002:000026a0       ??_7_AFX_BASE_MODULE_STATE@@6B@ 5f8ad6a0     afxstate.obj
 0002:000026a8       ??_7CThreadData@@6B@       5f8ad6a8     afxtls.obj
 0002:000026b0       ?classCSyncObject@CSyncObject@@2UCRuntimeClass@@B 5f8ad6b0     mtcore.obj
 0002:000026c8       ??_C@_0M@EHIL@CSyncObject?$AA@ 5f8ad6c8     mtcore.obj
 0002:000026d8       ?classCCriticalSection@CCriticalSection@@2UCRuntimeClass@@B 5f8ad6d8     mtcore.obj
 0002:000026f0       ??_C@_0BB@HCJ@CCriticalSection?$AA@ 5f8ad6f0     mtcore.obj
 0002:00002708       ??_7CSyncObject@@6B@       5f8ad708     mtcore.obj
 0002:00002728       ??_C@_07LNGA@?5named?5?$AA@ 5f8ad728     mtcore.obj
 0002:00002730       ??_C@_07MBHD@Object?5?$AA@ 5f8ad730     mtcore.obj
 0002:0000273c       ??_7CCriticalSection@@6B@  5f8ad73c     mtcore.obj
 0002:00002760       ?classCMutex@CMutex@@2UCRuntimeClass@@B 5f8ad760     mtex.obj
 0002:00002778       ??_C@_06HCIL@CMutex?$AA@   5f8ad778     mtex.obj
 0002:00002780       ?classCSemaphore@CSemaphore@@2UCRuntimeClass@@B 5f8ad780     mtex.obj
 0002:00002798       ??_C@_0L@NFMO@CSemaphore?$AA@ 5f8ad798     mtex.obj
 0002:000027a8       ?classCEvent@CEvent@@2UCRuntimeClass@@B 5f8ad7a8     mtex.obj
 0002:000027c0       ??_C@_06BPGE@CEvent?$AA@   5f8ad7c0     mtex.obj
 0002:000027cc       ??_7CSemaphore@@6B@        5f8ad7cc     mtex.obj
 0002:000027f0       ??_7CMutex@@6B@            5f8ad7f0     mtex.obj
 0002:00002814       ??_7CEvent@@6B@            5f8ad814     mtex.obj
 0002:00002838       ?classCTempWnd@CTempWnd@@2UCRuntimeClass@@B 5f8ad838     wincore.obj
 0002:00002850       ??_C@_08EHJM@CTempWnd?$AA@ 5f8ad850     wincore.obj
 0002:00002860       ?classCWnd@CWnd@@2UCRuntimeClass@@B 5f8ad860     wincore.obj
 0002:00002878       ??_C@_04MBPC@CWnd?$AA@     5f8ad878     wincore.obj
 0002:00002880       ?messageMap@CWnd@@1UAFX_MSGMAP@@B 5f8ad880     wincore.obj
 0002:00002888       ?_messageEntries@CWnd@@0QBUAFX_MSGMAP_ENTRY@@B 5f8ad888     wincore.obj
 0002:00002b28       ?_afxOldWndProc@@3QBGB     5f8adb28     wincore.obj
 0002:00002b4c       ?_afxWnd@@3QBGB            5f8adb4c     wincore.obj
 0002:00002b64       ?_afxWndControlBar@@3QBGB  5f8adb64     wincore.obj
 0002:00002b88       ?_afxWndMDIFrame@@3QBGB    5f8adb88     wincore.obj
 0002:00002ba8       ?_afxWndFrameOrView@@3QBGB 5f8adba8     wincore.obj
 0002:00002bd0       ?_afxWndOleControl@@3QBGB  5f8adbd0     wincore.obj
 0002:00002bf4       ??_C@_0BA@OPCN@GetMonitorInfoW?$AA@ 5f8adbf4     wincore.obj
 0002:00002c04       ??_C@_0BE@KPOG@EnumDisplayMonitors?$AA@ 5f8adc04     wincore.obj
 0002:00002c18       ??_C@_0BB@GJCM@MonitorFromPoint?$AA@ 5f8adc18     wincore.obj
 0002:00002c2c       ??_C@_0BA@GOHF@MonitorFromRect?$AA@ 5f8adc2c     wincore.obj
 0002:00002c3c       ??_C@_0BC@COEH@MonitorFromWindow?$AA@ 5f8adc3c     wincore.obj
 0002:00002c50       ??_C@_0BB@NDAA@GetSystemMetrics?$AA@ 5f8adc50     wincore.obj
 0002:00002c64       ??_C@_1O@EJK@?$AAU?$AAS?$AAE?$AAR?$AA3?$AA2?$AA?$AA@ 5f8adc64     wincore.obj
 0002:00002c74       ??_C@_1BA@FHJ@?$AAD?$AAI?$AAS?$AAP?$AAL?$AAA?$AAY?$AA?$AA@ 5f8adc74     wincore.obj
 0002:00002c84       ??_C@_1CK@HBPJ@?$AAc?$AAo?$AAm?$AAm?$AAc?$AAt?$AAr?$AAl?$AA_?$AAD?$AAr?$AAa?$AAg?$AAL?$AAi?$AAs?$AAt?$AAM?$AAs?$AAg@ 5f8adc84     wincore.obj
 0002:00002cb4       ??_7CWnd@@6B@              5f8adcb4     wincore.obj
 0002:00002d74       ??_C@_1HI@NNAA@?$AAW?$AAa?$AAr?$AAn?$AAi?$AAn?$AAg?$AA?3?$AA?5?$AAU?$AAn?$AAc?$AAa?$AAu?$AAg?$AAh?$AAt?$AA?5?$AAe?$AAx@ 5f8add74     wincore.obj
 0002:00002dec       ??_C@_1BA@KFMN@?$AAW?$AAn?$AAd?$AAP?$AAr?$AAo?$AAc?$AA?$AA@ 5f8addec     wincore.obj
 0002:00002dfc       ??_C@_1IO@PHDK@?$AAW?$AAa?$AAr?$AAn?$AAi?$AAn?$AAg?$AA?3?$AA?5?$AAU?$AAn?$AAc?$AAa?$AAu?$AAg?$AAh?$AAt?$AA?5?$AAe?$AAx@ 5f8addfc     wincore.obj
 0002:00002e8c       ??_C@_17NMLD@?$AAi?$AAm?$AAe?$AA?$AA@ 5f8ade8c     wincore.obj
 0002:00002e94       ??_C@_1HO@OOAB@?$AAW?$AAa?$AAr?$AAn?$AAi?$AAn?$AAg?$AA?3?$AA?5?$AAW?$AAi?$AAn?$AAd?$AAo?$AAw?$AA?5?$AAc?$AAr?$AAe?$AAa@ 5f8ade94     wincore.obj
 0002:00002f14       ??_C@_1OA@CIKK@?$AAW?$AAa?$AAr?$AAn?$AAi?$AAn?$AAg?$AA?3?$AA?5?$AAc?$AAa?$AAl?$AAl?$AAi?$AAn?$AAg?$AA?5?$AAD?$AAe?$AAs@ 5f8adf14     wincore.obj
 0002:00002ff4       ??_C@_06BHKF@?6id?5?$DN?5?$AA@ 5f8adff4     wincore.obj
 0002:00002ffc       ??_C@_09MMEE@?6style?5?$DN?5?$AA@ 5f8adffc     wincore.obj
 0002:00003008       ??_C@_0BB@OKDO@?6parent?5CWnd?$CK?5?$DN?5?$AA@ 5f8ae008     wincore.obj
 0002:0000301c       ??_C@_08IIAM@?6rect?5?$DN?5?$AA@ 5f8ae01c     wincore.obj
 0002:00003028       ??_C@_0BA@JMEP@?6class?5name?5?$DN?5?$CC?$AA@ 5f8ae028     wincore.obj
 0002:00003038       ??_C@_0N@EELD@?6caption?5?$DN?5?$CC?$AA@ 5f8ae038     wincore.obj
 0002:00003048       ??_C@_0BE@EMJB@?5?$CIpermanent?5window?$CJ?$AA@ 5f8ae048     wincore.obj
 0002:0000305c       ??_C@_0CA@HEAL@?5?$CIDetached?5or?5temporary?5window?$CJ?$AA@ 5f8ae05c     wincore.obj
 0002:0000307c       ??_C@_0BA@NCHM@?5?$CIillegal?5HWND?$CJ?$AA@ 5f8ae07c     wincore.obj
 0002:0000308c       ??_C@_0L@HLEE@?6m_hWnd?5?$DN?5?$AA@ 5f8ae08c     wincore.obj
 0002:00003098       ??_C@_1GO@BJLB@?$AAW?$AAa?$AAr?$AAn?$AAi?$AAn?$AAg?$AA?3?$AA?5?$AAu?$AAn?$AAk?$AAn?$AAo?$AAw?$AAn?$AA?5?$AAW?$AAM?$AA_@ 5f8ae098     wincore.obj
 0002:00003108       ??_C@_1EM@OKFH@?$AAC?$AAa?$AAn?$AA?8?$AAt?$AA?5?$AAr?$AAe?$AAg?$AAi?$AAs?$AAt?$AAe?$AAr?$AA?5?$AAw?$AAi?$AAn?$AAd?$AAo@ 5f8ae108     wincore.obj
 0002:00003154       ??_C@_1CG@HFFM@?$AAA?$AAf?$AAx?$AA?3?$AA?$CF?$AAx?$AA?3?$AA?$CF?$AAx?$AA?3?$AA?$CF?$AAx?$AA?3?$AA?$CF?$AAx?$AA?3?$AA?$CF?$AAx?$AA?$AA@ 5f8ae154     wincore.obj
 0002:0000317c       ??_C@_1BE@KCHN@?$AAA?$AAf?$AAx?$AA?3?$AA?$CF?$AAx?$AA?3?$AA?$CF?$AAx?$AA?$AA@ 5f8ae17c     wincore.obj
 0002:00003190       ??_C@_1HG@BIMO@?$AAW?$AAi?$AAn?$AAH?$AAe?$AAl?$AAp?$AA?3?$AA?5?$AAp?$AAs?$AAz?$AAH?$AAe?$AAl?$AAp?$AAF?$AAi?$AAl?$AAe@ 5f8ae190     wincore.obj
 0002:0000320c       ??_7CTestCmdUI@@6B@        5f8ae20c     wincore.obj
 0002:0000321c       ??_C@_1GK@IJAD@?$AAI?$AAm?$AAp?$AAl?$AAe?$AAm?$AAe?$AAn?$AAt?$AAa?$AAt?$AAi?$AAo?$AAn?$AA?5?$AAW?$AAa?$AAr?$AAn?$AAi@ 5f8ae21c     wincore.obj
 0002:00003288       ??_C@_1FI@PDNK@?$AAW?$AAa?$AAr?$AAn?$AAi?$AAn?$AAg?$AA?3?$AA?5?$AAn?$AAo?$AAt?$AA?5?$AAe?$AAx?$AAe?$AAc?$AAu?$AAt?$AAi@ 5f8ae288     wincore.obj
 0002:000032e0       ??_C@_1HA@LPHL@?$AAW?$AAa?$AAr?$AAn?$AAi?$AAn?$AAg?$AA?3?$AA?5?$AAD?$AAe?$AAf?$AAe?$AAr?$AAW?$AAi?$AAn?$AAd?$AAo?$AAw@ 5f8ae2e0     wincore.obj
 0002:00003350       ??_C@_1JA@JGEC@?$AAW?$AAa?$AAr?$AAn?$AAi?$AAn?$AAg?$AA?3?$AA?5?$AAh?$AAD?$AAC?$AA?5?$AAi?$AAs?$AA?5?$AAN?$AAU?$AAL?$AAL@ 5f8ae350     wincore.obj
 0002:000033e0       ??_C@_0BF@CELH@InitCommonControlsEx?$AA@ 5f8ae3e0     wincore.obj
 0002:000033f8       ??_C@_0N@BMKC@COMCTL32?4DLL?$AA@ 5f8ae3f8     wincore.obj
 0002:00003408       ??_C@_1FE@IHBG@?$AA?7?$AAh?$AAW?$AAn?$AAd?$AA?5?$AA?$DN?$AA?5?$AA$?$AA?$CF?$AA0?$AA4?$AAX?$AA?5?$AA?$CI?$AAn?$AAI?$AAD?$AAC?$AA?$DN@ 5f8ae408     wincore.obj
 0002:0000345c       ??_C@_1CC@BBNA@?$AA?7?$AAd?$AAe?$AAr?$AAi?$AAv?$AAe?$AAd?$AA?5?$AAc?$AAl?$AAa?$AAs?$AAs?$AA?4?$AA?6?$AA?$AA@ 5f8ae45c     wincore.obj
 0002:00003480       ??_C@_1HC@NHDM@?$AAE?$AAr?$AAr?$AAo?$AAr?$AA?3?$AA?5?$AAT?$AAr?$AAy?$AAi?$AAn?$AAg?$AA?5?$AAt?$AAo?$AA?5?$AAu?$AAs?$AAe@ 5f8ae480     wincore.obj
 0002:000034f8       ??_7CTempWnd@@6B@          5f8ae4f8     wincore.obj
 0002:000035bc       ??_7_AFX_CTL3D_STATE@@6B@  5f8ae5bc     wincore.obj
 0002:000035c0       ?classCControlBar@CControlBar@@2UCRuntimeClass@@B 5f8ae5c0     winfrm.obj
 0002:000035d8       ??_C@_0M@GCON@CControlBar?$AA@ 5f8ae5d8     winfrm.obj
 0002:000035e8       ?classCView@CView@@2UCRuntimeClass@@B 5f8ae5e8     winfrm.obj
 0002:00003600       ??_C@_05KON@CView?$AA@     5f8ae600     winfrm.obj
 0002:00003608       ?classCFrameWnd@CFrameWnd@@2UCRuntimeClass@@B 5f8ae608     winfrm.obj
 0002:00003620       ??_C@_09HNKJ@CFrameWnd?$AA@ 5f8ae620     winfrm.obj
 0002:00003630       ?messageMap@CFrameWnd@@1UAFX_MSGMAP@@B 5f8ae630     winfrm.obj
 0002:00003638       ?_messageEntries@CFrameWnd@@0QBUAFX_MSGMAP_ENTRY@@B 5f8ae638     winfrm.obj
 0002:00003aa0       ??_C@_1CA@JHCA@?$AAM?$AAS?$AAW?$AAH?$AAE?$AAE?$AAL?$AA_?$AAR?$AAO?$AAL?$AAL?$AAM?$AAS?$AAG?$AA?$AA@ 5f8aeaa0     winfrm.obj
 0002:00003ac4       ??_7CFrameWnd@@6B@         5f8aeac4     winfrm.obj
 0002:00003bc0       ??_C@_1EM@DDNK@?$AAW?$AAa?$AAr?$AAn?$AAi?$AAn?$AAg?$AA?3?$AA?5?$AAf?$AAa?$AAi?$AAl?$AAe?$AAd?$AA?5?$AAt?$AAo?$AA?5?$AAc@ 5f8aebc0     winfrm.obj
 0002:00003c0c       ??_C@_1FK@IOMB@?$AAW?$AAa?$AAr?$AAn?$AAi?$AAn?$AAg?$AA?3?$AA?5?$AAf?$AAa?$AAi?$AAl?$AAe?$AAd?$AA?5?$AAt?$AAo?$AA?5?$AAl@ 5f8aec0c     winfrm.obj
 0002:00003c68       ??_C@_1FG@DHFK@?$AAW?$AAa?$AAr?$AAn?$AAi?$AAn?$AAg?$AA?3?$AA?5?$AAc?$AAo?$AAu?$AAl?$AAd?$AA?5?$AAn?$AAo?$AAt?$AA?5?$AAc@ 5f8aec68     winfrm.obj
 0002:00003cc0       ??_C@_1GE@OKMP@?$AAW?$AAa?$AAr?$AAn?$AAi?$AAn?$AAg?$AA?3?$AA?5?$AAD?$AAy?$AAn?$AAa?$AAm?$AAi?$AAc?$AA?5?$AAc?$AAr?$AAe@ 5f8aecc0     winfrm.obj
 0002:00003d24       ??_C@_1FM@MAKN@?$AAF?$AAa?$AAi?$AAl?$AAe?$AAd?$AA?5?$AAt?$AAo?$AA?5?$AAc?$AAr?$AAe?$AAa?$AAt?$AAe?$AA?5?$AAc?$AAl?$AAi@ 5f8aed24     winfrm.obj
 0002:00003d80       ??_C@_1FI@CHH@?$AAE?$AAr?$AAr?$AAo?$AAr?$AA?3?$AA?5?$AAf?$AAa?$AAi?$AAl?$AAe?$AAd?$AA?5?$AAt?$AAo?$AA?5?$AAe?$AAx?$AAe@ 5f8aed80     winfrm.obj
 0002:00003dd8       ??_C@_1HO@HABA@?$AAW?$AAa?$AAr?$AAn?$AAi?$AAn?$AAg?$AA?3?$AA?5?$AAD?$AAD?$AAE?$AA?5?$AAc?$AAo?$AAm?$AAm?$AAa?$AAn?$AAd@ 5f8aedd8     winfrm.obj
 0002:00003e58       ??_C@_1GA@KHGF@?$AAW?$AAa?$AAr?$AAn?$AAi?$AAn?$AAg?$AA?3?$AA?5?$AAn?$AAo?$AA?5?$AAm?$AAe?$AAs?$AAs?$AAa?$AAg?$AAe?$AA?5@ 5f8aee58     winfrm.obj
 0002:00003eb8       ??_C@_1HG@CHFH@?$AAW?$AAa?$AAr?$AAn?$AAi?$AAn?$AAg?$AA?3?$AA?5?$AAO?$AAn?$AAU?$AAp?$AAd?$AAa?$AAt?$AAe?$AAK?$AAe?$AAy@ 5f8aeeb8     winfrm.obj
 0002:00003f30       ??_C@_17LFFB@?$AA?5?$AA?9?$AA?5?$AA?$AA@ 5f8aef30     winfrm.obj
 0002:00003f38       ??_C@_17LJFH@?$AA?3?$AA?$CF?$AAd?$AA?$AA@ 5f8aef38     winfrm.obj
 0002:00003f40       ??_C@_1II@MAFK@?$AAW?$AAa?$AAr?$AAn?$AAi?$AAn?$AAg?$AA?3?$AA?5?$AAs?$AAc?$AAr?$AAo?$AAl?$AAl?$AA?5?$AAb?$AAa?$AAr?$AAs@ 5f8aef40     winfrm.obj
 0002:00003fc8       ??_C@_0BA@OBND@?6no?5active?5view?$AA@ 5f8aefc8     winfrm.obj
 0002:00003fd8       ??_C@_0BE@LNEN@?6with?5active?5view?3?5?$AA@ 5f8aefd8     winfrm.obj
 0002:00003fec       ??_C@_0BF@GBOK@?6m_nIDLastMessage?5?$DN?5?$AA@ 5f8aefec     winfrm.obj
 0002:00004004       ??_C@_0BC@GNPE@?6m_nIDTracking?5?$DN?5?$AA@ 5f8af004     winfrm.obj
 0002:00004018       ??_C@_0O@BBAD@?6m_nIDHelp?5?$DN?5?$AA@ 5f8af018     winfrm.obj
 0002:00004028       ??_C@_0O@DMPK@?6m_nWindow?5?$DN?5?$AA@ 5f8af028     winfrm.obj
 0002:00004038       ??_C@_0BB@HLGH@m_hAccelTable?5?$DN?5?$AA@ 5f8af038     winfrm.obj
 0002:0000404c       ?dwDockBarMap@CFrameWnd@@1QAY01$$CBKA 5f8af04c     winfrm2.obj
 0002:0000406c       ??_C@_1HM@LAGL@?$AAE?$AAr?$AAr?$AAo?$AAr?$AA?3?$AA?5?$AAa?$AAn?$AA?5?$AAi?$AAn?$AA?9?$AAp?$AAl?$AAa?$AAc?$AAe?$AA?5?$AAs@ 5f8af06c     winfrmx.obj
 0002:000040e8       ?classCMDIChildWnd@CMDIChildWnd@@2UCRuntimeClass@@B 5f8af0e8     winmdi.obj
 0002:00004100       ??_C@_0N@NPHP@CMDIChildWnd?$AA@ 5f8af100     winmdi.obj
 0002:00004110       ?classCMDIFrameWnd@CMDIFrameWnd@@2UCRuntimeClass@@B 5f8af110     winmdi.obj
 0002:00004128       ??_C@_0N@FPEB@CMDIFrameWnd?$AA@ 5f8af128     winmdi.obj
 0002:00004138       ?messageMap@CMDIChildWnd@@1UAFX_MSGMAP@@B 5f8af138     winmdi.obj
 0002:00004140       ?_messageEntries@CMDIChildWnd@@0QBUAFX_MSGMAP_ENTRY@@B 5f8af140     winmdi.obj
 0002:00004248       ?messageMap@CMDIFrameWnd@@1UAFX_MSGMAP@@B 5f8af248     winmdi.obj
 0002:00004250       ?_messageEntries@CMDIFrameWnd@@0QBUAFX_MSGMAP_ENTRY@@B 5f8af250     winmdi.obj
 0002:000043d4       ??_7CMDIFrameWnd@@6B@      5f8af3d4     winmdi.obj
 0002:000044d8       ??_C@_1MC@OCII@?$AAW?$AAa?$AAr?$AAn?$AAi?$AAn?$AAg?$AA?3?$AA?5?$AAC?$AAM?$AAD?$AAI?$AAF?$AAr?$AAa?$AAm?$AAe?$AAW?$AAn@ 5f8af4d8     winmdi.obj
 0002:0000459c       ??_C@_1BE@MFDJ@?$AAm?$AAd?$AAi?$AAc?$AAl?$AAi?$AAe?$AAn?$AAt?$AA?$AA@ 5f8af59c     winmdi.obj
 0002:000045b0       ??_C@_1FO@CGDK@?$AAW?$AAa?$AAr?$AAn?$AAi?$AAn?$AAg?$AA?3?$AA?5?$AAC?$AAM?$AAD?$AAI?$AAF?$AAr?$AAa?$AAm?$AAe?$AAW?$AAn@ 5f8af5b0     winmdi.obj
 0002:00004610       ??_C@_1DK@EJFG@?$AAC?$AAo?$AAu?$AAl?$AAd?$AAn?$AA?8?$AAt?$AA?5?$AAl?$AAo?$AAa?$AAd?$AA?5?$AAf?$AAr?$AAa?$AAm?$AAe?$AA?5@ 5f8af610     winmdi.obj
 0002:0000464c       ??_C@_0BD@PBFF@?6m_hMenuDefault?5?$DN?5?$AA@ 5f8af64c     winmdi.obj
 0002:00004660       ??_C@_0BD@IENL@m_hWndMDIClient?5?$DN?5?$AA@ 5f8af660     winmdi.obj
 0002:00004678       ??_7CMDIChildWnd@@6B@      5f8af678     winmdi.obj
 0002:0000477c       ??_C@_1HE@JNPH@?$AAW?$AAa?$AAr?$AAn?$AAi?$AAn?$AAg?$AA?3?$AA?5?$AAn?$AAo?$AA?5?$AAs?$AAh?$AAa?$AAr?$AAe?$AAd?$AA?5?$AAm@ 5f8af77c     winmdi.obj
 0002:000047f0       ??_C@_0BB@DJLO@m_hMenuShared?5?$DN?5?$AA@ 5f8af7f0     winmdi.obj
 0002:00004804       ??_C@_1EK@LEIL@?$AAW?$AAa?$AAr?$AAn?$AAi?$AAn?$AAg?$AA?3?$AA?5?$AAG?$AAe?$AAt?$AAW?$AAi?$AAn?$AAd?$AAo?$AAw?$AAM?$AAe@ 5f8af804     winmdi.obj
 0002:00004850       ??_C@_1EM@GEBA@?$AAW?$AAa?$AAr?$AAn?$AAi?$AAn?$AAg?$AA?3?$AA?5?$AAf?$AAa?$AAi?$AAl?$AAe?$AAd?$AA?5?$AAt?$AAo?$AA?5?$AAc@ 5f8af850     winmdi.obj
 0002:0000489c       ??_C@_1GI@BAGO@?$AAW?$AAa?$AAr?$AAn?$AAi?$AAn?$AAg?$AA?3?$AA?5?$AAN?$AAo?$AA?5?$AAa?$AAc?$AAt?$AAi?$AAv?$AAe?$AA?5?$AAd@ 5f8af89c     winmdi.obj
 0002:00004908       ?classCToolTipCtrl@CToolTipCtrl@@2UCRuntimeClass@@B 5f8af908     tooltip.obj
 0002:00004920       ??_C@_0N@OELH@CToolTipCtrl?$AA@ 5f8af920     tooltip.obj
 0002:00004930       ?messageMap@CToolTipCtrl@@1UAFX_MSGMAP@@B 5f8af930     tooltip.obj
 0002:00004938       ?_messageEntries@CToolTipCtrl@@0QBUAFX_MSGMAP_ENTRY@@B 5f8af938     tooltip.obj
 0002:000049b4       ??_7CToolTipCtrl@@6B@      5f8af9b4     tooltip.obj
 0002:00004a74       ??_C@_1CC@BIKB@?$AAt?$AAo?$AAo?$AAl?$AAt?$AAi?$AAp?$AAs?$AA_?$AAc?$AAl?$AAa?$AAs?$AAs?$AA3?$AA2?$AA?$AA@ 5f8afa74     tooltip.obj
 0002:00004a98       ?classCMiniFrameWnd@CMiniFrameWnd@@2UCRuntimeClass@@B 5f8afa98     winmini.obj
 0002:00004ab0       ??_C@_0O@NPLL@CMiniFrameWnd?$AA@ 5f8afab0     winmini.obj
 0002:00004ac0       ?messageMap@CMiniFrameWnd@@1UAFX_MSGMAP@@B 5f8afac0     winmini.obj
 0002:00004ac8       ?_messageEntries@CMiniFrameWnd@@0QBUAFX_MSGMAP_ENTRY@@B 5f8afac8     winmini.obj
 0002:00004c4c       ??_7CMiniFrameWnd@@6B@     5f8afc4c     winmini.obj
 0002:00004d48       ??_C@_1BI@PPN@?$AAS?$AAm?$AAa?$AAl?$AAl?$AA?5?$AAF?$AAo?$AAn?$AAt?$AAs?$AA?$AA@ 5f8afd48     winmini.obj
 0002:00004d60       ??_C@_1BC@NHJA@?$AAT?$AAe?$AAr?$AAm?$AAi?$AAn?$AAa?$AAl?$AA?$AA@ 5f8afd60     winmini.obj
 0002:00004d74       ??_C@_1HK@GNFN@?$AAW?$AAa?$AAr?$AAn?$AAi?$AAn?$AAg?$AA?3?$AA?5?$AAf?$AAa?$AAi?$AAl?$AAe?$AAd?$AA?5?$AAt?$AAo?$AA?5?$AAr@ 5f8afd74     winhand.obj
 0002:00004df0       ??_C@_1FM@FGMM@?$AAW?$AAa?$AAr?$AAn?$AAi?$AAn?$AAg?$AA?3?$AA?5?$AAT?$AAe?$AAm?$AAp?$AA?5?$AAm?$AAa?$AAp?$AA?5?$AAl?$AAo@ 5f8afdf0     winmain.obj
 0002:00004e4c       ??_C@_1FC@IBEO@?$AAW?$AAa?$AAr?$AAn?$AAi?$AAn?$AAg?$AA?3?$AA?5?$AAD?$AAe?$AAs?$AAt?$AAr?$AAo?$AAy?$AAi?$AAn?$AAg?$AA?5@ 5f8afe4c     winmain.obj
 0002:00004ea0       ??_C@_0M@BKC@winmain?4cpp?$AA@ 5f8afea0     winmain.obj
 0002:00004eb0       ?messageMap@CControlBar@@1UAFX_MSGMAP@@B 5f8afeb0     barcore.obj
 0002:00004eb8       ?_messageEntries@CControlBar@@0QBUAFX_MSGMAP_ENTRY@@B 5f8afeb8     barcore.obj
 0002:0000506c       ??_7CControlBar@@6B@       5f8b006c     barcore.obj
 0002:00005154       ??_C@_0BC@BDB@?6m_bAutoDelete?5?$DN?5?$AA@ 5f8b0154     barcore.obj
 0002:00005168       ??_C@_0N@DDAM@?6m_nCount?5?$DN?5?$AA@ 5f8b0168     barcore.obj
 0002:00005178       ??_C@_0BD@OGL@?6m_cxDefaultGap?5?$DN?5?$AA@ 5f8b0178     barcore.obj
 0002:0000518c       ??_C@_0BF@HKFD@?6m_cyBottomBorder?5?$DN?5?$AA@ 5f8b018c     barcore.obj
 0002:000051a4       ??_C@_0BC@JBOA@?6m_cyTopBorder?5?$DN?5?$AA@ 5f8b01a4     barcore.obj
 0002:000051b8       ??_C@_0BE@MIIC@?6m_cxRightBorder?5?$DN?5?$AA@ 5f8b01b8     barcore.obj
 0002:000051cc       ??_C@_0BD@BEEP@?6m_cxLeftBorder?5?$DN?5?$AA@ 5f8b01cc     barcore.obj
 0002:000051e0       ?classCToolBar@CToolBar@@2UCRuntimeClass@@B 5f8b01e0     bartool.obj
 0002:000051f8       ??_C@_08NCEL@CToolBar?$AA@ 5f8b01f8     bartool.obj
 0002:00005208       ?messageMap@CToolBar@@1UAFX_MSGMAP@@B 5f8b0208     bartool.obj
 0002:00005210       ?_messageEntries@CToolBar@@0QBUAFX_MSGMAP_ENTRY@@B 5f8b0210     bartool.obj
 0002:00005348       ?_afxSysColorMap@@3QBUAFX_COLORMAP@@B 5f8b0348     bartool.obj
 0002:00005368       ??_C@_0O@CDEE@DllGetVersion?$AA@ 5f8b0368     bartool.obj
 0002:00005378       ??_C@_1BA@NPHH@?$AAM?$AAa?$AAr?$AAl?$AAe?$AAt?$AAt?$AA?$AA@ 5f8b0378     bartool.obj
 0002:0000538c       ??_7CToolBar@@6B@          5f8b038c     bartool.obj
 0002:00005478       ??_C@_1CA@IKCD@?$AAT?$AAo?$AAo?$AAl?$AAb?$AAa?$AAr?$AAW?$AAi?$AAn?$AAd?$AAo?$AAw?$AA3?$AA2?$AA?$AA@ 5f8b0478     bartool.obj
 0002:00005498       ??_C@_1HE@GHHH@?$AAW?$AAa?$AAr?$AAn?$AAi?$AAn?$AAg?$AA?3?$AA?5?$AAC?$AAT?$AAo?$AAo?$AAl?$AAB?$AAa?$AAr?$AA?3?$AA?3?$AAS@ 5f8b0498     bartool.obj
 0002:00005510       ??_7CToolCmdUI@@6B@        5f8b0510     bartool.obj
 0002:00005520       ??_C@_02JCCC@?6?$HN?$AA@   5f8b0520     bartool.obj
 0002:00005524       ??_C@_0CB@DJKL@?6?7iImage?5?$CIbitmap?5image?5index?$CJ?5?$DN?5@ 5f8b0524     bartool.obj
 0002:00005548       ??_C@_0BO@PCPI@?6?7iImage?5?$CIseparator?5width?$CJ?5?$DN?5?$AA@ 5f8b0548     bartool.obj
 0002:00005568       ??_C@_0M@GLAJ@?6?7nStyle?5?$DN?5?$AA@ 5f8b0568     bartool.obj
 0002:00005574       ??_C@_08LINB@?6?7nID?5?$DN?5?$AA@ 5f8b0574     bartool.obj
 0002:00005580       ??_C@_0BB@ELCK@?6toolbar?5button?$FL?$AA@ 5f8b0580     bartool.obj
 0002:00005594       ??_C@_05EJJM@?$FN?5?$DN?5?$HL?$AA@ 5f8b0594     bartool.obj
 0002:0000559c       ??_C@_0BA@BCFB@?6m_sizeImage?5?$DN?5?$AA@ 5f8b059c     bartool.obj
 0002:000055ac       ??_C@_0BB@BMHK@?6m_sizeButton?5?$DN?5?$AA@ 5f8b05ac     bartool.obj
 0002:000055c0       ??_C@_0BF@GKOI@?6m_hRsrcImageWell?5?$DN?5?$AA@ 5f8b05c0     bartool.obj
 0002:000055d8       ??_C@_0BF@ONDI@?6m_hInstImageWell?5?$DN?5?$AA@ 5f8b05d8     bartool.obj
 0002:000055f0       ??_C@_0BC@DKGE@m_hbmImageWell?5?$DN?5?$AA@ 5f8b05f0     bartool.obj
 0002:00005608       ?classCDialogBar@CDialogBar@@2UCRuntimeClass@@B 5f8b0608     bardlg.obj
 0002:00005620       ??_C@_0L@KJOE@CDialogBar?$AA@ 5f8b0620     bardlg.obj
 0002:00005630       ?messageMap@CDialogBar@@1UAFX_MSGMAP@@B 5f8b0630     bardlg.obj
 0002:00005638       ?_messageEntries@CDialogBar@@0QBUAFX_MSGMAP_ENTRY@@B 5f8b0638     bardlg.obj
 0002:0000566c       ??_7CDialogBar@@6B@        5f8b066c     bardlg.obj
 0002:00005754       ??_C@_1HG@BJFF@?$AAW?$AAa?$AAr?$AAn?$AAi?$AAn?$AAg?$AA?3?$AA?5?$AAC?$AAr?$AAe?$AAa?$AAt?$AAe?$AAD?$AAl?$AAg?$AAC?$AAo@ 5f8b0754     bardlg.obj
 0002:000057d0       ?classCStatusBar@CStatusBar@@2UCRuntimeClass@@B 5f8b07d0     barstat.obj
 0002:000057e8       ??_C@_0L@BNMI@CStatusBar?$AA@ 5f8b07e8     barstat.obj
 0002:000057f8       ?messageMap@CStatusBar@@1UAFX_MSGMAP@@B 5f8b07f8     barstat.obj
 0002:00005800       ?_messageEntries@CStatusBar@@0QBUAFX_MSGMAP_ENTRY@@B 5f8b0800     barstat.obj
 0002:0000590c       ??_7CStatusBar@@6B@        5f8b090c     barstat.obj
 0002:000059f8       ??_C@_1CG@LDD@?$AAm?$AAs?$AAc?$AAt?$AAl?$AAs?$AA_?$AAs?$AAt?$AAa?$AAt?$AAu?$AAs?$AAb?$AAa?$AAr?$AA3?$AA2?$AA?$AA@ 5f8b09f8     barstat.obj
 0002:00005a20       ??_C@_1GE@LEPD@?$AAW?$AAa?$AAr?$AAn?$AAi?$AAn?$AAg?$AA?3?$AA?5?$AAf?$AAa?$AAi?$AAl?$AAe?$AAd?$AA?5?$AAt?$AAo?$AA?5?$AAl@ 5f8b0a20     barstat.obj
 0002:00005a88       ??_7CStatusCmdUI@@6B@      5f8b0a88     barstat.obj
 0002:00005a98       ??_C@_03JNEF@?6?7?$HN?$AA@ 5f8b0a98     barstat.obj
 0002:00005a9c       ??_C@_0N@LFK@?6?7strText?5?$DN?5?$AA@ 5f8b0a9c     barstat.obj
 0002:00005aac       ??_C@_0M@KPHB@?6?7cxText?5?$DN?5?$AA@ 5f8b0aac     barstat.obj
 0002:00005ab8       ??_C@_0O@EBFM@?6status?5pane?$FL?$AA@ 5f8b0ab8     barstat.obj
 0002:00005ac8       ?classCMiniDockFrameWnd@CMiniDockFrameWnd@@2UCRuntimeClass@@B 5f8b0ac8     bardock.obj
 0002:00005ae0       ??_C@_0BC@NGKE@CMiniDockFrameWnd?$AA@ 5f8b0ae0     bardock.obj
 0002:00005af8       ?classCDockBar@CDockBar@@2UCRuntimeClass@@B 5f8b0af8     bardock.obj
 0002:00005b10       ??_C@_08EABA@CDockBar?$AA@ 5f8b0b10     bardock.obj
 0002:00005b20       ?messageMap@CMiniDockFrameWnd@@1UAFX_MSGMAP@@B 5f8b0b20     bardock.obj
 0002:00005b28       ?_messageEntries@CMiniDockFrameWnd@@0QBUAFX_MSGMAP_ENTRY@@B 5f8b0b28     bardock.obj
 0002:00005ba0       ?messageMap@CDockBar@@1UAFX_MSGMAP@@B 5f8b0ba0     bardock.obj
 0002:00005ba8       ?_messageEntries@CDockBar@@0QBUAFX_MSGMAP_ENTRY@@B 5f8b0ba8     bardock.obj
 0002:00005c3c       ??_7CDockBar@@6B@          5f8b0c3c     bardock.obj
 0002:00005d28       ??_C@_0O@PMCC@?6m_bFloating?5?$AA@ 5f8b0d28     bardock.obj
 0002:00005d38       ??_C@_0L@KJHL@m_arrBars?5?$AA@ 5f8b0d38     bardock.obj
 0002:00005d48       ??_7CMiniDockFrameWnd@@6B@ 5f8b0d48     bardock.obj
 0002:00005e4c       ??_7CDockContext@@6B@      5f8b0e4c     dockcont.obj
 0002:00005e58       ??_C@_0L@HPAN@CDockState?$AA@ 5f8b0e58     dockstat.obj
 0002:00005e64       ?_afxBar@@3QBGB            5f8b0e64     dockstat.obj
 0002:00005e74       ?_afxScreenCY@@3QBGB       5f8b0e74     dockstat.obj
 0002:00005e88       ?_afxScreenCX@@3QBGB       5f8b0e88     dockstat.obj
 0002:00005e9c       ?_afxBars@@3QBGB           5f8b0e9c     dockstat.obj
 0002:00005ea8       ?_afxFloating@@3QBGB       5f8b0ea8     dockstat.obj
 0002:00005ebc       ?_afxHorz@@3QBGB           5f8b0ebc     dockstat.obj
 0002:00005ec8       ?_afxBarID@@3QBGB          5f8b0ec8     dockstat.obj
 0002:00005ed4       ?_afxMRUFloatYPos@@3QBGB   5f8b0ed4     dockstat.obj
 0002:00005ef0       ?_afxMRUFloatXPos@@3QBGB   5f8b0ef0     dockstat.obj
 0002:00005f0c       ?_afxMRUFloatStyle@@3QBGB  5f8b0f0c     dockstat.obj
 0002:00005f28       ?_afxMRUDockBottomPos@@3QBGB 5f8b0f28     dockstat.obj
 0002:00005f4c       ?_afxMRUDockTopPos@@3QBGB  5f8b0f4c     dockstat.obj
 0002:00005f68       ?_afxMRUDockRightPos@@3QBGB 5f8b0f68     dockstat.obj
 0002:00005f88       ?_afxMRUDockLeftPos@@3QBGB 5f8b0f88     dockstat.obj
 0002:00005fa8       ?_afxMRUDockID@@3QBGB      5f8b0fa8     dockstat.obj
 0002:00005fbc       ?_afxDocking@@3QBGB        5f8b0fbc     dockstat.obj
 0002:00005fcc       ?_afxMRUWidth@@3QBGB       5f8b0fcc     dockstat.obj
 0002:00005fe0       ?_afxYPos@@3QBGB           5f8b0fe0     dockstat.obj
 0002:00005fec       ?_afxXPos@@3QBGB           5f8b0fec     dockstat.obj
 0002:00005ff8       ?_afxSummarySection@@3QBGB 5f8b0ff8     dockstat.obj
 0002:00006010       ?_afxBarSection@@3QBGB     5f8b1010     dockstat.obj
 0002:00006024       ?_afxVisible@@3QBGB        5f8b1024     dockstat.obj
 0002:00006038       ??_7CDockState@@6B@        5f8b1038     dockstat.obj
 0002:00006050       ?classCPreviewDC@CPreviewDC@@2UCRuntimeClass@@B 5f8b1050     dcprev.obj
 0002:00006068       ??_C@_0L@MCGA@CPreviewDC?$AA@ 5f8b1068     dcprev.obj
 0002:00006078       ??_7CPreviewDC@@6B@        5f8b1078     dcprev.obj
 0002:000060f4       ??_C@_0P@DFJI@Scale?5Factor?3?5?$AA@ 5f8b10f4     dcprev.obj
 0002:00006104       ??_C@_01FDLN@?1?$AA@       5f8b1104     dcprev.obj
 0002:00006108       ??_C@_01POCP@?7?$AA@       5f8b1108     dcprev.obj
 0002:0000610c       ??_C@_01PFH@A?$AA@         5f8b110c     dcprev.obj
 0002:00006110       ??_C@_1HE@MPEO@?$AAT?$AAe?$AAx?$AAt?$AAO?$AAu?$AAt?$AA?$CI?$AA?$CJ?$AA?5?$AAs?$AAu?$AAb?$AAs?$AAt?$AAi?$AAt?$AAu?$AAt?$AAe@ 5f8b1110     dcprev.obj
 0002:00006188       ?classCMetaFileDC@CMetaFileDC@@2UCRuntimeClass@@B 5f8b1188     dcmeta.obj
 0002:000061a0       ??_C@_0M@MIEC@CMetaFileDC?$AA@ 5f8b11a0     dcmeta.obj
 0002:000061b0       ??_7CMetaFileDC@@6B@       5f8b11b0     dcmeta.obj
 0002:0000622c       ??_C@_1GO@BKCN@?$AAM?$AAu?$AAs?$AAt?$AA?5?$AAu?$AAs?$AAe?$AA?5?$AAC?$AAr?$AAe?$AAa?$AAt?$AAe?$AA?$CI?$AA?$CJ?$AA?5?$AAo?$AAr@ 5f8b122c     dcmeta.obj
 0002:0000629c       ??_C@_1GC@JNEN@?$AAM?$AAu?$AAs?$AAt?$AA?5?$AAu?$AAs?$AAe?$AA?5?$AAC?$AAl?$AAo?$AAs?$AAe?$AA?$CI?$AA?$CJ?$AA?5?$AAt?$AAo?$AA?5@ 5f8b129c     dcmeta.obj
 0002:00006300       ??_C@_1GE@PPOB@?$AAW?$AAa?$AAr?$AAn?$AAi?$AAn?$AAg?$AA?$CB?$AA?5?$AAD?$AAe?$AAs?$AAt?$AAr?$AAo?$AAy?$AAi?$AAn?$AAg?$AA?5@ 5f8b1300     dcmeta.obj
 0002:000063a0       ?_afxRectInfo@@3QBUAFX_RECTINFO@@B 5f8b13a0     trckrect.obj
 0002:000063c0       ?_afxHandleInfo@@3QBUAFX_HANDLEINFO@@B 5f8b13c0     trckrect.obj
 0002:000064c0       ?classCReBar@CReBar@@2UCRuntimeClass@@B 5f8b14c0     barcool.obj
 0002:000064d8       ??_C@_06JANL@CReBar?$AA@   5f8b14d8     barcool.obj
 0002:000064e0       ?messageMap@CReBar@@1UAFX_MSGMAP@@B 5f8b14e0     barcool.obj
 0002:000064e8       ?_messageEntries@CReBar@@0QBUAFX_MSGMAP_ENTRY@@B 5f8b14e8     barcool.obj
 0002:000065dc       ??_7CReBar@@6B@            5f8b15dc     barcool.obj
 0002:000066c4       ??_C@_1BM@CPLN@?$AAR?$AAe?$AAB?$AAa?$AAr?$AAW?$AAi?$AAn?$AAd?$AAo?$AAw?$AA3?$AA2?$AA?$AA@ 5f8b16c4     barcool.obj
 0002:000066e0       ?classCScrollBar@CScrollBar@@2UCRuntimeClass@@B 5f8b16e0     winctrl1.obj
 0002:000066f8       ??_C@_0L@JCLK@CScrollBar?$AA@ 5f8b16f8     winctrl1.obj
 0002:00006708       ?classCEdit@CEdit@@2UCRuntimeClass@@B 5f8b1708     winctrl1.obj
 0002:00006720       ??_C@_05KKIE@CEdit?$AA@    5f8b1720     winctrl1.obj
 0002:00006728       ?classCComboBox@CComboBox@@2UCRuntimeClass@@B 5f8b1728     winctrl1.obj
 0002:00006740       ??_C@_09JMHE@CComboBox?$AA@ 5f8b1740     winctrl1.obj
 0002:00006750       ?classCListBox@CListBox@@2UCRuntimeClass@@B 5f8b1750     winctrl1.obj
 0002:00006768       ??_C@_08NBK@CListBox?$AA@  5f8b1768     winctrl1.obj
 0002:00006778       ?classCButton@CButton@@2UCRuntimeClass@@B 5f8b1778     winctrl1.obj
 0002:00006790       ??_C@_07NNHJ@CButton?$AA@  5f8b1790     winctrl1.obj
 0002:00006798       ?classCStatic@CStatic@@2UCRuntimeClass@@B 5f8b1798     winctrl1.obj
 0002:000067b0       ??_C@_07HEEJ@CStatic?$AA@  5f8b17b0     winctrl1.obj
 0002:000067b8       ??_C@_1O@GCMM@?$AAS?$AAT?$AAA?$AAT?$AAI?$AAC?$AA?$AA@ 5f8b17b8     winctrl1.obj
 0002:000067c8       ??_C@_1O@GKDM@?$AAB?$AAU?$AAT?$AAT?$AAO?$AAN?$AA?$AA@ 5f8b17c8     winctrl1.obj
 0002:000067d8       ??_C@_1BA@BJGI@?$AAL?$AAI?$AAS?$AAT?$AAB?$AAO?$AAX?$AA?$AA@ 5f8b17d8     winctrl1.obj
 0002:000067e8       ??_C@_1BC@DNEF@?$AAC?$AAO?$AAM?$AAB?$AAO?$AAB?$AAO?$AAX?$AA?$AA@ 5f8b17e8     winctrl1.obj
 0002:000067fc       ??_C@_19CJM@?$AAE?$AAD?$AAI?$AAT?$AA?$AA@ 5f8b17fc     winctrl1.obj
 0002:00006808       ??_C@_1BE@JGEP@?$AAS?$AAC?$AAR?$AAO?$AAL?$AAL?$AAB?$AAA?$AAR?$AA?$AA@ 5f8b1808     winctrl1.obj
 0002:00006820       ?classCRichEditCtrl@CRichEditCtrl@@2UCRuntimeClass@@B 5f8b1820     winctrl2.obj
 0002:00006838       ??_C@_0O@KLOD@CRichEditCtrl?$AA@ 5f8b1838     winctrl2.obj
 0002:00006848       ?classCTempImageList@CTempImageList@@2UCRuntimeClass@@B 5f8b1848     winctrl2.obj
 0002:00006860       ??_C@_0P@OCOD@CTempImageList?$AA@ 5f8b1860     winctrl2.obj
 0002:00006870       ?classCImageList@CImageList@@2UCRuntimeClass@@B 5f8b1870     winctrl2.obj
 0002:00006888       ??_C@_0L@HBAH@CImageList?$AA@ 5f8b1888     winctrl2.obj
 0002:00006898       ?classCStatusBarCtrl@CStatusBarCtrl@@2UCRuntimeClass@@B 5f8b1898     winctrl2.obj
 0002:000068b0       ??_C@_0P@NMO@CStatusBarCtrl?$AA@ 5f8b18b0     winctrl2.obj
 0002:000068c0       ?classCToolBarCtrl@CToolBarCtrl@@2UCRuntimeClass@@B 5f8b18c0     winctrl2.obj
 0002:000068d8       ??_C@_0N@HNL@CToolBarCtrl?$AA@ 5f8b18d8     winctrl2.obj
 0002:000068e8       ?classCListCtrl@CListCtrl@@2UCRuntimeClass@@B 5f8b18e8     winctrl2.obj
 0002:00006900       ??_C@_09IAHO@CListCtrl?$AA@ 5f8b1900     winctrl2.obj
 0002:00006910       ?classCTreeCtrl@CTreeCtrl@@2UCRuntimeClass@@B 5f8b1910     winctrl2.obj
 0002:00006928       ??_C@_09CIBI@CTreeCtrl?$AA@ 5f8b1928     winctrl2.obj
 0002:00006938       ?classCTabCtrl@CTabCtrl@@2UCRuntimeClass@@B 5f8b1938     winctrl2.obj
 0002:00006950       ??_C@_08IFFI@CTabCtrl?$AA@ 5f8b1950     winctrl2.obj
 0002:00006960       ?classCAnimateCtrl@CAnimateCtrl@@2UCRuntimeClass@@B 5f8b1960     winctrl2.obj
 0002:00006978       ??_C@_0N@PPEM@CAnimateCtrl?$AA@ 5f8b1978     winctrl2.obj
 0002:00006988       ?classCHotKeyCtrl@CHotKeyCtrl@@2UCRuntimeClass@@B 5f8b1988     winctrl2.obj
 0002:000069a0       ??_C@_0M@IPHC@CHotKeyCtrl?$AA@ 5f8b19a0     winctrl2.obj
 0002:000069b0       ?classCHeaderCtrl@CHeaderCtrl@@2UCRuntimeClass@@B 5f8b19b0     winctrl2.obj
 0002:000069c8       ??_C@_0M@HNGK@CHeaderCtrl?$AA@ 5f8b19c8     winctrl2.obj
 0002:000069d8       ?classCComboBoxEx@CComboBoxEx@@2UCRuntimeClass@@B 5f8b19d8     winctrl2.obj
 0002:000069f0       ??_C@_0M@BDBF@CComboBoxEx?$AA@ 5f8b19f0     winctrl2.obj
 0002:00006a00       ?classCProgressCtrl@CProgressCtrl@@2UCRuntimeClass@@B 5f8b1a00     winctrl2.obj
 0002:00006a18       ??_C@_0O@ECFI@CProgressCtrl?$AA@ 5f8b1a18     winctrl2.obj
 0002:00006a28       ?classCSliderCtrl@CSliderCtrl@@2UCRuntimeClass@@B 5f8b1a28     winctrl2.obj
 0002:00006a40       ??_C@_0M@POGH@CSliderCtrl?$AA@ 5f8b1a40     winctrl2.obj
 0002:00006a50       ?classCSpinButtonCtrl@CSpinButtonCtrl@@2UCRuntimeClass@@B 5f8b1a50     winctrl2.obj
 0002:00006a68       ??_C@_0BA@MANL@CSpinButtonCtrl?$AA@ 5f8b1a68     winctrl2.obj
 0002:00006a78       ?classCDragListBox@CDragListBox@@2UCRuntimeClass@@B 5f8b1a78     winctrl2.obj
 0002:00006a90       ??_C@_0N@BPBM@CDragListBox?$AA@ 5f8b1a90     winctrl2.obj
 0002:00006ab0       ?messageMap@CTabCtrl@@1UAFX_MSGMAP@@B 5f8b1ab0     winctrl2.obj
 0002:00006ab8       ?_messageEntries@CTabCtrl@@0QBUAFX_MSGMAP_ENTRY@@B 5f8b1ab8     winctrl2.obj
 0002:00006ae8       ?messageMap@CTreeCtrl@@1UAFX_MSGMAP@@B 5f8b1ae8     winctrl2.obj
 0002:00006af0       ?_messageEntries@CTreeCtrl@@0QBUAFX_MSGMAP_ENTRY@@B 5f8b1af0     winctrl2.obj
 0002:00006b20       ?messageMap@CListCtrl@@1UAFX_MSGMAP@@B 5f8b1b20     winctrl2.obj
 0002:00006b28       ?_messageEntries@CListCtrl@@0QBUAFX_MSGMAP_ENTRY@@B 5f8b1b28     winctrl2.obj
 0002:00006b58       ?messageMap@CToolBarCtrl@@1UAFX_MSGMAP@@B 5f8b1b58     winctrl2.obj
 0002:00006b60       ?_messageEntries@CToolBarCtrl@@0QBUAFX_MSGMAP_ENTRY@@B 5f8b1b60     winctrl2.obj
 0002:00006b94       ??_7CDragListBox@@6B@      5f8b1b94     winctrl2.obj
 0002:00006c84       ??_7CToolBarCtrl@@6B@      5f8b1c84     winctrl2.obj
 0002:00006d48       ??_7CStatusBarCtrl@@6B@    5f8b1d48     winctrl2.obj
 0002:00006e0c       ??_C@_1BM@DGLL@?$AAS?$AAy?$AAs?$AAL?$AAi?$AAs?$AAt?$AAV?$AAi?$AAe?$AAw?$AA3?$AA2?$AA?$AA@ 5f8b1e0c     winctrl2.obj
 0002:00006e2c       ??_7CListCtrl@@6B@         5f8b1e2c     winctrl2.obj
 0002:00006ef0       ??_C@_1BM@DBCI@?$AAS?$AAy?$AAs?$AAT?$AAr?$AAe?$AAe?$AAV?$AAi?$AAe?$AAw?$AA3?$AA2?$AA?$AA@ 5f8b1ef0     winctrl2.obj
 0002:00006f10       ??_7CTreeCtrl@@6B@         5f8b1f10     winctrl2.obj
 0002:00006fd0       ??_C@_1CA@JDKO@?$AAm?$AAs?$AAc?$AAt?$AAl?$AAs?$AA_?$AAu?$AAp?$AAd?$AAo?$AAw?$AAn?$AA3?$AA2?$AA?$AA@ 5f8b1fd0     winctrl2.obj
 0002:00006ff4       ??_7CSpinButtonCtrl@@6B@   5f8b1ff4     winctrl2.obj
 0002:000070b4       ??_C@_1CE@EHFJ@?$AAm?$AAs?$AAc?$AAt?$AAl?$AAs?$AA_?$AAt?$AAr?$AAa?$AAc?$AAk?$AAb?$AAa?$AAr?$AA3?$AA2?$AA?$AA@ 5f8b20b4     winctrl2.obj
 0002:000070dc       ??_7CSliderCtrl@@6B@       5f8b20dc     winctrl2.obj
 0002:0000719c       ??_C@_1CE@ECOJ@?$AAm?$AAs?$AAc?$AAt?$AAl?$AAs?$AA_?$AAp?$AAr?$AAo?$AAg?$AAr?$AAe?$AAs?$AAs?$AA3?$AA2?$AA?$AA@ 5f8b219c     winctrl2.obj
 0002:000071c4       ??_7CProgressCtrl@@6B@     5f8b21c4     winctrl2.obj
 0002:00007284       ??_C@_1BI@FFDG@?$AAS?$AAy?$AAs?$AAH?$AAe?$AAa?$AAd?$AAe?$AAr?$AA3?$AA2?$AA?$AA@ 5f8b2284     winctrl2.obj
 0002:000072a0       ??_7CHeaderCtrl@@6B@       5f8b22a0     winctrl2.obj
 0002:00007364       ??_C@_1CA@BKDN@?$AAm?$AAs?$AAc?$AAt?$AAl?$AAs?$AA_?$AAh?$AAo?$AAt?$AAk?$AAe?$AAy?$AA3?$AA2?$AA?$AA@ 5f8b2364     winctrl2.obj
 0002:00007388       ??_7CHotKeyCtrl@@6B@       5f8b2388     winctrl2.obj
 0002:00007448       ??_C@_1CA@OIHL@?$AAS?$AAy?$AAs?$AAT?$AAa?$AAb?$AAC?$AAo?$AAn?$AAt?$AAr?$AAo?$AAl?$AA3?$AA2?$AA?$AA@ 5f8b2448     winctrl2.obj
 0002:0000746c       ??_7CTabCtrl@@6B@          5f8b246c     winctrl2.obj
 0002:00007530       ??_C@_1BK@MPBJ@?$AAS?$AAy?$AAs?$AAA?$AAn?$AAi?$AAm?$AAa?$AAt?$AAe?$AA3?$AA2?$AA?$AA@ 5f8b2530     winctrl2.obj
 0002:00007550       ??_7CAnimateCtrl@@6B@      5f8b2550     winctrl2.obj
 0002:00007614       ??_7CRichEditCtrl@@6B@     5f8b2614     winctrl2.obj
 0002:000076d8       ??_7CImageList@@6B@        5f8b26d8     winctrl2.obj
 0002:000076ec       ??_C@_0BA@ENPN@m_hImageList?5?$DN?5?$AA@ 5f8b26ec     winctrl2.obj
 0002:00007700       ??_7CTempImageList@@6B@    5f8b2700     winctrl2.obj
 0002:00007718       ?classCCheckListBox@CCheckListBox@@2UCRuntimeClass@@B 5f8b2718     winctrl3.obj
 0002:00007730       ??_C@_0O@KOFM@CCheckListBox?$AA@ 5f8b2730     winctrl3.obj
 0002:00007740       ?messageMap@CCheckListBox@@1UAFX_MSGMAP@@B 5f8b2740     winctrl3.obj
 0002:00007748       ?_messageEntries@CCheckListBox@@0QBUAFX_MSGMAP_ENTRY@@B 5f8b2748     winctrl3.obj
 0002:000078b4       ??_7_AFX_CHECKLIST_STATE@@6B@ 5f8b28b4     winctrl3.obj
 0002:000078bc       ??_7_AFX_RICHEDIT_STATE@@6B@ 5f8b28bc     winctrl4.obj
 0002:000078c0       ??_C@_0N@GEKM@RICHED32?4DLL?$AA@ 5f8b28c0     winctrl4.obj
 0002:000078d0       ??_C@_1BC@IAEH@?$AAR?$AAI?$AAC?$AAH?$AAE?$AAD?$AAI?$AAT?$AA?$AA@ 5f8b28d0     winctrl4.obj
 0002:000078e8       ?classCBitmapButton@CBitmapButton@@2UCRuntimeClass@@B 5f8b28e8     winbtn.obj
 0002:00007900       ??_C@_0O@FPOC@CBitmapButton?$AA@ 5f8b2900     winbtn.obj
 0002:00007910       ??_C@_1FG@FIPG@?$AAF?$AAa?$AAi?$AAl?$AAe?$AAd?$AA?5?$AAt?$AAo?$AA?5?$AAl?$AAo?$AAa?$AAd?$AA?5?$AAb?$AAi?$AAt?$AAm?$AAa@ 5f8b2910     winbtn.obj
 0002:00007968       ??_C@_1FC@CJBJ@?$AAF?$AAa?$AAi?$AAl?$AAe?$AAd?$AA?5?$AAt?$AAo?$AA?5?$AAl?$AAo?$AAa?$AAd?$AA?5?$AAb?$AAi?$AAt?$AAm?$AAa@ 5f8b2968     winbtn.obj
 0002:000079bc       ??_C@_13LOIM@?$AAU?$AA?$AA@ 5f8b29bc     winbtn.obj
 0002:000079c0       ??_C@_13MNPA@?$AAD?$AA?$AA@ 5f8b29c0     winbtn.obj
 0002:000079c4       ??_C@_13GJNN@?$AAF?$AA?$AA@ 5f8b29c4     winbtn.obj
 0002:000079c8       ??_C@_13DEHF@?$AAX?$AA?$AA@ 5f8b29c8     winbtn.obj
 0002:000079cc       ??_C@_0BF@DEP@?6m_bitmapDisabled?5?$DN?5?$AA@ 5f8b29cc     winbtn.obj
 0002:000079e4       ??_C@_0BC@BPAL@?6m_bitmapFocus?5?$DN?5?$AA@ 5f8b29e4     winbtn.obj
 0002:000079f8       ??_C@_0BA@CKJB@?6m_bitmapSel?5?$DN?5?$AA@ 5f8b29f8     winbtn.obj
 0002:00007a08       ??_C@_0M@KFMF@m_bitmap?5?$DN?5?$AA@ 5f8b2a08     winbtn.obj
 0002:00007a18       ?classCDialog@CDialog@@2UCRuntimeClass@@B 5f8b2a18     dlgcore.obj
 0002:00007a30       ??_C@_07IJJI@CDialog?$AA@  5f8b2a30     dlgcore.obj
 0002:00007a38       ?messageMap@CDialog@@1UAFX_MSGMAP@@B 5f8b2a38     dlgcore.obj
 0002:00007a40       ?_messageEntries@CDialog@@0QBUAFX_MSGMAP_ENTRY@@B 5f8b2a40     dlgcore.obj
 0002:00007b18       ??_C@_19JGFH@?$AAE?$AAd?$AAi?$AAt?$AA?$AA@ 5f8b2b18     dlgcore.obj
 0002:00007b24       ??_C@_1GA@EDDJ@?$AAI?$AAG?$AAN?$AAO?$AAR?$AAI?$AAN?$AAG?$AA?5?$AAc?$AAo?$AAm?$AAm?$AAa?$AAn?$AAd?$AA?5?$AAi?$AAd?$AA?5@ 5f8b2b24     dlgcore.obj
 0002:00007b84       ??_C@_1EG@EKMI@?$AAR?$AAo?$AAu?$AAt?$AAi?$AAn?$AAg?$AA?5?$AAc?$AAo?$AAm?$AAm?$AAa?$AAn?$AAd?$AA?5?$AAi?$AAd?$AA?5?$AA0@ 5f8b2b84     dlgcore.obj
 0002:00007bcc       ??_C@_1FI@EEBE@?$AAR?$AAo?$AAu?$AAt?$AAi?$AAn?$AAg?$AA?5?$AAc?$AAo?$AAm?$AAm?$AAa?$AAn?$AAd?$AA?5?$AAi?$AAd?$AA?5?$AA0@ 5f8b2bcc     dlgcore.obj
 0002:00007c28       ??_7CDialog@@6B@           5f8b2c28     dlgcore.obj
 0002:00007d00       ??_C@_1IE@PFFC@?$AA?7?$AAO?$AAn?$AAD?$AAe?$AAs?$AAt?$AAr?$AAo?$AAy?$AA?5?$AAo?$AAr?$AA?5?$AAP?$AAo?$AAs?$AAt?$AAN?$AAc@ 5f8b2d00     dlgcore.obj
 0002:00007d84       ??_C@_1HA@CDGA@?$AAW?$AAa?$AAr?$AAn?$AAi?$AAn?$AAg?$AA?3?$AA?5?$AAc?$AAa?$AAl?$AAl?$AAi?$AAn?$AAg?$AA?5?$AAD?$AAe?$AAs@ 5f8b2d84     dlgcore.obj
 0002:00007df4       ??_C@_1IA@FHOC@?$AAW?$AAa?$AAr?$AAn?$AAi?$AAn?$AAg?$AA?3?$AA?5?$AAD?$AAi?$AAa?$AAl?$AAo?$AAg?$AA?5?$AAc?$AAr?$AAe?$AAa@ 5f8b2df4     dlgcore.obj
 0002:00007e74       ??_C@_1HK@MLHB@?$AA?$DO?$AA?$DO?$AA?$DO?$AA?5?$AAY?$AAo?$AAu?$AA?5?$AAs?$AAh?$AAo?$AAu?$AAl?$AAd?$AA?5?$AAc?$AAa?$AAl?$AAl?$AA?5@ 5f8b2e74     dlgcore.obj
 0002:00007ef0       ??_C@_1HA@MEAE@?$AA?$DO?$AA?$DO?$AA?$DO?$AA?5?$AAA?$AAf?$AAx?$AAE?$AAn?$AAa?$AAb?$AAl?$AAe?$AAC?$AAo?$AAn?$AAt?$AAr?$AAo?$AAl@ 5f8b2ef0     dlgcore.obj
 0002:00007f60       ??_C@_1EM@OJLL@?$AA?$DO?$AA?$DO?$AA?$DO?$AA?5?$AAI?$AAf?$AA?5?$AAt?$AAh?$AAi?$AAs?$AA?5?$AAd?$AAi?$AAa?$AAl?$AAo?$AAg?$AA?5?$AAh@ 5f8b2f60     dlgcore.obj
 0002:00007fac       ??_C@_19OFHG@?$AAH?$AAe?$AAl?$AAv?$AA?$AA@ 5f8b2fac     dlgcore.obj
 0002:00007fb8       ??_C@_1BM@LDDO@?$AAM?$AAS?$AA?5?$AAS?$AAa?$AAn?$AAs?$AA?5?$AAS?$AAe?$AAr?$AAi?$AAf?$AA?$AA@ 5f8b2fb8     dlgcore.obj
 0002:00007fd4       ??_C@_1BK@PLLM@?$AAM?$AAS?$AA?5?$AAS?$AAh?$AAe?$AAl?$AAl?$AA?5?$AAD?$AAl?$AAg?$AA?$AA@ 5f8b2fd4     dlgcore.obj
 0002:00007ff0       ??_C@_1GO@DMJG@?$AAW?$AAa?$AAr?$AAn?$AAi?$AAn?$AAg?$AA?3?$AA?5?$AAC?$AAr?$AAe?$AAa?$AAt?$AAe?$AAD?$AAl?$AAg?$AAC?$AAo@ 5f8b2ff0     dlgcore.obj
 0002:00008060       ??_C@_1GA@HAPJ@?$AAW?$AAa?$AAr?$AAn?$AAi?$AAn?$AAg?$AA?3?$AA?5?$AAU?$AAp?$AAd?$AAa?$AAt?$AAe?$AAD?$AAa?$AAt?$AAa?$AA?5@ 5f8b3060     dlgcore.obj
 0002:000080c0       ??_C@_1GI@HBII@?$AAW?$AAa?$AAr?$AAn?$AAi?$AAn?$AAg?$AA?3?$AA?5?$AAE?$AAx?$AAe?$AAc?$AAu?$AAt?$AAe?$AAD?$AAl?$AAg?$AAI@ 5f8b30c0     dlgcore.obj
 0002:00008128       ??_C@_1FM@KEKB@?$AAU?$AAp?$AAd?$AAa?$AAt?$AAe?$AAD?$AAa?$AAt?$AAa?$AA?5?$AAf?$AAa?$AAi?$AAl?$AAe?$AAd?$AA?5?$AAd?$AAu@ 5f8b3128     dlgcore.obj
 0002:00008184       ??_C@_0BB@MJBE@?6m_pParentWnd?5?$DN?5?$AA@ 5f8b3184     dlgcore.obj
 0002:00008198       ??_C@_0BH@IMJH@?6m_lpDialogTemplate?5?$DN?5?$AA@ 5f8b3198     dlgcore.obj
 0002:000081b0       ??_C@_0BG@BCJN@?6m_hDialogTemplate?5?$DN?5?$AA@ 5f8b31b0     dlgcore.obj
 0002:000081c8       ??_C@_0BG@FAML@m_lpszTemplateName?5?$DN?5?$AA@ 5f8b31c8     dlgcore.obj
 0002:000081e0       ??_C@_1HE@HEMG@?$AAE?$AAR?$AAR?$AAO?$AAR?$AA?3?$AA?5?$AAD?$AAi?$AAa?$AAl?$AAo?$AAg?$AA?5?$AAw?$AAi?$AAt?$AAh?$AA?5?$AAI@ 5f8b31e0     dlgcore.obj
 0002:00008254       ??_C@_1GK@PAKD@?$AAE?$AAR?$AAR?$AAO?$AAR?$AA?3?$AA?5?$AAD?$AAi?$AAa?$AAl?$AAo?$AAg?$AA?5?$AAn?$AAa?$AAm?$AAe?$AAd?$AA?5@ 5f8b3254     dlgcore.obj
 0002:000082c0       ??_C@_1GE@IKGH@?$AAE?$AAR?$AAR?$AAO?$AAR?$AA?3?$AA?5?$AAD?$AAi?$AAa?$AAl?$AAo?$AAg?$AA?5?$AAw?$AAi?$AAt?$AAh?$AA?5?$AAI@ 5f8b32c0     dlgcore.obj
 0002:00008324       ??_C@_1FK@HEHB@?$AAE?$AAR?$AAR?$AAO?$AAR?$AA?3?$AA?5?$AAD?$AAi?$AAa?$AAl?$AAo?$AAg?$AA?5?$AAn?$AAa?$AAm?$AAe?$AAd?$AA?5@ 5f8b3324     dlgcore.obj
 0002:00008380       ??_C@_1GG@GKLA@?$AAW?$AAa?$AAr?$AAn?$AAi?$AAn?$AAg?$AA?3?$AA?5?$AAL?$AAo?$AAa?$AAd?$AAR?$AAe?$AAs?$AAo?$AAu?$AAr?$AAc@ 5f8b3380     dlgcore.obj
 0002:000083e8       ??_C@_1GK@BGD@?$AAE?$AAR?$AAR?$AAO?$AAR?$AA?3?$AA?5?$AAC?$AAa?$AAn?$AAn?$AAo?$AAt?$AA?5?$AAf?$AAi?$AAn?$AAd?$AA?5?$AAd@ 5f8b33e8     dlgcore.obj
 0002:00008454       ??_C@_1GA@GOLA@?$AAE?$AAR?$AAR?$AAO?$AAR?$AA?3?$AA?5?$AAC?$AAa?$AAn?$AAn?$AAo?$AAt?$AA?5?$AAf?$AAi?$AAn?$AAd?$AA?5?$AAd@ 5f8b3454     dlgcore.obj
 0002:000084b4       ??_C@_1GC@NIHI@?$AAE?$AAr?$AAr?$AAo?$AAr?$AA?3?$AA?5?$AAn?$AAo?$AA?5?$AAd?$AAa?$AAt?$AAa?$AA?5?$AAe?$AAx?$AAc?$AAh?$AAa@ 5f8b34b4     dlgdata.obj
 0002:00008518       ??_C@_1HK@MBCF@?$AAE?$AAr?$AAr?$AAo?$AAr?$AA?3?$AA?5?$AAf?$AAa?$AAi?$AAl?$AA?5?$AAv?$AAa?$AAl?$AAi?$AAd?$AAa?$AAt?$AAi@ 5f8b3518     dlgdata.obj
 0002:00008594       ??_C@_1HE@KHBN@?$AAW?$AAa?$AAr?$AAn?$AAi?$AAn?$AAg?$AA?3?$AA?5?$AAC?$AAD?$AAa?$AAt?$AAa?$AAE?$AAx?$AAc?$AAh?$AAa?$AAn@ 5f8b3594     dlgdata.obj
 0002:00008608       ??_C@_17MFIG@?$AA?$CF?$AAh?$AAd?$AA?$AA@ 5f8b3608     dlgdata.obj
 0002:00008610       ??_C@_17CGJG@?$AA?$CF?$AAs?$AAd?$AA?$AA@ 5f8b3610     dlgdata.obj
 0002:00008618       ??_C@_1HC@KKK@?$AAT?$AAe?$AAx?$AAt?$AA?5?$AAi?$AAn?$AA?5?$AAc?$AAo?$AAn?$AAt?$AAr?$AAo?$AAl?$AA?5?$AAI?$AAD?$AA?5?$AA?$CF@ 5f8b3618     dlgdata.obj
 0002:0000868c       ??_C@_1HA@DPGA@?$AAW?$AAa?$AAr?$AAn?$AAi?$AAn?$AAg?$AA?3?$AA?5?$AAd?$AAi?$AAa?$AAl?$AAo?$AAg?$AA?5?$AAd?$AAa?$AAt?$AAa@ 5f8b368c     dlgdata.obj
 0002:000086fc       ??_C@_1FM@JLBD@?$AAW?$AAa?$AAr?$AAn?$AAi?$AAn?$AAg?$AA?3?$AA?5?$AAs?$AAk?$AAi?$AAp?$AAp?$AAi?$AAn?$AAg?$AA?5?$AAn?$AAo@ 5f8b36fc     dlgdata.obj
 0002:00008758       ??_C@_1EI@FFBM@?$AAW?$AAa?$AAr?$AAn?$AAi?$AAn?$AAg?$AA?3?$AA?5?$AAn?$AAo?$AA?5?$AAl?$AAi?$AAs?$AAt?$AAb?$AAo?$AAx?$AA?5@ 5f8b3758     dlgdata.obj
 0002:000087a0       ??_C@_1FO@BCAI@?$AAW?$AAa?$AAr?$AAn?$AAi?$AAn?$AAg?$AA?3?$AA?5?$AAi?$AAn?$AAi?$AAt?$AAi?$AAa?$AAl?$AA?5?$AAd?$AAi?$AAa@ 5f8b37a0     dlgdata.obj
 0002:00008800       ??_C@_1IA@EPBF@?$AAW?$AAa?$AAr?$AAn?$AAi?$AAn?$AAg?$AA?3?$AA?5?$AAi?$AAn?$AAi?$AAt?$AAi?$AAa?$AAl?$AA?5?$AAd?$AAi?$AAa@ 5f8b3800     dlgdata.obj
 0002:00008880       __real@8@00000000000000000000 5f8b3880     dlgfloat.obj
 0002:00008888       ??_C@_19PPNN@?$AA?$CF?$AA?4?$AA?$CK?$AAg?$AA?$AA@ 5f8b3888     dlgfloat.obj
 0002:00008898       ?classCPropertySheetEx@CPropertySheetEx@@2UCRuntimeClass@@B 5f8b3898     dlgprop.obj
 0002:000088b0       ??_C@_0BB@NMHF@CPropertySheetEx?$AA@ 5f8b38b0     dlgprop.obj
 0002:000088c8       ?classCPropertyPageEx@CPropertyPageEx@@2UCRuntimeClass@@B 5f8b38c8     dlgprop.obj
 0002:000088e0       ??_C@_0BA@MOPN@CPropertyPageEx?$AA@ 5f8b38e0     dlgprop.obj
 0002:000088f0       ?classCPropertySheet@CPropertySheet@@2UCRuntimeClass@@B 5f8b38f0     dlgprop.obj
 0002:00008908       ??_C@_0P@PIP@CPropertySheet?$AA@ 5f8b3908     dlgprop.obj
 0002:00008918       ?classCPropertyPage@CPropertyPage@@2UCRuntimeClass@@B 5f8b3918     dlgprop.obj
 0002:00008930       ??_C@_0O@DMH@CPropertyPage?$AA@ 5f8b3930     dlgprop.obj
 0002:00008940       ?_afxPropSheetIDs@@3QBHB   5f8b3940     dlgprop.obj
 0002:00008950       ?messageMap@CPropertySheet@@1UAFX_MSGMAP@@B 5f8b3950     dlgprop.obj
 0002:00008958       ?_messageEntries@CPropertySheet@@0QBUAFX_MSGMAP_ENTRY@@B 5f8b3958     dlgprop.obj
 0002:00008a18       ?messageMap@CPropertyPage@@1UAFX_MSGMAP@@B 5f8b3a18     dlgprop.obj
 0002:00008a20       ?_messageEntries@CPropertyPage@@0QBUAFX_MSGMAP_ENTRY@@B 5f8b3a20     dlgprop.obj
 0002:00008a6c       ??_7CPropertyPage@@6B@     5f8b3a6c     dlgprop.obj
 0002:00008b64       ??_C@_1BK@BFED@?$AAC?$AAO?$AAM?$AAC?$AAT?$AAL?$AA3?$AA2?$AA?4?$AAD?$AAL?$AAL?$AA?$AA@ 5f8b3b64     dlgprop.obj
 0002:00008b80       ??_C@_1FI@LFAF@?$AAU?$AAp?$AAd?$AAa?$AAt?$AAe?$AAD?$AAa?$AAt?$AAa?$AA?5?$AAf?$AAa?$AAi?$AAl?$AAe?$AAd?$AA?5?$AAd?$AAu@ 5f8b3b80     dlgprop.obj
 0002:00008bd8       ??_C@_0BB@OCIA@m_psp?4dwFlags?5?$DN?5?$AA@ 5f8b3bd8     dlgprop.obj
 0002:00008bec       ??_C@_0BA@OFIG@m_strCaption?5?$DN?5?$AA@ 5f8b3bec     dlgprop.obj
 0002:00008c00       ??_7CPropertySheet@@6B@    5f8b3c00     dlgprop.obj
 0002:00008ccc       ??_C@_1GE@PNCH@?$AAP?$AAr?$AAo?$AAp?$AAe?$AAr?$AAt?$AAy?$AAS?$AAh?$AAe?$AAe?$AAt?$AA?$CI?$AA?$CJ?$AA?5?$AAf?$AAa?$AAi?$AAl@ 5f8b3ccc     dlgprop.obj
 0002:00008d30       ??_C@_0M@BDB@Modeless?5?$DN?5?$AA@ 5f8b3d30     dlgprop.obj
 0002:00008d3c       ??_C@_0L@PHNA@Stacked?5?$DN?5?$AA@ 5f8b3d3c     dlgprop.obj
 0002:00008d48       ??_C@_0BD@JEML@Number?5of?5Pages?5?$DN?5?$AA@ 5f8b3d48     dlgprop.obj
 0002:00008d60       ??_7CPropertyPageEx@@6B@   5f8b3d60     dlgprop.obj
 0002:00008e58       ??_C@_0BH@MOOO@m_strHeaderSubTitle?5?$DN?5?$AA@ 5f8b3e58     dlgprop.obj
 0002:00008e70       ??_C@_0BE@ICMN@m_strHeaderTitle?5?$DN?5?$AA@ 5f8b3e70     dlgprop.obj
 0002:00008e88       ??_7CPropertySheetEx@@6B@  5f8b3e88     dlgprop.obj
 0002:00008f58       ?messageMap@CCommonDialog@@1UAFX_MSGMAP@@B 5f8b3f58     dlgcomm.obj
 0002:00008f60       ?_messageEntries@CCommonDialog@@0QBUAFX_MSGMAP_ENTRY@@B 5f8b3f60     dlgcomm.obj
 0002:00008f90       ??_C@_1CI@HAOL@?$AAc?$AAo?$AAm?$AAm?$AAd?$AAl?$AAg?$AA_?$AAS?$AAe?$AAt?$AAR?$AAG?$AAB?$AAC?$AAo?$AAl?$AAo?$AAr?$AA?$AA@ 5f8b3f90     dlgcomm.obj
 0002:00008fb8       ??_C@_1BK@KCME@?$AAc?$AAo?$AAm?$AAm?$AAd?$AAl?$AAg?$AA_?$AAh?$AAe?$AAl?$AAp?$AA?$AA@ 5f8b3fb8     dlgcomm.obj
 0002:00008fd4       ??_C@_1CA@HL@?$AAc?$AAo?$AAm?$AAm?$AAd?$AAl?$AAg?$AA_?$AAC?$AAo?$AAl?$AAo?$AAr?$AAO?$AAK?$AA?$AA@ 5f8b3fd4     dlgcomm.obj
 0002:00008ff4       ??_C@_1CG@GOBL@?$AAc?$AAo?$AAm?$AAm?$AAd?$AAl?$AAg?$AA_?$AAF?$AAi?$AAl?$AAe?$AAN?$AAa?$AAm?$AAe?$AAO?$AAK?$AA?$AA@ 5f8b3ff4     dlgcomm.obj
 0002:0000901c       ??_C@_1CO@EDLA@?$AAc?$AAo?$AAm?$AAm?$AAd?$AAl?$AAg?$AA_?$AAS?$AAh?$AAa?$AAr?$AAe?$AAV?$AAi?$AAo?$AAl?$AAa?$AAt?$AAi@ 5f8b401c     dlgcomm.obj
 0002:0000904c       ??_C@_1DG@FJGG@?$AAc?$AAo?$AAm?$AAm?$AAd?$AAl?$AAg?$AA_?$AAL?$AAB?$AAS?$AAe?$AAl?$AAC?$AAh?$AAa?$AAn?$AAg?$AAe?$AAd@ 5f8b404c     dlgcomm.obj
 0002:00009088       ?classCFileDialog@CFileDialog@@2UCRuntimeClass@@B 5f8b4088     dlgfile.obj
 0002:000090a0       ??_C@_0M@JEJA@CFileDialog?$AA@ 5f8b40a0     dlgfile.obj
 0002:000090b0       ??_7CFileDialog@@6B@       5f8b40b0     dlgfile.obj
 0002:000091a4       ??_C@_0DB@BLDH@?6hook?5function?5set?5to?5non?9standa@ 5f8b41a4     dlgfile.obj
 0002:000091d8       ??_C@_0DB@MAOJ@?6hook?5function?5set?5to?5standard?5M@ 5f8b41d8     dlgfile.obj
 0002:0000920c       ??_C@_0BM@FJOE@?6m_ofn?4lpstrCustomFilter?5?$DN?5?$AA@ 5f8b420c     dlgfile.obj
 0002:00009228       ??_C@_13DOPK@?$AA?$HM?$AA?$AA@ 5f8b4228     dlgfile.obj
 0002:0000922c       ??_C@_0BG@EAND@?6m_ofn?4lpstrFilter?5?$DN?5?$AA@ 5f8b422c     dlgfile.obj
 0002:00009244       ??_C@_0BJ@OLAM@?6m_ofn?4nFileExtension?5?$DN?5?$AA@ 5f8b4244     dlgfile.obj
 0002:00009260       ??_C@_0BG@GOAA@?6m_ofn?4nFileOffset?5?$DN?5?$AA@ 5f8b4260     dlgfile.obj
 0002:00009278       ??_C@_0BG@LIO@?6m_ofn?4lpstrDefExt?5?$DN?5?$AA@ 5f8b4278     dlgfile.obj
 0002:00009290       ??_C@_0BA@MNIM@?6m_ofn?4Flags?5?$DN?5?$AA@ 5f8b4290     dlgfile.obj
 0002:000092a0       ??_C@_0BF@LLBJ@?6m_ofn?4lpstrTitle?5?$DN?5?$AA@ 5f8b42a0     dlgfile.obj
 0002:000092b8       ??_C@_0BI@FHDD@?6m_ofn?4nMaxFileTitle?5?$DN?5?$AA@ 5f8b42b8     dlgfile.obj
 0002:000092d0       ??_C@_0BJ@IPCF@?6m_ofn?4lpstrFileTitle?5?$DN?5?$AA@ 5f8b42d0     dlgfile.obj
 0002:000092ec       ??_C@_0BD@NECP@?6m_ofn?4nMaxFile?5?$DN?5?$AA@ 5f8b42ec     dlgfile.obj
 0002:00009300       ??_C@_0BE@LAEE@?6m_ofn?4lpstrFile?5?$DN?5?$AA@ 5f8b4300     dlgfile.obj
 0002:00009314       ??_C@_0BH@IOFB@?6m_ofn?4nFilterIndex?5?$DN?5?$AA@ 5f8b4314     dlgfile.obj
 0002:0000932c       ??_C@_0BE@NJGO@?6m_ofn?4hwndOwner?5?$DN?5?$AA@ 5f8b432c     dlgfile.obj
 0002:00009340       ??_C@_0BB@BCDD@File?5save?5dialog?$AA@ 5f8b4340     dlgfile.obj
 0002:00009354       ??_C@_0BB@MMDF@File?5open?5dialog?$AA@ 5f8b4354     dlgfile.obj
 0002:00009368       ?classCPageSetupDialog@CPageSetupDialog@@2UCRuntimeClass@@B 5f8b4368     dlgprnt.obj
 0002:00009380       ??_C@_0BB@KMEP@CPageSetupDialog?$AA@ 5f8b4380     dlgprnt.obj
 0002:00009398       ?classCPrintDialog@CPrintDialog@@2UCRuntimeClass@@B 5f8b4398     dlgprnt.obj
 0002:000093b0       ??_C@_0N@KDJG@CPrintDialog?$AA@ 5f8b43b0     dlgprnt.obj
 0002:000093c0       ?messageMap@CPrintDialog@@1UAFX_MSGMAP@@B 5f8b43c0     dlgprnt.obj
 0002:000093c8       ?_messageEntries@CPrintDialog@@0QBUAFX_MSGMAP_ENTRY@@B 5f8b43c8     dlgprnt.obj
 0002:000093fc       ??_7CPageSetupDialog@@6B@  5f8b43fc     dlgprnt.obj
 0002:000094dc       ??_C@_0DH@COIM@?6print?5hook?5function?5set?5to?5non?9@ 5f8b44dc     dlgprnt.obj
 0002:00009514       ??_C@_0DH@PFFC@?6print?5hook?5function?5set?5to?5stan@ 5f8b4514     dlgprnt.obj
 0002:0000954c       ??_C@_0DH@EDE@?6setup?5hook?5function?5set?5to?5non?9@ 5f8b454c     dlgprnt.obj
 0002:00009584       ??_C@_0DH@NPOK@?6setup?5hook?5function?5set?5to?5stan@ 5f8b4584     dlgprnt.obj
 0002:000095bc       ??_C@_0BG@PAAH@?6m_psd?4rtMinMargin?5?$DN?5?$AA@ 5f8b45bc     dlgprnt.obj
 0002:000095d4       ??_C@_0BG@KHLO@?6m_psd?4ptPaperSize?5?$DN?5?$AA@ 5f8b45d4     dlgprnt.obj
 0002:000095ec       ??_C@_0BA@PEDP@?6m_psd?4Flags?5?$DN?5?$AA@ 5f8b45ec     dlgprnt.obj
 0002:000095fc       ??_C@_0BD@ICJF@m_psd?4hwndOwner?5?$DN?5?$AA@ 5f8b45fc     dlgprnt.obj
 0002:00009614       ??_7CPrintDialog@@6B@      5f8b4614     dlgprnt.obj
 0002:000096f0       ??_C@_0BB@IEIJ@?6m_pd?4nCopies?5?$DN?5?$AA@ 5f8b46f0     dlgprnt.obj
 0002:00009704       ??_C@_0BC@KGBJ@?6m_pd?4nMaxPage?5?$DN?5?$AA@ 5f8b4704     dlgprnt.obj
 0002:00009718       ??_C@_0BC@IGFG@?6m_pd?4nMinPage?5?$DN?5?$AA@ 5f8b4718     dlgprnt.obj
 0002:0000972c       ??_C@_0BB@FKMB@?6m_pd?4nToPage?5?$DN?5?$AA@ 5f8b472c     dlgprnt.obj
 0002:00009740       ??_C@_0BD@CAGL@?6m_pd?4nFromPage?5?$DN?5?$AA@ 5f8b4740     dlgprnt.obj
 0002:00009754       ??_C@_0P@GOAF@?6m_pd?4Flags?5?$DN?5?$AA@ 5f8b4754     dlgprnt.obj
 0002:00009764       ??_C@_0N@IKKN@?6m_pd?4hDC?5?$DN?5?$AA@ 5f8b4764     dlgprnt.obj
 0002:00009774       ??_C@_0BC@BGBH@m_pd?4hwndOwner?5?$DN?5?$AA@ 5f8b4774     dlgprnt.obj
 0002:00009788       ?classCColorDialog@CColorDialog@@2UCRuntimeClass@@B 5f8b4788     dlgclr.obj
 0002:000097a0       ??_C@_0N@GCDM@CColorDialog?$AA@ 5f8b47a0     dlgclr.obj
 0002:000097b0       ?messageMap@CColorDialog@@1UAFX_MSGMAP@@B 5f8b47b0     dlgclr.obj
 0002:000097b8       ?_messageEntries@CColorDialog@@0QBUAFX_MSGMAP_ENTRY@@B 5f8b47b8     dlgclr.obj
 0002:000097ec       ??_7_AFX_COLOR_STATE@@6B@  5f8b47ec     dlgclr.obj
 0002:000097f4       ??_7CColorDialog@@6B@      5f8b47f4     dlgclr.obj
 0002:000098d0       ??_C@_0BE@OCAE@?6m_cc?4lpCustColors?5?$AA@ 5f8b48d0     dlgclr.obj
 0002:000098e4       ??_C@_0P@FGCG@?6m_cc?4Flags?5?$DN?5?$AA@ 5f8b48e4     dlgclr.obj
 0002:000098f4       ??_C@_0BD@KEFJ@?6m_cc?4rgbResult?5?$DN?5?$AA@ 5f8b48f4     dlgclr.obj
 0002:00009908       ??_C@_0BC@BKEE@m_cc?4hwndOwner?5?$DN?5?$AA@ 5f8b4908     dlgclr.obj
 0002:00009920       ?classCFontDialog@CFontDialog@@2UCRuntimeClass@@B 5f8b4920     dlgfnt.obj
 0002:00009938       ??_C@_0M@EOLC@CFontDialog?$AA@ 5f8b4938     dlgfnt.obj
 0002:00009948       ??_7CFontDialog@@6B@       5f8b4948     dlgfnt.obj
 0002:00009a20       ??_C@_0BD@DOM@?6m_cf?4rgbColors?5?$DN?5?$AA@ 5f8b4a20     dlgfnt.obj
 0002:00009a34       ??_C@_0BD@FJNA@?6m_cf?4nFontType?5?$DN?5?$AA@ 5f8b4a34     dlgfnt.obj
 0002:00009a48       ??_C@_0BC@COFM@?6m_cf?4nSizeMax?5?$DN?5?$AA@ 5f8b4a48     dlgfnt.obj
 0002:00009a5c       ??_C@_0BC@KFLL@?6m_cf?4nSizeMin?5?$DN?5?$AA@ 5f8b4a5c     dlgfnt.obj
 0002:00009a70       ??_C@_0BD@DIPJ@?6m_cf?4lpszStyle?5?$DN?5?$AA@ 5f8b4a70     dlgfnt.obj
 0002:00009a84       ??_C@_0P@OGON@?6m_cf?4Flags?5?$DN?5?$AA@ 5f8b4a84     dlgfnt.obj
 0002:00009a94       ??_C@_0BE@DCEE@?6m_cf?4iPointSize?5?$DN?5?$AA@ 5f8b4a94     dlgfnt.obj
 0002:00009aa8       ??_C@_0N@HIKK@?6m_cf?4hDC?5?$DN?5?$AA@ 5f8b4aa8     dlgfnt.obj
 0002:00009ab8       ??_C@_0BC@DLFA@m_cf?4hwndOwner?5?$DN?5?$AA@ 5f8b4ab8     dlgfnt.obj
 0002:00009ad0       ?classCFindReplaceDialog@CFindReplaceDialog@@2UCRuntimeClass@@B 5f8b4ad0     dlgfr.obj
 0002:00009ae8       ??_C@_0BD@HPIP@CFindReplaceDialog?$AA@ 5f8b4ae8     dlgfr.obj
 0002:00009b00       ??_7CFindReplaceDialog@@6B@ 5f8b4b00     dlgfr.obj
 0002:00009bd8       ??_C@_0BK@NHOK@?6m_fr?4lpstrReplaceWith?5?$DN?5?$AA@ 5f8b4bd8     dlgfr.obj
 0002:00009bf4       ??_C@_0BH@KCOO@?6m_fr?4lpstrFindWhat?5?$DN?5?$AA@ 5f8b4bf4     dlgfr.obj
 0002:00009c0c       ??_C@_0P@GFHA@?6m_fr?4Flags?5?$DN?5?$AA@ 5f8b4c0c     dlgfr.obj
 0002:00009c1c       ??_C@_0BC@HHCC@m_fr?4hwndOwner?5?$DN?5?$AA@ 5f8b4c1c     dlgfr.obj
 0002:00009c30       ??_C@_0L@CKOP@ccdata?4cpp?$AA@ 5f8b4c30     ccdata.obj
 0002:00009c40       ??_7_AFX_PROPPAGEFONTINFO@@6B@ 5f8b4c40     ccdata.obj
 0002:00009c44       ??_C@_1GK@FNIL@?$AAA?$AAB?$AAC?$AAD?$AAE?$AAF?$AAG?$AAH?$AAI?$AAJ?$AAK?$AAL?$AAM?$AAN?$AAO?$AAP?$AAQ?$AAR?$AAS?$AAT@ 5f8b4c44     dlgtempl.obj
 0002:00009cb0       ??_C@_1O@KHFL@?$AAS?$AAy?$AAs?$AAt?$AAe?$AAm?$AA?$AA@ 5f8b4cb0     dlgtempl.obj
 0002:00009cc0       ?classCReBarCtrl@CReBarCtrl@@2UCRuntimeClass@@B 5f8b4cc0     winctrl6.obj
 0002:00009cd8       ??_C@_0L@GONC@CReBarCtrl?$AA@ 5f8b4cd8     winctrl6.obj
 0002:00009ce8       ?classCIPAddressCtrl@CIPAddressCtrl@@2UCRuntimeClass@@B 5f8b4ce8     winctrl6.obj
 0002:00009d00       ??_C@_0P@PBFM@CIPAddressCtrl?$AA@ 5f8b4d00     winctrl6.obj
 0002:00009d20       ??_7CIPAddressCtrl@@6B@    5f8b4d20     winctrl6.obj
 0002:00009de0       ??_C@_1BO@OJBJ@?$AAS?$AAy?$AAs?$AAI?$AAP?$AAA?$AAd?$AAd?$AAr?$AAe?$AAs?$AAs?$AA3?$AA2?$AA?$AA@ 5f8b4de0     winctrl6.obj
 0002:00009e00       ??_C@_0N@DEPF@winctrl6?4cpp?$AA@ 5f8b4e00     winctrl6.obj
 0002:00009e10       ??_C@_1BK@JEIN@?$AAC?$AAo?$AAm?$AAb?$AAo?$AAB?$AAo?$AAx?$AAE?$AAx?$AA3?$AA2?$AA?$AA@ 5f8b4e10     winctrl6.obj
 0002:00009e30       ??_7CComboBoxEx@@6B@       5f8b4e30     winctrl6.obj
 0002:00009f04       ??_7CReBarCtrl@@6B@        5f8b4f04     winctrl6.obj
 0002:00009fc8       ?classCTempGdiObject@CTempGdiObject@@2UCRuntimeClass@@B 5f8b4fc8     wingdi.obj
 0002:00009fe0       ??_C@_0P@LOPC@CTempGdiObject?$AA@ 5f8b4fe0     wingdi.obj
 0002:00009ff0       ?classCTempDC@CTempDC@@2UCRuntimeClass@@B 5f8b4ff0     wingdi.obj
 0002:0000a008       ??_C@_07LHDN@CTempDC?$AA@  5f8b5008     wingdi.obj
 0002:0000a010       ?classCRgn@CRgn@@2UCRuntimeClass@@B 5f8b5010     wingdi.obj
 0002:0000a028       ??_C@_04HJNG@CRgn?$AA@     5f8b5028     wingdi.obj
 0002:0000a030       ?classCPalette@CPalette@@2UCRuntimeClass@@B 5f8b5030     wingdi.obj
 0002:0000a048       ??_C@_08CIF@CPalette?$AA@  5f8b5048     wingdi.obj
 0002:0000a058       ?classCBitmap@CBitmap@@2UCRuntimeClass@@B 5f8b5058     wingdi.obj
 0002:0000a070       ??_C@_07HNEL@CBitmap?$AA@  5f8b5070     wingdi.obj
 0002:0000a078       ?classCFont@CFont@@2UCRuntimeClass@@B 5f8b5078     wingdi.obj
 0002:0000a090       ??_C@_05MCKJ@CFont?$AA@    5f8b5090     wingdi.obj
 0002:0000a098       ?classCBrush@CBrush@@2UCRuntimeClass@@B 5f8b5098     wingdi.obj
 0002:0000a0b0       ??_C@_06PNF@CBrush?$AA@    5f8b50b0     wingdi.obj
 0002:0000a0b8       ?classCPen@CPen@@2UCRuntimeClass@@B 5f8b50b8     wingdi.obj
 0002:0000a0d0       ??_C@_04PAKO@CPen?$AA@     5f8b50d0     wingdi.obj
 0002:0000a0d8       ?classCGdiObject@CGdiObject@@2UCRuntimeClass@@B 5f8b50d8     wingdi.obj
 0002:0000a0f0       ??_C@_0L@CNBG@CGdiObject?$AA@ 5f8b50f0     wingdi.obj
 0002:0000a100       ?classCPaintDC@CPaintDC@@2UCRuntimeClass@@B 5f8b5100     wingdi.obj
 0002:0000a118       ??_C@_08HFDK@CPaintDC?$AA@ 5f8b5118     wingdi.obj
 0002:0000a128       ?classCWindowDC@CWindowDC@@2UCRuntimeClass@@B 5f8b5128     wingdi.obj
 0002:0000a140       ??_C@_09NFPO@CWindowDC?$AA@ 5f8b5140     wingdi.obj
 0002:0000a150       ?classCClientDC@CClientDC@@2UCRuntimeClass@@B 5f8b5150     wingdi.obj
 0002:0000a168       ??_C@_09HIEC@CClientDC?$AA@ 5f8b5168     wingdi.obj
 0002:0000a178       ?classCDC@CDC@@2UCRuntimeClass@@B 5f8b5178     wingdi.obj
 0002:0000a190       ??_C@_03NJOH@CDC?$AA@      5f8b5190     wingdi.obj
 0002:0000a198       ?classCUserException@CUserException@@2UCRuntimeClass@@B 5f8b5198     wingdi.obj
 0002:0000a1b0       ??_C@_0P@BHHD@CUserException?$AA@ 5f8b51b0     wingdi.obj
 0002:0000a1c0       ?classCResourceException@CResourceException@@2UCRuntimeClass@@B 5f8b51c0     wingdi.obj
 0002:0000a1d8       ??_C@_0BD@GMHI@CResourceException?$AA@ 5f8b51d8     wingdi.obj
 0002:0000a1ec       ??_C@_01GFI@?$CI?$AA@      5f8b51ec     wingdi.obj
 0002:0000a1f0       ??_C@_03LADP@?5x?5?$AA@    5f8b51f0     wingdi.obj
 0002:0000a1f4       ??_C@_02GIEM@?0?5?$AA@     5f8b51f4     wingdi.obj
 0002:0000a1f8       ??_C@_03MFNL@?$CIL?5?$AA@  5f8b51f8     wingdi.obj
 0002:0000a1fc       ??_C@_04JPAJ@?0?5T?5?$AA@  5f8b51fc     wingdi.obj
 0002:0000a204       ??_C@_04OIPG@?0?5R?5?$AA@  5f8b5204     wingdi.obj
 0002:0000a20c       ??_C@_04ICFP@?0?5B?5?$AA@  5f8b520c     wingdi.obj
 0002:0000a218       ??_7CDC@@6B@               5f8b5218     wingdi.obj
 0002:0000a294       ??_C@_0BA@ILEG@?6m_bPrinting?5?$DN?5?$AA@ 5f8b5294     wingdi.obj
 0002:0000a2a4       ??_C@_0BA@CDKA@?6m_hAttribDC?5?$DN?5?$AA@ 5f8b52a4     wingdi.obj
 0002:0000a2b4       ??_C@_08EDME@m_hDC?5?$DN?5?$AA@ 5f8b52b4     wingdi.obj
 0002:0000a2c0       ??_C@_1FA@OKCP@?$AAC?$AAa?$AAn?$AAn?$AAo?$AAt?$AA?5?$AAS?$AAe?$AAt?$AA?5?$AAO?$AAu?$AAt?$AAp?$AAu?$AAt?$AA?5?$AAh?$AAD@ 5f8b52c0     wingdi.obj
 0002:0000a310       ??_C@_1FI@NHOF@?$AAC?$AAa?$AAn?$AAn?$AAo?$AAt?$AA?5?$AAR?$AAe?$AAl?$AAe?$AAa?$AAs?$AAe?$AA?5?$AAO?$AAu?$AAt?$AAp?$AAu@ 5f8b5310     wingdi.obj
 0002:0000a368       ??_C@_09EBEO@GetLayout?$AA@ 5f8b5368     wingdi.obj
 0002:0000a374       ??_C@_09JDFO@GDI32?4DLL?$AA@ 5f8b5374     wingdi.obj
 0002:0000a380       ??_C@_09GMOM@SetLayout?$AA@ 5f8b5380     wingdi.obj
 0002:0000a38c       ??_C@_1HO@CIMJ@?$AAE?$AAr?$AAr?$AAo?$AAr?$AA?3?$AA?5?$AAu?$AAn?$AAa?$AAb?$AAl?$AAe?$AA?5?$AAt?$AAo?$AA?5?$AAt?$AAr?$AAa@ 5f8b538c     wingdi.obj
 0002:0000a40c       ??_C@_09BKNC@m_hWnd?5?$DN?5?$AA@ 5f8b540c     wingdi.obj
 0002:0000a41c       ??_7CClientDC@@6B@         5f8b541c     wingdi.obj
 0002:0000a49c       ??_7CWindowDC@@6B@         5f8b549c     wingdi.obj
 0002:0000a518       ??_C@_0BB@ENDM@?6m_ps?4rcPaint?5?$DN?5?$AA@ 5f8b5518     wingdi.obj
 0002:0000a52c       ??_C@_0BA@EPIF@?6m_ps?4fErase?5?$DN?5?$AA@ 5f8b552c     wingdi.obj
 0002:0000a53c       ??_C@_0N@FOGF@?6m_ps?4hdc?5?$DN?5?$AA@ 5f8b553c     wingdi.obj
 0002:0000a550       ??_7CPaintDC@@6B@          5f8b5550     wingdi.obj
 0002:0000a5cc       ??_C@_0N@FLLI@m_hObject?5?$DN?5?$AA@ 5f8b55cc     wingdi.obj
 0002:0000a5dc       ??_C@_0BD@OHGG@?6lgpn?4lopnColor?5?$DN?5?$AA@ 5f8b55dc     wingdi.obj
 0002:0000a5f0       ??_C@_0BN@MJJM@?6lgpn?4lopnWidth?4x?5?$CIwidth?$CJ?5?$DN?5?$AA@ 5f8b55f0     wingdi.obj
 0002:0000a610       ??_C@_0BC@NJFN@lgpn?4lopnStyle?5?$DN?5?$AA@ 5f8b5610     wingdi.obj
 0002:0000a624       ??_C@_0BC@KGMJ@has?5ILLEGAL?5HPEN?$CB?$AA@ 5f8b5624     wingdi.obj
 0002:0000a638       ??_C@_0P@GPNM@?6lb?4lbColor?5?$DN?5?$AA@ 5f8b5638     wingdi.obj
 0002:0000a648       ??_C@_0P@CGKC@?6lb?4lbHatch?5?$DN?5?$AA@ 5f8b5648     wingdi.obj
 0002:0000a658       ??_C@_0O@JHIH@lb?4lbStyle?5?$DN?5?$AA@ 5f8b5658     wingdi.obj
 0002:0000a668       ??_C@_0BE@EOKH@has?5ILLEGAL?5HBRUSH?$CB?$AA@ 5f8b5668     wingdi.obj
 0002:0000a67c       ??_C@_0BC@MKGI@?6lf?4lfFaceName?5?$DN?5?$AA@ 5f8b567c     wingdi.obj
 0002:0000a690       ??_C@_0BI@KPDF@?6lf?4lfPitchAndFamily?5?$DN?5?$AA@ 5f8b5690     wingdi.obj
 0002:0000a6a8       ??_C@_0BB@HDME@?6lf?4lfQuality?5?$DN?5?$AA@ 5f8b56a8     wingdi.obj
 0002:0000a6bc       ??_C@_0BH@BHDK@?6lf?4lfClipPrecision?5?$DN?5?$AA@ 5f8b56bc     wingdi.obj
 0002:0000a6d4       ??_C@_0BG@LDPK@?6lf?4lfOutPrecision?5?$DN?5?$AA@ 5f8b56d4     wingdi.obj
 0002:0000a6ec       ??_C@_0BB@EHPI@?6lf?4lfCharSet?5?$DN?5?$AA@ 5f8b56ec     wingdi.obj
 0002:0000a700       ??_C@_0BD@CLIK@?6lf?4lfStrikeOut?5?$DN?5?$AA@ 5f8b5700     wingdi.obj
 0002:0000a714       ??_C@_0BD@CCIM@?6lf?4lfUnderline?5?$DN?5?$AA@ 5f8b5714     wingdi.obj
 0002:0000a728       ??_C@_0BA@PNIN@?6lf?4lfItalic?5?$DN?5?$AA@ 5f8b5728     wingdi.obj
 0002:0000a738       ??_C@_0BA@OEMP@?6lf?4lfWeight?5?$DN?5?$AA@ 5f8b5738     wingdi.obj
 0002:0000a748       ??_C@_0BF@BCNP@?6lf?4lfOrientation?5?$DN?5?$AA@ 5f8b5748     wingdi.obj
 0002:0000a760       ??_C@_0BE@FCLM@?6lf?4lfEscapement?5?$DN?5?$AA@ 5f8b5760     wingdi.obj
 0002:0000a774       ??_C@_0P@OPHM@?6lf?4lfWidth?5?$DN?5?$AA@ 5f8b5774     wingdi.obj
 0002:0000a784       ??_C@_0P@NLG@lf?4lfHeight?5?$DN?5?$AA@ 5f8b5784     wingdi.obj
 0002:0000a794       ??_C@_0BD@LADB@has?5ILLEGAL?5HFONT?$CB?$AA@ 5f8b5794     wingdi.obj
 0002:0000a7a8       ??_C@_0BD@FDEM@?6bm?4bmBitsPixel?5?$DN?5?$AA@ 5f8b57a8     wingdi.obj
 0002:0000a7bc       ??_C@_0BA@ELPK@?6bm?4bmPlanes?5?$DN?5?$AA@ 5f8b57bc     wingdi.obj
 0002:0000a7cc       ??_C@_0BE@PBD@?6bm?4bmWidthBytes?5?$DN?5?$AA@ 5f8b57cc     wingdi.obj
 0002:0000a7e0       ??_C@_0P@FABC@?6bm?4bmWidth?5?$DN?5?$AA@ 5f8b57e0     wingdi.obj
 0002:0000a7f0       ??_C@_0BA@ODEL@?6bm?4bmHeight?5?$DN?5?$AA@ 5f8b57f0     wingdi.obj
 0002:0000a800       ??_C@_0N@HLBI@bm?4bmType?5?$DN?5?$AA@ 5f8b5800     wingdi.obj
 0002:0000a810       ??_C@_0BF@LCPF@has?5ILLEGAL?5HBITMAP?$CB?$AA@ 5f8b5810     wingdi.obj
 0002:0000a82c       ??_7CTempDC@@6B@           5f8b582c     wingdi.obj
 0002:0000a8ac       ??_7CTempGdiObject@@6B@    5f8b58ac     wingdi.obj
 0002:0000a8c0       ?classCTempMenu@CTempMenu@@2UCRuntimeClass@@B 5f8b58c0     winmenu.obj
 0002:0000a8d8       ??_C@_09NDEG@CTempMenu?$AA@ 5f8b58d8     winmenu.obj
 0002:0000a8e8       ?classCMenu@CMenu@@2UCRuntimeClass@@B 5f8b58e8     winmenu.obj
 0002:0000a900       ??_C@_05BJMA@CMenu?$AA@    5f8b5900     winmenu.obj
 0002:0000a908       ??_C@_0L@LJHH@m_hMenu?5?$DN?5?$AA@ 5f8b5908     winmenu.obj
 0002:0000a918       ??_7CTempMenu@@6B@         5f8b5918     winmenu.obj
 0002:0000aee0       ??_C@_0BA@BCKA@WM_DEVICECHANGE?$AA@ 5f8b5ee0     afxtrace.obj
 0002:0000aef0       ??_C@_0BC@FLPI@WM_CAPTURECHANGED?$AA@ 5f8b5ef0     afxtrace.obj
 0002:0000af04       ??_C@_0L@JPGD@WM_SETICON?$AA@ 5f8b5f04     afxtrace.obj
 0002:0000af10       ??_C@_0BB@DEEK@WM_DISPLAYCHANGE?$AA@ 5f8b5f10     afxtrace.obj
 0002:0000af24       ??_C@_0BB@NJHD@WM_ENTERMENULOOP?$AA@ 5f8b5f24     afxtrace.obj
 0002:0000af38       ??_C@_0BA@HLKE@WM_EXITMENULOOP?$AA@ 5f8b5f38     afxtrace.obj
 0002:0000af48       ??_C@_0L@MMGP@WM_GETICON?$AA@ 5f8b5f48     afxtrace.obj
 0002:0000af54       ??_C@_09OEDN@WM_HOTKEY?$AA@ 5f8b5f54     afxtrace.obj
 0002:0000af60       ??_C@_0BC@HECE@WM_POWERBROADCAST?$AA@ 5f8b5f60     afxtrace.obj
 0002:0000af74       ??_C@_0P@HMNB@WM_PRINTCLIENT?$AA@ 5f8b5f74     afxtrace.obj
 0002:0000af84       ??_C@_08IKAD@WM_PRINT?$AA@ 5f8b5f84     afxtrace.obj
 0002:0000af90       ??_C@_0N@GEDB@WM_SETHOTKEY?$AA@ 5f8b5f90     afxtrace.obj
 0002:0000afa0       ??_C@_09LAEB@WM_SIZING?$AA@ 5f8b5fa0     afxtrace.obj
 0002:0000afac       ??_C@_0BB@DICO@WM_STYLECHANGING?$AA@ 5f8b5fac     afxtrace.obj
 0002:0000afc0       ??_C@_0BA@OFOA@WM_STYLECHANGED?$AA@ 5f8b5fc0     afxtrace.obj
 0002:0000afd0       ??_C@_09EFIF@WM_MOVING?$AA@ 5f8b5fd0     afxtrace.obj
 0002:0000afdc       ??_C@_0BC@MNNI@WM_MDIREFRESHMENU?$AA@ 5f8b5fdc     afxtrace.obj
 0002:0000aff0       ??_C@_08MGHH@WM_TCARD?$AA@ 5f8b5ff0     afxtrace.obj
 0002:0000affc       ??_C@_0P@HHPE@WM_CONTEXTMENU?$AA@ 5f8b5ffc     afxtrace.obj
 0002:0000b00c       ??_C@_09GCP@WM_NOTIFY?$AA@ 5f8b600c     afxtrace.obj
 0002:0000b018       ??_C@_07EBDL@WM_HELP?$AA@  5f8b6018     afxtrace.obj
 0002:0000b020       ??_C@_0BA@BKIC@WM_EXITHELPMODE?$AA@ 5f8b6020     afxtrace.obj
 0002:0000b030       ??_C@_0P@JFOD@WM_HELPHITTEST?$AA@ 5f8b6030     afxtrace.obj
 0002:0000b040       ??_C@_0P@LINK@WM_COMMANDHELP?$AA@ 5f8b6040     afxtrace.obj
 0002:0000b050       ??_C@_0BB@OBCK@WM_INITIALUPDATE?$AA@ 5f8b6050     afxtrace.obj
 0002:0000b064       ??_C@_0BD@GBKN@WM_IDLEUPDATECMDUI?$AA@ 5f8b6064     afxtrace.obj
 0002:0000b078       ??_C@_0BE@BKCA@WM_SETMESSAGESTRING?$AA@ 5f8b6078     afxtrace.obj
 0002:0000b08c       ??_C@_0O@MIIN@WM_SIZEPARENT?$AA@ 5f8b608c     afxtrace.obj
 0002:0000b09c       ??_C@_0BF@LNAM@WM_WINDOWPOSCHANGING?$AA@ 5f8b609c     afxtrace.obj
 0002:0000b0b4       ??_C@_0BE@MHJM@WM_WINDOWPOSCHANGED?$AA@ 5f8b60b4     afxtrace.obj
 0002:0000b0c8       ??_C@_08GJNJ@WM_POWER?$AA@ 5f8b60c8     afxtrace.obj
 0002:0000b0d4       ??_C@_0N@LNHC@WM_DROPFILES?$AA@ 5f8b60d4     afxtrace.obj
 0002:0000b0e4       ??_C@_0P@OMCP@WM_DDE_EXECUTE?$AA@ 5f8b60e4     afxtrace.obj
 0002:0000b0f4       ??_C@_0M@JFNO@WM_DDE_POKE?$AA@ 5f8b60f4     afxtrace.obj
 0002:0000b100       ??_C@_0P@LDGL@WM_DDE_REQUEST?$AA@ 5f8b6100     afxtrace.obj
 0002:0000b110       ??_C@_0M@DNIB@WM_DDE_DATA?$AA@ 5f8b6110     afxtrace.obj
 0002:0000b11c       ??_C@_0L@EJNE@WM_DDE_ACK?$AA@ 5f8b611c     afxtrace.obj
 0002:0000b128       ??_C@_0BA@IDGA@WM_DDE_UNADVISE?$AA@ 5f8b6128     afxtrace.obj
 0002:0000b138       ??_C@_0O@ILOI@WM_DDE_ADVISE?$AA@ 5f8b6138     afxtrace.obj
 0002:0000b148       ??_C@_0BB@EJPN@WM_DDE_TERMINATE?$AA@ 5f8b6148     afxtrace.obj
 0002:0000b15c       ??_C@_0BA@LLPM@WM_DDE_INITIATE?$AA@ 5f8b615c     afxtrace.obj
 0002:0000b16c       ??_C@_0BC@PIEK@WM_PALETTECHANGED?$AA@ 5f8b616c     afxtrace.obj
 0002:0000b180       ??_C@_0BF@EKBE@WM_PALETTEISCHANGING?$AA@ 5f8b6180     afxtrace.obj
 0002:0000b198       ??_C@_0BD@DMNM@WM_QUERYNEWPALETTE?$AA@ 5f8b6198     afxtrace.obj
 0002:0000b1ac       ??_C@_0BE@PKKP@WM_HSCROLLCLIPBOARD?$AA@ 5f8b61ac     afxtrace.obj
 0002:0000b1c0       ??_C@_0BB@LIFP@WM_CHANGECBCHAIN?$AA@ 5f8b61c0     afxtrace.obj
 0002:0000b1d4       ??_C@_0BD@PGGG@WM_ASKCBFORMATNAME?$AA@ 5f8b61d4     afxtrace.obj
 0002:0000b1e8       ??_C@_0BB@JJM@WM_SIZECLIPBOARD?$AA@ 5f8b61e8     afxtrace.obj
 0002:0000b1fc       ??_C@_0BE@CMBP@WM_VSCROLLCLIPBOARD?$AA@ 5f8b61fc     afxtrace.obj
 0002:0000b210       ??_C@_0BC@NHPH@WM_PAINTCLIPBOARD?$AA@ 5f8b6210     afxtrace.obj
 0002:0000b224       ??_C@_0BB@IODC@WM_DRAWCLIPBOARD?$AA@ 5f8b6224     afxtrace.obj
 0002:0000b238       ??_C@_0BE@CMMN@WM_DESTROYCLIPBOARD?$AA@ 5f8b6238     afxtrace.obj
 0002:0000b24c       ??_C@_0BE@BJAC@WM_RENDERALLFORMATS?$AA@ 5f8b624c     afxtrace.obj
 0002:0000b260       ??_C@_0BA@HABD@WM_RENDERFORMAT?$AA@ 5f8b6260     afxtrace.obj
 0002:0000b270       ??_C@_07PFGH@WM_UNDO?$AA@  5f8b6270     afxtrace.obj
 0002:0000b278       ??_C@_08DLPI@WM_CLEAR?$AA@ 5f8b6278     afxtrace.obj
 0002:0000b284       ??_C@_08FEGJ@WM_PASTE?$AA@ 5f8b6284     afxtrace.obj
 0002:0000b290       ??_C@_07ELLN@WM_COPY?$AA@  5f8b6290     afxtrace.obj
 0002:0000b298       ??_C@_0M@JLKG@WM_COPYDATA?$AA@ 5f8b6298     afxtrace.obj
 0002:0000b2a4       ??_C@_06HKFO@WM_CUT?$AA@   5f8b62a4     afxtrace.obj
 0002:0000b2ac       ??_C@_0O@HDPN@WM_MDISETMENU?$AA@ 5f8b62ac     afxtrace.obj
 0002:0000b2bc       ??_C@_0BA@NCGN@WM_MDIGETACTIVE?$AA@ 5f8b62bc     afxtrace.obj
 0002:0000b2cc       ??_C@_0BC@KCHC@WM_MDIICONARRANGE?$AA@ 5f8b62cc     afxtrace.obj
 0002:0000b2e0       ??_C@_0O@CAIK@WM_MDICASCADE?$AA@ 5f8b62e0     afxtrace.obj
 0002:0000b2f0       ??_C@_0L@DIEL@WM_MDITILE?$AA@ 5f8b62f0     afxtrace.obj
 0002:0000b2fc       ??_C@_0P@KOLA@WM_MDIMAXIMIZE?$AA@ 5f8b62fc     afxtrace.obj
 0002:0000b30c       ??_C@_0L@OGFF@WM_MDINEXT?$AA@ 5f8b630c     afxtrace.obj
 0002:0000b318       ??_C@_0O@HPMO@WM_MDIRESTORE?$AA@ 5f8b6318     afxtrace.obj
 0002:0000b328       ??_C@_0P@CLIN@WM_MDIACTIVATE?$AA@ 5f8b6328     afxtrace.obj
 0002:0000b338       ??_C@_0O@BOBD@WM_MDIDESTROY?$AA@ 5f8b6338     afxtrace.obj
 0002:0000b348       ??_C@_0N@MBAK@WM_MDICREATE?$AA@ 5f8b6348     afxtrace.obj
 0002:0000b358       ??_C@_0BA@PGF@WM_PARENTNOTIFY?$AA@ 5f8b6358     afxtrace.obj
 0002:0000b368       ??_C@_0BB@MPK@WM_MBUTTONDBLCLK?$AA@ 5f8b6368     afxtrace.obj
 0002:0000b37c       ??_C@_0N@NFAA@WM_MBUTTONUP?$AA@ 5f8b637c     afxtrace.obj
 0002:0000b38c       ??_C@_0P@CEIM@WM_MBUTTONDOWN?$AA@ 5f8b638c     afxtrace.obj
 0002:0000b39c       ??_C@_0BB@CHEK@WM_RBUTTONDBLCLK?$AA@ 5f8b639c     afxtrace.obj
 0002:0000b3b0       ??_C@_0N@KMDL@WM_RBUTTONUP?$AA@ 5f8b63b0     afxtrace.obj
 0002:0000b3c0       ??_C@_0P@ENKB@WM_RBUTTONDOWN?$AA@ 5f8b63c0     afxtrace.obj
 0002:0000b3d0       ??_C@_0BB@FNJH@WM_LBUTTONDBLCLK?$AA@ 5f8b63d0     afxtrace.obj
 0002:0000b3e4       ??_C@_0N@BHEI@WM_LBUTTONUP?$AA@ 5f8b63e4     afxtrace.obj
 0002:0000b3f4       ??_C@_0P@MOAD@WM_LBUTTONDOWN?$AA@ 5f8b63f4     afxtrace.obj
 0002:0000b404       ??_C@_0N@DMAG@WM_MOUSEMOVE?$AA@ 5f8b6404     afxtrace.obj
 0002:0000b414       ??_C@_0O@ENMC@WM_MOUSEWHEEL?$AA@ 5f8b6414     afxtrace.obj
 0002:0000b424       ??_C@_0N@MPP@WM_ENTERIDLE?$AA@ 5f8b6424     afxtrace.obj
 0002:0000b434       ??_C@_0M@LC@WM_MENUCHAR?$AA@ 5f8b6434     afxtrace.obj
 0002:0000b440       ??_C@_0O@FNCC@WM_MENUSELECT?$AA@ 5f8b6440     afxtrace.obj
 0002:0000b450       ??_C@_0BB@BMJA@WM_INITMENUPOPUP?$AA@ 5f8b6450     afxtrace.obj
 0002:0000b464       ??_C@_0M@JBDP@WM_INITMENU?$AA@ 5f8b6464     afxtrace.obj
 0002:0000b470       ??_C@_0L@OILE@WM_VSCROLL?$AA@ 5f8b6470     afxtrace.obj
 0002:0000b47c       ??_C@_0L@JCDO@WM_HSCROLL?$AA@ 5f8b647c     afxtrace.obj
 0002:0000b488       ??_C@_08CDFC@WM_TIMER?$AA@ 5f8b6488     afxtrace.obj
 0002:0000b494       ??_C@_0O@PINB@WM_SYSCOMMAND?$AA@ 5f8b6494     afxtrace.obj
 0002:0000b4a4       ??_C@_0L@HFHL@WM_COMMAND?$AA@ 5f8b64a4     afxtrace.obj
 0002:0000b4b0       ??_C@_0O@DCCN@WM_INITDIALOG?$AA@ 5f8b64b0     afxtrace.obj
 0002:0000b4c0       ??_C@_0L@BKII@WM_KEYLAST?$AA@ 5f8b64c0     afxtrace.obj
 0002:0000b4cc       ??_C@_0P@OCHE@WM_SYSDEADCHAR?$AA@ 5f8b64cc     afxtrace.obj
 0002:0000b4dc       ??_C@_0L@MNJP@WM_SYSCHAR?$AA@ 5f8b64dc     afxtrace.obj
 0002:0000b4e8       ??_C@_0M@GKFH@WM_SYSKEYUP?$AA@ 5f8b64e8     afxtrace.obj
 0002:0000b4f4       ??_C@_0O@DDDM@WM_SYSKEYDOWN?$AA@ 5f8b64f4     afxtrace.obj
 0002:0000b504       ??_C@_0M@OOPJ@WM_DEADCHAR?$AA@ 5f8b6504     afxtrace.obj
 0002:0000b510       ??_C@_07CCNO@WM_CHAR?$AA@  5f8b6510     afxtrace.obj
 0002:0000b518       ??_C@_08KJLI@WM_KEYUP?$AA@ 5f8b6518     afxtrace.obj
 0002:0000b524       ??_C@_0L@LOJG@WM_KEYDOWN?$AA@ 5f8b6524     afxtrace.obj
 0002:0000b530       ??_C@_0BD@FIJ@WM_NCMBUTTONDBLCLK?$AA@ 5f8b6530     afxtrace.obj
 0002:0000b544       ??_C@_0P@IMMP@WM_NCMBUTTONUP?$AA@ 5f8b6544     afxtrace.obj
 0002:0000b554       ??_C@_0BB@CPBP@WM_NCMBUTTONDOWN?$AA@ 5f8b6554     afxtrace.obj
 0002:0000b568       ??_C@_0BD@CODJ@WM_NCRBUTTONDBLCLK?$AA@ 5f8b6568     afxtrace.obj
 0002:0000b57c       ??_C@_0P@PFPE@WM_NCRBUTTONUP?$AA@ 5f8b657c     afxtrace.obj
 0002:0000b58c       ??_C@_0BB@EGDC@WM_NCRBUTTONDOWN?$AA@ 5f8b658c     afxtrace.obj
 0002:0000b5a0       ??_C@_0BD@FEOE@WM_NCLBUTTONDBLCLK?$AA@ 5f8b65a0     afxtrace.obj
 0002:0000b5b4       ??_C@_0P@EOIH@WM_NCLBUTTONUP?$AA@ 5f8b65b4     afxtrace.obj
 0002:0000b5c4       ??_C@_0BB@MFJA@WM_NCLBUTTONDOWN?$AA@ 5f8b65c4     afxtrace.obj
 0002:0000b5d8       ??_C@_0P@GFMJ@WM_NCMOUSEMOVE?$AA@ 5f8b65d8     afxtrace.obj
 0002:0000b5e8       ??_C@_0O@HBJG@WM_GETDLGCODE?$AA@ 5f8b65e8     afxtrace.obj
 0002:0000b5f8       ??_C@_0O@OLMF@WM_NCACTIVATE?$AA@ 5f8b65f8     afxtrace.obj
 0002:0000b608       ??_C@_0L@MLEG@WM_NCPAINT?$AA@ 5f8b6608     afxtrace.obj
 0002:0000b614       ??_C@_0N@ENIL@WM_NCHITTEST?$AA@ 5f8b6614     afxtrace.obj
 0002:0000b624       ??_C@_0O@HCNE@WM_NCCALCSIZE?$AA@ 5f8b6624     afxtrace.obj
 0002:0000b634       ??_C@_0N@FGCE@WM_NCDESTROY?$AA@ 5f8b6634     afxtrace.obj
 0002:0000b644       ??_C@_0M@PGBE@WM_NCCREATE?$AA@ 5f8b6644     afxtrace.obj
 0002:0000b650       ??_C@_0O@GAIC@WM_COMPACTING?$AA@ 5f8b6650     afxtrace.obj
 0002:0000b660       ??_C@_0P@BKKG@WM_COMPAREITEM?$AA@ 5f8b6660     afxtrace.obj
 0002:0000b670       ??_C@_0BB@IMIB@WM_QUERYDRAGICON?$AA@ 5f8b6670     afxtrace.obj
 0002:0000b684       ??_C@_0L@HKOC@WM_GETFONT?$AA@ 5f8b6684     afxtrace.obj
 0002:0000b690       ??_C@_0L@CJOO@WM_SETFONT?$AA@ 5f8b6690     afxtrace.obj
 0002:0000b69c       ??_C@_0O@OAAH@WM_CHARTOITEM?$AA@ 5f8b669c     afxtrace.obj
 0002:0000b6ac       ??_C@_0O@MNJJ@WM_VKEYTOITEM?$AA@ 5f8b66ac     afxtrace.obj
 0002:0000b6bc       ??_C@_0O@NOFD@WM_DELETEITEM?$AA@ 5f8b66bc     afxtrace.obj
 0002:0000b6cc       ??_C@_0P@MAHA@WM_MEASUREITEM?$AA@ 5f8b66cc     afxtrace.obj
 0002:0000b6dc       ??_C@_0M@EHEH@WM_DRAWITEM?$AA@ 5f8b66dc     afxtrace.obj
 0002:0000b6e8       ??_C@_0BB@MJAK@WM_SPOOLERSTATUS?$AA@ 5f8b66e8     afxtrace.obj
 0002:0000b6fc       ??_C@_0O@JNLH@WM_NEXTDLGCTL?$AA@ 5f8b66fc     afxtrace.obj
 0002:0000b70c       ??_C@_0BC@KHMF@WM_ICONERASEBKGND?$AA@ 5f8b670c     afxtrace.obj
 0002:0000b720       ??_C@_0BB@INDA@WM_GETMINMAXINFO?$AA@ 5f8b6720     afxtrace.obj
 0002:0000b734       ??_C@_0N@IJHA@WM_QUEUESYNC?$AA@ 5f8b6734     afxtrace.obj
 0002:0000b744       ??_C@_0BB@GLME@WM_CHILDACTIVATE?$AA@ 5f8b6744     afxtrace.obj
 0002:0000b758       ??_C@_0BB@LPNO@WM_MOUSEACTIVATE?$AA@ 5f8b6758     afxtrace.obj
 0002:0000b76c       ??_C@_0N@GJNG@WM_SETCURSOR?$AA@ 5f8b676c     afxtrace.obj
 0002:0000b77c       ??_C@_0O@PBAP@WM_CANCELMODE?$AA@ 5f8b677c     afxtrace.obj
 0002:0000b78c       ??_C@_0O@KEEP@WM_TIMECHANGE?$AA@ 5f8b678c     afxtrace.obj
 0002:0000b79c       ??_C@_0O@NFOD@WM_FONTCHANGE?$AA@ 5f8b679c     afxtrace.obj
 0002:0000b7ac       ??_C@_0P@MIOO@WM_ACTIVATEAPP?$AA@ 5f8b67ac     afxtrace.obj
 0002:0000b7bc       ??_C@_0BB@JHBE@WM_DEVMODECHANGE?$AA@ 5f8b67bc     afxtrace.obj
 0002:0000b7d0       ??_C@_0BB@OOJC@WM_SETTINGCHANGE?$AA@ 5f8b67d0     afxtrace.obj
 0002:0000b7e4       ??_C@_0BA@OBFL@WM_WININICHANGE?$AA@ 5f8b67e4     afxtrace.obj
 0002:0000b7f4       ??_C@_0BC@IELM@WM_CTLCOLORSTATIC?$AA@ 5f8b67f4     afxtrace.obj
 0002:0000b808       ??_C@_0BF@CNIA@WM_CTLCOLORSCROLLBAR?$AA@ 5f8b6808     afxtrace.obj
 0002:0000b820       ??_C@_0P@FLDC@WM_CTLCOLORDLG?$AA@ 5f8b6820     afxtrace.obj
 0002:0000b830       ??_C@_0P@JGJH@WM_CTLCOLORBTN?$AA@ 5f8b6830     afxtrace.obj
 0002:0000b840       ??_C@_0BD@CBNP@WM_CTLCOLORLISTBOX?$AA@ 5f8b6840     afxtrace.obj
 0002:0000b854       ??_C@_0BA@LJPL@WM_CTLCOLOREDIT?$AA@ 5f8b6854     afxtrace.obj
 0002:0000b864       ??_C@_0BC@JPK@WM_CTLCOLORMSGBOX?$AA@ 5f8b6864     afxtrace.obj
 0002:0000b878       ??_C@_0O@OMHP@WM_SHOWWINDOW?$AA@ 5f8b6878     afxtrace.obj
 0002:0000b888       ??_C@_0O@LOEN@WM_ENDSESSION?$AA@ 5f8b6888     afxtrace.obj
 0002:0000b898       ??_C@_0BC@FPLF@WM_SYSCOLORCHANGE?$AA@ 5f8b6898     afxtrace.obj
 0002:0000b8ac       ??_C@_0O@FPAF@WM_ERASEBKGND?$AA@ 5f8b68ac     afxtrace.obj
 0002:0000b8bc       ??_C@_0N@BAHI@WM_QUERYOPEN?$AA@ 5f8b68bc     afxtrace.obj
 0002:0000b8cc       ??_C@_07NMOO@WM_QUIT?$AA@  5f8b68cc     afxtrace.obj
 0002:0000b8d4       ??_C@_0BD@PEGN@WM_QUERYENDSESSION?$AA@ 5f8b68d4     afxtrace.obj
 0002:0000b8e8       ??_C@_08LEAJ@WM_CLOSE?$AA@ 5f8b68e8     afxtrace.obj
 0002:0000b8f4       ??_C@_08LANE@WM_PAINT?$AA@ 5f8b68f4     afxtrace.obj
 0002:0000b900       ??_C@_0BB@HNCD@WM_GETTEXTLENGTH?$AA@ 5f8b6900     afxtrace.obj
 0002:0000b914       ??_C@_0L@EMKJ@WM_GETTEXT?$AA@ 5f8b6914     afxtrace.obj
 0002:0000b920       ??_C@_0L@BPKF@WM_SETTEXT?$AA@ 5f8b6920     afxtrace.obj
 0002:0000b92c       ??_C@_0N@LOJK@WM_SETREDRAW?$AA@ 5f8b692c     afxtrace.obj
 0002:0000b93c       ??_C@_09PJML@WM_ENABLE?$AA@ 5f8b693c     afxtrace.obj
 0002:0000b948       ??_C@_0N@LCIJ@WM_KILLFOCUS?$AA@ 5f8b6948     afxtrace.obj
 0002:0000b958       ??_C@_0M@OHD@WM_SETFOCUS?$AA@ 5f8b6958     afxtrace.obj
 0002:0000b964       ??_C@_0M@CEAM@WM_ACTIVATE?$AA@ 5f8b6964     afxtrace.obj
 0002:0000b970       ??_C@_07DNHO@WM_SIZE?$AA@  5f8b6970     afxtrace.obj
 0002:0000b978       ??_C@_07JOKK@WM_MOVE?$AA@  5f8b6978     afxtrace.obj
 0002:0000b980       ??_C@_0L@JPGJ@WM_DESTROY?$AA@ 5f8b6980     afxtrace.obj
 0002:0000b98c       ??_C@_09LLGP@WM_CREATE?$AA@ 5f8b698c     afxtrace.obj
 0002:0000b998       ??_C@_1GC@IALP@?$AA?$CF?$AAs?$AA?3?$AA?5?$AAh?$AAw?$AAn?$AAd?$AA?$DN?$AA0?$AAx?$AA?$CF?$AA0?$AA4?$AAX?$AA?0?$AA?5?$AAm?$AAs?$AAg@ 5f8b6998     afxtrace.obj
 0002:0000b9fc       ??_C@_1FM@BOB@?$AA?$CF?$AAs?$AA?3?$AA?5?$AAh?$AAw?$AAn?$AAd?$AA?$DN?$AA0?$AAx?$AA?$CF?$AA0?$AA4?$AAX?$AA?0?$AA?5?$AAm?$AAs?$AAg@ 5f8b69fc     afxtrace.obj
 0002:0000ba58       ??_C@_0P@BIFO@WM_USER?$CL0x?$CF04X?$AA@ 5f8b6a58     afxtrace.obj
 0002:0000ba68       ??_C@_1HK@JOC@?$AA?$CF?$AAs?$AA?3?$AA?5?$AAA?$AAd?$AAv?$AAi?$AAs?$AAe?$AA?5?$AAi?$AAt?$AAe?$AAm?$AA?$DN?$AA?8?$AA?$CF?$AAs?$AA?8@ 5f8b6a68     afxtrace.obj
 0002:0000bae4       ??_C@_1GO@NPAK@?$AAW?$AAa?$AAr?$AAn?$AAi?$AAn?$AAg?$AA?3?$AA?5?$AAU?$AAn?$AAa?$AAb?$AAl?$AAe?$AA?5?$AAt?$AAo?$AA?5?$AAu@ 5f8b6ae4     afxtrace.obj
 0002:0000bb54       ??_C@_1CG@GLAK@?$AA?$CF?$AAs?$AA?3?$AA?5?$AAE?$AAx?$AAe?$AAc?$AAu?$AAt?$AAe?$AA?5?$AA?8?$AA?$CF?$AAs?$AA?8?$AA?4?$AA?6?$AA?$AA@ 5f8b6b54     afxtrace.obj
 0002:0000bb7c       ??_C@_1HA@JODE@?$AAW?$AAa?$AAr?$AAn?$AAi?$AAn?$AAg?$AA?3?$AA?5?$AAU?$AAn?$AAa?$AAb?$AAl?$AAe?$AA?5?$AAt?$AAo?$AA?5?$AAu@ 5f8b6b7c     afxtrace.obj
 0002:0000bbec       ??_C@_1BC@EMPM@?$AAc?$AAo?$AAm?$AAb?$AAo?$AAb?$AAo?$AAx?$AA?$AA@ 5f8b6bec     winutil.obj
 0002:0000bc00       ??_C@_1HI@POIA@?$AAE?$AAR?$AAR?$AAO?$AAR?$AA?3?$AA?5?$AAC?$AAr?$AAi?$AAt?$AAi?$AAc?$AAa?$AAl?$AA?5?$AAm?$AAe?$AAm?$AAo@ 5f8b6c00     winutil.obj
 0002:0000bc78       ??_C@_1JM@GINF@?$AAW?$AAa?$AAr?$AAn?$AAi?$AAn?$AAg?$AA?3?$AA?5?$AAS?$AAh?$AAr?$AAi?$AAn?$AAk?$AAi?$AAn?$AAg?$AA?5?$AAs@ 5f8b6c78     winutil.obj
 0002:0000bd14       ??_C@_1GI@DBFF@?$AAW?$AAa?$AAr?$AAn?$AAi?$AAn?$AAg?$AA?3?$AA?5?$AAF?$AAr?$AAe?$AAe?$AAi?$AAn?$AAg?$AA?5?$AAa?$AAp?$AAp@ 5f8b6d14     winutil.obj
 0002:0000bd7c       ??_C@_1FK@FPPA@?$AAW?$AAa?$AAr?$AAn?$AAi?$AAn?$AAg?$AA?3?$AA?5?$AAC?$AAr?$AAi?$AAt?$AAi?$AAc?$AAa?$AAl?$AA?5?$AAm?$AAe@ 5f8b6d7c     winutil.obj
 0002:0000bdd8       ?classCCmdTarget@CCmdTarget@@2UCRuntimeClass@@B 5f8b6dd8     cmdtarg.obj
 0002:0000bdf0       ??_C@_0L@MION@CCmdTarget?$AA@ 5f8b6df0     cmdtarg.obj
 0002:0000bdfc       ?_afxDot@@3QBEB            5f8b6dfc     cmdtarg.obj
 0002:0000be08       ?messageMap@CCmdTarget@@1UAFX_MSGMAP@@B 5f8b6e08     cmdtarg.obj
 0002:0000be10       ?_messageEntries@CCmdTarget@@0QBUAFX_MSGMAP_ENTRY@@B 5f8b6e10     cmdtarg.obj
 0002:0000be28       ?dispatchMap@CCmdTarget@@1UAFX_DISPMAP@@B 5f8b6e28     cmdtarg.obj
 0002:0000be38       ?_dispatchEntries@CCmdTarget@@0QBUAFX_DISPMAP_ENTRY@@B 5f8b6e38     cmdtarg.obj
 0002:0000be58       ?eventsinkMap@CCmdTarget@@1UAFX_EVENTSINKMAP@@B 5f8b6e58     cmdtarg.obj
 0002:0000be68       ?_eventsinkEntries@CCmdTarget@@0QBUAFX_EVENTSINKMAP_ENTRY@@B 5f8b6e68     cmdtarg.obj
 0002:0000be90       ?interfaceMap@CCmdTarget@@1UAFX_INTERFACEMAP@@B 5f8b6e90     cmdtarg.obj
 0002:0000be98       ?_interfaceEntries@CCmdTarget@@0QBUAFX_INTERFACEMAP_ENTRY@@B 5f8b6e98     cmdtarg.obj
 0002:0000bea8       ?connectionMap@CCmdTarget@@1UAFX_CONNECTIONMAP@@B 5f8b6ea8     cmdtarg.obj
 0002:0000beb0       ?_connectionEntries@CCmdTarget@@0QBUAFX_CONNECTIONMAP_ENTRY@@B 5f8b6eb0     cmdtarg.obj
 0002:0000beb8       ?commandMap@CCmdTarget@@1UAFX_OLECMDMAP@@B 5f8b6eb8     cmdtarg.obj
 0002:0000bec0       ?_commandEntries@CCmdTarget@@0QBUAFX_OLECMDMAP_ENTRY@@B 5f8b6ec0     cmdtarg.obj
 0002:0000bed0       ??_7CCmdTarget@@6B@        5f8b6ed0     cmdtarg.obj
 0002:0000bf28       ??_C@_1IO@HDFI@?$AAS?$AAE?$AAN?$AAD?$AAI?$AAN?$AAG?$AA?5?$AAc?$AAo?$AAn?$AAt?$AAr?$AAo?$AAl?$AA?5?$AAn?$AAo?$AAt?$AAi@ 5f8b6f28     cmdtarg.obj
 0002:0000bfb8       ??_C@_1FE@HCMG@?$AAS?$AAE?$AAN?$AAD?$AAI?$AAN?$AAG?$AA?5?$AAc?$AAo?$AAm?$AAm?$AAa?$AAn?$AAd?$AA?5?$AAi?$AAd?$AA?5?$AA0@ 5f8b6fb8     cmdtarg.obj
 0002:0000c010       ??_7CCmdUI@@6B@            5f8b7010     cmdtarg.obj
 0002:0000c020       ??_C@_1GC@BFBK@?$AAN?$AAo?$AA?5?$AAh?$AAa?$AAn?$AAd?$AAl?$AAe?$AAr?$AA?5?$AAf?$AAo?$AAr?$AA?5?$AAc?$AAo?$AAm?$AAm?$AAa@ 5f8b7020     cmdtarg.obj
 0002:0000c084       ??_C@_1GI@JKGO@?$AAW?$AAa?$AAr?$AAn?$AAi?$AAn?$AAg?$AA?3?$AA?5?$AAu?$AAs?$AAi?$AAn?$AAg?$AA?5?$AAs?$AAy?$AAs?$AAt?$AAe@ 5f8b7084     cmdtarg.obj
 0002:0000c0ec       ??_C@_0BN@LGCD@?6with?5aggregation?5capability?$AA@ 5f8b70ec     cmdtarg.obj
 0002:0000c10c       ??_C@_0BE@MMK@?6m_pOuterUnknown?5?$DN?5?$AA@ 5f8b710c     cmdtarg.obj
 0002:0000c120       ??_C@_0M@JGEE@?6m_dwRef?5?$DN?5?$AA@ 5f8b7120     cmdtarg.obj
 0002:0000c12c       ??_C@_0BE@JODL@with?5OLE?5capability?$AA@ 5f8b712c     cmdtarg.obj
 0002:0000c140       ??_C@_0CG@PJHG@with?5OLE?5Connection?5Point?5capabi@ 5f8b7140     cmdtarg.obj
 0002:0000c168       ??_C@_0BF@JADO@m_bResultExpected?5?$DN?5?$AA@ 5f8b7168     cmdtarg.obj
 0002:0000c180       ??_C@_0CM@INHM@with?5IDispatch?5?$CIOLE?5Automation?$CJ?5@ 5f8b7180     cmdtarg.obj
 0002:0000c1b0       ?classCDocument@CDocument@@2UCRuntimeClass@@B 5f8b71b0     doccore.obj
 0002:0000c1c8       ??_C@_09IIIN@CDocument?$AA@ 5f8b71c8     doccore.obj
 0002:0000c1d8       ?messageMap@CDocument@@1UAFX_MSGMAP@@B 5f8b71d8     doccore.obj
 0002:0000c1e0       ?_messageEntries@CDocument@@0QBUAFX_MSGMAP_ENTRY@@B 5f8b71e0     doccore.obj
 0002:0000c244       ??_7CDocument@@6B@         5f8b7244     doccore.obj
 0002:0000c2fc       ??_C@_1FE@OHLE@?$AAW?$AAa?$AAr?$AAn?$AAi?$AAn?$AAg?$AA?3?$AA?5?$AAd?$AAe?$AAs?$AAt?$AAr?$AAo?$AAy?$AAi?$AAn?$AAg?$AA?5@ 5f8b72fc     doccore.obj
 0002:0000c350       ??_C@_1DO@DEGD@?$AAW?$AAa?$AAr?$AAn?$AAi?$AAn?$AAg?$AA?3?$AA?5?$AAF?$AAi?$AAl?$AAe?$AA?5?$AAs?$AAa?$AAv?$AAe?$AA?9?$AAa@ 5f8b7350     doccore.obj
 0002:0000c390       ??_C@_1DI@PFCB@?$AAW?$AAa?$AAr?$AAn?$AAi?$AAn?$AAg?$AA?3?$AA?5?$AAF?$AAi?$AAl?$AAe?$AA?5?$AAs?$AAa?$AAv?$AAe?$AA?5?$AAf@ 5f8b7390     doccore.obj
 0002:0000c3c8       ??_C@_1FE@KIHP@?$AAW?$AAa?$AAr?$AAn?$AAi?$AAn?$AAg?$AA?3?$AA?5?$AAF?$AAi?$AAl?$AAe?$AA?5?$AAs?$AAa?$AAv?$AAe?$AA?5?$AAw@ 5f8b73c8     doccore.obj
 0002:0000c41c       ??_C@_1GK@IGPN@?$AAW?$AAa?$AAr?$AAn?$AAi?$AAn?$AAg?$AA?3?$AA?5?$AAf?$AAa?$AAi?$AAl?$AAe?$AAd?$AA?5?$AAt?$AAo?$AA?5?$AAd@ 5f8b741c     doccore.obj
 0002:0000c488       ??_C@_1O@OEBA@?$AA?5?$AA?$CD?$AA?$CF?$AA?$DL?$AA?1?$AA?2?$AA?$AA@ 5f8b7488     doccore.obj
 0002:0000c498       ??_C@_1IC@OCAA@?$AAR?$AAe?$AAp?$AAo?$AAr?$AAt?$AAi?$AAn?$AAg?$AA?5?$AAf?$AAi?$AAl?$AAe?$AA?5?$AAI?$AA?1?$AAO?$AA?5?$AAe@ 5f8b7498     doccore.obj
 0002:0000c51c       ??_C@_17PPBM@?$AAM?$AAF?$AAC?$AA?$AA@ 5f8b751c     doccore.obj
 0002:0000c524       ??_C@_0M@JIL@ReplaceFile?$AA@ 5f8b7524     doccore.obj
 0002:0000c530       ??_C@_08OBID@KERNEL32?$AA@ 5f8b7530     doccore.obj
 0002:0000c540       ??_7CMirrorFile@@6B@       5f8b7540     doccore.obj
 0002:0000c59c       ??_C@_1GM@HBGH@?$AAW?$AAa?$AAr?$AAn?$AAi?$AAn?$AAg?$AA?3?$AA?5?$AAO?$AAn?$AAN?$AAe?$AAw?$AAD?$AAo?$AAc?$AAu?$AAm?$AAe@ 5f8b759c     doccore.obj
 0002:0000c608       ??_C@_1GO@PBDE@?$AAW?$AAa?$AAr?$AAn?$AAi?$AAn?$AAg?$AA?3?$AA?5?$AAO?$AAn?$AAO?$AAp?$AAe?$AAn?$AAD?$AAo?$AAc?$AAu?$AAm@ 5f8b7608     doccore.obj
 0002:0000c678       ??_C@_0M@PCO@?6with?5view?5?$AA@ 5f8b7678     doccore.obj
 0002:0000c684       ??_C@_0BD@IDHL@?6m_pDocTemplate?5?$DN?5?$AA@ 5f8b7684     doccore.obj
 0002:0000c698       ??_C@_0BA@BOKL@?6m_bModified?5?$DN?5?$AA@ 5f8b7698     doccore.obj
 0002:0000c6a8       ??_C@_0BC@BBCA@?6m_strPathName?5?$DN?5?$AA@ 5f8b76a8     doccore.obj
 0002:0000c6bc       ??_C@_0O@DGKN@m_strTitle?5?$DN?5?$AA@ 5f8b76bc     doccore.obj
 0002:0000c6d0       ?classCDocTemplate@CDocTemplate@@2UCRuntimeClass@@B 5f8b76d0     doctempl.obj
 0002:0000c6e8       ??_C@_0N@BKAE@CDocTemplate?$AA@ 5f8b76e8     doctempl.obj
 0002:0000c6fc       ??_7CDocTemplate@@6B@      5f8b76fc     doctempl.obj
 0002:0000c790       ??_C@_1HA@MBGK@?$AAW?$AAa?$AAr?$AAn?$AAi?$AAn?$AAg?$AA?3?$AA?5?$AAn?$AAo?$AA?5?$AAd?$AAo?$AAc?$AAu?$AAm?$AAe?$AAn?$AAt@ 5f8b7790     doctempl.obj
 0002:0000c800       ??_C@_1GM@IAHF@?$AAW?$AAa?$AAr?$AAn?$AAi?$AAn?$AAg?$AA?3?$AA?5?$AAD?$AAy?$AAn?$AAa?$AAm?$AAi?$AAc?$AA?5?$AAc?$AAr?$AAe@ 5f8b7800     doctempl.obj
 0002:0000c86c       ??_C@_1HG@PIDB@?$AAE?$AAr?$AAr?$AAo?$AAr?$AA?3?$AA?5?$AAy?$AAo?$AAu?$AA?5?$AAm?$AAu?$AAs?$AAt?$AA?5?$AAo?$AAv?$AAe?$AAr@ 5f8b786c     doctempl.obj
 0002:0000c8e4       ??_C@_1GA@OKDH@?$AAW?$AAa?$AAr?$AAn?$AAi?$AAn?$AAg?$AA?3?$AA?5?$AAC?$AAD?$AAo?$AAc?$AAT?$AAe?$AAm?$AAp?$AAl?$AAa?$AAt@ 5f8b78e4     doctempl.obj
 0002:0000c944       ??_C@_1FO@PBD@?$AAW?$AAa?$AAr?$AAn?$AAi?$AAn?$AAg?$AA?3?$AA?5?$AAc?$AAr?$AAe?$AAa?$AAt?$AAi?$AAn?$AAg?$AA?5?$AAf?$AAr@ 5f8b7944     doctempl.obj
 0002:0000c9a4       ??_C@_1FM@IFDE@?$AAW?$AAa?$AAr?$AAn?$AAi?$AAn?$AAg?$AA?3?$AA?5?$AAD?$AAy?$AAn?$AAa?$AAm?$AAi?$AAc?$AA?5?$AAc?$AAr?$AAe@ 5f8b79a4     doctempl.obj
 0002:0000ca00       ??_C@_1HA@KHGO@?$AAE?$AAr?$AAr?$AAo?$AAr?$AA?3?$AA?5?$AAy?$AAo?$AAu?$AA?5?$AAm?$AAu?$AAs?$AAt?$AA?5?$AAo?$AAv?$AAe?$AAr@ 5f8b7a00     doctempl.obj
 0002:0000ca70       ??_C@_1GK@HABI@?$AAW?$AAa?$AAr?$AAn?$AAi?$AAn?$AAg?$AA?3?$AA?5?$AAC?$AAD?$AAo?$AAc?$AAT?$AAe?$AAm?$AAp?$AAl?$AAa?$AAt@ 5f8b7a70     doctempl.obj
 0002:0000cadc       ??_C@_1HC@BHOO@?$AAW?$AAa?$AAr?$AAn?$AAi?$AAn?$AAg?$AA?3?$AA?5?$AAp?$AAO?$AAl?$AAe?$AAF?$AAr?$AAa?$AAm?$AAe?$AAC?$AAl@ 5f8b7adc     doctempl.obj
 0002:0000cb50       ??_C@_0L@IBCP@?6document?5?$AA@ 5f8b7b50     doctempl.obj
 0002:0000cb5c       ??_C@_0BD@MDEG@?6document?5list?5?$DN?5?$HL?$AA@ 5f8b7b5c     doctempl.obj
 0002:0000cb70       ??_C@_0BE@PGDF@?6m_pDocClass?5?$DN?5NULL?$AA@ 5f8b7b70     doctempl.obj
 0002:0000cb84       ??_C@_0BA@NHLG@?6m_pDocClass?5?$DN?5?$AA@ 5f8b7b84     doctempl.obj
 0002:0000cb94       ??_C@_0BD@HDBA@?6m_strDocStrings?3?5?$AA@ 5f8b7b94     doctempl.obj
 0002:0000cba8       ??_C@_0BB@JBHJ@m_nIDResource?5?$DN?5?$AA@ 5f8b7ba8     doctempl.obj
 0002:0000cbc0       ?classCSingleDocTemplate@CSingleDocTemplate@@2UCRuntimeClass@@B 5f8b7bc0     docsingl.obj
 0002:0000cbd8       ??_C@_0BD@BIBJ@CSingleDocTemplate?$AA@ 5f8b7bd8     docsingl.obj
 0002:0000cbf0       ??_7CSingleDocTemplate@@6B@ 5f8b7bf0     docsingl.obj
 0002:0000cc84       ??_C@_1HI@LGBO@?$AAW?$AAa?$AAr?$AAn?$AAi?$AAn?$AAg?$AA?3?$AA?5?$AAd?$AAe?$AAs?$AAt?$AAr?$AAo?$AAy?$AAi?$AAn?$AAg?$AA?5@ 5f8b7c84     docsingl.obj
 0002:0000ccfc       ??_C@_1KG@HIJG@?$AAE?$AAr?$AAr?$AAo?$AAr?$AA?3?$AA?5?$AAO?$AAn?$AAN?$AAe?$AAw?$AAD?$AAo?$AAc?$AAu?$AAm?$AAe?$AAn?$AAt@ 5f8b7cfc     docsingl.obj
 0002:0000cda4       ??_C@_1FG@HJEH@?$AAC?$AAD?$AAo?$AAc?$AAu?$AAm?$AAe?$AAn?$AAt?$AA?3?$AA?3?$AAO?$AAn?$AAO?$AAp?$AAe?$AAn?$AAD?$AAo?$AAc@ 5f8b7da4     docsingl.obj
 0002:0000cdfc       ??_C@_1FE@BP@?$AAC?$AAD?$AAo?$AAc?$AAu?$AAm?$AAe?$AAn?$AAt?$AA?3?$AA?3?$AAO?$AAn?$AAN?$AAe?$AAw?$AAD?$AAo?$AAc?$AAu@ 5f8b7dfc     docsingl.obj
 0002:0000ce50       ??_C@_0BB@FAKC@with?5no?5document?$AA@ 5f8b7e50     docsingl.obj
 0002:0000ce64       ??_C@_0BA@NJIO@with?5document?3?5?$AA@ 5f8b7e64     docsingl.obj
 0002:0000ce78       ?classCMultiDocTemplate@CMultiDocTemplate@@2UCRuntimeClass@@B 5f8b7e78     docmulti.obj
 0002:0000ce90       ??_C@_0BC@HJJP@CMultiDocTemplate?$AA@ 5f8b7e90     docmulti.obj
 0002:0000cea8       ??_7CMultiDocTemplate@@6B@ 5f8b7ea8     docmulti.obj
 0002:0000cf3c       ??_C@_1GI@FBOH@?$AAW?$AAa?$AAr?$AAn?$AAi?$AAn?$AAg?$AA?3?$AA?5?$AAn?$AAo?$AA?5?$AAs?$AAh?$AAa?$AAr?$AAe?$AAd?$AA?5?$AAm@ 5f8b7f3c     docmulti.obj
 0002:0000cfa4       ??_C@_1IA@MBAG@?$AAW?$AAa?$AAr?$AAn?$AAi?$AAn?$AAg?$AA?3?$AA?5?$AAd?$AAe?$AAs?$AAt?$AAr?$AAo?$AAy?$AAi?$AAn?$AAg?$AA?5@ 5f8b7fa4     docmulti.obj
 0002:0000d024       ??_C@_1GA@EOKF@?$AAC?$AAD?$AAo?$AAc?$AAT?$AAe?$AAm?$AAp?$AAl?$AAa?$AAt?$AAe?$AA?3?$AA?3?$AAC?$AAr?$AAe?$AAa?$AAt?$AAe@ 5f8b8024     docmulti.obj
 0002:0000d084       ??_C@_0BA@FGCH@?6with?5document?5?$AA@ 5f8b8084     docmulti.obj
 0002:0000d094       ??_C@_06COBJ@?6with?5?$AA@ 5f8b8094     docmulti.obj
 0002:0000d09c       ??_C@_0BA@GGEF@?5open?5documents?$AA@ 5f8b809c     docmulti.obj
 0002:0000d0ac       ??_C@_0BF@HCCI@?6m_nUntitledCount?5?$DN?5?$AA@ 5f8b80ac     docmulti.obj
 0002:0000d0c4       ??_C@_0BC@DCCK@?6m_hAccelTable?5?$DN?5?$AA@ 5f8b80c4     docmulti.obj
 0002:0000d0d8       ?classCDocManager@CDocManager@@2UCRuntimeClass@@B 5f8b80d8     docmgr.obj
 0002:0000d0f0       ??_C@_0M@FJOK@CDocManager?$AA@ 5f8b80f0     docmgr.obj
 0002:0000d100       ?messageMap@CNewTypeDlg@@1UAFX_MSGMAP@@B 5f8b8100     docmgr.obj
 0002:0000d108       ?_messageEntries@CNewTypeDlg@@0QBUAFX_MSGMAP_ENTRY@@B 5f8b8108     docmgr.obj
 0002:0000d138       ?_afxShellNewValue@@3QBGB  5f8b8138     docmgr.obj
 0002:0000d13c       ?_afxShellNewValueName@@3QBGB 5f8b813c     docmgr.obj
 0002:0000d150       ?_afxDDEPrintTo@@3QBGB     5f8b8150     docmgr.obj
 0002:0000d190       ?_afxDDEPrint@@3QBGB       5f8b8190     docmgr.obj
 0002:0000d1ac       ?_afxDDEOpen@@3QBGB        5f8b81ac     docmgr.obj
 0002:0000d1c8       ?_afxDDEExec@@3QBGB        5f8b81c8     docmgr.obj
 0002:0000d1d8       ?_afxDDEArg@@3QBGB         5f8b81d8     docmgr.obj
 0002:0000d1e4       ?_afxPrintToArg@@3QBGB     5f8b81e4     docmgr.obj
 0002:0000d218       ?_afxPrintArg@@3QBGB       5f8b8218     docmgr.obj
 0002:0000d22c       ?_afxOpenArg@@3QBGB        5f8b822c     docmgr.obj
 0002:0000d238       ?_afxCommand@@3QBGB        5f8b8238     docmgr.obj
 0002:0000d248       ?_afxIconIndexFmt@@3QBGB   5f8b8248     docmgr.obj
 0002:0000d250       ?_afxShellNewFmt@@3QBGB    5f8b8250     docmgr.obj
 0002:0000d268       ?_afxDefaultIconFmt@@3QBGB 5f8b8268     docmgr.obj
 0002:0000d288       ?_afxShellPrintToFmt@@3QBGB 5f8b8288     docmgr.obj
 0002:0000d2b0       ?_afxShellPrintFmt@@3QBGB  5f8b82b0     docmgr.obj
 0002:0000d2d4       ?_afxShellOpenFmt@@3QBGB   5f8b82d4     docmgr.obj
 0002:0000d2f8       ??_C@_1HI@EIDD@?$AAW?$AAa?$AAr?$AAn?$AAi?$AAn?$AAg?$AA?3?$AA?5?$AAr?$AAe?$AAg?$AAi?$AAs?$AAt?$AAr?$AAa?$AAt?$AAi?$AAo@ 5f8b82f8     docmgr.obj
 0002:0000d374       ??_7CDocManager@@6B@       5f8b8374     docmgr.obj
 0002:0000d3b8       ??_C@_1FM@CLJG@?$AAE?$AAr?$AAr?$AAo?$AAr?$AA?3?$AA?5?$AAn?$AAo?$AA?5?$AAd?$AAo?$AAc?$AAu?$AAm?$AAe?$AAn?$AAt?$AA?5?$AAt@ 5f8b83b8     docmgr.obj
 0002:0000d414       ??_C@_17EICA@?$AA?$CK?$AA?4?$AA?$CK?$AA?$AA@ 5f8b8414     docmgr.obj
 0002:0000d41c       ??_C@_17OMHC@?$AA?$CC?$AA?0?$AA?$CC?$AA?$AA@ 5f8b841c     docmgr.obj
 0002:0000d424       ??_C@_1BG@LIGO@?$AA?$FL?$AAp?$AAr?$AAi?$AAn?$AAt?$AAt?$AAo?$AA?$CI?$AA?$CC?$AA?$AA@ 5f8b8424     docmgr.obj
 0002:0000d43c       ??_C@_1BC@CMHH@?$AA?$FL?$AAp?$AAr?$AAi?$AAn?$AAt?$AA?$CI?$AA?$CC?$AA?$AA@ 5f8b843c     docmgr.obj
 0002:0000d450       ??_C@_1BA@NGLM@?$AA?$FL?$AAo?$AAp?$AAe?$AAn?$AA?$CI?$AA?$CC?$AA?$AA@ 5f8b8450     docmgr.obj
 0002:0000d460       ??_C@_1GO@HEOJ@?$AAE?$AAr?$AAr?$AAo?$AAr?$AA?3?$AA?5?$AAn?$AAo?$AA?5?$AAd?$AAo?$AAc?$AAu?$AAm?$AAe?$AAn?$AAt?$AA?5?$AAt@ 5f8b8460     docmgr.obj
 0002:0000d4d4       ??_7CNewTypeDlg@@6B@       5f8b84d4     docmgr.obj
 0002:0000d5ac       ??_C@_01KCD@?$HN?$AA@      5f8b85ac     docmgr.obj
 0002:0000d5b0       ??_C@_0L@HIOI@?6template?5?$AA@ 5f8b85b0     docmgr.obj
 0002:0000d5bc       ??_C@_0BG@EOJI@?6m_templateList?$FL?$FN?5?$DN?5?$HL?$AA@ 5f8b85bc     docmgr.obj
 0002:0000d5d4       ??_C@_1GM@PNGI@?$AAE?$AAr?$AAr?$AAo?$AAr?$AA?3?$AA?5?$AAC?$AAa?$AAn?$AA?5?$AAn?$AAo?$AAt?$AA?5?$AAf?$AAi?$AAn?$AAd?$AA?5@ 5f8b85d4     docmgr.obj
 0002:0000d640       ??_C@_1GO@KHMA@?$AAE?$AAr?$AAr?$AAo?$AAr?$AA?3?$AA?5?$AAC?$AAa?$AAn?$AA?5?$AAn?$AAo?$AAt?$AA?5?$AAf?$AAi?$AAn?$AAd?$AA?5@ 5f8b8640     docmgr.obj
 0002:0000d6b0       ?classCCtrlView@CCtrlView@@2UCRuntimeClass@@B 5f8b86b0     viewcore.obj
 0002:0000d6c8       ??_C@_09OBAN@CCtrlView?$AA@ 5f8b86c8     viewcore.obj
 0002:0000d6d8       ?classCSplitterWnd@CSplitterWnd@@2UCRuntimeClass@@B 5f8b86d8     viewcore.obj
 0002:0000d6f0       ??_C@_0N@JGP@CSplitterWnd?$AA@ 5f8b86f0     viewcore.obj
 0002:0000d700       ?messageMap@CCtrlView@@1UAFX_MSGMAP@@B 5f8b8700     viewcore.obj
 0002:0000d708       ?_messageEntries@CCtrlView@@0QBUAFX_MSGMAP_ENTRY@@B 5f8b8708     viewcore.obj
 0002:0000d738       ?messageMap@CView@@1UAFX_MSGMAP@@B 5f8b8738     viewcore.obj
 0002:0000d740       ?_messageEntries@CView@@0QBUAFX_MSGMAP_ENTRY@@B 5f8b8740     viewcore.obj
 0002:0000d864       ??_7CView@@6B@             5f8b8864     viewcore.obj
 0002:0000d974       ??_C@_1FK@CBOF@?$AAW?$AAa?$AAr?$AAn?$AAi?$AAn?$AAg?$AA?3?$AA?5?$AAC?$AAr?$AAe?$AAa?$AAt?$AAi?$AAn?$AAg?$AA?5?$AAa?$AA?5@ 5f8b8974     viewcore.obj
 0002:0000d9d0       ??_C@_0BC@DEMG@with?5no?5document?6?$AA@ 5f8b89d0     viewcore.obj
 0002:0000d9e8       ??_7CCtrlView@@6B@         5f8b89e8     viewcore.obj
 0002:0000daf8       ??_C@_0BB@ODLP@?6Default?5Style?3?5?$AA@ 5f8b8af8     viewcore.obj
 0002:0000db0c       ??_C@_0O@IIAC@?6Class?5Name?3?5?$AA@ 5f8b8b0c     viewcore.obj
 0002:0000db20       ??_7CPrintingDialog@@6B@   5f8b8b20     viewprnt.obj
 0002:0000dbf8       ?messageMap@CSplitterWnd@@1UAFX_MSGMAP@@B 5f8b8bf8     winsplit.obj
 0002:0000dc00       ?_messageEntries@CSplitterWnd@@0QBUAFX_MSGMAP_ENTRY@@B 5f8b8c00     winsplit.obj
 0002:0000ddb0       ??_C@_1FO@FOEM@?$AAW?$AAa?$AAr?$AAn?$AAi?$AAn?$AAg?$AA?3?$AA?5?$AAC?$AAS?$AAp?$AAl?$AAi?$AAt?$AAt?$AAe?$AAr?$AAW?$AAn@ 5f8b8db0     winsplit.obj
 0002:0000de14       ??_7CSplitterWnd@@6B@      5f8b8e14     winsplit.obj
 0002:0000df3c       ??_C@_1GI@KEKL@?$AAW?$AAa?$AAr?$AAn?$AAi?$AAn?$AAg?$AA?3?$AA?5?$AAc?$AAo?$AAu?$AAl?$AAd?$AAn?$AA?8?$AAt?$AA?5?$AAc?$AAr@ 5f8b8f3c     winsplit.obj
 0002:0000dfa4       ??_C@_1FC@IDNJ@?$AAO?$AAu?$AAt?$AA?5?$AAo?$AAf?$AA?5?$AAm?$AAe?$AAm?$AAo?$AAr?$AAy?$AA?5?$AAc?$AAr?$AAe?$AAa?$AAt?$AAi@ 5f8b8fa4     winsplit.obj
 0002:0000dff8       ??_C@_1HK@LEDL@?$AAE?$AAr?$AAr?$AAo?$AAr?$AA?3?$AA?5?$AAC?$AAr?$AAe?$AAa?$AAt?$AAe?$AAV?$AAi?$AAe?$AAw?$AA?5?$AA?9?$AA?5@ 5f8b8ff8     winsplit.obj
 0002:0000e074       ??_C@_1FM@FJD@?$AAW?$AAa?$AAr?$AAn?$AAi?$AAn?$AAg?$AA?3?$AA?5?$AAs?$AAp?$AAl?$AAi?$AAt?$AA?5?$AAt?$AAo?$AAo?$AA?5?$AAs@ 5f8b9074     winsplit.obj
 0002:0000e0d0       ??_C@_1FM@OJCH@?$AAW?$AAa?$AAr?$AAn?$AAi?$AAn?$AAg?$AA?3?$AA?5?$AAs?$AAp?$AAl?$AAi?$AAt?$AA?5?$AAt?$AAo?$AAo?$AA?5?$AAs@ 5f8b90d0     winsplit.obj
 0002:0000e12c       ??_C@_1GA@CKNC@?$AAW?$AAa?$AAr?$AAn?$AAi?$AAn?$AAg?$AA?3?$AA?5?$AAs?$AAp?$AAl?$AAi?$AAt?$AA?5?$AAt?$AAo?$AAo?$AA?5?$AAs@ 5f8b912c     winsplit.obj
 0002:0000e18c       ??_C@_1FK@OBLD@?$AAW?$AAa?$AAr?$AAn?$AAi?$AAn?$AAg?$AA?3?$AA?5?$AAS?$AAp?$AAl?$AAi?$AAt?$AAR?$AAo?$AAw?$AA?5?$AAf?$AAa@ 5f8b918c     winsplit.obj
 0002:0000e1e8       ??_C@_1GA@NDIF@?$AAW?$AAa?$AAr?$AAn?$AAi?$AAn?$AAg?$AA?3?$AA?5?$AAS?$AAp?$AAl?$AAi?$AAt?$AAR?$AAo?$AAw?$AA?5?$AAf?$AAa@ 5f8b91e8     winsplit.obj
 0002:0000e248       ??_C@_1GG@BBNE@?$AAW?$AAa?$AAr?$AAn?$AAi?$AAn?$AAg?$AA?3?$AA?5?$AAS?$AAp?$AAl?$AAi?$AAt?$AAC?$AAo?$AAl?$AAu?$AAm?$AAn@ 5f8b9248     winsplit.obj
 0002:0000e2b0       ??_C@_1EG@MKEH@?$AAE?$AAr?$AAr?$AAo?$AAr?$AA?3?$AA?5?$AAG?$AAe?$AAt?$AAH?$AAi?$AAt?$AAR?$AAe?$AAc?$AAt?$AA?$CI?$AA?$CF?$AAd@ 5f8b92b0     winsplit.obj
 0002:0000e2f8       ??_C@_1JM@MLAF@?$AAW?$AAa?$AAr?$AAn?$AAi?$AAn?$AAg?$AA?3?$AA?5?$AAC?$AAo?$AAu?$AAl?$AAd?$AA?5?$AAn?$AAo?$AAt?$AA?5?$AAf@ 5f8b92f8     winsplit.obj
 0002:0000e394       ??_C@_1HG@CCEH@?$AAW?$AAa?$AAr?$AAn?$AAi?$AAn?$AAg?$AA?3?$AA?5?$AAs?$AAc?$AAr?$AAo?$AAl?$AAl?$AA?5?$AAp?$AAa?$AAn?$AAe@ 5f8b9394     winsplit.obj
 0002:0000e40c       ??_C@_1HI@KMLH@?$AAW?$AAa?$AAr?$AAn?$AAi?$AAn?$AAg?$AA?3?$AA?5?$AAC?$AAa?$AAn?$AA?8?$AAt?$AA?5?$AAg?$AAo?$AA?5?$AAt?$AAo@ 5f8b940c     winsplit.obj
 0002:0000e484       ??_C@_1HK@OHDB@?$AAW?$AAa?$AAr?$AAn?$AAi?$AAn?$AAg?$AA?3?$AA?5?$AAC?$AAa?$AAn?$AAn?$AAo?$AAt?$AA?5?$AAg?$AAo?$AA?5?$AAt@ 5f8b9484     winsplit.obj
 0002:0000e500       ??_C@_1GM@PACN@?$AAW?$AAa?$AAr?$AAn?$AAi?$AAn?$AAg?$AA?3?$AA?5?$AAN?$AAe?$AAx?$AAt?$AA?5?$AAp?$AAa?$AAn?$AAe?$AA?5?$AAi@ 5f8b9500     winsplit.obj
 0002:0000e56c       ??_C@_0BD@LJP@?6m_rectTracker2?5?$DN?5?$AA@ 5f8b956c     winsplit.obj
 0002:0000e580       ??_C@_0BC@JECF@?6m_rectTracker?5?$DN?5?$AA@ 5f8b9580     winsplit.obj
 0002:0000e594       ??_C@_0BE@MCJF@?6m_ptTrackOffset?5?$DN?5?$AA@ 5f8b9594     winsplit.obj
 0002:0000e5a8       ??_C@_0BA@PCAB@?6m_rectLimit?5?$DN?5?$AA@ 5f8b95a8     winsplit.obj
 0002:0000e5b8       ??_C@_0BI@CEEL@?6TRACKING?3?5m_htTrack?5?$DN?5?$AA@ 5f8b95b8     winsplit.obj
 0002:0000e5d0       ??_C@_0BB@OJKA@?6m_cySplitter?5?$DN?5?$AA@ 5f8b95d0     winsplit.obj
 0002:0000e5e4       ??_C@_0BB@IEEK@?6m_cxSplitter?5?$DN?5?$AA@ 5f8b95e4     winsplit.obj
 0002:0000e5f8       ??_C@_0BC@PJMI@?6m_bHasVScroll?5?$DN?5?$AA@ 5f8b95f8     winsplit.obj
 0002:0000e60c       ??_C@_0BC@FLHD@?6m_bHasHScroll?5?$DN?5?$AA@ 5f8b960c     winsplit.obj
 0002:0000e620       ??_C@_0M@CMG@?6m_nCols?5?$DN?5?$AA@ 5f8b9620     winsplit.obj
 0002:0000e62c       ??_C@_0M@CGBJ@?6m_nRows?5?$DN?5?$AA@ 5f8b962c     winsplit.obj
 0002:0000e638       ??_C@_0P@DFB@?6m_nMaxCols?5?$DN?5?$AA@ 5f8b9638     winsplit.obj
 0002:0000e648       ??_C@_0P@CHIO@?6m_nMaxRows?5?$DN?5?$AA@ 5f8b9648     winsplit.obj
 0002:0000e658       ??_C@_0BH@KHOP@m_pDynamicViewClass?5?$DN?5?$AA@ 5f8b9658     winsplit.obj
 0002:0000e670       ?classCScrollView@CScrollView@@2UCRuntimeClass@@B 5f8b9670     viewscrl.obj
 0002:0000e688       ??_C@_0M@DAH@CScrollView?$AA@ 5f8b9688     viewscrl.obj
 0002:0000e698       ?sizeDefault@CScrollView@@2UtagSIZE@@B 5f8b9698     viewscrl.obj
 0002:0000e6a0       ?messageMap@CScrollView@@1UAFX_MSGMAP@@B 5f8b96a0     viewscrl.obj
 0002:0000e6a8       ?_messageEntries@CScrollView@@0QBUAFX_MSGMAP_ENTRY@@B 5f8b96a8     viewscrl.obj
 0002:0000e720       ??_C@_1CC@BFDC@?$AAW?$AAh?$AAe?$AAe?$AAl?$AAS?$AAc?$AAr?$AAo?$AAl?$AAl?$AAL?$AAi?$AAn?$AAe?$AAs?$AA?$AA@ 5f8b9720     viewscrl.obj
 0002:0000e744       ??_C@_1CM@EIGA@?$AAC?$AAo?$AAn?$AAt?$AAr?$AAo?$AAl?$AA?5?$AAP?$AAa?$AAn?$AAe?$AAl?$AA?2?$AAD?$AAe?$AAs?$AAk?$AAt?$AAo@ 5f8b9744     viewscrl.obj
 0002:0000e770       ??_C@_1O@JDNM@?$AAM?$AAo?$AAu?$AAs?$AAe?$AAZ?$AA?$AA@ 5f8b9770     viewscrl.obj
 0002:0000e780       ??_C@_1CC@LAMD@?$AAM?$AAa?$AAg?$AAe?$AAl?$AAl?$AAa?$AAn?$AA?5?$AAM?$AAS?$AAW?$AAH?$AAE?$AAE?$AAL?$AA?$AA@ 5f8b9780     viewscrl.obj
 0002:0000e7a4       ??_C@_1CK@GMOB@?$AAM?$AAS?$AAH?$AA_?$AAS?$AAC?$AAR?$AAO?$AAL?$AAL?$AA_?$AAL?$AAI?$AAN?$AAE?$AAS?$AA_?$AAM?$AAS?$AAG@ 5f8b97a4     viewscrl.obj
 0002:0000e7d4       ??_7CScrollView@@6B@       5f8b97d4     viewscrl.obj
 0002:0000e8e4       ??_C@_1FC@CLG@?$AAW?$AAa?$AAr?$AAn?$AAi?$AAn?$AAg?$AA?3?$AA?5?$AAC?$AAS?$AAc?$AAr?$AAo?$AAl?$AAl?$AAV?$AAi?$AAe?$AAw@ 5f8b98e4     viewscrl.obj
 0002:0000e938       ??_C@_1DO@JBEG@?$AA?7?$AAb?$AAe?$AAf?$AAo?$AAr?$AAe?$AA?5?$AAp?$AAa?$AAi?$AAn?$AAt?$AAi?$AAn?$AAg?$AA?5?$AAs?$AAc?$AAr@ 5f8b9938     viewscrl.obj
 0002:0000e978       ??_C@_1HC@OKNA@?$AAE?$AAr?$AAr?$AAo?$AAr?$AA?3?$AA?5?$AAm?$AAu?$AAs?$AAt?$AA?5?$AAc?$AAa?$AAl?$AAl?$AA?5?$AAS?$AAe?$AAt@ 5f8b9978     viewscrl.obj
 0002:0000e9ec       ??_C@_1JI@GBPK@?$AAW?$AAa?$AAr?$AAn?$AAi?$AAn?$AAg?$AA?3?$AA?5?$AAC?$AAS?$AAc?$AAr?$AAo?$AAl?$AAl?$AAV?$AAi?$AAe?$AAw@ 5f8b99ec     viewscrl.obj
 0002:0000ea84       ??_C@_09EEIC@?$CKunknown?$CK?$AA@ 5f8b9a84     viewscrl.obj
 0002:0000ea90       ??_C@_08BEKL@MM_TWIPS?$AA@ 5f8b9a90     viewscrl.obj
 0002:0000ea9c       ??_C@_0N@GBMF@MM_HIENGLISH?$AA@ 5f8b9a9c     viewscrl.obj
 0002:0000eaac       ??_C@_0N@NIAC@MM_LOENGLISH?$AA@ 5f8b9aac     viewscrl.obj
 0002:0000eabc       ??_C@_0M@DPCL@MM_HIMETRIC?$AA@ 5f8b9abc     viewscrl.obj
 0002:0000eac8       ??_C@_0M@PIOM@MM_LOMETRIC?$AA@ 5f8b9ac8     viewscrl.obj
 0002:0000ead4       ??_C@_07PBEB@MM_TEXT?$AA@  5f8b9ad4     viewscrl.obj
 0002:0000eadc       ??_C@_0O@MDOC@MM_SCALETOFIT?$AA@ 5f8b9adc     viewscrl.obj
 0002:0000eaec       ??_C@_07OOHN@MM_NONE?$AA@  5f8b9aec     viewscrl.obj
 0002:0000eaf4       ??_C@_0P@FKBC@?6m_nMapMode?5?$DN?5?$AA@ 5f8b9af4     viewscrl.obj
 0002:0000eb04       ??_C@_0BE@PIDK@?6m_bInsideUpdate?5?$DN?5?$AA@ 5f8b9b04     viewscrl.obj
 0002:0000eb18       ??_C@_0O@JKPF@?6m_bCenter?5?$DN?5?$AA@ 5f8b9b18     viewscrl.obj
 0002:0000eb28       ??_C@_0O@POOE@?6m_lineDev?5?$DN?5?$AA@ 5f8b9b28     viewscrl.obj
 0002:0000eb38       ??_C@_0O@FIMA@?6m_pageDev?5?$DN?5?$AA@ 5f8b9b38     viewscrl.obj
 0002:0000eb48       ??_C@_0P@HAFJ@?6m_totalDev?5?$DN?5?$AA@ 5f8b9b48     viewscrl.obj
 0002:0000eb58       ??_C@_0O@KOGC@m_totalLog?5?$DN?5?$AA@ 5f8b9b58     viewscrl.obj
 0002:0000eb68       ?classCFormView@CFormView@@2UCRuntimeClass@@B 5f8b9b68     viewform.obj
 0002:0000eb80       ??_C@_09MHPF@CFormView?$AA@ 5f8b9b80     viewform.obj
 0002:0000eb90       ?messageMap@CFormView@@1UAFX_MSGMAP@@B 5f8b9b90     viewform.obj
 0002:0000eb98       ?_messageEntries@CFormView@@0QBUAFX_MSGMAP_ENTRY@@B 5f8b9b98     viewform.obj
 0002:0000ec14       ??_7CFormView@@6B@         5f8b9c14     viewform.obj
 0002:0000ed24       ??_C@_1GG@COBA@?$AAU?$AAp?$AAd?$AAa?$AAt?$AAe?$AAD?$AAa?$AAt?$AAa?$AA?5?$AAf?$AAa?$AAi?$AAl?$AAe?$AAd?$AA?5?$AAd?$AAu@ 5f8b9d24     viewform.obj
 0002:0000ed8c       ??_C@_1FO@JGEE@?$AAW?$AAa?$AAr?$AAn?$AAi?$AAn?$AAg?$AA?3?$AA?5?$AAC?$AAF?$AAo?$AAr?$AAm?$AAV?$AAi?$AAe?$AAw?$AA?5?$AAd@ 5f8b9d8c     viewform.obj
 0002:0000edec       ??_C@_1HE@LGBF@?$AAW?$AAa?$AAr?$AAn?$AAi?$AAn?$AAg?$AA?3?$AA?5?$AAC?$AAr?$AAe?$AAa?$AAt?$AAe?$AAD?$AAl?$AAg?$AAC?$AAo@ 5f8b9dec     viewform.obj
 0002:0000ee60       ?classCEditView@CEditView@@2UCRuntimeClass@@B 5f8b9e60     viewedit.obj
 0002:0000ee78       ??_C@_09PCCM@CEditView?$AA@ 5f8b9e78     viewedit.obj
 0002:0000ee84       ?dwStyleDefault@CEditView@@2KB 5f8b9e84     viewedit.obj
 0002:0000ee88       ?nMaxSize@CEditView@@2IB   5f8b9e88     viewedit.obj
 0002:0000ee90       ?messageMap@CEditView@@1UAFX_MSGMAP@@B 5f8b9e90     viewedit.obj
 0002:0000ee98       ?_messageEntries@CEditView@@0QBUAFX_MSGMAP_ENTRY@@B 5f8b9e98     viewedit.obj
 0002:0000f108       ??_C@_1CI@PGNH@?$AAc?$AAo?$AAm?$AAm?$AAd?$AAl?$AAg?$AA_?$AAF?$AAi?$AAn?$AAd?$AAR?$AAe?$AAp?$AAl?$AAa?$AAc?$AAe?$AA?$AA@ 5f8ba108     viewedit.obj
 0002:0000f134       ??_7_AFX_EDIT_STATE@@6B@   5f8ba134     viewedit.obj
 0002:0000f13c       ??_7CEditView@@6B@         5f8ba13c     viewedit.obj
 0002:0000f260       ??_C@_1EK@KBHO@?$AAU?$AAn?$AAa?$AAb?$AAl?$AAe?$AA?5?$AAt?$AAo?$AA?5?$AAc?$AAr?$AAe?$AAa?$AAt?$AAe?$AA?5?$AAu?$AAn?$AAi@ 5f8ba260     viewedit.obj
 0002:0000f2ac       ??_C@_1CI@IJEE@?$AAL?$AAu?$AAc?$AAi?$AAd?$AAa?$AA?5?$AAS?$AAa?$AAn?$AAs?$AA?5?$AAU?$AAn?$AAi?$AAc?$AAo?$AAd?$AAe?$AA?$AA@ 5f8ba2ac     viewedit.obj
 0002:0000f2d4       ??_C@_13MCKD@?$AA?7?$AA?$AA@ 5f8ba2d4     viewedit.obj
 0002:0000f2d8       ??_C@_09EHNL@?6bNext?5?$DN?5?$AA@ 5f8ba2d8     viewedit.obj
 0002:0000f2e4       ??_C@_09GAAD@?6bCase?5?$DN?5?$AA@ 5f8ba2e4     viewedit.obj
 0002:0000f2f0       ??_C@_0P@HKAL@?6strReplace?5?$DN?5?$AA@ 5f8ba2f0     viewedit.obj
 0002:0000f300       ??_C@_0M@FIBA@?6strFind?5?$DN?5?$AA@ 5f8ba300     viewedit.obj
 0002:0000f30c       ??_C@_0O@BAGE@?6bFindOnly?5?$DN?5?$AA@ 5f8ba30c     viewedit.obj
 0002:0000f31c       ??_C@_0BE@BDLE@?6pFindReplaceDlg?5?$DN?5?$AA@ 5f8ba31c     viewedit.obj
 0002:0000f330       ??_C@_0BF@IHOD@?6static?5member?5data?3?$AA@ 5f8ba330     viewedit.obj
 0002:0000f348       ??_C@_0BA@HBLG@?6m_aPageStart?3?5?$AA@ 5f8ba348     viewedit.obj
 0002:0000f358       ??_C@_0BA@HKDA@?6m_hMirrorFont?5?$AA@ 5f8ba358     viewedit.obj
 0002:0000f368       ??_C@_0BB@NGNO@?6m_hPrinterFont?5?$AA@ 5f8ba368     viewedit.obj
 0002:0000f37c       ??_C@_0P@IBOM@m_nTabStops?5?$DN?5?$AA@ 5f8ba37c     viewedit.obj
 0002:0000f390       ?classCPreviewView@CPreviewView@@2UCRuntimeClass@@B 5f8ba390     viewprev.obj
 0002:0000f3a8       ??_C@_0N@LOLK@CPreviewView?$AA@ 5f8ba3a8     viewprev.obj
 0002:0000f3b8       ?messageMap@CPreviewView@@1UAFX_MSGMAP@@B 5f8ba3b8     viewprev.obj
 0002:0000f3c0       ?_messageEntries@CPreviewView@@0QBUAFX_MSGMAP_ENTRY@@B 5f8ba3c0     viewprev.obj
 0002:0000f5a0       ??_C@_1DO@OHCL@?$AAE?$AAr?$AAr?$AAo?$AAr?$AA?3?$AA?5?$AAD?$AAo?$AAP?$AAr?$AAi?$AAn?$AAt?$AAP?$AAr?$AAe?$AAv?$AAi?$AAe@ 5f8ba5a0     viewprev.obj
 0002:0000f5e0       ??_C@_1GA@MJLF@?$AAE?$AAr?$AAr?$AAo?$AAr?$AA?3?$AA?5?$AAc?$AAo?$AAu?$AAl?$AAd?$AAn?$AA?8?$AAt?$AA?5?$AAc?$AAr?$AAe?$AAa@ 5f8ba5e0     viewprev.obj
 0002:0000f640       ??_C@_1GC@EPKA@?$AAE?$AAr?$AAr?$AAo?$AAr?$AA?3?$AA?5?$AAP?$AAr?$AAe?$AAv?$AAi?$AAe?$AAw?$AA?5?$AAc?$AAo?$AAu?$AAl?$AAd@ 5f8ba640     viewprev.obj
 0002:0000f6a4       ??_C@_1EO@EGBN@?$AAE?$AAr?$AAr?$AAo?$AAr?$AA?3?$AA?5?$AAF?$AAa?$AAi?$AAl?$AAe?$AAd?$AA?5?$AAt?$AAo?$AA?5?$AAc?$AAr?$AAe@ 5f8ba6a4     viewprev.obj
 0002:0000f6f8       ??_7CPreviewView@@6B@      5f8ba6f8     viewprev.obj
 0002:0000f814       ??_C@_1FM@KDFI@?$AA?7?$AAD?$AAi?$AAd?$AA?5?$AAy?$AAo?$AAu?$AA?5?$AAr?$AAe?$AAm?$AAe?$AAm?$AAb?$AAe?$AAr?$AA?5?$AAt?$AAo@ 5f8ba814     viewprev.obj
 0002:0000f870       ??_C@_1EI@NBPG@?$AAE?$AAr?$AAr?$AAo?$AAr?$AA?3?$AA?5?$AAh?$AAD?$AAC?$AA?5?$AAn?$AAo?$AAt?$AA?5?$AAs?$AAe?$AAt?$AA?5?$AAf@ 5f8ba870     viewprev.obj
 0002:0000f8b8       ??_C@_1HK@OGEJ@?$AAM?$AAa?$AAl?$AAf?$AAo?$AAr?$AAm?$AAe?$AAd?$AA?5?$AAP?$AAa?$AAg?$AAe?$AA?5?$AAD?$AAe?$AAs?$AAc?$AAr@ 5f8ba8b8     viewprev.obj
 0002:0000f934       ??_C@_0BB@PBHN@?6m_pPreviewDC?5?$DN?5?$AA@ 5f8ba934     viewprev.obj
 0002:0000f948       ??_C@_0O@DBPJ@?6m_dcPrint?5?$DN?5?$AA@ 5f8ba948     viewprev.obj
 0002:0000f958       ??_C@_0P@IJCK@MM_ANISOTROPIC?$AA@ 5f8ba958     viewprev.obj
 0002:0000f968       ??_C@_0N@PCPL@MM_ISOTROPIC?$AA@ 5f8ba968     viewprev.obj
 0002:0000f978       ??_C@_0M@PFDM@ZOOM_MIDDLE?$AA@ 5f8ba978     viewprev.obj
 0002:0000f984       ??_C@_07GDBC@ZOOM_IN?$AA@  5f8ba984     viewprev.obj
 0002:0000f98c       ??_C@_08BFPK@ZOOM_OUT?$AA@ 5f8ba98c     viewprev.obj
 0002:0000f998       ??_C@_0BB@FHNA@?6m_nZoomState?5?$DN?5?$AA@ 5f8ba998     viewprev.obj
 0002:0000f9ac       ??_C@_0BE@OPKL@?6m_ptCenterPoint?5?$DN?5?$AA@ 5f8ba9ac     viewprev.obj
 0002:0000f9c0       ??_C@_0BF@PDIA@?6m_sizePrinterPPI?5?$DN?5?$AA@ 5f8ba9c0     viewprev.obj
 0002:0000f9d8       ??_C@_0BA@JPPO@?6m_nMaxPages?5?$DN?5?$AA@ 5f8ba9d8     viewprev.obj
 0002:0000f9e8       ??_C@_0BG@BFDN@?6m_nSecondPageOffset?5?$AA@ 5f8ba9e8     viewprev.obj
 0002:0000fa00       ??_C@_0BB@NIFL@?6m_nCurrentPage?5?$AA@ 5f8baa00     viewprev.obj
 0002:0000fa14       ??_C@_0N@JAPP@?6m_nPages?5?$DN?5?$AA@ 5f8baa14     viewprev.obj
 0002:0000fa24       ??_C@_0BI@FEFH@?6m_bPageNumDisplayed?5?$DN?5?$AA@ 5f8baa24     viewprev.obj
 0002:0000fa3c       ??_C@_0BA@NFLH@?6m_pOrigView?5?$DN?5?$AA@ 5f8baa3c     viewprev.obj
 0002:0000fa4c       ??_C@_0BA@GMAL@m_pPrintView?5?$DN?5?$AA@ 5f8baa4c     viewprev.obj
 0002:0000fa60       ?classCTreeView@CTreeView@@2UCRuntimeClass@@B 5f8baa60     viewcmn.obj
 0002:0000fa78       ??_C@_09GPDN@CTreeView?$AA@ 5f8baa78     viewcmn.obj
 0002:0000fa88       ?classCListView@CListView@@2UCRuntimeClass@@B 5f8baa88     viewcmn.obj
 0002:0000faa0       ??_C@_09MHFL@CListView?$AA@ 5f8baaa0     viewcmn.obj
 0002:0000fac0       ?messageMap@CTreeView@@1UAFX_MSGMAP@@B 5f8baac0     viewcmn.obj
 0002:0000fac8       ?_messageEntries@CTreeView@@0QBUAFX_MSGMAP_ENTRY@@B 5f8baac8     viewcmn.obj
 0002:0000faf8       ?messageMap@CListView@@1UAFX_MSGMAP@@B 5f8baaf8     viewcmn.obj
 0002:0000fb00       ?_messageEntries@CListView@@0QBUAFX_MSGMAP_ENTRY@@B 5f8bab00     viewcmn.obj
 0002:0000fb34       ??_7CListView@@6B@         5f8bab34     viewcmn.obj
 0002:0000fc4c       ??_7CTreeView@@6B@         5f8bac4c     viewcmn.obj
 0002:0000fd60       ??_7_AFX_MAIL_STATE@@6B@   5f8bad60     docmapi.obj
 0002:0000fd64       ??_C@_1GE@CNKP@?$AAW?$AAa?$AAr?$AAn?$AAi?$AAn?$AAg?$AA?3?$AA?5?$AAf?$AAi?$AAl?$AAe?$AA?5?$AAs?$AAa?$AAv?$AAe?$AA?5?$AAf@ 5f8bad64     docmapi.obj
 0002:0000fdc8       ??_C@_17OCMI@?$AAa?$AAf?$AAx?$AA?$AA@ 5f8badc8     docmapi.obj
 0002:0000fdd0       ??_C@_0N@HFFA@MAPISendMail?$AA@ 5f8badd0     docmapi.obj
 0002:0000fde0       ??_C@_0L@ICPG@MAPI32?4DLL?$AA@ 5f8bade0     docmapi.obj
 0002:0000fdec       ??_C@_1BG@PFLE@?$AAM?$AAA?$AAP?$AAI?$AA3?$AA2?$AA?4?$AAD?$AAL?$AAL?$AA?$AA@ 5f8badec     docmapi.obj
 0002:0000fe04       ??_C@_19DFMB@?$AAM?$AAA?$AAI?$AAL?$AA?$AA@ 5f8bae04     docmapi.obj
 0002:0000fe10       ??_C@_19IMNH@?$AAM?$AAA?$AAP?$AAI?$AA?$AA@ 5f8bae10     docmapi.obj
 0002:0000fe20       ?classCWinThread@CWinThread@@2UCRuntimeClass@@B 5f8bae20     thrdcore.obj
 0002:0000fe38       ??_C@_0L@BKIL@CWinThread?$AA@ 5f8bae38     thrdcore.obj
 0002:0000fe44       ??_C@_1FM@KGED@?$AAW?$AAa?$AAr?$AAn?$AAi?$AAn?$AAg?$AA?3?$AA?5?$AAE?$AAr?$AAr?$AAo?$AAr?$AA?5?$AAd?$AAu?$AAr?$AAi?$AAn@ 5f8bae44     thrdcore.obj
 0002:0000fea4       ??_7CWinThread@@6B@        5f8baea4     thrdcore.obj
 0002:0000ff28       ??_C@_1HE@EAH@?$AAW?$AAa?$AAr?$AAn?$AAi?$AAn?$AAg?$AA?3?$AA?5?$AAC?$AAr?$AAe?$AAa?$AAt?$AAe?$AAE?$AAv?$AAe?$AAn?$AAt@ 5f8baf28     thrdcore.obj
 0002:0000ff9c       ??_C@_1BI@FLOA@?$AAP?$AAu?$AAm?$AAp?$AAM?$AAe?$AAs?$AAs?$AAa?$AAg?$AAe?$AA?$AA@ 5f8baf9c     thrdcore.obj
 0002:0000ffb4       ??_C@_1HG@OHCD@?$AAE?$AAr?$AAr?$AAo?$AAr?$AA?3?$AA?5?$AAC?$AAW?$AAi?$AAn?$AAT?$AAh?$AAr?$AAe?$AAa?$AAd?$AA?3?$AA?3?$AAP@ 5f8bafb4     thrdcore.obj
 0002:0001002c       ??_C@_1FK@CIFA@?$AAC?$AAW?$AAi?$AAn?$AAT?$AAh?$AAr?$AAe?$AAa?$AAd?$AA?3?$AA?3?$AAP?$AAu?$AAm?$AAp?$AAM?$AAe?$AAs?$AAs@ 5f8bb02c     thrdcore.obj
 0002:00010088       ??_C@_0P@GMKI@?6m_nMsgLast?5?$DN?5?$AA@ 5f8bb088     thrdcore.obj
 0002:00010098       ??_C@_0BD@PJHD@?6m_ptCursorLast?5?$DN?5?$AA@ 5f8bb098     thrdcore.obj
 0002:000100ac       ??_C@_0BE@PBKK@?6m_pThreadParams?5?$DN?5?$AA@ 5f8bb0ac     thrdcore.obj
 0002:000100c0       ??_C@_07HGLI@?6?7pt?5?$DN?5?$AA@ 5f8bb0c0     thrdcore.obj
 0002:000100c8       ??_C@_09GLNE@?6?7time?5?$DN?5?$AA@ 5f8bb0c8     thrdcore.obj
 0002:000100d4       ??_C@_0M@FCJI@?6?7lParam?5?$DN?5?$AA@ 5f8bb0d4     thrdcore.obj
 0002:000100e0       ??_C@_0M@CCID@?6?7wParam?5?$DN?5?$AA@ 5f8bb0e0     thrdcore.obj
 0002:000100ec       ??_C@_0N@FJCP@?6?7message?5?$DN?5?$AA@ 5f8bb0ec     thrdcore.obj
 0002:000100fc       ??_C@_09DIL@?6?7hwnd?5?$DN?5?$AA@ 5f8bb0fc     thrdcore.obj
 0002:00010108       ??_C@_0O@KHHI@?6m_msgCur?5?$DN?5?$HL?$AA@ 5f8bb108     thrdcore.obj
 0002:00010118       ??_C@_0P@NEDM@?6m_pMainWnd?5?$DN?5?$AA@ 5f8bb118     thrdcore.obj
 0002:00010128       ??_C@_0BI@HNBD@?6m_nDisablePumpCount?5?$DN?5?$AA@ 5f8bb128     thrdcore.obj
 0002:00010140       ??_C@_0BA@DPHF@?6m_nThreadID?5?$DN?5?$AA@ 5f8bb140     thrdcore.obj
 0002:00010150       ??_C@_0O@FLKC@?6m_hThread?5?$DN?5?$AA@ 5f8bb150     thrdcore.obj
 0002:00010160       ??_C@_0BE@BFCE@?6m_pfnThreadProc?5?$DN?5?$AA@ 5f8bb160     thrdcore.obj
 0002:00010174       ??_C@_0BD@PNCO@m_pThreadParams?5?$DN?5?$AA@ 5f8bb174     thrdcore.obj
 0002:0001018c       ??_7_AFX_CTL3D_THREAD@@6B@ 5f8bb18c     thrdcore.obj
 0002:00010190       ?classCWinApp@CWinApp@@2UCRuntimeClass@@B 5f8bb190     appcore.obj
 0002:000101a8       ??_C@_07DHEF@CWinApp?$AA@  5f8bb1a8     appcore.obj
 0002:000101b0       ?messageMap@CWinApp@@1UAFX_MSGMAP@@B 5f8bb1b0     appcore.obj
 0002:000101b8       ?_messageEntries@CWinApp@@0QBUAFX_MSGMAP_ENTRY@@B 5f8bb1b8     appcore.obj
 0002:00010218       ?_afxPreviewEntry@@3QBGB   5f8bb218     appcore.obj
 0002:00010234       ?_afxPreviewSection@@3QBGB 5f8bb234     appcore.obj
 0002:00010248       ?_afxFileEntry@@3QBGB      5f8bb248     appcore.obj
 0002:00010258       ?_afxFileSection@@3QBGB    5f8bb258     appcore.obj
 0002:00010280       ??_7_AFX_WIN_STATE@@6B@    5f8bb280     appcore.obj
 0002:00010288       ??_7CWinApp@@6B@           5f8bb288     appcore.obj
 0002:00010330       ??_7CCommandLineInfo@@6B@  5f8bb330     appcore.obj
 0002:0001034c       ??_C@_0L@POJA@Automation?$AA@ 5f8bb34c     appcore.obj
 0002:00010358       ??_C@_09LHIP@Embedding?$AA@ 5f8bb358     appcore.obj
 0002:00010364       ??_C@_03FNJD@dde?$AA@      5f8bb364     appcore.obj
 0002:00010368       ??_C@_0M@HIDL@Unregserver?$AA@ 5f8bb368     appcore.obj
 0002:00010374       ??_C@_0L@MNBE@Unregister?$AA@ 5f8bb374     appcore.obj
 0002:00010380       ??_C@_01FOFA@p?$AA@        5f8bb380     appcore.obj
 0002:00010384       ??_C@_02OBFC@pt?$AA@       5f8bb384     appcore.obj
 0002:00010388       ??_C@_1IK@MNJF@?$AAW?$AAa?$AAr?$AAn?$AAi?$AAn?$AAg?$AA?3?$AA?5?$AAm?$AA_?$AAp?$AAM?$AAa?$AAi?$AAn?$AAW?$AAn?$AAd?$AA?5@ 5f8bb388     appcore.obj
 0002:00010414       ??_C@_0BH@PIJH@?6m_nNumPreviewPages?5?$DN?5?$AA@ 5f8bb414     appcore.obj
 0002:0001042c       ??_C@_0BM@ONLF@?6m_hcurWaitCursorRestore?5?$DN?5?$AA@ 5f8bb42c     appcore.obj
 0002:00010448       ??_C@_0BH@HIBE@?6m_nWaitCursorCount?5?$DN?5?$AA@ 5f8bb448     appcore.obj
 0002:00010460       ??_C@_08NLBP@?6?7File?3?5?$AA@ 5f8bb460     appcore.obj
 0002:0001046c       ??_C@_0BH@IMKH@?6m_strRecentFiles?$FL?$FN?5?$DN?5?$AA@ 5f8bb46c     appcore.obj
 0002:00010484       ??_C@_0BG@IPJO@?6m_dwPromptContext?5?$DN?5?$AA@ 5f8bb484     appcore.obj
 0002:0001049c       ??_C@_0BA@BILD@?6m_hDevNames?5?$DN?5?$AA@ 5f8bb49c     appcore.obj
 0002:000104ac       ??_C@_0P@GNCF@?6m_hDevMode?5?$DN?5?$AA@ 5f8bb4ac     appcore.obj
 0002:000104bc       ??_C@_0BF@JALM@?6m_pszProfileName?5?$DN?5?$AA@ 5f8bb4bc     appcore.obj
 0002:000104d4       ??_C@_0BG@OAHJ@?6m_pszHelpFilePath?5?$DN?5?$AA@ 5f8bb4d4     appcore.obj
 0002:000104ec       ??_C@_0BB@IKHF@?6m_pszExeName?5?$DN?5?$AA@ 5f8bb4ec     appcore.obj
 0002:00010500       ??_C@_0BA@ILGP@?6m_bHelpMode?5?$DN?5?$AA@ 5f8bb500     appcore.obj
 0002:00010510       ??_C@_0BB@ENEA@?6m_pszAppName?5?$DN?5?$AA@ 5f8bb510     appcore.obj
 0002:00010524       ??_C@_0P@NBJF@?6m_nCmdShow?5?$DN?5?$AA@ 5f8bb524     appcore.obj
 0002:00010534       ??_C@_0BA@IPNE@?6m_lpCmdLine?5?$DN?5?$AA@ 5f8bb534     appcore.obj
 0002:00010544       ??_C@_0BE@HDGO@?6m_hPrevInstance?5?$DN?5?$AA@ 5f8bb544     appcore.obj
 0002:00010558       ??_C@_0P@BLOD@m_hInstance?5?$DN?5?$AA@ 5f8bb558     appcore.obj
 0002:00010568       ??_C@_0CG@NLNA@E?3?28168?2vc98?2mfc?2mfc?2include?2afx@ 5f8bb568     appcore.obj
 0002:00010590       ??_C@_19KGAM@?$AA?4?$AAI?$AAN?$AAI?$AA?$AA@ 5f8bb590     appinit.obj
 0002:0001059c       ??_C@_19CLBK@?$AA?4?$AAH?$AAL?$AAP?$AA?$AA@ 5f8bb59c     appinit.obj
 0002:000105a8       ??_C@_1DG@EHDI@?$AAM?$AAR?$AAU?$AA?3?$AA?5?$AAo?$AAp?$AAe?$AAn?$AA?5?$AAf?$AAi?$AAl?$AAe?$AA?5?$AA?$CI?$AA?$CF?$AAd?$AA?$CJ?$AA?5@ 5f8bb5a8     appui.obj
 0002:000105e0       ??_C@_1FK@BFAO@?$AAW?$AAa?$AAr?$AAn?$AAi?$AAn?$AAg?$AA?3?$AA?5?$AAn?$AAo?$AA?5?$AAi?$AAc?$AAo?$AAn?$AA?5?$AAs?$AAp?$AAe@ 5f8bb5e0     appui1.obj
 0002:0001063c       ??_C@_1HC@OMKM@?$AAE?$AAr?$AAr?$AAo?$AAr?$AA?3?$AA?5?$AAf?$AAa?$AAi?$AAl?$AAe?$AAd?$AA?5?$AAt?$AAo?$AA?5?$AAl?$AAo?$AAa@ 5f8bb63c     appui1.obj
 0002:000106b0       ??_C@_13HMCP@?$AA?2?$AA?$AA@ 5f8bb6b0     appui2.obj
 0002:000106b4       ??_C@_1BE@JFBP@?$AAS?$AAo?$AAf?$AAt?$AAw?$AAa?$AAr?$AAe?$AA?2?$AA?$AA@ 5f8bb6b4     appui2.obj
 0002:000106c8       ??_C@_1O@IKOG@?$AAs?$AAy?$AAs?$AAt?$AAe?$AAm?$AA?$AA@ 5f8bb6c8     appui2.obj
 0002:000106d8       ??_C@_1BC@GMME@?$AAs?$AAo?$AAf?$AAt?$AAw?$AAa?$AAr?$AAe?$AA?$AA@ 5f8bb6d8     appui3.obj
 0002:000106ec       ??_C@_0M@PMCB@CTL3D32?4DLL?$AA@ 5f8bb6ec     app3d.obj
 0002:000106f8       ??_C@_1GM@GFJL@?$AAE?$AAr?$AAr?$AAo?$AAr?$AA?3?$AA?5?$AAf?$AAa?$AAi?$AAl?$AAe?$AAd?$AA?5?$AAt?$AAo?$AA?5?$AAl?$AAo?$AAa@ 5f8bb6f8     apphelp.obj
 0002:00010764       ??_C@_1FG@POBE@?$AAE?$AAr?$AAr?$AAo?$AAr?$AA?3?$AA?5?$AAi?$AAl?$AAl?$AAe?$AAg?$AAa?$AAl?$AA?5?$AAs?$AAt?$AAr?$AAi?$AAn@ 5f8bb764     apphelp.obj
 0002:000107bc       ??_C@_19BHME@?$AA?2?$AA?4?$AA?4?$AA?4?$AA?$AA@ 5f8bb7bc     filelist.obj
 0002:000107cc       ??_7CRecentFileList@@6B@   5f8bb7cc     filelist.obj
 0002:000107e4       ??_C@_19ENHM@?$AA?$CG?$AA?$CF?$AAd?$AA?5?$AA?$AA@ 5f8bb7e4     filelist.obj
 0002:000107f0       ??_C@_1JC@JPME@?$AAW?$AAa?$AAr?$AAn?$AAi?$AAn?$AAg?$AA?3?$AA?5?$AAA?$AAf?$AAx?$AAO?$AAl?$AAe?$AAS?$AAe?$AAt?$AAU?$AAs@ 5f8bb7f0     olelock.obj
 0002:00010888       ?classCGopherFileFind@CGopherFileFind@@2UCRuntimeClass@@B 5f8bb888     inet.obj
 0002:000108a0       ??_C@_0BA@FPGB@CGopherFileFind?$AA@ 5f8bb8a0     inet.obj
 0002:000108b0       ?classCFtpFileFind@CFtpFileFind@@2UCRuntimeClass@@B 5f8bb8b0     inet.obj
 0002:000108c8       ??_C@_0N@NGMH@CFtpFileFind?$AA@ 5f8bb8c8     inet.obj
 0002:000108d8       ?classCGopherConnection@CGopherConnection@@2UCRuntimeClass@@B 5f8bb8d8     inet.obj
 0002:000108f0       ??_C@_0BC@JCEC@CGopherConnection?$AA@ 5f8bb8f0     inet.obj
 0002:00010908       ?classCHttpConnection@CHttpConnection@@2UCRuntimeClass@@B 5f8bb908     inet.obj
 0002:00010920       ??_C@_0BA@OLNH@CHttpConnection?$AA@ 5f8bb920     inet.obj
 0002:00010930       ?classCFtpConnection@CFtpConnection@@2UCRuntimeClass@@B 5f8bb930     inet.obj
 0002:00010948       ??_C@_0P@HPOD@CFtpConnection?$AA@ 5f8bb948     inet.obj
 0002:00010958       ?classCInternetConnection@CInternetConnection@@2UCRuntimeClass@@B 5f8bb958     inet.obj
 0002:00010970       ??_C@_0BE@NNFJ@CInternetConnection?$AA@ 5f8bb970     inet.obj
 0002:00010988       ?classCInternetSession@CInternetSession@@2UCRuntimeClass@@B 5f8bb988     inet.obj
 0002:000109a0       ??_C@_0BB@BEAH@CInternetSession?$AA@ 5f8bb9a0     inet.obj
 0002:000109b8       ?classCGopherFile@CGopherFile@@2UCRuntimeClass@@B 5f8bb9b8     inet.obj
 0002:000109d0       ??_C@_0M@HDHO@CGopherFile?$AA@ 5f8bb9d0     inet.obj
 0002:000109e0       ?classCHttpFile@CHttpFile@@2UCRuntimeClass@@B 5f8bb9e0     inet.obj
 0002:000109f8       ??_C@_09IMKB@CHttpFile?$AA@ 5f8bb9f8     inet.obj
 0002:00010a08       ?classCInternetFile@CInternetFile@@2UCRuntimeClass@@B 5f8bba08     inet.obj
 0002:00010a20       ??_C@_0O@FDJM@CInternetFile?$AA@ 5f8bba20     inet.obj
 0002:00010a30       ?classCInternetException@CInternetException@@2UCRuntimeClass@@B 5f8bba30     inet.obj
 0002:00010a48       ??_C@_0BD@EMID@CInternetException?$AA@ 5f8bba48     inet.obj
 0002:00010a5c       ?szHtmlVerbs@CHttpConnection@@1QBQBGB 5f8bba5c     inet.obj
 0002:00010a78       ??_C@_1O@IMGP@?$AAU?$AAN?$AAL?$AAI?$AAN?$AAK?$AA?$AA@ 5f8bba78     inet.obj
 0002:00010a88       ??_C@_1O@FBDO@?$AAD?$AAE?$AAL?$AAE?$AAT?$AAE?$AA?$AA@ 5f8bba88     inet.obj
 0002:00010a98       ??_C@_19FNLP@?$AAL?$AAI?$AAN?$AAK?$AA?$AA@ 5f8bba98     inet.obj
 0002:00010aa4       ??_C@_17ILBJ@?$AAP?$AAU?$AAT?$AA?$AA@ 5f8bbaa4     inet.obj
 0002:00010aac       ??_C@_19NFGA@?$AAH?$AAE?$AAA?$AAD?$AA?$AA@ 5f8bbaac     inet.obj
 0002:00010ab8       ??_C@_17KJPO@?$AAG?$AAE?$AAT?$AA?$AA@ 5f8bbab8     inet.obj
 0002:00010ac0       ??_C@_19KJFA@?$AAP?$AAO?$AAS?$AAT?$AA?$AA@ 5f8bbac0     inet.obj
 0002:00010acc       ?_afxURLhttp@@3QBGB        5f8bbacc     inet.obj
 0002:00010adc       ?_afxURLftp@@3QBGB         5f8bbadc     inet.obj
 0002:00010aec       ??_C@_1CI@JKPN@?$AAU?$AAn?$AAk?$AAn?$AAo?$AAw?$AAn?$AA?5?$AAs?$AAt?$AAa?$AAt?$AAu?$AAs?$AA?3?$AA?5?$AA?$CF?$AAd?$AA?6?$AA?$AA@ 5f8bbaec     inet.obj
 0002:00010b14       ??_C@_1CG@JFMO@?$AAr?$AAe?$AAq?$AAu?$AAe?$AAs?$AAt?$AA?5?$AAc?$AAo?$AAm?$AAp?$AAl?$AAe?$AAt?$AAe?$AA?4?$AA?6?$AA?$AA@ 5f8bbb14     inet.obj
 0002:00010b3c       ??_C@_1GK@BKEA@?$AAr?$AAe?$AAq?$AAu?$AAe?$AAs?$AAt?$AA?5?$AAc?$AAo?$AAm?$AAp?$AAl?$AAe?$AAt?$AAe?$AA?0?$AA?5?$AAd?$AAw@ 5f8bbb3c     inet.obj
 0002:00010ba8       ??_C@_1CM@OCOM@?$AAh?$AAa?$AAn?$AAd?$AAl?$AAe?$AA?5?$AA?$CF?$AA8?$AA?4?$AA8?$AAX?$AA?5?$AAc?$AAl?$AAo?$AAs?$AAe?$AAd?$AA?$CB@ 5f8bbba8     inet.obj
 0002:00010bd4       ??_C@_1DE@KFJB@?$AAc?$AAo?$AAn?$AAn?$AAe?$AAc?$AAt?$AAi?$AAo?$AAn?$AA?5?$AA?$CF?$AA8?$AA?4?$AA8?$AAX?$AA?5?$AAc?$AAl?$AAo@ 5f8bbbd4     inet.obj
 0002:00010c08       ??_C@_1DE@OGJA@?$AAc?$AAl?$AAo?$AAs?$AAi?$AAn?$AAg?$AA?5?$AAc?$AAo?$AAn?$AAn?$AAe?$AAc?$AAt?$AAi?$AAo?$AAn?$AA?5?$AA?$CF@ 5f8bbc08     inet.obj
 0002:00010c3c       ??_C@_1CI@MDEA@?$AAr?$AAe?$AAs?$AAp?$AAo?$AAn?$AAs?$AAe?$AA?5?$AAr?$AAe?$AAc?$AAe?$AAi?$AAv?$AAe?$AAd?$AA?$CB?$AA?6?$AA?$AA@ 5f8bbc3c     inet.obj
 0002:00010c64       ??_C@_1CO@ENDF@?$AAr?$AAe?$AAc?$AAe?$AAi?$AAv?$AAi?$AAn?$AAg?$AA?5?$AAr?$AAe?$AAs?$AAp?$AAo?$AAn?$AAs?$AAe?$AA?4?$AA?4@ 5f8bbc64     inet.obj
 0002:00010c94       ??_C@_1DM@HJAA@?$AAc?$AAo?$AAn?$AAn?$AAe?$AAc?$AAt?$AAe?$AAd?$AA?5?$AAt?$AAo?$AA?5?$AAs?$AAo?$AAc?$AAk?$AAe?$AAt?$AA?5@ 5f8bbc94     inet.obj
 0002:00010cd0       ??_C@_1CI@IGPM@?$AAs?$AAe?$AAn?$AAd?$AAi?$AAn?$AAg?$AA?5?$AAr?$AAe?$AAq?$AAu?$AAe?$AAs?$AAt?$AA?4?$AA?4?$AA?4?$AA?6?$AA?$AA@ 5f8bbcd0     inet.obj
 0002:00010cf8       ??_C@_1BO@IILD@?$AAr?$AAe?$AAq?$AAu?$AAe?$AAs?$AAt?$AA?5?$AAs?$AAe?$AAn?$AAt?$AA?$CB?$AA?6?$AA?$AA@ 5f8bbcf8     inet.obj
 0002:00010d18       ??_C@_1EG@KDCF@?$AAc?$AAo?$AAn?$AAn?$AAe?$AAc?$AAt?$AAi?$AAn?$AAg?$AA?5?$AAt?$AAo?$AA?5?$AAs?$AAo?$AAc?$AAk?$AAe?$AAt@ 5f8bbd18     inet.obj
 0002:00010d60       ??_C@_1CM@OHMG@?$AAh?$AAa?$AAn?$AAd?$AAl?$AAe?$AA?5?$AA?$CF?$AA8?$AA?4?$AA8?$AAX?$AA?5?$AAc?$AAr?$AAe?$AAa?$AAt?$AAe?$AAd@ 5f8bbd60     inet.obj
 0002:00010d8c       ??_C@_1CO@MKEC@?$AAr?$AAe?$AAs?$AAo?$AAl?$AAv?$AAe?$AAd?$AA?5?$AAn?$AAa?$AAm?$AAe?$AA?5?$AAf?$AAo?$AAr?$AA?5?$AA?$CF?$AAs@ 5f8bbd8c     inet.obj
 0002:00010dbc       ??_C@_1CO@FDOL@?$AAr?$AAe?$AAs?$AAo?$AAl?$AAv?$AAi?$AAn?$AAg?$AA?5?$AAn?$AAa?$AAm?$AAe?$AA?5?$AAf?$AAo?$AAr?$AA?5?$AA?$CF@ 5f8bbdbc     inet.obj
 0002:00010dec       ??_C@_1CG@LKHP@?$AAI?$AAn?$AAt?$AAe?$AAr?$AAn?$AAe?$AAt?$AA?5?$AAc?$AAt?$AAx?$AAt?$AA?$DN?$AA?$CF?$AAd?$AA?3?$AA?5?$AA?$AA@ 5f8bbdec     inet.obj
 0002:00010e18       ??_7CInternetSession@@6B@  5f8bbe18     inet.obj
 0002:00010e34       ??_C@_1FC@CAPM@?$AAE?$AAr?$AAr?$AAo?$AAr?$AA?3?$AA?5?$AAU?$AAn?$AAi?$AAd?$AAe?$AAn?$AAt?$AAi?$AAf?$AAi?$AAe?$AAd?$AA?5@ 5f8bbe34     inet.obj
 0002:00010e88       ??_C@_0BA@CGKN@?6m_dwContext?5?$DN?5?$AA@ 5f8bbe88     inet.obj
 0002:00010e98       ??_C@_0O@GFCO@m_hSession?5?$DN?5?$AA@ 5f8bbe98     inet.obj
 0002:00010eac       ??_7CInternetFile@@6B@     5f8bbeac     inet.obj
 0002:00010f14       ??_C@_1GE@BEFK@?$AAW?$AAa?$AAr?$AAn?$AAi?$AAn?$AAg?$AA?3?$AA?5?$AAd?$AAe?$AAs?$AAt?$AAr?$AAo?$AAy?$AAi?$AAn?$AAg?$AA?5@ 5f8bbf14     inet.obj
 0002:00010f78       ??_C@_0O@ONDP@?5with?5handle?5?$AA@ 5f8bbf78     inet.obj
 0002:00010f88       ??_C@_03PCF@?6a?5?$AA@     5f8bbf88     inet.obj
 0002:00010f90       ??_7CInternetConnection@@6B@ 5f8bbf90     inet.obj
 0002:00010fa8       ??_C@_1JC@GBFE@?$AAW?$AAa?$AAr?$AAn?$AAi?$AAn?$AAg?$AA?3?$AA?5?$AAD?$AAi?$AAs?$AAc?$AAo?$AAn?$AAn?$AAe?$AAc?$AAt?$AAi@ 5f8bbfa8     inet.obj
 0002:0001103c       ??_C@_0BB@JPFC@m_hConnection?5?$DN?5?$AA@ 5f8bc03c     inet.obj
 0002:00011054       ??_7CFtpConnection@@6B@    5f8bc054     inet.obj
 0002:0001106c       ??_C@_0BE@LGJ@?6m_strServerName?5?$DN?5?$AA@ 5f8bc06c     inet.obj
 0002:00011084       ??_7CGopherConnection@@6B@ 5f8bc084     inet.obj
 0002:000110a0       ??_7CHttpConnection@@6B@   5f8bc0a0     inet.obj
 0002:000110b8       ??_C@_1BC@IFNG@?$AAH?$AAT?$AAT?$AAP?$AA?1?$AA1?$AA?4?$AA0?$AA?$AA@ 5f8bc0b8     inet.obj
 0002:000110d0       ??_7CHttpFile@@6B@         5f8bc0d0     inet.obj
 0002:0001113c       ??_C@_0O@GCD@?6m_strVerb?5?$DN?5?$AA@ 5f8bc13c     inet.obj
 0002:0001114c       ??_C@_0BC@KHMN@?6m_strFileName?5?$DN?5?$AA@ 5f8bc14c     inet.obj
 0002:00011164       ??_7CGopherFile@@6B@       5f8bc164     inet.obj
 0002:000111d0       ??_7CFtpFileFind@@6B@      5f8bc1d0     inet.obj
 0002:00011224       ??_C@_15OGLP@?$AA?2?$AA?1?$AA?$AA@ 5f8bc224     inet.obj
 0002:0001122c       ??_C@_13HGEN@?$AA?$CK?$AA?$AA@ 5f8bc22c     inet.obj
 0002:00011230       ??_C@_0O@MBAB@m_hContext?5?$DN?5?$AA@ 5f8bc230     inet.obj
 0002:00011244       ??_7CGopherFileFind@@6B@   5f8bc244     inet.obj
 0002:000112a8       ??_7CGopherLocator@@6B@    5f8bc2a8     inet.obj
 0002:000112bc       ??_C@_1GG@MPDM@?$AAW?$AAa?$AAr?$AAn?$AAi?$AAn?$AAg?$AA?3?$AA?5?$AAt?$AAh?$AAr?$AAo?$AAw?$AAi?$AAn?$AAg?$AA?5?$AAC?$AAI@ 5f8bc2bc     inet.obj
 0002:00011324       ??_C@_1HA@LAJN@?$AAW?$AAa?$AAr?$AAn?$AAi?$AAn?$AAg?$AA?3?$AA?5?$AAE?$AAx?$AAt?$AAe?$AAn?$AAd?$AAe?$AAd?$AA?5?$AAe?$AAr@ 5f8bc324     inet.obj
 0002:00011394       ??_C@_0M@KFA@WININET?4DLL?$AA@ 5f8bc394     inet.obj
 0002:000113a4       ??_7CInternetException@@6B@ 5f8bc3a4     inet.obj
 0002:000113c0       ??_C@_0N@OJLI@m_dwError?5?$DN?5?$AA@ 5f8bc3c0     inet.obj
 0002:000113d4       ??_7CSessionMapPtrToPtr@@6B@ 5f8bc3d4     inet.obj
 0002:000113e8       ?classCFileFind@CFileFind@@2UCRuntimeClass@@B 5f8bc3e8     filefind.obj
 0002:00011400       ??_C@_09CGCC@CFileFind?$AA@ 5f8bc400     filefind.obj
 0002:00011410       ??_7CFileFind@@6B@         5f8bc410     filefind.obj
 0002:00011464       ??_C@_0N@IJHF@filefind?4cpp?$AA@ 5f8bc464     filefind.obj
 0002:00011474       ??_C@_07LDFI@file?3?1?1?$AA@ 5f8bc474     filefind.obj
 0002:0001147c       ??_C@_0P@IDCI@?6m_hContext?5?$DN?5?$AA@ 5f8bc47c     filefind.obj
 0002:000114a0       ?classCDynLinkLibrary@CDynLinkLibrary@@2UCRuntimeClass@@B 5f8bc4a0     dllinit.obj
 0002:000114b8       ??_C@_0BA@FNMJ@CDynLinkLibrary?$AA@ 5f8bc4b8     dllinit.obj
 0002:000114cc       ??_7CDynLinkLibrary@@6B@   5f8bc4cc     dllinit.obj
 0002:00011524       ??_C@_0BI@LMNE@?6module?5name?5is?5unknown?$AA@ 5f8bc524     dllinit.obj
 0002:0001153c       ??_C@_0BA@EJOI@?6module?5name?5?$DN?5?$AA@ 5f8bc53c     dllinit.obj
 0002:0001154c       ??_C@_0BA@EPIG@?6m_hResource?5?$DN?5?$AA@ 5f8bc54c     dllinit.obj
 0002:0001155c       ??_C@_0N@COLJ@m_hModule?5?$DN?5?$AA@ 5f8bc55c     dllinit.obj
 0002:0001156c       ??_C@_0JB@KLFG@This?5application?5or?5DLL?5can?5not?5@ 5f8bc56c     dllinit.obj
 0002:00011600       ??_C@_0BD@CCKL@MFC?5Runtime?5Module?$AA@ 5f8bc600     dllinit.obj
 0002:00011614       ??_C@_0M@LDMD@MSVCRTD?4DLL?$AA@ 5f8bc614     dllinit.obj
 0002:00011624       ??_7type_info@@6B@         5f8bc624     msvcrtd:ti_inst.obj
 0002:00011654       ??_C@_08JKC@crtdll?4c?$AA@ 5f8bc654     msvcrtd:crtdll.obj
 0002:00011660       _IID_IStream               5f8bc660     uuid:objidl_i_guid18.obj
 0002:00011670       _IID_IUnknown              5f8bc670     uuid:unknwn_i_guid0.obj
 0002:00011680       _IID_IClassFactory         5f8bc680     uuid:unknwn_i_guid1.obj
 0002:00011690       _IID_IPersistFile          5f8bc690     uuid:objidl_i_guid21.obj
 0002:000116a0       _IID_IDropTarget           5f8bc6a0     uuid:oleidl_i_guid20.obj
 0002:000116b0       _IID_IDispatch             5f8bc6b0     uuid:oaidl_i_guid4.obj
 0002:000116c0       __sz_ADVAPI32              5f8bc6c0     advapi32:ADVAPI32.dll
 0002:000116d0       __sz_COMCTL32              5f8bc6d0     comctl32:COMCTL32.dll
 0002:000116e0       __sz_SHELL32               5f8bc6e0     shell32:SHELL32.dll
 0002:000116f0       __sz_comdlg32              5f8bc6f0     comdlg32:comdlg32.dll
 0002:00011700       __sz_WINSPOOL              5f8bc700     winspool:WINSPOOL.DRV
 0002:00011710       __sz_WININET               5f8bc710     wininet:WININET.dll
 0002:00011720       ??_R1A@?0A@A@CObject@@8    5f8bc720     except.obj
 0002:00011738       ??_R1A@?0A@A@CException@@8 5f8bc738     except.obj
 0002:00011750       ??_R2CException@@8         5f8bc750     except.obj
 0002:00011760       ??_R3CException@@8         5f8bc760     except.obj
 0002:00011770       ??_R4CException@@6B@       5f8bc770     except.obj
 0002:00011788       ??_R1A@?0A@A@IUnknown@@8   5f8bc788     arcstrm.obj
 0002:000117a0       ??_R1A@?0A@A@ISequentialStream@@8 5f8bc7a0     arcstrm.obj
 0002:000117b8       ??_R1A@?0A@A@IStream@@8    5f8bc7b8     arcstrm.obj
 0002:000117d0       ??_R1A@?0A@A@CArchiveStream@@8 5f8bc7d0     arcstrm.obj
 0002:000117e8       ??_R2CArchiveStream@@8     5f8bc7e8     arcstrm.obj
 0002:00011800       ??_R3CArchiveStream@@8     5f8bc800     arcstrm.obj
 0002:00011810       ??_R4CArchiveStream@@6B@   5f8bc810     arcstrm.obj
 0002:00011828       ??_R1A@?0A@A@CNoTrackObject@@8 5f8bc828     dumpinit.obj
 0002:00011840       ??_R1A@?0A@A@_AFX_DEBUG_STATE@@8 5f8bc840     dumpinit.obj
 0002:00011858       ??_R2_AFX_DEBUG_STATE@@8   5f8bc858     dumpinit.obj
 0002:00011868       ??_R3_AFX_DEBUG_STATE@@8   5f8bc868     dumpinit.obj
 0002:00011878       ??_R4_AFX_DEBUG_STATE@@6B@ 5f8bc878     dumpinit.obj
 0002:0001188c       ??_R2CNoTrackObject@@8     5f8bc88c     dumpinit.obj
 0002:00011898       ??_R3CNoTrackObject@@8     5f8bc898     dumpinit.obj
 0002:000118a8       ??_R4CNoTrackObject@@6B@   5f8bc8a8     dumpinit.obj
 0002:000118bc       ??_R2CObject@@8            5f8bc8bc     afxinl1.obj
 0002:000118c8       ??_R3CObject@@8            5f8bc8c8     afxinl1.obj
 0002:000118d8       ??_R4CObject@@6B@          5f8bc8d8     afxinl1.obj
 0002:000118f0       ??_R1A@?0A@A@CSimpleException@@8 5f8bc8f0     afxinl1.obj
 0002:00011908       ??_R2CSimpleException@@8   5f8bc908     afxinl1.obj
 0002:00011918       ??_R3CSimpleException@@8   5f8bc918     afxinl1.obj
 0002:00011928       ??_R4CSimpleException@@6B@ 5f8bc928     afxinl1.obj
 0002:00011940       ??_R1A@?0A@A@CMemoryException@@8 5f8bc940     afxinl1.obj
 0002:00011958       ??_R2CMemoryException@@8   5f8bc958     afxinl1.obj
 0002:00011970       ??_R3CMemoryException@@8   5f8bc970     afxinl1.obj
 0002:00011980       ??_R4CMemoryException@@6B@ 5f8bc980     afxinl1.obj
 0002:00011998       ??_R1A@?0A@A@CNotSupportedException@@8 5f8bc998     afxinl1.obj
 0002:000119b0       ??_R2CNotSupportedException@@8 5f8bc9b0     afxinl1.obj
 0002:000119c8       ??_R3CNotSupportedException@@8 5f8bc9c8     afxinl1.obj
 0002:000119d8       ??_R4CNotSupportedException@@6B@ 5f8bc9d8     afxinl1.obj
 0002:000119f0       ??_R1A@?0A@A@CArchiveException@@8 5f8bc9f0     afxinl1.obj
 0002:00011a08       ??_R2CArchiveException@@8  5f8bca08     afxinl1.obj
 0002:00011a18       ??_R3CArchiveException@@8  5f8bca18     afxinl1.obj
 0002:00011a28       ??_R4CArchiveException@@6B@ 5f8bca28     afxinl1.obj
 0002:00011a40       ??_R1A@?0A@A@CFileException@@8 5f8bca40     afxinl1.obj
 0002:00011a58       ??_R2CFileException@@8     5f8bca58     afxinl1.obj
 0002:00011a68       ??_R3CFileException@@8     5f8bca68     afxinl1.obj
 0002:00011a78       ??_R4CFileException@@6B@   5f8bca78     afxinl1.obj
 0002:00011a90       ??_R1A@?0A@A@CCmdTarget@@8 5f8bca90     afxinl1.obj
 0002:00011aa8       ??_R1A@?0A@A@CWnd@@8       5f8bcaa8     afxinl1.obj
 0002:00011ac0       ??_R1A@?0A@A@CDialog@@8    5f8bcac0     afxinl1.obj
 0002:00011ad8       ??_R1A@?0A@A@CCommonDialog@@8 5f8bcad8     afxinl1.obj
 0002:00011af0       ??_R2CCommonDialog@@8      5f8bcaf0     afxinl1.obj
 0002:00011b08       ??_R3CCommonDialog@@8      5f8bcb08     afxinl1.obj
 0002:00011b18       ??_R4CCommonDialog@@6B@    5f8bcb18     afxinl1.obj
 0002:00011b30       ??_R1A@?0A@A@CRectTracker@@8 5f8bcb30     afxinl1.obj
 0002:00011b48       ??_R2CRectTracker@@8       5f8bcb48     afxinl1.obj
 0002:00011b50       ??_R3CRectTracker@@8       5f8bcb50     afxinl1.obj
 0002:00011b60       ??_R4CRectTracker@@6B@     5f8bcb60     afxinl1.obj
 0002:00011b78       ??_R1A@?0A@A@CButton@@8    5f8bcb78     afxinl1.obj
 0002:00011b90       ??_R1A@?0A@A@CBitmapButton@@8 5f8bcb90     afxinl1.obj
 0002:00011ba8       ??_R2CBitmapButton@@8      5f8bcba8     afxinl1.obj
 0002:00011bc0       ??_R3CBitmapButton@@8      5f8bcbc0     afxinl1.obj
 0002:00011bd0       ??_R4CBitmapButton@@6B@    5f8bcbd0     afxinl1.obj
 0002:00011be8       ??_R1A@?0A@A@CResourceException@@8 5f8bcbe8     afxinl2.obj
 0002:00011c00       ??_R2CResourceException@@8 5f8bcc00     afxinl2.obj
 0002:00011c18       ??_R3CResourceException@@8 5f8bcc18     afxinl2.obj
 0002:00011c28       ??_R4CResourceException@@6B@ 5f8bcc28     afxinl2.obj
 0002:00011c40       ??_R1A@?0A@A@CUserException@@8 5f8bcc40     afxinl2.obj
 0002:00011c58       ??_R2CUserException@@8     5f8bcc58     afxinl2.obj
 0002:00011c70       ??_R3CUserException@@8     5f8bcc70     afxinl2.obj
 0002:00011c80       ??_R4CUserException@@6B@   5f8bcc80     afxinl2.obj
 0002:00011c98       ??_R1A@?0A@A@CGdiObject@@8 5f8bcc98     afxinl2.obj
 0002:00011cb0       ??_R2CGdiObject@@8         5f8bccb0     afxinl2.obj
 0002:00011cc0       ??_R3CGdiObject@@8         5f8bccc0     afxinl2.obj
 0002:00011cd0       ??_R4CGdiObject@@6B@       5f8bccd0     afxinl2.obj
 0002:00011ce8       ??_R1A@?0A@A@CPen@@8       5f8bcce8     afxinl2.obj
 0002:00011d00       ??_R2CPen@@8               5f8bcd00     afxinl2.obj
 0002:00011d10       ??_R3CPen@@8               5f8bcd10     afxinl2.obj
 0002:00011d20       ??_R4CPen@@6B@             5f8bcd20     afxinl2.obj
 0002:00011d38       ??_R1A@?0A@A@CBrush@@8     5f8bcd38     afxinl2.obj
 0002:00011d50       ??_R2CBrush@@8             5f8bcd50     afxinl2.obj
 0002:00011d60       ??_R3CBrush@@8             5f8bcd60     afxinl2.obj
 0002:00011d70       ??_R4CBrush@@6B@           5f8bcd70     afxinl2.obj
 0002:00011d88       ??_R1A@?0A@A@CFont@@8      5f8bcd88     afxinl2.obj
 0002:00011da0       ??_R2CFont@@8              5f8bcda0     afxinl2.obj
 0002:00011db0       ??_R3CFont@@8              5f8bcdb0     afxinl2.obj
 0002:00011dc0       ??_R4CFont@@6B@            5f8bcdc0     afxinl2.obj
 0002:00011dd8       ??_R1A@?0A@A@CBitmap@@8    5f8bcdd8     afxinl2.obj
 0002:00011df0       ??_R2CBitmap@@8            5f8bcdf0     afxinl2.obj
 0002:00011e00       ??_R3CBitmap@@8            5f8bce00     afxinl2.obj
 0002:00011e10       ??_R4CBitmap@@6B@          5f8bce10     afxinl2.obj
 0002:00011e28       ??_R1A@?0A@A@CPalette@@8   5f8bce28     afxinl2.obj
 0002:00011e40       ??_R2CPalette@@8           5f8bce40     afxinl2.obj
 0002:00011e50       ??_R3CPalette@@8           5f8bce50     afxinl2.obj
 0002:00011e60       ??_R4CPalette@@6B@         5f8bce60     afxinl2.obj
 0002:00011e78       ??_R1A@?0A@A@CRgn@@8       5f8bce78     afxinl2.obj
 0002:00011e90       ??_R2CRgn@@8               5f8bce90     afxinl2.obj
 0002:00011ea0       ??_R3CRgn@@8               5f8bcea0     afxinl2.obj
 0002:00011eb0       ??_R4CRgn@@6B@             5f8bceb0     afxinl2.obj
 0002:00011ec8       ??_R1A@?0A@A@CMenu@@8      5f8bcec8     afxinl2.obj
 0002:00011ee0       ??_R2CMenu@@8              5f8bcee0     afxinl2.obj
 0002:00011ef0       ??_R3CMenu@@8              5f8bcef0     afxinl2.obj
 0002:00011f00       ??_R4CMenu@@6B@            5f8bcf00     afxinl2.obj
 0002:00011f18       ??_R1A@?0A@A@CStatic@@8    5f8bcf18     afxinl3.obj
 0002:00011f30       ??_R2CStatic@@8            5f8bcf30     afxinl3.obj
 0002:00011f48       ??_R3CStatic@@8            5f8bcf48     afxinl3.obj
 0002:00011f58       ??_R4CStatic@@6B@          5f8bcf58     afxinl3.obj
 0002:00011f70       ??_R2CButton@@8            5f8bcf70     afxinl3.obj
 0002:00011f88       ??_R3CButton@@8            5f8bcf88     afxinl3.obj
 0002:00011f98       ??_R4CButton@@6B@          5f8bcf98     afxinl3.obj
 0002:00011fb0       ??_R1A@?0A@A@CListBox@@8   5f8bcfb0     afxinl3.obj
 0002:00011fc8       ??_R2CListBox@@8           5f8bcfc8     afxinl3.obj
 0002:00011fe0       ??_R3CListBox@@8           5f8bcfe0     afxinl3.obj
 0002:00011ff0       ??_R4CListBox@@6B@         5f8bcff0     afxinl3.obj
 0002:00012008       ??_R1A@?0A@A@CCheckListBox@@8 5f8bd008     afxinl3.obj
 0002:00012020       ??_R2CCheckListBox@@8      5f8bd020     afxinl3.obj
 0002:00012038       ??_R3CCheckListBox@@8      5f8bd038     afxinl3.obj
 0002:00012048       ??_R4CCheckListBox@@6B@    5f8bd048     afxinl3.obj
 0002:00012060       ??_R1A@?0A@A@CComboBox@@8  5f8bd060     afxinl3.obj
 0002:00012078       ??_R2CComboBox@@8          5f8bd078     afxinl3.obj
 0002:00012090       ??_R3CComboBox@@8          5f8bd090     afxinl3.obj
 0002:000120a0       ??_R4CComboBox@@6B@        5f8bd0a0     afxinl3.obj
 0002:000120b8       ??_R1A@?0A@A@CEdit@@8      5f8bd0b8     afxinl3.obj
 0002:000120d0       ??_R2CEdit@@8              5f8bd0d0     afxinl3.obj
 0002:000120e8       ??_R3CEdit@@8              5f8bd0e8     afxinl3.obj
 0002:000120f8       ??_R4CEdit@@6B@            5f8bd0f8     afxinl3.obj
 0002:00012110       ??_R1A@?0A@A@CScrollBar@@8 5f8bd110     afxinl3.obj
 0002:00012128       ??_R2CScrollBar@@8         5f8bd128     afxinl3.obj
 0002:00012140       ??_R3CScrollBar@@8         5f8bd140     afxinl3.obj
 0002:00012150       ??_R4CScrollBar@@6B@       5f8bd150     afxinl3.obj
 0002:00012168       ??_R1A@?0A@A@CFile@@8      5f8bd168     filecore.obj
 0002:00012180       ??_R2CFile@@8              5f8bd180     filecore.obj
 0002:00012190       ??_R3CFile@@8              5f8bd190     filecore.obj
 0002:000121a0       ??_R4CFile@@6B@            5f8bd1a0     filecore.obj
 0002:000121b8       ??_R1A@?0A@A@CStdioFile@@8 5f8bd1b8     filetxt.obj
 0002:000121d0       ??_R2CStdioFile@@8         5f8bd1d0     filetxt.obj
 0002:000121e0       ??_R3CStdioFile@@8         5f8bd1e0     filetxt.obj
 0002:000121f0       ??_R4CStdioFile@@6B@       5f8bd1f0     filetxt.obj
 0002:00012208       ??_R1A@?0A@A@CMemFile@@8   5f8bd208     filemem.obj
 0002:00012220       ??_R2CMemFile@@8           5f8bd220     filemem.obj
 0002:00012230       ??_R3CMemFile@@8           5f8bd230     filemem.obj
 0002:00012240       ??_R4CMemFile@@6B@         5f8bd240     filemem.obj
 0002:00012258       ??_R1A@?0A@A@CSharedFile@@8 5f8bd258     fileshrd.obj
 0002:00012270       ??_R2CSharedFile@@8        5f8bd270     fileshrd.obj
 0002:00012288       ??_R3CSharedFile@@8        5f8bd288     fileshrd.obj
 0002:00012298       ??_R4CSharedFile@@6B@      5f8bd298     fileshrd.obj
 0002:000122b0       ??_R1A@?0A@A@CByteArray@@8 5f8bd2b0     array_b.obj
 0002:000122c8       ??_R2CByteArray@@8         5f8bd2c8     array_b.obj
 0002:000122d8       ??_R3CByteArray@@8         5f8bd2d8     array_b.obj
 0002:000122e8       ??_R4CByteArray@@6B@       5f8bd2e8     array_b.obj
 0002:00012300       ??_R1A@?0A@A@CDWordArray@@8 5f8bd300     array_d.obj
 0002:00012318       ??_R2CDWordArray@@8        5f8bd318     array_d.obj
 0002:00012328       ??_R3CDWordArray@@8        5f8bd328     array_d.obj
 0002:00012338       ??_R4CDWordArray@@6B@      5f8bd338     array_d.obj
 0002:00012350       ??_R1A@?0A@A@CPtrArray@@8  5f8bd350     array_p.obj
 0002:00012368       ??_R2CPtrArray@@8          5f8bd368     array_p.obj
 0002:00012378       ??_R3CPtrArray@@8          5f8bd378     array_p.obj
 0002:00012388       ??_R4CPtrArray@@6B@        5f8bd388     array_p.obj
 0002:000123a0       ??_R1A@?0A@A@CObArray@@8   5f8bd3a0     array_o.obj
 0002:000123b8       ??_R2CObArray@@8           5f8bd3b8     array_o.obj
 0002:000123c8       ??_R3CObArray@@8           5f8bd3c8     array_o.obj
 0002:000123d8       ??_R4CObArray@@6B@         5f8bd3d8     array_o.obj
 0002:000123f0       ??_R1A@?0A@A@CStringArray@@8 5f8bd3f0     array_s.obj
 0002:00012408       ??_R2CStringArray@@8       5f8bd408     array_s.obj
 0002:00012418       ??_R3CStringArray@@8       5f8bd418     array_s.obj
 0002:00012428       ??_R4CStringArray@@6B@     5f8bd428     array_s.obj
 0002:00012440       ??_R1A@?0A@A@CUIntArray@@8 5f8bd440     array_u.obj
 0002:00012458       ??_R2CUIntArray@@8         5f8bd458     array_u.obj
 0002:00012468       ??_R3CUIntArray@@8         5f8bd468     array_u.obj
 0002:00012478       ??_R4CUIntArray@@6B@       5f8bd478     array_u.obj
 0002:00012490       ??_R1A@?0A@A@CWordArray@@8 5f8bd490     array_w.obj
 0002:000124a8       ??_R2CWordArray@@8         5f8bd4a8     array_w.obj
 0002:000124b8       ??_R3CWordArray@@8         5f8bd4b8     array_w.obj
 0002:000124c8       ??_R4CWordArray@@6B@       5f8bd4c8     array_w.obj
 0002:000124e0       ??_R1A@?0A@A@CObList@@8    5f8bd4e0     list_o.obj
 0002:000124f8       ??_R2CObList@@8            5f8bd4f8     list_o.obj
 0002:00012508       ??_R3CObList@@8            5f8bd508     list_o.obj
 0002:00012518       ??_R4CObList@@6B@          5f8bd518     list_o.obj
 0002:00012530       ??_R1A@?0A@A@CPtrList@@8   5f8bd530     list_p.obj
 0002:00012548       ??_R2CPtrList@@8           5f8bd548     list_p.obj
 0002:00012558       ??_R3CPtrList@@8           5f8bd558     list_p.obj
 0002:00012568       ??_R4CPtrList@@6B@         5f8bd568     list_p.obj
 0002:00012580       ??_R1A@?0A@A@CStringList@@8 5f8bd580     list_s.obj
 0002:00012598       ??_R2CStringList@@8        5f8bd598     list_s.obj
 0002:000125a8       ??_R3CStringList@@8        5f8bd5a8     list_s.obj
 0002:000125b8       ??_R4CStringList@@6B@      5f8bd5b8     list_s.obj
 0002:000125d0       ??_R1A@?0A@A@CMapPtrToPtr@@8 5f8bd5d0     map_pp.obj
 0002:000125e8       ??_R2CMapPtrToPtr@@8       5f8bd5e8     map_pp.obj
 0002:000125f8       ??_R3CMapPtrToPtr@@8       5f8bd5f8     map_pp.obj
 0002:00012608       ??_R4CMapPtrToPtr@@6B@     5f8bd608     map_pp.obj
 0002:00012620       ??_R1A@?0A@A@CMapPtrToWord@@8 5f8bd620     map_pw.obj
 0002:00012638       ??_R2CMapPtrToWord@@8      5f8bd638     map_pw.obj
 0002:00012648       ??_R3CMapPtrToWord@@8      5f8bd648     map_pw.obj
 0002:00012658       ??_R4CMapPtrToWord@@6B@    5f8bd658     map_pw.obj
 0002:00012670       ??_R1A@?0A@A@CMapStringToOb@@8 5f8bd670     map_so.obj
 0002:00012688       ??_R2CMapStringToOb@@8     5f8bd688     map_so.obj
 0002:00012698       ??_R3CMapStringToOb@@8     5f8bd698     map_so.obj
 0002:000126a8       ??_R4CMapStringToOb@@6B@   5f8bd6a8     map_so.obj
 0002:000126c0       ??_R1A@?0A@A@CMapStringToPtr@@8 5f8bd6c0     map_sp.obj
 0002:000126d8       ??_R2CMapStringToPtr@@8    5f8bd6d8     map_sp.obj
 0002:000126e8       ??_R3CMapStringToPtr@@8    5f8bd6e8     map_sp.obj
 0002:000126f8       ??_R4CMapStringToPtr@@6B@  5f8bd6f8     map_sp.obj
 0002:00012710       ??_R1A@?0A@A@CMapStringToString@@8 5f8bd710     map_ss.obj
 0002:00012728       ??_R2CMapStringToString@@8 5f8bd728     map_ss.obj
 0002:00012738       ??_R3CMapStringToString@@8 5f8bd738     map_ss.obj
 0002:00012748       ??_R4CMapStringToString@@6B@ 5f8bd748     map_ss.obj
 0002:00012760       ??_R1A@?0A@A@CMapWordToOb@@8 5f8bd760     map_wo.obj
 0002:00012778       ??_R2CMapWordToOb@@8       5f8bd778     map_wo.obj
 0002:00012788       ??_R3CMapWordToOb@@8       5f8bd788     map_wo.obj
 0002:00012798       ??_R4CMapWordToOb@@6B@     5f8bd798     map_wo.obj
 0002:000127b0       ??_R1A@?0A@A@CMapWordToPtr@@8 5f8bd7b0     map_wp.obj
 0002:000127c8       ??_R2CMapWordToPtr@@8      5f8bd7c8     map_wp.obj
 0002:000127d8       ??_R3CMapWordToPtr@@8      5f8bd7d8     map_wp.obj
 0002:000127e8       ??_R4CMapWordToPtr@@6B@    5f8bd7e8     map_wp.obj
 0002:00012800       ??_R1A@?0A@A@_AFX_THREAD_STATE@@8 5f8bd800     afxstate.obj
 0002:00012818       ??_R2_AFX_THREAD_STATE@@8  5f8bd818     afxstate.obj
 0002:00012828       ??_R3_AFX_THREAD_STATE@@8  5f8bd828     afxstate.obj
 0002:00012838       ??_R4_AFX_THREAD_STATE@@6B@ 5f8bd838     afxstate.obj
 0002:00012850       ??_R1A@?0A@A@AFX_MODULE_STATE@@8 5f8bd850     afxstate.obj
 0002:00012868       ??_R2AFX_MODULE_STATE@@8   5f8bd868     afxstate.obj
 0002:00012878       ??_R3AFX_MODULE_STATE@@8   5f8bd878     afxstate.obj
 0002:00012888       ??_R4AFX_MODULE_STATE@@6B@ 5f8bd888     afxstate.obj
 0002:000128a0       ??_R1A@?0A@A@AFX_MODULE_THREAD_STATE@@8 5f8bd8a0     afxstate.obj
 0002:000128b8       ??_R2AFX_MODULE_THREAD_STATE@@8 5f8bd8b8     afxstate.obj
 0002:000128c8       ??_R3AFX_MODULE_THREAD_STATE@@8 5f8bd8c8     afxstate.obj
 0002:000128d8       ??_R4AFX_MODULE_THREAD_STATE@@6B@ 5f8bd8d8     afxstate.obj
 0002:000128f0       ??_R1A@?0A@A@_AFX_BASE_MODULE_STATE@@8 5f8bd8f0     afxstate.obj
 0002:00012908       ??_R2_AFX_BASE_MODULE_STATE@@8 5f8bd908     afxstate.obj
 0002:00012918       ??_R3_AFX_BASE_MODULE_STATE@@8 5f8bd918     afxstate.obj
 0002:00012928       ??_R4_AFX_BASE_MODULE_STATE@@6B@ 5f8bd928     afxstate.obj
 0002:00012940       ??_R1A@?0A@A@CThreadData@@8 5f8bd940     afxtls.obj
 0002:00012958       ??_R2CThreadData@@8        5f8bd958     afxtls.obj
 0002:00012968       ??_R3CThreadData@@8        5f8bd968     afxtls.obj
 0002:00012978       ??_R4CThreadData@@6B@      5f8bd978     afxtls.obj
 0002:00012990       ??_R1A@?0A@A@CSyncObject@@8 5f8bd990     mtcore.obj
 0002:000129a8       ??_R2CSyncObject@@8        5f8bd9a8     mtcore.obj
 0002:000129b8       ??_R3CSyncObject@@8        5f8bd9b8     mtcore.obj
 0002:000129c8       ??_R4CSyncObject@@6B@      5f8bd9c8     mtcore.obj
 0002:000129e0       ??_R1A@?0A@A@CCriticalSection@@8 5f8bd9e0     mtcore.obj
 0002:000129f8       ??_R2CCriticalSection@@8   5f8bd9f8     mtcore.obj
 0002:00012a08       ??_R3CCriticalSection@@8   5f8bda08     mtcore.obj
 0002:00012a18       ??_R4CCriticalSection@@6B@ 5f8bda18     mtcore.obj
 0002:00012a30       ??_R1A@?0A@A@CSemaphore@@8 5f8bda30     mtex.obj
 0002:00012a48       ??_R2CSemaphore@@8         5f8bda48     mtex.obj
 0002:00012a58       ??_R3CSemaphore@@8         5f8bda58     mtex.obj
 0002:00012a68       ??_R4CSemaphore@@6B@       5f8bda68     mtex.obj
 0002:00012a80       ??_R1A@?0A@A@CMutex@@8     5f8bda80     mtex.obj
 0002:00012a98       ??_R2CMutex@@8             5f8bda98     mtex.obj
 0002:00012aa8       ??_R3CMutex@@8             5f8bdaa8     mtex.obj
 0002:00012ab8       ??_R4CMutex@@6B@           5f8bdab8     mtex.obj
 0002:00012ad0       ??_R1A@?0A@A@CEvent@@8     5f8bdad0     mtex.obj
 0002:00012ae8       ??_R2CEvent@@8             5f8bdae8     mtex.obj
 0002:00012af8       ??_R3CEvent@@8             5f8bdaf8     mtex.obj
 0002:00012b08       ??_R4CEvent@@6B@           5f8bdb08     mtex.obj
 0002:00012b20       ??_R2CWnd@@8               5f8bdb20     wincore.obj
 0002:00012b30       ??_R3CWnd@@8               5f8bdb30     wincore.obj
 0002:00012b40       ??_R4CWnd@@6B@             5f8bdb40     wincore.obj
 0002:00012b58       ??_R1A@?0A@A@CCmdUI@@8     5f8bdb58     wincore.obj
 0002:00012b70       ??_R1A@?0A@A@CTestCmdUI@@8 5f8bdb70     wincore.obj
 0002:00012b88       ??_R2CTestCmdUI@@8         5f8bdb88     wincore.obj
 0002:00012b98       ??_R3CTestCmdUI@@8         5f8bdb98     wincore.obj
 0002:00012ba8       ??_R4CTestCmdUI@@6B@       5f8bdba8     wincore.obj
 0002:00012bc0       ??_R1A@?0A@A@CTempWnd@@8   5f8bdbc0     wincore.obj
 0002:00012bd8       ??_R2CTempWnd@@8           5f8bdbd8     wincore.obj
 0002:00012bf0       ??_R3CTempWnd@@8           5f8bdbf0     wincore.obj
 0002:00012c00       ??_R4CTempWnd@@6B@         5f8bdc00     wincore.obj
 0002:00012c18       ??_R1A@?0A@A@_AFX_CTL3D_STATE@@8 5f8bdc18     wincore.obj
 0002:00012c30       ??_R2_AFX_CTL3D_STATE@@8   5f8bdc30     wincore.obj
 0002:00012c40       ??_R3_AFX_CTL3D_STATE@@8   5f8bdc40     wincore.obj
 0002:00012c50       ??_R4_AFX_CTL3D_STATE@@6B@ 5f8bdc50     wincore.obj
 0002:00012c68       ??_R1A@?0A@A@CFrameWnd@@8  5f8bdc68     winfrm.obj
 0002:00012c80       ??_R2CFrameWnd@@8          5f8bdc80     winfrm.obj
 0002:00012c98       ??_R3CFrameWnd@@8          5f8bdc98     winfrm.obj
 0002:00012ca8       ??_R4CFrameWnd@@6B@        5f8bdca8     winfrm.obj
 0002:00012cc0       ??_R1A@?0A@A@CMDIFrameWnd@@8 5f8bdcc0     winmdi.obj
 0002:00012cd8       ??_R2CMDIFrameWnd@@8       5f8bdcd8     winmdi.obj
 0002:00012cf0       ??_R3CMDIFrameWnd@@8       5f8bdcf0     winmdi.obj
 0002:00012d00       ??_R4CMDIFrameWnd@@6B@     5f8bdd00     winmdi.obj
 0002:00012d18       ??_R1A@?0A@A@CMDIChildWnd@@8 5f8bdd18     winmdi.obj
 0002:00012d30       ??_R2CMDIChildWnd@@8       5f8bdd30     winmdi.obj
 0002:00012d48       ??_R3CMDIChildWnd@@8       5f8bdd48     winmdi.obj
 0002:00012d58       ??_R4CMDIChildWnd@@6B@     5f8bdd58     winmdi.obj
 0002:00012d70       ??_R1A@?0A@A@CToolTipCtrl@@8 5f8bdd70     tooltip.obj
 0002:00012d88       ??_R2CToolTipCtrl@@8       5f8bdd88     tooltip.obj
 0002:00012da0       ??_R3CToolTipCtrl@@8       5f8bdda0     tooltip.obj
 0002:00012db0       ??_R4CToolTipCtrl@@6B@     5f8bddb0     tooltip.obj
 0002:00012dc8       ??_R1A@?0A@A@CMiniFrameWnd@@8 5f8bddc8     winmini.obj
 0002:00012de0       ??_R2CMiniFrameWnd@@8      5f8bdde0     winmini.obj
 0002:00012df8       ??_R3CMiniFrameWnd@@8      5f8bddf8     winmini.obj
 0002:00012e08       ??_R4CMiniFrameWnd@@6B@    5f8bde08     winmini.obj
 0002:00012e20       ??_R1A@?0A@A@CControlBar@@8 5f8bde20     barcore.obj
 0002:00012e38       ??_R2CControlBar@@8        5f8bde38     barcore.obj
 0002:00012e50       ??_R3CControlBar@@8        5f8bde50     barcore.obj
 0002:00012e60       ??_R4CControlBar@@6B@      5f8bde60     barcore.obj
 0002:00012e78       ??_R1A@?0A@A@CToolBar@@8   5f8bde78     bartool.obj
 0002:00012e90       ??_R2CToolBar@@8           5f8bde90     bartool.obj
 0002:00012ea8       ??_R3CToolBar@@8           5f8bdea8     bartool.obj
 0002:00012eb8       ??_R4CToolBar@@6B@         5f8bdeb8     bartool.obj
 0002:00012ed0       ??_R1A@?0A@A@CToolCmdUI@@8 5f8bded0     bartool.obj
 0002:00012ee8       ??_R2CToolCmdUI@@8         5f8bdee8     bartool.obj
 0002:00012ef8       ??_R3CToolCmdUI@@8         5f8bdef8     bartool.obj
 0002:00012f08       ??_R4CToolCmdUI@@6B@       5f8bdf08     bartool.obj
 0002:00012f20       ??_R1A@?0A@A@CDialogBar@@8 5f8bdf20     bardlg.obj
 0002:00012f38       ??_R2CDialogBar@@8         5f8bdf38     bardlg.obj
 0002:00012f50       ??_R3CDialogBar@@8         5f8bdf50     bardlg.obj
 0002:00012f60       ??_R4CDialogBar@@6B@       5f8bdf60     bardlg.obj
 0002:00012f78       ??_R1A@?0A@A@CStatusBar@@8 5f8bdf78     barstat.obj
 0002:00012f90       ??_R2CStatusBar@@8         5f8bdf90     barstat.obj
 0002:00012fa8       ??_R3CStatusBar@@8         5f8bdfa8     barstat.obj
 0002:00012fb8       ??_R4CStatusBar@@6B@       5f8bdfb8     barstat.obj
 0002:00012fd0       ??_R1A@?0A@A@CStatusCmdUI@@8 5f8bdfd0     barstat.obj
 0002:00012fe8       ??_R2CStatusCmdUI@@8       5f8bdfe8     barstat.obj
 0002:00012ff8       ??_R3CStatusCmdUI@@8       5f8bdff8     barstat.obj
 0002:00013008       ??_R4CStatusCmdUI@@6B@     5f8be008     barstat.obj
 0002:00013020       ??_R1A@?0A@A@CDockBar@@8   5f8be020     bardock.obj
 0002:00013038       ??_R2CDockBar@@8           5f8be038     bardock.obj
 0002:00013050       ??_R3CDockBar@@8           5f8be050     bardock.obj
 0002:00013060       ??_R4CDockBar@@6B@         5f8be060     bardock.obj
 0002:00013078       ??_R1A@?0A@A@CMiniDockFrameWnd@@8 5f8be078     bardock.obj
 0002:00013090       ??_R2CMiniDockFrameWnd@@8  5f8be090     bardock.obj
 0002:000130b0       ??_R3CMiniDockFrameWnd@@8  5f8be0b0     bardock.obj
 0002:000130c0       ??_R4CMiniDockFrameWnd@@6B@ 5f8be0c0     bardock.obj
 0002:000130d8       ??_R1A@?0A@A@CDockContext@@8 5f8be0d8     dockcont.obj
 0002:000130f0       ??_R2CDockContext@@8       5f8be0f0     dockcont.obj
 0002:000130f8       ??_R3CDockContext@@8       5f8be0f8     dockcont.obj
 0002:00013108       ??_R4CDockContext@@6B@     5f8be108     dockcont.obj
 0002:00013120       ??_R1A@?0A@A@CDockState@@8 5f8be120     dockstat.obj
 0002:00013138       ??_R2CDockState@@8         5f8be138     dockstat.obj
 0002:00013148       ??_R3CDockState@@8         5f8be148     dockstat.obj
 0002:00013158       ??_R4CDockState@@6B@       5f8be158     dockstat.obj
 0002:00013170       ??_R1A@?0A@A@CDC@@8        5f8be170     dcprev.obj
 0002:00013188       ??_R1A@?0A@A@CPreviewDC@@8 5f8be188     dcprev.obj
 0002:000131a0       ??_R2CPreviewDC@@8         5f8be1a0     dcprev.obj
 0002:000131b0       ??_R3CPreviewDC@@8         5f8be1b0     dcprev.obj
 0002:000131c0       ??_R4CPreviewDC@@6B@       5f8be1c0     dcprev.obj
 0002:000131d8       ??_R1A@?0A@A@CMetaFileDC@@8 5f8be1d8     dcmeta.obj
 0002:000131f0       ??_R2CMetaFileDC@@8        5f8be1f0     dcmeta.obj
 0002:00013200       ??_R3CMetaFileDC@@8        5f8be200     dcmeta.obj
 0002:00013210       ??_R4CMetaFileDC@@6B@      5f8be210     dcmeta.obj
 0002:00013228       ??_R1A@?0A@A@CReBar@@8     5f8be228     barcool.obj
 0002:00013240       ??_R2CReBar@@8             5f8be240     barcool.obj
 0002:00013258       ??_R3CReBar@@8             5f8be258     barcool.obj
 0002:00013268       ??_R4CReBar@@6B@           5f8be268     barcool.obj
 0002:00013280       ??_R1A@?0A@A@CDragListBox@@8 5f8be280     winctrl2.obj
 0002:00013298       ??_R2CDragListBox@@8       5f8be298     winctrl2.obj
 0002:000132b0       ??_R3CDragListBox@@8       5f8be2b0     winctrl2.obj
 0002:000132c0       ??_R4CDragListBox@@6B@     5f8be2c0     winctrl2.obj
 0002:000132d8       ??_R1A@?0A@A@CToolBarCtrl@@8 5f8be2d8     winctrl2.obj
 0002:000132f0       ??_R2CToolBarCtrl@@8       5f8be2f0     winctrl2.obj
 0002:00013308       ??_R3CToolBarCtrl@@8       5f8be308     winctrl2.obj
 0002:00013318       ??_R4CToolBarCtrl@@6B@     5f8be318     winctrl2.obj
 0002:00013330       ??_R1A@?0A@A@CStatusBarCtrl@@8 5f8be330     winctrl2.obj
 0002:00013348       ??_R2CStatusBarCtrl@@8     5f8be348     winctrl2.obj
 0002:00013360       ??_R3CStatusBarCtrl@@8     5f8be360     winctrl2.obj
 0002:00013370       ??_R4CStatusBarCtrl@@6B@   5f8be370     winctrl2.obj
 0002:00013388       ??_R1A@?0A@A@CListCtrl@@8  5f8be388     winctrl2.obj
 0002:000133a0       ??_R2CListCtrl@@8          5f8be3a0     winctrl2.obj
 0002:000133b8       ??_R3CListCtrl@@8          5f8be3b8     winctrl2.obj
 0002:000133c8       ??_R4CListCtrl@@6B@        5f8be3c8     winctrl2.obj
 0002:000133e0       ??_R1A@?0A@A@CTreeCtrl@@8  5f8be3e0     winctrl2.obj
 0002:000133f8       ??_R2CTreeCtrl@@8          5f8be3f8     winctrl2.obj
 0002:00013410       ??_R3CTreeCtrl@@8          5f8be410     winctrl2.obj
 0002:00013420       ??_R4CTreeCtrl@@6B@        5f8be420     winctrl2.obj
 0002:00013438       ??_R1A@?0A@A@CSpinButtonCtrl@@8 5f8be438     winctrl2.obj
 0002:00013450       ??_R2CSpinButtonCtrl@@8    5f8be450     winctrl2.obj
 0002:00013468       ??_R3CSpinButtonCtrl@@8    5f8be468     winctrl2.obj
 0002:00013478       ??_R4CSpinButtonCtrl@@6B@  5f8be478     winctrl2.obj
 0002:00013490       ??_R1A@?0A@A@CSliderCtrl@@8 5f8be490     winctrl2.obj
 0002:000134a8       ??_R2CSliderCtrl@@8        5f8be4a8     winctrl2.obj
 0002:000134c0       ??_R3CSliderCtrl@@8        5f8be4c0     winctrl2.obj
 0002:000134d0       ??_R4CSliderCtrl@@6B@      5f8be4d0     winctrl2.obj
 0002:000134e8       ??_R1A@?0A@A@CProgressCtrl@@8 5f8be4e8     winctrl2.obj
 0002:00013500       ??_R2CProgressCtrl@@8      5f8be500     winctrl2.obj
 0002:00013518       ??_R3CProgressCtrl@@8      5f8be518     winctrl2.obj
 0002:00013528       ??_R4CProgressCtrl@@6B@    5f8be528     winctrl2.obj
 0002:00013540       ??_R1A@?0A@A@CHeaderCtrl@@8 5f8be540     winctrl2.obj
 0002:00013558       ??_R2CHeaderCtrl@@8        5f8be558     winctrl2.obj
 0002:00013570       ??_R3CHeaderCtrl@@8        5f8be570     winctrl2.obj
 0002:00013580       ??_R4CHeaderCtrl@@6B@      5f8be580     winctrl2.obj
 0002:00013598       ??_R1A@?0A@A@CHotKeyCtrl@@8 5f8be598     winctrl2.obj
 0002:000135b0       ??_R2CHotKeyCtrl@@8        5f8be5b0     winctrl2.obj
 0002:000135c8       ??_R3CHotKeyCtrl@@8        5f8be5c8     winctrl2.obj
 0002:000135d8       ??_R4CHotKeyCtrl@@6B@      5f8be5d8     winctrl2.obj
 0002:000135f0       ??_R1A@?0A@A@CTabCtrl@@8   5f8be5f0     winctrl2.obj
 0002:00013608       ??_R2CTabCtrl@@8           5f8be608     winctrl2.obj
 0002:00013620       ??_R3CTabCtrl@@8           5f8be620     winctrl2.obj
 0002:00013630       ??_R4CTabCtrl@@6B@         5f8be630     winctrl2.obj
 0002:00013648       ??_R1A@?0A@A@CAnimateCtrl@@8 5f8be648     winctrl2.obj
 0002:00013660       ??_R2CAnimateCtrl@@8       5f8be660     winctrl2.obj
 0002:00013678       ??_R3CAnimateCtrl@@8       5f8be678     winctrl2.obj
 0002:00013688       ??_R4CAnimateCtrl@@6B@     5f8be688     winctrl2.obj
 0002:000136a0       ??_R1A@?0A@A@CRichEditCtrl@@8 5f8be6a0     winctrl2.obj
 0002:000136b8       ??_R2CRichEditCtrl@@8      5f8be6b8     winctrl2.obj
 0002:000136d0       ??_R3CRichEditCtrl@@8      5f8be6d0     winctrl2.obj
 0002:000136e0       ??_R4CRichEditCtrl@@6B@    5f8be6e0     winctrl2.obj
 0002:000136f8       ??_R1A@?0A@A@CImageList@@8 5f8be6f8     winctrl2.obj
 0002:00013710       ??_R2CImageList@@8         5f8be710     winctrl2.obj
 0002:00013720       ??_R3CImageList@@8         5f8be720     winctrl2.obj
 0002:00013730       ??_R4CImageList@@6B@       5f8be730     winctrl2.obj
 0002:00013748       ??_R1A@?0A@A@CTempImageList@@8 5f8be748     winctrl2.obj
 0002:00013760       ??_R2CTempImageList@@8     5f8be760     winctrl2.obj
 0002:00013770       ??_R3CTempImageList@@8     5f8be770     winctrl2.obj
 0002:00013780       ??_R4CTempImageList@@6B@   5f8be780     winctrl2.obj
 0002:00013798       ??_R1A@?0A@A@_AFX_CHECKLIST_STATE@@8 5f8be798     winctrl3.obj
 0002:000137b0       ??_R2_AFX_CHECKLIST_STATE@@8 5f8be7b0     winctrl3.obj
 0002:000137c0       ??_R3_AFX_CHECKLIST_STATE@@8 5f8be7c0     winctrl3.obj
 0002:000137d0       ??_R4_AFX_CHECKLIST_STATE@@6B@ 5f8be7d0     winctrl3.obj
 0002:000137e8       ??_R1A@?0A@A@_AFX_EDIT_STATE@@8 5f8be7e8     winctrl4.obj
 0002:00013800       ??_R1A@?0A@A@_AFX_RICHEDIT_STATE@@8 5f8be800     winctrl4.obj
 0002:00013818       ??_R2_AFX_RICHEDIT_STATE@@8 5f8be818     winctrl4.obj
 0002:00013828       ??_R3_AFX_RICHEDIT_STATE@@8 5f8be828     winctrl4.obj
 0002:00013838       ??_R4_AFX_RICHEDIT_STATE@@6B@ 5f8be838     winctrl4.obj
 0002:00013850       ??_R2CDialog@@8            5f8be850     dlgcore.obj
 0002:00013868       ??_R3CDialog@@8            5f8be868     dlgcore.obj
 0002:00013878       ??_R4CDialog@@6B@          5f8be878     dlgcore.obj
 0002:00013890       ??_R1A@?0A@A@CPropertyPage@@8 5f8be890     dlgprop.obj
 0002:000138a8       ??_R2CPropertyPage@@8      5f8be8a8     dlgprop.obj
 0002:000138c0       ??_R3CPropertyPage@@8      5f8be8c0     dlgprop.obj
 0002:000138d0       ??_R4CPropertyPage@@6B@    5f8be8d0     dlgprop.obj
 0002:000138e8       ??_R1A@?0A@A@CPropertySheet@@8 5f8be8e8     dlgprop.obj
 0002:00013900       ??_R2CPropertySheet@@8     5f8be900     dlgprop.obj
 0002:00013918       ??_R3CPropertySheet@@8     5f8be918     dlgprop.obj
 0002:00013928       ??_R4CPropertySheet@@6B@   5f8be928     dlgprop.obj
 0002:00013940       ??_R1A@?0A@A@CPropertyPageEx@@8 5f8be940     dlgprop.obj
 0002:00013958       ??_R2CPropertyPageEx@@8    5f8be958     dlgprop.obj
 0002:00013978       ??_R3CPropertyPageEx@@8    5f8be978     dlgprop.obj
 0002:00013988       ??_R4CPropertyPageEx@@6B@  5f8be988     dlgprop.obj
 0002:000139a0       ??_R1A@?0A@A@CPropertySheetEx@@8 5f8be9a0     dlgprop.obj
 0002:000139b8       ??_R2CPropertySheetEx@@8   5f8be9b8     dlgprop.obj
 0002:000139d0       ??_R3CPropertySheetEx@@8   5f8be9d0     dlgprop.obj
 0002:000139e0       ??_R4CPropertySheetEx@@6B@ 5f8be9e0     dlgprop.obj
 0002:000139f8       ??_R1A@?0A@A@CFileDialog@@8 5f8be9f8     dlgfile.obj
 0002:00013a10       ??_R2CFileDialog@@8        5f8bea10     dlgfile.obj
 0002:00013a30       ??_R3CFileDialog@@8        5f8bea30     dlgfile.obj
 0002:00013a40       ??_R4CFileDialog@@6B@      5f8bea40     dlgfile.obj
 0002:00013a58       ??_R1A@?0A@A@CPageSetupDialog@@8 5f8bea58     dlgprnt.obj
 0002:00013a70       ??_R2CPageSetupDialog@@8   5f8bea70     dlgprnt.obj
 0002:00013a90       ??_R3CPageSetupDialog@@8   5f8bea90     dlgprnt.obj
 0002:00013aa0       ??_R4CPageSetupDialog@@6B@ 5f8beaa0     dlgprnt.obj
 0002:00013ab8       ??_R1A@?0A@A@CPrintDialog@@8 5f8beab8     dlgprnt.obj
 0002:00013ad0       ??_R2CPrintDialog@@8       5f8bead0     dlgprnt.obj
 0002:00013af0       ??_R3CPrintDialog@@8       5f8beaf0     dlgprnt.obj
 0002:00013b00       ??_R4CPrintDialog@@6B@     5f8beb00     dlgprnt.obj
 0002:00013b18       ??_R1A@?0A@A@_AFX_COLOR_STATE@@8 5f8beb18     dlgclr.obj
 0002:00013b30       ??_R2_AFX_COLOR_STATE@@8   5f8beb30     dlgclr.obj
 0002:00013b40       ??_R3_AFX_COLOR_STATE@@8   5f8beb40     dlgclr.obj
 0002:00013b50       ??_R4_AFX_COLOR_STATE@@6B@ 5f8beb50     dlgclr.obj
 0002:00013b68       ??_R1A@?0A@A@CColorDialog@@8 5f8beb68     dlgclr.obj
 0002:00013b80       ??_R2CColorDialog@@8       5f8beb80     dlgclr.obj
 0002:00013ba0       ??_R3CColorDialog@@8       5f8beba0     dlgclr.obj
 0002:00013bb0       ??_R4CColorDialog@@6B@     5f8bebb0     dlgclr.obj
 0002:00013bc8       ??_R1A@?0A@A@CFontDialog@@8 5f8bebc8     dlgfnt.obj
 0002:00013be0       ??_R2CFontDialog@@8        5f8bebe0     dlgfnt.obj
 0002:00013c00       ??_R3CFontDialog@@8        5f8bec00     dlgfnt.obj
 0002:00013c10       ??_R4CFontDialog@@6B@      5f8bec10     dlgfnt.obj
 0002:00013c28       ??_R1A@?0A@A@CFindReplaceDialog@@8 5f8bec28     dlgfr.obj
 0002:00013c40       ??_R2CFindReplaceDialog@@8 5f8bec40     dlgfr.obj
 0002:00013c60       ??_R3CFindReplaceDialog@@8 5f8bec60     dlgfr.obj
 0002:00013c70       ??_R4CFindReplaceDialog@@6B@ 5f8bec70     dlgfr.obj
 0002:00013c88       ??_R1A@?0A@A@_AFX_PROPPAGEFONTINFO@@8 5f8bec88     ccdata.obj
 0002:00013ca0       ??_R2_AFX_PROPPAGEFONTINFO@@8 5f8beca0     ccdata.obj
 0002:00013cb0       ??_R3_AFX_PROPPAGEFONTINFO@@8 5f8becb0     ccdata.obj
 0002:00013cc0       ??_R4_AFX_PROPPAGEFONTINFO@@6B@ 5f8becc0     ccdata.obj
 0002:00013cd8       ??_R1A@?0A@A@CIPAddressCtrl@@8 5f8becd8     winctrl6.obj
 0002:00013cf0       ??_R2CIPAddressCtrl@@8     5f8becf0     winctrl6.obj
 0002:00013d08       ??_R3CIPAddressCtrl@@8     5f8bed08     winctrl6.obj
 0002:00013d18       ??_R4CIPAddressCtrl@@6B@   5f8bed18     winctrl6.obj
 0002:00013d30       ??_R1A@?0A@A@CComboBoxEx@@8 5f8bed30     winctrl6.obj
 0002:00013d48       ??_R2CComboBoxEx@@8        5f8bed48     winctrl6.obj
 0002:00013d60       ??_R3CComboBoxEx@@8        5f8bed60     winctrl6.obj
 0002:00013d70       ??_R4CComboBoxEx@@6B@      5f8bed70     winctrl6.obj
 0002:00013d88       ??_R1A@?0A@A@CReBarCtrl@@8 5f8bed88     winctrl6.obj
 0002:00013da0       ??_R2CReBarCtrl@@8         5f8beda0     winctrl6.obj
 0002:00013db8       ??_R3CReBarCtrl@@8         5f8bedb8     winctrl6.obj
 0002:00013dc8       ??_R4CReBarCtrl@@6B@       5f8bedc8     winctrl6.obj
 0002:00013de0       ??_R2CDC@@8                5f8bede0     wingdi.obj
 0002:00013df0       ??_R3CDC@@8                5f8bedf0     wingdi.obj
 0002:00013e00       ??_R4CDC@@6B@              5f8bee00     wingdi.obj
 0002:00013e18       ??_R1A@?0A@A@CClientDC@@8  5f8bee18     wingdi.obj
 0002:00013e30       ??_R2CClientDC@@8          5f8bee30     wingdi.obj
 0002:00013e40       ??_R3CClientDC@@8          5f8bee40     wingdi.obj
 0002:00013e50       ??_R4CClientDC@@6B@        5f8bee50     wingdi.obj
 0002:00013e68       ??_R1A@?0A@A@CWindowDC@@8  5f8bee68     wingdi.obj
 0002:00013e80       ??_R2CWindowDC@@8          5f8bee80     wingdi.obj
 0002:00013e90       ??_R3CWindowDC@@8          5f8bee90     wingdi.obj
 0002:00013ea0       ??_R4CWindowDC@@6B@        5f8beea0     wingdi.obj
 0002:00013eb8       ??_R1A@?0A@A@CPaintDC@@8   5f8beeb8     wingdi.obj
 0002:00013ed0       ??_R2CPaintDC@@8           5f8beed0     wingdi.obj
 0002:00013ee0       ??_R3CPaintDC@@8           5f8beee0     wingdi.obj
 0002:00013ef0       ??_R4CPaintDC@@6B@         5f8beef0     wingdi.obj
 0002:00013f08       ??_R1A@?0A@A@CTempDC@@8    5f8bef08     wingdi.obj
 0002:00013f20       ??_R2CTempDC@@8            5f8bef20     wingdi.obj
 0002:00013f30       ??_R3CTempDC@@8            5f8bef30     wingdi.obj
 0002:00013f40       ??_R4CTempDC@@6B@          5f8bef40     wingdi.obj
 0002:00013f58       ??_R1A@?0A@A@CTempGdiObject@@8 5f8bef58     wingdi.obj
 0002:00013f70       ??_R2CTempGdiObject@@8     5f8bef70     wingdi.obj
 0002:00013f80       ??_R3CTempGdiObject@@8     5f8bef80     wingdi.obj
 0002:00013f90       ??_R4CTempGdiObject@@6B@   5f8bef90     wingdi.obj
 0002:00013fa8       ??_R1A@?0A@A@CTempMenu@@8  5f8befa8     winmenu.obj
 0002:00013fc0       ??_R2CTempMenu@@8          5f8befc0     winmenu.obj
 0002:00013fd0       ??_R3CTempMenu@@8          5f8befd0     winmenu.obj
 0002:00013fe0       ??_R4CTempMenu@@6B@        5f8befe0     winmenu.obj
 0002:00013ff8       ??_R2CCmdTarget@@8         5f8beff8     cmdtarg.obj
 0002:00014008       ??_R3CCmdTarget@@8         5f8bf008     cmdtarg.obj
 0002:00014018       ??_R4CCmdTarget@@6B@       5f8bf018     cmdtarg.obj
 0002:0001402c       ??_R2CCmdUI@@8             5f8bf02c     cmdtarg.obj
 0002:00014038       ??_R3CCmdUI@@8             5f8bf038     cmdtarg.obj
 0002:00014048       ??_R4CCmdUI@@6B@           5f8bf048     cmdtarg.obj
 0002:00014060       ??_R1A@?0A@A@CDocument@@8  5f8bf060     doccore.obj
 0002:00014078       ??_R2CDocument@@8          5f8bf078     doccore.obj
 0002:00014088       ??_R3CDocument@@8          5f8bf088     doccore.obj
 0002:00014098       ??_R4CDocument@@6B@        5f8bf098     doccore.obj
 0002:000140b0       ??_R1A@?0A@A@CMirrorFile@@8 5f8bf0b0     doccore.obj
 0002:000140c8       ??_R2CMirrorFile@@8        5f8bf0c8     doccore.obj
 0002:000140d8       ??_R3CMirrorFile@@8        5f8bf0d8     doccore.obj
 0002:000140e8       ??_R4CMirrorFile@@6B@      5f8bf0e8     doccore.obj
 0002:00014100       ??_R1A@?0A@A@CDocTemplate@@8 5f8bf100     doctempl.obj
 0002:00014118       ??_R2CDocTemplate@@8       5f8bf118     doctempl.obj
 0002:00014128       ??_R3CDocTemplate@@8       5f8bf128     doctempl.obj
 0002:00014138       ??_R4CDocTemplate@@6B@     5f8bf138     doctempl.obj
 0002:00014150       ??_R1A@?0A@A@CSingleDocTemplate@@8 5f8bf150     docsingl.obj
 0002:00014168       ??_R2CSingleDocTemplate@@8 5f8bf168     docsingl.obj
 0002:00014180       ??_R3CSingleDocTemplate@@8 5f8bf180     docsingl.obj
 0002:00014190       ??_R4CSingleDocTemplate@@6B@ 5f8bf190     docsingl.obj
 0002:000141a8       ??_R1A@?0A@A@CMultiDocTemplate@@8 5f8bf1a8     docmulti.obj
 0002:000141c0       ??_R2CMultiDocTemplate@@8  5f8bf1c0     docmulti.obj
 0002:000141d8       ??_R3CMultiDocTemplate@@8  5f8bf1d8     docmulti.obj
 0002:000141e8       ??_R4CMultiDocTemplate@@6B@ 5f8bf1e8     docmulti.obj
 0002:00014200       ??_R1A@?0A@A@CDocManager@@8 5f8bf200     docmgr.obj
 0002:00014218       ??_R2CDocManager@@8        5f8bf218     docmgr.obj
 0002:00014228       ??_R3CDocManager@@8        5f8bf228     docmgr.obj
 0002:00014238       ??_R4CDocManager@@6B@      5f8bf238     docmgr.obj
 0002:00014250       ??_R1A@?0A@A@CNewTypeDlg@@8 5f8bf250     docmgr.obj
 0002:00014268       ??_R2CNewTypeDlg@@8        5f8bf268     docmgr.obj
 0002:00014280       ??_R3CNewTypeDlg@@8        5f8bf280     docmgr.obj
 0002:00014290       ??_R4CNewTypeDlg@@6B@      5f8bf290     docmgr.obj
 0002:000142a8       ??_R1A@?0A@A@CView@@8      5f8bf2a8     viewcore.obj
 0002:000142c0       ??_R2CView@@8              5f8bf2c0     viewcore.obj
 0002:000142d8       ??_R3CView@@8              5f8bf2d8     viewcore.obj
 0002:000142e8       ??_R4CView@@6B@            5f8bf2e8     viewcore.obj
 0002:00014300       ??_R1A@?0A@A@CCtrlView@@8  5f8bf300     viewcore.obj
 0002:00014318       ??_R2CCtrlView@@8          5f8bf318     viewcore.obj
 0002:00014330       ??_R3CCtrlView@@8          5f8bf330     viewcore.obj
 0002:00014340       ??_R4CCtrlView@@6B@        5f8bf340     viewcore.obj
 0002:00014358       ??_R1A@?0A@A@CPrintingDialog@@8 5f8bf358     viewprnt.obj
 0002:00014370       ??_R2CPrintingDialog@@8    5f8bf370     viewprnt.obj
 0002:00014388       ??_R3CPrintingDialog@@8    5f8bf388     viewprnt.obj
 0002:00014398       ??_R4CPrintingDialog@@6B@  5f8bf398     viewprnt.obj
 0002:000143b0       ??_R1A@?0A@A@CSplitterWnd@@8 5f8bf3b0     winsplit.obj
 0002:000143c8       ??_R2CSplitterWnd@@8       5f8bf3c8     winsplit.obj
 0002:000143e0       ??_R3CSplitterWnd@@8       5f8bf3e0     winsplit.obj
 0002:000143f0       ??_R4CSplitterWnd@@6B@     5f8bf3f0     winsplit.obj
 0002:00014408       ??_R1A@?0A@A@CScrollView@@8 5f8bf408     viewscrl.obj
 0002:00014420       ??_R2CScrollView@@8        5f8bf420     viewscrl.obj
 0002:00014438       ??_R3CScrollView@@8        5f8bf438     viewscrl.obj
 0002:00014448       ??_R4CScrollView@@6B@      5f8bf448     viewscrl.obj
 0002:00014460       ??_R1A@?0A@A@CFormView@@8  5f8bf460     viewform.obj
 0002:00014478       ??_R2CFormView@@8          5f8bf478     viewform.obj
 0002:00014498       ??_R3CFormView@@8          5f8bf498     viewform.obj
 0002:000144a8       ??_R4CFormView@@6B@        5f8bf4a8     viewform.obj
 0002:000144c0       ??_R2_AFX_EDIT_STATE@@8    5f8bf4c0     viewedit.obj
 0002:000144d0       ??_R3_AFX_EDIT_STATE@@8    5f8bf4d0     viewedit.obj
 0002:000144e0       ??_R4_AFX_EDIT_STATE@@6B@  5f8bf4e0     viewedit.obj
 0002:000144f8       ??_R1A@?0A@A@CEditView@@8  5f8bf4f8     viewedit.obj
 0002:00014510       ??_R2CEditView@@8          5f8bf510     viewedit.obj
 0002:00014530       ??_R3CEditView@@8          5f8bf530     viewedit.obj
 0002:00014540       ??_R4CEditView@@6B@        5f8bf540     viewedit.obj
 0002:00014558       ??_R1A@?0A@A@CPreviewView@@8 5f8bf558     viewprev.obj
 0002:00014570       ??_R2CPreviewView@@8       5f8bf570     viewprev.obj
 0002:00014590       ??_R3CPreviewView@@8       5f8bf590     viewprev.obj
 0002:000145a0       ??_R4CPreviewView@@6B@     5f8bf5a0     viewprev.obj
 0002:000145b8       ??_R1A@?0A@A@CListView@@8  5f8bf5b8     viewcmn.obj
 0002:000145d0       ??_R2CListView@@8          5f8bf5d0     viewcmn.obj
 0002:000145f0       ??_R3CListView@@8          5f8bf5f0     viewcmn.obj
 0002:00014600       ??_R4CListView@@6B@        5f8bf600     viewcmn.obj
 0002:00014618       ??_R1A@?0A@A@CTreeView@@8  5f8bf618     viewcmn.obj
 0002:00014630       ??_R2CTreeView@@8          5f8bf630     viewcmn.obj
 0002:00014650       ??_R3CTreeView@@8          5f8bf650     viewcmn.obj
 0002:00014660       ??_R4CTreeView@@6B@        5f8bf660     viewcmn.obj
 0002:00014678       ??_R1A@?0A@A@_AFX_MAIL_STATE@@8 5f8bf678     docmapi.obj
 0002:00014690       ??_R2_AFX_MAIL_STATE@@8    5f8bf690     docmapi.obj
 0002:000146a0       ??_R3_AFX_MAIL_STATE@@8    5f8bf6a0     docmapi.obj
 0002:000146b0       ??_R4_AFX_MAIL_STATE@@6B@  5f8bf6b0     docmapi.obj
 0002:000146c8       ??_R1A@?0A@A@CWinThread@@8 5f8bf6c8     thrdcore.obj
 0002:000146e0       ??_R2CWinThread@@8         5f8bf6e0     thrdcore.obj
 0002:000146f0       ??_R3CWinThread@@8         5f8bf6f0     thrdcore.obj
 0002:00014700       ??_R4CWinThread@@6B@       5f8bf700     thrdcore.obj
 0002:00014718       ??_R1A@?0A@A@_AFX_CTL3D_THREAD@@8 5f8bf718     thrdcore.obj
 0002:00014730       ??_R2_AFX_CTL3D_THREAD@@8  5f8bf730     thrdcore.obj
 0002:00014740       ??_R3_AFX_CTL3D_THREAD@@8  5f8bf740     thrdcore.obj
 0002:00014750       ??_R4_AFX_CTL3D_THREAD@@6B@ 5f8bf750     thrdcore.obj
 0002:00014768       ??_R1A@?0A@A@_AFX_WIN_STATE@@8 5f8bf768     appcore.obj
 0002:00014780       ??_R2_AFX_WIN_STATE@@8     5f8bf780     appcore.obj
 0002:00014790       ??_R3_AFX_WIN_STATE@@8     5f8bf790     appcore.obj
 0002:000147a0       ??_R4_AFX_WIN_STATE@@6B@   5f8bf7a0     appcore.obj
 0002:000147b8       ??_R1A@?0A@A@CWinApp@@8    5f8bf7b8     appcore.obj
 0002:000147d0       ??_R2CWinApp@@8            5f8bf7d0     appcore.obj
 0002:000147e8       ??_R3CWinApp@@8            5f8bf7e8     appcore.obj
 0002:000147f8       ??_R4CWinApp@@6B@          5f8bf7f8     appcore.obj
 0002:00014810       ??_R1A@?0A@A@CCommandLineInfo@@8 5f8bf810     appcore.obj
 0002:00014828       ??_R2CCommandLineInfo@@8   5f8bf828     appcore.obj
 0002:00014838       ??_R3CCommandLineInfo@@8   5f8bf838     appcore.obj
 0002:00014848       ??_R4CCommandLineInfo@@6B@ 5f8bf848     appcore.obj
 0002:00014860       ??_R1A@?0A@A@CRecentFileList@@8 5f8bf860     filelist.obj
 0002:00014878       ??_R2CRecentFileList@@8    5f8bf878     filelist.obj
 0002:00014880       ??_R3CRecentFileList@@8    5f8bf880     filelist.obj
 0002:00014890       ??_R4CRecentFileList@@6B@  5f8bf890     filelist.obj
 0002:000148a8       ??_R1A@?0A@A@CInternetSession@@8 5f8bf8a8     inet.obj
 0002:000148c0       ??_R2CInternetSession@@8   5f8bf8c0     inet.obj
 0002:000148d0       ??_R3CInternetSession@@8   5f8bf8d0     inet.obj
 0002:000148e0       ??_R4CInternetSession@@6B@ 5f8bf8e0     inet.obj
 0002:000148f8       ??_R1A@?0A@A@CInternetFile@@8 5f8bf8f8     inet.obj
 0002:00014910       ??_R2CInternetFile@@8      5f8bf910     inet.obj
 0002:00014928       ??_R3CInternetFile@@8      5f8bf928     inet.obj
 0002:00014938       ??_R4CInternetFile@@6B@    5f8bf938     inet.obj
 0002:00014950       ??_R1A@?0A@A@CInternetConnection@@8 5f8bf950     inet.obj
 0002:00014968       ??_R2CInternetConnection@@8 5f8bf968     inet.obj
 0002:00014978       ??_R3CInternetConnection@@8 5f8bf978     inet.obj
 0002:00014988       ??_R4CInternetConnection@@6B@ 5f8bf988     inet.obj
 0002:000149a0       ??_R1A@?0A@A@CFtpConnection@@8 5f8bf9a0     inet.obj
 0002:000149b8       ??_R2CFtpConnection@@8     5f8bf9b8     inet.obj
 0002:000149c8       ??_R3CFtpConnection@@8     5f8bf9c8     inet.obj
 0002:000149d8       ??_R4CFtpConnection@@6B@   5f8bf9d8     inet.obj
 0002:000149f0       ??_R1A@?0A@A@CGopherConnection@@8 5f8bf9f0     inet.obj
 0002:00014a08       ??_R2CGopherConnection@@8  5f8bfa08     inet.obj
 0002:00014a18       ??_R3CGopherConnection@@8  5f8bfa18     inet.obj
 0002:00014a28       ??_R4CGopherConnection@@6B@ 5f8bfa28     inet.obj
 0002:00014a40       ??_R1A@?0A@A@CHttpConnection@@8 5f8bfa40     inet.obj
 0002:00014a58       ??_R2CHttpConnection@@8    5f8bfa58     inet.obj
 0002:00014a68       ??_R3CHttpConnection@@8    5f8bfa68     inet.obj
 0002:00014a78       ??_R4CHttpConnection@@6B@  5f8bfa78     inet.obj
 0002:00014a90       ??_R1A@?0A@A@CHttpFile@@8  5f8bfa90     inet.obj
 0002:00014aa8       ??_R2CHttpFile@@8          5f8bfaa8     inet.obj
 0002:00014ac0       ??_R3CHttpFile@@8          5f8bfac0     inet.obj
 0002:00014ad0       ??_R4CHttpFile@@6B@        5f8bfad0     inet.obj
 0002:00014ae8       ??_R1A@?0A@A@CGopherFile@@8 5f8bfae8     inet.obj
 0002:00014b00       ??_R2CGopherFile@@8        5f8bfb00     inet.obj
 0002:00014b18       ??_R3CGopherFile@@8        5f8bfb18     inet.obj
 0002:00014b28       ??_R4CGopherFile@@6B@      5f8bfb28     inet.obj
 0002:00014b40       ??_R1A@?0A@A@CFileFind@@8  5f8bfb40     inet.obj
 0002:00014b58       ??_R1A@?0A@A@CFtpFileFind@@8 5f8bfb58     inet.obj
 0002:00014b70       ??_R2CFtpFileFind@@8       5f8bfb70     inet.obj
 0002:00014b80       ??_R3CFtpFileFind@@8       5f8bfb80     inet.obj
 0002:00014b90       ??_R4CFtpFileFind@@6B@     5f8bfb90     inet.obj
 0002:00014ba8       ??_R1A@?0A@A@CGopherFileFind@@8 5f8bfba8     inet.obj
 0002:00014bc0       ??_R2CGopherFileFind@@8    5f8bfbc0     inet.obj
 0002:00014bd0       ??_R3CGopherFileFind@@8    5f8bfbd0     inet.obj
 0002:00014be0       ??_R4CGopherFileFind@@6B@  5f8bfbe0     inet.obj
 0002:00014bf8       ??_R1A@?0A@A@CGopherLocator@@8 5f8bfbf8     inet.obj
 0002:00014c10       ??_R2CGopherLocator@@8     5f8bfc10     inet.obj
 0002:00014c20       ??_R3CGopherLocator@@8     5f8bfc20     inet.obj
 0002:00014c30       ??_R4CGopherLocator@@6B@   5f8bfc30     inet.obj
 0002:00014c48       ??_R1A@?0A@A@CInternetException@@8 5f8bfc48     inet.obj
 0002:00014c60       ??_R2CInternetException@@8 5f8bfc60     inet.obj
 0002:00014c70       ??_R3CInternetException@@8 5f8bfc70     inet.obj
 0002:00014c80       ??_R4CInternetException@@6B@ 5f8bfc80     inet.obj
 0002:00014c98       ??_R1A@?0A@A@CSessionMapPtrToPtr@@8 5f8bfc98     inet.obj
 0002:00014cb0       ??_R2CSessionMapPtrToPtr@@8 5f8bfcb0     inet.obj
 0002:00014cc0       ??_R3CSessionMapPtrToPtr@@8 5f8bfcc0     inet.obj
 0002:00014cd0       ??_R4CSessionMapPtrToPtr@@6B@ 5f8bfcd0     inet.obj
 0002:00014ce8       ??_R2CFileFind@@8          5f8bfce8     filefind.obj
 0002:00014cf8       ??_R3CFileFind@@8          5f8bfcf8     filefind.obj
 0002:00014d08       ??_R4CFileFind@@6B@        5f8bfd08     filefind.obj
 0002:00014d20       ??_R1A@?0A@A@CDynLinkLibrary@@8 5f8bfd20     dllinit.obj
 0002:00014d38       ??_R2CDynLinkLibrary@@8    5f8bfd38     dllinit.obj
 0002:00014d48       ??_R3CDynLinkLibrary@@8    5f8bfd48     dllinit.obj
 0002:00014d58       ??_R4CDynLinkLibrary@@6B@  5f8bfd58     dllinit.obj
 0002:00014d70       ??_R1A@?0A@A@type_info@@8  5f8bfd70     msvcrtd:ti_inst.obj
 0002:00014d88       ??_R2type_info@@8          5f8bfd88     msvcrtd:ti_inst.obj
 0002:00014d90       ??_R3type_info@@8          5f8bfd90     msvcrtd:ti_inst.obj
 0002:00014da0       ??_R4type_info@@6B@        5f8bfda0     msvcrtd:ti_inst.obj
 0002:00014e10       __CT??_R0PAX@84            5f8bfe10     except.obj
 0002:00014e30       __CT??_R0PAVCObject@@@84   5f8bfe30     except.obj
 0002:00014e50       __CT??_R0PAVCException@@@84 5f8bfe50     except.obj
 0002:00014e70       __CT??_R0PAVCSimpleException@@@84 5f8bfe70     except.obj
 0002:00014e90       __CT??_R0PAVCMemoryException@@@84 5f8bfe90     except.obj
 0002:00014eb0       __CTA5PAVCMemoryException@@ 5f8bfeb0     except.obj
 0002:00014ec8       __TI5PAVCMemoryException@@ 5f8bfec8     except.obj
 0002:00014ed8       __CT??_R0PAVCNotSupportedException@@@84 5f8bfed8     except.obj
 0002:00014ef8       __CTA5PAVCNotSupportedException@@ 5f8bfef8     except.obj
 0002:00014f10       __TI5PAVCNotSupportedException@@ 5f8bff10     except.obj
 0002:000150a0       __CT??_R0PAVCArchiveException@@@84 5f8c00a0     arcex.obj
 0002:000150c0       __CTA4PAVCArchiveException@@ 5f8c00c0     arcex.obj
 0002:000150d8       __TI4PAVCArchiveException@@ 5f8c00d8     arcex.obj
 0002:00015670       __CT??_R0PAVCFileException@@@84 5f8c0670     filex.obj
 0002:00015690       __CTA4PAVCFileException@@  5f8c0690     filex.obj
 0002:000156a8       __TI4PAVCFileException@@   5f8c06a8     filex.obj
 0002:00018830       __CT??_R0PAVCResourceException@@@84 5f8c3830     wingdi.obj
 0002:00018850       __CTA5PAVCResourceException@@ 5f8c3850     wingdi.obj
 0002:00018868       __TI5PAVCResourceException@@ 5f8c3868     wingdi.obj
 0002:00018878       __CT??_R0PAVCUserException@@@84 5f8c3878     wingdi.obj
 0002:00018898       __CTA5PAVCUserException@@  5f8c3898     wingdi.obj
 0002:000188b0       __TI5PAVCUserException@@   5f8c38b0     wingdi.obj
 0002:0001a800       __CT??_R0PAVCInternetException@@@84 5f8c5800     inet.obj
 0002:0001a820       __CTA4PAVCInternetException@@ 5f8c5820     inet.obj
 0002:0001a838       __TI4PAVCInternetException@@ 5f8c5838     inet.obj
 0002:0001ad08       __DELAY_IMPORT_DESCRIPTOR_ADVAPI32 5f8c5d08     advapi32:ADVAPI32.dll
 0002:0001ad28       __DELAY_IMPORT_DESCRIPTOR_COMCTL32 5f8c5d28     comctl32:COMCTL32.dll
 0002:0001ad48       __DELAY_IMPORT_DESCRIPTOR_SHELL32 5f8c5d48     shell32:SHELL32.dll
 0002:0001ad68       __DELAY_IMPORT_DESCRIPTOR_comdlg32 5f8c5d68     comdlg32:comdlg32.dll
 0002:0001ad88       __DELAY_IMPORT_DESCRIPTOR_WINSPOOL 5f8c5d88     winspool:WINSPOOL.DRV
 0002:0001ada8       __DELAY_IMPORT_DESCRIPTOR_WININET 5f8c5da8     wininet:WININET.dll
 0002:0001adc8       __NULL_DELAY_IMPORT_DESCRIPTOR 5f8c5dc8     advapi32:ADVAPI32.dll
 0002:0001ae20       \177ADVAPI32_NULL_THUNK_DATA_DLN 5f8c5e20     advapi32:ADVAPI32.dll
 0002:0001aebc       \177COMCTL32_NULL_THUNK_DATA_DLN 5f8c5ebc     comctl32:COMCTL32.dll
 0002:0001aed4       \177SHELL32_NULL_THUNK_DATA_DLN 5f8c5ed4     shell32:SHELL32.dll
 0002:0001af74       \177WININET_NULL_THUNK_DATA_DLN 5f8c5f74     wininet:WININET.dll
 0002:0001af84       \177WINSPOOL_NULL_THUNK_DATA_DLN 5f8c5f84     winspool:WINSPOOL.DRV
 0002:0001afb0       \177comdlg32_NULL_THUNK_DATA_DLN 5f8c5fb0     comdlg32:comdlg32.dll
 0002:0001b82c       \177ADVAPI32_NULL_THUNK_DATA_DLB 5f8c682c     advapi32:ADVAPI32.dll
 0002:0001b868       \177COMCTL32_NULL_THUNK_DATA_DLB 5f8c6868     comctl32:COMCTL32.dll
 0002:0001b904       \177SHELL32_NULL_THUNK_DATA_DLB 5f8c6904     shell32:SHELL32.dll
 0002:0001b91c       \177comdlg32_NULL_THUNK_DATA_DLB 5f8c691c     comdlg32:comdlg32.dll
 0002:0001b948       \177WINSPOOL_NULL_THUNK_DATA_DLB 5f8c6948     winspool:WINSPOOL.DRV
 0002:0001b958       \177WININET_NULL_THUNK_DATA_DLB 5f8c6958     wininet:WININET.dll
 0002:0001b9f4       __IMPORT_DESCRIPTOR_MSVCRTD 5f8c69f4     msvcrtd:MSVCRTD.dll
 0002:0001ba08       __IMPORT_DESCRIPTOR_KERNEL32 5f8c6a08     kernel32:KERNEL32.dll
 0002:0001ba1c       __IMPORT_DESCRIPTOR_GDI32  5f8c6a1c     gdi32:GDI32.dll
 0002:0001ba30       __IMPORT_DESCRIPTOR_USER32 5f8c6a30     user32:USER32.dll
 0002:0001ba44       __NULL_IMPORT_DESCRIPTOR   5f8c6a44     msvcrtd:MSVCRTD.dll
 0003:00000000       ___xc_a                    5f8cf000     msvcrtd:cinitexe.obj
 0003:000000b0       ___xc_z                    5f8cf0b0     msvcrtd:cinitexe.obj
 0003:000000b4       ___xi_a                    5f8cf0b4     msvcrtd:cinitexe.obj
 0003:000000b8       ___xi_z                    5f8cf0b8     msvcrtd:cinitexe.obj
 0003:000000d0       ??_R0PAVCException@@@8     5f8cf0d0     objcore.obj
 0003:000000f8       ??_R0?AVCObject@@@8        5f8cf0f8     except.obj
 0003:00000110       ??_R0?AVCException@@@8     5f8cf110     except.obj
 0003:00000130       ??_R0PAX@8                 5f8cf130     except.obj
 0003:00000140       ??_R0PAVCObject@@@8        5f8cf140     except.obj
 0003:00000158       ??_R0PAVCSimpleException@@@8 5f8cf158     except.obj
 0003:00000178       ??_R0PAVCMemoryException@@@8 5f8cf178     except.obj
 0003:00000198       ??_R0PAVCNotSupportedException@@@8 5f8cf198     except.obj
 0003:000001f8       ??_R0PAVCArchiveException@@@8 5f8cf1f8     arccore.obj
 0003:00000240       ??_R0?AUIUnknown@@@8       5f8cf240     arcstrm.obj
 0003:00000258       ??_R0?AUISequentialStream@@@8 5f8cf258     arcstrm.obj
 0003:00000278       ??_R0?AUIStream@@@8        5f8cf278     arcstrm.obj
 0003:00000290       ??_R0?AVCArchiveStream@@@8 5f8cf290     arcstrm.obj
 0003:000002b0       ??_R0?AVCNoTrackObject@@@8 5f8cf2b0     dumpinit.obj
 0003:000002d0       ??_R0?AV_AFX_DEBUG_STATE@@@8 5f8cf2d0     dumpinit.obj
 0003:0000030c       ?pfnAllocHook@@3P6GHIHJ@ZA 5f8cf30c     afxmem.obj
 0003:00000320       ??_R0?AVCSimpleException@@@8 5f8cf320     afxinl1.obj
 0003:00000340       ??_R0?AVCMemoryException@@@8 5f8cf340     afxinl1.obj
 0003:00000360       ??_R0?AVCNotSupportedException@@@8 5f8cf360     afxinl1.obj
 0003:00000388       ??_R0?AVCArchiveException@@@8 5f8cf388     afxinl1.obj
 0003:000003a8       ??_R0?AVCFileException@@@8 5f8cf3a8     afxinl1.obj
 0003:000003c8       ??_R0?AVCCmdTarget@@@8     5f8cf3c8     afxinl1.obj
 0003:000003e8       ??_R0?AVCWnd@@@8           5f8cf3e8     afxinl1.obj
 0003:00000400       ??_R0?AVCDialog@@@8        5f8cf400     afxinl1.obj
 0003:00000418       ??_R0?AVCCommonDialog@@@8  5f8cf418     afxinl1.obj
 0003:00000438       ??_R0?AVCRectTracker@@@8   5f8cf438     afxinl1.obj
 0003:00000458       ??_R0?AVCButton@@@8        5f8cf458     afxinl1.obj
 0003:00000470       ??_R0?AVCBitmapButton@@@8  5f8cf470     afxinl1.obj
 0003:00000490       ??_R0?AVCResourceException@@@8 5f8cf490     afxinl2.obj
 0003:000004b8       ??_R0?AVCUserException@@@8 5f8cf4b8     afxinl2.obj
 0003:000004d8       ??_R0?AVCGdiObject@@@8     5f8cf4d8     afxinl2.obj
 0003:000004f8       ??_R0?AVCPen@@@8           5f8cf4f8     afxinl2.obj
 0003:00000510       ??_R0?AVCBrush@@@8         5f8cf510     afxinl2.obj
 0003:00000528       ??_R0?AVCFont@@@8          5f8cf528     afxinl2.obj
 0003:00000540       ??_R0?AVCBitmap@@@8        5f8cf540     afxinl2.obj
 0003:00000558       ??_R0?AVCPalette@@@8       5f8cf558     afxinl2.obj
 0003:00000570       ??_R0?AVCRgn@@@8           5f8cf570     afxinl2.obj
 0003:00000588       ??_R0?AVCMenu@@@8          5f8cf588     afxinl2.obj
 0003:000005a0       ??_R0?AVCStatic@@@8        5f8cf5a0     afxinl3.obj
 0003:000005b8       ??_R0?AVCListBox@@@8       5f8cf5b8     afxinl3.obj
 0003:000005d0       ??_R0?AVCCheckListBox@@@8  5f8cf5d0     afxinl3.obj
 0003:000005f0       ??_R0?AVCComboBox@@@8      5f8cf5f0     afxinl3.obj
 0003:00000608       ??_R0?AVCEdit@@@8          5f8cf608     afxinl3.obj
 0003:00000620       ??_R0?AVCScrollBar@@@8     5f8cf620     afxinl3.obj
 0003:00000650       ??_R0?AVCFile@@@8          5f8cf650     filecore.obj
 0003:00000670       ??_R0?AVCStdioFile@@@8     5f8cf670     filetxt.obj
 0003:00000698       ??_R0?AVCMemFile@@@8       5f8cf698     filemem.obj
 0003:000006c0       ??_R0?AVCSharedFile@@@8    5f8cf6c0     fileshrd.obj
 0003:000006e8       ??_R0PAVCFileException@@@8 5f8cf6e8     filex.obj
 0003:00000718       ?classCByteArray@CByteArray@@2UCRuntimeClass@@A 5f8cf718     array_b.obj
 0003:00000740       ??_R0?AVCByteArray@@@8     5f8cf740     array_b.obj
 0003:00000760       ?classCDWordArray@CDWordArray@@2UCRuntimeClass@@A 5f8cf760     array_d.obj
 0003:00000788       ??_R0?AVCDWordArray@@@8    5f8cf788     array_d.obj
 0003:000007b0       ??_R0?AVCPtrArray@@@8      5f8cf7b0     array_p.obj
 0003:000007c8       ?classCObArray@CObArray@@2UCRuntimeClass@@A 5f8cf7c8     array_o.obj
 0003:000007f0       ??_R0?AVCObArray@@@8       5f8cf7f0     array_o.obj
 0003:00000808       ?classCStringArray@CStringArray@@2UCRuntimeClass@@A 5f8cf808     array_s.obj
 0003:00000830       ??_R0?AVCStringArray@@@8   5f8cf830     array_s.obj
 0003:00000858       ??_R0?AVCUIntArray@@@8     5f8cf858     array_u.obj
 0003:00000878       ?classCWordArray@CWordArray@@2UCRuntimeClass@@A 5f8cf878     array_w.obj
 0003:000008a0       ??_R0?AVCWordArray@@@8     5f8cf8a0     array_w.obj
 0003:000008c0       ?classCObList@CObList@@2UCRuntimeClass@@A 5f8cf8c0     list_o.obj
 0003:000008e8       ??_R0?AVCObList@@@8        5f8cf8e8     list_o.obj
 0003:00000910       ??_R0?AVCPtrList@@@8       5f8cf910     list_p.obj
 0003:00000928       ?classCStringList@CStringList@@2UCRuntimeClass@@A 5f8cf928     list_s.obj
 0003:00000950       ??_R0?AVCStringList@@@8    5f8cf950     list_s.obj
 0003:00000978       ??_R0?AVCMapPtrToPtr@@@8   5f8cf978     map_pp.obj
 0003:000009a0       ??_R0?AVCMapPtrToWord@@@8  5f8cf9a0     map_pw.obj
 0003:000009c0       ?classCMapStringToOb@CMapStringToOb@@2UCRuntimeClass@@A 5f8cf9c0     map_so.obj
 0003:000009e8       ??_R0?AVCMapStringToOb@@@8 5f8cf9e8     map_so.obj
 0003:00000a18       ??_R0?AVCMapStringToPtr@@@8 5f8cfa18     map_sp.obj
 0003:00000a38       ?classCMapStringToString@CMapStringToString@@2UCRuntimeClass@@A 5f8cfa38     map_ss.obj
 0003:00000a60       ??_R0?AVCMapStringToString@@@8 5f8cfa60     map_ss.obj
 0003:00000a88       ?classCMapWordToOb@CMapWordToOb@@2UCRuntimeClass@@A 5f8cfa88     map_wo.obj
 0003:00000ab0       ??_R0?AVCMapWordToOb@@@8   5f8cfab0     map_wo.obj
 0003:00000ad8       ??_R0?AVCMapWordToPtr@@@8  5f8cfad8     map_wp.obj
 0003:00000b00       ?_afxPchNil@@3PBGB         5f8cfb00     strcore.obj
 0003:00000b04       ?_afxDataNil@@3PAUCStringData@@A 5f8cfb04     strcore.obj
 0003:00000b08       ?_afxInitData@@3PAHA       5f8cfb08     strcore.obj
 0003:00000b60       ??_R0?AV_AFX_THREAD_STATE@@@8 5f8cfb60     afxstate.obj
 0003:00000b80       ??_R0?AVAFX_MODULE_STATE@@@8 5f8cfb80     afxstate.obj
 0003:00000ba0       ??_R0?AVAFX_MODULE_THREAD_STATE@@@8 5f8cfba0     afxstate.obj
 0003:00000bc8       ??_R0?AV_AFX_BASE_MODULE_STATE@@@8 5f8cfbc8     afxstate.obj
 0003:00000c00       ??_R0?AUCThreadData@@@8    5f8cfc00     afxtls.obj
 0003:00000c48       ??_R0?AVCSyncObject@@@8    5f8cfc48     mtcore.obj
 0003:00000c68       ??_R0?AVCCriticalSection@@@8 5f8cfc68     mtcore.obj
 0003:00000c98       ??_R0?AVCSemaphore@@@8     5f8cfc98     mtex.obj
 0003:00000cb8       ??_R0?AVCMutex@@@8         5f8cfcb8     mtex.obj
 0003:00000cd0       ??_R0?AVCEvent@@@8         5f8cfcd0     mtex.obj
 0003:00000cf8       ??_R0?AVCCmdUI@@@8         5f8cfcf8     wincore.obj
 0003:00000d10       ??_R0?AVCTestCmdUI@@@8     5f8cfd10     wincore.obj
 0003:00000d30       ??_R0PAVCUserException@@@8 5f8cfd30     wincore.obj
 0003:00000d50       ??_R0?AVCTempWnd@@@8       5f8cfd50     wincore.obj
 0003:00000d68       ??_R0?AV_AFX_CTL3D_STATE@@@8 5f8cfd68     wincore.obj
 0003:00000d98       ??_R0?AVCFrameWnd@@@8      5f8cfd98     winfrm.obj
 0003:00000dd8       ??_R0?AVCMDIFrameWnd@@@8   5f8cfdd8     winmdi.obj
 0003:00000df8       ??_R0?AVCMDIChildWnd@@@8   5f8cfdf8     winmdi.obj
 0003:00000e20       ??_R0?AVCToolTipCtrl@@@8   5f8cfe20     tooltip.obj
 0003:00000e48       ??_R0?AVCMiniFrameWnd@@@8  5f8cfe48     winmini.obj
 0003:00000e80       ??_R0?AVCControlBar@@@8    5f8cfe80     barcore.obj
 0003:00000ea8       ?_afxComCtlVersion@@3HA    5f8cfea8     bartool.obj
 0003:00000eac       ?_afxDropDownWidth@@3HA    5f8cfeac     bartool.obj
 0003:00000eb0       ??_R0?AVCToolBar@@@8       5f8cfeb0     bartool.obj
 0003:00000ec8       ??_R0?AVCToolCmdUI@@@8     5f8cfec8     bartool.obj
 0003:00000ef0       ??_R0?AVCDialogBar@@@8     5f8cfef0     bardlg.obj
 0003:00000f18       ??_R0?AVCStatusBar@@@8     5f8cff18     barstat.obj
 0003:00000f38       ??_R0?AVCStatusCmdUI@@@8   5f8cff38     barstat.obj
 0003:00000f60       ??_R0?AVCDockBar@@@8       5f8cff60     bardock.obj
 0003:00000f78       ??_R0?AVCMiniDockFrameWnd@@@8 5f8cff78     bardock.obj
 0003:00000fa8       ??_R0?AVCDockContext@@@8   5f8cffa8     dockcont.obj
 0003:00000fc8       ?classCDockState@CDockState@@2UCRuntimeClass@@A 5f8cffc8     dockstat.obj
 0003:00000ff0       ??_R0?AVCDockState@@@8     5f8cfff0     dockstat.obj
 0003:00001018       ??_R0?AVCDC@@@8            5f8d0018     dcprev.obj
 0003:00001030       ??_R0?AVCPreviewDC@@@8     5f8d0030     dcprev.obj
 0003:00001058       ??_R0?AVCMetaFileDC@@@8    5f8d0058     dcmeta.obj
 0003:00001090       ??_R0?AVCReBar@@@8         5f8d0090     barcool.obj
 0003:000010c8       ??_R0?AVCDragListBox@@@8   5f8d00c8     winctrl2.obj
 0003:000010e8       ??_R0?AVCToolBarCtrl@@@8   5f8d00e8     winctrl2.obj
 0003:00001108       ??_R0?AVCStatusBarCtrl@@@8 5f8d0108     winctrl2.obj
 0003:00001128       ??_R0?AVCListCtrl@@@8      5f8d0128     winctrl2.obj
 0003:00001140       ??_R0?AVCTreeCtrl@@@8      5f8d0140     winctrl2.obj
 0003:00001158       ??_R0?AVCSpinButtonCtrl@@@8 5f8d0158     winctrl2.obj
 0003:00001178       ??_R0?AVCSliderCtrl@@@8    5f8d0178     winctrl2.obj
 0003:00001198       ??_R0?AVCProgressCtrl@@@8  5f8d0198     winctrl2.obj
 0003:000011b8       ??_R0?AVCHeaderCtrl@@@8    5f8d01b8     winctrl2.obj
 0003:000011d8       ??_R0?AVCHotKeyCtrl@@@8    5f8d01d8     winctrl2.obj
 0003:000011f8       ??_R0?AVCTabCtrl@@@8       5f8d01f8     winctrl2.obj
 0003:00001210       ??_R0?AVCAnimateCtrl@@@8   5f8d0210     winctrl2.obj
 0003:00001230       ??_R0?AVCRichEditCtrl@@@8  5f8d0230     winctrl2.obj
 0003:00001250       ??_R0?AVCImageList@@@8     5f8d0250     winctrl2.obj
 0003:00001270       ??_R0?AVCTempImageList@@@8 5f8d0270     winctrl2.obj
 0003:000012a0       ??_R0?AV_AFX_CHECKLIST_STATE@@@8 5f8d02a0     winctrl3.obj
 0003:000012d8       ??_R0?AV_AFX_EDIT_STATE@@@8 5f8d02d8     winctrl4.obj
 0003:000012f8       ??_R0?AV_AFX_RICHEDIT_STATE@@@8 5f8d02f8     winctrl4.obj
 0003:00001350       ?_afxPropSheetButtons@@3PAHA 5f8d0350     dlgprop.obj
 0003:00001370       ??_R0?AVCPropertyPage@@@8  5f8d0370     dlgprop.obj
 0003:00001390       ??_R0?AVCPropertySheet@@@8 5f8d0390     dlgprop.obj
 0003:000013b0       ??_R0?AVCPropertyPageEx@@@8 5f8d03b0     dlgprop.obj
 0003:000013d0       ??_R0?AVCPropertySheetEx@@@8 5f8d03d0     dlgprop.obj
 0003:00001408       ??_R0?AVCFileDialog@@@8    5f8d0408     dlgfile.obj
 0003:00001430       ??_R0?AVCPageSetupDialog@@@8 5f8d0430     dlgprnt.obj
 0003:00001450       ??_R0?AVCPrintDialog@@@8   5f8d0450     dlgprnt.obj
 0003:00001478       ??_R0?AV_AFX_COLOR_STATE@@@8 5f8d0478     dlgclr.obj
 0003:00001498       ??_R0?AVCColorDialog@@@8   5f8d0498     dlgclr.obj
 0003:000014c0       ??_R0?AVCFontDialog@@@8    5f8d04c0     dlgfnt.obj
 0003:000014e8       ??_R0?AVCFindReplaceDialog@@@8 5f8d04e8     dlgfr.obj
 0003:00001510       ??_R0?AU_AFX_PROPPAGEFONTINFO@@@8 5f8d0510     ccdata.obj
 0003:00001548       ??_R0?AVCIPAddressCtrl@@@8 5f8d0548     winctrl6.obj
 0003:00001568       ??_R0?AVCComboBoxEx@@@8    5f8d0568     winctrl6.obj
 0003:00001588       ??_R0?AVCReBarCtrl@@@8     5f8d0588     winctrl6.obj
 0003:000015c0       ??_R0?AVCClientDC@@@8      5f8d05c0     wingdi.obj
 0003:000015d8       ??_R0?AVCWindowDC@@@8      5f8d05d8     wingdi.obj
 0003:000015f0       ??_R0?AVCPaintDC@@@8       5f8d05f0     wingdi.obj
 0003:00001608       ??_R0?AVCTempDC@@@8        5f8d0608     wingdi.obj
 0003:00001620       ??_R0?AVCTempGdiObject@@@8 5f8d0620     wingdi.obj
 0003:00001640       ??_R0PAVCResourceException@@@8 5f8d0640     wingdi.obj
 0003:00001688       ??_R0?AVCTempMenu@@@8      5f8d0688     winmenu.obj
 0003:000016ec       ?_dispatchEntryCount@CCmdTarget@@0IA 5f8d06ec     cmdtarg.obj
 0003:000016f0       ?_dwStockPropMask@CCmdTarget@@0KA 5f8d06f0     cmdtarg.obj
 0003:000016f4       ?_eventsinkEntryCount@CCmdTarget@@0IA 5f8d06f4     cmdtarg.obj
 0003:00001708       ??_R0?AVCDocument@@@8      5f8d0708     doccore.obj
 0003:00001720       ??_R0?AVCMirrorFile@@@8    5f8d0720     doccore.obj
 0003:00001750       ??_R0?AVCDocTemplate@@@8   5f8d0750     doctempl.obj
 0003:00001780       ??_R0?AVCSingleDocTemplate@@@8 5f8d0780     docsingl.obj
 0003:000017b8       ??_R0?AVCMultiDocTemplate@@@8 5f8d07b8     docmulti.obj
 0003:000017e8       ??_R0?AVCDocManager@@@8    5f8d07e8     docmgr.obj
 0003:00001808       ??_R0?AVCNewTypeDlg@@@8    5f8d0808     docmgr.obj
 0003:00001838       ??_R0?AVCView@@@8          5f8d0838     viewcore.obj
 0003:00001850       ??_R0?AVCCtrlView@@@8      5f8d0850     viewcore.obj
 0003:00001878       ??_R0?AVCPrintingDialog@@@8 5f8d0878     viewprnt.obj
 0003:000018a8       ??_R0?AVCSplitterWnd@@@8   5f8d08a8     winsplit.obj
 0003:000018d8       ??_R0?AVCScrollView@@@8    5f8d08d8     viewscrl.obj
 0003:00001908       ??_R0?AVCFormView@@@8      5f8d0908     viewform.obj
 0003:00001930       ??_R0?AVCEditView@@@8      5f8d0930     viewedit.obj
 0003:00001958       ??_R0?AVCPreviewView@@@8   5f8d0958     viewprev.obj
 0003:00001980       ??_R0?AVCListView@@@8      5f8d0980     viewcmn.obj
 0003:00001998       ??_R0?AVCTreeView@@@8      5f8d0998     viewcmn.obj
 0003:000019b0       ?_afxIsMailAvail@@3HA      5f8d09b0     docmapi.obj
 0003:000019c0       ??_R0?AV_AFX_MAIL_STATE@@@8 5f8d09c0     docmapi.obj
 0003:000019f0       ??_R0?AVCWinThread@@@8     5f8d09f0     thrdcore.obj
 0003:00001a10       ??_R0?AV_AFX_CTL3D_THREAD@@@8 5f8d0a10     thrdcore.obj
 0003:00001a3c       ?bStaticInit@CDocManager@@2HA 5f8d0a3c     appcore.obj
 0003:00001a40       ??_R0?AV_AFX_WIN_STATE@@@8 5f8d0a40     appcore.obj
 0003:00001a60       ??_R0?AVCWinApp@@@8        5f8d0a60     appcore.obj
 0003:00001a78       ??_R0?AVCCommandLineInfo@@@8 5f8d0a78     appcore.obj
 0003:00001b40       ??_R0?AVCRecentFileList@@@8 5f8d0b40     filelist.obj
 0003:00001b90       ??_R0?AVCInternetSession@@@8 5f8d0b90     inet.obj
 0003:00001bb0       ??_R0?AVCInternetFile@@@8  5f8d0bb0     inet.obj
 0003:00001bd0       ??_R0?AVCInternetConnection@@@8 5f8d0bd0     inet.obj
 0003:00001bf8       ??_R0?AVCFtpConnection@@@8 5f8d0bf8     inet.obj
 0003:00001c18       ??_R0?AVCGopherConnection@@@8 5f8d0c18     inet.obj
 0003:00001c38       ??_R0?AVCHttpConnection@@@8 5f8d0c38     inet.obj
 0003:00001c58       ??_R0?AVCHttpFile@@@8      5f8d0c58     inet.obj
 0003:00001c70       ??_R0?AVCGopherFile@@@8    5f8d0c70     inet.obj
 0003:00001c90       ??_R0?AVCFileFind@@@8      5f8d0c90     inet.obj
 0003:00001ca8       ??_R0?AVCFtpFileFind@@@8   5f8d0ca8     inet.obj
 0003:00001cc8       ??_R0?AVCGopherFileFind@@@8 5f8d0cc8     inet.obj
 0003:00001ce8       ??_R0?AVCGopherLocator@@@8 5f8d0ce8     inet.obj
 0003:00001d08       ??_R0PAVCInternetException@@@8 5f8d0d08     inet.obj
 0003:00001d30       ??_R0?AVCInternetException@@@8 5f8d0d30     inet.obj
 0003:00001d58       ??_R0?AVCSessionMapPtrToPtr@@@8 5f8d0d58     inet.obj
 0003:00001d88       __pRawDllMain              5f8d0d88     dllinit.obj
 0003:00001d8c       ?_afxForceVectorDelete_mfc@@3P6AXXZA 5f8d0d8c     dllinit.obj
 0003:00001d90       ??_R0?AVCDynLinkLibrary@@@8 5f8d0d90     dllinit.obj
 0003:00001db0       ??_R0?AVtype_info@@@8      5f8d0db0     msvcrtd:ti_inst.obj
 0003:00001dd0       __imp__RegDeleteValueW@8   5f8d0dd0     advapi32:ADVAPI32.dll
 0003:00001dd4       __imp__RegQueryValueExW@24 5f8d0dd4     advapi32:ADVAPI32.dll
 0003:00001dd8       __imp__RegOpenKeyW@12      5f8d0dd8     advapi32:ADVAPI32.dll
 0003:00001ddc       __imp__SetFileSecurityW@12 5f8d0ddc     advapi32:ADVAPI32.dll
 0003:00001de0       __imp__GetFileSecurityW@20 5f8d0de0     advapi32:ADVAPI32.dll
 0003:00001de4       __imp__RegDeleteKeyW@8     5f8d0de4     advapi32:ADVAPI32.dll
 0003:00001de8       __imp__RegEnumKeyW@16      5f8d0de8     advapi32:ADVAPI32.dll
 0003:00001dec       __imp__RegSetValueExW@24   5f8d0dec     advapi32:ADVAPI32.dll
 0003:00001df0       __imp__RegCreateKeyW@12    5f8d0df0     advapi32:ADVAPI32.dll
 0003:00001df4       __imp__RegSetValueW@20     5f8d0df4     advapi32:ADVAPI32.dll
 0003:00001df8       __imp__RegQueryValueW@16   5f8d0df8     advapi32:ADVAPI32.dll
 0003:00001dfc       __imp__RegOpenKeyExW@20    5f8d0dfc     advapi32:ADVAPI32.dll
 0003:00001e00       __imp__RegCreateKeyExW@36  5f8d0e00     advapi32:ADVAPI32.dll
 0003:00001e04       __imp__RegCloseKey@4       5f8d0e04     advapi32:ADVAPI32.dll
 0003:00001e08       \177ADVAPI32_NULL_THUNK_DATA_DLA 5f8d0e08     advapi32:ADVAPI32.dll
 0003:00001e0c       __imp__ImageList_Create@20 5f8d0e0c     comctl32:COMCTL32.dll
 0003:00001e10       __imp__InitCommonControlsEx@4 5f8d0e10     comctl32:COMCTL32.dll
 0003:00001e14       __imp__InitCommonControls@0 5f8d0e14     comctl32:COMCTL32.dll
 0003:00001e18       __imp__MakeDragList@4      5f8d0e18     comctl32:COMCTL32.dll
 0003:00001e1c       __imp__ImageList_Destroy@4 5f8d0e1c     comctl32:COMCTL32.dll
 0003:00001e20       __imp__CreateMappedBitmap@20 5f8d0e20     comctl32:COMCTL32.dll
 0003:00001e24       __imp__ImageList_LoadImageW@28 5f8d0e24     comctl32:COMCTL32.dll
 0003:00001e28       __imp__ImageList_Merge@24  5f8d0e28     comctl32:COMCTL32.dll
 0003:00001e2c       __imp__ImageList_Read@4    5f8d0e2c     comctl32:COMCTL32.dll
 0003:00001e30       __imp__ImageList_Write@8   5f8d0e30     comctl32:COMCTL32.dll
 0003:00001e34       __imp__LBItemFromPt@16     5f8d0e34     comctl32:COMCTL32.dll
 0003:00001e38       __imp__ImageList_GetImageCount@4 5f8d0e38     comctl32:COMCTL32.dll
 0003:00001e3c       __imp__ImageList_Add@12    5f8d0e3c     comctl32:COMCTL32.dll
 0003:00001e40       __imp__ImageList_AddMasked@12 5f8d0e40     comctl32:COMCTL32.dll
 0003:00001e44       __imp__ImageList_Remove@8  5f8d0e44     comctl32:COMCTL32.dll
 0003:00001e48       __imp__ImageList_Replace@16 5f8d0e48     comctl32:COMCTL32.dll
 0003:00001e4c       __imp__ImageList_ReplaceIcon@12 5f8d0e4c     comctl32:COMCTL32.dll
 0003:00001e50       __imp__ImageList_GetIcon@12 5f8d0e50     comctl32:COMCTL32.dll
 0003:00001e54       __imp__ImageList_Draw@24   5f8d0e54     comctl32:COMCTL32.dll
 0003:00001e58       __imp__ImageList_SetBkColor@8 5f8d0e58     comctl32:COMCTL32.dll
 0003:00001e5c       __imp__ImageList_GetBkColor@4 5f8d0e5c     comctl32:COMCTL32.dll
 0003:00001e60       __imp__ImageList_SetOverlayImage@12 5f8d0e60     comctl32:COMCTL32.dll
 0003:00001e64       __imp__ImageList_GetImageInfo@12 5f8d0e64     comctl32:COMCTL32.dll
 0003:00001e68       __imp__ImageList_BeginDrag@16 5f8d0e68     comctl32:COMCTL32.dll
 0003:00001e6c       __imp__ImageList_EndDrag@0 5f8d0e6c     comctl32:COMCTL32.dll
 0003:00001e70       __imp__ImageList_DragMove@8 5f8d0e70     comctl32:COMCTL32.dll
 0003:00001e74       __imp__ImageList_SetDragCursorImage@16 5f8d0e74     comctl32:COMCTL32.dll
 0003:00001e78       __imp__ImageList_DragShowNolock@4 5f8d0e78     comctl32:COMCTL32.dll
 0003:00001e7c       __imp__ImageList_GetDragImage@8 5f8d0e7c     comctl32:COMCTL32.dll
 0003:00001e80       __imp__ImageList_DragEnter@12 5f8d0e80     comctl32:COMCTL32.dll
 0003:00001e84       __imp__ImageList_DragLeave@4 5f8d0e84     comctl32:COMCTL32.dll
 0003:00001e88       __imp__PropertySheetW@4    5f8d0e88     comctl32:COMCTL32.dll
 0003:00001e8c       __imp__DestroyPropertySheetPage@4 5f8d0e8c     comctl32:COMCTL32.dll
 0003:00001e90       __imp__CreatePropertySheetPageW@4 5f8d0e90     comctl32:COMCTL32.dll
 0003:00001e94       __imp__ImageList_SetImageCount@8 5f8d0e94     comctl32:COMCTL32.dll
 0003:00001e98       __imp__ImageList_Copy@20   5f8d0e98     comctl32:COMCTL32.dll
 0003:00001e9c       __imp__ImageList_DrawIndirect@4 5f8d0e9c     comctl32:COMCTL32.dll
 0003:00001ea0       __imp__ImageList_Duplicate@4 5f8d0ea0     comctl32:COMCTL32.dll
 0003:00001ea4       \177COMCTL32_NULL_THUNK_DATA_DLA 5f8d0ea4     comctl32:COMCTL32.dll
 0003:00001ea8       __imp__DragAcceptFiles@8   5f8d0ea8     shell32:SHELL32.dll
 0003:00001eac       __imp__SHGetFileInfoW@20   5f8d0eac     shell32:SHELL32.dll
 0003:00001eb0       __imp__DragFinish@4        5f8d0eb0     shell32:SHELL32.dll
 0003:00001eb4       __imp__DragQueryFileW@16   5f8d0eb4     shell32:SHELL32.dll
 0003:00001eb8       __imp__ExtractIconW@12     5f8d0eb8     shell32:SHELL32.dll
 0003:00001ebc       \177SHELL32_NULL_THUNK_DATA_DLA 5f8d0ebc     shell32:SHELL32.dll
 0003:00001ec0       __imp__InternetWriteFile@16 5f8d0ec0     wininet:WININET.dll
 0003:00001ec4       __imp__InternetReadFile@16 5f8d0ec4     wininet:WININET.dll
 0003:00001ec8       __imp__InternetGetLastResponseInfoW@12 5f8d0ec8     wininet:WININET.dll
 0003:00001ecc       __imp__GopherFindFirstFileW@24 5f8d0ecc     wininet:WININET.dll
 0003:00001ed0       __imp__GopherGetLocatorTypeW@8 5f8d0ed0     wininet:WININET.dll
 0003:00001ed4       __imp__FtpFindFirstFileW@20 5f8d0ed4     wininet:WININET.dll
 0003:00001ed8       __imp__HttpQueryInfoW@20   5f8d0ed8     wininet:WININET.dll
 0003:00001edc       __imp__InternetFindNextFileW@8 5f8d0edc     wininet:WININET.dll
 0003:00001ee0       __imp__HttpEndRequestW@16  5f8d0ee0     wininet:WININET.dll
 0003:00001ee4       __imp__HttpSendRequestW@20 5f8d0ee4     wininet:WININET.dll
 0003:00001ee8       __imp__HttpSendRequestExW@20 5f8d0ee8     wininet:WININET.dll
 0003:00001eec       __imp__InternetErrorDlg@20 5f8d0eec     wininet:WININET.dll
 0003:00001ef0       __imp__HttpOpenRequestW@32 5f8d0ef0     wininet:WININET.dll
 0003:00001ef4       __imp__HttpAddRequestHeadersW@16 5f8d0ef4     wininet:WININET.dll
 0003:00001ef8       __imp__GopherGetAttributeW@32 5f8d0ef8     wininet:WININET.dll
 0003:00001efc       __imp__InternetCrackUrlW@16 5f8d0efc     wininet:WININET.dll
 0003:00001f00       __imp__InternetCanonicalizeUrlW@16 5f8d0f00     wininet:WININET.dll
 0003:00001f04       __imp__InternetQueryOptionW@16 5f8d0f04     wininet:WININET.dll
 0003:00001f08       __imp__InternetOpenW@20    5f8d0f08     wininet:WININET.dll
 0003:00001f0c       __imp__InternetCloseHandle@4 5f8d0f0c     wininet:WININET.dll
 0003:00001f10       __imp__InternetOpenUrlW@24 5f8d0f10     wininet:WININET.dll
 0003:00001f14       __imp__InternetSetOptionExW@20 5f8d0f14     wininet:WININET.dll
 0003:00001f18       __imp__InternetSetStatusCallback@8 5f8d0f18     wininet:WININET.dll
 0003:00001f1c       __imp__InternetSetCookieW@12 5f8d0f1c     wininet:WININET.dll
 0003:00001f20       __imp__InternetGetCookieW@16 5f8d0f20     wininet:WININET.dll
 0003:00001f24       __imp__InternetSetFilePointer@20 5f8d0f24     wininet:WININET.dll
 0003:00001f28       __imp__GopherCreateLocatorW@28 5f8d0f28     wininet:WININET.dll
 0003:00001f2c       __imp__GopherOpenFileW@20  5f8d0f2c     wininet:WININET.dll
 0003:00001f30       __imp__InternetQueryDataAvailable@16 5f8d0f30     wininet:WININET.dll
 0003:00001f34       __imp__InternetConnectW@32 5f8d0f34     wininet:WININET.dll
 0003:00001f38       __imp__FtpDeleteFileW@8    5f8d0f38     wininet:WININET.dll
 0003:00001f3c       __imp__FtpRenameFileW@12   5f8d0f3c     wininet:WININET.dll
 0003:00001f40       __imp__FtpCreateDirectoryW@8 5f8d0f40     wininet:WININET.dll
 0003:00001f44       __imp__FtpRemoveDirectoryW@8 5f8d0f44     wininet:WININET.dll
 0003:00001f48       __imp__FtpSetCurrentDirectoryW@8 5f8d0f48     wininet:WININET.dll
 0003:00001f4c       __imp__FtpGetCurrentDirectoryW@12 5f8d0f4c     wininet:WININET.dll
 0003:00001f50       __imp__FtpOpenFileW@20     5f8d0f50     wininet:WININET.dll
 0003:00001f54       __imp__FtpPutFileW@20      5f8d0f54     wininet:WININET.dll
 0003:00001f58       __imp__FtpGetFileW@28      5f8d0f58     wininet:WININET.dll
 0003:00001f5c       \177WININET_NULL_THUNK_DATA_DLA 5f8d0f5c     wininet:WININET.dll
 0003:00001f60       __imp__OpenPrinterW@12     5f8d0f60     winspool:WINSPOOL.DRV
 0003:00001f64       __imp__DocumentPropertiesW@24 5f8d0f64     winspool:WINSPOOL.DRV
 0003:00001f68       __imp__ClosePrinter@4      5f8d0f68     winspool:WINSPOOL.DRV
 0003:00001f6c       \177WINSPOOL_NULL_THUNK_DATA_DLA 5f8d0f6c     winspool:WINSPOOL.DRV
 0003:00001f70       __imp__FindTextW@4         5f8d0f70     comdlg32:comdlg32.dll
 0003:00001f74       __imp__CommDlgExtendedError@0 5f8d0f74     comdlg32:comdlg32.dll
 0003:00001f78       __imp__ChooseColorW@4      5f8d0f78     comdlg32:comdlg32.dll
 0003:00001f7c       __imp__ReplaceTextW@4      5f8d0f7c     comdlg32:comdlg32.dll
 0003:00001f80       __imp__ChooseFontW@4       5f8d0f80     comdlg32:comdlg32.dll
 0003:00001f84       __imp__GetOpenFileNameW@4  5f8d0f84     comdlg32:comdlg32.dll
 0003:00001f88       __imp__PrintDlgW@4         5f8d0f88     comdlg32:comdlg32.dll
 0003:00001f8c       __imp__PageSetupDlgW@4     5f8d0f8c     comdlg32:comdlg32.dll
 0003:00001f90       __imp__GetFileTitleW@12    5f8d0f90     comdlg32:comdlg32.dll
 0003:00001f94       __imp__GetSaveFileNameW@4  5f8d0f94     comdlg32:comdlg32.dll
 0003:00001f98       \177comdlg32_NULL_THUNK_DATA_DLA 5f8d0f98     comdlg32:comdlg32.dll
 0003:00001fa0       ?_simpleNotSupportedException@@3VCNotSupportedException@@A 5f8d0fa0     except.obj
 0003:000020c0       ?_simpleMemoryException@@3VCMemoryException@@A 5f8d10c0     except.obj
 0003:000021e0       ?afxDebugState@@3V?$CProcessLocal@V_AFX_DEBUG_STATE@@@@A 5f8d11e0     dumpinit.obj
 0003:000021e4       ?_afxDiagnosticInit@@3HA   5f8d11e4     dumpinit.obj
 0003:000021e8       ?afxTraceFlags@@3IA        5f8d11e8     dumpinit.obj
 0003:000021ec       ?afxTraceEnabled@@3HA      5f8d11ec     dumpinit.obj
 0003:000021f0       ?afxDump@@3VCDumpContext@@A 5f8d11f0     dumpinit.obj
 0003:00002200       ?_afxMemoryLeakOverride@@3HA 5f8d1200     afxmem.obj
 0003:00002204       ?pfnCrtAllocHook@@3P6AHHPAXIHJPBEH@ZA 5f8d1204     afxmem.obj
 0003:00002208       ?_init_CByteArray@@3UAFX_CLASSINIT@@A 5f8d1208     array_b.obj
 0003:0000220c       ?_init_CDWordArray@@3UAFX_CLASSINIT@@A 5f8d120c     array_d.obj
 0003:00002210       ?_init_CObArray@@3UAFX_CLASSINIT@@A 5f8d1210     array_o.obj
 0003:00002214       ?_init_CStringArray@@3UAFX_CLASSINIT@@A 5f8d1214     array_s.obj
 0003:00002218       ?_init_CWordArray@@3UAFX_CLASSINIT@@A 5f8d1218     array_w.obj
 0003:0000221c       ?_init_CObList@@3UAFX_CLASSINIT@@A 5f8d121c     list_o.obj
 0003:00002220       ?_init_CStringList@@3UAFX_CLASSINIT@@A 5f8d1220     list_s.obj
 0003:00002224       ?_init_CMapStringToOb@@3UAFX_CLASSINIT@@A 5f8d1224     map_so.obj
 0003:00002228       ?_init_CMapStringToString@@3UAFX_CLASSINIT@@A 5f8d1228     map_ss.obj
 0003:0000222c       ?_init_CMapWordToOb@@3UAFX_CLASSINIT@@A 5f8d122c     map_wo.obj
 0003:00002230       ?afxChNil@@3GA             5f8d1230     strcore.obj
 0003:00002234       ?_afxBaseModuleState@@3V?$CProcessLocal@V_AFX_BASE_MODULE_STATE@@@@A 5f8d1234     afxstate.obj
 0003:00002238       ?_afxThreadState@@3V?$CThreadLocal@V_AFX_THREAD_STATE@@@@A 5f8d1238     afxstate.obj
 0003:0000223c       ?_afxTlsRef@@3JA           5f8d123c     afxtls.obj
 0003:00002240       ?_afxThreadData@@3PAVCThreadSlotData@@A 5f8d1240     afxtls.obj
 0003:00002244       ?__afxThreadData@@3PAEA    5f8d1244     afxtls.obj
 0003:00002278       ?_afxGotScrollLines@@3HA   5f8d1278     wincore.obj
 0003:00002280       ?_afxMsgCache@@3PAUAFX_MSG_CACHE@@A 5f8d1280     wincore.obj
 0003:00003a80       ?wndNoTopMost@CWnd@@2V1@B  5f8d2a80     wincore.obj
 0003:00003ac0       ?wndTopMost@CWnd@@2V1@B    5f8d2ac0     wincore.obj
 0003:00003b00       ?wndBottom@CWnd@@2V1@B     5f8d2b00     wincore.obj
 0003:00003b48       ?wndTop@CWnd@@2V1@B        5f8d2b48     wincore.obj
 0003:00003b88       ?m_nMsgDragList@CWnd@@1IB  5f8d2b88     wincore.obj
 0003:00003b8c       _g_pfnGetSystemMetrics     5f8d2b8c     wincore.obj
 0003:00003b90       _g_pfnMonitorFromWindow    5f8d2b90     wincore.obj
 0003:00003b94       _g_pfnMonitorFromRect      5f8d2b94     wincore.obj
 0003:00003b98       _g_pfnMonitorFromPoint     5f8d2b98     wincore.obj
 0003:00003b9c       _g_pfnGetMonitorInfo       5f8d2b9c     wincore.obj
 0003:00003ba0       _g_pfnEnumDisplayMonitors  5f8d2ba0     wincore.obj
 0003:00003ba4       _g_fMultiMonInitDone       5f8d2ba4     wincore.obj
 0003:00003ba8       ?_afxMsgMouseWheel@@3IA    5f8d2ba8     winfrm.obj
 0003:00003bb0       ?rectDefault@CFrameWnd@@2VCRect@@B 5f8d2bb0     winfrm.obj
 0003:00003bc0       ?_afx_sizeMiniSys@@3UtagSIZE@@A 5f8d2bc0     winmini.obj
 0003:00003bc8       ?_afx_hfontMiniSys@@3PAUHFONT__@@A 5f8d2bc8     winmini.obj
 0003:00003bcc       ?_afx_hbmMiniSys@@3PAUHBITMAP__@@A 5f8d2bcc     winmini.obj
 0003:00003bd0       ?_afxWinminiTerm@@3HA      5f8d2bd0     winmini.obj
 0003:00003bd4       ?_init_CDockState@@3UAFX_CLASSINIT@@A 5f8d2bd4     dockstat.obj
 0003:00003bd8       ?_afxHandleSize@@3HA       5f8d2bd8     trckrect.obj
 0003:00003bdc       ?_afxBlackDottedPen@@3PAUHPEN__@@A 5f8d2bdc     trckrect.obj
 0003:00003be0       ?_afxHatchBrush@@3PAUHBRUSH__@@A 5f8d2be0     trckrect.obj
 0003:00003be4       ?_afxCursors@@3PAPAUHICON__@@A 5f8d2be4     trckrect.obj
 0003:00003c10       ?_afxTrackerTerm@@3DA      5f8d2c10     trckrect.obj
 0003:00003c14       ?_afxChecklistState@@3V?$CProcessLocal@V_AFX_CHECKLIST_STATE@@@@A 5f8d2c14     winctrl3.obj
 0003:00003c18       ?_afxRichEditState@@3V?$CProcessLocal@V_AFX_RICHEDIT_STATE@@@@A 5f8d2c18     winctrl4.obj
 0003:00003c1c       ?_afxMsgSETRGB@@3IA        5f8d2c1c     dlgcomm.obj
 0003:00003c20       ?_afxMsgHELP@@3IA          5f8d2c20     dlgcomm.obj
 0003:00003c24       ?_afxMsgCOLOROK@@3IA       5f8d2c24     dlgcomm.obj
 0003:00003c28       ?_afxMsgFILEOK@@3IA        5f8d2c28     dlgcomm.obj
 0003:00003c2c       ?_afxMsgSHAREVI@@3IA       5f8d2c2c     dlgcomm.obj
 0003:00003c30       ?_afxMsgLBSELCHANGE@@3IA   5f8d2c30     dlgcomm.obj
 0003:00003c34       ?_afxClrState@@3V?$CProcessLocal@V_AFX_COLOR_STATE@@@@A 5f8d2c34     dlgclr.obj
 0003:00003c38       ?_afxPropPageFontInfo@@3V?$CProcessLocal@U_AFX_PROPPAGEFONTINFO@@@@A 5f8d2c38     ccdata.obj
 0003:00003c40       ?_simpleUserException@@3VCUserException@@A 5f8d2c40     wingdi.obj
 0003:00003d60       ?_simpleResourceException@@3VCResourceException@@A 5f8d2d60     wingdi.obj
 0003:00003e80       ?_afxHalftoneBrush@@3PAUHBRUSH__@@A 5f8d2e80     wingdix.obj
 0003:00003e84       ?_afxWingdixTerm@@3DA      5f8d2e84     wingdix.obj
 0003:00003e88       ?afxData@@3UAUX_DATA@@A    5f8d2e88     auxdata.obj
 0003:00003ef4       ?_afxResourceLocked@@3PAHA 5f8d2ef4     afxcrit.obj
 0003:00003f38       ?_afxLockInit@@3PAHA       5f8d2f38     afxcrit.obj
 0003:00003f80       ?_afxLockInitLock@@3U_RTL_CRITICAL_SECTION@@A 5f8d2f80     afxcrit.obj
 0003:00003f98       ?_afxResourceLock@@3PAU_RTL_CRITICAL_SECTION@@A 5f8d2f98     afxcrit.obj
 0003:00004130       ?_afxCriticalWin32s@@3HA   5f8d3130     afxcrit.obj
 0003:00004134       ?_afxCriticalInit@@3HA     5f8d3134     afxcrit.obj
 0003:00004138       ?_afx_idcPrimaryLast@@3IA  5f8d3138     winsplit.obj
 0003:0000413c       ?_afx_hcurDestroy@@3PAUHICON__@@A 5f8d313c     winsplit.obj
 0003:00004140       ?_afx_hcurLast@@3PAUHICON__@@A 5f8d3140     winsplit.obj
 0003:00004150       ?_afxUnicodeFont@@3PAUHFONT__@@A 5f8d3150     viewedit.obj
 0003:00004154       ?_afxEditState@@3V?$CProcessLocal@V_AFX_EDIT_STATE@@@@A 5f8d3154     viewedit.obj
 0003:00004158       ?_afxEditviewTerm@@3DA     5f8d3158     viewedit.obj
 0003:0000415c       ?_afxMsgFindReplace@@3IB   5f8d315c     viewedit.obj
 0003:00004160       ?_afxMailState@@3V?$CProcessLocal@V_AFX_MAIL_STATE@@@@A 5f8d3160     docmapi.obj
 0003:00004164       ?_afxWinState@@3V?$CProcessLocal@V_AFX_WIN_STATE@@@@A 5f8d3164     appcore.obj
 0003:00004168       ?pStaticDocManager@CDocManager@@2PAV1@A 5f8d3168     appcore.obj
 0003:0000416c       ?pStaticList@CDocManager@@2PAVCPtrList@@A 5f8d316c     appcore.obj
 0003:00004170       ?_afxCtl3dThread@@3V?$CThreadLocal@V_AFX_CTL3D_THREAD@@@@A 5f8d3170     app3d.obj
 0003:00004174       ?_afxCtl3dState@@3V?$CProcessLocal@V_AFX_CTL3D_STATE@@@@A 5f8d3174     app3d.obj
 0003:00004178       ?_afxSessionMap@@3VCSessionMapPtrToPtr@@A 5f8d3178     inet.obj
 0003:000041d0       __hmod__ADVAPI32           5f8d31d0     advapi32:ADVAPI32.dll
 0003:000041d4       __hmod__COMCTL32           5f8d31d4     comctl32:COMCTL32.dll
 0003:000041d8       __hmod__SHELL32            5f8d31d8     shell32:SHELL32.dll
 0003:000041dc       __hmod__COMDLG32           5f8d31dc     comdlg32:comdlg32.dll
 0003:000041e0       __hmod__WINSPOOL           5f8d31e0     winspool:WINSPOOL.DRV
 0003:000041e4       __hmod__WININET            5f8d31e4     wininet:WININET.dll
 0003:000041e8       ___puiHead                 5f8d31e8     delayimp:delayhlp.obj
 0003:000041ec       ___pfnDliFailureHook       5f8d31ec     delayimp:delayhk1.obj
 0003:000041f0       ___pfnDliNotifyHook        5f8d31f0     delayimp:delayhk2.obj
 0003:000041f4       __adjust_fdiv              5f8d31f4     <common>
 0003:000041f8       ___onexitend               5f8d31f8     <common>
 0003:000041fc       ___onexitbegin             5f8d31fc     <common>

 entry point at        0001:00002d20

 Static symbols

 0001:000a14e0       ?_AfxForceVectorDelete@@YAXXZ 5f8a24e0 f   dllinit.obj
 0001:00098b3e       _$E375                     5f899b3e f   inet.obj
 0001:00098b4d       _$E372                     5f899b4d f   inet.obj
 0001:00098b5c       _$E374                     5f899b5c f   inet.obj
 0001:00098b6e       _$E373                     5f899b6e f   inet.obj
 0001:000989b6       _$E375                     5f8999b6 f   app3d.obj
 0001:000989c5       _$E372                     5f8999c5 f   app3d.obj
 0001:000989ca       _$E374                     5f8999ca f   app3d.obj
 0001:000989dc       _$E373                     5f8999dc f   app3d.obj
 0001:000989eb       _$E380                     5f8999eb f   app3d.obj
 0001:000989fa       _$E377                     5f8999fa f   app3d.obj
 0001:000989ff       _$E379                     5f8999ff f   app3d.obj
 0001:00098a11       _$E378                     5f899a11 f   app3d.obj
 0001:00096fe3       _$E375                     5f897fe3 f   appcore.obj
 0001:00096ff2       _$E372                     5f897ff2 f   appcore.obj
 0001:00096ff7       _$E374                     5f897ff7 f   appcore.obj
 0001:00097009       _$E373                     5f898009 f   appcore.obj
 0001:00095eb0       _$E375                     5f896eb0 f   docmapi.obj
 0001:00095ebf       _$E372                     5f896ebf f   docmapi.obj
 0001:00095ec4       _$E374                     5f896ec4 f   docmapi.obj
 0001:00095ed6       _$E373                     5f896ed6 f   docmapi.obj
 0001:000720e0       _$E373                     5f8730e0 f   viewedit.obj
 0001:000720ea       _$E372                     5f8730ea f   viewedit.obj
 0001:0007210e       _$E376                     5f87310e f   viewedit.obj
 0001:00072118       _$E375                     5f873118 f   viewedit.obj
 0001:00095bf8       _$E381                     5f896bf8 f   viewedit.obj
 0001:00095c07       _$E378                     5f896c07 f   viewedit.obj
 0001:00095c0c       _$E380                     5f896c0c f   viewedit.obj
 0001:00095c1e       _$E379                     5f896c1e f   viewedit.obj
 0001:0007a02d       ?TraceDDE@@YGXPBGPBUtagMSG@@@Z 5f87b02d f   afxtrace.obj
 0001:000942b0       _$E375                     5f8952b0 f   auxdata.obj
 0001:000942bf       _$E372                     5f8952bf f   auxdata.obj
 0001:000942ce       _$E374                     5f8952ce f   auxdata.obj
 0001:000942e0       _$E373                     5f8952e0 f   auxdata.obj
 0001:0007142f       _$E373                     5f87242f f   wingdix.obj
 0001:00071439       _$E372                     5f872439 f   wingdix.obj
 0001:00093cba       _$E377                     5f894cba f   wingdi.obj
 0001:00093cc9       _$E374                     5f894cc9 f   wingdi.obj
 0001:00093cdf       _$E376                     5f894cdf f   wingdi.obj
 0001:00093cf1       _$E375                     5f894cf1 f   wingdi.obj
 0001:00093d1a       _$E382                     5f894d1a f   wingdi.obj
 0001:00093d29       _$E379                     5f894d29 f   wingdi.obj
 0001:00093d3f       _$E381                     5f894d3f f   wingdi.obj
 0001:00093d51       _$E380                     5f894d51 f   wingdi.obj
 0001:000939a0       _$E375                     5f8949a0 f   ccdata.obj
 0001:000939af       _$E372                     5f8949af f   ccdata.obj
 0001:000939b4       _$E374                     5f8949b4 f   ccdata.obj
 0001:000939c6       _$E373                     5f8949c6 f   ccdata.obj
 0001:0009382a       _$E375                     5f89482a f   dlgclr.obj
 0001:00093839       _$E372                     5f894839 f   dlgclr.obj
 0001:0009383e       _$E374                     5f89483e f   dlgclr.obj
 0001:00093850       _$E373                     5f894850 f   dlgclr.obj
 0001:000160a8       _$E375                     5f8170a8 f   winctrl4.obj
 0001:000160b7       _$E372                     5f8170b7 f   winctrl4.obj
 0001:000160bc       _$E374                     5f8170bc f   winctrl4.obj
 0001:000160ce       _$E373                     5f8170ce f   winctrl4.obj
 0001:000935ea       _$E375                     5f8945ea f   winctrl3.obj
 0001:000935f9       _$E372                     5f8945f9 f   winctrl3.obj
 0001:000935fe       _$E374                     5f8945fe f   winctrl3.obj
 0001:00093610       _$E373                     5f894610 f   winctrl3.obj
 0001:00069b69       _$E373                     5f86ab69 f   trckrect.obj
 0001:00069b73       _$E372                     5f86ab73 f   trckrect.obj
 0001:00093198       _$E373                     5f894198 f   dockstat.obj
 0001:000931a2       _$E372                     5f8941a2 f   dockstat.obj
 0001:00068139       _$E373                     5f869139 f   winmini.obj
 0001:00068143       _$E372                     5f869143 f   winmini.obj
 0001:00061180       _$E373                     5f862180 f   winfrm.obj
 0001:0006118a       _$E372                     5f86218a f   winfrm.obj
 0001:000611a7       _$E376                     5f8621a7 f   winfrm.obj
 0001:000611b1       _$E375                     5f8621b1 f   winfrm.obj
 0001:0002b2e0       _$E381                     5f82c2e0 f   wincore.obj
 0001:0002b2ea       _$E380                     5f82c2ea f   wincore.obj
 0001:0002b2ff       _$E387                     5f82c2ff f   wincore.obj
 0001:0002b30e       _$E383                     5f82c30e f   wincore.obj
 0001:0002b31f       _$E386                     5f82c31f f   wincore.obj
 0001:0002b331       _$E384                     5f82c331 f   wincore.obj
 0001:0002b35d       _$E392                     5f82c35d f   wincore.obj
 0001:0002b36c       _$E389                     5f82c36c f   wincore.obj
 0001:0002b37d       _$E391                     5f82c37d f   wincore.obj
 0001:0002b38f       _$E390                     5f82c38f f   wincore.obj
 0001:0002b3bb       _$E397                     5f82c3bb f   wincore.obj
 0001:0002b3ca       _$E394                     5f82c3ca f   wincore.obj
 0001:0002b3db       _$E396                     5f82c3db f   wincore.obj
 0001:0002b3ed       _$E395                     5f82c3ed f   wincore.obj
 0001:0002b419       _$E402                     5f82c419 f   wincore.obj
 0001:0002b428       _$E399                     5f82c428 f   wincore.obj
 0001:0002b439       _$E401                     5f82c439 f   wincore.obj
 0001:0002b44b       _$E400                     5f82c44b f   wincore.obj
 0001:0008f162       _$E375                     5f890162 f   afxstate.obj
 0001:0008f171       _$E372                     5f890171 f   afxstate.obj
 0001:0008f176       _$E374                     5f890176 f   afxstate.obj
 0001:0008f188       _$E373                     5f890188 f   afxstate.obj
 0001:0008f6fe       _$E380                     5f8906fe f   afxstate.obj
 0001:0008f70d       _$E377                     5f89070d f   afxstate.obj
 0001:0008f712       _$E379                     5f890712 f   afxstate.obj
 0001:0008f724       _$E378                     5f890724 f   afxstate.obj
 0001:0008ef1a       _$E373                     5f88ff1a f   map_wo.obj
 0001:0008ef24       _$E372                     5f88ff24 f   map_wo.obj
 0001:00023e4b       ?DestructElement@@YAXPAVCString@@@Z 5f824e4b f   map_ss.obj
 0001:00023ff5       ?ConstructElement@@YAXPAVCString@@@Z 5f824ff5 f   map_ss.obj
 0001:0008ee4a       _$E373                     5f88fe4a f   map_ss.obj
 0001:0008ee54       _$E372                     5f88fe54 f   map_ss.obj
 0001:000234bc       ?DestructElement@@YAXPAVCString@@@Z 5f8244bc f   map_sp.obj
 0001:000229cc       ?DestructElement@@YAXPAVCString@@@Z 5f8239cc f   map_so.obj
 0001:0008ed5a       _$E373                     5f88fd5a f   map_so.obj
 0001:0008ed64       _$E372                     5f88fd64 f   map_so.obj
 0001:00020670       ?DestructElement@@YAXPAVCString@@@Z 5f821670 f   list_s.obj
 0001:00020810       ?ConstructElement@@YAXPAVCString@@@Z 5f821810 f   list_s.obj
 0001:0008ec4a       _$E373                     5f88fc4a f   list_s.obj
 0001:0008ec54       _$E372                     5f88fc54 f   list_s.obj
 0001:0008eb5a       _$E373                     5f88fb5a f   list_o.obj
 0001:0008eb64       _$E372                     5f88fb64 f   list_o.obj
 0001:0008ea88       _$E373                     5f88fa88 f   array_w.obj
 0001:0008ea92       _$E372                     5f88fa92 f   array_w.obj
 0001:0001c6ed       ?DestructElements@@YAXPAVCString@@H@Z 5f81d6ed f   array_s.obj
 0001:0001c73c       ?DestructElement@@YAXPAVCString@@@Z 5f81d73c f   array_s.obj
 0001:0001ca7f       ?ConstructElements@@YAXPAVCString@@H@Z 5f81da7f f   array_s.obj
 0001:0001cace       ?ConstructElement@@YAXPAVCString@@@Z 5f81dace f   array_s.obj
 0001:0001cb77       ?CopyElements@@YAXPAVCString@@0H@Z 5f81db77 f   array_s.obj
 0001:0008e998       _$E373                     5f88f998 f   array_s.obj
 0001:0008e9a2       _$E372                     5f88f9a2 f   array_s.obj
 0001:0008e8c8       _$E373                     5f88f8c8 f   array_o.obj
 0001:0008e8d2       _$E372                     5f88f8d2 f   array_o.obj
 0001:0008e7d8       _$E373                     5f88f7d8 f   array_d.obj
 0001:0008e7e2       _$E372                     5f88f7e2 f   array_d.obj
 0001:0008e708       _$E373                     5f88f708 f   array_b.obj
 0001:0008e712       _$E372                     5f88f712 f   array_b.obj
 0001:00003a30       _$E373                     5f804a30 f   dumpinit.obj
 0001:00003a3a       _$E372                     5f804a3a f   dumpinit.obj
 0001:00003a4b       _$E376                     5f804a4b f   dumpinit.obj
 0001:00003a55       _$E375                     5f804a55 f   dumpinit.obj
 0001:00003d91       _$E381                     5f804d91 f   dumpinit.obj
 0001:00003da0       _$E378                     5f804da0 f   dumpinit.obj
 0001:00003da5       _$E380                     5f804da5 f   dumpinit.obj
 0001:00003db7       _$E379                     5f804db7 f   dumpinit.obj
 0001:0008e434       _$E375                     5f88f434 f   except.obj
 0001:0008e443       _$E372                     5f88f443 f   except.obj
 0001:0008e459       _$E374                     5f88f459 f   except.obj
 0001:0008e46b       _$E373                     5f88f46b f   except.obj
 0001:0008e494       _$E380                     5f88f494 f   except.obj
 0001:0008e4a3       _$E377                     5f88f4a3 f   except.obj
 0001:0008e4b9       _$E379                     5f88f4b9 f   except.obj
 0001:0008e4cb       _$E378                     5f88f4cb f   except.obj
 0001:00002be0       ?ArrayUnwindFilter@@YAHPAU_EXCEPTION_POINTERS@@@Z 5f803be0 f   msvcrtd:ehvecdtr.obj
 0001:000029e9       hard                       5f8039e9 f   msvcrtd:llmul.obj
 0001:000029b0       MORE32                     5f8039b0 f   msvcrtd:llshr.obj
 0001:000029bb       RETSIGN                    5f8039bb f   msvcrtd:llshr.obj
 0001:00002911       L1                         5f803911 f   msvcrtd:lldiv.obj
 0001:0000292d       L2                         5f80392d f   msvcrtd:lldiv.obj
 0001:00002949       L3                         5f803949 f   msvcrtd:lldiv.obj
 0001:00002957       L5                         5f803957 f   msvcrtd:lldiv.obj
 0001:00002985       L6                         5f803985 f   msvcrtd:lldiv.obj
 0001:00002986       L7                         5f803986 f   msvcrtd:lldiv.obj
 0001:0000298a       L4                         5f80398a f   msvcrtd:lldiv.obj
 0001:00002994       L8                         5f803994 f   msvcrtd:lldiv.obj
 0001:000028a0       _$$$00001                  5f8038a0 f   msvcrtd:chkstk.obj
 0001:000028ac       probepages                 5f8038ac f   msvcrtd:chkstk.obj
 0001:000028c0       lastpage                   5f8038c0 f   msvcrtd:chkstk.obj
 0001:0000382f       ?OverlayIAT@@YGXPAU_IMAGE_THUNK_DATA32@@PBU1@@Z 5f80482f f   delayimp:delayhlp.obj

 1237 bytes saved through ICF

